 ProcList

 Timestamp is 61f9ea6d (Wed Feb  2 02:20:29 2022)

 Preferred load address is 0000000180000000

 Start         Length     Name                   Class
 0001:00000000 00000ae0H .text                   CODE
 0001:00000ae0 000000b0H .text$di                CODE
 0001:00000b90 00041bc8H .text$mn                CODE
 0001:00042758 00001a80H .text$x                 CODE
 0001:000441d8 00000244H .text$yd                CODE
 0002:00000000 00000498H .idata$5                DATA
 0002:00000498 00000008H .00cfg                  DATA
 0002:000004a0 00000008H .CRT$XCA                DATA
 0002:000004a8 00000018H .CRT$XCC                DATA
 0002:000004c0 00000010H .CRT$XCL                DATA
 0002:000004d0 00000018H .CRT$XCU                DATA
 0002:000004e8 00000008H .CRT$XCZ                DATA
 0002:000004f0 00000008H .CRT$XIA                DATA
 0002:000004f8 00000020H .CRT$XIC                DATA
 0002:00000518 00000008H .CRT$XIZ                DATA
 0002:00000520 00000008H .CRT$XPA                DATA
 0002:00000528 00000010H .CRT$XPX                DATA
 0002:00000538 00000008H .CRT$XPXA               DATA
 0002:00000540 00000008H .CRT$XPZ                DATA
 0002:00000548 00000008H .CRT$XTA                DATA
 0002:00000550 00000010H .CRT$XTZ                DATA
 0002:00000558 00000000H .gehcont$y              DATA
 0002:00000558 00000000H .gfids$y                DATA
 0002:00000560 0000e520H .rdata                  DATA
 0002:0000ea80 00000000H .rdata$CastGuardVftablesA DATA
 0002:0000ea80 00000000H .rdata$CastGuardVftablesC DATA
 0002:0000ea80 00000facH .rdata$r                DATA
 0002:0000fa2c 0000038cH .rdata$zzzdbg           DATA
 0002:0000fdb8 00000008H .rtc$IAA                DATA
 0002:0000fdc0 00000008H .rtc$IZZ                DATA
 0002:0000fdc8 00000008H .rtc$TAA                DATA
 0002:0000fdd0 00000010H .rtc$TZZ                DATA
 0002:0000fde0 00004b98H .xdata                  DATA
 0002:00014978 000003d8H .xdata$x                DATA
 0002:00014d50 000001a0H .edata                  DATA
 0002:00014ef0 000000a0H .idata$2                DATA
 0002:00014f90 00000018H .idata$3                DATA
 0002:00014fa8 00000498H .idata$4                DATA
 0002:00015440 00000a2cH .idata$6                DATA
 0003:00000000 00000b80H .data                   DATA
 0003:00000b80 00000370H .data$r                 DATA
 0003:00000ef0 00000670H .data$rs                DATA
 0003:00001560 00002bbcH .bss                    DATA
 0004:00000000 00002098H .pdata                  DATA
 0005:00000000 00000060H .rsrc$01                DATA
 0005:00000060 00000340H .rsrc$02                DATA

  Address         Publics by Value              Rva+Base               Lib:Object

 0000:00000000       __x64_code_ranges_to_entry_points 0000000000000000     <absolute>
 0000:00000000       __guard_fids_count         0000000000000000     <absolute>
 0000:00000000       ___safe_se_handler_table   0000000000000000     <absolute>
 0000:00000000       __x64_code_ranges_to_entry_points_count 0000000000000000     <absolute>
 0000:00000000       __arm64x_extra_rfe_table   0000000000000000     <absolute>
 0000:00000000       __hybrid_code_map          0000000000000000     <absolute>
 0000:00000000       __arm64x_redirection_metadata 0000000000000000     <absolute>
 0000:00000000       __volatile_metadata        0000000000000000     <absolute>
 0000:00000000       __arm64x_extra_rfe_table_size 0000000000000000     <absolute>
 0000:00000000       __guard_iat_table          0000000000000000     <absolute>
 0000:00000000       ___safe_se_handler_count   0000000000000000     <absolute>
 0000:00000000       __guard_longjmp_table      0000000000000000     <absolute>
 0000:00000000       __guard_iat_count          0000000000000000     <absolute>
 0000:00000000       __guard_longjmp_count      0000000000000000     <absolute>
 0000:00000000       __dynamic_value_reloc_table 0000000000000000     <absolute>
 0000:00000000       __hybrid_auxiliary_iat     0000000000000000     <absolute>
 0000:00000000       __hybrid_auxiliary_iat_copy 0000000000000000     <absolute>
 0000:00000000       __guard_eh_cont_count      0000000000000000     <absolute>
 0000:00000000       __AbsoluteZero             0000000000000000     <absolute>
 0000:00000000       __guard_check_icall_a64n_fptr 0000000000000000     <absolute>
 0000:00000000       __guard_fids_table         0000000000000000     <absolute>
 0000:00000000       __arm64x_redirection_metadata_count 0000000000000000     <absolute>
 0000:00000000       __enclave_config           0000000000000000     <absolute>
 0000:00000000       __guard_eh_cont_table      0000000000000000     <absolute>
 0000:00000000       __arm64x_native_entrypoint 0000000000000000     <absolute>
 0000:00000000       __hybrid_code_map_count    0000000000000000     <absolute>
 0000:00000100       __guard_flags              0000000000000100     <absolute>
 0000:00000000       __ImageBase                0000000180000000     <linker-defined>
 0001:00000000       __security_check_cookie    0000000180001000 f   LIBCMT:arm64secgs.obj
 0001:00000018       __gsfailure                0000000180001018 f   LIBCMT:arm64secgs.obj
 0001:00000050       __security_push_cookie     0000000180001050 f   LIBCMT:secpushpop.obj
 0001:00000070       __security_pop_cookie      0000000180001070 f   LIBCMT:secpushpop.obj
 0001:000000a0       __ppgsfailure              00000001800010a0 f   LIBCMT:secpushpop.obj
 0001:000000c0       _alloca_probe              00000001800010c0 f   LIBCMT:chkstk.obj
 0001:000000c0       __chkstk                   00000001800010c0 f   LIBCMT:chkstk.obj
 0001:00000100       memmove                    0000000180001100 f   libvcruntime:memcpy.obj
 0001:00000100       memcpy                     0000000180001100 f   libvcruntime:memcpy.obj
 0001:00000110       __memcpy_forward           0000000180001110     libvcruntime:memcpy.obj
 0001:00000110       _memcpy_strict_align       0000000180001110     libvcruntime:memcpy.obj
 0001:00000160       __memcpy_forward_large_neon 0000000180001160 f   libvcruntime:memcpy.obj
 0001:00000260       __memcpy_reverse           0000000180001260 f   libvcruntime:memcpy.obj
 0001:000002c0       __memcpy_reverse_large_neon 00000001800012c0 f   libvcruntime:memcpy.obj
 0001:000003e0       memset                     00000001800013e0 f   libvcruntime:memset.obj
 0001:00000580       memcmp                     0000000180001580 f   libvcruntime:memcmp.obj
 0001:00000968       _NLG_Notify                0000000180001968 f   libvcruntime:notify.obj
 0001:0000097c       __NLG_Dispatch2            000000018000197c     libvcruntime:notify.obj
 0001:00000984       __NLG_Return2              0000000180001984 f   libvcruntime:notify.obj
 0001:00000990       __C_ExecuteExceptionFilter 0000000180001990 f   libvcruntime:handler.obj
 0001:000009e4       __C_ExecuteTerminationHandler 00000001800019e4 f   libvcruntime:handler.obj
 0001:00000a38       _CallSettingFrame          0000000180001a38 f   libvcruntime:handlers.obj
 0001:00000b90       ?WriteToFile@@YA_KPEAXAEBV?$basic_string_view@_WU?$char_traits@_W@std@@@std@@@Z 0000000180001b90 f   fileio.obj
 0001:00000be0       ??1PerfLib@@QEAA@XZ        0000000180001be0 f i perfthread.obj
 0001:00000be0       ??1?$basic_string@_WU?$char_traits@_W@std@@V?$allocator@_W@2@@std@@QEAA@XZ 0000000180001be0 f i fileio.obj
 0001:00000c20       ??1mode@@QEAA@XZ           0000000180001c20 f i fileio.obj
 0001:00000d20       ??1columns@@QEAA@XZ        0000000180001d20 f i fileio.obj
 0001:00000da8       __local_stdio_printf_options 0000000180001da8 f i format.obj
 0001:00000db8       ??0exception@std@@QEAA@AEBV01@@Z 0000000180001db8 f i format.obj
 0001:00000df8       ?what@exception@std@@UEBAPEBDXZ 0000000180001df8 f i format.obj
 0001:00000e10       ??_Eruntime_error@std@@UEAAPEAXI@Z 0000000180001e10 f i * CIL library *:* CIL module *
 0001:00000e10       ??_Gruntime_error@std@@UEAAPEAXI@Z 0000000180001e10 f i format.obj
 0001:00000e10       ??_Eformat_error@v8@fmt@@UEAAPEAXI@Z 0000000180001e10 f i * CIL library *:* CIL module *
 0001:00000e10       ??_Gbad_cast@std@@UEAAPEAXI@Z 0000000180001e10 f i format.obj
 0001:00000e10       ??_Eexception@std@@UEAAPEAXI@Z 0000000180001e10 f i * CIL library *:* CIL module *
 0001:00000e10       ??_Ebad_alloc@std@@UEAAPEAXI@Z 0000000180001e10 f i * CIL library *:* CIL module *
 0001:00000e10       ??_Ebad_array_new_length@std@@UEAAPEAXI@Z 0000000180001e10 f i * CIL library *:* CIL module *
 0001:00000e10       ??_Gbad_alloc@std@@UEAAPEAXI@Z 0000000180001e10 f i format.obj
 0001:00000e10       ??_Gexception@std@@UEAAPEAXI@Z 0000000180001e10 f i format.obj
 0001:00000e10       ??_Ebad_cast@std@@UEAAPEAXI@Z 0000000180001e10 f i * CIL library *:* CIL module *
 0001:00000e10       ??_Gformat_error@v8@fmt@@UEAAPEAXI@Z 0000000180001e10 f i format.obj
 0001:00000e10       ??_Gbad_array_new_length@std@@UEAAPEAXI@Z 0000000180001e10 f i format.obj
 0001:00000e58       ??1bad_cast@std@@UEAA@XZ   0000000180001e58 f i format.obj
 0001:00000e58       ??1bad_array_new_length@std@@UEAA@XZ 0000000180001e58 f i format.obj
 0001:00000e58       ??1bad_function_call@std@@UEAA@XZ 0000000180001e58 f i libcpmt:xthrow.obj
 0001:00000e58       ??1format_error@v8@fmt@@UEAA@XZ 0000000180001e58 f i format.obj
 0001:00000e58       ??1out_of_range@std@@UEAA@XZ 0000000180001e58 f i libcpmt:xthrow.obj
 0001:00000e58       ??1bad_alloc@std@@UEAA@XZ  0000000180001e58 f i format.obj
 0001:00000e58       ??1runtime_error@std@@UEAA@XZ 0000000180001e58 f i format.obj
 0001:00000e58       ??1length_error@std@@UEAA@XZ 0000000180001e58 f i libcpmt:xthrow.obj
 0001:00000e58       ??1bad_exception@std@@UEAA@XZ 0000000180001e58 f i libvcruntime:frame.obj
 0001:00000e68       ??0bad_array_new_length@std@@QEAA@XZ 0000000180001e68 f i format.obj
 0001:00000e88       ?_Throw_bad_array_new_length@std@@YAXXZ 0000000180001e88 f i format.obj
 0001:00000ea8       ??0bad_array_new_length@std@@QEAA@AEBV01@@Z 0000000180001ea8 f i format.obj
 0001:00000ef0       ??0bad_alloc@std@@QEAA@AEBV01@@Z 0000000180001ef0 f i format.obj
 0001:00000f38       ??0bad_cast@std@@QEAA@XZ   0000000180001f38 f i format.obj
 0001:00000f58       ?_Throw_bad_cast@std@@YAXXZ 0000000180001f58 f i format.obj
 0001:00000f78       ??0bad_cast@std@@QEAA@AEBV01@@Z 0000000180001f78 f i format.obj
 0001:00000fc0       ?_Xlen_string@std@@YAXXZ   0000000180001fc0 f i format.obj
 0001:00000fd0       ??0runtime_error@std@@QEAA@PEBD@Z 0000000180001fd0 f i format.obj
 0001:00001028       ??0runtime_error@std@@QEAA@AEBV01@@Z 0000000180002028 f i format.obj
 0001:00001070       ?on_error@?$specs_handler@_W@detail@v8@fmt@@QEAAXPEBD@Z 0000000180002070 f i handles.obj
 0001:00001070       ?on_error@error_handler@detail@v8@fmt@@QEAAXPEBD@Z 0000000180002070 f i format.obj
 0001:000010f8       ??1?$thousands_sep_result@_W@detail@v8@fmt@@QEAA@XZ 00000001800020f8 f i format.obj
 0001:000010f8       ??1?$digit_grouping@_W@detail@v8@fmt@@QEAA@XZ 00000001800020f8 f i handles.obj
 0001:000010f8       ??1?$basic_string@DU?$char_traits@D@std@@V?$allocator@D@2@@std@@QEAA@XZ 00000001800020f8 f i format.obj
 0001:00001138       ??_G_Facet_base@std@@UEAAPEAXI@Z 0000000180002138 f i format.obj
 0001:00001138       ??_E_Facet_base@std@@UEAAPEAXI@Z 0000000180002138 f i * CIL library *:* CIL module *
 0001:00001170       ??1_Locinfo@std@@QEAA@XZ   0000000180002170 f i format.obj
 0001:00001200       ?_Incref@facet@locale@std@@UEAAXXZ 0000000180002200 f i format.obj
 0001:00001218       ?_Decref@facet@locale@std@@UEAAPEAV_Facet_base@3@XZ 0000000180002218 f i format.obj
 0001:00001238       ??1facet@locale@std@@MEAA@XZ 0000000180002238 f i format.obj
 0001:00001248       ??1locale@std@@QEAA@XZ     0000000180002248 f i format.obj
 0001:00001280       ?throw_format_error@detail@v8@fmt@@YAXPEBD@Z 0000000180002280 f   format.obj
 0001:00001308       ?fmt_snprintf@detail@v8@fmt@@YAHPEAD_KPEBDZZ 0000000180002308 f i format.obj
 0001:00001370       ??1bigint@detail@v8@fmt@@QEAA@XZ 0000000180002370 f i format.obj
 0001:00001370       ??1?$basic_memory_buffer@I$0CA@V?$allocator@I@std@@@v8@fmt@@QEAA@XZ 0000000180002370 f i format.obj
 0001:000013a0       ??_3bigint@detail@v8@fmt@@QEAAAEAV0123@H@Z 00000001800023a0 f i format.obj
 0001:00001458       ?compare@detail@v8@fmt@@YAHAEBVbigint@123@0@Z 0000000180002458 f i format.obj
 0001:00001508       ?add_compare@detail@v8@fmt@@YAHAEBVbigint@123@00@Z 0000000180002508 f i format.obj
 0001:00001638       ?assign_pow10@bigint@detail@v8@fmt@@QEAAXH@Z 0000000180002638 f i format.obj
 0001:000017a0       ?square@bigint@detail@v8@fmt@@QEAAXXZ 00000001800027a0 f i format.obj
 0001:00001a28       ?align@bigint@detail@v8@fmt@@QEAAXAEBV1234@@Z 0000000180002a28 f i format.obj
 0001:00001b48       ?on_digit@gen_digits_handler@detail@v8@fmt@@QEAA?AW4result@digits@234@D_K00_N@Z 0000000180002b48 f i format.obj
 0001:00001c98       ?grisu_gen_digits@detail@v8@fmt@@YA?AW4result@digits@123@Ufp@123@_KAEAHAEAUgen_digits_handler@123@@Z 0000000180002c98 f i format.obj
 0001:00001f40       ?get_cached_power@?$cache_accessor@N@dragonbox@detail@v8@fmt@@SA?AUuint128_wrapper@345@H@Z 0000000180002f40 f i format.obj
 0001:000020f0       ?remove_trailing_zeros@dragonbox@detail@v8@fmt@@YAHAEAI@Z 00000001800030f0 f i format.obj
 0001:00002198       ?remove_trailing_zeros@dragonbox@detail@v8@fmt@@YAHAEA_K@Z 0000000180003198 f i format.obj
 0001:000023a0       ?format_dragon@detail@v8@fmt@@YAXUfp@123@_NHAEAV?$buffer@D@123@AEAH@Z 00000001800033a0 f i format.obj
 0001:000037f0       ??1?$_Yarn@D@std@@QEAA@XZ  00000001800047f0 f i format.obj
 0001:000037f0       ??1?$_Yarn@_W@std@@QEAA@XZ 00000001800047f0 f i format.obj
 0001:00003818       ??1?$basic_memory_buffer@D$0BPE@V?$allocator@D@std@@@v8@fmt@@QEAA@XZ 0000000180004818 f i format.obj
 0001:00003848       ??1?$basic_memory_buffer@_W$0BPE@V?$allocator@_W@std@@@v8@fmt@@QEAA@XZ 0000000180004848 f i format.obj
 0001:00003878       ?try_resize@?$buffer@D@detail@v8@fmt@@QEAAX_K@Z 0000000180004878 f i format.obj
 0001:000038c0       ?assign@?$basic_string@_WU?$char_traits@_W@std@@V?$allocator@_W@2@@std@@QEAAAEAV12@QEB_W_K@Z 00000001800048c0 f i format.obj
 0001:000039e8       ?assign@?$basic_string@DU?$char_traits@D@std@@V?$allocator@D@2@@std@@QEAAAEAV12@QEBD_K@Z 00000001800049e8 f i format.obj
 0001:00003af8       ?grow@?$basic_memory_buffer@D$0BPE@V?$allocator@D@std@@@v8@fmt@@MEAAX_K@Z 0000000180004af8 f i format.obj
 0001:00003b78       ??$thousands_sep_impl@_W@detail@v8@fmt@@YA?AU?$thousands_sep_result@_W@012@Vlocale_ref@012@@Z 0000000180004b78 f i format.obj
 0001:00003cc0       ?grow@?$basic_memory_buffer@_W$0BPE@V?$allocator@_W@std@@@v8@fmt@@MEAAX_K@Z 0000000180004cc0 f i format.obj
 0001:00003d68       ?grow@?$basic_memory_buffer@H$0BPE@V?$allocator@H@std@@@v8@fmt@@MEAAX_K@Z 0000000180004d68 f i format.obj
 0001:00003d68       ?grow@?$basic_memory_buffer@I$0CA@V?$allocator@I@std@@@v8@fmt@@MEAAX_K@Z 0000000180004d68 f i format.obj
 0001:00003e10       ??$format_float@N@detail@v8@fmt@@YAHNHUfloat_specs@012@AEAV?$buffer@D@012@@Z 0000000180004e10 f i format.obj
 0001:000041e0       ??$format_float@O@detail@v8@fmt@@YAHOHUfloat_specs@012@AEAV?$buffer@D@012@@Z 00000001800051e0 f i format.obj
 0001:000045b0       ??$snprintf_float@N@detail@v8@fmt@@YAHNHUfloat_specs@012@AEAV?$buffer@D@012@@Z 00000001800055b0 f i format.obj
 0001:000048d8       ??$snprintf_float@O@detail@v8@fmt@@YAHOHUfloat_specs@012@AEAV?$buffer@D@012@@Z 00000001800058d8 f i format.obj
 0001:00004c08       ??$to_decimal@M@dragonbox@detail@v8@fmt@@YA?AU?$decimal_fp@M@0123@M@Z 0000000180005c08 f i format.obj
 0001:00004e80       ??$to_decimal@N@dragonbox@detail@v8@fmt@@YA?AU?$decimal_fp@N@0123@N@Z 0000000180005e80 f i format.obj
 0001:000052d0       ??0format_error@v8@fmt@@QEAA@AEBV012@@Z 00000001800062d0 f i format.obj
 0001:00005318       ??1?$unique_ptr@V_Facet_base@std@@U?$default_delete@V_Facet_base@std@@@2@@std@@QEAA@XZ 0000000180006318 f i format.obj
 0001:00005338       ?do_truename@?$numpunct@_W@std@@MEBA?AV?$basic_string@_WU?$char_traits@_W@std@@V?$allocator@_W@2@@2@XZ 0000000180006338 f i format.obj
 0001:00005398       ?do_falsename@?$numpunct@_W@std@@MEBA?AV?$basic_string@_WU?$char_traits@_W@std@@V?$allocator@_W@2@@2@XZ 0000000180006398 f i format.obj
 0001:000053f8       ?do_grouping@?$numpunct@_W@std@@MEBA?AV?$basic_string@DU?$char_traits@D@std@@V?$allocator@D@2@@2@XZ 00000001800063f8 f i format.obj
 0001:00005458       ?do_thousands_sep@?$numpunct@_W@std@@MEBA_WXZ 0000000180006458 f i format.obj
 0001:00005460       ?do_decimal_point@?$numpunct@_W@std@@MEBA_WXZ 0000000180006460 f i format.obj
 0001:00005468       ??_G?$numpunct@_W@std@@MEAAPEAXI@Z 0000000180006468 f i format.obj
 0001:00005468       ??_E?$numpunct@_W@std@@MEAAPEAXI@Z 0000000180006468 f i * CIL library *:* CIL module *
 0001:000054c8       ??0?$basic_string@_WU?$char_traits@_W@std@@V?$allocator@_W@2@@std@@QEAA@QEB_W@Z 00000001800064c8 f i format.obj
 0001:00005520       ??$use_facet@V?$numpunct@_W@std@@@std@@YAAEBV?$numpunct@_W@0@AEBVlocale@0@@Z 0000000180006520 f i format.obj
 0001:00005650       ??$write@DVappender@v8@fmt@@I$0A@@detail@v8@fmt@@YA?AVappender@12@V312@I@Z 0000000180006650 f i format.obj
 0001:00005768       ??$write@DVappender@v8@fmt@@_K$0A@@detail@v8@fmt@@YA?AVappender@12@V312@_K@Z 0000000180006768 f i format.obj
 0001:00005890       ??$shorter_interval_case@M@dragonbox@detail@v8@fmt@@YA?AU?$decimal_fp@M@0123@H@Z 0000000180006890 f i format.obj
 0001:00005a20       ??$is_endpoint_integer@M@dragonbox@detail@v8@fmt@@YA_NIHH@Z 0000000180006a20 f i format.obj
 0001:00005a70       ??$is_endpoint_integer@N@dragonbox@detail@v8@fmt@@YA_N_KHH@Z 0000000180006a70 f i format.obj
 0001:00005ac0       ?_Getcat@?$numpunct@_W@std@@SA_KPEAPEBVfacet@locale@2@PEBV42@@Z 0000000180006ac0 f i format.obj
 0001:00005c38       ?_Init@?$numpunct@_W@std@@IEAAXAEBV_Locinfo@2@_N@Z 0000000180006c38 f i format.obj
 0001:00005f38       ??1?$_Tidy_guard@V?$numpunct@_W@std@@@std@@QEAA@XZ 0000000180006f38 f i format.obj
 0001:00005f70       ??$format_decimal@DIVappender@v8@fmt@@$0A@@detail@v8@fmt@@YA?AU?$format_decimal_result@Vappender@v8@fmt@@@012@Vappender@12@IH@Z 0000000180006f70 f i format.obj
 0001:00006088       ??$format_decimal@D_KVappender@v8@fmt@@$0A@@detail@v8@fmt@@YA?AU?$format_decimal_result@Vappender@v8@fmt@@@012@Vappender@12@_KH@Z 0000000180007088 f i format.obj
 0001:00006198       ??$?RH$0A@@?$width_checker@Uerror_handler@detail@v8@fmt@@@detail@v8@fmt@@QEAA_KH@Z 0000000180007198 f i format.obj
 0001:00006240       ??$?RH$0A@@?$precision_checker@Uerror_handler@detail@v8@fmt@@@detail@v8@fmt@@QEAA_KH@Z 0000000180007240 f i format.obj
 0001:000062e8       ??$?R_J$0A@@?$width_checker@Uerror_handler@detail@v8@fmt@@@detail@v8@fmt@@QEAA_K_J@Z 00000001800072e8 f i format.obj
 0001:00006390       ??$?RPEBX$0A@@?$width_checker@Uerror_handler@detail@v8@fmt@@@detail@v8@fmt@@QEAA_KPEBX@Z 0000000180007390 f i format.obj
 0001:00006390       ??$?RN$0A@@?$width_checker@Uerror_handler@detail@v8@fmt@@@detail@v8@fmt@@QEAA_KN@Z 0000000180007390 f i format.obj
 0001:00006390       ??$?RO$0A@@?$width_checker@Uerror_handler@detail@v8@fmt@@@detail@v8@fmt@@QEAA_KO@Z 0000000180007390 f i format.obj
 0001:00006390       ??$?RM$0A@@?$width_checker@Uerror_handler@detail@v8@fmt@@@detail@v8@fmt@@QEAA_KM@Z 0000000180007390 f i format.obj
 0001:00006390       ??$?R_N$0A@@?$width_checker@Uerror_handler@detail@v8@fmt@@@detail@v8@fmt@@QEAA_K_N@Z 0000000180007390 f i format.obj
 0001:00006390       ??$?RUmonostate@v8@fmt@@$0A@@?$width_checker@Uerror_handler@detail@v8@fmt@@@detail@v8@fmt@@QEAA_KUmonostate@23@@Z 0000000180007390 f i format.obj
 0001:00006428       ??$?R_J$0A@@?$precision_checker@Uerror_handler@detail@v8@fmt@@@detail@v8@fmt@@QEAA_K_J@Z 0000000180007428 f i format.obj
 0001:000064d0       ??$?RM$0A@@?$precision_checker@Uerror_handler@detail@v8@fmt@@@detail@v8@fmt@@QEAA_KM@Z 00000001800074d0 f i format.obj
 0001:000064d0       ??$?RUmonostate@v8@fmt@@$0A@@?$precision_checker@Uerror_handler@detail@v8@fmt@@@detail@v8@fmt@@QEAA_KUmonostate@23@@Z 00000001800074d0 f i format.obj
 0001:000064d0       ??$?RPEBX$0A@@?$precision_checker@Uerror_handler@detail@v8@fmt@@@detail@v8@fmt@@QEAA_KPEBX@Z 00000001800074d0 f i format.obj
 0001:000064d0       ??$?RN$0A@@?$precision_checker@Uerror_handler@detail@v8@fmt@@@detail@v8@fmt@@QEAA_KN@Z 00000001800074d0 f i format.obj
 0001:000064d0       ??$?R_N$0A@@?$precision_checker@Uerror_handler@detail@v8@fmt@@@detail@v8@fmt@@QEAA_K_N@Z 00000001800074d0 f i format.obj
 0001:000064d0       ??$?RO$0A@@?$precision_checker@Uerror_handler@detail@v8@fmt@@@detail@v8@fmt@@QEAA_KO@Z 00000001800074d0 f i format.obj
 0001:00006568       ??1?$basic_memory_buffer@H$0BPE@V?$allocator@H@std@@@v8@fmt@@QEAA@XZ 0000000180007568 f i format.obj
 0001:00006598       ??$decimal_point@_W@detail@v8@fmt@@YA_WVlocale_ref@012@@Z 0000000180007598 f i handles.obj
 0001:00006668       ??1DebugToken@@QEAA@XZ     0000000180007668 f i handles.obj
 0001:00007218       ?PrintHandleInfo@@YA_NKPEAX_NPEAVPerfThread@@@Z 0000000180008218 f   handles.obj
 0001:00007830       ?c_str@?$basic_string@_WU?$char_traits@_W@std@@V?$allocator@_W@2@@std@@QEBAPEB_WXZ 0000000180008830 f i handles.obj
 0001:00007848       ??1?$unique_ptr@UPROCLIST_SYSTEM_HANDLE_INFORMATION@@Uvirtual_deleter@@@std@@QEAA@XZ 0000000180008848 f i handles.obj
 0001:00007870       ??1?$scoped_lock@VPerfThread@@@std@@QEAA@XZ 0000000180008870 f i handles.obj
 0001:00007890       ??1?$unique_ptr@_WUlocal_deleter@@@std@@QEAA@XZ 0000000180008890 f i handles.obj
 0001:000078b0       ??1?$unique_ptr@$$BY0A@DU?$default_delete@$$BY0A@D@std@@@std@@QEAA@XZ 00000001800088b0 f i handles.obj
 0001:000078b0       ??1?$unique_ptr@$$BY0A@_WU?$default_delete@$$BY0A@_W@std@@@std@@QEAA@XZ 00000001800088b0 f i handles.obj
 0001:000078c0       ??1?$unique_ptr@UPluginPanelItem@@Ufree_deleter@@@std@@QEAA@XZ 00000001800088c0 f i Pclass.obj
 0001:000078c0       ??1?$unique_ptr@XUfree_deleter@@@std@@QEAA@XZ 00000001800088c0 f i handles.obj
 0001:000078d0       ??1?$unique_ptr@XUhandle_closer@@@std@@QEAA@XZ 00000001800088d0 f i handles.obj
 0001:000078f0       ?empty@?$basic_string@_WU?$char_traits@_W@std@@V?$allocator@_W@2@@std@@QEBA_NXZ 00000001800088f0 f i handles.obj
 0001:00007900       ??B?$basic_string@_WU?$char_traits@_W@std@@V?$allocator@_W@2@@std@@QEBA?AV?$basic_string_view@_WU?$char_traits@_W@std@@@1@XZ 0000000180008900 f i handles.obj
 0001:00007920       ??0?$basic_string@_WU?$char_traits@_W@std@@V?$allocator@_W@2@@std@@QEAA@XZ 0000000180008920 f i handles.obj
 0001:00007948       ??0?$basic_string@_WU?$char_traits@_W@std@@V?$allocator@_W@2@@std@@QEAA@AEBV01@@Z 0000000180008948 f i handles.obj
 0001:000079f0       ?on_text@format_handler@?1???$vformat_to@_W@detail@v8@fmt@@YAXAEAV?$buffer@_W@234@V?$basic_string_view@_W@34@V?$basic_format_args@V?$basic_format_context@V?$back_insert_iterator@V?$buffer@_W@detail@v8@fmt@@@std@@_W@v8@fmt@@@34@Vlocale_ref@234@@Z@QEAAXPEB_W4@Z 00000001800089f0 f i handles.obj
 0001:00007a70       ?on_replacement_field@format_handler@?1???$vformat_to@_W@detail@v8@fmt@@YAXAEAV?$buffer@_W@234@V?$basic_string_view@_W@34@V?$basic_format_args@V?$basic_format_context@V?$back_insert_iterator@V?$buffer@_W@detail@v8@fmt@@@std@@_W@v8@fmt@@@34@Vlocale_ref@234@@Z@QEAAXHPEB_W@Z 0000000180008a70 f i handles.obj
 0001:00007ad0       ?check_arg_id@?$basic_format_parse_context@_WUerror_handler@detail@v8@fmt@@@v8@fmt@@QEAAXH@Z 0000000180008ad0 f i handles.obj
 0001:00007b88       ?next_arg_id@?$basic_format_parse_context@_WUerror_handler@detail@v8@fmt@@@v8@fmt@@QEAAHXZ 0000000180008b88 f i handles.obj
 0001:00007c40       ?append@?$basic_string@_WU?$char_traits@_W@std@@V?$allocator@_W@2@@std@@QEAAAEAV12@QEB_W_K@Z 0000000180008c40 f i handles.obj
 0001:00007db8       ??$visit_format_arg@U?$default_arg_formatter@_W@detail@v8@fmt@@V?$basic_format_context@V?$back_insert_iterator@V?$buffer@_W@detail@v8@fmt@@@std@@_W@34@@v8@fmt@@YA?AV?$back_insert_iterator@V?$buffer@_W@detail@v8@fmt@@@std@@$$QEAU?$default_arg_formatter@_W@detail@01@AEBV?$basic_format_arg@V?$basic_format_context@V?$back_insert_iterator@V?$buffer@_W@detail@v8@fmt@@@std@@_W@v8@fmt@@@01@@Z 0000000180008db8 f i handles.obj
 0001:000084e0       ??$get_arg@V?$basic_format_context@V?$back_insert_iterator@V?$buffer@_W@detail@v8@fmt@@@std@@_W@v8@fmt@@H@detail@v8@fmt@@YA?AV?$basic_format_arg@V?$basic_format_context@V?$back_insert_iterator@V?$buffer@_W@detail@v8@fmt@@@std@@_W@v8@fmt@@@12@AEAV?$basic_format_context@V?$back_insert_iterator@V?$buffer@_W@detail@v8@fmt@@@std@@_W@12@H@Z 00000001800094e0 f i handles.obj
 0001:00008608       ??$parse_format_specs@_WAEAV?$specs_checker@V?$specs_handler@_W@detail@v8@fmt@@@detail@v8@fmt@@@detail@v8@fmt@@YAPEB_WPEB_W0AEAV?$specs_checker@V?$specs_handler@_W@detail@v8@fmt@@@012@@Z 0000000180009608 f i handles.obj
 0001:00008800       ??$visit_format_arg@AEAU?$arg_formatter@_W@detail@v8@fmt@@V?$basic_format_context@V?$back_insert_iterator@V?$buffer@_W@detail@v8@fmt@@@std@@_W@34@@v8@fmt@@YA?AV?$back_insert_iterator@V?$buffer@_W@detail@v8@fmt@@@std@@AEAU?$arg_formatter@_W@detail@01@AEBV?$basic_format_arg@V?$basic_format_context@V?$back_insert_iterator@V?$buffer@_W@detail@v8@fmt@@@std@@_W@v8@fmt@@@01@@Z 0000000180009800 f i handles.obj
 0001:00008c30       ??$parse_format_string@$0A@_WUformat_handler@?1???$vformat_to@_W@detail@v8@fmt@@YAXAEAV?$buffer@_W@234@V?$basic_string_view@_W@34@V?$basic_format_args@V?$basic_format_context@V?$back_insert_iterator@V?$buffer@_W@detail@v8@fmt@@@std@@_W@v8@fmt@@@34@Vlocale_ref@234@@Z@@detail@v8@fmt@@YAXV?$basic_string_view@_W@12@$$QEAUformat_handler@?1???$vformat_to@_W@012@YAXAEAV?$buffer@_W@012@0V?$basic_format_args@V?$basic_format_context@V?$back_insert_iterator@V?$buffer@_W@detail@v8@fmt@@@std@@_W@v8@fmt@@@12@Vlocale_ref@012@@Z@@Z 0000000180009c30 f i handles.obj
 0001:00008ea8       ??Rwriter@?1???$parse_format_string@$0A@_WUformat_handler@?1???$vformat_to@_W@detail@v8@fmt@@YAXAEAV?$buffer@_W@234@V?$basic_string_view@_W@34@V?$basic_format_args@V?$basic_format_context@V?$back_insert_iterator@V?$buffer@_W@detail@v8@fmt@@@std@@_W@v8@fmt@@@34@Vlocale_ref@234@@Z@@detail@v8@fmt@@YAXV?$basic_string_view@_W@23@$$QEAUformat_handler@?1???$vformat_to@_W@123@YAXAEAV?$buffer@_W@123@0V?$basic_format_args@V?$basic_format_context@V?$back_insert_iterator@V?$buffer@_W@detail@v8@fmt@@@std@@_W@v8@fmt@@@23@Vlocale_ref@123@@Z@@Z@QEAAXPEB_W5@Z 0000000180009ea8 f i handles.obj
 0001:00009070       ??$parse_presentation_type@_W@detail@v8@fmt@@YA?AW4presentation_type@12@_W@Z 000000018000a070 f i handles.obj
 0001:00009158       ??$vformat@_W$0A@@v8@fmt@@YA?AV?$basic_string@_WU?$char_traits@_W@std@@V?$allocator@_W@2@@std@@V?$basic_string_view@_W@01@V?$basic_format_args@V?$basic_format_context@V?$back_insert_iterator@V?$buffer@_W@detail@v8@fmt@@@std@@_W@v8@fmt@@@01@@Z 000000018000a158 f i handles.obj
 0001:00009368       ??$get_id@_W@?$basic_format_args@V?$basic_format_context@V?$back_insert_iterator@V?$buffer@_W@detail@v8@fmt@@@std@@_W@v8@fmt@@@v8@fmt@@QEBAHV?$basic_string_view@_W@12@@Z 000000018000a368 f i handles.obj
 0001:00009430       ?on_sign@?$specs_checker@V?$specs_handler@_W@detail@v8@fmt@@@detail@v8@fmt@@QEAAXW4type@sign@34@@Z 000000018000a430 f i handles.obj
 0001:000094a0       ?require_numeric_argument@?$specs_checker@V?$specs_handler@_W@detail@v8@fmt@@@detail@v8@fmt@@AEAAXXZ 000000018000a4a0 f i handles.obj
 0001:00009548       ??$?RM@?$default_arg_formatter@_W@detail@v8@fmt@@QEAA?AV?$back_insert_iterator@V?$buffer@_W@detail@v8@fmt@@@std@@M@Z 000000018000a548 f i handles.obj
 0001:000096e8       ??$?RN@?$default_arg_formatter@_W@detail@v8@fmt@@QEAA?AV?$back_insert_iterator@V?$buffer@_W@detail@v8@fmt@@@std@@N@Z 000000018000a6e8 f i handles.obj
 0001:00009888       ??$?RO@?$default_arg_formatter@_W@detail@v8@fmt@@QEAA?AV?$back_insert_iterator@V?$buffer@_W@detail@v8@fmt@@@std@@O@Z 000000018000a888 f i handles.obj
 0001:00009a28       ??$parse_align@_WAEAV?$specs_checker@V?$specs_handler@_W@detail@v8@fmt@@@detail@v8@fmt@@@detail@v8@fmt@@YAPEB_WPEB_W0AEAV?$specs_checker@V?$specs_handler@_W@detail@v8@fmt@@@012@@Z 000000018000aa28 f i handles.obj
 0001:00009c18       ??$parse_width@_WAEAV?$specs_checker@V?$specs_handler@_W@detail@v8@fmt@@@detail@v8@fmt@@@detail@v8@fmt@@YAPEB_WPEB_W0AEAV?$specs_checker@V?$specs_handler@_W@detail@v8@fmt@@@012@@Z 000000018000ac18 f i handles.obj
 0001:00009f08       ?on_error@precision_adapter@?1???$parse_precision@_WAEAV?$specs_checker@V?$specs_handler@_W@detail@v8@fmt@@@detail@v8@fmt@@@detail@v8@fmt@@YAPEB_WPEB_W0AEAV?$specs_checker@V?$specs_handler@_W@detail@v8@fmt@@@234@@Z@QEAAXPEBD@Z 000000018000af08 f i handles.obj
 0001:00009f08       ?on_error@id_adapter@?1???$parse_replacement_field@_WAEAUformat_handler@?1???$vformat_to@_W@detail@v8@fmt@@YAXAEAV?$buffer@_W@234@V?$basic_string_view@_W@34@V?$basic_format_args@V?$basic_format_context@V?$back_insert_iterator@V?$buffer@_W@detail@v8@fmt@@@std@@_W@v8@fmt@@@34@Vlocale_ref@234@@Z@@detail@v8@fmt@@YAPEB_WPEB_W0AEAUformat_handler@?1???$vformat_to@_W@234@YAXAEAV?$buffer@_W@234@V?$basic_string_view@_W@34@V?$basic_format_args@V?$basic_format_context@V?$back_insert_iterator@V?$buffer@_W@detail@v8@fmt@@@std@@_W@v8@fmt@@@34@Vlocale_ref@234@@Z@@Z@QEAAXPEBD@Z 000000018000af08 f i handles.obj
 0001:00009f08       ?on_error@width_adapter@?1???$parse_width@_WAEAV?$specs_checker@V?$specs_handler@_W@detail@v8@fmt@@@detail@v8@fmt@@@detail@v8@fmt@@YAPEB_WPEB_W0AEAV?$specs_checker@V?$specs_handler@_W@detail@v8@fmt@@@234@@Z@QEAAXPEBD@Z 000000018000af08 f i handles.obj
 0001:00009fa0       ??$parse_precision@_WAEAV?$specs_checker@V?$specs_handler@_W@detail@v8@fmt@@@detail@v8@fmt@@@detail@v8@fmt@@YAPEB_WPEB_W0AEAV?$specs_checker@V?$specs_handler@_W@detail@v8@fmt@@@012@@Z 000000018000afa0 f i handles.obj
 0001:0000a3b8       ??$parse_replacement_field@_WAEAUformat_handler@?1???$vformat_to@_W@detail@v8@fmt@@YAXAEAV?$buffer@_W@234@V?$basic_string_view@_W@34@V?$basic_format_args@V?$basic_format_context@V?$back_insert_iterator@V?$buffer@_W@detail@v8@fmt@@@std@@_W@v8@fmt@@@34@Vlocale_ref@234@@Z@@detail@v8@fmt@@YAPEB_WPEB_W0AEAUformat_handler@?1???$vformat_to@_W@012@YAXAEAV?$buffer@_W@012@V?$basic_string_view@_W@12@V?$basic_format_args@V?$basic_format_context@V?$back_insert_iterator@V?$buffer@_W@detail@v8@fmt@@@std@@_W@v8@fmt@@@12@Vlocale_ref@012@@Z@@Z 000000018000b3b8 f i handles.obj
 0001:0000a720       ??$write@_WV?$back_insert_iterator@V?$buffer@_W@detail@v8@fmt@@@std@@@detail@v8@fmt@@YA?AV?$back_insert_iterator@V?$buffer@_W@detail@v8@fmt@@@std@@V34@V?$basic_string_view@_W@12@AEBU?$basic_format_specs@_W@12@Vlocale_ref@012@@Z 000000018000b720 f i handles.obj
 0001:0000a838       ??$write@_WV?$back_insert_iterator@V?$buffer@_W@detail@v8@fmt@@@std@@_N$0A@@detail@v8@fmt@@YA?AV?$back_insert_iterator@V?$buffer@_W@detail@v8@fmt@@@std@@V34@_NAEBU?$basic_format_specs@_W@12@Vlocale_ref@012@@Z 000000018000b838 f i handles.obj
 0001:0000a920       ??$write@_WV?$back_insert_iterator@V?$buffer@_W@detail@v8@fmt@@@std@@X$0A@@detail@v8@fmt@@YA?AV?$back_insert_iterator@V?$buffer@_W@detail@v8@fmt@@@std@@V34@PEBXAEBU?$basic_format_specs@_W@12@Vlocale_ref@012@@Z 000000018000b920 f i handles.obj
 0001:0000aa00       ??$write@_WV?$back_insert_iterator@V?$buffer@_W@detail@v8@fmt@@@std@@@detail@v8@fmt@@YA?AV?$back_insert_iterator@V?$buffer@_W@detail@v8@fmt@@@std@@V34@_WAEBU?$basic_format_specs@_W@12@Vlocale_ref@012@@Z 000000018000ba00 f i handles.obj
 0001:0000ac00       ??$write@_WV?$back_insert_iterator@V?$buffer@_W@detail@v8@fmt@@@std@@M$0A@@detail@v8@fmt@@YA?AV?$back_insert_iterator@V?$buffer@_W@detail@v8@fmt@@@std@@V34@MU?$basic_format_specs@_W@12@Vlocale_ref@012@@Z 000000018000bc00 f i handles.obj
 0001:0000af48       ??$write@_WV?$back_insert_iterator@V?$buffer@_W@detail@v8@fmt@@@std@@N$0A@@detail@v8@fmt@@YA?AV?$back_insert_iterator@V?$buffer@_W@detail@v8@fmt@@@std@@V34@NU?$basic_format_specs@_W@12@Vlocale_ref@012@@Z 000000018000bf48 f i handles.obj
 0001:0000b280       ??$write@_WV?$back_insert_iterator@V?$buffer@_W@detail@v8@fmt@@@std@@O$0A@@detail@v8@fmt@@YA?AV?$back_insert_iterator@V?$buffer@_W@detail@v8@fmt@@@std@@V34@OU?$basic_format_specs@_W@12@Vlocale_ref@012@@Z 000000018000c280 f i handles.obj
 0001:0000b5b8       ?get_arg@?$specs_handler@_W@detail@v8@fmt@@AEAA?AV?$basic_format_arg@V?$basic_format_context@V?$back_insert_iterator@V?$buffer@_W@detail@v8@fmt@@@std@@_W@v8@fmt@@@34@V?$basic_string_view@_W@34@@Z 000000018000c5b8 f i handles.obj
 0001:0000b710       ??$format_decimal@_WI@detail@v8@fmt@@YA?AU?$format_decimal_result@PEA_W@012@PEA_WIH@Z 000000018000c710 f i handles.obj
 0001:0000b7a0       ??$format_decimal@_WIV?$back_insert_iterator@V?$buffer@_W@detail@v8@fmt@@@std@@$0A@@detail@v8@fmt@@YA?AU?$format_decimal_result@V?$back_insert_iterator@V?$buffer@_W@detail@v8@fmt@@@std@@@012@V?$back_insert_iterator@V?$buffer@_W@detail@v8@fmt@@@std@@IH@Z 000000018000c7a0 f i handles.obj
 0001:0000b8b0       ??$format_decimal@_W_K@detail@v8@fmt@@YA?AU?$format_decimal_result@PEA_W@012@PEA_W_KH@Z 000000018000c8b0 f i handles.obj
 0001:0000b938       ??$format_decimal@_W_KV?$back_insert_iterator@V?$buffer@_W@detail@v8@fmt@@@std@@$0A@@detail@v8@fmt@@YA?AU?$format_decimal_result@V?$back_insert_iterator@V?$buffer@_W@detail@v8@fmt@@@std@@@012@V?$back_insert_iterator@V?$buffer@_W@detail@v8@fmt@@@std@@_KH@Z 000000018000c938 f i handles.obj
 0001:0000ba38       ??$write_ptr@_WV?$back_insert_iterator@V?$buffer@_W@detail@v8@fmt@@@std@@_K@detail@v8@fmt@@YA?AV?$back_insert_iterator@V?$buffer@_W@detail@v8@fmt@@@std@@V34@_KPEBU?$basic_format_specs@_W@12@@Z 000000018000ca38 f i handles.obj
 0001:0000bc10       ??$do_parse_arg_id@_WAEAUwidth_adapter@?1???$parse_width@_WAEAV?$specs_checker@V?$specs_handler@_W@detail@v8@fmt@@@detail@v8@fmt@@@detail@v8@fmt@@YAPEB_WPEB_W0AEAV?$specs_checker@V?$specs_handler@_W@detail@v8@fmt@@@234@@Z@@detail@v8@fmt@@YAPEB_WPEB_W0AEAUwidth_adapter@?1???$parse_width@_WAEAV?$specs_checker@V?$specs_handler@_W@detail@v8@fmt@@@detail@v8@fmt@@@012@YAPEB_W00AEAV?$specs_checker@V?$specs_handler@_W@detail@v8@fmt@@@012@@Z@@Z 000000018000cc10 f i handles.obj
 0001:0000bf60       ??$do_parse_arg_id@_WAEAUprecision_adapter@?1???$parse_precision@_WAEAV?$specs_checker@V?$specs_handler@_W@detail@v8@fmt@@@detail@v8@fmt@@@detail@v8@fmt@@YAPEB_WPEB_W0AEAV?$specs_checker@V?$specs_handler@_W@detail@v8@fmt@@@234@@Z@@detail@v8@fmt@@YAPEB_WPEB_W0AEAUprecision_adapter@?1???$parse_precision@_WAEAV?$specs_checker@V?$specs_handler@_W@detail@v8@fmt@@@detail@v8@fmt@@@012@YAPEB_W00AEAV?$specs_checker@V?$specs_handler@_W@detail@v8@fmt@@@012@@Z@@Z 000000018000cf60 f i handles.obj
 0001:0000c2b0       ??$parse_float_type_spec@Uerror_handler@detail@v8@fmt@@_W@detail@v8@fmt@@YA?AUfloat_specs@012@AEBU?$basic_format_specs@_W@12@$$QEAUerror_handler@012@@Z 000000018000d2b0 f i handles.obj
 0001:0000c470       ??$do_parse_arg_id@_WAEAUid_adapter@?1???$parse_replacement_field@_WAEAUformat_handler@?1???$vformat_to@_W@detail@v8@fmt@@YAXAEAV?$buffer@_W@234@V?$basic_string_view@_W@34@V?$basic_format_args@V?$basic_format_context@V?$back_insert_iterator@V?$buffer@_W@detail@v8@fmt@@@std@@_W@v8@fmt@@@34@Vlocale_ref@234@@Z@@detail@v8@fmt@@YAPEB_WPEB_W0AEAUformat_handler@?1???$vformat_to@_W@234@YAXAEAV?$buffer@_W@234@V?$basic_string_view@_W@34@V?$basic_format_args@V?$basic_format_context@V?$back_insert_iterator@V?$buffer@_W@detail@v8@fmt@@@std@@_W@v8@fmt@@@34@Vlocale_ref@234@@Z@@Z@@detail@v8@fmt@@YAPEB_WPEB_W0AEAUid_adapter@?1???$parse_replacement_field@_WAEAUformat_handler@?1???$vformat_to@_W@detail@v8@fmt@@YAXAEAV?$buffer@_W@234@V?$basic_string_view@_W@34@V?$basic_format_args@V?$basic_format_context@V?$back_insert_iterator@V?$buffer@_W@detail@v8@fmt@@@std@@_W@v8@fmt@@@34@Vlocale_ref@234@@Z@@012@YAPEB_W00AEAUformat_handler@?1???$vformat_to@_W@012@YAXAEAV?$buffer@_W@012@V?$basic_string_view@_W@12@V?$basic_format_args@V?$basic_format_context@V?$back_insert_iterator@V?$buffer@_W@detail@v8@fmt@@@std@@_W@v8@fmt@@@12@Vlocale_ref@012@@Z@@Z@@Z 000000018000d470 f i handles.obj
 0001:0000c6d0       ??$write_padded@$00V?$back_insert_iterator@V?$buffer@_W@detail@v8@fmt@@@std@@_WV<lambda_1>@?1???$write@_WV?$back_insert_iterator@V?$buffer@_W@detail@v8@fmt@@@std@@@detail@v8@fmt@@YA?AV12@V12@V?$basic_string_view@_W@56@AEBU?$basic_format_specs@_W@56@@Z@@detail@v8@fmt@@YA?AV?$back_insert_iterator@V?$buffer@_W@detail@v8@fmt@@@std@@V34@AEBU?$basic_format_specs@_W@12@_K2$$QEAV<lambda_1>@?1???$write@_WV?$back_insert_iterator@V?$buffer@_W@detail@v8@fmt@@@std@@@012@YA?AV34@0V?$basic_string_view@_W@12@1@Z@@Z 000000018000d6d0 f i handles.obj
 0001:0000c890       ??$write_int@_WV?$back_insert_iterator@V?$buffer@_W@detail@v8@fmt@@@std@@I@detail@v8@fmt@@YA?AV?$back_insert_iterator@V?$buffer@_W@detail@v8@fmt@@@std@@V34@U?$write_int_arg@I@012@AEBU?$basic_format_specs@_W@12@Vlocale_ref@012@@Z 000000018000d890 f i handles.obj
 0001:0000cd88       ??R<lambda_2>@?8???$write_int@_WV?$back_insert_iterator@V?$buffer@_W@detail@v8@fmt@@@std@@I@detail@v8@fmt@@YA?AV?$back_insert_iterator@V?$buffer@_W@detail@v8@fmt@@@std@@V45@U?$write_int_arg@I@123@AEBU?$basic_format_specs@_W@23@Vlocale_ref@123@@Z@QEBA@0@Z 000000018000dd88 f i handles.obj
 0001:0000cec8       ??$do_write_float@V?$back_insert_iterator@V?$buffer@_W@detail@v8@fmt@@@std@@U?$decimal_fp@M@dragonbox@detail@v8@fmt@@_WV?$digit_grouping@_W@567@@detail@v8@fmt@@YA?AV?$back_insert_iterator@V?$buffer@_W@detail@v8@fmt@@@std@@V34@AEBU?$decimal_fp@M@dragonbox@012@AEBU?$basic_format_specs@_W@12@Ufloat_specs@012@Vlocale_ref@012@@Z 000000018000dec8 f i handles.obj
 0001:0000d2e8       ??R<lambda_2>@?4???$do_write_float@V?$back_insert_iterator@V?$buffer@_W@detail@v8@fmt@@@std@@U?$decimal_fp@M@dragonbox@detail@v8@fmt@@_WV?$digit_grouping@_W@567@@detail@v8@fmt@@YA?AV?$back_insert_iterator@V?$buffer@_W@detail@v8@fmt@@@std@@V45@AEBU?$decimal_fp@M@dragonbox@123@AEBU?$basic_format_specs@_W@23@Ufloat_specs@123@Vlocale_ref@123@@Z@QEBA@0@Z 000000018000e2e8 f i handles.obj
 0001:0000d488       ??R<lambda_3>@?BD@???$do_write_float@V?$back_insert_iterator@V?$buffer@_W@detail@v8@fmt@@@std@@U?$decimal_fp@M@dragonbox@detail@v8@fmt@@_WV?$digit_grouping@_W@567@@detail@v8@fmt@@YA?AV?$back_insert_iterator@V?$buffer@_W@detail@v8@fmt@@@std@@V45@AEBU?$decimal_fp@M@dragonbox@123@AEBU?$basic_format_specs@_W@23@Ufloat_specs@123@Vlocale_ref@123@@Z@QEBA@0@Z 000000018000e488 f i handles.obj
 0001:0000d708       ??R<lambda_5>@?1???$do_write_float@V?$back_insert_iterator@V?$buffer@_W@detail@v8@fmt@@@std@@U?$decimal_fp@M@dragonbox@detail@v8@fmt@@_WV?$digit_grouping@_W@567@@detail@v8@fmt@@YA?AV?$back_insert_iterator@V?$buffer@_W@detail@v8@fmt@@@std@@V45@AEBU?$decimal_fp@M@dragonbox@123@AEBU?$basic_format_specs@_W@23@Ufloat_specs@123@Vlocale_ref@123@@Z@QEBA@0@Z 000000018000e708 f i handles.obj
 0001:0000d890       ??$do_write_float@V?$back_insert_iterator@V?$buffer@_W@detail@v8@fmt@@@std@@U?$decimal_fp@N@dragonbox@detail@v8@fmt@@_WV?$digit_grouping@_W@567@@detail@v8@fmt@@YA?AV?$back_insert_iterator@V?$buffer@_W@detail@v8@fmt@@@std@@V34@AEBU?$decimal_fp@N@dragonbox@012@AEBU?$basic_format_specs@_W@12@Ufloat_specs@012@Vlocale_ref@012@@Z 000000018000e890 f i handles.obj
 0001:0000dcc8       ??R<lambda_2>@?4???$do_write_float@V?$back_insert_iterator@V?$buffer@_W@detail@v8@fmt@@@std@@U?$decimal_fp@N@dragonbox@detail@v8@fmt@@_WV?$digit_grouping@_W@567@@detail@v8@fmt@@YA?AV?$back_insert_iterator@V?$buffer@_W@detail@v8@fmt@@@std@@V45@AEBU?$decimal_fp@N@dragonbox@123@AEBU?$basic_format_specs@_W@23@Ufloat_specs@123@Vlocale_ref@123@@Z@QEBA@0@Z 000000018000ecc8 f i handles.obj
 0001:0000de08       ??R<lambda_3>@?BD@???$do_write_float@V?$back_insert_iterator@V?$buffer@_W@detail@v8@fmt@@@std@@U?$decimal_fp@N@dragonbox@detail@v8@fmt@@_WV?$digit_grouping@_W@567@@detail@v8@fmt@@YA?AV?$back_insert_iterator@V?$buffer@_W@detail@v8@fmt@@@std@@V45@AEBU?$decimal_fp@N@dragonbox@123@AEBU?$basic_format_specs@_W@23@Ufloat_specs@123@Vlocale_ref@123@@Z@QEBA@0@Z 000000018000ee08 f i handles.obj
 0001:0000e088       ??R<lambda_4>@?BO@???$do_write_float@V?$back_insert_iterator@V?$buffer@_W@detail@v8@fmt@@@std@@U?$decimal_fp@N@dragonbox@detail@v8@fmt@@_WV?$digit_grouping@_W@567@@detail@v8@fmt@@YA?AV?$back_insert_iterator@V?$buffer@_W@detail@v8@fmt@@@std@@V45@AEBU?$decimal_fp@N@dragonbox@123@AEBU?$basic_format_specs@_W@23@Ufloat_specs@123@Vlocale_ref@123@@Z@QEBA@0@Z 000000018000f088 f i handles.obj
 0001:0000e290       ??R<lambda_5>@?1???$do_write_float@V?$back_insert_iterator@V?$buffer@_W@detail@v8@fmt@@@std@@U?$decimal_fp@N@dragonbox@detail@v8@fmt@@_WV?$digit_grouping@_W@567@@detail@v8@fmt@@YA?AV?$back_insert_iterator@V?$buffer@_W@detail@v8@fmt@@@std@@V45@AEBU?$decimal_fp@N@dragonbox@123@AEBU?$basic_format_specs@_W@23@Ufloat_specs@123@Vlocale_ref@123@@Z@QEBA@0@Z 000000018000f290 f i handles.obj
 0001:0000e418       ??$format_uint@$03_WV?$back_insert_iterator@V?$buffer@_W@detail@v8@fmt@@@std@@_K@detail@v8@fmt@@YA?AV?$back_insert_iterator@V?$buffer@_W@detail@v8@fmt@@@std@@V34@_KH_N@Z 000000018000f418 f i handles.obj
 0001:0000e550       ??$visit_format_arg@V?$width_checker@Uerror_handler@detail@v8@fmt@@@detail@v8@fmt@@V?$basic_format_context@V?$back_insert_iterator@V?$buffer@_W@detail@v8@fmt@@@std@@_W@34@@v8@fmt@@YA_K$$QEAV?$width_checker@Uerror_handler@detail@v8@fmt@@@detail@01@AEBV?$basic_format_arg@V?$basic_format_context@V?$back_insert_iterator@V?$buffer@_W@detail@v8@fmt@@@std@@_W@v8@fmt@@@01@@Z 000000018000f550 f i handles.obj
 0001:0000e888       ??$visit_format_arg@V?$precision_checker@Uerror_handler@detail@v8@fmt@@@detail@v8@fmt@@V?$basic_format_context@V?$back_insert_iterator@V?$buffer@_W@detail@v8@fmt@@@std@@_W@34@@v8@fmt@@YA_K$$QEAV?$precision_checker@Uerror_handler@detail@v8@fmt@@@detail@01@AEBV?$basic_format_arg@V?$basic_format_context@V?$back_insert_iterator@V?$buffer@_W@detail@v8@fmt@@@std@@_W@v8@fmt@@@01@@Z 000000018000f888 f i handles.obj
 0001:0000ebc0       ??$write_int@_WV?$back_insert_iterator@V?$buffer@_W@detail@v8@fmt@@@std@@_K@detail@v8@fmt@@YA?AV?$back_insert_iterator@V?$buffer@_W@detail@v8@fmt@@@std@@V34@U?$write_int_arg@_K@012@AEBU?$basic_format_specs@_W@12@Vlocale_ref@012@@Z 000000018000fbc0 f i handles.obj
 0001:0000f0a8       ??$do_write_float@V?$back_insert_iterator@V?$buffer@_W@detail@v8@fmt@@@std@@Ubig_decimal_fp@detail@v8@fmt@@_WV?$digit_grouping@_W@456@@detail@v8@fmt@@YA?AV?$back_insert_iterator@V?$buffer@_W@detail@v8@fmt@@@std@@V34@AEBUbig_decimal_fp@012@AEBU?$basic_format_specs@_W@12@Ufloat_specs@012@Vlocale_ref@012@@Z 00000001800100a8 f i handles.obj
 0001:0000f4a8       ??R<lambda_2>@?4???$do_write_float@V?$back_insert_iterator@V?$buffer@_W@detail@v8@fmt@@@std@@Ubig_decimal_fp@detail@v8@fmt@@_WV?$digit_grouping@_W@456@@detail@v8@fmt@@YA?AV?$back_insert_iterator@V?$buffer@_W@detail@v8@fmt@@@std@@V45@AEBUbig_decimal_fp@123@AEBU?$basic_format_specs@_W@23@Ufloat_specs@123@Vlocale_ref@123@@Z@QEBA@0@Z 00000001800104a8 f i handles.obj
 0001:0000f5e8       ??R<lambda_3>@?BD@???$do_write_float@V?$back_insert_iterator@V?$buffer@_W@detail@v8@fmt@@@std@@Ubig_decimal_fp@detail@v8@fmt@@_WV?$digit_grouping@_W@456@@detail@v8@fmt@@YA?AV?$back_insert_iterator@V?$buffer@_W@detail@v8@fmt@@@std@@V45@AEBUbig_decimal_fp@123@AEBU?$basic_format_specs@_W@23@Ufloat_specs@123@Vlocale_ref@123@@Z@QEBA@0@Z 00000001800105e8 f i handles.obj
 0001:0000f738       ??R<lambda_4>@?BO@???$do_write_float@V?$back_insert_iterator@V?$buffer@_W@detail@v8@fmt@@@std@@Ubig_decimal_fp@detail@v8@fmt@@_WV?$digit_grouping@_W@456@@detail@v8@fmt@@YA?AV?$back_insert_iterator@V?$buffer@_W@detail@v8@fmt@@@std@@V45@AEBUbig_decimal_fp@123@AEBU?$basic_format_specs@_W@23@Ufloat_specs@123@Vlocale_ref@123@@Z@QEBA@0@Z 0000000180010738 f i handles.obj
 0001:0000f940       ??R<lambda_5>@?1???$do_write_float@V?$back_insert_iterator@V?$buffer@_W@detail@v8@fmt@@@std@@Ubig_decimal_fp@detail@v8@fmt@@_WV?$digit_grouping@_W@456@@detail@v8@fmt@@YA?AV?$back_insert_iterator@V?$buffer@_W@detail@v8@fmt@@@std@@V45@AEBUbig_decimal_fp@123@AEBU?$basic_format_specs@_W@23@Ufloat_specs@123@Vlocale_ref@123@@Z@QEBA@0@Z 0000000180010940 f i handles.obj
 0001:0000fb00       ?count_separators@?$digit_grouping@_W@detail@v8@fmt@@QEBAHH@Z 0000000180010b00 f i handles.obj
 0001:0000fba8       ??0?$digit_grouping@_W@detail@v8@fmt@@QEAA@Vlocale_ref@123@_N@Z 0000000180010ba8 f i handles.obj
 0001:0000fc88       ??$fill@V?$back_insert_iterator@V?$buffer@_W@detail@v8@fmt@@@std@@_W@detail@v8@fmt@@YA?AV?$back_insert_iterator@V?$buffer@_W@detail@v8@fmt@@@std@@V34@_KAEBU?$fill_t@_W@012@@Z 0000000180010c88 f i handles.obj
 0001:0000fd80       ??$write_int_localized@V?$back_insert_iterator@V?$buffer@_W@detail@v8@fmt@@@std@@_K_W@detail@v8@fmt@@YA_NAEAV?$back_insert_iterator@V?$buffer@_W@detail@v8@fmt@@@std@@_KIAEBU?$basic_format_specs@_W@12@Vlocale_ref@012@@Z 0000000180010d80 f i handles.obj
 0001:0000ffc8       ??$write_int@V?$back_insert_iterator@V?$buffer@_W@detail@v8@fmt@@@std@@_WV<lambda_3>@?M@???$write_int@_WV?$back_insert_iterator@V?$buffer@_W@detail@v8@fmt@@@std@@I@detail@v8@fmt@@YA?AV12@V12@U?$write_int_arg@I@456@AEBU?$basic_format_specs@_W@56@Vlocale_ref@456@@Z@@detail@v8@fmt@@YA?AV?$back_insert_iterator@V?$buffer@_W@detail@v8@fmt@@@std@@V34@HIAEBU?$basic_format_specs@_W@12@V<lambda_3>@?M@???$write_int@_WV?$back_insert_iterator@V?$buffer@_W@detail@v8@fmt@@@std@@I@012@YA?AV34@0U?$write_int_arg@I@012@1Vlocale_ref@012@@Z@@Z 0000000180010fc8 f i handles.obj
 0001:000101c0       ??$write_int@V?$back_insert_iterator@V?$buffer@_W@detail@v8@fmt@@@std@@_WV<lambda_4>@?P@???$write_int@_WV?$back_insert_iterator@V?$buffer@_W@detail@v8@fmt@@@std@@I@detail@v8@fmt@@YA?AV12@V12@U?$write_int_arg@I@456@AEBU?$basic_format_specs@_W@56@Vlocale_ref@456@@Z@@detail@v8@fmt@@YA?AV?$back_insert_iterator@V?$buffer@_W@detail@v8@fmt@@@std@@V34@HIAEBU?$basic_format_specs@_W@12@V<lambda_4>@?P@???$write_int@_WV?$back_insert_iterator@V?$buffer@_W@detail@v8@fmt@@@std@@I@012@YA?AV34@0U?$write_int_arg@I@012@1Vlocale_ref@012@@Z@@Z 00000001800111c0 f i handles.obj
 0001:000103b8       ??$write_padded@$00V?$back_insert_iterator@V?$buffer@_W@detail@v8@fmt@@@std@@_WAEAV<lambda_1>@?1???$write_bytes@$00_WV?$back_insert_iterator@V?$buffer@_W@detail@v8@fmt@@@std@@@detail@v8@fmt@@YA?AV12@V12@V?$basic_string_view@D@56@AEBU?$basic_format_specs@_W@56@@Z@@detail@v8@fmt@@YA?AV?$back_insert_iterator@V?$buffer@_W@detail@v8@fmt@@@std@@V34@AEBU?$basic_format_specs@_W@12@_K2AEAV<lambda_1>@?1???$write_bytes@$00_WV?$back_insert_iterator@V?$buffer@_W@detail@v8@fmt@@@std@@@012@YA?AV34@0V?$basic_string_view@D@12@1@Z@@Z 00000001800113b8 f i handles.obj
 0001:00010578       ??$write_padded@$00V?$back_insert_iterator@V?$buffer@_W@detail@v8@fmt@@@std@@_WAEAV<lambda_1>@?1???$write_nonfinite@_WV?$back_insert_iterator@V?$buffer@_W@detail@v8@fmt@@@std@@@detail@v8@fmt@@YA?AV12@V12@_NU?$basic_format_specs@_W@56@AEBUfloat_specs@456@@Z@@detail@v8@fmt@@YA?AV?$back_insert_iterator@V?$buffer@_W@detail@v8@fmt@@@std@@V34@AEBU?$basic_format_specs@_W@12@_K2AEAV<lambda_1>@?1???$write_nonfinite@_WV?$back_insert_iterator@V?$buffer@_W@detail@v8@fmt@@@std@@@012@YA?AV34@0_NU512@AEBUfloat_specs@012@@Z@@Z 0000000180011578 f i handles.obj
 0001:00010788       ??$write_exponent@_WV?$back_insert_iterator@V?$buffer@_W@detail@v8@fmt@@@std@@@detail@v8@fmt@@YA?AV?$back_insert_iterator@V?$buffer@_W@detail@v8@fmt@@@std@@HV34@@Z 0000000180011788 f i handles.obj
 0001:00010960       ??$write_significand@V?$back_insert_iterator@V?$buffer@_W@detail@v8@fmt@@@std@@_WIV?$digit_grouping@_W@detail@v8@fmt@@@detail@v8@fmt@@YA?AV?$back_insert_iterator@V?$buffer@_W@detail@v8@fmt@@@std@@V34@IHH_WAEBV?$digit_grouping@_W@012@@Z 0000000180011960 f i handles.obj
 0001:00010b70       ??$write_significand@V?$back_insert_iterator@V?$buffer@_W@detail@v8@fmt@@@std@@_K_W$0A@@detail@v8@fmt@@YA?AV?$back_insert_iterator@V?$buffer@_W@detail@v8@fmt@@@std@@V34@_KHH_W@Z 0000000180011b70 f i handles.obj
 0001:00010d08       ??$write_padded@$01V?$back_insert_iterator@V?$buffer@_W@detail@v8@fmt@@@std@@_WAEAV<lambda_1>@?1???$write_ptr@_WV?$back_insert_iterator@V?$buffer@_W@detail@v8@fmt@@@std@@_K@detail@v8@fmt@@YA?AV12@V12@_KPEBU?$basic_format_specs@_W@56@@Z@@detail@v8@fmt@@YA?AV?$back_insert_iterator@V?$buffer@_W@detail@v8@fmt@@@std@@V34@AEBU?$basic_format_specs@_W@12@_K2AEAV<lambda_1>@?1???$write_ptr@_WV?$back_insert_iterator@V?$buffer@_W@detail@v8@fmt@@@std@@_K@012@YA?AV34@02PEBU512@@Z@@Z 0000000180011d08 f i handles.obj
 0001:00010fd0       ??$write_int@V?$back_insert_iterator@V?$buffer@_W@detail@v8@fmt@@@std@@_WV<lambda_3>@?M@???$write_int@_WV?$back_insert_iterator@V?$buffer@_W@detail@v8@fmt@@@std@@_K@detail@v8@fmt@@YA?AV12@V12@U?$write_int_arg@_K@456@AEBU?$basic_format_specs@_W@56@Vlocale_ref@456@@Z@@detail@v8@fmt@@YA?AV?$back_insert_iterator@V?$buffer@_W@detail@v8@fmt@@@std@@V34@HIAEBU?$basic_format_specs@_W@12@V<lambda_3>@?M@???$write_int@_WV?$back_insert_iterator@V?$buffer@_W@detail@v8@fmt@@@std@@_K@012@YA?AV34@0U?$write_int_arg@_K@012@1Vlocale_ref@012@@Z@@Z 0000000180011fd0 f i handles.obj
 0001:000111d0       ??$write_int@V?$back_insert_iterator@V?$buffer@_W@detail@v8@fmt@@@std@@_WV<lambda_4>@?P@???$write_int@_WV?$back_insert_iterator@V?$buffer@_W@detail@v8@fmt@@@std@@_K@detail@v8@fmt@@YA?AV12@V12@U?$write_int_arg@_K@456@AEBU?$basic_format_specs@_W@56@Vlocale_ref@456@@Z@@detail@v8@fmt@@YA?AV?$back_insert_iterator@V?$buffer@_W@detail@v8@fmt@@@std@@V34@HIAEBU?$basic_format_specs@_W@12@V<lambda_4>@?P@???$write_int@_WV?$back_insert_iterator@V?$buffer@_W@detail@v8@fmt@@@std@@_K@012@YA?AV34@0U?$write_int_arg@_K@012@1Vlocale_ref@012@@Z@@Z 00000001800121d0 f i handles.obj
 0001:000113d0       ??$write_padded@$00V?$back_insert_iterator@V?$buffer@_W@detail@v8@fmt@@@std@@_WAEAV<lambda_1>@?1???$write_char@_WV?$back_insert_iterator@V?$buffer@_W@detail@v8@fmt@@@std@@@detail@v8@fmt@@YA?AV12@V12@_WAEBU?$basic_format_specs@_W@56@@Z@@detail@v8@fmt@@YA?AV?$back_insert_iterator@V?$buffer@_W@detail@v8@fmt@@@std@@V34@AEBU?$basic_format_specs@_W@12@_K2AEAV<lambda_1>@?1???$write_char@_WV?$back_insert_iterator@V?$buffer@_W@detail@v8@fmt@@@std@@@012@YA?AV34@0_W1@Z@@Z 00000001800123d0 f i handles.obj
 0001:00011578       ??$write_padded@$01V?$back_insert_iterator@V?$buffer@_W@detail@v8@fmt@@@std@@_WAEAV<lambda_1>@?1???$write_bytes@$01_WV?$back_insert_iterator@V?$buffer@_W@detail@v8@fmt@@@std@@@detail@v8@fmt@@YA?AV12@V12@V?$basic_string_view@D@56@AEBU?$basic_format_specs@_W@56@@Z@@detail@v8@fmt@@YA?AV?$back_insert_iterator@V?$buffer@_W@detail@v8@fmt@@@std@@V34@AEBU?$basic_format_specs@_W@12@_K2AEAV<lambda_1>@?1???$write_bytes@$01_WV?$back_insert_iterator@V?$buffer@_W@detail@v8@fmt@@@std@@@012@YA?AV34@0V?$basic_string_view@D@12@1@Z@@Z 0000000180012578 f i handles.obj
 0001:00011738       ??$write_significand@V?$back_insert_iterator@V?$buffer@_W@detail@v8@fmt@@@std@@_W@detail@v8@fmt@@YA?AV?$back_insert_iterator@V?$buffer@_W@detail@v8@fmt@@@std@@V34@PEBDHH_W@Z 0000000180012738 f i handles.obj
 0001:00011870       ??$write_significand@_WV?$back_insert_iterator@V?$buffer@_W@detail@v8@fmt@@@std@@PEBDV?$digit_grouping@_W@detail@v8@fmt@@@detail@v8@fmt@@YA?AV?$back_insert_iterator@V?$buffer@_W@detail@v8@fmt@@@std@@V34@PEBDHHAEBV?$digit_grouping@_W@012@@Z 0000000180012870 f i handles.obj
 0001:00011a98       ??$write_significand@_WI$0A@@detail@v8@fmt@@YAPEA_WPEA_WIHH_W@Z 0000000180012a98 f i handles.obj
 0001:00011bb8       ??$write_padded@$01V?$back_insert_iterator@V?$buffer@_W@detail@v8@fmt@@@std@@_WAEAV<lambda_2>@?4???$do_write_float@V?$back_insert_iterator@V?$buffer@_W@detail@v8@fmt@@@std@@U?$decimal_fp@M@dragonbox@detail@v8@fmt@@_WV?$digit_grouping@_W@567@@detail@v8@fmt@@YA?AV12@V12@AEBU?$decimal_fp@M@dragonbox@456@AEBU?$basic_format_specs@_W@56@Ufloat_specs@456@Vlocale_ref@456@@Z@@detail@v8@fmt@@YA?AV?$back_insert_iterator@V?$buffer@_W@detail@v8@fmt@@@std@@V34@AEBU?$basic_format_specs@_W@12@_K2AEAV<lambda_2>@?4???$do_write_float@V?$back_insert_iterator@V?$buffer@_W@detail@v8@fmt@@@std@@U?$decimal_fp@M@dragonbox@detail@v8@fmt@@_WV?$digit_grouping@_W@567@@012@YA?AV34@0AEBU?$decimal_fp@M@dragonbox@012@1Ufloat_specs@012@Vlocale_ref@012@@Z@@Z 0000000180012bb8 f i handles.obj
 0001:00011d30       ??$apply@V?$back_insert_iterator@V?$buffer@_W@detail@v8@fmt@@@std@@D@?$digit_grouping@_W@detail@v8@fmt@@QEBA?AV?$back_insert_iterator@V?$buffer@_W@detail@v8@fmt@@@std@@V45@V?$basic_string_view@D@23@@Z 0000000180012d30 f i handles.obj
 0001:00011f78       ??$write_padded@$01V?$back_insert_iterator@V?$buffer@_W@detail@v8@fmt@@@std@@_WAEAV<lambda_3>@?BD@???$do_write_float@V?$back_insert_iterator@V?$buffer@_W@detail@v8@fmt@@@std@@U?$decimal_fp@M@dragonbox@detail@v8@fmt@@_WV?$digit_grouping@_W@567@@detail@v8@fmt@@YA?AV12@V12@AEBU?$decimal_fp@M@dragonbox@456@AEBU?$basic_format_specs@_W@56@Ufloat_specs@456@Vlocale_ref@456@@Z@@detail@v8@fmt@@YA?AV?$back_insert_iterator@V?$buffer@_W@detail@v8@fmt@@@std@@V34@AEBU?$basic_format_specs@_W@12@_K2AEAV<lambda_3>@?BD@???$do_write_float@V?$back_insert_iterator@V?$buffer@_W@detail@v8@fmt@@@std@@U?$decimal_fp@M@dragonbox@detail@v8@fmt@@_WV?$digit_grouping@_W@567@@012@YA?AV34@0AEBU?$decimal_fp@M@dragonbox@012@1Ufloat_specs@012@Vlocale_ref@012@@Z@@Z 0000000180012f78 f i handles.obj
 0001:000120f0       ??$apply@V?$back_insert_iterator@V?$buffer@_W@detail@v8@fmt@@@std@@_W@?$digit_grouping@_W@detail@v8@fmt@@QEBA?AV?$back_insert_iterator@V?$buffer@_W@detail@v8@fmt@@@std@@V45@V?$basic_string_view@_W@23@@Z 00000001800130f0 f i handles.obj
 0001:00012338       ??$write_padded@$01V?$back_insert_iterator@V?$buffer@_W@detail@v8@fmt@@@std@@_WAEAV<lambda_4>@?BO@???$do_write_float@V?$back_insert_iterator@V?$buffer@_W@detail@v8@fmt@@@std@@U?$decimal_fp@M@dragonbox@detail@v8@fmt@@_WV?$digit_grouping@_W@567@@detail@v8@fmt@@YA?AV12@V12@AEBU?$decimal_fp@M@dragonbox@456@AEBU?$basic_format_specs@_W@56@Ufloat_specs@456@Vlocale_ref@456@@Z@@detail@v8@fmt@@YA?AV?$back_insert_iterator@V?$buffer@_W@detail@v8@fmt@@@std@@V34@AEBU?$basic_format_specs@_W@12@_K2AEAV<lambda_4>@?BO@???$do_write_float@V?$back_insert_iterator@V?$buffer@_W@detail@v8@fmt@@@std@@U?$decimal_fp@M@dragonbox@detail@v8@fmt@@_WV?$digit_grouping@_W@567@@012@YA?AV34@0AEBU?$decimal_fp@M@dragonbox@012@1Ufloat_specs@012@Vlocale_ref@012@@Z@@Z 0000000180013338 f i handles.obj
 0001:00012578       ??$write_padded@$01V?$back_insert_iterator@V?$buffer@_W@detail@v8@fmt@@@std@@_WAEAV<lambda_5>@?1???$do_write_float@V?$back_insert_iterator@V?$buffer@_W@detail@v8@fmt@@@std@@U?$decimal_fp@M@dragonbox@detail@v8@fmt@@_WV?$digit_grouping@_W@567@@detail@v8@fmt@@YA?AV12@V12@AEBU?$decimal_fp@M@dragonbox@456@AEBU?$basic_format_specs@_W@56@Ufloat_specs@456@Vlocale_ref@456@@Z@@detail@v8@fmt@@YA?AV?$back_insert_iterator@V?$buffer@_W@detail@v8@fmt@@@std@@V34@AEBU?$basic_format_specs@_W@12@_K2AEAV<lambda_5>@?1???$do_write_float@V?$back_insert_iterator@V?$buffer@_W@detail@v8@fmt@@@std@@U?$decimal_fp@M@dragonbox@detail@v8@fmt@@_WV?$digit_grouping@_W@567@@012@YA?AV34@0AEBU?$decimal_fp@M@dragonbox@012@1Ufloat_specs@012@Vlocale_ref@012@@Z@@Z 0000000180013578 f i handles.obj
 0001:000126f0       ??$write_padded@$01V?$back_insert_iterator@V?$buffer@_W@detail@v8@fmt@@@std@@_WAEAV<lambda_2>@?4???$do_write_float@V?$back_insert_iterator@V?$buffer@_W@detail@v8@fmt@@@std@@U?$decimal_fp@N@dragonbox@detail@v8@fmt@@_WV?$digit_grouping@_W@567@@detail@v8@fmt@@YA?AV12@V12@AEBU?$decimal_fp@N@dragonbox@456@AEBU?$basic_format_specs@_W@56@Ufloat_specs@456@Vlocale_ref@456@@Z@@detail@v8@fmt@@YA?AV?$back_insert_iterator@V?$buffer@_W@detail@v8@fmt@@@std@@V34@AEBU?$basic_format_specs@_W@12@_K2AEAV<lambda_2>@?4???$do_write_float@V?$back_insert_iterator@V?$buffer@_W@detail@v8@fmt@@@std@@U?$decimal_fp@N@dragonbox@detail@v8@fmt@@_WV?$digit_grouping@_W@567@@012@YA?AV34@0AEBU?$decimal_fp@N@dragonbox@012@1Ufloat_specs@012@Vlocale_ref@012@@Z@@Z 00000001800136f0 f i handles.obj
 0001:00012868       ??$write_padded@$01V?$back_insert_iterator@V?$buffer@_W@detail@v8@fmt@@@std@@_WAEAV<lambda_3>@?BD@???$do_write_float@V?$back_insert_iterator@V?$buffer@_W@detail@v8@fmt@@@std@@U?$decimal_fp@N@dragonbox@detail@v8@fmt@@_WV?$digit_grouping@_W@567@@detail@v8@fmt@@YA?AV12@V12@AEBU?$decimal_fp@N@dragonbox@456@AEBU?$basic_format_specs@_W@56@Ufloat_specs@456@Vlocale_ref@456@@Z@@detail@v8@fmt@@YA?AV?$back_insert_iterator@V?$buffer@_W@detail@v8@fmt@@@std@@V34@AEBU?$basic_format_specs@_W@12@_K2AEAV<lambda_3>@?BD@???$do_write_float@V?$back_insert_iterator@V?$buffer@_W@detail@v8@fmt@@@std@@U?$decimal_fp@N@dragonbox@detail@v8@fmt@@_WV?$digit_grouping@_W@567@@012@YA?AV34@0AEBU?$decimal_fp@N@dragonbox@012@1Ufloat_specs@012@Vlocale_ref@012@@Z@@Z 0000000180013868 f i handles.obj
 0001:000129e0       ??$write_padded@$01V?$back_insert_iterator@V?$buffer@_W@detail@v8@fmt@@@std@@_WAEAV<lambda_4>@?BO@???$do_write_float@V?$back_insert_iterator@V?$buffer@_W@detail@v8@fmt@@@std@@U?$decimal_fp@N@dragonbox@detail@v8@fmt@@_WV?$digit_grouping@_W@567@@detail@v8@fmt@@YA?AV12@V12@AEBU?$decimal_fp@N@dragonbox@456@AEBU?$basic_format_specs@_W@56@Ufloat_specs@456@Vlocale_ref@456@@Z@@detail@v8@fmt@@YA?AV?$back_insert_iterator@V?$buffer@_W@detail@v8@fmt@@@std@@V34@AEBU?$basic_format_specs@_W@12@_K2AEAV<lambda_4>@?BO@???$do_write_float@V?$back_insert_iterator@V?$buffer@_W@detail@v8@fmt@@@std@@U?$decimal_fp@N@dragonbox@detail@v8@fmt@@_WV?$digit_grouping@_W@567@@012@YA?AV34@0AEBU?$decimal_fp@N@dragonbox@012@1Ufloat_specs@012@Vlocale_ref@012@@Z@@Z 00000001800139e0 f i handles.obj
 0001:00012b58       ??$write_padded@$01V?$back_insert_iterator@V?$buffer@_W@detail@v8@fmt@@@std@@_WAEAV<lambda_5>@?1???$do_write_float@V?$back_insert_iterator@V?$buffer@_W@detail@v8@fmt@@@std@@U?$decimal_fp@N@dragonbox@detail@v8@fmt@@_WV?$digit_grouping@_W@567@@detail@v8@fmt@@YA?AV12@V12@AEBU?$decimal_fp@N@dragonbox@456@AEBU?$basic_format_specs@_W@56@Ufloat_specs@456@Vlocale_ref@456@@Z@@detail@v8@fmt@@YA?AV?$back_insert_iterator@V?$buffer@_W@detail@v8@fmt@@@std@@V34@AEBU?$basic_format_specs@_W@12@_K2AEAV<lambda_5>@?1???$do_write_float@V?$back_insert_iterator@V?$buffer@_W@detail@v8@fmt@@@std@@U?$decimal_fp@N@dragonbox@detail@v8@fmt@@_WV?$digit_grouping@_W@567@@012@YA?AV34@0AEBU?$decimal_fp@N@dragonbox@012@1Ufloat_specs@012@Vlocale_ref@012@@Z@@Z 0000000180013b58 f i handles.obj
 0001:00012cd0       ??$write_padded@$01V?$back_insert_iterator@V?$buffer@_W@detail@v8@fmt@@@std@@_WAEAV<lambda_2>@?4???$do_write_float@V?$back_insert_iterator@V?$buffer@_W@detail@v8@fmt@@@std@@Ubig_decimal_fp@detail@v8@fmt@@_WV?$digit_grouping@_W@456@@detail@v8@fmt@@YA?AV12@V12@AEBUbig_decimal_fp@456@AEBU?$basic_format_specs@_W@56@Ufloat_specs@456@Vlocale_ref@456@@Z@@detail@v8@fmt@@YA?AV?$back_insert_iterator@V?$buffer@_W@detail@v8@fmt@@@std@@V34@AEBU?$basic_format_specs@_W@12@_K2AEAV<lambda_2>@?4???$do_write_float@V?$back_insert_iterator@V?$buffer@_W@detail@v8@fmt@@@std@@Ubig_decimal_fp@detail@v8@fmt@@_WV?$digit_grouping@_W@456@@012@YA?AV34@0AEBUbig_decimal_fp@012@1Ufloat_specs@012@Vlocale_ref@012@@Z@@Z 0000000180013cd0 f i handles.obj
 0001:00012e48       ??$write_padded@$01V?$back_insert_iterator@V?$buffer@_W@detail@v8@fmt@@@std@@_WAEAV<lambda_3>@?BD@???$do_write_float@V?$back_insert_iterator@V?$buffer@_W@detail@v8@fmt@@@std@@Ubig_decimal_fp@detail@v8@fmt@@_WV?$digit_grouping@_W@456@@detail@v8@fmt@@YA?AV12@V12@AEBUbig_decimal_fp@456@AEBU?$basic_format_specs@_W@56@Ufloat_specs@456@Vlocale_ref@456@@Z@@detail@v8@fmt@@YA?AV?$back_insert_iterator@V?$buffer@_W@detail@v8@fmt@@@std@@V34@AEBU?$basic_format_specs@_W@12@_K2AEAV<lambda_3>@?BD@???$do_write_float@V?$back_insert_iterator@V?$buffer@_W@detail@v8@fmt@@@std@@Ubig_decimal_fp@detail@v8@fmt@@_WV?$digit_grouping@_W@456@@012@YA?AV34@0AEBUbig_decimal_fp@012@1Ufloat_specs@012@Vlocale_ref@012@@Z@@Z 0000000180013e48 f i handles.obj
 0001:00012fc0       ??$write_padded@$01V?$back_insert_iterator@V?$buffer@_W@detail@v8@fmt@@@std@@_WAEAV<lambda_4>@?BO@???$do_write_float@V?$back_insert_iterator@V?$buffer@_W@detail@v8@fmt@@@std@@Ubig_decimal_fp@detail@v8@fmt@@_WV?$digit_grouping@_W@456@@detail@v8@fmt@@YA?AV12@V12@AEBUbig_decimal_fp@456@AEBU?$basic_format_specs@_W@56@Ufloat_specs@456@Vlocale_ref@456@@Z@@detail@v8@fmt@@YA?AV?$back_insert_iterator@V?$buffer@_W@detail@v8@fmt@@@std@@V34@AEBU?$basic_format_specs@_W@12@_K2AEAV<lambda_4>@?BO@???$do_write_float@V?$back_insert_iterator@V?$buffer@_W@detail@v8@fmt@@@std@@Ubig_decimal_fp@detail@v8@fmt@@_WV?$digit_grouping@_W@456@@012@YA?AV34@0AEBUbig_decimal_fp@012@1Ufloat_specs@012@Vlocale_ref@012@@Z@@Z 0000000180013fc0 f i handles.obj
 0001:00013138       ??$write_padded@$01V?$back_insert_iterator@V?$buffer@_W@detail@v8@fmt@@@std@@_WAEAV<lambda_5>@?1???$do_write_float@V?$back_insert_iterator@V?$buffer@_W@detail@v8@fmt@@@std@@Ubig_decimal_fp@detail@v8@fmt@@_WV?$digit_grouping@_W@456@@detail@v8@fmt@@YA?AV12@V12@AEBUbig_decimal_fp@456@AEBU?$basic_format_specs@_W@56@Ufloat_specs@456@Vlocale_ref@456@@Z@@detail@v8@fmt@@YA?AV?$back_insert_iterator@V?$buffer@_W@detail@v8@fmt@@@std@@V34@AEBU?$basic_format_specs@_W@12@_K2AEAV<lambda_5>@?1???$do_write_float@V?$back_insert_iterator@V?$buffer@_W@detail@v8@fmt@@@std@@Ubig_decimal_fp@detail@v8@fmt@@_WV?$digit_grouping@_W@456@@012@YA?AV34@0AEBUbig_decimal_fp@012@1Ufloat_specs@012@Vlocale_ref@012@@Z@@Z 0000000180014138 f i handles.obj
 0001:000132b0       ??$write_padded@$01V?$back_insert_iterator@V?$buffer@_W@detail@v8@fmt@@@std@@_WV<lambda_1>@?1???$write_int_localized@V?$back_insert_iterator@V?$buffer@_W@detail@v8@fmt@@@std@@_K_W@detail@v8@fmt@@YA?AV12@V12@_KIAEBU?$basic_format_specs@_W@56@AEBV?$digit_grouping@_W@456@@Z@@detail@v8@fmt@@YA?AV?$back_insert_iterator@V?$buffer@_W@detail@v8@fmt@@@std@@V34@AEBU?$basic_format_specs@_W@12@_K2$$QEAV<lambda_1>@?1???$write_int_localized@V?$back_insert_iterator@V?$buffer@_W@detail@v8@fmt@@@std@@_K_W@012@YA?AV34@02I1AEBV?$digit_grouping@_W@012@@Z@@Z 00000001800142b0 f i handles.obj
 0001:00013480       ??$write_padded@$01V?$back_insert_iterator@V?$buffer@_W@detail@v8@fmt@@@std@@_WAEAV<lambda_1>@?1???$write_int@V?$back_insert_iterator@V?$buffer@_W@detail@v8@fmt@@@std@@_WV<lambda_1>@?4???$write_int@_WV?$back_insert_iterator@V?$buffer@_W@detail@v8@fmt@@@std@@I@detail@v8@fmt@@YA?AV12@V12@U?$write_int_arg@I@456@AEBU?$basic_format_specs@_W@56@Vlocale_ref@456@@Z@@detail@v8@fmt@@YA?AV12@V12@HIAEBU?$basic_format_specs@_W@56@V3?4???$write_int@_WV?$back_insert_iterator@V?$buffer@_W@detail@v8@fmt@@@std@@I@456@YA?AV12@0U?$write_int_arg@I@456@1Vlocale_ref@456@@Z@@Z@@detail@v8@fmt@@YA?AV?$back_insert_iterator@V?$buffer@_W@detail@v8@fmt@@@std@@V34@AEBU?$basic_format_specs@_W@12@_K2AEAV<lambda_1>@?1???$write_int@V?$back_insert_iterator@V?$buffer@_W@detail@v8@fmt@@@std@@_WV<lambda_1>@?4???$write_int@_WV?$back_insert_iterator@V?$buffer@_W@detail@v8@fmt@@@std@@I@detail@v8@fmt@@YA?AV12@V12@U?$write_int_arg@I@456@AEBU?$basic_format_specs@_W@56@Vlocale_ref@456@@Z@@012@YA?AV34@0HI1V6?4???$write_int@_WV?$back_insert_iterator@V?$buffer@_W@detail@v8@fmt@@@std@@I@012@YA?AV34@0U?$write_int_arg@I@012@1Vlocale_ref@012@@Z@@Z@@Z 0000000180014480 f i handles.obj
 0001:00013698       ??$write_padded@$01V?$back_insert_iterator@V?$buffer@_W@detail@v8@fmt@@@std@@_WAEAV<lambda_1>@?1???$write_int@V?$back_insert_iterator@V?$buffer@_W@detail@v8@fmt@@@std@@_WV<lambda_2>@?8???$write_int@_WV?$back_insert_iterator@V?$buffer@_W@detail@v8@fmt@@@std@@I@detail@v8@fmt@@YA?AV12@V12@U?$write_int_arg@I@456@AEBU?$basic_format_specs@_W@56@Vlocale_ref@456@@Z@@detail@v8@fmt@@YA?AV12@V12@HIAEBU?$basic_format_specs@_W@56@V<lambda_2>@?8???$write_int@_WV?$back_insert_iterator@V?$buffer@_W@detail@v8@fmt@@@std@@I@456@YA?AV12@0U?$write_int_arg@I@456@1Vlocale_ref@456@@Z@@Z@@detail@v8@fmt@@YA?AV?$back_insert_iterator@V?$buffer@_W@detail@v8@fmt@@@std@@V34@AEBU?$basic_format_specs@_W@12@_K2AEAV<lambda_1>@?1???$write_int@V?$back_insert_iterator@V?$buffer@_W@detail@v8@fmt@@@std@@_WV<lambda_2>@?8???$write_int@_WV?$back_insert_iterator@V?$buffer@_W@detail@v8@fmt@@@std@@I@detail@v8@fmt@@YA?AV12@V12@U?$write_int_arg@I@456@AEBU?$basic_format_specs@_W@56@Vlocale_ref@456@@Z@@012@YA?AV34@0HI1V<lambda_2>@?8???$write_int@_WV?$back_insert_iterator@V?$buffer@_W@detail@v8@fmt@@@std@@I@012@YA?AV34@0U?$write_int_arg@I@012@1Vlocale_ref@012@@Z@@Z@@Z 0000000180014698 f i handles.obj
 0001:000138b8       ??$write_padded@$01V?$back_insert_iterator@V?$buffer@_W@detail@v8@fmt@@@std@@_WAEAV<lambda_1>@?1???$write_int@V?$back_insert_iterator@V?$buffer@_W@detail@v8@fmt@@@std@@_WV<lambda_3>@?M@???$write_int@_WV?$back_insert_iterator@V?$buffer@_W@detail@v8@fmt@@@std@@I@detail@v8@fmt@@YA?AV12@V12@U?$write_int_arg@I@456@AEBU?$basic_format_specs@_W@56@Vlocale_ref@456@@Z@@detail@v8@fmt@@YA?AV12@V12@HIAEBU?$basic_format_specs@_W@56@V<lambda_3>@?M@???$write_int@_WV?$back_insert_iterator@V?$buffer@_W@detail@v8@fmt@@@std@@I@456@YA?AV12@0U?$write_int_arg@I@456@1Vlocale_ref@456@@Z@@Z@@detail@v8@fmt@@YA?AV?$back_insert_iterator@V?$buffer@_W@detail@v8@fmt@@@std@@V34@AEBU?$basic_format_specs@_W@12@_K2AEAV<lambda_1>@?1???$write_int@V?$back_insert_iterator@V?$buffer@_W@detail@v8@fmt@@@std@@_WV<lambda_3>@?M@???$write_int@_WV?$back_insert_iterator@V?$buffer@_W@detail@v8@fmt@@@std@@I@detail@v8@fmt@@YA?AV12@V12@U?$write_int_arg@I@456@AEBU?$basic_format_specs@_W@56@Vlocale_ref@456@@Z@@012@YA?AV34@0HI1V<lambda_3>@?M@???$write_int@_WV?$back_insert_iterator@V?$buffer@_W@detail@v8@fmt@@@std@@I@012@YA?AV34@0U?$write_int_arg@I@012@1Vlocale_ref@012@@Z@@Z@@Z 00000001800148b8 f i handles.obj
 0001:00013b98       ??$write_padded@$01V?$back_insert_iterator@V?$buffer@_W@detail@v8@fmt@@@std@@_WAEAV<lambda_1>@?1???$write_int@V?$back_insert_iterator@V?$buffer@_W@detail@v8@fmt@@@std@@_WV<lambda_4>@?P@???$write_int@_WV?$back_insert_iterator@V?$buffer@_W@detail@v8@fmt@@@std@@I@detail@v8@fmt@@YA?AV12@V12@U?$write_int_arg@I@456@AEBU?$basic_format_specs@_W@56@Vlocale_ref@456@@Z@@detail@v8@fmt@@YA?AV12@V12@HIAEBU?$basic_format_specs@_W@56@V<lambda_4>@?P@???$write_int@_WV?$back_insert_iterator@V?$buffer@_W@detail@v8@fmt@@@std@@I@456@YA?AV12@0U?$write_int_arg@I@456@1Vlocale_ref@456@@Z@@Z@@detail@v8@fmt@@YA?AV?$back_insert_iterator@V?$buffer@_W@detail@v8@fmt@@@std@@V34@AEBU?$basic_format_specs@_W@12@_K2AEAV<lambda_1>@?1???$write_int@V?$back_insert_iterator@V?$buffer@_W@detail@v8@fmt@@@std@@_WV<lambda_4>@?P@???$write_int@_WV?$back_insert_iterator@V?$buffer@_W@detail@v8@fmt@@@std@@I@detail@v8@fmt@@YA?AV12@V12@U?$write_int_arg@I@456@AEBU?$basic_format_specs@_W@56@Vlocale_ref@456@@Z@@012@YA?AV34@0HI1V<lambda_4>@?P@???$write_int@_WV?$back_insert_iterator@V?$buffer@_W@detail@v8@fmt@@@std@@I@012@YA?AV34@0U?$write_int_arg@I@012@1Vlocale_ref@012@@Z@@Z@@Z 0000000180014b98 f i handles.obj
 0001:00013e78       ??$write_padded@$01V?$back_insert_iterator@V?$buffer@_W@detail@v8@fmt@@@std@@_WAEAV<lambda_1>@?1???$write_int@V?$back_insert_iterator@V?$buffer@_W@detail@v8@fmt@@@std@@_WV<lambda_1>@?4???$write_int@_WV?$back_insert_iterator@V?$buffer@_W@detail@v8@fmt@@@std@@_K@detail@v8@fmt@@YA?AV12@V12@U?$write_int_arg@_K@456@AEBU?$basic_format_specs@_W@56@Vlocale_ref@456@@Z@@detail@v8@fmt@@YA?AV12@V12@HIAEBU?$basic_format_specs@_W@56@V3?4???$write_int@_WV?$back_insert_iterator@V?$buffer@_W@detail@v8@fmt@@@std@@_K@456@YA?AV12@0U?$write_int_arg@_K@456@1Vlocale_ref@456@@Z@@Z@@detail@v8@fmt@@YA?AV?$back_insert_iterator@V?$buffer@_W@detail@v8@fmt@@@std@@V34@AEBU?$basic_format_specs@_W@12@_K2AEAV<lambda_1>@?1???$write_int@V?$back_insert_iterator@V?$buffer@_W@detail@v8@fmt@@@std@@_WV<lambda_1>@?4???$write_int@_WV?$back_insert_iterator@V?$buffer@_W@detail@v8@fmt@@@std@@_K@detail@v8@fmt@@YA?AV12@V12@U?$write_int_arg@_K@456@AEBU?$basic_format_specs@_W@56@Vlocale_ref@456@@Z@@012@YA?AV34@0HI1V6?4???$write_int@_WV?$back_insert_iterator@V?$buffer@_W@detail@v8@fmt@@@std@@_K@012@YA?AV34@0U?$write_int_arg@_K@012@1Vlocale_ref@012@@Z@@Z@@Z 0000000180014e78 f i handles.obj
 0001:00014098       ??$write_padded@$01V?$back_insert_iterator@V?$buffer@_W@detail@v8@fmt@@@std@@_WAEAV<lambda_1>@?1???$write_int@V?$back_insert_iterator@V?$buffer@_W@detail@v8@fmt@@@std@@_WV<lambda_2>@?8???$write_int@_WV?$back_insert_iterator@V?$buffer@_W@detail@v8@fmt@@@std@@_K@detail@v8@fmt@@YA?AV12@V12@U?$write_int_arg@_K@456@AEBU?$basic_format_specs@_W@56@Vlocale_ref@456@@Z@@detail@v8@fmt@@YA?AV12@V12@HIAEBU?$basic_format_specs@_W@56@V<lambda_2>@?8???$write_int@_WV?$back_insert_iterator@V?$buffer@_W@detail@v8@fmt@@@std@@_K@456@YA?AV12@0U?$write_int_arg@_K@456@1Vlocale_ref@456@@Z@@Z@@detail@v8@fmt@@YA?AV?$back_insert_iterator@V?$buffer@_W@detail@v8@fmt@@@std@@V34@AEBU?$basic_format_specs@_W@12@_K2AEAV<lambda_1>@?1???$write_int@V?$back_insert_iterator@V?$buffer@_W@detail@v8@fmt@@@std@@_WV<lambda_2>@?8???$write_int@_WV?$back_insert_iterator@V?$buffer@_W@detail@v8@fmt@@@std@@_K@detail@v8@fmt@@YA?AV12@V12@U?$write_int_arg@_K@456@AEBU?$basic_format_specs@_W@56@Vlocale_ref@456@@Z@@012@YA?AV34@0HI1V<lambda_2>@?8???$write_int@_WV?$back_insert_iterator@V?$buffer@_W@detail@v8@fmt@@@std@@_K@012@YA?AV34@0U?$write_int_arg@_K@012@1Vlocale_ref@012@@Z@@Z@@Z 0000000180015098 f i handles.obj
 0001:000142c0       ??$write_padded@$01V?$back_insert_iterator@V?$buffer@_W@detail@v8@fmt@@@std@@_WAEAV<lambda_1>@?1???$write_int@V?$back_insert_iterator@V?$buffer@_W@detail@v8@fmt@@@std@@_WV<lambda_3>@?M@???$write_int@_WV?$back_insert_iterator@V?$buffer@_W@detail@v8@fmt@@@std@@_K@detail@v8@fmt@@YA?AV12@V12@U?$write_int_arg@_K@456@AEBU?$basic_format_specs@_W@56@Vlocale_ref@456@@Z@@detail@v8@fmt@@YA?AV12@V12@HIAEBU?$basic_format_specs@_W@56@V<lambda_3>@?M@???$write_int@_WV?$back_insert_iterator@V?$buffer@_W@detail@v8@fmt@@@std@@_K@456@YA?AV12@0U?$write_int_arg@_K@456@1Vlocale_ref@456@@Z@@Z@@detail@v8@fmt@@YA?AV?$back_insert_iterator@V?$buffer@_W@detail@v8@fmt@@@std@@V34@AEBU?$basic_format_specs@_W@12@_K2AEAV<lambda_1>@?1???$write_int@V?$back_insert_iterator@V?$buffer@_W@detail@v8@fmt@@@std@@_WV<lambda_3>@?M@???$write_int@_WV?$back_insert_iterator@V?$buffer@_W@detail@v8@fmt@@@std@@_K@detail@v8@fmt@@YA?AV12@V12@U?$write_int_arg@_K@456@AEBU?$basic_format_specs@_W@56@Vlocale_ref@456@@Z@@012@YA?AV34@0HI1V<lambda_3>@?M@???$write_int@_WV?$back_insert_iterator@V?$buffer@_W@detail@v8@fmt@@@std@@_K@012@YA?AV34@0U?$write_int_arg@_K@012@1Vlocale_ref@012@@Z@@Z@@Z 00000001800152c0 f i handles.obj
 0001:000145a8       ??$write_padded@$01V?$back_insert_iterator@V?$buffer@_W@detail@v8@fmt@@@std@@_WAEAV<lambda_1>@?1???$write_int@V?$back_insert_iterator@V?$buffer@_W@detail@v8@fmt@@@std@@_WV<lambda_4>@?P@???$write_int@_WV?$back_insert_iterator@V?$buffer@_W@detail@v8@fmt@@@std@@_K@detail@v8@fmt@@YA?AV12@V12@U?$write_int_arg@_K@456@AEBU?$basic_format_specs@_W@56@Vlocale_ref@456@@Z@@detail@v8@fmt@@YA?AV12@V12@HIAEBU?$basic_format_specs@_W@56@V<lambda_4>@?P@???$write_int@_WV?$back_insert_iterator@V?$buffer@_W@detail@v8@fmt@@@std@@_K@456@YA?AV12@0U?$write_int_arg@_K@456@1Vlocale_ref@456@@Z@@Z@@detail@v8@fmt@@YA?AV?$back_insert_iterator@V?$buffer@_W@detail@v8@fmt@@@std@@V34@AEBU?$basic_format_specs@_W@12@_K2AEAV<lambda_1>@?1???$write_int@V?$back_insert_iterator@V?$buffer@_W@detail@v8@fmt@@@std@@_WV<lambda_4>@?P@???$write_int@_WV?$back_insert_iterator@V?$buffer@_W@detail@v8@fmt@@@std@@_K@detail@v8@fmt@@YA?AV12@V12@U?$write_int_arg@_K@456@AEBU?$basic_format_specs@_W@56@Vlocale_ref@456@@Z@@012@YA?AV34@0HI1V<lambda_4>@?P@???$write_int@_WV?$back_insert_iterator@V?$buffer@_W@detail@v8@fmt@@@std@@_K@012@YA?AV34@0U?$write_int_arg@_K@012@1Vlocale_ref@012@@Z@@Z@@Z 00000001800155a8 f i handles.obj
 0001:00014890       ??0PluginSettings@@QEAA@AEBU_GUID@@P6A_JPEAXW4FAR_SETTINGS_CONTROL_COMMANDS@@_J1@Z@Z 0000000180015890 f i Pcfg.obj
 0001:00014908       ??1PluginSettings@@QEAA@XZ 0000000180015908 f i Pcfg.obj
 0001:00014938       ?SaveValue@PluginCheckBoxBinding@@UEAAXPEBUFarDialogItem@@H@Z 0000000180015938 f i Pcfg.obj
 0001:000149d8       ??_GPluginCheckBoxBinding@@UEAAPEAXI@Z 00000001800159d8 f i Pcfg.obj
 0001:000149d8       ??_EPluginEditFieldBinding@@UEAAPEAXI@Z 00000001800159d8 f i * CIL library *:* CIL module *
 0001:000149d8       ??_GPluginEditFieldBinding@@UEAAPEAXI@Z 00000001800159d8 f i Pclass.obj
 0001:000149d8       ??_EPluginCheckBoxBinding@@UEAAPEAXI@Z 00000001800159d8 f i * CIL library *:* CIL module *
 0001:00014a00       ??0PluginDialogBuilder@@QEAA@AEBUPluginStartupInfo@@AEBU_GUID@@1HPEB_WP6A_JPEAX_J43@Z3_K@Z 0000000180015a00 f i Pcfg.obj
 0001:00014aa0       ??1PluginDialogBuilder@@QEAA@XZ 0000000180015aa0 f i Pcfg.obj
 0001:00014b20       ?AddText@PluginDialogBuilder@@QEAAPEAUFarDialogItem@@H@Z 0000000180015b20 f i Pcfg.obj
 0001:00014b88       ?AddCheckbox@PluginDialogBuilder@@QEAAPEAUFarDialogItem@@HPEAHH_N@Z 0000000180015b88 f i Pcfg.obj
 0001:00014ce0       ?AddOKCancel@PluginDialogBuilder@@QEAAXHHH_N@Z 0000000180015ce0 f i Pcfg.obj
 0001:00014ea8       ?ShowDialogEx@PluginDialogBuilder@@QEAA_JXZ 0000000180015ea8 f i Pcfg.obj
 0001:00015030       ?AddDialogItem@PluginDialogBuilder@@AEAAPEAUFarDialogItem@@W4FARDIALOGITEMTYPES@@PEB_W@Z 0000000180016030 f i Pcfg.obj
 0001:000151d0       ?ItemWidth@PluginDialogBuilder@@CA_JAEBUFarDialogItem@@@Z 00000001800161d0 f i Pcfg.obj
 0001:00015260       ?UpdateBorderSize@PluginDialogBuilder@@AEAAXXZ 0000000180016260 f i Pcfg.obj
 0001:00015420       ?Config@@YAHXZ             0000000180016420 f   Pcfg.obj
 0001:000156a8       ?Write@options@@QEBAXXZ    00000001800166a8 f   Pcfg.obj
 0001:00015928       ?Read@options@@QEAAXXZ     0000000180016928 f   Pcfg.obj
 0001:00015c30       ?SmartReread@PerfThread@@QEAAXXZ 0000000180016c30 f i Pclass.obj
 0001:00015ca8       ?SaveValue@PluginEditFieldBinding@@UEAAXPEBUFarDialogItem@@H@Z 0000000180016ca8 f i Pclass.obj
 0001:00015d38       ?AddEditField@PluginDialogBuilder@@QEAAPEAUFarDialogItem@@PEA_WHHPEB_W_N@Z 0000000180016d38 f i Pclass.obj
 0001:00015e30       ?OpenSubKey@PluginSettings@@QEAAH_KPEB_W@Z 0000000180016e30 f i Pclass.obj
 0001:00015e68       ?Get@PluginSettings@@QEAAPEB_W_KPEB_W1@Z 0000000180016e68 f i Pclass.obj
 0001:00015ec8       ?Get@PluginSettings@@QEAA_N_KPEB_W_N@Z 0000000180016ec8 f i Pclass.obj
 0001:000164a8       ??0Plist@@QEAA@XZ          00000001800174a8 f   Pclass.obj
 0001:00016920       ?InitializePanelModes@Plist@@SAXXZ 0000000180017920 f   Pclass.obj
 0001:000175f0       ?SavePanelModes@Plist@@SAXXZ 00000001800185f0 f   Pclass.obj
 0001:00017bb0       ??1StrTok@@QEAA@XZ         0000000180018bb0 f i Pclass.obj
 0001:00017bc0       ?PanelModes@Plist@@QEAAPEAUPanelMode@@AEA_K@Z 0000000180018bc0 f   Pclass.obj
 0001:00017dd0       ?GetOpenPanelInfo@Plist@@QEAAXPEAUOpenPanelInfo@@@Z 0000000180018dd0 f   Pclass.obj
 0001:000181a8       ?GetFindData@Plist@@QEAAHAEAPEAUPluginPanelItem@@AEA_K_K@Z 00000001800191a8 f   Pclass.obj
 0001:00018df0       ??1?$unordered_map@KPEAUHWND__@@U?$hash@K@std@@U?$equal_to@K@3@V?$allocator@U?$pair@$$CBKPEAUHWND__@@@std@@@3@@std@@QEAA@XZ 0000000180019df0 f i Pclass.obj
 0001:00018fd8       ??1?$pair@_JV?$basic_string@_WU?$char_traits@_W@std@@V?$allocator@_W@2@@std@@@std@@QEAA@XZ 0000000180019fd8 f i Pclass.obj
 0001:00018fd8       ??1?$pair@KV?$basic_string@_WU?$char_traits@_W@std@@V?$allocator@_W@2@@std@@@std@@QEAA@XZ 0000000180019fd8 f i Pclass.obj
 0001:00019608       ?GetFiles@Plist@@QEAAHPEAUPluginPanelItem@@_KHPEAPEB_W1AEAUoptions@@@Z 000000018001a608 f   Pclass.obj
 0001:0001b258       ??1ProcessData@@QEAA@XZ    000000018001c258 f i Pclass.obj
 0001:0001b2c0       ?DeleteFiles@Plist@@QEAAHPEAUPluginPanelItem@@_K1@Z 000000018001c2c0 f   Pclass.obj
 0001:0001b8a0       ?Reread@Plist@@AEAAXXZ     000000018001c8a0 f   Pclass.obj
 0001:0001b978       ?Connect@Plist@@QEAA_NPEB_W00@Z 000000018001c978 f   Pclass.obj
 0001:0001bcd0       ?ProcessKey@Plist@@QEAAHPEBU_INPUT_RECORD@@@Z 000000018001ccd0 f   Pclass.obj
 0001:0001d658       ?DurationToText@@YA?AV?$basic_string@_WU?$char_traits@_W@std@@V?$allocator@_W@2@@std@@_K@Z 000000018001e658 f   Pclass.obj
 0001:0001d7d0       ?GetVersionInfo@Plist@@SA_NPEB_WAEAV?$unique_ptr@$$BY0A@DU?$default_delete@$$BY0A@D@std@@@std@@AEAPEB_W2@Z 000000018001e7d0 f   Pclass.obj
 0001:0001db98       ?PrintVersionInfo@Plist@@CAXPEAXPEB_W@Z 000000018001eb98 f   Pclass.obj
 0001:0001df78       ?ConnectWMI@Plist@@AEAA_NXZ 000000018001ef78 f   Pclass.obj
 0001:0001e090       ?PrintOwnerInfo@Plist@@AEAAXPEAXK@Z 000000018001f090 f   Pclass.obj
 0001:0001e648       ?Compare@Plist@@QEBAHPEBUPluginPanelItem@@0I@Z 000000018001f648 f   Pclass.obj
 0001:0001e7f8       ?WmiError@Plist@@AEBAXXZ   000000018001f7f8 f   Pclass.obj
 0001:0001e840       ??1?$vector@PEAUHINSTANCE__@@V?$allocator@PEAUHINSTANCE__@@@std@@@std@@QEAA@XZ 000000018001f840 f i Plist.obj
 0001:0001e840       ??1?$vector@_KV?$allocator@_K@std@@@std@@QEAA@XZ 000000018001f840 f i Pclass.obj
 0001:0001e878       ??1?$vector@UFarMenuItem@@V?$allocator@UFarMenuItem@@@std@@@std@@QEAA@XZ 000000018001f878 f i Pclass.obj
 0001:0001e8b8       ?_Tidy@?$vector@V?$basic_string@_WU?$char_traits@_W@std@@V?$allocator@_W@2@@std@@V?$allocator@V?$basic_string@_WU?$char_traits@_W@std@@V?$allocator@_W@2@@std@@@2@@std@@AEAAXXZ 000000018001f8b8 f i Pclass.obj
 0001:0001e8b8       ??1?$vector@V?$basic_string@_WU?$char_traits@_W@std@@V?$allocator@_W@2@@std@@V?$allocator@V?$basic_string@_WU?$char_traits@_W@std@@V?$allocator@_W@2@@std@@@2@@std@@QEAA@XZ 000000018001f8b8 f i Pclass.obj
 0001:0001e948       ??1?$_Hash_vec@V?$allocator@V?$_List_unchecked_iterator@V?$_List_val@U?$_List_simple_types@U?$pair@$$CBKPEAUHWND__@@@std@@@std@@@std@@@std@@@std@@@std@@QEAA@XZ 000000018001f948 f i Pclass.obj
 0001:0001e948       ??1?$_Hash_vec@V?$allocator@V?$_List_unchecked_iterator@V?$_List_val@U?$_List_simple_types@U?$pair@$$CBKUProcessPerfData@@@std@@@std@@@std@@@std@@@std@@@std@@QEAA@XZ 000000018001f948 f i perfthread.obj
 0001:0001e978       ??1?$list@U?$pair@$$CBKPEAUHWND__@@@std@@V?$allocator@U?$pair@$$CBKPEAUHWND__@@@std@@@2@@std@@QEAA@XZ 000000018001f978 f i Pclass.obj
 0001:0001e9c8       ??1?$scoped_lock@Vrefresh_lock@Plist@@@std@@QEAA@XZ 000000018001f9c8 f i Pclass.obj
 0001:0001e9e0       ??0?$initializer_list@Umode@@@std@@QEAA@PEBUmode@@0@Z 000000018001f9e0 f i Pclass.obj
 0001:0001e9e8       ??4?$vector@Umode@@V?$allocator@Umode@@@std@@@std@@QEAAAEAV01@V?$initializer_list@Umode@@@1@@Z 000000018001f9e8 f i Pclass.obj
 0001:0001ea08       ??1?$unique_ptr@VWMIConnection@@U?$default_delete@VWMIConnection@@@std@@@std@@QEAA@XZ 000000018001fa08 f i Pclass.obj
 0001:0001ea18       ??1?$unique_ptr@VPerfThread@@U?$default_delete@VPerfThread@@@std@@@std@@QEAA@XZ 000000018001fa18 f i Pclass.obj
 0001:0001ea48       ??4?$unique_ptr@VPerfThread@@U?$default_delete@VPerfThread@@@std@@@std@@QEAAAEAV01@$$T@Z 000000018001fa48 f i Pclass.obj
 0001:0001ea88       ?push_back@?$basic_string@_WU?$char_traits@_W@std@@V?$allocator@_W@2@@std@@QEAAX_W@Z 000000018001fa88 f i Pclass.obj
 0001:0001ebd8       ??4?$basic_string@_WU?$char_traits@_W@std@@V?$allocator@_W@2@@std@@QEAAAEAV01@QEB_W@Z 000000018001fbd8 f i Pclass.obj
 0001:0001ebf8       ?_Xlength@?$vector@UProcessPerfData@@V?$allocator@UProcessPerfData@@@std@@@std@@CAXXZ 000000018001fbf8 f i perfthread.obj
 0001:0001ebf8       ?_Xlength@?$vector@PEAUHINSTANCE__@@V?$allocator@PEAUHINSTANCE__@@@std@@@std@@CAXXZ 000000018001fbf8 f i Plist.obj
 0001:0001ebf8       ?_Xlength@?$vector@V?$basic_string@_WU?$char_traits@_W@std@@V?$allocator@_W@2@@std@@V?$allocator@V?$basic_string@_WU?$char_traits@_W@std@@V?$allocator@_W@2@@std@@@2@@std@@CAXXZ 000000018001fbf8 f i Pclass.obj
 0001:0001ebf8       ?_Xlength@?$vector@PEB_WV?$allocator@PEB_W@std@@@std@@CAXXZ 000000018001fbf8 f i Pclass.obj
 0001:0001ebf8       ?_Xlength@?$vector@UFarMenuItem@@V?$allocator@UFarMenuItem@@@std@@@std@@CAXXZ 000000018001fbf8 f i Pclass.obj
 0001:0001ebf8       ?_Xlength@?$vector@EV?$allocator@E@std@@@std@@CAXXZ 000000018001fbf8 f i perfthread.obj
 0001:0001ebf8       ?_Xlength@?$vector@_KV?$allocator@_K@std@@@std@@CAXXZ 000000018001fbf8 f i Pclass.obj
 0001:0001ebf8       ?_Xlength@?$vector@Umode@@V?$allocator@Umode@@@std@@@std@@CAXXZ 000000018001fbf8 f i Pclass.obj
 0001:0001ec08       ?_Reallocate_exactly@?$vector@_KV?$allocator@_K@std@@@std@@AEAAX_K@Z 000000018001fc08 f i Pclass.obj
 0001:0001eca0       ?_Reallocate_exactly@?$vector@UFarMenuItem@@V?$allocator@UFarMenuItem@@@std@@@std@@AEAAX_K@Z 000000018001fca0 f i Pclass.obj
 0001:0001ed48       ?_Reallocate_exactly@?$vector@V?$basic_string@_WU?$char_traits@_W@std@@V?$allocator@_W@2@@std@@V?$allocator@V?$basic_string@_WU?$char_traits@_W@std@@V?$allocator@_W@2@@std@@@2@@std@@AEAAX_K@Z 000000018001fd48 f i Pclass.obj
 0001:0001ee10       ??R?$default_delete@VWMIConnection@@@std@@QEBAXPEAVWMIConnection@@@Z 000000018001fe10 f i Pclass.obj
 0001:0001eeb0       ?insert@?$basic_string@_WU?$char_traits@_W@std@@V?$allocator@_W@2@@std@@QEAAAEAV12@_KQEB_W0@Z 000000018001feb0 f i Pclass.obj
 0001:0001f080       ?_Change_array@?$vector@V?$basic_string@_WU?$char_traits@_W@std@@V?$allocator@_W@2@@std@@V?$allocator@V?$basic_string@_WU?$char_traits@_W@std@@V?$allocator@_W@2@@std@@@2@@std@@AEAAXQEAV?$basic_string@_WU?$char_traits@_W@std@@V?$allocator@_W@2@@2@_K1@Z 0000000180020080 f i Pclass.obj
 0001:0001f140       ?_Assign_grow@?$_Hash_vec@V?$allocator@V?$_List_unchecked_iterator@V?$_List_val@U?$_List_simple_types@U?$pair@$$CBKPEAUHWND__@@@std@@@std@@@std@@@std@@@std@@@std@@QEAAX_KV?$_List_unchecked_iterator@V?$_List_val@U?$_List_simple_types@U?$pair@$$CBKPEAUHWND__@@@std@@@std@@@std@@@2@@Z 0000000180020140 f i Pclass.obj
 0001:0001f140       ?_Assign_grow@?$_Hash_vec@V?$allocator@V?$_List_unchecked_iterator@V?$_List_val@U?$_List_simple_types@U?$pair@$$CBKUProcessPerfData@@@std@@@std@@@std@@@std@@@std@@@std@@QEAAX_KV?$_List_unchecked_iterator@V?$_List_val@U?$_List_simple_types@U?$pair@$$CBKUProcessPerfData@@@std@@@std@@@std@@@2@@Z 0000000180020140 f i perfthread.obj
 0001:0001f208       ?_Xran@?$_String_val@U?$_Simple_types@_W@std@@@std@@SAXXZ 0000000180020208 f i Pclass.obj
 0001:0001f218       ??$?4U?$default_delete@VPerfThread@@@std@@$0A@@?$unique_ptr@VPerfThread@@U?$default_delete@VPerfThread@@@std@@@std@@QEAAAEAV01@$$QEAV01@@Z 0000000180020218 f i Pclass.obj
 0001:0001f268       ??$_Emplace_reallocate@V?$basic_string@_WU?$char_traits@_W@std@@V?$allocator@_W@2@@std@@@?$vector@V?$basic_string@_WU?$char_traits@_W@std@@V?$allocator@_W@2@@std@@V?$allocator@V?$basic_string@_WU?$char_traits@_W@std@@V?$allocator@_W@2@@std@@@2@@std@@QEAAPEAV?$basic_string@_WU?$char_traits@_W@std@@V?$allocator@_W@2@@1@QEAV21@$$QEAV21@@Z 0000000180020268 f i Pclass.obj
 0001:0001f418       ??$format@AEAV?$basic_string@_WU?$char_traits@_W@std@@V?$allocator@_W@2@@std@@AEAK@v8@fmt@@YA?AV?$basic_string@_WU?$char_traits@_W@std@@V?$allocator@_W@2@@std@@V?$basic_format_string@_WAEAV?$basic_string@_WU?$char_traits@_W@std@@V?$allocator@_W@2@@std@@AEAK@01@AEAV23@AEAK@Z 0000000180020418 f i Pclass.obj
 0001:0001f4a0       ??$_Emplace_reallocate@AEB_K@?$vector@_KV?$allocator@_K@std@@@std@@QEAAPEA_KQEA_KAEB_K@Z 00000001800204a0 f i Pclass.obj
 0001:0001f4a0       ??$_Emplace_reallocate@_K@?$vector@_KV?$allocator@_K@std@@@std@@QEAAPEA_KQEA_K$$QEA_K@Z 00000001800204a0 f i Pclass.obj
 0001:0001f5c8       ??$_Emplace_reallocate@UFarMenuItem@@@?$vector@UFarMenuItem@@V?$allocator@UFarMenuItem@@@std@@@std@@QEAAPEAUFarMenuItem@@QEAU2@$$QEAU2@@Z 00000001800205c8 f i Pclass.obj
 0001:0001f720       ??$_Try_emplace@AEBK$$V@?$_Hash@V?$_Umap_traits@KPEAUHWND__@@V?$_Uhash_compare@KU?$hash@K@std@@U?$equal_to@K@2@@std@@V?$allocator@U?$pair@$$CBKPEAUHWND__@@@std@@@3@$0A@@std@@@std@@IEAA?AU?$pair@PEAU?$_List_node@U?$pair@$$CBKPEAUHWND__@@@std@@PEAX@std@@_N@1@AEBK@Z 0000000180020720 f i Pclass.obj
 0001:0001f9c8       ??$_Assign_range@PEBUmode@@@?$vector@Umode@@V?$allocator@Umode@@@std@@@std@@AEAAXPEBUmode@@0Uforward_iterator_tag@1@@Z 00000001800209c8 f i Pclass.obj
 0001:0001fb50       ??$_Reallocate_grow_by@V<lambda_1>@?1??insert@?$basic_string@_WU?$char_traits@_W@std@@V?$allocator@_W@2@@std@@QEAAAEAV34@_K0_W@Z@_K_K_W@?$basic_string@_WU?$char_traits@_W@std@@V?$allocator@_W@2@@std@@AEAAAEAV01@_KV<lambda_1>@?1??insert@01@QEAAAEAV01@00_W@Z@_K3_W@Z 0000000180020b50 f i Pclass.obj
 0001:0001fcd8       ??$_Reallocate_grow_by@V<lambda_1>@?1??append@?$basic_string@_WU?$char_traits@_W@std@@V?$allocator@_W@2@@std@@QEAAAEAV34@_K_W@Z@_K_W@?$basic_string@_WU?$char_traits@_W@std@@V?$allocator@_W@2@@std@@AEAAAEAV01@_KV<lambda_1>@?1??append@01@QEAAAEAV01@0_W@Z@_K_W@Z 0000000180020cd8 f i Pclass.obj
 0001:0001fe38       ??1?$_Alloc_construct_ptr@V?$allocator@U?$_List_node@U?$pair@$$CBKPEAUHWND__@@@std@@PEAX@std@@@std@@@std@@QEAA@XZ 0000000180020e38 f i Pclass.obj
 0001:0001fe38       ??1?$_List_node_emplace_op2@V?$allocator@U?$_List_node@U?$pair@$$CBKPEAUHWND__@@@std@@PEAX@std@@@std@@@std@@QEAA@XZ 0000000180020e38 f i Pclass.obj
 0001:0001fe50       ?_Umove@?$vector@V?$basic_string@_WU?$char_traits@_W@std@@V?$allocator@_W@2@@std@@V?$allocator@V?$basic_string@_WU?$char_traits@_W@std@@V?$allocator@_W@2@@std@@@2@@std@@AEAAPEAV?$basic_string@_WU?$char_traits@_W@std@@V?$allocator@_W@2@@2@PEAV32@00@Z 0000000180020e50 f i Pclass.obj
 0001:0001feb0       ?_Forced_rehash@?$_Hash@V?$_Umap_traits@KUProcessPerfData@@V?$_Uhash_compare@KU?$hash@K@std@@U?$equal_to@K@2@@std@@V?$allocator@U?$pair@$$CBKUProcessPerfData@@@std@@@3@$00@std@@@std@@IEAAX_K@Z 0000000180020eb0 f i perfthread.obj
 0001:0001feb0       ?_Forced_rehash@?$_Hash@V?$_Umap_traits@KPEAUHWND__@@V?$_Uhash_compare@KU?$hash@K@std@@U?$equal_to@K@2@@std@@V?$allocator@U?$pair@$$CBKPEAUHWND__@@@std@@@3@$0A@@std@@@std@@IEAAX_K@Z 0000000180020eb0 f i Pclass.obj
 0001:00020080       ??$_Resize_reallocate@U_Value_init_tag@std@@@?$vector@PEAUHINSTANCE__@@V?$allocator@PEAUHINSTANCE__@@@std@@@std@@AEAAX_KAEBU_Value_init_tag@1@@Z 0000000180021080 f i Plist.obj
 0001:00020080       ??$_Resize_reallocate@U_Value_init_tag@std@@@?$vector@PEB_WV?$allocator@PEB_W@std@@@std@@AEAAX_KAEBU_Value_init_tag@1@@Z 0000000180021080 f i Pclass.obj
 0001:00020170       ??$_Copy_unchecked@PEBUmode@@PEAU1@@std@@YAPEAUmode@@PEBU1@0PEAU1@@Z 0000000180021170 f i Pclass.obj
 0001:000202a0       ??$_Uninitialized_copy@PEBUmode@@V?$allocator@Umode@@@std@@@std@@YAPEAUmode@@QEBU1@0PEAU1@AEAV?$allocator@Umode@@@0@@Z 00000001800212a0 f i Pclass.obj
 0001:000204f0       ??1?$_Uninitialized_backout_al@V?$allocator@Umode@@@std@@@std@@QEAA@XZ 00000001800214f0 f i Pclass.obj
 0001:00020528       ??0PerfThread@@QEAA@PEAVPlist@@PEB_W11@Z 0000000180021528 f   perfthread.obj
 0001:00020d08       ??1?$unordered_multimap@KUProcessPerfData@@U?$hash@K@std@@U?$equal_to@K@3@V?$allocator@U?$pair@$$CBKUProcessPerfData@@@std@@@3@@std@@QEAA@XZ 0000000180021d08 f i perfthread.obj
 0001:00020d50       ??1PerfThread@@QEAA@XZ     0000000180021d50 f   perfthread.obj
 0001:00020f88       ?GetProcessData@PerfThread@@QEAAPEAUProcessPerfData@@KK@Z 0000000180021f88 f   perfthread.obj
 0001:00021088       ?Refresh@PerfThread@@AEAAXXZ 0000000180022088 f   perfthread.obj
 0001:00022428       ??1ProcessPerfData@@QEAA@XZ 0000000180023428 f i perfthread.obj
 0001:000224d8       ??4ProcessPerfData@@QEAAAEAU0@AEBU0@@Z 00000001800234d8 f i perfthread.obj
 0001:00022750       ?RefreshWMIData@PerfThread@@AEAAXXZ 0000000180023750 f   perfthread.obj
 0001:00022d40       ?ThreadProc@PerfThread@@CAKPEAX@Z 0000000180023d40 f   perfthread.obj
 0001:00022de0       ?WmiThreadProc@PerfThread@@CAKPEAX@Z 0000000180023de0 f   perfthread.obj
 0001:00022f28       ??1?$vector@UProcessPerfData@@V?$allocator@UProcessPerfData@@@std@@@std@@QEAA@XZ 0000000180023f28 f i perfthread.obj
 0001:00022f78       ??1?$vector@EV?$allocator@E@std@@@std@@QEAA@XZ 0000000180023f78 f i perfthread.obj
 0001:00022fb0       ??1?$vector@_WV?$allocator@_W@std@@@std@@QEAA@XZ 0000000180023fb0 f i perfthread.obj
 0001:00022fe8       ??0?$unordered_multimap@KUProcessPerfData@@U?$hash@K@std@@U?$equal_to@K@3@V?$allocator@U?$pair@$$CBKUProcessPerfData@@@std@@@3@@std@@QEAA@XZ 0000000180023fe8 f i perfthread.obj
 0001:000230c0       ??1?$list@U?$pair@$$CBKUProcessPerfData@@@std@@V?$allocator@U?$pair@$$CBKUProcessPerfData@@@std@@@2@@std@@QEAA@XZ 00000001800240c0 f i perfthread.obj
 0001:000230f0       ?_Reallocate_exactly@?$vector@UProcessPerfData@@V?$allocator@UProcessPerfData@@@std@@@std@@AEAAX_K@Z 00000001800240f0 f i perfthread.obj
 0001:000231c0       ?_Unchecked_erase@?$_Hash@V?$_Umap_traits@KUProcessPerfData@@V?$_Uhash_compare@KU?$hash@K@std@@U?$equal_to@K@2@@std@@V?$allocator@U?$pair@$$CBKUProcessPerfData@@@std@@@3@$00@std@@@std@@AEAAPEAU?$_List_node@U?$pair@$$CBKUProcessPerfData@@@std@@PEAX@2@PEAU32@QEAU32@@Z 00000001800241c0 f i perfthread.obj
 0001:00023440       ??$?0PEAUProcessPerfData@@_K$0A@@?$pair@PEAUProcessPerfData@@_K@std@@QEAA@XZ 0000000180024440 f i perfthread.obj
 0001:00023448       ??$emplace@AEBKUProcessPerfData@@@?$_Hash@V?$_Umap_traits@KUProcessPerfData@@V?$_Uhash_compare@KU?$hash@K@std@@U?$equal_to@K@2@@std@@V?$allocator@U?$pair@$$CBKUProcessPerfData@@@std@@@3@$00@std@@@std@@QEAA?AV?$_List_iterator@V?$_List_val@U?$_List_simple_types@U?$pair@$$CBKUProcessPerfData@@@std@@@std@@@std@@@1@AEBK$$QEAUProcessPerfData@@@Z 0000000180024448 f i perfthread.obj
 0001:00023a58       ??0ProcessPerfData@@QEAA@AEBU0@@Z 0000000180024a58 f i perfthread.obj
 0001:00023b60       ??$_Free_non_head@V?$allocator@U?$_List_node@U?$pair@$$CBKUProcessPerfData@@@std@@PEAX@std@@@std@@@?$_List_node@U?$pair@$$CBKUProcessPerfData@@@std@@PEAX@std@@SAXAEAV?$allocator@U?$_List_node@U?$pair@$$CBKUProcessPerfData@@@std@@PEAX@std@@@1@PEAU01@@Z 0000000180024b60 f i perfthread.obj
 0001:00023c40       ??$_Destroy_range@V?$allocator@UProcessPerfData@@@std@@@std@@YAXPEAUProcessPerfData@@QEAU1@AEAV?$allocator@UProcessPerfData@@@0@@Z 0000000180024c40 f i perfthread.obj
 0001:00023d10       ??1?$_List_node_emplace_op2@V?$allocator@U?$_List_node@U?$pair@$$CBKUProcessPerfData@@@std@@PEAX@std@@@std@@@std@@QEAA@XZ 0000000180024d10 f i perfthread.obj
 0001:00023d48       ??1?$_Alloc_construct_ptr@V?$allocator@U?$_List_node@U?$pair@$$CBKUProcessPerfData@@@std@@PEAX@std@@@std@@@std@@QEAA@XZ 0000000180024d48 f i perfthread.obj
 0001:00023d60       ??$_Resize_reallocate@U_Value_init_tag@std@@@?$vector@EV?$allocator@E@std@@@std@@AEAAX_KAEBU_Value_init_tag@1@@Z 0000000180024d60 f i perfthread.obj
 0001:00023e30       ??$_Emplace_reallocate@UProcessPerfData@@@?$vector@UProcessPerfData@@V?$allocator@UProcessPerfData@@@std@@@std@@QEAAPEAUProcessPerfData@@QEAU2@$$QEAU2@@Z 0000000180024e30 f i perfthread.obj
 0001:00023fd8       ??0ProcessPerfData@@QEAA@$$QEAU0@@Z 0000000180024fd8 f i perfthread.obj
 0001:00024118       ?GetPData@@YA_NAEAUProcessData@@AEBUProcessPerfData@@@Z 0000000180025118 f   Plist.obj
 0001:000242a0       ?GetList@@YA_NAEAPEAUPluginPanelItem@@AEA_KAEAVPerfThread@@@Z 00000001800252a0 f   Plist.obj
 0001:000246d0       ?Enable@DebugToken@@QEAA_NXZ 00000001800256d0 f   Plist.obj
 0001:000247b0       ?KillProcess@@YA_NKPEAUHWND__@@@Z 00000001800257b0 f   Plist.obj
 0001:00024998       ?PrintNTCurDirAndEnv@@YAXPEAX0H@Z 0000000180025998 f   Plist.obj
 0001:00025050       ?PrintModules@@YAXPEAXKAEAUoptions@@@Z 0000000180026050 f   Plist.obj
 0001:00025490       ??1?$function@$$A6A_NPEA_W_K@Z@std@@QEAA@XZ 0000000180026490 f i Plist.obj
 0001:00025490       ??1?$function@$$A6AXAEBUtagVARIANT@@@Z@std@@QEAA@XZ 0000000180026490 f i wmi.obj
 0001:000254c8       ?PrintModules@?$ipc_functions@$0A@@@SAXPEAX0AEAUoptions@@@Z 00000001800264c8 f i Plist.obj
 0001:00025740       ?GetOpenProcessData@?$ipc_functions@$0A@@@SAXPEAXPEAV?$basic_string@_WU?$char_traits@_W@std@@V?$allocator@_W@2@@std@@1111@Z 0000000180026740 f i Plist.obj
 0001:00025c30       ?read_string@?$ipc_functions@$0A@@@SA?AV?$basic_string@_WU?$char_traits@_W@std@@V?$allocator@_W@2@@std@@PEAXAEBUUNICODE_STRING_SAME@detail@@@Z 0000000180026c30 f i Plist.obj
 0001:00025d80       ?resize@?$basic_string@_WU?$char_traits@_W@std@@V?$allocator@_W@2@@std@@QEAAX_K_W@Z 0000000180026d80 f i Plist.obj
 0001:00025f38       ??$insert@V?$_List_unchecked_const_iterator@V?$_List_val@U?$_List_simple_types@U?$pair@$$CBKUProcessPerfData@@@std@@@std@@@std@@U_Iterator_base0@2@@std@@@?$_Hash@V?$_Umap_traits@KUProcessPerfData@@V?$_Uhash_compare@KU?$hash@K@std@@U?$equal_to@K@2@@std@@V?$allocator@U?$pair@$$CBKUProcessPerfData@@@std@@@3@$00@std@@@std@@QEAAXV?$_List_unchecked_const_iterator@V?$_List_val@U?$_List_simple_types@U?$pair@$$CBKUProcessPerfData@@@std@@@std@@@std@@U_Iterator_base0@2@@1@0@Z 0000000180026f38 f i Plist.obj
 0001:00026160       ?_Delete_this@?$_Func_impl_no_alloc@V<lambda_1>@?6??PrintModules@?$ipc_functions@$0A@@@SAXPEAX0AEAUoptions@@@Z@_NPEA_W_K@std@@EEAAX_N@Z 0000000180027160 f i Plist.obj
 0001:00026178       ?_Get@?$_Func_impl_no_alloc@V<lambda_1>@?6??PrintModules@?$ipc_functions@$0A@@@SAXPEAX0AEAUoptions@@@Z@_NPEA_W_K@std@@EEBAPEBXXZ 0000000180027178 f i Plist.obj
 0001:00026180       ?_Target_type@?$_Func_impl_no_alloc@V<lambda_1>@?6??PrintModules@?$ipc_functions@$0A@@@SAXPEAX0AEAUoptions@@@Z@_NPEA_W_K@std@@EEBAAEBVtype_info@@XZ 0000000180027180 f i Plist.obj
 0001:00026190       ?_Do_call@?$_Func_impl_no_alloc@V<lambda_1>@?6??PrintModules@?$ipc_functions@$0A@@@SAXPEAX0AEAUoptions@@@Z@_NPEA_W_K@std@@EEAA_N$$QEAPEA_W$$QEA_K@Z 0000000180027190 f i Plist.obj
 0001:000261d0       ?_Move@?$_Func_impl_no_alloc@V<lambda_1>@?6??PrintModules@?$ipc_functions@$0A@@@SAXPEAX0AEAUoptions@@@Z@_NPEA_W_K@std@@EEAAPEAV?$_Func_base@_NPEA_W_K@2@PEAX@Z 00000001800271d0 f i Plist.obj
 0001:000261d0       ?_Copy@?$_Func_impl_no_alloc@V<lambda_1>@?6??PrintModules@?$ipc_functions@$0A@@@SAXPEAX0AEAUoptions@@@Z@_NPEA_W_K@std@@EEBAPEAV?$_Func_base@_NPEA_W_K@2@PEAX@Z 00000001800271d0 f i Plist.obj
 0001:00026258       ?GetMsg@@YAPEB_WH@Z        0000000180027258 f   Pmix.obj
 0001:00026270       ?WinError@@YAHPEB_W@Z      0000000180027270 f   Pmix.obj
 0001:00026550       ?find_last_not_of@?$basic_string@_WU?$char_traits@_W@std@@V?$allocator@_W@2@@std@@QEBA_KQEB_W_K@Z 0000000180027550 f i Pmix.obj
 0001:000266b8       ??1bstr@@QEAA@XZ           00000001800276b8 f i wmi.obj
 0001:000266d8       ??1WMIConnection@@QEAA@XZ  00000001800276d8 f   wmi.obj
 0001:00026768       ?GetProcessOwner@WMIConnection@@QEAA?AV?$basic_string@_WU?$char_traits@_W@std@@V?$allocator@_W@2@@std@@KPEAV23@@Z 0000000180027768 f   wmi.obj
 0001:00026a68       ?GetProcessUserSid@WMIConnection@@QEAA?AV?$basic_string@_WU?$char_traits@_W@std@@V?$allocator@_W@2@@std@@K@Z 0000000180027a68 f   wmi.obj
 0001:00026cc0       ?GetProcessSessionId@WMIConnection@@QEAAKK@Z 0000000180027cc0 f   wmi.obj
 0001:00026d48       ?ExecMethod@WMIConnection@@AEAAHKPEB_W0K@Z 0000000180027d48 f   wmi.obj
 0001:00027150       ?GetProcessProperty@WMIConnection@@AEAA_NKPEB_WAEBV?$function@$$A6AXAEBUtagVARIANT@@@Z@std@@@Z 0000000180028150 f   wmi.obj
 0001:00027328       ?Connect@WMIConnection@@QEAA_NPEB_W00@Z 0000000180028328 f   wmi.obj
 0001:000275d0       ??1?$unique_ptr@UIWbemClassObject@@Ucom_closer@@@std@@QEAA@XZ 00000001800285d0 f i wmi.obj
 0001:000275d0       ??1?$unique_ptr@UIWbemLocator@@Ucom_closer@@@std@@QEAA@XZ 00000001800285d0 f i wmi.obj
 0001:00027600       ??1?$ptr_setter@V?$unique_ptr@UIWbemClassObject@@Ucom_closer@@@std@@@@QEAA@XZ 0000000180028600 f i wmi.obj
 0001:00027718       __isa_available_init       0000000180028718 f   LIBCMT:cpu_disp.obj
 0001:000279f8       GetGlobalInfoW             00000001800289f8 f   Proclist.obj
 0001:00027a90       SetStartupInfoW            0000000180028a90 f   Proclist.obj
 0001:00027be0       OpenW                      0000000180028be0 f   Proclist.obj
 0001:00027cf8       ClosePanelW                0000000180028cf8 f   Proclist.obj
 0001:00027da8       GetFindDataW               0000000180028da8 f   Proclist.obj
 0001:00027dd0       FreeFindDataW              0000000180028dd0 f   Proclist.obj
 0001:00027ef0       GetPluginInfoW             0000000180028ef0 f   Proclist.obj
 0001:00027fb8       GetOpenPanelInfoW          0000000180028fb8 f   Proclist.obj
 0001:00027fc8       GetFilesW                  0000000180028fc8 f   Proclist.obj
 0001:00028000       DeleteFilesW               0000000180029000 f   Proclist.obj
 0001:00028020       ProcessPanelEventW         0000000180029020 f   Proclist.obj
 0001:000281e8       ProcessPanelInputW         00000001800291e8 f   Proclist.obj
 0001:00028208       ConfigureW                 0000000180029208 f   Proclist.obj
 0001:00028220       CompareW                   0000000180029220 f   Proclist.obj
 0001:00028248       ProcessSynchroEventW       0000000180029248 f   Proclist.obj
 0001:00028270       _Mbrtowc                   0000000180029270 f   libcpmt:xmbtowc.obj
 0001:00028410       ??0_Init_locks@std@@QEAA@XZ 0000000180029410 f   libcpmt:xlock.obj
 0001:00028478       ??0_Lockit@std@@QEAA@H@Z   0000000180029478 f   libcpmt:xlock.obj
 0001:000284c8       ??1_Init_locks@std@@QEAA@XZ 00000001800294c8 f   libcpmt:xlock.obj
 0001:00028520       ??1_Lockit@std@@QEAA@XZ    0000000180029520 f   libcpmt:xlock.obj
 0001:00028550       ??0bad_alloc@std@@QEAA@XZ  0000000180029550 f i libcpmt:xthrow.obj
 0001:00028570       ??0bad_function_call@std@@QEAA@AEBV01@@Z 0000000180029570 f i libcpmt:xthrow.obj
 0001:000285c0       ??0bad_function_call@std@@QEAA@XZ 00000001800295c0 f i libcpmt:xthrow.obj
 0001:000285d8       ??0length_error@std@@QEAA@AEBV01@@Z 00000001800295d8 f i libcpmt:xthrow.obj
 0001:00028628       ??0length_error@std@@QEAA@PEBD@Z 0000000180029628 f i libcpmt:xthrow.obj
 0001:00028680       ??0logic_error@std@@QEAA@AEBV01@@Z 0000000180029680 f i libcpmt:xthrow.obj
 0001:000286d0       ??0out_of_range@std@@QEAA@AEBV01@@Z 00000001800296d0 f i libcpmt:xthrow.obj
 0001:00028720       ??0out_of_range@std@@QEAA@PEBD@Z 0000000180029720 f i libcpmt:xthrow.obj
 0001:00028778       ??_Gout_of_range@std@@UEAAPEAXI@Z 0000000180029778 f i libcpmt:xthrow.obj
 0001:00028778       ??_Ebad_function_call@std@@UEAAPEAXI@Z 0000000180029778 f i libcpmt:xthrow.obj
 0001:00028778       ??_Eout_of_range@std@@UEAAPEAXI@Z 0000000180029778 f i libcpmt:xthrow.obj
 0001:00028778       ??_Elength_error@std@@UEAAPEAXI@Z 0000000180029778 f i libcpmt:xthrow.obj
 0001:00028778       ??_Gbad_exception@std@@UEAAPEAXI@Z 0000000180029778 f i libvcruntime:frame.obj
 0001:00028778       ??_Elogic_error@std@@UEAAPEAXI@Z 0000000180029778 f i libcpmt:xthrow.obj
 0001:00028778       ??_Glogic_error@std@@UEAAPEAXI@Z 0000000180029778 f i libcpmt:xthrow.obj
 0001:00028778       ??_Ebad_exception@std@@UEAAPEAXI@Z 0000000180029778 f i libvcruntime:frame.obj
 0001:00028778       ??_Gbad_function_call@std@@UEAAPEAXI@Z 0000000180029778 f i libcpmt:xthrow.obj
 0001:00028778       ??_Glength_error@std@@UEAAPEAXI@Z 0000000180029778 f i libcpmt:xthrow.obj
 0001:000287c0       ?_Xbad_alloc@std@@YAXXZ    00000001800297c0 f   libcpmt:xthrow.obj
 0001:000287c0       ?__scrt_throw_std_bad_alloc@@YAXXZ 00000001800297c0 f   LIBCMT:throw_bad_alloc.obj
 0001:000287e0       ?_Xbad_function_call@std@@YAXXZ 00000001800297e0 f   libcpmt:xthrow.obj
 0001:00028800       ?_Xlength_error@std@@YAXPEBD@Z 0000000180029800 f   libcpmt:xthrow.obj
 0001:00028828       ?_Xout_of_range@std@@YAXPEBD@Z 0000000180029828 f   libcpmt:xthrow.obj
 0001:00028850       ?_Xruntime_error@std@@YAXPEBD@Z 0000000180029850 f   libcpmt:xthrow.obj
 0001:00028878       ?what@bad_function_call@std@@UEBAPEBDXZ 0000000180029878 f i libcpmt:xthrow.obj
 0001:00028888       ??1_Fac_tidy_reg_t@std@@QEAA@XZ 0000000180029888 f i libcpmt:locale0.obj
 0001:00028920       ??_G_Locimp@locale@std@@MEAAPEAXI@Z 0000000180029920 f i libcpmt:locale0.obj
 0001:00028920       ??_E_Locimp@locale@std@@MEAAPEAXI@Z 0000000180029920 f i libcpmt:locale0.obj
 0001:00028980       ?_Facet_Register@std@@YAXPEAV_Facet_base@1@@Z 0000000180029980 f   libcpmt:locale0.obj
 0001:000289c8       ?_Getgloballocale@locale@std@@CAPEAV_Locimp@12@XZ 00000001800299c8 f   libcpmt:locale0.obj
 0001:000289d8       ?_Init@locale@std@@CAPEAV_Locimp@12@_N@Z 00000001800299d8 f   libcpmt:locale0.obj
 0001:00028af8       ?_Locimp_dtor@_Locimp@locale@std@@CAXPEAV123@@Z 0000000180029af8 f   libcpmt:locale0.obj
 0001:00028bb0       ?_Locinfo_ctor@_Locinfo@std@@SAXPEAV12@PEBD@Z 0000000180029bb0 f   libcpmt:locale0.obj
 0001:00028cb8       ?_Locinfo_dtor@_Locinfo@std@@SAXPEAV12@@Z 0000000180029cb8 f   libcpmt:locale0.obj
 0001:00028cd0       ?_New_Locimp@_Locimp@locale@std@@CAPEAV123@_N@Z 0000000180029cd0 f   libcpmt:locale0.obj
 0001:00028d70       ?_Setgloballocale@locale@std@@CAXPEAX@Z 0000000180029d70 f   libcpmt:locale0.obj
 0001:00028db8       _Deletegloballocale        0000000180029db8 f   libcpmt:locale0.obj
 0001:00028e68       _Getcvt                    0000000180029e68 f   libcpmt:xwctomb.obj
 0001:00028f00       _Mtxdst                    0000000180029f00 f   libcpmt:xmtx.obj
 0001:00028f20       _Mtxinit                   0000000180029f20 f   libcpmt:xmtx.obj
 0001:00028f48       _Mtxlock                   0000000180029f48 f   libcpmt:xmtx.obj
 0001:00028f68       _Mtxunlock                 0000000180029f68 f   libcpmt:xmtx.obj
 0001:00028f88       ??1_Init_atexit@@QEAA@XZ   0000000180029f88 f i libcpmt:iosptrs.obj
 0001:00029018       ?_Atexit@@YAXP6AXXZ@Z      000000018002a018 f   libcpmt:iosptrs.obj
 0001:00029068       __scrt_acquire_startup_lock 000000018002a068 f   LIBCMT:utility.obj
 0001:000290d8       __scrt_dllmain_after_initialize_c 000000018002a0d8 f   LIBCMT:utility.obj
 0001:00029118       __scrt_dllmain_before_initialize_c 000000018002a118 f   LIBCMT:utility.obj
 0001:00029140       __scrt_dllmain_crt_thread_attach 000000018002a140 f   LIBCMT:utility.obj
 0001:00029180       __scrt_dllmain_crt_thread_detach 000000018002a180 f   LIBCMT:utility.obj
 0001:000291a0       __scrt_dllmain_exception_filter 000000018002a1a0 f   LIBCMT:utility.obj
 0001:00029220       __scrt_dllmain_uninitialize_c 000000018002a220 f   LIBCMT:utility.obj
 0001:00029258       __scrt_dllmain_uninitialize_critical 000000018002a258 f   LIBCMT:utility.obj
 0001:00029278       __scrt_initialize_crt      000000018002a278 f   LIBCMT:utility.obj
 0001:000292d8       __scrt_initialize_onexit_tables 000000018002a2d8 f   LIBCMT:utility.obj
 0001:00029378       __scrt_is_nonwritable_in_current_image 000000018002a378 f   LIBCMT:utility.obj
 0001:00029448       __scrt_release_startup_lock 000000018002a448 f   LIBCMT:utility.obj
 0001:00029480       __scrt_uninitialize_crt    000000018002a480 f   LIBCMT:utility.obj
 0001:000294c8       _onexit                    000000018002a4c8 f   LIBCMT:utility.obj
 0001:00029510       atexit                     000000018002a510 f   LIBCMT:utility.obj
 0001:00029530       ??3@YAXPEAX@Z              000000018002a530 f   LIBCMT:delete_scalar.obj
 0001:00029538       ??3@YAXPEAX_K@Z            000000018002a538 f   LIBCMT:delete_scalar_size.obj
 0001:00029538       ??_V@YAXPEAX@Z             000000018002a538 f   LIBCMT:delete_array.obj
 0001:00029540       ??2@YAPEAX_K@Z             000000018002a540 f   LIBCMT:new_scalar.obj
 0001:00029588       ??_Gtype_info@@UEAAPEAXI@Z 000000018002a588 f i LIBCMT:std_type_info_static.obj
 0001:00029588       ??_Etype_info@@UEAAPEAXI@Z 000000018002a588 f i LIBCMT:std_type_info_static.obj
 0001:000295c0       ??_U@YAPEAX_K@Z            000000018002a5c0 f   LIBCMT:new_array.obj
 0001:000295c8       ??_M@YAXPEAX_K1P6AX0@Z@Z   000000018002a5c8 f   LIBCMT:ehvecdtr.obj
 0001:00029650       ?__ArrayUnwind@@YAXPEAX_K1P6AX0@Z@Z 000000018002a650 f   LIBCMT:ehvecdtr.obj
 0001:00029a98       _DllMainCRTStartup         000000018002aa98 f   LIBCMT:dll_dllmain.obj
 0001:00029ae0       _guard_check_icall_nop     000000018002aae0 f i LIBCMT:guard_support.obj
 0001:00029ae8       __GSHandlerCheck           000000018002aae8 f   LIBCMT:gshandler.obj
 0001:00029b20       __GSHandlerCheckCommon     000000018002ab20 f   LIBCMT:gshandler.obj
 0001:00029b40       __GSHandlerCheck_EH        000000018002ab40 f   LIBCMT:gshandlereh.obj
 0001:00029bd0       __report_gsfailure         000000018002abd0 f   LIBCMT:gs_report.obj
 0001:00029be8       __report_rangecheckfailure 000000018002abe8 f   LIBCMT:gs_report.obj
 0001:00029c00       __report_securityfailure   000000018002ac00 f   LIBCMT:gs_report.obj
 0001:00029c18       DllMain                    000000018002ac18 f   LIBCMT:dll_dllmain_stub.obj
 0001:00029c18       __acrt_uninitialize_command_line 000000018002ac18 f   libucrt:argv_data.obj
 0001:00029c18       _get_startup_argv_mode     000000018002ac18 f   LIBCMT:argv_mode.obj
 0001:00029c20       __scrt_is_ucrt_dll_in_use  000000018002ac20 f   LIBCMT:ucrt_detection.obj
 0001:00029c38       _invoke_watson             000000018002ac38 f   libucrt:invalid_parameter.obj
 0001:00029c38       __scrt_fastfail            000000018002ac38 f   LIBCMT:utility_desktop.obj
 0001:00029c40       ?__scrt_throw_std_bad_array_new_length@@YAXXZ 000000018002ac40 f   LIBCMT:throw_bad_alloc.obj
 0001:00029c60       __security_init_cookie     000000018002ac60 f   LIBCMT:gs_support.obj
 0001:00029d50       ?__scrt_initialize_type_info@@YAXXZ 000000018002ad50 f   LIBCMT:tncleanup.obj
 0001:00029d68       ?__scrt_uninitialize_type_info@@YAXXZ 000000018002ad68 f   LIBCMT:tncleanup.obj
 0001:00029d78       __local_stdio_scanf_options 000000018002ad78 f i LIBCMT:default_local_stdio_options.obj
 0001:00029d88       __scrt_initialize_default_local_stdio_options 000000018002ad88 f   LIBCMT:default_local_stdio_options.obj
 0001:00029dc0       __scrt_get_dyn_tls_init_callback 000000018002adc0 f   LIBCMT:dyn_tls_init.obj
 0001:00029dd0       _RTC_Initialize            000000018002add0 f   LIBCMT:initsect.obj
 0001:00029e38       _RTC_Terminate             000000018002ae38 f   LIBCMT:initsect.obj
 0001:00029ea0       ??$_CallSETranslator@V__FrameHandler3@@@@YAHPEAUEHExceptionRecord@@PEA_KPEAU_CONTEXT@@PEAU_xDISPATCHER_CONTEXT@@PEBU_s_FuncInfo@@K1H@Z 000000018002aea0 f i libvcruntime:risctrnsctrl.obj
 0001:00029f10       ?CatchTryBlock@__FrameHandler3@@SAPEBU_s_TryBlockMapEntry@@PEBU_s_FuncInfo@@H@Z 000000018002af10 f   libvcruntime:risctrnsctrl.obj
 0001:00029f80       ?ExecutionInCatch@__FrameHandler3@@SA_NPEAU_xDISPATCHER_CONTEXT@@PEBU_s_FuncInfo@@@Z 000000018002af80 f   libvcruntime:risctrnsctrl.obj
 0001:00029fc0       ?FrameUnwindToEmptyState@__FrameHandler3@@SAXPEA_KPEAU_xDISPATCHER_CONTEXT@@PEBU_s_FuncInfo@@@Z 000000018002afc0 f   libvcruntime:risctrnsctrl.obj
 0001:0002a030       ?GetEstablisherFrame@__FrameHandler3@@SAPEA_KPEA_KPEAU_xDISPATCHER_CONTEXT@@PEBU_s_FuncInfo@@0@Z 000000018002b030 f   libvcruntime:risctrnsctrl.obj
 0001:0002a138       ?GetRangeOfTrysToCheck@__FrameHandler3@@SA?AU?$pair@Viterator@TryBlockMap@__FrameHandler3@@V123@@std@@AEAVTryBlockMap@1@HPEAU_xDISPATCHER_CONTEXT@@PEBU_s_FuncInfo@@H@Z 000000018002b138 f   libvcruntime:risctrnsctrl.obj
 0001:0002a298       ?UnwindNestedFrames@__FrameHandler3@@SAXPEA_KPEAUEHExceptionRecord@@PEAU_CONTEXT@@0PEAXPEBU_s_FuncInfo@@HHPEBU_s_HandlerType@@PEAU_xDISPATCHER_CONTEXT@@E@Z 000000018002b298 f   libvcruntime:risctrnsctrl.obj
 0001:0002a348       _CreateFrameInfo           000000018002b348 f   libvcruntime:risctrnsctrl.obj
 0001:0002a398       _FindAndUnlinkFrame        000000018002b398 f   libvcruntime:risctrnsctrl.obj
 0001:0002a3f8       _GetImageBase              000000018002b3f8 f   libvcruntime:risctrnsctrl.obj
 0001:0002a410       _GetThrowImageBase         000000018002b410 f   libvcruntime:risctrnsctrl.obj
 0001:0002a428       _SetImageBase              000000018002b428 f   libvcruntime:risctrnsctrl.obj
 0001:0002a450       _SetThrowImageBase         000000018002b450 f   libvcruntime:risctrnsctrl.obj
 0001:0002a478       __CxxFrameHandler3         000000018002b478 f   libvcruntime:risctrnsctrl.obj
 0001:0002a4f8       __DestructExceptionObject  000000018002b4f8 f   libvcruntime:ehhelpers.obj
 0001:0002a5b0       ?_CallMemberFunction0@@YAXQEAX0@Z 000000018002b5b0 f i libvcruntime:ehhelpers.obj
 0001:0002a5b8       _IsExceptionObjectToBeDestroyed 000000018002b5b8 f   libvcruntime:ehhelpers.obj
 0001:0002a600       __AdjustPointer            000000018002b600 f   libvcruntime:ehhelpers.obj
 0001:0002a628       __FrameUnwindFilter        000000018002b628 f   libvcruntime:ehhelpers.obj
 0001:0002a6c0       __current_exception        000000018002b6c0 f   libvcruntime:ehhelpers.obj
 0001:0002a6d8       __current_exception_context 000000018002b6d8 f   libvcruntime:ehhelpers.obj
 0001:0002a6f0       __std_terminate            000000018002b6f0 f   libvcruntime:ehhelpers.obj
 0001:0002a6f8       __std_exception_copy       000000018002b6f8 f   libvcruntime:std_exception.obj
 0001:0002a790       __std_exception_destroy    000000018002b790 f   libvcruntime:std_exception.obj
 0001:0002a7c8       _get_purecall_handler      000000018002b7c8 f   libvcruntime:purevirt.obj
 0001:0002a7d8       _purecall                  000000018002b7d8 f   libvcruntime:purevirt.obj
 0001:0002a808       wcschr                     000000018002b808 f   libvcruntime:wcschr.obj
 0001:0002a9f0       _CxxThrowException         000000018002b9f0 f   libvcruntime:throw.obj
 0001:0002aac8       __vcrt_initialize          000000018002bac8 f   libvcruntime:initialization.obj
 0001:0002ab08       __vcrt_thread_attach       000000018002bb08 f   libvcruntime:initialization.obj
 0001:0002ab28       __vcrt_thread_detach       000000018002bb28 f   libvcruntime:initialization.obj
 0001:0002ab48       __vcrt_uninitialize        000000018002bb48 f   libvcruntime:initialization.obj
 0001:0002ab70       __vcrt_uninitialize_critical 000000018002bb70 f   libvcruntime:initialization.obj
 0001:0002ab88       __C_specific_handler       000000018002bb88 f   libvcruntime:riscchandler.obj
 0001:0002ae30       __std_type_info_compare    000000018002be30 f   libvcruntime:std_type_info.obj
 0001:0002ae50       __std_type_info_destroy_list 000000018002be50 f   libvcruntime:std_type_info.obj
 0001:0002ae90       __vcrt_freefls             000000018002be90 f   libvcruntime:per_thread_data.obj
 0001:0002aeb0       __vcrt_freeptd             000000018002beb0 f   libvcruntime:per_thread_data.obj
 0001:0002af28       __vcrt_getptd              000000018002bf28 f   libvcruntime:per_thread_data.obj
 0001:0002af48       __vcrt_getptd_noexit       000000018002bf48 f   libvcruntime:per_thread_data.obj
 0001:0002b060       __vcrt_initialize_ptd      000000018002c060 f   libvcruntime:per_thread_data.obj
 0001:0002b0d8       __vcrt_uninitialize_ptd    000000018002c0d8 f   libvcruntime:per_thread_data.obj
 0001:0002b120       ?GetCurrentState@__FrameHandler3@@SAHPEA_KPEAU_xDISPATCHER_CONTEXT@@PEBU_s_FuncInfo@@@Z 000000018002c120 f   libvcruntime:ehstate.obj
 0001:0002b148       ?GetUnwindTryBlock@__FrameHandler3@@SAHPEA_KPEAU_xDISPATCHER_CONTEXT@@PEBU_s_FuncInfo@@@Z 000000018002c148 f   libvcruntime:ehstate.obj
 0001:0002b180       ?SetState@__FrameHandler3@@SAXPEA_KPEBU_s_FuncInfo@@H@Z 000000018002c180 f   libvcruntime:ehstate.obj
 0001:0002b190       ?SetUnwindTryBlock@__FrameHandler3@@SAXPEA_KPEAU_xDISPATCHER_CONTEXT@@PEBU_s_FuncInfo@@H@Z 000000018002c190 f   libvcruntime:ehstate.obj
 0001:0002b1d8       ?StateFromControlPc@__FrameHandler3@@SAHPEBU_s_FuncInfo@@PEAU_xDISPATCHER_CONTEXT@@@Z 000000018002c1d8 f   libvcruntime:ehstate.obj
 0001:0002b1e0       ?StateFromIp@__FrameHandler3@@SAHPEBU_s_FuncInfo@@PEAU_xDISPATCHER_CONTEXT@@_K@Z 000000018002c1e0 f   libvcruntime:ehstate.obj
 0001:0002bd88       ??$TypeMatchHelper@V__FrameHandler3@@@@YAHPEBU_s_HandlerType@@PEBU_s_CatchableType@@PEBU_s_ThrowInfo@@@Z 000000018002cd88 f i libvcruntime:frame.obj
 0001:0002bea8       ??$__InternalCxxFrameHandler@V__FrameHandler3@@@@YA?AW4_EXCEPTION_DISPOSITION@@PEAUEHExceptionRecord@@PEA_KPEAU_CONTEXT@@PEAU_xDISPATCHER_CONTEXT@@PEBU_s_FuncInfo@@H1E@Z 000000018002cea8 f i libvcruntime:frame.obj
 0001:0002c130       ??0bad_exception@std@@QEAA@AEBV01@@Z 000000018002d130 f i libvcruntime:frame.obj
 0001:0002c180       ??0bad_exception@std@@QEAA@XZ 000000018002d180 f i libvcruntime:frame.obj
 0001:0002c1a0       ?CxxCallCatchBlock@__FrameHandler3@@SAPEAXPEAU_EXCEPTION_RECORD@@@Z 000000018002d1a0 f   libvcruntime:frame.obj
 0001:0002c470       ?FrameUnwindToState@__FrameHandler3@@SAXPEA_KPEAU_xDISPATCHER_CONTEXT@@PEBU_s_FuncInfo@@H@Z 000000018002d470 f   libvcruntime:frame.obj
 0001:0002c650       ?GetHandlerSearchState@__FrameHandler3@@SAHPEA_KPEAU_xDISPATCHER_CONTEXT@@PEBU_s_FuncInfo@@@Z 000000018002d650 f i libvcruntime:frame.obj
 0001:0002c7e8       ?_CallMemberFunction1@@YAXQEAX00@Z 000000018002d7e8 f i libvcruntime:frame.obj
 0001:0002c7f8       ?_CallMemberFunction2@@YAXQEAX00H@Z 000000018002d7f8 f i libvcruntime:frame.obj
 0001:0002c808       __vcrt_initialize_locks    000000018002d808 f   libvcruntime:locks.obj
 0001:0002c860       __vcrt_uninitialize_locks  000000018002d860 f   libvcruntime:locks.obj
 0001:0002c8d0       __except_validate_context_record 000000018002d8d0 f   libvcruntime:jbcxrval.obj
 0001:0002c910       calloc                     000000018002d910 f   libucrt:calloc.obj
 0001:0002c918       __acrt_lowio_create_handle_array 000000018002d918 f   libucrt:osfinfo.obj
 0001:0002c9e8       __acrt_lowio_destroy_handle_array 000000018002d9e8 f   libucrt:osfinfo.obj
 0001:0002ca50       __acrt_lowio_ensure_fh_exists 000000018002da50 f   libucrt:osfinfo.obj
 0001:0002cb08       __acrt_lowio_lock_fh       000000018002db08 f   libucrt:osfinfo.obj
 0001:0002cb38       __acrt_lowio_unlock_fh     000000018002db38 f   libucrt:osfinfo.obj
 0001:0002cb68       _free_osfhnd               000000018002db68 f   libucrt:osfinfo.obj
 0001:0002cc58       _get_osfhandle             000000018002dc58 f   libucrt:osfinfo.obj
 0001:0002cce8       __acrt_initialize_stdio    000000018002dce8 f   libucrt:_file.obj
 0001:0002ce08       __acrt_uninitialize_stdio  000000018002de08 f   libucrt:_file.obj
 0001:0002ce80       _lock_file                 000000018002de80 f   libucrt:_file.obj
 0001:0002ce98       _unlock_file               000000018002de98 f   libucrt:_file.obj
 0001:0002ceb0       _dclass                    000000018002deb0 f   libucrt:nan.obj
 0001:0002ced0       _dsign                     000000018002ded0 f   libucrt:nan.obj
 0001:0002ced0       _ldsign                    000000018002ded0 f   libucrt:nanl.obj
 0001:0002d070       ??$ensure_buffer_is_big_enough@D@formatting_buffer@__crt_stdio_output@@QEAA_N_K@Z 000000018002e070 f i libucrt:output.obj
 0001:0002d118       ??$is_wide_character_specifier@D@__crt_stdio_output@@YA_N_KDW4length_modifier@0@@Z 000000018002e118 f i libucrt:output.obj
 0001:0002d160       ??$type_case_integer_parse_into_buffer@I@?$output_processor@DV?$string_output_adapter@D@__crt_stdio_output@@V?$format_validation_base@DV?$string_output_adapter@D@__crt_stdio_output@@@2@@__crt_stdio_output@@AEAAXII_N@Z 000000018002e160 f i libucrt:output.obj
 0001:0002d210       ??$type_case_integer_parse_into_buffer@_K@?$output_processor@DV?$string_output_adapter@D@__crt_stdio_output@@V?$format_validation_base@DV?$string_output_adapter@D@__crt_stdio_output@@@2@@__crt_stdio_output@@AEAAX_KI_N@Z 000000018002e210 f i libucrt:output.obj
 0001:0002d2c8       ??$write_multiple_characters@V?$string_output_adapter@D@__crt_stdio_output@@D@__crt_stdio_output@@YAXAEBV?$string_output_adapter@D@0@DHQEAH@Z 000000018002e2c8 f i libucrt:output.obj
 0001:0002d338       ??0_LocaleUpdate@@QEAA@QEAU__crt_locale_pointers@@@Z 000000018002e338 f i libucrt:output.obj
 0001:0002d3d8       ??1_LocaleUpdate@@QEAA@XZ  000000018002e3d8 f i libucrt:output.obj
 0001:0002d3f8       ?crop_zeroes@__crt_stdio_output@@YAXPEADQEAU__crt_locale_pointers@@@Z 000000018002e3f8 f i libucrt:output.obj
 0001:0002d490       ?force_decimal_point@__crt_stdio_output@@YAXPEADQEAU__crt_locale_pointers@@@Z 000000018002e490 f i libucrt:output.obj
 0001:0002d510       ?parse_int_from_format_string@?$output_processor@DV?$string_output_adapter@D@__crt_stdio_output@@V?$format_validation_base@DV?$string_output_adapter@D@__crt_stdio_output@@@2@@__crt_stdio_output@@AEAA_NQEAH@Z 000000018002e510 f i libucrt:output.obj
 0001:0002d5c0       ?process@?$output_processor@DV?$string_output_adapter@D@__crt_stdio_output@@V?$format_validation_base@DV?$string_output_adapter@D@__crt_stdio_output@@@2@@__crt_stdio_output@@QEAAHXZ 000000018002e5c0 f i libucrt:output.obj
 0001:0002d818       ?state_case_flag@?$output_processor@DV?$string_output_adapter@D@__crt_stdio_output@@V?$format_validation_base@DV?$string_output_adapter@D@__crt_stdio_output@@@2@@__crt_stdio_output@@AEAA_NXZ 000000018002e818 f i libucrt:output.obj
 0001:0002d888       ?state_case_normal_tchar@?$output_processor@DV?$string_output_adapter@D@__crt_stdio_output@@V?$format_validation_base@DV?$string_output_adapter@D@__crt_stdio_output@@@2@@__crt_stdio_output@@AEAA_ND@Z 000000018002e888 f i libucrt:output.obj
 0001:0002d910       ?state_case_size@?$output_processor@DV?$string_output_adapter@D@__crt_stdio_output@@V?$format_validation_base@DV?$string_output_adapter@D@__crt_stdio_output@@@2@@__crt_stdio_output@@AEAA_NXZ 000000018002e910 f i libucrt:output.obj
 0001:0002dad0       ?state_case_type@?$output_processor@DV?$string_output_adapter@D@__crt_stdio_output@@V?$format_validation_base@DV?$string_output_adapter@D@__crt_stdio_output@@@2@@__crt_stdio_output@@AEAA_NXZ 000000018002ead0 f i libucrt:output.obj
 0001:0002de18       ?type_case_Z@?$output_processor@DV?$string_output_adapter@D@__crt_stdio_output@@V?$format_validation_base@DV?$string_output_adapter@D@__crt_stdio_output@@@2@@__crt_stdio_output@@AEAA_NXZ 000000018002ee18 f i libucrt:output.obj
 0001:0002dec0       ?type_case_a@?$output_processor@DV?$string_output_adapter@D@__crt_stdio_output@@V?$format_validation_base@DV?$string_output_adapter@D@__crt_stdio_output@@@2@@__crt_stdio_output@@AEAA_NXZ 000000018002eec0 f i libucrt:output.obj
 0001:0002e0d8       ?type_case_c_tchar@?$output_processor@DV?$string_output_adapter@D@__crt_stdio_output@@V?$format_validation_base@DV?$string_output_adapter@D@__crt_stdio_output@@@2@@__crt_stdio_output@@AEAA_ND@Z 000000018002f0d8 f i libucrt:output.obj
 0001:0002e1a8       ?type_case_integer@?$output_processor@DV?$string_output_adapter@D@__crt_stdio_output@@V?$format_validation_base@DV?$string_output_adapter@D@__crt_stdio_output@@@2@@__crt_stdio_output@@AEAA_NI_N@Z 000000018002f1a8 f i libucrt:output.obj
 0001:0002e3e8       ?type_case_n@?$output_processor@DV?$string_output_adapter@D@__crt_stdio_output@@V?$format_validation_base@DV?$string_output_adapter@D@__crt_stdio_output@@@2@@__crt_stdio_output@@AEAA_NXZ 000000018002f3e8 f i libucrt:output.obj
 0001:0002e4a0       ?type_case_s@?$output_processor@DV?$string_output_adapter@D@__crt_stdio_output@@V?$format_validation_base@DV?$string_output_adapter@D@__crt_stdio_output@@@2@@__crt_stdio_output@@AEAA_NXZ 000000018002f4a0 f i libucrt:output.obj
 0001:0002e560       ?write_character@?$string_output_adapter@D@__crt_stdio_output@@QEBA_NDQEAH@Z 000000018002f560 f i libucrt:output.obj
 0001:0002e5e0       ?write_stored_string_tchar@?$output_processor@DV?$string_output_adapter@D@__crt_stdio_output@@V?$format_validation_base@DV?$string_output_adapter@D@__crt_stdio_output@@@2@@__crt_stdio_output@@AEAA_ND@Z 000000018002f5e0 f i libucrt:output.obj
 0001:0002e6a8       ?write_string@?$string_output_adapter@D@__crt_stdio_output@@QEBAXQEBDHQEAHAEAV__crt_deferred_errno_cache@@@Z 000000018002f6a8 f i libucrt:output.obj
 0001:0002e770       __stdio_common_vsnprintf_s 000000018002f770 f   libucrt:output.obj
 0001:0002e890       _isatty                    000000018002f890 f   libucrt:isatty.obj
 0001:0002e910       terminate                  000000018002f910 f   libucrt:terminate.obj
 0001:0002e948       localeconv                 000000018002f948 f   libucrt:localeconv.obj
 0001:0002e978       _fileno                    000000018002f978 f   libucrt:fileno.obj
 0001:0002e9b0       __acrt_errno_from_os_error 000000018002f9b0 f   libucrt:errno.obj
 0001:0002ea18       __acrt_errno_map_os_error  000000018002fa18 f   libucrt:errno.obj
 0001:0002ea78       __doserrno                 000000018002fa78 f   libucrt:errno.obj
 0001:0002eaa0       _errno                     000000018002faa0 f   libucrt:errno.obj
 0001:0002eac8       _fdclass                   000000018002fac8 f   libucrt:nanf.obj
 0001:0002eae8       _fdsign                    000000018002fae8 f   libucrt:nanf.obj
 0001:0002eb00       _ldclass                   000000018002fb00 f   libucrt:nanl.obj
 0001:0002eb20       free                       000000018002fb20 f   libucrt:free.obj
 0001:0002eb38       malloc                     000000018002fb38 f   libucrt:malloc.obj
 0001:0002eb40       modf                       000000018002fb40 f   libucrt:modf.obj
 0001:0002ebe0       log2                       000000018002fbe0 f   libucrt:log2.obj
 0001:0002ee30       _isleadbyte_l              000000018002fe30 f i libucrt:_wctype.obj
 0001:0002ee90       iswdigit                   000000018002fe90 f i libucrt:_wctype.obj
 0001:0002eea0       wcspbrk                    000000018002fea0 f   libucrt:wcspbrk.obj
 0001:0002eee0       wcstok                     000000018002fee0 f   libucrt:wcstok.obj
 0001:0002ef18       round                      000000018002ff18 f   libucrt:round.obj
 0001:0002ef88       wcsncpy_s                  000000018002ff88 f   libucrt:wcsncpy_s.obj
 0001:0002f068       wcscspn                    0000000180030068 f   libucrt:wcscspn.obj
 0001:0002f0b0       __acrt_initialize_locks    00000001800300b0 f   libucrt:locks.obj
 0001:0002f128       __acrt_lock                0000000180030128 f   libucrt:locks.obj
 0001:0002f150       __acrt_uninitialize_locks  0000000180030150 f   libucrt:locks.obj
 0001:0002f1c0       __acrt_unlock              00000001800301c0 f   libucrt:locks.obj
 0001:0002f1e8       _lock_locales              00000001800301e8 f   libucrt:locks.obj
 0001:0002f218       _unlock_locales            0000000180030218 f   libucrt:locks.obj
 0001:0002f510       setlocale                  0000000180030510 f   libucrt:setlocale.obj
 0001:0002f558       ___lc_codepage_func        0000000180030558 f   libucrt:initctype.obj
 0001:0002f588       ___lc_locale_name_func     0000000180030588 f   libucrt:initctype.obj
 0001:0002f5b8       ___mb_cur_max_func         00000001800305b8 f   libucrt:initctype.obj
 0001:0002f5e8       __acrt_locale_initialize_ctype 00000001800305e8 f   libucrt:initctype.obj
 0001:0002fae0       __pctype_func              0000000180030ae0 f   libucrt:ctype.obj
 0001:0002fb10       ?divide@__crt_strtox@@YA_KAEAUbig_integer@1@AEBU21@@Z 0000000180030b10 f i libucrt:strtod.obj
 0001:0002ff00       pow                        0000000180030f00 f   libucrt:pow.obj
 0001:00030570       strcmp                     0000000180031570 f   libucrt:strcmp.obj
 0001:000305b0       abort                      00000001800315b0 f   libucrt:abort.obj
 0001:000305e0       wcsdup                     00000001800315e0 f   libucrt:wcsdup.obj
 0001:000305e0       _wcsdup                    00000001800315e0 f   libucrt:wcsdup.obj
 0001:00030670       ??$__acrt_mbs_to_wcs_cp@U__crt_win32_buffer_internal_dynamic_resizing@@@@YAHQEBDAEAV?$__crt_win32_buffer@_WU__crt_win32_buffer_internal_dynamic_resizing@@@@I@Z 0000000180031670 f i libucrt:strftime.obj
 0001:000307f8       ??$__acrt_wcs_to_mbs_cp@U__crt_win32_buffer_no_resizing@@@@YAHQEB_WAEAV?$__crt_win32_buffer@DU__crt_win32_buffer_no_resizing@@@@I@Z 00000001800317f8 f i libucrt:strftime.obj
 0001:00030920       __strncnt                  0000000180031920 f   libucrt:strncnt.obj
 0001:00030948       strnlen                    0000000180031948 f   libucrt:strnlen.obj
 0001:00030978       wcsnlen                    0000000180031978 f   libucrt:strnlen.obj
 0001:000309a8       __initialize_lconv_for_unsigned_char 00000001800319a8 f   libucrt:lconv_unsigned_char_initialization.obj
 0001:000309e0       _seh_filter_dll            00000001800319e0 f   libucrt:exception_filter.obj
 0001:00030a08       _seh_filter_exe            0000000180031a08 f   libucrt:exception_filter.obj
 0001:00030f80       __acrt_initialize_thread_local_exit_callback 0000000180031f80 f   libucrt:exit.obj
 0001:00030f90       _cexit                     0000000180031f90 f   libucrt:exit.obj
 0001:00030fa0       _exit                      0000000180031fa0 f   libucrt:exit.obj
 0001:00030fb0       _is_c_termination_complete 0000000180031fb0 f   libucrt:exit.obj
 0001:00031210       __acrt_allocate_buffer_for_argv 0000000180032210 f   libucrt:argv_parsing.obj
 0001:00031280       _configure_narrow_argv     0000000180032280 f   libucrt:argv_parsing.obj
 0001:00031670       __dcrt_uninitialize_environments_nolock 0000000180032670 f   libucrt:environment_initialization.obj
 0001:00031700       _initialize_narrow_environment 0000000180032700 f   libucrt:environment_initialization.obj
 0001:00031aa0       _crt_atexit                0000000180032aa0 f   libucrt:onexit.obj
 0001:00031ab0       _execute_onexit_table      0000000180032ab0 f   libucrt:onexit.obj
 0001:00031af0       _initialize_onexit_table   0000000180032af0 f   libucrt:onexit.obj
 0001:00031b28       _register_onexit_function  0000000180032b28 f   libucrt:onexit.obj
 0001:00031cf8       __acrt_initialize          0000000180032cf8 f   libucrt:initialization.obj
 0001:00031d20       __acrt_thread_attach       0000000180032d20 f   libucrt:initialization.obj
 0001:00031d40       __acrt_thread_detach       0000000180032d40 f   libucrt:initialization.obj
 0001:00031d58       __acrt_uninitialize        0000000180032d58 f   libucrt:initialization.obj
 0001:00031da0       __acrt_uninitialize_critical 0000000180032da0 f   libucrt:initialization.obj
 0001:00031dc0       __acrt_initialize_new_handler 0000000180032dc0 f   libucrt:new_handler.obj
 0001:00031dd0       _callnewh                  0000000180032dd0 f   libucrt:new_handler.obj
 0001:00031e20       _query_new_handler         0000000180032e20 f   libucrt:new_handler.obj
 0001:00031e68       _initterm                  0000000180032e68 f   libucrt:initterm.obj
 0001:00031ed8       _initterm_e                0000000180032ed8 f   libucrt:initterm.obj
 0001:00031f38       strcpy_s                   0000000180032f38 f   libucrt:strcpy_s.obj
 0001:00031fb8       ??$is_overflow_condition@K@__crt_strtox@@YA_NIK@Z 0000000180032fb8 f i libucrt:atox.obj
 0001:00031fe8       ??$parse_integer@KV?$c_string_character_source@D@__crt_strtox@@@__crt_strtox@@YAKQEAU__crt_locale_pointers@@V?$c_string_character_source@D@0@H_N@Z 0000000180032fe8 f i libucrt:atox.obj
 0001:00032368       ??$parse_integer@KV?$c_string_character_source@_W@__crt_strtox@@@__crt_strtox@@YAKQEAU__crt_locale_pointers@@V?$c_string_character_source@_W@0@H_N@Z 0000000180033368 f i libucrt:atox.obj
 0001:00032a50       _wtol                      0000000180033a50 f   libucrt:atox.obj
 0001:00032a78       __acrt_initialize_invalid_parameter_handler 0000000180033a78 f   libucrt:invalid_parameter.obj
 0001:00032a88       _invalid_parameter         0000000180033a88 f   libucrt:invalid_parameter.obj
 0001:00032b38       _invalid_parameter_noinfo  0000000180033b38 f   libucrt:invalid_parameter.obj
 0001:00032d98       __acrt_initialize_lowio    0000000180033d98 f   libucrt:ioinit.obj
 0001:00032de0       __acrt_uninitialize_lowio  0000000180033de0 f   libucrt:ioinit.obj
 0001:00032e28       _calloc_base               0000000180033e28 f   libucrt:calloc_base.obj
 0001:00032ed8       _query_app_type            0000000180033ed8 f   libucrt:report_runtime_error.obj
 0001:00032ee8       _free_base                 0000000180033ee8 f   libucrt:free_base.obj
 0001:00033260       __acrt_AppPolicyGetProcessTerminationMethodInternal 0000000180034260 f   libucrt:winapi_thunks.obj
 0001:000332d0       __acrt_AreFileApisANSI     00000001800342d0 f   libucrt:winapi_thunks.obj
 0001:00033328       __acrt_EnumSystemLocalesEx 0000000180034328 f   libucrt:winapi_thunks.obj
 0001:000333d0       __acrt_FlsAlloc            00000001800343d0 f   libucrt:winapi_thunks.obj
 0001:00033440       __acrt_FlsFree             0000000180034440 f   libucrt:winapi_thunks.obj
 0001:000334b0       __acrt_FlsGetValue         00000001800344b0 f   libucrt:winapi_thunks.obj
 0001:00033520       __acrt_FlsSetValue         0000000180034520 f   libucrt:winapi_thunks.obj
 0001:000335a8       __acrt_GetLocaleInfoEx     00000001800345a8 f   libucrt:winapi_thunks.obj
 0001:00033658       __acrt_GetUserDefaultLocaleName 0000000180034658 f   libucrt:winapi_thunks.obj
 0001:000336e8       __acrt_InitializeCriticalSectionEx 00000001800346e8 f   libucrt:winapi_thunks.obj
 0001:00033778       __acrt_IsValidLocaleName   0000000180034778 f   libucrt:winapi_thunks.obj
 0001:000337f8       __acrt_LCIDToLocaleName    00000001800347f8 f   libucrt:winapi_thunks.obj
 0001:00033890       __acrt_LCMapStringEx       0000000180034890 f   libucrt:winapi_thunks.obj
 0001:00033988       __acrt_LocaleNameToLCID    0000000180034988 f   libucrt:winapi_thunks.obj
 0001:00033a00       __acrt_can_use_vista_locale_apis 0000000180034a00 f   libucrt:winapi_thunks.obj
 0001:00033a38       __acrt_eagerly_load_locale_apis 0000000180034a38 f   libucrt:winapi_thunks.obj
 0001:00033b80       __acrt_initialize_winapi_thunks 0000000180034b80 f   libucrt:winapi_thunks.obj
 0001:00033bc0       __acrt_uninitialize_winapi_thunks 0000000180034bc0 f   libucrt:winapi_thunks.obj
 0001:00033c28       _fcloseall                 0000000180034c28 f   libucrt:closeall.obj
 0001:00033f18       __acrt_stdio_flush_nolock  0000000180034f18 f   libucrt:fflush.obj
 0001:00033fd0       _fflush_nolock             0000000180034fd0 f   libucrt:fflush.obj
 0001:00034038       _flushall                  0000000180035038 f   libucrt:fflush.obj
 0001:00034040       __acrt_stdio_free_buffer_nolock 0000000180035040 f   libucrt:_freebuf.obj
 0001:000340a8       _d_int                     00000001800350a8 f   libucrt:_test.obj
 0001:000341c8       _dtest                     00000001800351c8 f   libucrt:_test.obj
 0001:00034248       _fdtest                    0000000180035248 f   libucrt:_test.obj
 0001:000342a8       _ldtest                    00000001800352a8 f   libucrt:_test.obj
 0001:000342c0       _malloc_base               00000001800352c0 f   libucrt:malloc_base.obj
 0001:00034360       strtol                     0000000180035360 f   libucrt:strtox.obj
 0001:00034390       _mbtowc_l                  0000000180035390 f   libucrt:mbtowc.obj
 0001:00034508       mbtowc                     0000000180035508 f   libucrt:mbtowc.obj
 0001:00034510       _wctomb_s_l                0000000180035510 f   libucrt:wctomb.obj
 0001:000346e0       wctomb_s                   00000001800356e0 f   libucrt:wctomb.obj
 0001:00034ae0       __acrt_freeptd             0000000180035ae0 f   libucrt:per_thread_data.obj
 0001:00034b30       __acrt_getptd              0000000180035b30 f   libucrt:per_thread_data.obj
 0001:00034c20       __acrt_getptd_head         0000000180035c20 f   libucrt:per_thread_data.obj
 0001:00034cd8       __acrt_getptd_noexit       0000000180035cd8 f   libucrt:per_thread_data.obj
 0001:00034dc0       __acrt_initialize_ptd      0000000180035dc0 f   libucrt:per_thread_data.obj
 0001:00034e10       __acrt_uninitialize_ptd    0000000180035e10 f   libucrt:per_thread_data.obj
 0001:00034e48       __acrt_update_locale_info  0000000180035e48 f   libucrt:locale_update.obj
 0001:00034e98       __acrt_update_multibyte_info 0000000180035e98 f   libucrt:locale_update.obj
 0001:000358c0       __acrt_fp_format           00000001800368c0 f   libucrt:cvt.obj
 0001:00035ac8       _get_printf_count_output   0000000180036ac8 f   libucrt:printf_count_output.obj
 0001:00035d90       __acrt_copy_locale_name    0000000180036d90 f   libucrt:wsetlocale.obj
 0001:00035e18       __acrt_set_locale_changed  0000000180036e18 f   libucrt:wsetlocale.obj
 0001:00035e30       __acrt_uninitialize_locale 0000000180036e30 f   libucrt:wsetlocale.obj
 0001:00035e60       __lc_lctowcs               0000000180036e60 f   libucrt:wsetlocale.obj
 0001:00035ef8       __lc_wcstolc               0000000180036ef8 f   libucrt:wsetlocale.obj
 0001:00036450       _wcscats                   0000000180037450 f   libucrt:wsetlocale.obj
 0001:000364e8       _wsetlocale                00000001800374e8 f   libucrt:wsetlocale.obj
 0001:00037b40       _write                     0000000180038b40 f   libucrt:write.obj
 0001:00037c58       _write_nolock              0000000180038c58 f   libucrt:write.obj
 0001:00038040       _handle_error              0000000180039040 f   libucrt:libm_error.obj
 0001:00038178       _handle_nan                0000000180039178 f   libucrt:libm_error.obj
 0001:00038188       iswctype                   0000000180039188 f   libucrt:iswctype.obj
 0001:00038200       __acrt_wcstok_s_novalidation 0000000180039200 f   libucrt:wcstok_s.obj
 0001:000384b0       _mbstowcs_s_l              00000001800394b0 f   libucrt:mbstowcs.obj
 0001:000385f0       mbstowcs_s                 00000001800395f0 f   libucrt:mbstowcs.obj
 0001:00038910       _wcstombs_s_l              0000000180039910 f   libucrt:wcstombs.obj
 0001:00038b98       __acrt_GetLocaleInfoA      0000000180039b98 f   libucrt:getlocaleinfoa.obj
 0001:00038d80       __acrt_GetStringTypeA      0000000180039d80 f   libucrt:getstringtypea.obj
 0001:00039248       __acrt_LCMapStringA        000000018003a248 f   libucrt:lcmapstringa.obj
 0001:000392f0       _errcode                   000000018003a2f0 f   libucrt:fpexcept.obj
 0001:00039330       _except2                   000000018003a330 f   libucrt:fpexcept.obj
 0001:00039428       _handle_exc                000000018003a428 f   libucrt:fpexcept.obj
 0001:00039648       _handle_qnan2              000000018003a648 f   libucrt:fpexcept.obj
 0001:00039650       _raise_exc                 000000018003a650 f   libucrt:fpexcept.obj
 0001:00039658       _raise_exc_ex              000000018003a658 f   libucrt:fpexcept.obj
 0001:00039a88       _set_errno_from_matherr    000000018003aa88 f   libucrt:fpexcept.obj
 0001:00039ac8       _umatherr                  000000018003aac8 f   libucrt:fpexcept.obj
 0001:00039ba0       _decomp                    000000018003aba0 f   libucrt:util.obj
 0001:00039c78       _get_exp                   000000018003ac78 f   libucrt:util.obj
 0001:00039c98       _set_exp                   000000018003ac98 f   libucrt:util.obj
 0001:00039cc8       _sptype                    000000018003acc8 f   libucrt:util.obj
 0001:00039d50       _clrfp                     000000018003ad50 f   libucrt:fpctrl.obj
 0001:00039d68       _ctrlfp                    000000018003ad68 f   libucrt:fpctrl.obj
 0001:00039da0       _set_statfp                000000018003ada0 f   libucrt:fpctrl.obj
 0001:00039db8       _statfp                    000000018003adb8 f   libucrt:fpctrl.obj
 0001:00039dc8       _copysign                  000000018003adc8 f   libucrt:_copysign.obj
 0001:00039de8       _realloc_base              000000018003ade8 f   libucrt:realloc_base.obj
 0001:00039eb0       _d_inttype                 000000018003aeb0 f   libucrt:powhlp.obj
 0001:00039f18       _powhlp                    000000018003af18 f   libucrt:powhlp.obj
 0001:0003a058       _frnd                      000000018003b058 f   libucrt:frnd.obj
 0001:0003a1f0       _fpclass                   000000018003b1f0 f   libucrt:ieeemisc.obj
 0001:0003a2a0       log                        000000018003b2a0 f   libucrt:log.obj
 0001:0003a568       __acrt_get_sigabrt_handler 000000018003b568 f   libucrt:signal.obj
 0001:0003a598       __acrt_initialize_signal_handlers 000000018003b598 f   libucrt:signal.obj
 0001:0003a5b0       raise                      000000018003b5b0 f   libucrt:signal.obj
 0001:0003a820       wcscpy_s                   000000018003b820 f   libucrt:wcscpy_s.obj
 0001:0003a8a0       __acrt_MultiByteToWideChar 000000018003b8a0 f   libucrt:multibytetowidechar.obj
 0001:0003a928       __acrt_WideCharToMultiByte 000000018003b928 f   libucrt:widechartomultibyte.obj
 0001:0003a9d0       __ascii_wcsicmp            000000018003b9d0 f   libucrt:wcsicmp.obj
 0001:0003aa10       _wcsicmp                   000000018003ba10 f   libucrt:wcsicmp.obj
 0001:0003aa60       _wcsicmp_l                 000000018003ba60 f   libucrt:wcsicmp.obj
 0001:0003ab80       __acrt_initialize_timeset  000000018003bb80 f   libucrt:timeset.obj
 0001:0003abb8       __acrt_get_process_end_policy 000000018003bbb8 f   libucrt:win_policies.obj
 0001:0003ac20       ??$__acrt_wcs_to_mbs_cp@U__crt_win32_buffer_internal_dynamic_resizing@@@@YAHQEB_WAEAV?$__crt_win32_buffer@DU__crt_win32_buffer_internal_dynamic_resizing@@@@I@Z 000000018003bc20 f i libucrt:argv_wildcards.obj
 0001:0003b4f0       __acrt_expand_narrow_argv_wildcards 000000018003c4f0 f   libucrt:argv_wildcards.obj
 0001:0003b4f8       __acrt_GetModuleFileNameA  000000018003c4f8 f   libucrt:getmodulefilenamea.obj
 0001:0003bd20       __acrt_initialize_multibyte 000000018003cd20 f   libucrt:mbctype.obj
 0001:0003bd90       __acrt_update_thread_multibyte_data 000000018003cd90 f   libucrt:mbctype.obj
 0001:0003bdb0       _setmbcp_nolock            000000018003cdb0 f   libucrt:mbctype.obj
 0001:0003c0d8       _ismbblead                 000000018003d0d8 f   libucrt:ismbbyte.obj
 0001:0003c0f0       __acrt_initialize_command_line 000000018003d0f0 f   libucrt:argv_data.obj
 0001:0003c138       __dcrt_get_narrow_environment_from_os 000000018003d138 f   libucrt:get_environment_from_os.obj
 0001:0003c260       _recalloc_base             000000018003d260 f   libucrt:recalloc.obj
 0001:0003c300       __acrt_initialize_heap     000000018003d300 f   libucrt:heap_handle.obj
 0001:0003c330       __acrt_uninitialize_heap   000000018003d330 f   libucrt:heap_handle.obj
 0001:0003c340       __acrt_execute_initializers 000000018003d340 f   libucrt:shared_initialization.obj
 0001:0003c400       __acrt_execute_uninitializers 000000018003d400 f   libucrt:shared_initialization.obj
 0001:0003c460       __acrt_has_user_matherr    000000018003d460 f   libucrt:matherr.obj
 0001:0003c488       __acrt_initialize_user_matherr 000000018003d488 f   libucrt:matherr.obj
 0001:0003c498       __acrt_invoke_user_matherr 000000018003d498 f   libucrt:matherr.obj
 0001:0003c5b8       _lseeki64_nolock           000000018003d5b8 f   libucrt:lseek.obj
 0001:0003c5c0       _query_new_mode            000000018003d5c0 f   libucrt:new_mode.obj
 0001:0003c5d0       wcscat_s                   000000018003d5d0 f   libucrt:wcscat_s.obj
 0001:0003c668       wcsncmp                    000000018003d668 f   libucrt:wcsncmp.obj
 0001:0003c6b0       __acrt_DownlevelLCIDToLocaleName 000000018003d6b0 f   libucrt:lcidtoname_downlevel.obj
 0001:0003c7b0       __acrt_DownlevelLocaleNameToLCID 000000018003d7b0 f   libucrt:lcidtoname_downlevel.obj
 0001:0003c868       _fclose_nolock             000000018003d868 f   libucrt:fclose.obj
 0001:0003c900       fclose                     000000018003d900 f   libucrt:fclose.obj
 0001:0003ca30       _commit                    000000018003da30 f   libucrt:commit.obj
 0001:0003cad0       __acrt_fenv_get_control    000000018003dad0 f   libucrt:_fenvutils.obj
 0001:0003cb90       __acrt_fenv_get_status     000000018003db90 f   libucrt:_fenvutils.obj
 0001:0003cbf8       __acrt_fenv_set_control    000000018003dbf8 f   libucrt:_fenvutils.obj
 0001:0003cce0       __acrt_fenv_set_status     000000018003dce0 f   libucrt:_fenvutils.obj
 0001:0003cd60       ?__mbrtowc_utf8@__crt_mbstring@@YA_KPEA_WPEBD_KPEAU_Mbstatet@@@Z 000000018003dd60 f   libucrt:mbrtowc.obj
 0001:0003cda8       ?__mbsrtowcs_utf8@__crt_mbstring@@YA_KPEA_WPEAPEBD_KPEAU_Mbstatet@@@Z 000000018003dda8 f   libucrt:mbrtowc.obj
 0001:0003cf50       ?__c32rtomb_utf8@__crt_mbstring@@YA_KPEAD_UPEAU_Mbstatet@@@Z 000000018003df50 f   libucrt:c32rtomb.obj
 0001:0003d028       c32rtomb                   000000018003e028 f   libucrt:c32rtomb.obj
 0001:0003d030       __acrt_add_locale_ref      000000018003e030 f   libucrt:locale_refcounting.obj
 0001:0003d128       __acrt_free_locale         000000018003e128 f   libucrt:locale_refcounting.obj
 0001:0003d278       __acrt_locale_add_lc_time_reference 000000018003e278 f   libucrt:locale_refcounting.obj
 0001:0003d2b8       __acrt_locale_free_lc_time_if_unreferenced 000000018003e2b8 f   libucrt:locale_refcounting.obj
 0001:0003d300       __acrt_locale_release_lc_time_reference 000000018003e300 f   libucrt:locale_refcounting.obj
 0001:0003d340       __acrt_release_locale_ref  000000018003e340 f   libucrt:locale_refcounting.obj
 0001:0003d440       __acrt_update_thread_locale_data 000000018003e440 f   libucrt:locale_refcounting.obj
 0001:0003d4b0       _updatetlocinfoEx_nolock   000000018003e4b0 f   libucrt:locale_refcounting.obj
 0001:0003d528       __acrt_fp_strflt_to_string 000000018003e528 f   libucrt:_fptostr.obj
 0001:0003d660       __acrt_fltout              000000018003e660 f   libucrt:cfout.obj
 0001:0003e830       __acrt_locale_free_monetary 000000018003f830 f   libucrt:initmon.obj
 0001:0003e960       __acrt_locale_initialize_monetary 000000018003f960 f   libucrt:initmon.obj
 0001:0003ee70       __acrt_locale_free_numeric 000000018003fe70 f   libucrt:initnum.obj
 0001:0003ef00       __acrt_locale_initialize_numeric 000000018003ff00 f   libucrt:initnum.obj
 0001:0003f518       __acrt_locale_free_time    0000000180040518 f   libucrt:inittime.obj
 0001:0003f5e8       __acrt_locale_initialize_time 00000001800405e8 f   libucrt:inittime.obj
 0001:0003f680       wcsncat_s                  0000000180040680 f   libucrt:wcsncat_s.obj
 0001:0003fe90       __acrt_get_qualified_locale 0000000180040e90 f   libucrt:get_qualified_locale.obj
 0001:00040a08       __acrt_get_qualified_locale_downlevel 0000000180041a08 f   libucrt:getqloc_downlevel.obj
 0001:00040ca0       wcscmp                     0000000180041ca0 f   libucrt:wcscmp.obj
 0001:00040cd8       _putwch_nolock             0000000180041cd8 f   libucrt:putwch.obj
 0001:00040d18       __acrt_GetStringTypeW      0000000180041d18 f   libucrt:getstringtypew.obj
 0001:00040d28       ?__wcsrtombs_utf8@__crt_mbstring@@YA_KPEADPEAPEB_W_KPEAU_Mbstatet@@@Z 0000000180041d28 f   libucrt:wcrtomb.obj
 0001:00040e70       strncpy_s                  0000000180041e70 f   libucrt:strncpy_s.obj
 0001:00040fa8       _clearfp                   0000000180041fa8 f   libucrt:ieee.obj
 0001:00040fc0       _towlower_l                0000000180041fc0 f   libucrt:towlower.obj
 0001:00041080       qsort                      0000000180042080 f   libucrt:qsort.obj
 0001:000414a8       strpbrk                    00000001800424a8 f   libucrt:strpbrk.obj
 0001:00041558       _mbsdec                    0000000180042558 f   libucrt:mbsdec.obj
 0001:00041560       _mbsdec_l                  0000000180042560 f   libucrt:mbsdec.obj
 0001:00041630       _msize_base                0000000180042630 f   libucrt:msize.obj
 0001:00041680       __ascii_wcsnicmp           0000000180042680 f   libucrt:wcsnicmp.obj
 0001:000416d0       _wcsnicmp                  00000001800426d0 f   libucrt:wcsnicmp.obj
 0001:00041720       _wcsnicmp_l                0000000180042720 f   libucrt:wcsnicmp.obj
 0001:000418e8       _close                     00000001800428e8 f   libucrt:close.obj
 0001:00041998       _close_nolock              0000000180042998 f   libucrt:close.obj
 0001:00041a88       ?__acrt_stdio_free_stream@@YAXV__crt_stdio_stream@@@Z 0000000180042a88 f   libucrt:stream.obj
 0001:00041ab0       ?__mbrtoc32_utf8@__crt_mbstring@@YA_KPEA_UPEBD_KPEAU_Mbstatet@@@Z 0000000180042ab0 f   libucrt:mbrtoc32.obj
 0001:00041c78       fegetenv                   0000000180042c78 f   libucrt:fegetenv.obj
 0001:00041ca8       fesetenv                   0000000180042ca8 f   libucrt:fesetenv.obj
 0001:00041d10       feholdexcept               0000000180042d10 f   libucrt:feholdexcept.obj
 0001:00041d70       log10                      0000000180042d70 f   libucrt:log10.obj
 0001:00042120       _itow_s                    0000000180043120 f   libucrt:xtoa.obj
 0001:00042130       __dcrt_lowio_ensure_console_output_initialized 0000000180043130 f   libucrt:initcon.obj
 0001:00042198       __dcrt_terminate_console_output 0000000180043198 f   libucrt:initcon.obj
 0001:000421c0       __dcrt_write_console       00000001800431c0 f   libucrt:initcon.obj
 0001:000422b8       ?__c16rtomb_utf8@__crt_mbstring@@YA_KPEAD_SPEAU_Mbstatet@@@Z 00000001800432b8 f   libucrt:c16rtomb.obj
 0001:00042380       __acrt_LCMapStringW        0000000180043380 f   libucrt:lcmapstringw.obj
 0001:00042410       _FindPESection             0000000180043410 f   LIBCMT:pesect.obj
 0001:00042470       _IsNonwritableInCurrentImage 0000000180043470 f   LIBCMT:pesect.obj
 0001:000424d8       _ValidateImageBase         00000001800434d8 f   LIBCMT:pesect.obj
 0001:00042518       strrchr                    0000000180043518 f   libvcruntime:strrchr.obj
 0002:00000000       __imp_LookupPrivilegeValueW 0000000180046000     advapi32:ADVAPI32.dll
 0002:00000008       __imp_AdjustTokenPrivileges 0000000180046008     advapi32:ADVAPI32.dll
 0002:00000010       __imp_OpenProcessToken     0000000180046010     advapi32:ADVAPI32.dll
 0002:00000018       __imp_SetThreadToken       0000000180046018     advapi32:ADVAPI32.dll
 0002:00000020       __imp_DuplicateTokenEx     0000000180046020     advapi32:ADVAPI32.dll
 0002:00000028       __imp_OpenThreadToken      0000000180046028     advapi32:ADVAPI32.dll
 0002:00000030       __imp_RegCloseKey          0000000180046030     advapi32:ADVAPI32.dll
 0002:00000038       __imp_RegConnectRegistryW  0000000180046038     advapi32:ADVAPI32.dll
 0002:00000040       __imp_RegQueryValueExW     0000000180046040     advapi32:ADVAPI32.dll
 0002:00000048       __imp_ConvertSidToStringSidW 0000000180046048     advapi32:ADVAPI32.dll
 0002:00000050       __imp_GetUserNameW         0000000180046050     advapi32:ADVAPI32.dll
 0002:00000058       __imp_LookupAccountNameW   0000000180046058     advapi32:ADVAPI32.dll
 0002:00000060       \177ADVAPI32_NULL_THUNK_DATA 0000000180046060     advapi32:ADVAPI32.dll
 0002:00000068       __imp_lstrlenW             0000000180046068     kernel32:KERNEL32.dll
 0002:00000070       __imp_SetLastError         0000000180046070     kernel32:KERNEL32.dll
 0002:00000078       __imp_SetPriorityClass     0000000180046078     kernel32:KERNEL32.dll
 0002:00000080       __imp_lstrcpynW            0000000180046080     kernel32:KERNEL32.dll
 0002:00000088       __imp_CreateFileW          0000000180046088     kernel32:KERNEL32.dll
 0002:00000090       __imp_GetCurrentThreadId   0000000180046090     kernel32:KERNEL32.dll
 0002:00000098       __imp_SetEvent             0000000180046098     kernel32:KERNEL32.dll
 0002:000000a0       __imp_FileTimeToSystemTime 00000001800460a0     kernel32:KERNEL32.dll
 0002:000000a8       __imp_GetLocalTime         00000001800460a8     kernel32:KERNEL32.dll
 0002:000000b0       __imp_GetPriorityClass     00000001800460b0     kernel32:KERNEL32.dll
 0002:000000b8       __imp_SystemTimeToTzSpecificLocalTime 00000001800460b8     kernel32:KERNEL32.dll
 0002:000000c0       __imp_GetSystemTimeAsFileTime 00000001800460c0     kernel32:KERNEL32.dll
 0002:000000c8       __imp_GetTickCount         00000001800460c8     kernel32:KERNEL32.dll
 0002:000000d0       __imp_lstrcmpW             00000001800460d0     kernel32:KERNEL32.dll
 0002:000000d8       __imp_WaitForMultipleObjects 00000001800460d8     kernel32:KERNEL32.dll
 0002:000000e0       __imp_GetFileType          00000001800460e0     kernel32:KERNEL32.dll
 0002:000000e8       __imp_ReleaseMutex         00000001800460e8     kernel32:KERNEL32.dll
 0002:000000f0       __imp_CreateEventW         00000001800460f0     kernel32:KERNEL32.dll
 0002:000000f8       __imp_ResetEvent           00000001800460f8     kernel32:KERNEL32.dll
 0002:00000100       __imp_GetProcessTimes      0000000180046100     kernel32:KERNEL32.dll
 0002:00000108       __imp_TerminateProcess     0000000180046108     kernel32:KERNEL32.dll
 0002:00000110       __imp_OpenProcess          0000000180046110     kernel32:KERNEL32.dll
 0002:00000118       __imp_GetLastError         0000000180046118     kernel32:KERNEL32.dll
 0002:00000120       __imp_GetCurrentThread     0000000180046120     kernel32:KERNEL32.dll
 0002:00000128       __imp_ReadProcessMemory    0000000180046128     kernel32:KERNEL32.dll
 0002:00000130       __imp_FormatMessageW       0000000180046130     kernel32:KERNEL32.dll
 0002:00000138       __imp_FileTimeToLocalFileTime 0000000180046138     kernel32:KERNEL32.dll
 0002:00000140       __imp_GetTimeFormatW       0000000180046140     kernel32:KERNEL32.dll
 0002:00000148       __imp_GetModuleHandleW     0000000180046148     kernel32:KERNEL32.dll
 0002:00000150       __imp_GetDateFormatW       0000000180046150     kernel32:KERNEL32.dll
 0002:00000158       __imp_GetProcAddress       0000000180046158     kernel32:KERNEL32.dll
 0002:00000160       __imp_HeapSize             0000000180046160     kernel32:KERNEL32.dll
 0002:00000168       __imp_GetCurrentProcessId  0000000180046168     kernel32:KERNEL32.dll
 0002:00000170       __imp_LocalFree            0000000180046170     kernel32:KERNEL32.dll
 0002:00000178       __imp_CreateThread         0000000180046178     kernel32:KERNEL32.dll
 0002:00000180       __imp_CloseHandle          0000000180046180     kernel32:KERNEL32.dll
 0002:00000188       __imp_TerminateThread      0000000180046188     kernel32:KERNEL32.dll
 0002:00000190       __imp_DuplicateHandle      0000000180046190     kernel32:KERNEL32.dll
 0002:00000198       __imp_WaitForSingleObject  0000000180046198     kernel32:KERNEL32.dll
 0002:000001a0       __imp_VirtualAlloc         00000001800461a0     kernel32:KERNEL32.dll
 0002:000001a8       __imp_GetCurrentProcess    00000001800461a8     kernel32:KERNEL32.dll
 0002:000001b0       __imp_VirtualFree          00000001800461b0     kernel32:KERNEL32.dll
 0002:000001b8       __imp_WriteConsoleW        00000001800461b8     kernel32:KERNEL32.dll
 0002:000001c0       __imp_CreateMutexW         00000001800461c0     kernel32:KERNEL32.dll
 0002:000001c8       __imp_WriteFile            00000001800461c8     kernel32:KERNEL32.dll
 0002:000001d0       __imp_FlushFileBuffers     00000001800461d0     kernel32:KERNEL32.dll
 0002:000001d8       __imp_GetProcessHeap       00000001800461d8     kernel32:KERNEL32.dll
 0002:000001e0       __imp_FreeEnvironmentStringsW 00000001800461e0     kernel32:KERNEL32.dll
 0002:000001e8       __imp_GetEnvironmentStringsW 00000001800461e8     kernel32:KERNEL32.dll
 0002:000001f0       __imp_GetCommandLineW      00000001800461f0     kernel32:KERNEL32.dll
 0002:000001f8       __imp_GetCommandLineA      00000001800461f8     kernel32:KERNEL32.dll
 0002:00000200       __imp_GetOEMCP             0000000180046200     kernel32:KERNEL32.dll
 0002:00000208       __imp_GetACP               0000000180046208     kernel32:KERNEL32.dll
 0002:00000210       __imp_IsValidCodePage      0000000180046210     kernel32:KERNEL32.dll
 0002:00000218       __imp_FindNextFileW        0000000180046218     kernel32:KERNEL32.dll
 0002:00000220       __imp_FindFirstFileExW     0000000180046220     kernel32:KERNEL32.dll
 0002:00000228       __imp_FindClose            0000000180046228     kernel32:KERNEL32.dll
 0002:00000230       __imp_HeapReAlloc          0000000180046230     kernel32:KERNEL32.dll
 0002:00000238       __imp_GetConsoleMode       0000000180046238     kernel32:KERNEL32.dll
 0002:00000240       __imp_GetConsoleCP         0000000180046240     kernel32:KERNEL32.dll
 0002:00000248       __imp_EnumSystemLocalesW   0000000180046248     kernel32:KERNEL32.dll
 0002:00000250       __imp_GetUserDefaultLCID   0000000180046250     kernel32:KERNEL32.dll
 0002:00000258       __imp_IsValidLocale        0000000180046258     kernel32:KERNEL32.dll
 0002:00000260       __imp_GetLocaleInfoW       0000000180046260     kernel32:KERNEL32.dll
 0002:00000268       __imp_LCMapStringW         0000000180046268     kernel32:KERNEL32.dll
 0002:00000270       __imp_LoadLibraryExW       0000000180046270     kernel32:KERNEL32.dll
 0002:00000278       __imp_TlsFree              0000000180046278     kernel32:KERNEL32.dll
 0002:00000280       __imp_MultiByteToWideChar  0000000180046280     kernel32:KERNEL32.dll
 0002:00000288       __imp_WideCharToMultiByte  0000000180046288     kernel32:KERNEL32.dll
 0002:00000290       __imp_EnterCriticalSection 0000000180046290     kernel32:KERNEL32.dll
 0002:00000298       __imp_LeaveCriticalSection 0000000180046298     kernel32:KERNEL32.dll
 0002:000002a0       __imp_InitializeCriticalSectionEx 00000001800462a0     kernel32:KERNEL32.dll
 0002:000002a8       __imp_DeleteCriticalSection 00000001800462a8     kernel32:KERNEL32.dll
 0002:000002b0       __imp_EncodePointer        00000001800462b0     kernel32:KERNEL32.dll
 0002:000002b8       __imp_DecodePointer        00000001800462b8     kernel32:KERNEL32.dll
 0002:000002c0       __imp_GetStringTypeW       00000001800462c0     kernel32:KERNEL32.dll
 0002:000002c8       __imp_GetCPInfo            00000001800462c8     kernel32:KERNEL32.dll
 0002:000002d0       __imp_GetStartupInfoW      00000001800462d0     kernel32:KERNEL32.dll
 0002:000002d8       __imp_QueryPerformanceCounter 00000001800462d8     kernel32:KERNEL32.dll
 0002:000002e0       __imp_InitializeSListHead  00000001800462e0     kernel32:KERNEL32.dll
 0002:000002e8       __imp_RtlLookupFunctionEntry 00000001800462e8     kernel32:KERNEL32.dll
 0002:000002f0       __imp_RtlUnwindEx          00000001800462f0     kernel32:KERNEL32.dll
 0002:000002f8       __imp_RtlPcToFileHeader    00000001800462f8     kernel32:KERNEL32.dll
 0002:00000300       __imp_RaiseException       0000000180046300     kernel32:KERNEL32.dll
 0002:00000308       __imp_InterlockedFlushSList 0000000180046308     kernel32:KERNEL32.dll
 0002:00000310       __imp_FlsAlloc             0000000180046310     kernel32:KERNEL32.dll
 0002:00000318       __imp_FlsGetValue          0000000180046318     kernel32:KERNEL32.dll
 0002:00000320       __imp_FlsSetValue          0000000180046320     kernel32:KERNEL32.dll
 0002:00000328       __imp_FlsFree              0000000180046328     kernel32:KERNEL32.dll
 0002:00000330       __imp_SetStdHandle         0000000180046330     kernel32:KERNEL32.dll
 0002:00000338       __imp_ExitProcess          0000000180046338     kernel32:KERNEL32.dll
 0002:00000340       __imp_FreeLibrary          0000000180046340     kernel32:KERNEL32.dll
 0002:00000348       __imp_GetModuleHandleExW   0000000180046348     kernel32:KERNEL32.dll
 0002:00000350       __imp_GetModuleFileNameW   0000000180046350     kernel32:KERNEL32.dll
 0002:00000358       __imp_SetFilePointerEx     0000000180046358     kernel32:KERNEL32.dll
 0002:00000360       __imp_GetStdHandle         0000000180046360     kernel32:KERNEL32.dll
 0002:00000368       __imp_HeapAlloc            0000000180046368     kernel32:KERNEL32.dll
 0002:00000370       __imp_HeapFree             0000000180046370     kernel32:KERNEL32.dll
 0002:00000378       __imp_InitializeCriticalSectionAndSpinCount 0000000180046378     kernel32:KERNEL32.dll
 0002:00000380       __imp_TlsAlloc             0000000180046380     kernel32:KERNEL32.dll
 0002:00000388       __imp_TlsGetValue          0000000180046388     kernel32:KERNEL32.dll
 0002:00000390       __imp_TlsSetValue          0000000180046390     kernel32:KERNEL32.dll
 0002:00000398       \177KERNEL32_NULL_THUNK_DATA 0000000180046398     kernel32:KERNEL32.dll
 0002:000003a0       __imp_WNetCancelConnection2W 00000001800463a0     mpr:MPR.dll
 0002:000003a8       __imp_WNetAddConnection2W  00000001800463a8     mpr:MPR.dll
 0002:000003b0       \177MPR_NULL_THUNK_DATA    00000001800463b0     mpr:MPR.dll
 0002:000003b8       __imp_VariantClear         00000001800463b8     oleaut32:OLEAUT32.dll
 0002:000003c0       __imp_SysAllocString       00000001800463c0     oleaut32:OLEAUT32.dll
 0002:000003c8       __imp_SysFreeString        00000001800463c8     oleaut32:OLEAUT32.dll
 0002:000003d0       \177OLEAUT32_NULL_THUNK_DATA 00000001800463d0     oleaut32:OLEAUT32.dll
 0002:000003d8       __imp_GetModuleInformation 00000001800463d8     psapi:PSAPI.DLL
 0002:000003e0       __imp_GetModuleFileNameExW 00000001800463e0     psapi:PSAPI.DLL
 0002:000003e8       \177PSAPI_NULL_THUNK_DATA  00000001800463e8     psapi:PSAPI.DLL
 0002:000003f0       __imp_GetAncestor          00000001800463f0     user32:USER32.dll
 0002:000003f8       __imp_SetForegroundWindow  00000001800463f8     user32:USER32.dll
 0002:00000400       __imp_IsIconic             0000000180046400     user32:USER32.dll
 0002:00000408       __imp_GetWindowTextW       0000000180046408     user32:USER32.dll
 0002:00000410       __imp_GetParent            0000000180046410     user32:USER32.dll
 0002:00000418       __imp_CharUpperBuffW       0000000180046418     user32:USER32.dll
 0002:00000420       __imp_EnumWindows          0000000180046420     user32:USER32.dll
 0002:00000428       __imp_GetWindowThreadProcessId 0000000180046428     user32:USER32.dll
 0002:00000430       __imp_GetLastActivePopup   0000000180046430     user32:USER32.dll
 0002:00000438       __imp_ShowWindowAsync      0000000180046438     user32:USER32.dll
 0002:00000440       __imp_IsWindowVisible      0000000180046440     user32:USER32.dll
 0002:00000448       __imp_GetWindowLongPtrW    0000000180046448     user32:USER32.dll
 0002:00000450       \177USER32_NULL_THUNK_DATA 0000000180046450     user32:USER32.dll
 0002:00000458       __imp_GetFileVersionInfoSizeW 0000000180046458     version:VERSION.dll
 0002:00000460       __imp_GetFileVersionInfoW  0000000180046460     version:VERSION.dll
 0002:00000468       __imp_VerQueryValueW       0000000180046468     version:VERSION.dll
 0002:00000470       \177VERSION_NULL_THUNK_DATA 0000000180046470     version:VERSION.dll
 0002:00000478       __imp_CoUninitialize       0000000180046478     ole32:ole32.dll
 0002:00000480       __imp_CoInitialize         0000000180046480     ole32:ole32.dll
 0002:00000488       __imp_CoCreateInstance     0000000180046488     ole32:ole32.dll
 0002:00000490       \177ole32_NULL_THUNK_DATA  0000000180046490     ole32:ole32.dll
 0002:00000498       __guard_check_icall_fptr   0000000180046498     LIBCMT:guard_support.obj
 0002:000004a0       __xc_a                     00000001800464a0     LIBCMT:initializers.obj
 0002:000004e8       __xc_z                     00000001800464e8     LIBCMT:initializers.obj
 0002:000004f0       __xi_a                     00000001800464f0     LIBCMT:initializers.obj
 0002:00000500       __acrt_stdio_initializer   0000000180046500     libucrt:stdio_initializer.obj
 0002:00000508       __acrt_timeset_initializer 0000000180046508     libucrt:timeset_initializer.obj
 0002:00000510       __acrt_multibyte_initializer 0000000180046510     libucrt:multibyte_initializer.obj
 0002:00000518       __xi_z                     0000000180046518     LIBCMT:initializers.obj
 0002:00000520       __xp_a                     0000000180046520     LIBCMT:initializers.obj
 0002:00000528       __acrt_locale_terminator   0000000180046528     libucrt:locale_initializer.obj
 0002:00000530       __dcrt_console_output_terminator 0000000180046530     libucrt:console_output_initializer.obj
 0002:00000538       __acrt_stdio_terminator    0000000180046538     libucrt:stdio_initializer.obj
 0002:00000540       __xp_z                     0000000180046540     LIBCMT:initializers.obj
 0002:00000548       __xt_a                     0000000180046548     LIBCMT:initializers.obj
 0002:00000550       __xt_z                     0000000180046550     LIBCMT:initializers.obj
 0002:00000560       CLSID_WbemLocator          0000000180046560     wbemuuid:wbemcli_i.obj
 0002:00000570       IID_IWbemLocator           0000000180046570     wbemuuid:wbemcli_i.obj
 0002:00000588       ??_7exception@std@@6B@     0000000180046588     libcpmt:xthrow.obj
 0002:000005a0       ??_7bad_alloc@std@@6B@     00000001800465a0     libcpmt:xthrow.obj
 0002:000005b0       ??_C@_0P@GHFPNOJB@bad?5allocation@ 00000001800465b0     libcpmt:xthrow.obj
 0002:000005c8       ??_7bad_function_call@std@@6B@ 00000001800465c8     libcpmt:xthrow.obj
 0002:000005d8       ??_C@_0BC@DPJNKNAF@bad?5function?5call@ 00000001800465d8     libcpmt:xthrow.obj
 0002:000005f8       ??_7logic_error@std@@6B@   00000001800465f8     libcpmt:xthrow.obj
 0002:00000610       ??_7length_error@std@@6B@  0000000180046610     libcpmt:xthrow.obj
 0002:00000628       ??_7out_of_range@std@@6B@  0000000180046628     libcpmt:xthrow.obj
 0002:00000640       ??_7runtime_error@std@@6B@ 0000000180046640     libcpmt:xthrow.obj
 0002:00000680       ??_7_Facet_base@std@@6B@   0000000180046680     libcpmt:locale0.obj
 0002:000006a0       ??_7_Locimp@locale@std@@6B@ 00000001800466a0     libcpmt:locale0.obj
 0002:000006b8       ??_C@_01NBENCBCI@?$CK@     00000001800466b8     libcpmt:locale0.obj
 0002:000006bc       ??_C@_01GFHCPBMG@C@        00000001800466bc     libcpmt:locale0.obj
 0002:00000e20       ??_C@_0BN@LKKBCCDB@address?5family?5not?5supported@ 0000000180046e20     libcpmt:syserror.obj
 0002:00000e40       ??_C@_0P@LDMLAFHI@address?5in?5use@ 0000000180046e40     libcpmt:syserror.obj
 0002:00000e50       ??_C@_0BG@DHPCNBJB@address?5not?5available@ 0000000180046e50     libcpmt:syserror.obj
 0002:00000e68       ??_C@_0BC@DFIBIBIL@already?5connected@ 0000000180046e68     libcpmt:syserror.obj
 0002:00000e80       ??_C@_0BH@CAKOHOMI@argument?5list?5too?5long@ 0000000180046e80     libcpmt:syserror.obj
 0002:00000e98       ??_C@_0BH@CGIMPKIM@argument?5out?5of?5domain@ 0000000180046e98     libcpmt:syserror.obj
 0002:00000eb0       ??_C@_0M@KGHGGJGL@bad?5address@ 0000000180046eb0     libcpmt:syserror.obj
 0002:00000ec0       ??_C@_0BE@MPJPGCEO@bad?5file?5descriptor@ 0000000180046ec0     libcpmt:syserror.obj
 0002:00000ed8       ??_C@_0M@PMMIEFCP@bad?5message@ 0000000180046ed8     libcpmt:syserror.obj
 0002:00000ee8       ??_C@_0M@KPHOFDBE@broken?5pipe@ 0000000180046ee8     libcpmt:syserror.obj
 0002:00000ef8       ??_C@_0BD@MGNDDEGM@connection?5aborted@ 0000000180046ef8     libcpmt:syserror.obj
 0002:00000f10       ??_C@_0BP@KAIHPOGN@connection?5already?5in?5progress@ 0000000180046f10     libcpmt:syserror.obj
 0002:00000f30       ??_C@_0BD@PJLIIJEL@connection?5refused@ 0000000180046f30     libcpmt:syserror.obj
 0002:00000f48       ??_C@_0BB@IECNJNOI@connection?5reset@ 0000000180046f48     libcpmt:syserror.obj
 0002:00000f60       ??_C@_0BC@PPHBOELF@cross?5device?5link@ 0000000180046f60     libcpmt:syserror.obj
 0002:00000f78       ??_C@_0BN@KDMIFEIP@destination?5address?5required@ 0000000180046f78     libcpmt:syserror.obj
 0002:00000f98       ??_C@_0BI@NGCEHDD@device?5or?5resource?5busy@ 0000000180046f98     libcpmt:syserror.obj
 0002:00000fb0       ??_C@_0BE@JIDOCPHM@directory?5not?5empty@ 0000000180046fb0     libcpmt:syserror.obj
 0002:00000fc8       ??_C@_0BI@BNCLIGPB@executable?5format?5error@ 0000000180046fc8     libcpmt:syserror.obj
 0002:00000fe0       ??_C@_0M@MIDIAGJP@file?5exists@ 0000000180046fe0     libcpmt:syserror.obj
 0002:00000ff0       ??_C@_0P@DNAJLBJK@file?5too?5large@ 0000000180046ff0     libcpmt:syserror.obj
 0002:00001000       ??_C@_0BC@EJHOMAAK@filename?5too?5long@ 0000000180047000     libcpmt:syserror.obj
 0002:00001018       ??_C@_0BH@KEFGLDAF@function?5not?5supported@ 0000000180047018     libcpmt:syserror.obj
 0002:00001030       ??_C@_0BB@DHFDFGDM@host?5unreachable@ 0000000180047030     libcpmt:syserror.obj
 0002:00001048       ??_C@_0BD@JPHBMONG@identifier?5removed@ 0000000180047048     libcpmt:syserror.obj
 0002:00001060       ??_C@_0BG@CDNPAGJK@illegal?5byte?5sequence@ 0000000180047060     libcpmt:syserror.obj
 0002:00001078       ??_C@_0CD@BNPLBMNA@inappropriate?5io?5control?5operat@ 0000000180047078     libcpmt:syserror.obj
 0002:000010a0       ??_C@_0M@EGEKIIMP@interrupted@ 00000001800470a0     libcpmt:syserror.obj
 0002:000010b0       ??_C@_0BB@FCMFBGOM@invalid?5argument@ 00000001800470b0     libcpmt:syserror.obj
 0002:000010c8       ??_C@_0N@OHAFKDEK@invalid?5seek@ 00000001800470c8     libcpmt:syserror.obj
 0002:000010d8       ??_C@_08GLNPIFBN@io?5error@ 00000001800470d8     libcpmt:syserror.obj
 0002:000010e8       ??_C@_0P@FLLDBIDK@is?5a?5directory@ 00000001800470e8     libcpmt:syserror.obj
 0002:000010f8       ??_C@_0N@IFLPBIOP@message?5size@ 00000001800470f8     libcpmt:syserror.obj
 0002:00001108       ??_C@_0N@KIIEAAIO@network?5down@ 0000000180047108     libcpmt:syserror.obj
 0002:00001118       ??_C@_0O@FNPDBHEE@network?5reset@ 0000000180047118     libcpmt:syserror.obj
 0002:00001128       ??_C@_0BE@IFNCKGE@network?5unreachable@ 0000000180047128     libcpmt:syserror.obj
 0002:00001140       ??_C@_0BA@PFFCAOFK@no?5buffer?5space@ 0000000180047140     libcpmt:syserror.obj
 0002:00001150       ??_C@_0BB@IEPBLJHK@no?5child?5process@ 0000000180047150     libcpmt:syserror.obj
 0002:00001168       ??_C@_07PLECNNKG@no?5link@ 0000000180047168     libcpmt:syserror.obj
 0002:00001170       ??_C@_0BC@NJECKMKE@no?5lock?5available@ 0000000180047170     libcpmt:syserror.obj
 0002:00001188       ??_C@_0BF@PBGGPKKE@no?5message?5available@ 0000000180047188     libcpmt:syserror.obj
 0002:000011a0       ??_C@_0L@EDOLMPAK@no?5message@ 00000001800471a0     libcpmt:syserror.obj
 0002:000011b0       ??_C@_0BD@EAMBFIDF@no?5protocol?5option@ 00000001800471b0     libcpmt:syserror.obj
 0002:000011c8       ??_C@_0BD@IJDJKDEA@no?5space?5on?5device@ 00000001800471c8     libcpmt:syserror.obj
 0002:000011e0       ??_C@_0BE@MKFDAFMP@no?5stream?5resources@ 00000001800471e0     libcpmt:syserror.obj
 0002:000011f8       ??_C@_0BK@IMCPHCBI@no?5such?5device?5or?5address@ 00000001800471f8     libcpmt:syserror.obj
 0002:00001218       ??_C@_0P@FDINDDOK@no?5such?5device@ 0000000180047218     libcpmt:syserror.obj
 0002:00001228       ??_C@_0BK@NDOCBPGE@no?5such?5file?5or?5directory@ 0000000180047228     libcpmt:syserror.obj
 0002:00001248       ??_C@_0BA@ENLPPKBN@no?5such?5process@ 0000000180047248     libcpmt:syserror.obj
 0002:00001258       ??_C@_0BA@DOCPFFJG@not?5a?5directory@ 0000000180047258     libcpmt:syserror.obj
 0002:00001268       ??_C@_0N@POEIPGGF@not?5a?5socket@ 0000000180047268     libcpmt:syserror.obj
 0002:00001278       ??_C@_0N@LGAPMMPI@not?5a?5stream@ 0000000180047278     libcpmt:syserror.obj
 0002:00001288       ??_C@_0O@GLMIBBEG@not?5connected@ 0000000180047288     libcpmt:syserror.obj
 0002:00001298       ??_C@_0BC@ENOOLCNF@not?5enough?5memory@ 0000000180047298     libcpmt:syserror.obj
 0002:000012b0       ??_C@_0O@NHEDABJP@not?5supported@ 00000001800472b0     libcpmt:syserror.obj
 0002:000012c0       ??_C@_0BD@MOLBPMEA@operation?5canceled@ 00000001800472c0     libcpmt:syserror.obj
 0002:000012d8       ??_C@_0BG@KDKHOPCO@operation?5in?5progress@ 00000001800472d8     libcpmt:syserror.obj
 0002:000012f0       ??_C@_0BI@OHIEJAAB@operation?5not?5permitted@ 00000001800472f0     libcpmt:syserror.obj
 0002:00001308       ??_C@_0BI@LNEGIFLN@operation?5not?5supported@ 0000000180047308     libcpmt:syserror.obj
 0002:00001320       ??_C@_0BG@OEMDKMEE@operation?5would?5block@ 0000000180047320     libcpmt:syserror.obj
 0002:00001338       ??_C@_0L@BLPOFLNJ@owner?5dead@ 0000000180047338     libcpmt:syserror.obj
 0002:00001348       ??_C@_0BC@CIJDGCDI@permission?5denied@ 0000000180047348     libcpmt:syserror.obj
 0002:00001360       ??_C@_0P@FNPOCJBE@protocol?5error@ 0000000180047360     libcpmt:syserror.obj
 0002:00001370       ??_C@_0BH@JPPPLHJB@protocol?5not?5supported@ 0000000180047370     libcpmt:syserror.obj
 0002:00001388       ??_C@_0BG@EICBIHDP@read?5only?5file?5system@ 0000000180047388     libcpmt:syserror.obj
 0002:000013a0       ??_C@_0BO@BJBOMOEJ@resource?5deadlock?5would?5occur@ 00000001800473a0     libcpmt:syserror.obj
 0002:000013c0       ??_C@_0BP@LKNGHENJ@resource?5unavailable?5try?5again@ 00000001800473c0     libcpmt:syserror.obj
 0002:000013e0       ??_C@_0BE@GOIPJJHG@result?5out?5of?5range@ 00000001800473e0     libcpmt:syserror.obj
 0002:000013f8       ??_C@_0BG@MPLKFPAE@state?5not?5recoverable@ 00000001800473f8     libcpmt:syserror.obj
 0002:00001410       ??_C@_0P@DIIFGFCG@stream?5timeout@ 0000000180047410     libcpmt:syserror.obj
 0002:00001420       ??_C@_0P@IPFDMIFL@text?5file?5busy@ 0000000180047420     libcpmt:syserror.obj
 0002:00001430       ??_C@_09KJPPMAOI@timed?5out@ 0000000180047430     libcpmt:syserror.obj
 0002:00001440       ??_C@_0BO@HACHBEKI@too?5many?5files?5open?5in?5system@ 0000000180047440     libcpmt:syserror.obj
 0002:00001460       ??_C@_0BE@GHAFMPAH@too?5many?5files?5open@ 0000000180047460     libcpmt:syserror.obj
 0002:00001478       ??_C@_0P@HCOMKFCC@too?5many?5links@ 0000000180047478     libcpmt:syserror.obj
 0002:00001488       ??_C@_0BO@EFGOJEF@too?5many?5symbolic?5link?5levels@ 0000000180047488     libcpmt:syserror.obj
 0002:000014a8       ??_C@_0BA@KGKGOOJA@value?5too?5large@ 00000001800474a8     libcpmt:syserror.obj
 0002:000014b8       ??_C@_0BE@MIEJDDNH@wrong?5protocol?5type@ 00000001800474b8     libcpmt:syserror.obj
 0002:000014d8       ??_7bad_cast@std@@6B@      00000001800474d8     libcpmt:locale.obj
 0002:00001628       ??_7bad_array_new_length@std@@6B@ 0000000180047628     libcpmt:wlocale.obj
 0002:00001640       ??_7?$numpunct@_W@std@@6B@ 0000000180047640     libcpmt:wlocale.obj
 0002:00001680       ??_C@_13IMODFHAA@?$AA?9@   0000000180047680     libcpmt:wlocale.obj
 0002:00001684       ??_C@_01JOAMLHOP@?9@       0000000180047684     libcpmt:wlocale.obj
 0002:00001730       ??_7type_info@@6B@         0000000180047730     LIBCMT:std_type_info_static.obj
 0002:00001738       _pRawDllMain               0000000180047738     LIBCMT:dll_dllmain.obj
 0002:00001738       _pDefaultRawDllMain        0000000180047738     LIBCMT:dll_dllmain.obj
 0002:000017e8       _pDestructExceptionObject  00000001800477e8     libvcruntime:ehhelpers.obj
 0002:000017f8       ??_7bad_exception@std@@6B@ 00000001800477f8     libvcruntime:frame.obj
 0002:00001808       ??_C@_0O@DPKOEFFH@bad?5exception@ 0000000180047808     libvcruntime:frame.obj
 0002:00001f20       ??_C@_08EHJDFFNH@__based?$CI@ 0000000180047f20     libvcruntime:undname.obj
 0002:00001f30       ??_C@_07KOLFKCDI@__cdecl@  0000000180047f30     libvcruntime:undname.obj
 0002:00001f38       ??_C@_08GHMPAG@__pascal@   0000000180047f38     libvcruntime:undname.obj
 0002:00001f48       ??_C@_09IFJBGAPI@__stdcall@ 0000000180047f48     libvcruntime:undname.obj
 0002:00001f58       ??_C@_0L@NPHFGOKO@__thiscall@ 0000000180047f58     libvcruntime:undname.obj
 0002:00001f68       ??_C@_0L@JMKHOMEK@__fastcall@ 0000000180047f68     libvcruntime:undname.obj
 0002:00001f78       ??_C@_0N@BCKKPABJ@__vectorcall@ 0000000180047f78     libvcruntime:undname.obj
 0002:00001f88       ??_C@_09HIJEGCPM@__clrcall@ 0000000180047f88     libvcruntime:undname.obj
 0002:00001f94       ??_C@_06GHPCKEAG@__eabi@   0000000180047f94     libvcruntime:undname.obj
 0002:00001fa0       ??_C@_09IOPIDJLG@__swift_1@ 0000000180047fa0     libvcruntime:undname.obj
 0002:00001fb0       ??_C@_09KFNFGKHF@__swift_2@ 0000000180047fb0     libvcruntime:undname.obj
 0002:00001fc0       ??_C@_07JOMMBBKO@__ptr64@  0000000180047fc0     libvcruntime:undname.obj
 0002:00001fc8       ??_C@_0L@PILCLIHE@__restrict@ 0000000180047fc8     libvcruntime:undname.obj
 0002:00001fd8       ??_C@_0M@GFIIJFMG@__unaligned@ 0000000180047fd8     libvcruntime:undname.obj
 0002:00001fe8       ??_C@_09DHDLOLLB@restrict?$CI@ 0000000180047fe8     libvcruntime:undname.obj
 0002:00001ff4       ??_C@_04NIHEBCM@?5new@     0000000180047ff4     libvcruntime:undname.obj
 0002:00002000       ??_C@_07FPCDHGMM@?5delete@ 0000000180048000     libvcruntime:undname.obj
 0002:00002008       ??_C@_01NEMOKFLO@?$DN@     0000000180048008     libvcruntime:undname.obj
 0002:0000200c       ??_C@_02GPIOPFAK@?$DO?$DO@ 000000018004800c     libvcruntime:undname.obj
 0002:00002010       ??_C@_02FODMEDOG@?$DM?$DM@ 0000000180048010     libvcruntime:undname.obj
 0002:00002014       ??_C@_01DCLJPIOD@?$CB@     0000000180048014     libvcruntime:undname.obj
 0002:00002018       ??_C@_02EGOFBIJA@?$DN?$DN@ 0000000180048018     libvcruntime:undname.obj
 0002:0000201c       ??_C@_02FDNJECIE@?$CB?$DN@ 000000018004801c     libvcruntime:undname.obj
 0002:00002020       ??_C@_02GPECMEKF@?$FL?$FN@ 0000000180048020     libvcruntime:undname.obj
 0002:00002028       ??_C@_08LHJFAFGD@operator@ 0000000180048028     libvcruntime:undname.obj
 0002:00002034       ??_C@_02HBOOOICD@?9?$DO@   0000000180048034     libvcruntime:undname.obj
 0002:00002038       ??_C@_02ECNGHCIF@?$CL?$CL@ 0000000180048038     libvcruntime:undname.obj
 0002:0000203c       ??_C@_02BAABKJLB@?9?9@     000000018004803c     libvcruntime:undname.obj
 0002:00002040       ??_C@_01MIFGBAGJ@?$CL@     0000000180048040     libvcruntime:undname.obj
 0002:00002044       ??_C@_01HNPIGOCE@?$CG@     0000000180048044     libvcruntime:undname.obj
 0002:00002048       ??_C@_03MNHNFDLC@?9?$DO?$CK@ 0000000180048048     libvcruntime:undname.obj
 0002:0000204c       ??_C@_01KMDKNFGN@?1@       000000018004804c     libvcruntime:undname.obj
 0002:00002050       ??_C@_01FGNFDNOH@?$CF@     0000000180048050     libvcruntime:undname.obj
 0002:00002054       ??_C@_01MNNFJEPP@?$DM@     0000000180048054     libvcruntime:undname.obj
 0002:00002058       ??_C@_02EHCHHCKH@?$DM?$DN@ 0000000180048058     libvcruntime:undname.obj
 0002:0000205c       ??_C@_01PPODPGHN@?$DO@     000000018004805c     libvcruntime:undname.obj
 0002:00002060       ??_C@_02EEKDKGMJ@?$DO?$DN@ 0000000180048060     libvcruntime:undname.obj
 0002:00002064       ??_C@_01IHBHIGKO@?0@       0000000180048064     libvcruntime:undname.obj
 0002:00002068       ??_C@_02HCKGKOFO@?$CI?$CJ@ 0000000180048068     libvcruntime:undname.obj
 0002:0000206c       ??_C@_01PJKLJHI@?$HO@      000000018004806c     libvcruntime:undname.obj
 0002:00002070       ??_C@_01JKBOJNNK@?$FO@     0000000180048070     libvcruntime:undname.obj
 0002:00002074       ??_C@_01DNKMNLPK@?$HM@     0000000180048074     libvcruntime:undname.obj
 0002:00002078       ??_C@_02PPKAJPJL@?$CG?$CG@ 0000000180048078     libvcruntime:undname.obj
 0002:0000207c       ??_C@_02NONPIBCD@?$HM?$HM@ 000000018004807c     libvcruntime:undname.obj
 0002:00002080       ??_C@_02FPIMKNGF@?$CK?$DN@ 0000000180048080     libvcruntime:undname.obj
 0002:00002084       ??_C@_02FOEOMHFC@?$CL?$DN@ 0000000180048084     libvcruntime:undname.obj
 0002:00002088       ??_C@_02FKMDLLOA@?9?$DN@   0000000180048088     libvcruntime:undname.obj
 0002:0000208c       ??_C@_02FJEHGPIO@?1?$DN@   000000018004808c     libvcruntime:undname.obj
 0002:00002090       ??_C@_02FENAOKFI@?$CF?$DN@ 0000000180048090     libvcruntime:undname.obj
 0002:00002094       ??_C@_03IKFCCPFF@?$DO?$DO?$DN@ 0000000180048094     libvcruntime:undname.obj
 0002:00002098       ??_C@_03CDNPDDLA@?$DM?$DM?$DN@ 0000000180048098     libvcruntime:undname.obj
 0002:0000209c       ??_C@_02FGJGFEAB@?$CG?$DN@ 000000018004809c     libvcruntime:undname.obj
 0002:000020a0       ??_C@_02DHLNPPGH@?$HM?$DN@ 00000001800480a0     libvcruntime:undname.obj
 0002:000020a4       ??_C@_02MHEGNOJ@?$FO?$DN@  00000001800480a4     libvcruntime:undname.obj
 0002:000020a8       ??_C@_09IFPLHPGF@?$GAvftable?8@ 00000001800480a8     libvcruntime:undname.obj
 0002:000020b8       ??_C@_09BLBHBJP@?$GAvbtable?8@ 00000001800480b8     libvcruntime:undname.obj
 0002:000020c8       ??_C@_07FEEIOKP@?$GAvcall?8@ 00000001800480c8     libvcruntime:undname.obj
 0002:000020d0       ??_C@_08LLFFHHDJ@?$GAtypeof?8@ 00000001800480d0     libvcruntime:undname.obj
 0002:000020e0       ??_C@_0BF@KDPPACIK@?$GAlocal?5static?5guard?8@ 00000001800480e0     libvcruntime:undname.obj
 0002:000020f8       ??_C@_08OBABFOLI@?$GAstring?8@ 00000001800480f8     libvcruntime:undname.obj
 0002:00002108       ??_C@_0BD@JDLKDPAB@?$GAvbase?5destructor?8@ 0000000180048108     libvcruntime:undname.obj
 0002:00002120       ??_C@_0BN@DEGPLNFK@?$GAvector?5deleting?5destructor?8@ 0000000180048120     libvcruntime:undname.obj
 0002:00002140       ??_C@_0BO@OBMKPJIG@?$GAdefault?5constructor?5closure?8@ 0000000180048140     libvcruntime:undname.obj
 0002:00002160       ??_C@_0BN@IMDCHIKM@?$GAscalar?5deleting?5destructor?8@ 0000000180048160     libvcruntime:undname.obj
 0002:00002180       ??_C@_0BO@PFGOCPJJ@?$GAvector?5constructor?5iterator?8@ 0000000180048180     libvcruntime:undname.obj
 0002:000021a0       ??_C@_0BN@LFPFMEDL@?$GAvector?5destructor?5iterator?8@ 00000001800481a0     libvcruntime:undname.obj
 0002:000021c0       ??_C@_0CE@IKBNEHA@?$GAvector?5vbase?5constructor?5itera@ 00000001800481c0     libvcruntime:undname.obj
 0002:000021e8       ??_C@_0BL@NILFHHPC@?$GAvirtual?5displacement?5map?8@ 00000001800481e8     libvcruntime:undname.obj
 0002:00002208       ??_C@_0CB@JONCMFFK@?$GAeh?5vector?5constructor?5iterator@ 0000000180048208     libvcruntime:undname.obj
 0002:00002230       ??_C@_0CA@GCEOPDGL@?$GAeh?5vector?5destructor?5iterator?8@ 0000000180048230     libvcruntime:undname.obj
 0002:00002250       ??_C@_0CH@OOJPLCPH@?$GAeh?5vector?5vbase?5constructor?5it@ 0000000180048250     libvcruntime:undname.obj
 0002:00002278       ??_C@_0BL@LLKPOHJI@?$GAcopy?5constructor?5closure?8@ 0000000180048278     libvcruntime:undname.obj
 0002:00002298       ??_C@_0BA@KBCDOMBN@?$GAudt?5returning?8@ 0000000180048298     libvcruntime:undname.obj
 0002:000022a8       ??_C@_03KLGMFNMG@?$GAEH@   00000001800482a8     libvcruntime:undname.obj
 0002:000022ac       ??_C@_05KHLCHHI@?$GARTTI@  00000001800482ac     libvcruntime:undname.obj
 0002:000022b8       ??_C@_0BA@KKLDJDLB@?$GAlocal?5vftable?8@ 00000001800482b8     libvcruntime:undname.obj
 0002:000022c8       ??_C@_0CE@IIHCMGGL@?$GAlocal?5vftable?5constructor?5clos@ 00000001800482c8     libvcruntime:undname.obj
 0002:000022ec       ??_C@_06FHBGPFGH@?5new?$FL?$FN@ 00000001800482ec     libvcruntime:undname.obj
 0002:000022f8       ??_C@_09LBNFPBCA@?5delete?$FL?$FN@ 00000001800482f8     libvcruntime:undname.obj
 0002:00002308       ??_C@_0P@HJKNJFNN@?$GAomni?5callsig?8@ 0000000180048308     libvcruntime:undname.obj
 0002:00002318       ??_C@_0BL@CNOONJFP@?$GAplacement?5delete?5closure?8@ 0000000180048318     libvcruntime:undname.obj
 0002:00002338       ??_C@_0BN@CKNJLHMB@?$GAplacement?5delete?$FL?$FN?5closure?8@ 0000000180048338     libvcruntime:undname.obj
 0002:00002358       ??_C@_0CG@CFDHKGGD@?$GAmanaged?5vector?5constructor?5ite@ 0000000180048358     libvcruntime:undname.obj
 0002:00002380       ??_C@_0CF@IMGKMJNO@?$GAmanaged?5vector?5destructor?5iter@ 0000000180048380     libvcruntime:undname.obj
 0002:000023a8       ??_C@_0CG@HLDDJMAG@?$GAeh?5vector?5copy?5constructor?5ite@ 00000001800483a8     libvcruntime:undname.obj
 0002:000023d0       ??_C@_0CM@FCBBDIGB@?$GAeh?5vector?5vbase?5copy?5construct@ 00000001800483d0     libvcruntime:undname.obj
 0002:00002400       ??_C@_0BL@CLIPGLGB@?$GAdynamic?5initializer?5for?5?8@ 0000000180048400     libvcruntime:undname.obj
 0002:00002420       ??_C@_0CB@PDBIFEP@?$GAdynamic?5atexit?5destructor?5for?5@ 0000000180048420     libvcruntime:undname.obj
 0002:00002448       ??_C@_0CD@CGAJBKEJ@?$GAvector?5copy?5constructor?5iterat@ 0000000180048448     libvcruntime:undname.obj
 0002:00002470       ??_C@_0CJ@GJELGAMM@?$GAvector?5vbase?5copy?5constructor?5@ 0000000180048470     libvcruntime:undname.obj
 0002:000024a0       ??_C@_0CL@FGIJHLCE@?$GAmanaged?5vector?5copy?5constructo@ 00000001800484a0     libvcruntime:undname.obj
 0002:000024d0       ??_C@_0BM@PMGGMLDN@?$GAlocal?5static?5thread?5guard?8@ 00000001800484d0     libvcruntime:undname.obj
 0002:000024f0       ??_C@_0N@BDNMDMOL@operator?5?$CC?$CC?5@ 00000001800484f0     libvcruntime:undname.obj
 0002:00002500       ??_C@_0BC@GGEBGALA@operator?5co_await@ 0000000180048500     libvcruntime:undname.obj
 0002:00002518       ??_C@_0M@GAAIMMOH@operator?$DM?$DN?$DO@ 0000000180048518     libvcruntime:undname.obj
 0002:00002528       ??_C@_0BC@DAFEJGAK@?5Type?5Descriptor?8@ 0000000180048528     libvcruntime:undname.obj
 0002:00002540       ??_C@_0BM@LDKODKLH@?5Base?5Class?5Descriptor?5at?5?$CI@ 0000000180048540     libvcruntime:undname.obj
 0002:00002560       ??_C@_0BD@LGICGFMM@?5Base?5Class?5Array?8@ 0000000180048560     libvcruntime:undname.obj
 0002:00002578       ??_C@_0BN@MECKDCOJ@?5Class?5Hierarchy?5Descriptor?8@ 0000000180048578     libvcruntime:undname.obj
 0002:00002598       ??_C@_0BK@CFCOFLF@?5Complete?5Object?5Locator?8@ 0000000180048598     libvcruntime:undname.obj
 0002:000025b8       ??_C@_0BG@JNJLAMPM@?$GAanonymous?5namespace?8@ 00000001800485b8     libvcruntime:undname.obj
 0002:000025d0       format_validation_lookup_table 00000001800485d0     libucrt:output.obj
 0002:00002630       ??_C@_1O@CEDCILHN@?$AA?$CI?$AAn?$AAu?$AAl?$AAl?$AA?$CJ@ 0000000180048630     libucrt:output.obj
 0002:00002640       ??_C@_06OJHGLDPL@?$CInull?$CJ@ 0000000180048640     libucrt:output.obj
 0002:00002bd8       ??_C@_04KGLCPMCP@log2@     0000000180048bd8     libucrt:log2.obj
 0002:00002be0       __newctype                 0000000180048be0     libucrt:ctype.obj
 0002:00002ee0       __newclmap                 0000000180048ee0     libucrt:ctype.obj
 0002:00003060       __newcumap                 0000000180049060     libucrt:ctype.obj
 0002:000031e0       _wctype                    00000001800491e0     libucrt:ctype.obj
 0002:000033f0       ?large_power_data@?1??multiply_by_power_of_ten@__crt_strtox@@YA_NAEAUbig_integer@2@I@Z@4QBIB 00000001800493f0     libucrt:strtod.obj
 0002:00003cf8       ?small_powers_of_ten@?1??multiply_by_power_of_ten@__crt_strtox@@YA_NAEAUbig_integer@2@I@Z@4QBIB 0000000180049cf8     libucrt:strtod.obj
 0002:00003e10       __acrt_exception_action_table 0000000180049e10     libucrt:exception_filter.obj
 0002:00003ed0       __acrt_signal_action_table_count 0000000180049ed0     libucrt:exception_filter.obj
 0002:00003ed8       __acrt_signal_action_first_fpe_index 0000000180049ed8     libucrt:exception_filter.obj
 0002:00003ee0       __acrt_signal_action_fpe_count 0000000180049ee0     libucrt:exception_filter.obj
 0002:00003ee8       ??_C@_1BI@BGOHAHKC@?$AAm?$AAs?$AAc?$AAo?$AAr?$AAe?$AAe?$AA?4?$AAd?$AAl?$AAl@ 0000000180049ee8     libucrt:exit.obj
 0002:00003f00       ??_C@_0P@MIGLKIOC@CorExitProcess@ 0000000180049f00     libucrt:exit.obj
 0002:000040b0       ??_C@_1EA@JGEFHKEI@?$AAa?$AAp?$AAi?$AA?9?$AAm?$AAs?$AA?9?$AAw?$AAi?$AAn?$AA?9?$AAc?$AAo?$AAr?$AAe@ 000000018004a0b0     libucrt:winapi_thunks.obj
 0002:000040f0       ??_C@_1DM@KHCHBNEB@?$AAa?$AAp?$AAi?$AA?9?$AAm?$AAs?$AA?9?$AAw?$AAi?$AAn?$AA?9?$AAc?$AAo?$AAr?$AAe@ 000000018004a0f0     libucrt:winapi_thunks.obj
 0002:00004130       ??_C@_1DI@IJCEHOCB@?$AAa?$AAp?$AAi?$AA?9?$AAm?$AAs?$AA?9?$AAw?$AAi?$AAn?$AA?9?$AAc?$AAo?$AAr?$AAe@ 000000018004a130     libucrt:winapi_thunks.obj
 0002:00004170       ??_C@_1EI@MPIAOHOC@?$AAa?$AAp?$AAi?$AA?9?$AAm?$AAs?$AA?9?$AAw?$AAi?$AAn?$AA?9?$AAc?$AAo?$AAr?$AAe@ 000000018004a170     libucrt:winapi_thunks.obj
 0002:000041c0       ??_C@_1FK@FPHCKFIE@?$AAa?$AAp?$AAi?$AA?9?$AAm?$AAs?$AA?9?$AAw?$AAi?$AAn?$AA?9?$AAc?$AAo?$AAr?$AAe@ 000000018004a1c0     libucrt:winapi_thunks.obj
 0002:00004220       ??_C@_1EM@DILCGIIO@?$AAa?$AAp?$AAi?$AA?9?$AAm?$AAs?$AA?9?$AAw?$AAi?$AAn?$AA?9?$AAc?$AAo?$AAr?$AAe@ 000000018004a220     libucrt:winapi_thunks.obj
 0002:00004270       ??_C@_1DM@LNCGDDPN@?$AAa?$AAp?$AAi?$AA?9?$AAm?$AAs?$AA?9?$AAw?$AAi?$AAn?$AA?9?$AAc?$AAo?$AAr?$AAe@ 000000018004a270     libucrt:winapi_thunks.obj
 0002:000042b0       ??_C@_1DK@LPPGFMPP@?$AAa?$AAp?$AAi?$AA?9?$AAm?$AAs?$AA?9?$AAw?$AAi?$AAn?$AA?9?$AAc?$AAo?$AAr?$AAe@ 000000018004a2b0     libucrt:winapi_thunks.obj
 0002:000042f0       ??_C@_1DO@FPAPJEMD@?$AAa?$AAp?$AAi?$AA?9?$AAm?$AAs?$AA?9?$AAw?$AAi?$AAn?$AA?9?$AAc?$AAo?$AAr?$AAe@ 000000018004a2f0     libucrt:winapi_thunks.obj
 0002:00004330       ??_C@_1DK@NDHNAHIO@?$AAa?$AAp?$AAi?$AA?9?$AAm?$AAs?$AA?9?$AAw?$AAi?$AAn?$AA?9?$AAc?$AAo?$AAr?$AAe@ 000000018004a330     libucrt:winapi_thunks.obj
 0002:00004370       ??_C@_1DM@KGHDGBCM@?$AAa?$AAp?$AAi?$AA?9?$AAm?$AAs?$AA?9?$AAw?$AAi?$AAn?$AA?9?$AAc?$AAo?$AAr?$AAe@ 000000018004a370     libucrt:winapi_thunks.obj
 0002:000043b0       ??_C@_1EO@IJIOEFOH@?$AAa?$AAp?$AAi?$AA?9?$AAm?$AAs?$AA?9?$AAw?$AAi?$AAn?$AA?9?$AAr?$AAt?$AAc?$AAo@ 000000018004a3b0     libucrt:winapi_thunks.obj
 0002:00004400       ??_C@_1FG@HHGEKANL@?$AAa?$AAp?$AAi?$AA?9?$AAm?$AAs?$AA?9?$AAw?$AAi?$AAn?$AA?9?$AAs?$AAe?$AAc?$AAu@ 000000018004a400     libucrt:winapi_thunks.obj
 0002:00004460       ??_C@_1EG@DBIOJECG@?$AAe?$AAx?$AAt?$AA?9?$AAm?$AAs?$AA?9?$AAw?$AAi?$AAn?$AA?9?$AAn?$AAt?$AAu?$AAs@ 000000018004a460     libucrt:winapi_thunks.obj
 0002:000044b0       ??_C@_1EO@FIHMJCLF@?$AAe?$AAx?$AAt?$AA?9?$AAm?$AAs?$AA?9?$AAw?$AAi?$AAn?$AA?9?$AAn?$AAt?$AAu?$AAs@ 000000018004a4b0     libucrt:winapi_thunks.obj
 0002:00004500       ??_C@_1EG@DPGNFKGC@?$AAa?$AAp?$AAi?$AA?9?$AAm?$AAs?$AA?9?$AAw?$AAi?$AAn?$AA?9?$AAa?$AAp?$AAp?$AAm@ 000000018004a500     libucrt:winapi_thunks.obj
 0002:00004548       ??_C@_1BA@PFFKHIOG@?$AAa?$AAp?$AAi?$AA?9?$AAm?$AAs?$AA?9@ 000000018004a548     libucrt:winapi_thunks.obj
 0002:00004558       ??_C@_1BA@IAIFMGEF@?$AAe?$AAx?$AAt?$AA?9?$AAm?$AAs?$AA?9@ 000000018004a558     libucrt:winapi_thunks.obj
 0002:00004570       ??_C@_0BA@FHFNEAED@AreFileApisANSI@ 000000018004a570     libucrt:winapi_thunks.obj
 0002:00004588       ??_C@_0BA@IHGNDAEB@CompareStringEx@ 000000018004a588     libucrt:winapi_thunks.obj
 0002:000045a0       ??_C@_0BE@LJANKFHF@EnumSystemLocalesEx@ 000000018004a5a0     libucrt:winapi_thunks.obj
 0002:000045c0       ??_C@_08KNHFBNJ@FlsAlloc@  000000018004a5c0     libucrt:winapi_thunks.obj
 0002:000045d8       ??_C@_07PEJMOBNF@FlsFree@  000000018004a5d8     libucrt:winapi_thunks.obj
 0002:000045e8       ??_C@_0M@GDNOONDI@FlsGetValue@ 000000018004a5e8     libucrt:winapi_thunks.obj
 0002:00004600       ??_C@_0M@JCPCPOEF@FlsSetValue@ 000000018004a600     libucrt:winapi_thunks.obj
 0002:00004618       ??_C@_0BA@EPCJIIPD@GetDateFormatEx@ 000000018004a618     libucrt:winapi_thunks.obj
 0002:00004630       ??_C@_0BA@ONOKGCMP@GetLocaleInfoEx@ 000000018004a630     libucrt:winapi_thunks.obj
 0002:00004648       ??_C@_0BA@CIJJKCJJ@GetTimeFormatEx@ 000000018004a648     libucrt:winapi_thunks.obj
 0002:00004660       ??_C@_0BJ@PBCCBIPI@GetUserDefaultLocaleName@ 000000018004a660     libucrt:winapi_thunks.obj
 0002:00004688       ??_C@_0BM@HCFOFFN@InitializeCriticalSectionEx@ 000000018004a688     libucrt:winapi_thunks.obj
 0002:000046b0       ??_C@_0BC@CELBKLLA@IsValidLocaleName@ 000000018004a6b0     libucrt:winapi_thunks.obj
 0002:000046d0       ??_C@_0O@KKBNKAPF@LCMapStringEx@ 000000018004a6d0     libucrt:winapi_thunks.obj
 0002:000046e8       ??_C@_0BB@CDHDDLLP@LCIDToLocaleName@ 000000018004a6e8     libucrt:winapi_thunks.obj
 0002:00004708       ??_C@_0BB@HBDEELFH@LocaleNameToLCID@ 000000018004a708     libucrt:winapi_thunks.obj
 0002:00004720       ??_C@_0CF@OJOFEIGO@AppPolicyGetProcessTerminationM@ 000000018004a720     libucrt:winapi_thunks.obj
 0002:00004810       ??_C@_09OFJJIMPC@NAN?$CISNAN?$CJ@ 000000018004a810     libucrt:cvt.obj
 0002:00004820       ??_C@_09IPFBKMDL@nan?$CIsnan?$CJ@ 000000018004a820     libucrt:cvt.obj
 0002:00004830       ??_C@_08IKHNHAJ@NAN?$CIIND?$CJ@ 000000018004a830     libucrt:cvt.obj
 0002:00004840       ??_C@_08OFCDMILK@nan?$CIind?$CJ@ 000000018004a840     libucrt:cvt.obj
 0002:0000484c       ??_C@_05KLBDPFGC@e?$CL000@ 000000018004a84c     libucrt:cvt.obj
 0002:000048e0       __lc_category              000000018004a8e0     libucrt:wsetlocale.obj
 0002:00004970       ??_C@_1O@GIFLHMA@?$AAL?$AAC?$AA_?$AAA?$AAL?$AAL@ 000000018004a970     libucrt:wsetlocale.obj
 0002:00004980       ??_C@_1BG@PPOMIBNJ@?$AAL?$AAC?$AA_?$AAC?$AAO?$AAL?$AAL?$AAA?$AAT?$AAE@ 000000018004a980     libucrt:wsetlocale.obj
 0002:00004998       ??_C@_1BC@FFJGAPJM@?$AAL?$AAC?$AA_?$AAC?$AAT?$AAY?$AAP?$AAE@ 000000018004a998     libucrt:wsetlocale.obj
 0002:000049b0       ??_C@_1BI@PCKFNJFB@?$AAL?$AAC?$AA_?$AAM?$AAO?$AAN?$AAE?$AAT?$AAA?$AAR?$AAY@ 000000018004a9b0     libucrt:wsetlocale.obj
 0002:000049c8       ??_C@_1BG@ENIEDKID@?$AAL?$AAC?$AA_?$AAN?$AAU?$AAM?$AAE?$AAR?$AAI?$AAC@ 000000018004a9c8     libucrt:wsetlocale.obj
 0002:000049e0       ??_C@_1BA@HAAOMIIG@?$AAL?$AAC?$AA_?$AAT?$AAI?$AAM?$AAE@ 000000018004a9e0     libucrt:wsetlocale.obj
 0002:000049f0       ??_C@_15NBPDDFIP@?$AA?$DN?$AA?$DL@ 000000018004a9f0     libucrt:wsetlocale.obj
 0002:000049f8       ??_C@_13PJJBFPED@?$AA?$DL@ 000000018004a9f8     libucrt:wsetlocale.obj
 0002:000049fc       ??_C@_13NMPKAAJP@?$AA?$DN@ 000000018004a9fc     libucrt:wsetlocale.obj
 0002:00004a00       ??_C@_17EFJLDFDO@?$AA?9?$AA_?$AA?4@ 000000018004aa00     libucrt:wsetlocale.obj
 0002:00004a08       ??_C@_13FHBKNHDA@?$AAC@    000000018004aa08     libucrt:wsetlocale.obj
 0002:00004a10       ??_C@_17MBJJLFDM@?$AA_?$AA?4?$AA?0@ 000000018004aa10     libucrt:wsetlocale.obj
 0002:00004a18       ??_C@_13ENNFDPBH@?$AA_@    000000018004aa18     libucrt:wsetlocale.obj
 0002:00004a20       __lc_time_c                000000018004aa20     libucrt:nlsdata.obj
 0002:00004ce0       ??_C@_03KOEHGMDN@Sun@      000000018004ace0     libucrt:nlsdata.obj
 0002:00004ce4       ??_C@_03PDAGKDH@Mon@       000000018004ace4     libucrt:nlsdata.obj
 0002:00004ce8       ??_C@_03NAGEINEP@Tue@      000000018004ace8     libucrt:nlsdata.obj
 0002:00004cec       ??_C@_03MHOMLAJA@Wed@      000000018004acec     libucrt:nlsdata.obj
 0002:00004cf0       ??_C@_03IOFIKPDN@Thu@      000000018004acf0     libucrt:nlsdata.obj
 0002:00004cf4       ??_C@_03IDIOELNC@Fri@      000000018004acf4     libucrt:nlsdata.obj
 0002:00004cf8       ??_C@_03FEFJNEK@Sat@       000000018004acf8     libucrt:nlsdata.obj
 0002:00004cfc       ??_C@_06OOPIFAJ@Sunday@    000000018004acfc     libucrt:nlsdata.obj
 0002:00004d04       ??_C@_06JLEDEDGH@Monday@   000000018004ad04     libucrt:nlsdata.obj
 0002:00004d10       ??_C@_07BAAGCFCM@Tuesday@  000000018004ad10     libucrt:nlsdata.obj
 0002:00004d18       ??_C@_09DLIGFAKA@Wednesday@ 000000018004ad18     libucrt:nlsdata.obj
 0002:00004d28       ??_C@_08HACCIKIA@Thursday@ 000000018004ad28     libucrt:nlsdata.obj
 0002:00004d34       ??_C@_06JECMNKMI@Friday@   000000018004ad34     libucrt:nlsdata.obj
 0002:00004d40       ??_C@_08INBOOONO@Saturday@ 000000018004ad40     libucrt:nlsdata.obj
 0002:00004d4c       ??_C@_03JIHJHPIE@Jan@      000000018004ad4c     libucrt:nlsdata.obj
 0002:00004d50       ??_C@_03HJBDCHOM@Feb@      000000018004ad50     libucrt:nlsdata.obj
 0002:00004d54       ??_C@_03ODNJBKGA@Mar@      000000018004ad54     libucrt:nlsdata.obj
 0002:00004d58       ??_C@_03LEOLGMJP@Apr@      000000018004ad58     libucrt:nlsdata.obj
 0002:00004d5c       ??_C@_03CNMDKL@May@        000000018004ad5c     libucrt:nlsdata.obj
 0002:00004d60       ??_C@_03IDFGHECI@Jun@      000000018004ad60     libucrt:nlsdata.obj
 0002:00004d64       ??_C@_03LBGABGKK@Jul@      000000018004ad64     libucrt:nlsdata.obj
 0002:00004d68       ??_C@_03IFJFEIGA@Aug@      000000018004ad68     libucrt:nlsdata.obj
 0002:00004d6c       ??_C@_03GGCAPAJC@Sep@      000000018004ad6c     libucrt:nlsdata.obj
 0002:00004d70       ??_C@_03BMAOKBAD@Oct@      000000018004ad70     libucrt:nlsdata.obj
 0002:00004d74       ??_C@_03JPJOFNIA@Nov@      000000018004ad74     libucrt:nlsdata.obj
 0002:00004d78       ??_C@_03MKABNOCG@Dec@      000000018004ad78     libucrt:nlsdata.obj
 0002:00004d80       ??_C@_07CGJPFGJA@January@  000000018004ad80     libucrt:nlsdata.obj
 0002:00004d88       ??_C@_08GNJGEPFN@February@ 000000018004ad88     libucrt:nlsdata.obj
 0002:00004d94       ??_C@_05HPCKOFNC@March@    000000018004ad94     libucrt:nlsdata.obj
 0002:00004d9c       ??_C@_05DMJDNLEJ@April@    000000018004ad9c     libucrt:nlsdata.obj
 0002:00004da4       ??_C@_04CNLMGBGM@June@     000000018004ada4     libucrt:nlsdata.obj
 0002:00004dac       ??_C@_04MIEPOIFP@July@     000000018004adac     libucrt:nlsdata.obj
 0002:00004db4       ??_C@_06LBBHFDDG@August@   000000018004adb4     libucrt:nlsdata.obj
 0002:00004dc0       ??_C@_09BHHEALKD@September@ 000000018004adc0     libucrt:nlsdata.obj
 0002:00004dd0       ??_C@_07JJNFCEND@October@  000000018004add0     libucrt:nlsdata.obj
 0002:00004dd8       ??_C@_08HCHEGEOA@November@ 000000018004add8     libucrt:nlsdata.obj
 0002:00004de8       ??_C@_08EDHMEBNP@December@ 000000018004ade8     libucrt:nlsdata.obj
 0002:00004df4       ??_C@_02DEDBPAFC@AM@       000000018004adf4     libucrt:nlsdata.obj
 0002:00004df8       ??_C@_02CJNFDJBF@PM@       000000018004adf8     libucrt:nlsdata.obj
 0002:00004e00       ??_C@_08BPBNCDIB@MM?1dd?1yy@ 000000018004ae00     libucrt:nlsdata.obj
 0002:00004e10       ??_C@_0BE@CKGJFCPC@dddd?0?5MMMM?5dd?0?5yyyy@ 000000018004ae10     libucrt:nlsdata.obj
 0002:00004e28       ??_C@_08JCCMCCIL@HH?3mm?3ss@ 000000018004ae28     libucrt:nlsdata.obj
 0002:00004e38       ??_C@_17MBGCMIPB@?$AAS?$AAu?$AAn@ 000000018004ae38     libucrt:nlsdata.obj
 0002:00004e40       ??_C@_17KBOMKBF@?$AAM?$AAo?$AAn@ 000000018004ae40     libucrt:nlsdata.obj
 0002:00004e48       ??_C@_17BMKGEGOJ@?$AAT?$AAu?$AAe@ 000000018004ae48     libucrt:nlsdata.obj
 0002:00004e50       ??_C@_17CJEDCEPE@?$AAW?$AAe?$AAd@ 000000018004ae50     libucrt:nlsdata.obj
 0002:00004e58       ??_C@_17PDPHAADD@?$AAT?$AAh?$AAu@ 000000018004ae58     libucrt:nlsdata.obj
 0002:00004e60       ??_C@_17HFOLPPLP@?$AAF?$AAr?$AAi@ 000000018004ae60     libucrt:nlsdata.obj
 0002:00004e68       ??_C@_17GGIBDPIH@?$AAS?$AAa?$AAt@ 000000018004ae68     libucrt:nlsdata.obj
 0002:00004e70       ??_C@_1O@IHNHDHPB@?$AAS?$AAu?$AAn?$AAd?$AAa?$AAy@ 000000018004ae70     libucrt:nlsdata.obj
 0002:00004e80       ??_C@_1O@MMNBFLIA@?$AAM?$AAo?$AAn?$AAd?$AAa?$AAy@ 000000018004ae80     libucrt:nlsdata.obj
 0002:00004e90       ??_C@_1BA@ENFBFFEK@?$AAT?$AAu?$AAe?$AAs?$AAd?$AAa?$AAy@ 000000018004ae90     libucrt:nlsdata.obj
 0002:00004ea0       ??_C@_1BE@EBOGMDOH@?$AAW?$AAe?$AAd?$AAn?$AAe?$AAs?$AAd?$AAa?$AAy@ 000000018004aea0     libucrt:nlsdata.obj
 0002:00004eb8       ??_C@_1BC@HHMNLIHE@?$AAT?$AAh?$AAu?$AAr?$AAs?$AAd?$AAa?$AAy@ 000000018004aeb8     libucrt:nlsdata.obj
 0002:00004ed0       ??_C@_1O@PDICJHAG@?$AAF?$AAr?$AAi?$AAd?$AAa?$AAy@ 000000018004aed0     libucrt:nlsdata.obj
 0002:00004ee0       ??_C@_1BC@ENMNNPAJ@?$AAS?$AAa?$AAt?$AAu?$AAr?$AAd?$AAa?$AAy@ 000000018004aee0     libucrt:nlsdata.obj
 0002:00004ef8       ??_C@_17DKNBKCHM@?$AAJ?$AAa?$AAn@ 000000018004aef8     libucrt:nlsdata.obj
 0002:00004f00       ??_C@_17LMDJEKJN@?$AAF?$AAe?$AAb@ 000000018004af00     libucrt:nlsdata.obj
 0002:00004f08       ??_C@_17CKNLEDEC@?$AAM?$AAa?$AAr@ 000000018004af08     libucrt:nlsdata.obj
 0002:00004f10       ??_C@_17LFPOIHDD@?$AAA?$AAp?$AAr@ 000000018004af10     libucrt:nlsdata.obj
 0002:00004f18       ??_C@_17PNNKMEED@?$AAM?$AAa?$AAy@ 000000018004af18     libucrt:nlsdata.obj
 0002:00004f20       ??_C@_17KCJGOCPB@?$AAJ?$AAu?$AAn@ 000000018004af20     libucrt:nlsdata.obj
 0002:00004f28       ??_C@_17IJPCKHK@?$AAJ?$AAu?$AAl@ 000000018004af28     libucrt:nlsdata.obj
 0002:00004f30       ??_C@_17ICPELBCN@?$AAA?$AAu?$AAg@ 000000018004af30     libucrt:nlsdata.obj
 0002:00004f38       ??_C@_17HCHCOKMG@?$AAS?$AAe?$AAp@ 000000018004af38     libucrt:nlsdata.obj
 0002:00004f40       ??_C@_17FNLKOI@?$AAO?$AAc?$AAt@ 000000018004af40     libucrt:nlsdata.obj
 0002:00004f48       ??_C@_17BBDMLCIG@?$AAN?$AAo?$AAv@ 000000018004af48     libucrt:nlsdata.obj
 0002:00004f50       ??_C@_17EGKACKIF@?$AAD?$AAe?$AAc@ 000000018004af50     libucrt:nlsdata.obj
 0002:00004f58       ??_C@_1BA@EFMEIEBA@?$AAJ?$AAa?$AAn?$AAu?$AAa?$AAr?$AAy@ 000000018004af58     libucrt:nlsdata.obj
 0002:00004f68       ??_C@_1BC@JGDDFFAM@?$AAF?$AAe?$AAb?$AAr?$AAu?$AAa?$AAr?$AAy@ 000000018004af68     libucrt:nlsdata.obj
 0002:00004f80       ??_C@_1M@IKEENEDF@?$AAM?$AAa?$AAr?$AAc?$AAh@ 000000018004af80     libucrt:nlsdata.obj
 0002:00004f90       ??_C@_1M@GJNLMHFD@?$AAA?$AAp?$AAr?$AAi?$AAl@ 000000018004af90     libucrt:nlsdata.obj
 0002:00004fa0       ??_C@_19EPFLPGAP@?$AAJ?$AAu?$AAn?$AAe@ 000000018004afa0     libucrt:nlsdata.obj
 0002:00004fb0       ??_C@_19BIFMLPCD@?$AAJ?$AAu?$AAl?$AAy@ 000000018004afb0     libucrt:nlsdata.obj
 0002:00004fc0       ??_C@_1O@PAHLKOAC@?$AAA?$AAu?$AAg?$AAu?$AAs?$AAt@ 000000018004afc0     libucrt:nlsdata.obj
 0002:00004fd0       ??_C@_1BE@DKAAMBJL@?$AAS?$AAe?$AAp?$AAt?$AAe?$AAm?$AAb?$AAe?$AAr@ 000000018004afd0     libucrt:nlsdata.obj
 0002:00004fe8       ??_C@_1BA@EPANDLNG@?$AAO?$AAc?$AAt?$AAo?$AAb?$AAe?$AAr@ 000000018004afe8     libucrt:nlsdata.obj
 0002:00004ff8       ??_C@_1BC@BGLIFPF@?$AAN?$AAo?$AAv?$AAe?$AAm?$AAb?$AAe?$AAr@ 000000018004aff8     libucrt:nlsdata.obj
 0002:00005010       ??_C@_1BC@FEMKIFH@?$AAD?$AAe?$AAc?$AAe?$AAm?$AAb?$AAe?$AAr@ 000000018004b010     libucrt:nlsdata.obj
 0002:00005024       ??_C@_15ODEHAHHF@?$AAA?$AAM@ 000000018004b024     libucrt:nlsdata.obj
 0002:0000502c       ??_C@_15CLMNNGEL@?$AAP?$AAM@ 000000018004b02c     libucrt:nlsdata.obj
 0002:00005038       ??_C@_1BC@IEBCMHCM@?$AAM?$AAM?$AA?1?$AAd?$AAd?$AA?1?$AAy?$AAy@ 000000018004b038     libucrt:nlsdata.obj
 0002:00005050       ??_C@_1CI@KNAKOEBC@?$AAd?$AAd?$AAd?$AAd?$AA?0?$AA?5?$AAM?$AAM?$AAM?$AAM?$AA?5?$AAd?$AAd?$AA?0?$AA?5@ 000000018004b050     libucrt:nlsdata.obj
 0002:00005078       ??_C@_1BC@GDGBMEMK@?$AAH?$AAH?$AA?3?$AAm?$AAm?$AA?3?$AAs?$AAs@ 000000018004b078     libucrt:nlsdata.obj
 0002:00005090       ??_C@_1M@BMHNFIME@?$AAe?$AAn?$AA?9?$AAU?$AAS@ 000000018004b090     libucrt:nlsdata.obj
 0002:000052a0       ??_C@_03KHJOGHMM@exp@      000000018004b2a0     libucrt:fpexcept.obj
 0002:000052a4       ??_C@_03JGHBODFD@pow@      000000018004b2a4     libucrt:fpexcept.obj
 0002:000052a8       ??_C@_03MGHMBJCF@log@      000000018004b2a8     libucrt:fpexcept.obj
 0002:000052ac       ??_C@_05HGHHAHAP@log10@    000000018004b2ac     libucrt:fpexcept.obj
 0002:000052b4       ??_C@_04COOMCNPB@sinh@     000000018004b2b4     libucrt:fpexcept.obj
 0002:000052bc       ??_C@_04HPJJNFIM@cosh@     000000018004b2bc     libucrt:fpexcept.obj
 0002:000052c4       ??_C@_04FJHINJAO@tanh@     000000018004b2c4     libucrt:fpexcept.obj
 0002:000052cc       ??_C@_04FIHNOPOL@asin@     000000018004b2cc     libucrt:fpexcept.obj
 0002:000052d4       ??_C@_04PDIFKINK@acos@     000000018004b2d4     libucrt:fpexcept.obj
 0002:000052dc       ??_C@_04MLLJIGOK@atan@     000000018004b2dc     libucrt:fpexcept.obj
 0002:000052e4       ??_C@_05KNGEOGJB@atan2@    000000018004b2e4     libucrt:fpexcept.obj
 0002:000052ec       ??_C@_04EIAKFFMI@sqrt@     000000018004b2ec     libucrt:fpexcept.obj
 0002:000052f4       ??_C@_03BLEJJJBH@sin@      000000018004b2f4     libucrt:fpexcept.obj
 0002:000052f8       ??_C@_03LALBNOCG@cos@      000000018004b2f8     libucrt:fpexcept.obj
 0002:000052fc       ??_C@_03IIINPABG@tan@      000000018004b2fc     libucrt:fpexcept.obj
 0002:00005300       ??_C@_04GFPJNGEK@ceil@     000000018004b300     libucrt:fpexcept.obj
 0002:00005308       ??_C@_05PBJFFIGL@floor@    000000018004b308     libucrt:fpexcept.obj
 0002:00005310       ??_C@_04ODHECPBC@fabs@     000000018004b310     libucrt:fpexcept.obj
 0002:00005318       ??_C@_04EHEDPDJG@modf@     000000018004b318     libucrt:fpexcept.obj
 0002:00005320       ??_C@_05CEJMAHNP@ldexp@    000000018004b320     libucrt:fpexcept.obj
 0002:00005328       ??_C@_05KBKMEMPO@_cabs@    000000018004b328     libucrt:fpexcept.obj
 0002:00005330       ??_C@_06MEIMCGCF@_hypot@   000000018004b330     libucrt:fpexcept.obj
 0002:00005338       ??_C@_04KEPJIHGP@fmod@     000000018004b338     libucrt:fpexcept.obj
 0002:00005340       ??_C@_05GKKHEGJL@frexp@    000000018004b340     libucrt:fpexcept.obj
 0002:00005348       ??_C@_03MJLDFKDL@_y0@      000000018004b348     libucrt:fpexcept.obj
 0002:0000534c       ??_C@_03NAKIGLHK@_y1@      000000018004b34c     libucrt:fpexcept.obj
 0002:00005350       ??_C@_03ONILCKOB@_yn@      000000018004b350     libucrt:fpexcept.obj
 0002:00005354       ??_C@_05JGDBENOH@_logb@    000000018004b354     libucrt:fpexcept.obj
 0002:00005360       ??_C@_0L@KDOEJCKC@_nextafter@ 000000018004b360     libucrt:fpexcept.obj
 0002:00005370       _d_inf                     000000018004b370     libucrt:util.obj
 0002:00005378       _d_ind                     000000018004b378     libucrt:util.obj
 0002:00005380       _d_max                     000000018004b380     libucrt:util.obj
 0002:00005388       _d_mzero                   000000018004b388     libucrt:util.obj
 0002:000057a8       ??_C@_1M@HPNHIDJI@?$AAj?$AAa?$AA?9?$AAJ?$AAP@ 000000018004b7a8     libucrt:mbctype.obj
 0002:000057b8       ??_C@_1M@BIBDDEMK@?$AAz?$AAh?$AA?9?$AAC?$AAN@ 000000018004b7b8     libucrt:mbctype.obj
 0002:000057c8       ??_C@_1M@JLOOOEGK@?$AAk?$AAo?$AA?9?$AAK?$AAR@ 000000018004b7c8     libucrt:mbctype.obj
 0002:000057d8       ??_C@_1M@CLNBBOPM@?$AAz?$AAh?$AA?9?$AAT?$AAW@ 000000018004b7d8     libucrt:mbctype.obj
 0002:00006630       ??_C@_15EMKDOKLE@?$AAa?$AAr@ 000000018004c630     libucrt:lcidtoname_downlevel.obj
 0002:00006638       ??_C@_15KNPADPLH@?$AAb?$AAg@ 000000018004c638     libucrt:lcidtoname_downlevel.obj
 0002:00006640       ??_C@_15EDMHLDMO@?$AAc?$AAa@ 000000018004c640     libucrt:lcidtoname_downlevel.obj
 0002:00006648       ??_C@_1O@BPEAJADD@?$AAz?$AAh?$AA?9?$AAC?$AAH?$AAS@ 000000018004c648     libucrt:lcidtoname_downlevel.obj
 0002:00006658       ??_C@_15LJNHCMNK@?$AAc?$AAs@ 000000018004c658     libucrt:lcidtoname_downlevel.obj
 0002:00006660       ??_C@_15FOMCIDHG@?$AAd?$AAa@ 000000018004c660     libucrt:lcidtoname_downlevel.obj
 0002:00006668       ??_C@_15NBKABECB@?$AAd?$AAe@ 000000018004c668     libucrt:lcidtoname_downlevel.obj
 0002:00006670       ??_C@_15GHPEIIAO@?$AAe?$AAl@ 000000018004c670     libucrt:lcidtoname_downlevel.obj
 0002:00006678       ??_C@_15MNPNEAIF@?$AAe?$AAn@ 000000018004c678     libucrt:lcidtoname_downlevel.obj
 0002:00006680       ??_C@_15GPIOMPMH@?$AAe?$AAs@ 000000018004c680     libucrt:lcidtoname_downlevel.obj
 0002:00006688       ??_C@_15NGLOAKJC@?$AAf?$AAi@ 000000018004c688     libucrt:lcidtoname_downlevel.obj
 0002:00006690       ??_C@_15FBKGNKAM@?$AAf?$AAr@ 000000018004c690     libucrt:lcidtoname_downlevel.obj
 0002:00006698       ??_C@_15KGGCNEFK@?$AAh?$AAe@ 000000018004c698     libucrt:lcidtoname_downlevel.obj
 0002:000066a0       ??_C@_15PGHLIDMF@?$AAh?$AAu@ 000000018004c6a0     libucrt:lcidtoname_downlevel.obj
 0002:000066a8       ??_C@_15BIEMAPLM@?$AAi?$AAs@ 000000018004c6a8     libucrt:lcidtoname_downlevel.obj
 0002:000066b0       ??_C@_15IFJLDHAF@?$AAi?$AAt@ 000000018004c6b0     libucrt:lcidtoname_downlevel.obj
 0002:000066b8       ??_C@_15GEMIOCAG@?$AAj?$AAa@ 000000018004c6b8     libucrt:lcidtoname_downlevel.obj
 0002:000066c0       ??_C@_15EPELEGJA@?$AAk?$AAo@ 000000018004c6c0     libucrt:lcidtoname_downlevel.obj
 0002:000066c8       ??_C@_15NDDHIMN@?$AAn?$AAl@ 000000018004c6c8     libucrt:lcidtoname_downlevel.obj
 0002:000066d0       ??_C@_15BPIGNHCD@?$AAn?$AAo@ 000000018004c6d0     libucrt:lcidtoname_downlevel.obj
 0002:000066d8       ??_C@_15DEOPBLCG@?$AAp?$AAl@ 000000018004c6d8     libucrt:lcidtoname_downlevel.obj
 0002:000066e0       ??_C@_15KBECGEFG@?$AAp?$AAt@ 000000018004c6e0     libucrt:lcidtoname_downlevel.obj
 0002:000066e8       ??_C@_15GLJCBFMD@?$AAr?$AAo@ 000000018004c6e8     libucrt:lcidtoname_downlevel.obj
 0002:000066f0       ??_C@_15FEDGKCDI@?$AAr?$AAu@ 000000018004c6f0     libucrt:lcidtoname_downlevel.obj
 0002:000066f8       ??_C@_15GLKMLLHM@?$AAh?$AAr@ 000000018004c6f8     libucrt:lcidtoname_downlevel.obj
 0002:00006700       ??_C@_15CPKMFBDB@?$AAs?$AAk@ 000000018004c700     libucrt:lcidtoname_downlevel.obj
 0002:00006708       ??_C@_15BAAIOGMK@?$AAs?$AAq@ 000000018004c708     libucrt:lcidtoname_downlevel.obj
 0002:00006710       ??_C@_15INNPNOHD@?$AAs?$AAv@ 000000018004c710     libucrt:lcidtoname_downlevel.obj
 0002:00006718       ??_C@_15CABMMOGH@?$AAt?$AAh@ 000000018004c718     libucrt:lcidtoname_downlevel.obj
 0002:00006720       ??_C@_15BPLIHJJM@?$AAt?$AAr@ 000000018004c720     libucrt:lcidtoname_downlevel.obj
 0002:00006728       ??_C@_15NEOEKKDJ@?$AAu?$AAr@ 000000018004c728     libucrt:lcidtoname_downlevel.obj
 0002:00006730       ??_C@_15NFICGAJK@?$AAi?$AAd@ 000000018004c730     libucrt:lcidtoname_downlevel.obj
 0002:00006738       ??_C@_15PJPFLCCM@?$AAu?$AAk@ 000000018004c738     libucrt:lcidtoname_downlevel.obj
 0002:00006740       ??_C@_15HPJPHDM@?$AAb?$AAe@ 000000018004c740     libucrt:lcidtoname_downlevel.obj
 0002:00006748       ??_C@_15LCHLGJII@?$AAs?$AAl@ 000000018004c748     libucrt:lcidtoname_downlevel.obj
 0002:00006750       ??_C@_15PCFJPHHO@?$AAe?$AAt@ 000000018004c750     libucrt:lcidtoname_downlevel.obj
 0002:00006758       ??_C@_15HPFPGODN@?$AAl?$AAv@ 000000018004c758     libucrt:lcidtoname_downlevel.obj
 0002:00006760       ??_C@_15NFFGKGLG@?$AAl?$AAt@ 000000018004c760     libucrt:lcidtoname_downlevel.obj
 0002:00006768       ??_C@_15BDAKCCHN@?$AAf?$AAa@ 000000018004c768     libucrt:lcidtoname_downlevel.obj
 0002:00006770       ??_C@_15NFGIAIAJ@?$AAv?$AAi@ 000000018004c770     libucrt:lcidtoname_downlevel.obj
 0002:00006778       ??_C@_15LMKNDMHN@?$AAh?$AAy@ 000000018004c778     libucrt:lcidtoname_downlevel.obj
 0002:00006780       ??_C@_15IJBHMCFL@?$AAa?$AAz@ 000000018004c780     libucrt:lcidtoname_downlevel.obj
 0002:00006788       ??_C@_15EKOFJABL@?$AAe?$AAu@ 000000018004c788     libucrt:lcidtoname_downlevel.obj
 0002:00006790       ??_C@_15BGHADCNK@?$AAm?$AAk@ 000000018004c790     libucrt:lcidtoname_downlevel.obj
 0002:00006798       ??_C@_15JDNICKHM@?$AAa?$AAf@ 000000018004c798     libucrt:lcidtoname_downlevel.obj
 0002:000067a0       ??_C@_15KPJEDBKD@?$AAk?$AAa@ 000000018004c7a0     libucrt:lcidtoname_downlevel.obj
 0002:000067a8       ??_C@_15PDNFFFEO@?$AAf?$AAo@ 000000018004c7a8     libucrt:lcidtoname_downlevel.obj
 0002:000067b0       ??_C@_15OMLEGLOC@?$AAh?$AAi@ 000000018004c7b0     libucrt:lcidtoname_downlevel.obj
 0002:000067b8       ??_C@_15IDNNENKK@?$AAm?$AAs@ 000000018004c7b8     libucrt:lcidtoname_downlevel.obj
 0002:000067c0       ??_C@_15MACJNBMH@?$AAk?$AAk@ 000000018004c7c0     libucrt:lcidtoname_downlevel.obj
 0002:000067c8       ??_C@_15DKDJEOND@?$AAk?$AAy@ 000000018004c7c8     libucrt:lcidtoname_downlevel.obj
 0002:000067d0       ??_C@_15DFGDLJBG@?$AAs?$AAw@ 000000018004c7d0     libucrt:lcidtoname_downlevel.obj
 0002:000067d8       ??_C@_15BBFAICNG@?$AAu?$AAz@ 000000018004c7d8     libucrt:lcidtoname_downlevel.obj
 0002:000067e0       ??_C@_15DKNDCGEA@?$AAt?$AAt@ 000000018004c7e0     libucrt:lcidtoname_downlevel.obj
 0002:000067e8       ??_C@_15MGIFMDPL@?$AAp?$AAa@ 000000018004c7e8     libucrt:lcidtoname_downlevel.obj
 0002:000067f0       ??_C@_15HCNDBBA@?$AAg?$AAu@ 000000018004c7f0     libucrt:lcidtoname_downlevel.obj
 0002:000067f8       ??_C@_15FNBEIBON@?$AAt?$AAa@ 000000018004c7f8     libucrt:lcidtoname_downlevel.obj
 0002:00006800       ??_C@_15NCHGBGLK@?$AAt?$AAe@ 000000018004c800     libucrt:lcidtoname_downlevel.obj
 0002:00006808       ??_C@_15PHPHCBPF@?$AAk?$AAn@ 000000018004c808     libucrt:lcidtoname_downlevel.obj
 0002:00006810       ??_C@_15DLGBCKMP@?$AAm?$AAr@ 000000018004c810     libucrt:lcidtoname_downlevel.obj
 0002:00006818       ??_C@_15EABBLBFF@?$AAs?$AAa@ 000000018004c818     libucrt:lcidtoname_downlevel.obj
 0002:00006820       ??_C@_15CBKOMCOI@?$AAm?$AAn@ 000000018004c820     libucrt:lcidtoname_downlevel.obj
 0002:00006828       ??_C@_15CKDMCJAF@?$AAg?$AAl@ 000000018004c828     libucrt:lcidtoname_downlevel.obj
 0002:00006830       ??_C@_17CNJFBPG@?$AAk?$AAo?$AAk@ 000000018004c830     libucrt:lcidtoname_downlevel.obj
 0002:00006838       ??_C@_17FFBJICPL@?$AAs?$AAy?$AAr@ 000000018004c838     libucrt:lcidtoname_downlevel.obj
 0002:00006840       ??_C@_17KPNDCPAF@?$AAd?$AAi?$AAv@ 000000018004c840     libucrt:lcidtoname_downlevel.obj
 0002:00006848       ??_C@_1M@OKAHONE@?$AAa?$AAr?$AA?9?$AAS?$AAA@ 000000018004c848     libucrt:lcidtoname_downlevel.obj
 0002:00006858       ??_C@_1M@FFFIGIGK@?$AAb?$AAg?$AA?9?$AAB?$AAG@ 000000018004c858     libucrt:lcidtoname_downlevel.obj
 0002:00006868       ??_C@_1M@BJNKEDC@?$AAc?$AAa?$AA?9?$AAE?$AAS@ 000000018004c868     libucrt:lcidtoname_downlevel.obj
 0002:00006878       ??_C@_1M@IJJHFJHA@?$AAc?$AAs?$AA?9?$AAC?$AAZ@ 000000018004c878     libucrt:lcidtoname_downlevel.obj
 0002:00006888       ??_C@_1M@CLPEOBGI@?$AAd?$AAa?$AA?9?$AAD?$AAK@ 000000018004c888     libucrt:lcidtoname_downlevel.obj
 0002:00006898       ??_C@_1M@MCMADGCB@?$AAd?$AAe?$AA?9?$AAD?$AAE@ 000000018004c898     libucrt:lcidtoname_downlevel.obj
 0002:000068a8       ??_C@_1M@OOCKEMAM@?$AAe?$AAl?$AA?9?$AAG?$AAR@ 000000018004c8a8     libucrt:lcidtoname_downlevel.obj
 0002:000068b8       ??_C@_1M@DDNJFGID@?$AAf?$AAi?$AA?9?$AAF?$AAI@ 000000018004c8b8     libucrt:lcidtoname_downlevel.obj
 0002:000068c8       ??_C@_1M@GLIPPMAC@?$AAf?$AAr?$AA?9?$AAF?$AAR@ 000000018004c8c8     libucrt:lcidtoname_downlevel.obj
 0002:000068d8       ??_C@_1M@GFMCHPE@?$AAh?$AAe?$AA?9?$AAI?$AAL@ 000000018004c8d8     libucrt:lcidtoname_downlevel.obj
 0002:000068e8       ??_C@_1M@MHLPGNKM@?$AAh?$AAu?$AA?9?$AAH?$AAU@ 000000018004c8e8     libucrt:lcidtoname_downlevel.obj
 0002:000068f8       ??_C@_1M@LPDDNNPN@?$AAi?$AAs?$AA?9?$AAI?$AAS@ 000000018004c8f8     libucrt:lcidtoname_downlevel.obj
 0002:00006908       ??_C@_1M@MADIPODN@?$AAi?$AAt?$AA?9?$AAI?$AAT@ 000000018004c908     libucrt:lcidtoname_downlevel.obj
 0002:00006918       ??_C@_1M@IHBJJGG@?$AAn?$AAl?$AA?9?$AAN?$AAL@ 000000018004c918     libucrt:lcidtoname_downlevel.obj
 0002:00006928       ??_C@_1M@EANAGDL@?$AAn?$AAb?$AA?9?$AAN?$AAO@ 000000018004c928     libucrt:lcidtoname_downlevel.obj
 0002:00006938       ??_C@_1M@NEIEMEGP@?$AAp?$AAl?$AA?9?$AAP?$AAL@ 000000018004c938     libucrt:lcidtoname_downlevel.obj
 0002:00006948       ??_C@_1M@BOCFIGEP@?$AAp?$AAt?$AA?9?$AAB?$AAR@ 000000018004c948     libucrt:lcidtoname_downlevel.obj
 0002:00006958       ??_C@_1M@IMPFOPBG@?$AAr?$AAo?$AA?9?$AAR?$AAO@ 000000018004c958     libucrt:lcidtoname_downlevel.obj
 0002:00006968       ??_C@_1M@IDNNEJMM@?$AAr?$AAu?$AA?9?$AAR?$AAU@ 000000018004c968     libucrt:lcidtoname_downlevel.obj
 0002:00006978       ??_C@_1M@LILEEOGM@?$AAh?$AAr?$AA?9?$AAH?$AAR@ 000000018004c978     libucrt:lcidtoname_downlevel.obj
 0002:00006988       ??_C@_1M@FKIFEHPB@?$AAs?$AAk?$AA?9?$AAS?$AAK@ 000000018004c988     libucrt:lcidtoname_downlevel.obj
 0002:00006998       ??_C@_1M@LJMAMNPJ@?$AAs?$AAq?$AA?9?$AAA?$AAL@ 000000018004c998     libucrt:lcidtoname_downlevel.obj
 0002:000069a8       ??_C@_1M@GIAKDKJK@?$AAs?$AAv?$AA?9?$AAS?$AAE@ 000000018004c9a8     libucrt:lcidtoname_downlevel.obj
 0002:000069b8       ??_C@_1M@MKJKIKCL@?$AAt?$AAh?$AA?9?$AAT?$AAH@ 000000018004c9b8     libucrt:lcidtoname_downlevel.obj
 0002:000069c8       ??_C@_1M@MFLCCMPB@?$AAt?$AAr?$AA?9?$AAT?$AAR@ 000000018004c9c8     libucrt:lcidtoname_downlevel.obj
 0002:000069d8       ??_C@_1M@OIJHDKJN@?$AAu?$AAr?$AA?9?$AAP?$AAK@ 000000018004c9d8     libucrt:lcidtoname_downlevel.obj
 0002:000069e8       ??_C@_1M@LHIPCIEK@?$AAi?$AAd?$AA?9?$AAI?$AAD@ 000000018004c9e8     libucrt:lcidtoname_downlevel.obj
 0002:000069f8       ??_C@_1M@MFMOBGI@?$AAu?$AAk?$AA?9?$AAU?$AAA@ 000000018004c9f8     libucrt:lcidtoname_downlevel.obj
 0002:00006a08       ??_C@_1M@OBGLJIPL@?$AAb?$AAe?$AA?9?$AAB?$AAY@ 000000018004ca08     libucrt:lcidtoname_downlevel.obj
 0002:00006a18       ??_C@_1M@BCFAJEAD@?$AAs?$AAl?$AA?9?$AAS?$AAI@ 000000018004ca18     libucrt:lcidtoname_downlevel.obj
 0002:00006a28       ??_C@_1M@FKFFEDDN@?$AAe?$AAt?$AA?9?$AAE?$AAE@ 000000018004ca28     libucrt:lcidtoname_downlevel.obj
 0002:00006a38       ??_C@_1M@KGKKAACI@?$AAl?$AAv?$AA?9?$AAL?$AAV@ 000000018004ca38     libucrt:lcidtoname_downlevel.obj
 0002:00006a48       ??_C@_1M@IFGBIJO@?$AAl?$AAt?$AA?9?$AAL?$AAT@ 000000018004ca48     libucrt:lcidtoname_downlevel.obj
 0002:00006a58       ??_C@_1M@FGEAHEDM@?$AAf?$AAa?$AA?9?$AAI?$AAR@ 000000018004ca58     libucrt:lcidtoname_downlevel.obj
 0002:00006a68       ??_C@_1M@KBMAIBFN@?$AAv?$AAi?$AA?9?$AAV?$AAN@ 000000018004ca68     libucrt:lcidtoname_downlevel.obj
 0002:00006a78       ??_C@_1M@GPCBKDJK@?$AAh?$AAy?$AA?9?$AAA?$AAM@ 000000018004ca78     libucrt:lcidtoname_downlevel.obj
 0002:00006a88       ??_C@_1BG@BECMDDJB@?$AAa?$AAz?$AA?9?$AAA?$AAZ?$AA?9?$AAL?$AAa?$AAt?$AAn@ 000000018004ca88     libucrt:lcidtoname_downlevel.obj
 0002:00006aa0       ??_C@_1M@MAOFCAEA@?$AAe?$AAu?$AA?9?$AAE?$AAS@ 000000018004caa0     libucrt:lcidtoname_downlevel.obj
 0002:00006ab0       ??_C@_1M@IGHABKPI@?$AAm?$AAk?$AA?9?$AAM?$AAK@ 000000018004cab0     libucrt:lcidtoname_downlevel.obj
 0002:00006ac0       ??_C@_1M@IAIGNEJG@?$AAt?$AAn?$AA?9?$AAZ?$AAA@ 000000018004cac0     libucrt:lcidtoname_downlevel.obj
 0002:00006ad0       ??_C@_1M@IIJCOJFA@?$AAx?$AAh?$AA?9?$AAZ?$AAA@ 000000018004cad0     libucrt:lcidtoname_downlevel.obj
 0002:00006ae0       ??_C@_1M@LGPJHNJH@?$AAz?$AAu?$AA?9?$AAZ?$AAA@ 000000018004cae0     libucrt:lcidtoname_downlevel.obj
 0002:00006af0       ??_C@_1M@HOKAOIO@?$AAa?$AAf?$AA?9?$AAZ?$AAA@ 000000018004caf0     libucrt:lcidtoname_downlevel.obj
 0002:00006b00       ??_C@_1M@DPCLHLIE@?$AAk?$AAa?$AA?9?$AAG?$AAE@ 000000018004cb00     libucrt:lcidtoname_downlevel.obj
 0002:00006b10       ??_C@_1M@BLKMHJBI@?$AAf?$AAo?$AA?9?$AAF?$AAO@ 000000018004cb10     libucrt:lcidtoname_downlevel.obj
 0002:00006b20       ??_C@_1M@LGGJAPPB@?$AAh?$AAi?$AA?9?$AAI?$AAN@ 000000018004cb20     libucrt:lcidtoname_downlevel.obj
 0002:00006b30       ??_C@_1M@FIKPIHFE@?$AAm?$AAt?$AA?9?$AAM?$AAT@ 000000018004cb30     libucrt:lcidtoname_downlevel.obj
 0002:00006b40       ??_C@_1M@HEGGPBFA@?$AAs?$AAe?$AA?9?$AAN?$AAO@ 000000018004cb40     libucrt:lcidtoname_downlevel.obj
 0002:00006b50       ??_C@_1M@EIBJEEPA@?$AAm?$AAs?$AA?9?$AAM?$AAY@ 000000018004cb50     libucrt:lcidtoname_downlevel.obj
 0002:00006b60       ??_C@_1M@FHLBGMPP@?$AAk?$AAk?$AA?9?$AAK?$AAZ@ 000000018004cb60     libucrt:lcidtoname_downlevel.obj
 0002:00006b70       ??_C@_1M@NGJJLCGI@?$AAk?$AAy?$AA?9?$AAK?$AAG@ 000000018004cb70     libucrt:lcidtoname_downlevel.obj
 0002:00006b80       ??_C@_1M@GIENNBFC@?$AAs?$AAw?$AA?9?$AAK?$AAE@ 000000018004cb80     libucrt:lcidtoname_downlevel.obj
 0002:00006b90       ??_C@_1BG@NDGMJIMJ@?$AAu?$AAz?$AA?9?$AAU?$AAZ?$AA?9?$AAL?$AAa?$AAt?$AAn@ 000000018004cb90     libucrt:lcidtoname_downlevel.obj
 0002:00006ba8       ??_C@_1M@IDCCIHBC@?$AAt?$AAt?$AA?9?$AAR?$AAU@ 000000018004cba8     libucrt:lcidtoname_downlevel.obj
 0002:00006bb8       ??_C@_1M@LOICPMOJ@?$AAb?$AAn?$AA?9?$AAI?$AAN@ 000000018004cbb8     libucrt:lcidtoname_downlevel.obj
 0002:00006bc8       ??_C@_1M@KPKKNEAH@?$AAp?$AAa?$AA?9?$AAI?$AAN@ 000000018004cbc8     libucrt:lcidtoname_downlevel.obj
 0002:00006bd8       ??_C@_1M@PJGPPBOG@?$AAg?$AAu?$AA?9?$AAI?$AAN@ 000000018004cbd8     libucrt:lcidtoname_downlevel.obj
 0002:00006be8       ??_C@_1M@KMKMOPHI@?$AAt?$AAa?$AA?9?$AAI?$AAN@ 000000018004cbe8     libucrt:lcidtoname_downlevel.obj
 0002:00006bf8       ??_C@_1M@KFEHEPAC@?$AAt?$AAe?$AA?9?$AAI?$AAN@ 000000018004cbf8     libucrt:lcidtoname_downlevel.obj
 0002:00006c08       ??_C@_1M@CDCLMGHI@?$AAk?$AAn?$AA?9?$AAI?$AAN@ 000000018004cc08     libucrt:lcidtoname_downlevel.obj
 0002:00006c18       ??_C@_1M@MIODLDKF@?$AAm?$AAl?$AA?9?$AAI?$AAN@ 000000018004cc18     libucrt:lcidtoname_downlevel.obj
 0002:00006c28       ??_C@_1M@PBIEACPO@?$AAm?$AAr?$AA?9?$AAI?$AAN@ 000000018004cc28     libucrt:lcidtoname_downlevel.obj
 0002:00006c38       ??_C@_1M@NIDEAGPH@?$AAs?$AAa?$AA?9?$AAI?$AAN@ 000000018004cc38     libucrt:lcidtoname_downlevel.obj
 0002:00006c48       ??_C@_1M@FHIHCBIO@?$AAm?$AAn?$AA?9?$AAM?$AAN@ 000000018004cc48     libucrt:lcidtoname_downlevel.obj
 0002:00006c58       ??_C@_1M@JAIJPENP@?$AAc?$AAy?$AA?9?$AAG?$AAB@ 000000018004cc58     libucrt:lcidtoname_downlevel.obj
 0002:00006c68       ??_C@_1M@PHGFBEPN@?$AAg?$AAl?$AA?9?$AAE?$AAS@ 000000018004cc68     libucrt:lcidtoname_downlevel.obj
 0002:00006c78       ??_C@_1O@KPIPDNCP@?$AAk?$AAo?$AAk?$AA?9?$AAI?$AAN@ 000000018004cc78     libucrt:lcidtoname_downlevel.obj
 0002:00006c88       ??_C@_1O@KNHJLDJA@?$AAs?$AAy?$AAr?$AA?9?$AAS?$AAY@ 000000018004cc88     libucrt:lcidtoname_downlevel.obj
 0002:00006c98       ??_C@_1O@MKEKBLAH@?$AAd?$AAi?$AAv?$AA?9?$AAM?$AAV@ 000000018004cc98     libucrt:lcidtoname_downlevel.obj
 0002:00006ca8       ??_C@_1O@OHDCKDDF@?$AAq?$AAu?$AAz?$AA?9?$AAB?$AAO@ 000000018004cca8     libucrt:lcidtoname_downlevel.obj
 0002:00006cb8       ??_C@_1M@LEPJNLFD@?$AAn?$AAs?$AA?9?$AAZ?$AAA@ 000000018004ccb8     libucrt:lcidtoname_downlevel.obj
 0002:00006cc8       ??_C@_1M@OMLEIIJB@?$AAm?$AAi?$AA?9?$AAN?$AAZ@ 000000018004ccc8     libucrt:lcidtoname_downlevel.obj
 0002:00006cd8       ??_C@_1M@PMPEAILG@?$AAa?$AAr?$AA?9?$AAI?$AAQ@ 000000018004ccd8     libucrt:lcidtoname_downlevel.obj
 0002:00006ce8       ??_C@_1M@CNKPNOEE@?$AAd?$AAe?$AA?9?$AAC?$AAH@ 000000018004cce8     libucrt:lcidtoname_downlevel.obj
 0002:00006cf8       ??_C@_1M@LKMGMLKO@?$AAe?$AAn?$AA?9?$AAG?$AAB@ 000000018004ccf8     libucrt:lcidtoname_downlevel.obj
 0002:00006d08       ??_C@_1M@PGKJFFGL@?$AAe?$AAs?$AA?9?$AAM?$AAX@ 000000018004cd08     libucrt:lcidtoname_downlevel.obj
 0002:00006d18       ??_C@_1M@DNNANBDC@?$AAf?$AAr?$AA?9?$AAB?$AAE@ 000000018004cd18     libucrt:lcidtoname_downlevel.obj
 0002:00006d28       ??_C@_1M@HLGMDFHM@?$AAi?$AAt?$AA?9?$AAC?$AAH@ 000000018004cd28     libucrt:lcidtoname_downlevel.obj
 0002:00006d38       ??_C@_1M@CLLBGJH@?$AAn?$AAl?$AA?9?$AAB?$AAE@ 000000018004cd38     libucrt:lcidtoname_downlevel.obj
 0002:00006d48       ??_C@_1M@BODBOGLF@?$AAn?$AAn?$AA?9?$AAN?$AAO@ 000000018004cd48     libucrt:lcidtoname_downlevel.obj
 0002:00006d58       ??_C@_1M@HFFAHKAD@?$AAp?$AAt?$AA?9?$AAP?$AAT@ 000000018004cd58     libucrt:lcidtoname_downlevel.obj
 0002:00006d68       ??_C@_1BG@LNOAKHIE@?$AAs?$AAr?$AA?9?$AAS?$AAP?$AA?9?$AAL?$AAa?$AAt?$AAn@ 000000018004cd68     libucrt:lcidtoname_downlevel.obj
 0002:00006d80       ??_C@_1M@HBMHBGAK@?$AAs?$AAv?$AA?9?$AAF?$AAI@ 000000018004cd80     libucrt:lcidtoname_downlevel.obj
 0002:00006d90       ??_C@_1BG@DGCJGJBE@?$AAa?$AAz?$AA?9?$AAA?$AAZ?$AA?9?$AAC?$AAy?$AAr?$AAl@ 000000018004cd90     libucrt:lcidtoname_downlevel.obj
 0002:00006da8       ??_C@_1M@KEJDAAHB@?$AAs?$AAe?$AA?9?$AAS?$AAE@ 000000018004cda8     libucrt:lcidtoname_downlevel.obj
 0002:00006db8       ??_C@_1M@HEIBJJAD@?$AAm?$AAs?$AA?9?$AAB?$AAN@ 000000018004cdb8     libucrt:lcidtoname_downlevel.obj
 0002:00006dc8       ??_C@_1BG@PBGJMCEM@?$AAu?$AAz?$AA?9?$AAU?$AAZ?$AA?9?$AAC?$AAy?$AAr?$AAl@ 000000018004cdc8     libucrt:lcidtoname_downlevel.obj
 0002:00006de0       ??_C@_1O@LAOBCMDF@?$AAq?$AAu?$AAz?$AA?9?$AAE?$AAC@ 000000018004cde0     libucrt:lcidtoname_downlevel.obj
 0002:00006df0       ??_C@_1M@POEEMAIO@?$AAa?$AAr?$AA?9?$AAE?$AAG@ 000000018004cdf0     libucrt:lcidtoname_downlevel.obj
 0002:00006e00       ??_C@_1M@EFAKDEDL@?$AAz?$AAh?$AA?9?$AAH?$AAK@ 000000018004ce00     libucrt:lcidtoname_downlevel.obj
 0002:00006e10       ??_C@_1M@HKKIJHGI@?$AAd?$AAe?$AA?9?$AAA?$AAT@ 000000018004ce10     libucrt:lcidtoname_downlevel.obj
 0002:00006e20       ??_C@_1M@KBFBEHJF@?$AAe?$AAn?$AA?9?$AAA?$AAU@ 000000018004ce20     libucrt:lcidtoname_downlevel.obj
 0002:00006e30       ??_C@_1M@MNPLFAAH@?$AAe?$AAs?$AA?9?$AAE?$AAS@ 000000018004ce30     libucrt:lcidtoname_downlevel.obj
 0002:00006e40       ??_C@_1M@HJOOJFMA@?$AAf?$AAr?$AA?9?$AAC?$AAA@ 000000018004ce40     libucrt:lcidtoname_downlevel.obj
 0002:00006e50       ??_C@_1BG@JPOFPNAB@?$AAs?$AAr?$AA?9?$AAS?$AAP?$AA?9?$AAC?$AAy?$AAr?$AAl@ 000000018004ce50     libucrt:lcidtoname_downlevel.obj
 0002:00006e68       ??_C@_1M@LNFOCMOB@?$AAs?$AAe?$AA?9?$AAF?$AAI@ 000000018004ce68     libucrt:lcidtoname_downlevel.obj
 0002:00006e78       ??_C@_1O@MGJBOAMB@?$AAq?$AAu?$AAz?$AA?9?$AAP?$AAE@ 000000018004ce78     libucrt:lcidtoname_downlevel.obj
 0002:00006e88       ??_C@_1M@GJINLBOK@?$AAa?$AAr?$AA?9?$AAL?$AAY@ 000000018004ce88     libucrt:lcidtoname_downlevel.obj
 0002:00006e98       ??_C@_1M@GGMNHJNL@?$AAz?$AAh?$AA?9?$AAS?$AAG@ 000000018004ce98     libucrt:lcidtoname_downlevel.obj
 0002:00006ea8       ??_C@_1M@HOIKODND@?$AAd?$AAe?$AA?9?$AAL?$AAU@ 000000018004cea8     libucrt:lcidtoname_downlevel.obj
 0002:00006eb8       ??_C@_1M@DDOCCGFG@?$AAe?$AAn?$AA?9?$AAC?$AAA@ 000000018004ceb8     libucrt:lcidtoname_downlevel.obj
 0002:00006ec8       ??_C@_1M@BNOEMJLF@?$AAe?$AAs?$AA?9?$AAG?$AAT@ 000000018004cec8     libucrt:lcidtoname_downlevel.obj
 0002:00006ed8       ??_C@_1M@EOGNKEK@?$AAf?$AAr?$AA?9?$AAC?$AAH@ 000000018004ced8     libucrt:lcidtoname_downlevel.obj
 0002:00006ee8       ??_C@_1M@FLIDJFHL@?$AAh?$AAr?$AA?9?$AAB?$AAA@ 000000018004cee8     libucrt:lcidtoname_downlevel.obj
 0002:00006ef8       ??_C@_1O@FMCELNAJ@?$AAs?$AAm?$AAj?$AA?9?$AAN?$AAO@ 000000018004cef8     libucrt:lcidtoname_downlevel.obj
 0002:00006f08       ??_C@_1M@JHGLJMGJ@?$AAa?$AAr?$AA?9?$AAD?$AAZ@ 000000018004cf08     libucrt:lcidtoname_downlevel.obj
 0002:00006f18       ??_C@_1M@JKKFDCNP@?$AAz?$AAh?$AA?9?$AAM?$AAO@ 000000018004cf18     libucrt:lcidtoname_downlevel.obj
 0002:00006f28       ??_C@_1M@GEEFALPE@?$AAd?$AAe?$AA?9?$AAL?$AAI@ 000000018004cf28     libucrt:lcidtoname_downlevel.obj
 0002:00006f38       ??_C@_1M@IGEOFBG@?$AAe?$AAn?$AA?9?$AAN?$AAZ@ 000000018004cf38     libucrt:lcidtoname_downlevel.obj
 0002:00006f48       ??_C@_1M@KDBONEHP@?$AAe?$AAs?$AA?9?$AAC?$AAR@ 000000018004cf48     libucrt:lcidtoname_downlevel.obj
 0002:00006f58       ??_C@_1M@FHMDOHNN@?$AAf?$AAr?$AA?9?$AAL?$AAU@ 000000018004cf58     libucrt:lcidtoname_downlevel.obj
 0002:00006f68       ??_C@_1BG@NFKKMAFG@?$AAb?$AAs?$AA?9?$AAB?$AAA?$AA?9?$AAL?$AAa?$AAt?$AAn@ 000000018004cf68     libucrt:lcidtoname_downlevel.obj
 0002:00006f80       ??_C@_1O@IMNBEMCI@?$AAs?$AAm?$AAj?$AA?9?$AAS?$AAE@ 000000018004cf80     libucrt:lcidtoname_downlevel.obj
 0002:00006f90       ??_C@_1M@DHHMBNDP@?$AAa?$AAr?$AA?9?$AAM?$AAA@ 000000018004cf90     libucrt:lcidtoname_downlevel.obj
 0002:00006fa0       ??_C@_1M@BNBLJCGH@?$AAe?$AAn?$AA?9?$AAI?$AAE@ 000000018004cfa0     libucrt:lcidtoname_downlevel.obj
 0002:00006fb0       ??_C@_1M@GEPAFMDL@?$AAe?$AAs?$AA?9?$AAP?$AAA@ 000000018004cfb0     libucrt:lcidtoname_downlevel.obj
 0002:00006fc0       ??_C@_1M@OJONDMDL@?$AAf?$AAr?$AA?9?$AAM?$AAC@ 000000018004cfc0     libucrt:lcidtoname_downlevel.obj
 0002:00006fd0       ??_C@_1BG@OBCNFJB@?$AAs?$AAr?$AA?9?$AAB?$AAA?$AA?9?$AAL?$AAa?$AAt?$AAn@ 000000018004cfd0     libucrt:lcidtoname_downlevel.obj
 0002:00006fe8       ??_C@_1O@KEMEEGPO@?$AAs?$AAm?$AAa?$AA?9?$AAN?$AAO@ 000000018004cfe8     libucrt:lcidtoname_downlevel.obj
 0002:00006ff8       ??_C@_1M@ELMGFODK@?$AAa?$AAr?$AA?9?$AAT?$AAN@ 000000018004cff8     libucrt:lcidtoname_downlevel.obj
 0002:00007008       ??_C@_1M@BHDLHFAF@?$AAe?$AAn?$AA?9?$AAZ?$AAA@ 000000018004d008     libucrt:lcidtoname_downlevel.obj
 0002:00007018       ??_C@_1M@BMGIGLIF@?$AAe?$AAs?$AA?9?$AAD?$AAO@ 000000018004d018     libucrt:lcidtoname_downlevel.obj
 0002:00007028       ??_C@_1BG@CMBHIPBE@?$AAs?$AAr?$AA?9?$AAB?$AAA?$AA?9?$AAC?$AAy?$AAr?$AAl@ 000000018004d028     libucrt:lcidtoname_downlevel.obj
 0002:00007040       ??_C@_1O@HEDBLHNP@?$AAs?$AAm?$AAa?$AA?9?$AAS?$AAE@ 000000018004d040     libucrt:lcidtoname_downlevel.obj
 0002:00007050       ??_C@_1M@DAGCADIM@?$AAa?$AAr?$AA?9?$AAO?$AAM@ 000000018004d050     libucrt:lcidtoname_downlevel.obj
 0002:00007060       ??_C@_1M@FODLMICG@?$AAe?$AAn?$AA?9?$AAJ?$AAM@ 000000018004d060     libucrt:lcidtoname_downlevel.obj
 0002:00007070       ??_C@_1M@DNMLCIHB@?$AAe?$AAs?$AA?9?$AAV?$AAE@ 000000018004d070     libucrt:lcidtoname_downlevel.obj
 0002:00007080       ??_C@_1O@EOKHMKJK@?$AAs?$AAm?$AAs?$AA?9?$AAF?$AAI@ 000000018004d080     libucrt:lcidtoname_downlevel.obj
 0002:00007090       ??_C@_1M@CAFJMKOF@?$AAa?$AAr?$AA?9?$AAY?$AAE@ 000000018004d090     libucrt:lcidtoname_downlevel.obj
 0002:000070a0       ??_C@_1M@CBFHIJLI@?$AAe?$AAn?$AA?9?$AAC?$AAB@ 000000018004d0a0     libucrt:lcidtoname_downlevel.obj
 0002:000070b0       ??_C@_1M@BGNFLDN@?$AAe?$AAs?$AA?9?$AAC?$AAO@ 000000018004d0b0     libucrt:lcidtoname_downlevel.obj
 0002:000070c0       ??_C@_1O@JMPHMAMC@?$AAs?$AAm?$AAn?$AA?9?$AAF?$AAI@ 000000018004d0c0     libucrt:lcidtoname_downlevel.obj
 0002:000070d0       ??_C@_1M@JLANABKE@?$AAa?$AAr?$AA?9?$AAS?$AAY@ 000000018004d0d0     libucrt:lcidtoname_downlevel.obj
 0002:000070e0       ??_C@_1M@HPKGCFGN@?$AAe?$AAn?$AA?9?$AAB?$AAZ@ 000000018004d0e0     libucrt:lcidtoname_downlevel.obj
 0002:000070f0       ??_C@_1M@OLJCMLGM@?$AAe?$AAs?$AA?9?$AAP?$AAE@ 000000018004d0f0     libucrt:lcidtoname_downlevel.obj
 0002:00007100       ??_C@_1M@MKKGFKLE@?$AAa?$AAr?$AA?9?$AAJ?$AAO@ 000000018004d100     libucrt:lcidtoname_downlevel.obj
 0002:00007110       ??_C@_1M@EKPGLDNI@?$AAe?$AAn?$AA?9?$AAT?$AAT@ 000000018004d110     libucrt:lcidtoname_downlevel.obj
 0002:00007120       ??_C@_1M@OONGHFHE@?$AAe?$AAs?$AA?9?$AAA?$AAR@ 000000018004d120     libucrt:lcidtoname_downlevel.obj
 0002:00007130       ??_C@_1M@OOJFGBHE@?$AAa?$AAr?$AA?9?$AAL?$AAB@ 000000018004d130     libucrt:lcidtoname_downlevel.obj
 0002:00007140       ??_C@_1M@GCEJHNEG@?$AAe?$AAn?$AA?9?$AAZ?$AAW@ 000000018004d140     libucrt:lcidtoname_downlevel.obj
 0002:00007150       ??_C@_1M@JNOCAHJI@?$AAe?$AAs?$AA?9?$AAE?$AAC@ 000000018004d150     libucrt:lcidtoname_downlevel.obj
 0002:00007160       ??_C@_1M@JEFHPGGB@?$AAa?$AAr?$AA?9?$AAK?$AAW@ 000000018004d160     libucrt:lcidtoname_downlevel.obj
 0002:00007170       ??_C@_1M@MLKIBJOJ@?$AAe?$AAn?$AA?9?$AAP?$AAH@ 000000018004d170     libucrt:lcidtoname_downlevel.obj
 0002:00007180       ??_C@_1M@BDNIPEND@?$AAe?$AAs?$AA?9?$AAC?$AAL@ 000000018004d180     libucrt:lcidtoname_downlevel.obj
 0002:00007190       ??_C@_1M@MPNMEKBD@?$AAa?$AAr?$AA?9?$AAA?$AAE@ 000000018004d190     libucrt:lcidtoname_downlevel.obj
 0002:000071a0       ??_C@_1M@KBJALCPI@?$AAe?$AAs?$AA?9?$AAU?$AAY@ 000000018004d1a0     libucrt:lcidtoname_downlevel.obj
 0002:000071b0       ??_C@_1M@LLCCOAGA@?$AAa?$AAr?$AA?9?$AAB?$AAH@ 000000018004d1b0     libucrt:lcidtoname_downlevel.obj
 0002:000071c0       ??_C@_1M@PBFNCDEL@?$AAe?$AAs?$AA?9?$AAP?$AAY@ 000000018004d1c0     libucrt:lcidtoname_downlevel.obj
 0002:000071d0       ??_C@_1M@EDGINPNP@?$AAa?$AAr?$AA?9?$AAQ?$AAA@ 000000018004d1d0     libucrt:lcidtoname_downlevel.obj
 0002:000071e0       ??_C@_1M@MKDBIIJI@?$AAe?$AAs?$AA?9?$AAB?$AAO@ 000000018004d1e0     libucrt:lcidtoname_downlevel.obj
 0002:000071f0       ??_C@_1M@CPKKEBLD@?$AAe?$AAs?$AA?9?$AAS?$AAV@ 000000018004d1f0     libucrt:lcidtoname_downlevel.obj
 0002:00007200       ??_C@_1M@NDBGMMJL@?$AAe?$AAs?$AA?9?$AAH?$AAN@ 000000018004d200     libucrt:lcidtoname_downlevel.obj
 0002:00007210       ??_C@_1M@JIJIBHDP@?$AAe?$AAs?$AA?9?$AAN?$AAI@ 000000018004d210     libucrt:lcidtoname_downlevel.obj
 0002:00007220       ??_C@_1M@CGFMKEEK@?$AAe?$AAs?$AA?9?$AAP?$AAR@ 000000018004d220     libucrt:lcidtoname_downlevel.obj
 0002:00007230       ??_C@_1O@ICJHKIIK@?$AAz?$AAh?$AA?9?$AAC?$AAH?$AAT@ 000000018004d230     libucrt:lcidtoname_downlevel.obj
 0002:00007240       ??_C@_15CLNEJCE@?$AAs?$AAr@ 000000018004d240     libucrt:lcidtoname_downlevel.obj
 0002:00008090       ??_C@_1M@KAHEKEIG@?$AAa?$AAf?$AA?9?$AAz?$AAa@ 000000018004e090     libucrt:lcidtoname_downlevel.obj
 0002:000080a0       ??_C@_1M@GIECOABL@?$AAa?$AAr?$AA?9?$AAa?$AAe@ 000000018004e0a0     libucrt:lcidtoname_downlevel.obj
 0002:000080b0       ??_C@_1M@BMLMEKGI@?$AAa?$AAr?$AA?9?$AAb?$AAh@ 000000018004e0b0     libucrt:lcidtoname_downlevel.obj
 0002:000080c0       ??_C@_1M@DAPFDGGB@?$AAa?$AAr?$AA?9?$AAd?$AAz@ 000000018004e0c0     libucrt:lcidtoname_downlevel.obj
 0002:000080d0       ??_C@_1M@FJNKGKIG@?$AAa?$AAr?$AA?9?$AAe?$AAg@ 000000018004e0d0     libucrt:lcidtoname_downlevel.obj
 0002:000080e0       ??_C@_1M@FLGKKCLO@?$AAa?$AAr?$AA?9?$AAi?$AAq@ 000000018004e0e0     libucrt:lcidtoname_downlevel.obj
 0002:000080f0       ??_C@_1M@GNDIPALM@?$AAa?$AAr?$AA?9?$AAj?$AAo@ 000000018004e0f0     libucrt:lcidtoname_downlevel.obj
 0002:00008100       ??_C@_1M@DDMJFMGJ@?$AAa?$AAr?$AA?9?$AAk?$AAw@ 000000018004e100     libucrt:lcidtoname_downlevel.obj
 0002:00008110       ??_C@_1M@EJALMLHM@?$AAa?$AAr?$AA?9?$AAl?$AAb@ 000000018004e110     libucrt:lcidtoname_downlevel.obj
 0002:00008120       ??_C@_1M@MOBDBLOC@?$AAa?$AAr?$AA?9?$AAl?$AAy@ 000000018004e120     libucrt:lcidtoname_downlevel.obj
 0002:00008130       ??_C@_1M@JAOCLHDH@?$AAa?$AAr?$AA?9?$AAm?$AAa@ 000000018004e130     libucrt:lcidtoname_downlevel.obj
 0002:00008140       ??_C@_1M@JHPMKJIE@?$AAa?$AAr?$AA?9?$AAo?$AAm@ 000000018004e140     libucrt:lcidtoname_downlevel.obj
 0002:00008150       ??_C@_1M@OEPGHFNH@?$AAa?$AAr?$AA?9?$AAq?$AAa@ 000000018004e150     libucrt:lcidtoname_downlevel.obj
 0002:00008160       ??_C@_1M@KJDONENM@?$AAa?$AAr?$AA?9?$AAs?$AAa@ 000000018004e160     libucrt:lcidtoname_downlevel.obj
 0002:00008170       ??_C@_1M@DMJDKLKM@?$AAa?$AAr?$AA?9?$AAs?$AAy@ 000000018004e170     libucrt:lcidtoname_downlevel.obj
 0002:00008180       ??_C@_1M@OMFIPEDC@?$AAa?$AAr?$AA?9?$AAt?$AAn@ 000000018004e180     libucrt:lcidtoname_downlevel.obj
 0002:00008190       ??_C@_1M@IHMHGAON@?$AAa?$AAr?$AA?9?$AAy?$AAe@ 000000018004e190     libucrt:lcidtoname_downlevel.obj
 0002:000081a0       ??_C@_1BG@KDCPGJGB@?$AAa?$AAz?$AA?9?$AAa?$AAz?$AA?9?$AAc?$AAy?$AAr?$AAl@ 000000018004e1a0     libucrt:lcidtoname_downlevel.obj
 0002:000081b8       ??_C@_1BG@IBCKDDOE@?$AAa?$AAz?$AA?9?$AAa?$AAz?$AA?9?$AAl?$AAa?$AAt?$AAn@ 000000018004e1b8     libucrt:lcidtoname_downlevel.obj
 0002:000081d0       ??_C@_1M@EGPFDCPD@?$AAb?$AAe?$AA?9?$AAb?$AAy@ 000000018004e1d0     libucrt:lcidtoname_downlevel.obj
 0002:000081e0       ??_C@_1M@PCMGMCGC@?$AAb?$AAg?$AA?9?$AAb?$AAg@ 000000018004e1e0     libucrt:lcidtoname_downlevel.obj
 0002:000081f0       ??_C@_1M@BJBMFGOB@?$AAb?$AAn?$AA?9?$AAi?$AAn@ 000000018004e1f0     libucrt:lcidtoname_downlevel.obj
 0002:00008200       ??_C@_1BG@EAKMMACD@?$AAb?$AAs?$AA?9?$AAb?$AAa?$AA?9?$AAl?$AAa?$AAt?$AAn@ 000000018004e200     libucrt:lcidtoname_downlevel.obj
 0002:00008218       ??_C@_1M@KGADAODK@?$AAc?$AAa?$AA?9?$AAe?$AAs@ 000000018004e218     libucrt:lcidtoname_downlevel.obj
 0002:00008228       ??_C@_1M@COAJPDHI@?$AAc?$AAs?$AA?9?$AAc?$AAz@ 000000018004e228     libucrt:lcidtoname_downlevel.obj
 0002:00008238       ??_C@_1M@DHBHFONH@?$AAc?$AAy?$AA?9?$AAg?$AAb@ 000000018004e238     libucrt:lcidtoname_downlevel.obj
 0002:00008248       ??_C@_1M@IMGKELGA@?$AAd?$AAa?$AA?9?$AAd?$AAk@ 000000018004e248     libucrt:lcidtoname_downlevel.obj
 0002:00008258       ??_C@_1M@NNDGDNGA@?$AAd?$AAe?$AA?9?$AAa?$AAt@ 000000018004e258     libucrt:lcidtoname_downlevel.obj
 0002:00008268       ??_C@_1M@IKDBHEEM@?$AAd?$AAe?$AA?9?$AAc?$AAh@ 000000018004e268     libucrt:lcidtoname_downlevel.obj
 0002:00008278       ??_C@_1M@GFFOJMCJ@?$AAd?$AAe?$AA?9?$AAd?$AAe@ 000000018004e278     libucrt:lcidtoname_downlevel.obj
 0002:00008288       ??_C@_1M@MDNLKBPM@?$AAd?$AAe?$AA?9?$AAl?$AAi@ 000000018004e288     libucrt:lcidtoname_downlevel.obj
 0002:00008298       ??_C@_1M@NJBEEJNL@?$AAd?$AAe?$AA?9?$AAl?$AAu@ 000000018004e298     libucrt:lcidtoname_downlevel.obj
 0002:000082a8       ??_C@_1O@GNNELBAP@?$AAd?$AAi?$AAv?$AA?9?$AAm?$AAv@ 000000018004e2a8     libucrt:lcidtoname_downlevel.obj
 0002:000082b8       ??_C@_1M@EJLEOGAE@?$AAe?$AAl?$AA?9?$AAg?$AAr@ 000000018004e2b8     libucrt:lcidtoname_downlevel.obj
 0002:000082c8       ??_C@_1M@GMPONJN@?$AAe?$AAn?$AA?9?$AAa?$AAu@ 000000018004e2c8     libucrt:lcidtoname_downlevel.obj
 0002:000082d8       ??_C@_1M@NIDIIPGF@?$AAe?$AAn?$AA?9?$AAb?$AAz@ 000000018004e2d8     libucrt:lcidtoname_downlevel.obj
 0002:000082e8       ??_C@_1M@JEHMIMFO@?$AAe?$AAn?$AA?9?$AAc?$AAa@ 000000018004e2e8     libucrt:lcidtoname_downlevel.obj
 0002:000082f8       ??_C@_1M@IGMJCDLA@?$AAe?$AAn?$AA?9?$AAc?$AAb@ 000000018004e2f8     libucrt:lcidtoname_downlevel.obj
 0002:00008308       ??_C@_1M@BNFIGBKG@?$AAe?$AAn?$AA?9?$AAg?$AAb@ 000000018004e308     libucrt:lcidtoname_downlevel.obj
 0002:00008318       ??_C@_1M@LKIFDIGP@?$AAe?$AAn?$AA?9?$AAi?$AAe@ 000000018004e318     libucrt:lcidtoname_downlevel.obj
 0002:00008328       ??_C@_1M@PJKFGCCO@?$AAe?$AAn?$AA?9?$AAj?$AAm@ 000000018004e328     libucrt:lcidtoname_downlevel.obj
 0002:00008338       ??_C@_1M@KPPKEPBO@?$AAe?$AAn?$AA?9?$AAn?$AAz@ 000000018004e338     libucrt:lcidtoname_downlevel.obj
 0002:00008348       ??_C@_1M@GMDGLDOB@?$AAe?$AAn?$AA?9?$AAp?$AAh@ 000000018004e348     libucrt:lcidtoname_downlevel.obj
 0002:00008358       ??_C@_1M@ONGIBJNA@?$AAe?$AAn?$AA?9?$AAt?$AAt@ 000000018004e358     libucrt:lcidtoname_downlevel.obj
 0002:00008368       ??_C@_1M@LLODPCMM@?$AAe?$AAn?$AA?9?$AAu?$AAs@ 000000018004e368     libucrt:lcidtoname_downlevel.obj
 0002:00008378       ??_C@_1M@LAKFNPAN@?$AAe?$AAn?$AA?9?$AAz?$AAa@ 000000018004e378     libucrt:lcidtoname_downlevel.obj
 0002:00008388       ??_C@_1M@MFNHNHEO@?$AAe?$AAn?$AA?9?$AAz?$AAw@ 000000018004e388     libucrt:lcidtoname_downlevel.obj
 0002:00008398       ??_C@_1M@EJEINPHM@?$AAe?$AAs?$AA?9?$AAa?$AAr@ 000000018004e398     libucrt:lcidtoname_downlevel.obj
 0002:000083a8       ??_C@_1M@GNKPCCJA@?$AAe?$AAs?$AA?9?$AAb?$AAo@ 000000018004e3a8     libucrt:lcidtoname_downlevel.obj
 0002:000083b8       ??_C@_1M@LEEGFONL@?$AAe?$AAs?$AA?9?$AAc?$AAl@ 000000018004e3b8     libucrt:lcidtoname_downlevel.obj
 0002:000083c8       ??_C@_1M@KGPDPBDF@?$AAe?$AAs?$AA?9?$AAc?$AAo@ 000000018004e3c8     libucrt:lcidtoname_downlevel.obj
 0002:000083d8       ??_C@_1M@EIAHOHH@?$AAe?$AAs?$AA?9?$AAc?$AAr@ 000000018004e3d8     libucrt:lcidtoname_downlevel.obj
 0002:000083e8       ??_C@_1M@LLPGMBIN@?$AAe?$AAs?$AA?9?$AAd?$AAo@ 000000018004e3e8     libucrt:lcidtoname_downlevel.obj
 0002:000083f8       ??_C@_1M@DKHMKNJA@?$AAe?$AAs?$AA?9?$AAe?$AAc@ 000000018004e3f8     libucrt:lcidtoname_downlevel.obj
 0002:00008408       ??_C@_1M@GKGFPKAP@?$AAe?$AAs?$AA?9?$AAe?$AAs@ 000000018004e408     libucrt:lcidtoname_downlevel.obj
 0002:00008418       ??_C@_1M@LKHKGDLN@?$AAe?$AAs?$AA?9?$AAg?$AAt@ 000000018004e418     libucrt:lcidtoname_downlevel.obj
 0002:00008428       ??_C@_1M@HEIIGGJD@?$AAe?$AAs?$AA?9?$AAh?$AAn@ 000000018004e428     libucrt:lcidtoname_downlevel.obj
 0002:00008438       ??_C@_1M@FBDHPPGD@?$AAe?$AAs?$AA?9?$AAm?$AAx@ 000000018004e438     libucrt:lcidtoname_downlevel.obj
 0002:00008448       ??_C@_1M@DPAGLNDH@?$AAe?$AAs?$AA?9?$AAn?$AAi@ 000000018004e448     libucrt:lcidtoname_downlevel.obj
 0002:00008458       ??_C@_1M@MDGOPGDD@?$AAe?$AAs?$AA?9?$AAp?$AAa@ 000000018004e458     libucrt:lcidtoname_downlevel.obj
 0002:00008468       ??_C@_1M@EMAMGBGE@?$AAe?$AAs?$AA?9?$AAp?$AAe@ 000000018004e468     libucrt:lcidtoname_downlevel.obj
 0002:00008478       ??_C@_1M@IBMCAOEC@?$AAe?$AAs?$AA?9?$AAp?$AAr@ 000000018004e478     libucrt:lcidtoname_downlevel.obj
 0002:00008488       ??_C@_1M@FGMDIJED@?$AAe?$AAs?$AA?9?$AAp?$AAy@ 000000018004e488     libucrt:lcidtoname_downlevel.obj
 0002:00008498       ??_C@_1M@IIDEOLLL@?$AAe?$AAs?$AA?9?$AAs?$AAv@ 000000018004e498     libucrt:lcidtoname_downlevel.obj
 0002:000084a8       ??_C@_1M@GAOBIPA@?$AAe?$AAs?$AA?9?$AAu?$AAy@ 000000018004e4a8     libucrt:lcidtoname_downlevel.obj
 0002:000084b8       ??_C@_1M@JKFFICHJ@?$AAe?$AAs?$AA?9?$AAv?$AAe@ 000000018004e4b8     libucrt:lcidtoname_downlevel.obj
 0002:000084c8       ??_C@_1M@PNMLOJDF@?$AAe?$AAt?$AA?9?$AAe?$AAe@ 000000018004e4c8     libucrt:lcidtoname_downlevel.obj
 0002:000084d8       ??_C@_1M@GHHLIKEI@?$AAe?$AAu?$AA?9?$AAe?$AAs@ 000000018004e4d8     libucrt:lcidtoname_downlevel.obj
 0002:000084e8       ??_C@_1M@PBNONODE@?$AAf?$AAa?$AA?9?$AAi?$AAr@ 000000018004e4e8     libucrt:lcidtoname_downlevel.obj
 0002:000084f8       ??_C@_1M@JEEHPMIL@?$AAf?$AAi?$AA?9?$AAf?$AAi@ 000000018004e4f8     libucrt:lcidtoname_downlevel.obj
 0002:00008508       ??_C@_1M@LMDCNDBA@?$AAf?$AAo?$AA?9?$AAf?$AAo@ 000000018004e508     libucrt:lcidtoname_downlevel.obj
 0002:00008518       ??_C@_1M@JKEOHLDK@?$AAf?$AAr?$AA?9?$AAb?$AAe@ 000000018004e518     libucrt:lcidtoname_downlevel.obj
 0002:00008528       ??_C@_1M@NOHADPMI@?$AAf?$AAr?$AA?9?$AAc?$AAa@ 000000018004e528     libucrt:lcidtoname_downlevel.obj
 0002:00008538       ??_C@_1M@KDHIHAEC@?$AAf?$AAr?$AA?9?$AAc?$AAh@ 000000018004e538     libucrt:lcidtoname_downlevel.obj
 0002:00008548       ??_C@_1M@MMBBFGAK@?$AAf?$AAr?$AA?9?$AAf?$AAr@ 000000018004e548     libucrt:lcidtoname_downlevel.obj
 0002:00008558       ??_C@_1M@PAFNENNF@?$AAf?$AAr?$AA?9?$AAl?$AAu@ 000000018004e558     libucrt:lcidtoname_downlevel.obj
 0002:00008568       ??_C@_1M@EOHDJGDD@?$AAf?$AAr?$AA?9?$AAm?$AAc@ 000000018004e568     libucrt:lcidtoname_downlevel.obj
 0002:00008578       ??_C@_1M@FAPLLOPF@?$AAg?$AAl?$AA?9?$AAe?$AAs@ 000000018004e578     libucrt:lcidtoname_downlevel.obj
 0002:00008588       ??_C@_1M@FOPBFLOO@?$AAg?$AAu?$AA?9?$AAi?$AAn@ 000000018004e588     libucrt:lcidtoname_downlevel.obj
 0002:00008598       ??_C@_1M@KBMCINPM@?$AAh?$AAe?$AA?9?$AAi?$AAl@ 000000018004e598     libucrt:lcidtoname_downlevel.obj
 0002:000085a8       ??_C@_1M@BBPHKFPJ@?$AAh?$AAi?$AA?9?$AAi?$AAn@ 000000018004e5a8     libucrt:lcidtoname_downlevel.obj
 0002:000085b8       ??_C@_1M@PMBNDPHD@?$AAh?$AAr?$AA?9?$AAb?$AAa@ 000000018004e5b8     libucrt:lcidtoname_downlevel.obj
 0002:000085c8       ??_C@_1M@BPCKOEGE@?$AAh?$AAr?$AA?9?$AAh?$AAr@ 000000018004e5c8     libucrt:lcidtoname_downlevel.obj
 0002:000085d8       ??_C@_1M@GACBMHKE@?$AAh?$AAu?$AA?9?$AAh?$AAu@ 000000018004e5d8     libucrt:lcidtoname_downlevel.obj
 0002:000085e8       ??_C@_1M@MILPAJJC@?$AAh?$AAy?$AA?9?$AAa?$AAm@ 000000018004e5e8     libucrt:lcidtoname_downlevel.obj
 0002:000085f8       ??_C@_1M@BABBICEC@?$AAi?$AAd?$AA?9?$AAi?$AAd@ 000000018004e5f8     libucrt:lcidtoname_downlevel.obj
 0002:00008608       ??_C@_1M@BIKNHHPF@?$AAi?$AAs?$AA?9?$AAi?$AAs@ 000000018004e608     libucrt:lcidtoname_downlevel.obj
 0002:00008618       ??_C@_1M@NMPCJPHE@?$AAi?$AAt?$AA?9?$AAc?$AAh@ 000000018004e618     libucrt:lcidtoname_downlevel.obj
 0002:00008628       ??_C@_1M@GHKGFEDF@?$AAi?$AAt?$AA?9?$AAi?$AAt@ 000000018004e628     libucrt:lcidtoname_downlevel.obj
 0002:00008638       ??_C@_1M@NIEJCJJA@?$AAj?$AAa?$AA?9?$AAj?$AAp@ 000000018004e638     libucrt:lcidtoname_downlevel.obj
 0002:00008648       ??_C@_1M@JILFNBIM@?$AAk?$AAa?$AA?9?$AAg?$AAe@ 000000018004e648     libucrt:lcidtoname_downlevel.obj
 0002:00008658       ??_C@_1M@PACPMGPH@?$AAk?$AAk?$AA?9?$AAk?$AAz@ 000000018004e658     libucrt:lcidtoname_downlevel.obj
 0002:00008668       ??_C@_1M@IELFGMHA@?$AAk?$AAn?$AA?9?$AAi?$AAn@ 000000018004e668     libucrt:lcidtoname_downlevel.obj
 0002:00008678       ??_C@_1O@IBBJHCH@?$AAk?$AAo?$AAk?$AA?9?$AAi?$AAn@ 000000018004e678     libucrt:lcidtoname_downlevel.obj
 0002:00008688       ??_C@_1M@DMHAEOGC@?$AAk?$AAo?$AA?9?$AAk?$AAr@ 000000018004e688     libucrt:lcidtoname_downlevel.obj
 0002:00008698       ??_C@_1M@HBAHBIGA@?$AAk?$AAy?$AA?9?$AAk?$AAg@ 000000018004e698     libucrt:lcidtoname_downlevel.obj
 0002:000086a8       ??_C@_1M@KPMILCJG@?$AAl?$AAt?$AA?9?$AAl?$AAt@ 000000018004e6a8     libucrt:lcidtoname_downlevel.obj
 0002:000086b8       ??_C@_1M@BDEKKCA@?$AAl?$AAv?$AA?9?$AAl?$AAv@ 000000018004e6b8     libucrt:lcidtoname_downlevel.obj
 0002:000086c8       ??_C@_1M@ELCKCCJJ@?$AAm?$AAi?$AA?9?$AAn?$AAz@ 000000018004e6c8     libucrt:lcidtoname_downlevel.obj
 0002:000086d8       ??_C@_1M@CBOOLAPA@?$AAm?$AAk?$AA?9?$AAm?$AAk@ 000000018004e6d8     libucrt:lcidtoname_downlevel.obj
 0002:000086e8       ??_C@_1M@GPHNBJKN@?$AAm?$AAl?$AA?9?$AAi?$AAn@ 000000018004e6e8     libucrt:lcidtoname_downlevel.obj
 0002:000086f8       ??_C@_1M@PABJILIG@?$AAm?$AAn?$AA?9?$AAm?$AAn@ 000000018004e6f8     libucrt:lcidtoname_downlevel.obj
 0002:00008708       ??_C@_1M@FGBKKIPG@?$AAm?$AAr?$AA?9?$AAi?$AAn@ 000000018004e708     libucrt:lcidtoname_downlevel.obj
 0002:00008718       ??_C@_1M@NDBPDDAL@?$AAm?$AAs?$AA?9?$AAb?$AAn@ 000000018004e718     libucrt:lcidtoname_downlevel.obj
 0002:00008728       ??_C@_1M@OPIHOOPI@?$AAm?$AAs?$AA?9?$AAm?$AAy@ 000000018004e728     libucrt:lcidtoname_downlevel.obj
 0002:00008738       ??_C@_1M@PPDBCNFM@?$AAm?$AAt?$AA?9?$AAm?$AAt@ 000000018004e738     libucrt:lcidtoname_downlevel.obj
 0002:00008748       ??_C@_1M@KDJDKMDD@?$AAn?$AAb?$AA?9?$AAn?$AAo@ 000000018004e748     libucrt:lcidtoname_downlevel.obj
 0002:00008758       ??_C@_1M@KFCFLMJP@?$AAn?$AAl?$AA?9?$AAb?$AAe@ 000000018004e758     libucrt:lcidtoname_downlevel.obj
 0002:00008768       ??_C@_1M@KPOPDDGO@?$AAn?$AAl?$AA?9?$AAn?$AAl@ 000000018004e768     libucrt:lcidtoname_downlevel.obj
 0002:00008778       ??_C@_1M@LJKPEMLN@?$AAn?$AAn?$AA?9?$AAn?$AAo@ 000000018004e778     libucrt:lcidtoname_downlevel.obj
 0002:00008788       ??_C@_1M@BDGHHBFL@?$AAn?$AAs?$AA?9?$AAz?$AAa@ 000000018004e788     libucrt:lcidtoname_downlevel.obj
 0002:00008798       ??_C@_1M@IDEHOAP@?$AAp?$AAa?$AA?9?$AAi?$AAn@ 000000018004e798     libucrt:lcidtoname_downlevel.obj
 0002:000087a8       ??_C@_1M@HDBKGOGH@?$AAp?$AAl?$AA?9?$AAp?$AAl@ 000000018004e7a8     libucrt:lcidtoname_downlevel.obj
 0002:000087b8       ??_C@_1M@LJLLCMEH@?$AAp?$AAt?$AA?9?$AAb?$AAr@ 000000018004e7b8     libucrt:lcidtoname_downlevel.obj
 0002:000087c8       ??_C@_1M@NCMONAAL@?$AAp?$AAt?$AA?9?$AAp?$AAt@ 000000018004e7c8     libucrt:lcidtoname_downlevel.obj
 0002:000087d8       ??_C@_1O@EAKMAJDN@?$AAq?$AAu?$AAz?$AA?9?$AAb?$AAo@ 000000018004e7d8     libucrt:lcidtoname_downlevel.obj
 0002:000087e8       ??_C@_1O@BHHPIGDN@?$AAq?$AAu?$AAz?$AA?9?$AAe?$AAc@ 000000018004e7e8     libucrt:lcidtoname_downlevel.obj
 0002:000087f8       ??_C@_1O@GBAPEKMJ@?$AAq?$AAu?$AAz?$AA?9?$AAp?$AAe@ 000000018004e7f8     libucrt:lcidtoname_downlevel.obj
 0002:00008808       ??_C@_1M@CLGLEFBO@?$AAr?$AAo?$AA?9?$AAr?$AAo@ 000000018004e808     libucrt:lcidtoname_downlevel.obj
 0002:00008818       ??_C@_1M@CEEDODME@?$AAr?$AAu?$AA?9?$AAr?$AAu@ 000000018004e818     libucrt:lcidtoname_downlevel.obj
 0002:00008828       ??_C@_1M@HPKKKMPP@?$AAs?$AAa?$AA?9?$AAi?$AAn@ 000000018004e828     libucrt:lcidtoname_downlevel.obj
 0002:00008838       ??_C@_1M@BKMAIGOJ@?$AAs?$AAe?$AA?9?$AAf?$AAi@ 000000018004e838     libucrt:lcidtoname_downlevel.obj
 0002:00008848       ??_C@_1M@NDPIFLFI@?$AAs?$AAe?$AA?9?$AAn?$AAo@ 000000018004e848     libucrt:lcidtoname_downlevel.obj
 0002:00008858       ??_C@_1M@DANKKHJ@?$AAs?$AAe?$AA?9?$AAs?$AAe@ 000000018004e858     libucrt:lcidtoname_downlevel.obj
 0002:00008868       ??_C@_1M@PNBLONPJ@?$AAs?$AAk?$AA?9?$AAs?$AAk@ 000000018004e868     libucrt:lcidtoname_downlevel.obj
 0002:00008878       ??_C@_1M@LFMODOAL@?$AAs?$AAl?$AA?9?$AAs?$AAi@ 000000018004e878     libucrt:lcidtoname_downlevel.obj
 0002:00008888       ??_C@_1O@DFKOMPG@?$AAs?$AAm?$AAa?$AA?9?$AAn?$AAo@ 000000018004e888     libucrt:lcidtoname_downlevel.obj
 0002:00008898       ??_C@_1O@NDKPBNNH@?$AAs?$AAm?$AAa?$AA?9?$AAs?$AAe@ 000000018004e898     libucrt:lcidtoname_downlevel.obj
 0002:000088a8       ??_C@_1O@PLLKBHAB@?$AAs?$AAm?$AAj?$AA?9?$AAn?$AAo@ 000000018004e8a8     libucrt:lcidtoname_downlevel.obj
 0002:000088b8       ??_C@_1O@CLEPOGCA@?$AAs?$AAm?$AAj?$AA?9?$AAs?$AAe@ 000000018004e8b8     libucrt:lcidtoname_downlevel.obj
 0002:000088c8       ??_C@_1O@DLGJGKMK@?$AAs?$AAm?$AAn?$AA?9?$AAf?$AAi@ 000000018004e8c8     libucrt:lcidtoname_downlevel.obj
 0002:000088d8       ??_C@_1O@OJDJGAJC@?$AAs?$AAm?$AAs?$AA?9?$AAf?$AAi@ 000000018004e8d8     libucrt:lcidtoname_downlevel.obj
 0002:000088e8       ??_C@_1M@BOFOGHPB@?$AAs?$AAq?$AA?9?$AAa?$AAl@ 000000018004e8e8     libucrt:lcidtoname_downlevel.obj
 0002:000088f8       ??_C@_1BG@LJBBIPGB@?$AAs?$AAr?$AA?9?$AAb?$AAa?$AA?9?$AAc?$AAy?$AAr?$AAl@ 000000018004e8f8     libucrt:lcidtoname_downlevel.obj
 0002:00008910       ??_C@_1BG@JLBENFOE@?$AAs?$AAr?$AA?9?$AAb?$AAa?$AA?9?$AAl?$AAa?$AAt?$AAn@ 000000018004e910     libucrt:lcidtoname_downlevel.obj
 0002:00008928       ??_C@_1BG@KODPNHE@?$AAs?$AAr?$AA?9?$AAs?$AAp?$AA?9?$AAc?$AAy?$AAr?$AAl@ 000000018004e928     libucrt:lcidtoname_downlevel.obj
 0002:00008940       ??_C@_1BG@CIOGKHPB@?$AAs?$AAr?$AA?9?$AAs?$AAp?$AA?9?$AAl?$AAa?$AAt?$AAn@ 000000018004e940     libucrt:lcidtoname_downlevel.obj
 0002:00008958       ??_C@_1M@NGFJLMAC@?$AAs?$AAv?$AA?9?$AAf?$AAi@ 000000018004e958     libucrt:lcidtoname_downlevel.obj
 0002:00008968       ??_C@_1M@MPJEJAJC@?$AAs?$AAv?$AA?9?$AAs?$AAe@ 000000018004e968     libucrt:lcidtoname_downlevel.obj
 0002:00008978       ??_C@_1M@MPNDHLFK@?$AAs?$AAw?$AA?9?$AAk?$AAe@ 000000018004e978     libucrt:lcidtoname_downlevel.obj
 0002:00008988       ??_C@_1O@KOHBJJI@?$AAs?$AAy?$AAr?$AA?9?$AAs?$AAy@ 000000018004e988     libucrt:lcidtoname_downlevel.obj
 0002:00008998       ??_C@_1M@LDCEFHA@?$AAt?$AAa?$AA?9?$AAi?$AAn@ 000000018004e998     libucrt:lcidtoname_downlevel.obj
 0002:000089a8       ??_C@_1M@CNJOFAK@?$AAt?$AAe?$AA?9?$AAi?$AAn@ 000000018004e9a8     libucrt:lcidtoname_downlevel.obj
 0002:000089b8       ??_C@_1M@GNAECACD@?$AAt?$AAh?$AA?9?$AAt?$AAh@ 000000018004e9b8     libucrt:lcidtoname_downlevel.obj
 0002:000089c8       ??_C@_1M@CHBIHOJO@?$AAt?$AAn?$AA?9?$AAz?$AAa@ 000000018004e9c8     libucrt:lcidtoname_downlevel.obj
 0002:000089d8       ??_C@_1M@GCCMIGPJ@?$AAt?$AAr?$AA?9?$AAt?$AAr@ 000000018004e9d8     libucrt:lcidtoname_downlevel.obj
 0002:000089e8       ??_C@_1M@CELMCNBK@?$AAt?$AAt?$AA?9?$AAr?$AAu@ 000000018004e9e8     libucrt:lcidtoname_downlevel.obj
 0002:000089f8       ??_C@_1M@KLMCELGA@?$AAu?$AAk?$AA?9?$AAu?$AAa@ 000000018004e9f8     libucrt:lcidtoname_downlevel.obj
 0002:00008a08       ??_C@_1M@EPAJJAJF@?$AAu?$AAr?$AA?9?$AAp?$AAk@ 000000018004ea08     libucrt:lcidtoname_downlevel.obj
 0002:00008a18       ??_C@_1BG@GEGPMCDJ@?$AAu?$AAz?$AA?9?$AAu?$AAz?$AA?9?$AAc?$AAy?$AAr?$AAl@ 000000018004ea18     libucrt:lcidtoname_downlevel.obj
 0002:00008a30       ??_C@_1BG@EGGKJILM@?$AAu?$AAz?$AA?9?$AAu?$AAz?$AA?9?$AAl?$AAa?$AAt?$AAn@ 000000018004ea30     libucrt:lcidtoname_downlevel.obj
 0002:00008a48       ??_C@_1M@GFOCLFF@?$AAv?$AAi?$AA?9?$AAv?$AAn@ 000000018004ea48     libucrt:lcidtoname_downlevel.obj
 0002:00008a58       ??_C@_1M@CPAMEDFI@?$AAx?$AAh?$AA?9?$AAz?$AAa@ 000000018004ea58     libucrt:lcidtoname_downlevel.obj
 0002:00008a68       ??_C@_1O@EBKIFIGN@?$AAz?$AAh?$AA?9?$AAc?$AAh?$AAs@ 000000018004ea68     libucrt:lcidtoname_downlevel.obj
 0002:00008a78       ??_C@_1O@NMHPGANE@?$AAz?$AAh?$AA?9?$AAc?$AAh?$AAt@ 000000018004ea78     libucrt:lcidtoname_downlevel.obj
 0002:00008a88       ??_C@_1M@LPINJOMC@?$AAz?$AAh?$AA?9?$AAc?$AAn@ 000000018004ea88     libucrt:lcidtoname_downlevel.obj
 0002:00008a98       ??_C@_1M@OCJEJODD@?$AAz?$AAh?$AA?9?$AAh?$AAk@ 000000018004ea98     libucrt:lcidtoname_downlevel.obj
 0002:00008aa8       ??_C@_1M@DNDLJINH@?$AAz?$AAh?$AA?9?$AAm?$AAo@ 000000018004eaa8     libucrt:lcidtoname_downlevel.obj
 0002:00008ab8       ??_C@_1M@MBFDNDND@?$AAz?$AAh?$AA?9?$AAs?$AAg@ 000000018004eab8     libucrt:lcidtoname_downlevel.obj
 0002:00008ac8       ??_C@_1M@IMEPLEPE@?$AAz?$AAh?$AA?9?$AAt?$AAw@ 000000018004eac8     libucrt:lcidtoname_downlevel.obj
 0002:00008ad8       ??_C@_1M@BBGHNHJP@?$AAz?$AAu?$AA?9?$AAz?$AAa@ 000000018004ead8     libucrt:lcidtoname_downlevel.obj
 0002:00008b88       ??_C@_01GBGANLPD@0@        000000018004eb88     libucrt:cfout.obj
 0002:00008b8c       ??_C@_05DNEBIAHO@1?$CDINF@ 000000018004eb8c     libucrt:cfout.obj
 0002:00008b94       ??_C@_06IMKFLFPG@1?$CDQNAN@ 000000018004eb94     libucrt:cfout.obj
 0002:00008b9c       ??_C@_06PGGFOGJG@1?$CDSNAN@ 000000018004eb9c     libucrt:cfout.obj
 0002:00008ba4       ??_C@_05PHHOCPM@1?$CDIND@  000000018004eba4     libucrt:cfout.obj
 0002:00008bb0       __acrt_rg_language         000000018004ebb0     libucrt:get_qualified_locale.obj
 0002:00008fc0       __acrt_rg_language_count   000000018004efc0     libucrt:get_qualified_locale.obj
 0002:00008fd0       __acrt_rg_country          000000018004efd0     libucrt:get_qualified_locale.obj
 0002:00009140       __acrt_rg_country_count    000000018004f140     libucrt:get_qualified_locale.obj
 0002:00009148       ??_C@_1BC@LLOKLNP@?$AAa?$AAm?$AAe?$AAr?$AAi?$AAc?$AAa?$AAn@ 000000018004f148     libucrt:get_qualified_locale.obj
 0002:00009160       ??_C@_1CC@HEIGCDGG@?$AAa?$AAm?$AAe?$AAr?$AAi?$AAc?$AAa?$AAn?$AA?5?$AAe?$AAn?$AAg?$AAl?$AAi?$AAs@ 000000018004f160     libucrt:get_qualified_locale.obj
 0002:00009188       ??_C@_1CC@IHCNOMIN@?$AAa?$AAm?$AAe?$AAr?$AAi?$AAc?$AAa?$AAn?$AA?9?$AAe?$AAn?$AAg?$AAl?$AAi?$AAs@ 000000018004f188     libucrt:get_qualified_locale.obj
 0002:000091b0       ??_C@_1BG@GKAGPCGG@?$AAa?$AAu?$AAs?$AAt?$AAr?$AAa?$AAl?$AAi?$AAa?$AAn@ 000000018004f1b0     libucrt:get_qualified_locale.obj
 0002:000091c8       ??_C@_1BA@GMENCENF@?$AAb?$AAe?$AAl?$AAg?$AAi?$AAa?$AAn@ 000000018004f1c8     libucrt:get_qualified_locale.obj
 0002:000091d8       ??_C@_1BC@PJMIIAAN@?$AAc?$AAa?$AAn?$AAa?$AAd?$AAi?$AAa?$AAn@ 000000018004f1d8     libucrt:get_qualified_locale.obj
 0002:000091f0       ??_C@_17NOIMNFBF@?$AAc?$AAh?$AAh@ 000000018004f1f0     libucrt:get_qualified_locale.obj
 0002:000091f8       ??_C@_17GGDALCHA@?$AAc?$AAh?$AAi@ 000000018004f1f8     libucrt:get_qualified_locale.obj
 0002:00009200       ??_C@_1BA@NPNJKIBL@?$AAc?$AAh?$AAi?$AAn?$AAe?$AAs?$AAe@ 000000018004f200     libucrt:get_qualified_locale.obj
 0002:00009210       ??_C@_1CC@DINBAMMJ@?$AAc?$AAh?$AAi?$AAn?$AAe?$AAs?$AAe?$AA?9?$AAh?$AAo?$AAn?$AAg?$AAk?$AAo?$AAn@ 000000018004f210     libucrt:get_qualified_locale.obj
 0002:00009238       ??_C@_1CG@IOBJPACO@?$AAc?$AAh?$AAi?$AAn?$AAe?$AAs?$AAe?$AA?9?$AAs?$AAi?$AAm?$AAp?$AAl?$AAi?$AAf@ 000000018004f238     libucrt:get_qualified_locale.obj
 0002:00009260       ??_C@_1CE@GAJNDCKG@?$AAc?$AAh?$AAi?$AAn?$AAe?$AAs?$AAe?$AA?9?$AAs?$AAi?$AAn?$AAg?$AAa?$AAp?$AAo@ 000000018004f260     libucrt:get_qualified_locale.obj
 0002:00009288       ??_C@_1CI@PAJPIOOD@?$AAc?$AAh?$AAi?$AAn?$AAe?$AAs?$AAe?$AA?9?$AAt?$AAr?$AAa?$AAd?$AAi?$AAt?$AAi@ 000000018004f288     libucrt:get_qualified_locale.obj
 0002:000092b0       ??_C@_1BM@NILJBMMD@?$AAd?$AAu?$AAt?$AAc?$AAh?$AA?9?$AAb?$AAe?$AAl?$AAg?$AAi?$AAa?$AAn@ 000000018004f2b0     libucrt:get_qualified_locale.obj
 0002:000092d0       ??_C@_1CC@OOJPJNEJ@?$AAe?$AAn?$AAg?$AAl?$AAi?$AAs?$AAh?$AA?9?$AAa?$AAm?$AAe?$AAr?$AAi?$AAc?$AAa@ 000000018004f2d0     libucrt:get_qualified_locale.obj
 0002:000092f8       ??_C@_1BI@IOLFEEM@?$AAe?$AAn?$AAg?$AAl?$AAi?$AAs?$AAh?$AA?9?$AAa?$AAu?$AAs@ 000000018004f2f8     libucrt:get_qualified_locale.obj
 0002:00009310       ??_C@_1BO@HFFNLENJ@?$AAe?$AAn?$AAg?$AAl?$AAi?$AAs?$AAh?$AA?9?$AAb?$AAe?$AAl?$AAi?$AAz?$AAe@ 000000018004f310     libucrt:get_qualified_locale.obj
 0002:00009330       ??_C@_1BI@HAPKJMPO@?$AAe?$AAn?$AAg?$AAl?$AAi?$AAs?$AAh?$AA?9?$AAc?$AAa?$AAn@ 000000018004f330     libucrt:get_qualified_locale.obj
 0002:00009348       ??_C@_1CE@HLNDMIOJ@?$AAe?$AAn?$AAg?$AAl?$AAi?$AAs?$AAh?$AA?9?$AAc?$AAa?$AAr?$AAi?$AAb?$AAb?$AAe@ 000000018004f348     libucrt:get_qualified_locale.obj
 0002:00009370       ??_C@_1BI@LDHJHHAC@?$AAe?$AAn?$AAg?$AAl?$AAi?$AAs?$AAh?$AA?9?$AAi?$AAr?$AAe@ 000000018004f370     libucrt:get_qualified_locale.obj
 0002:00009388       ??_C@_1CA@NJMMCFOC@?$AAe?$AAn?$AAg?$AAl?$AAi?$AAs?$AAh?$AA?9?$AAj?$AAa?$AAm?$AAa?$AAi?$AAc?$AAa@ 000000018004f388     libucrt:get_qualified_locale.obj
 0002:000093a8       ??_C@_1BG@BHJEBBGG@?$AAe?$AAn?$AAg?$AAl?$AAi?$AAs?$AAh?$AA?9?$AAn?$AAz@ 000000018004f3a8     libucrt:get_qualified_locale.obj
 0002:000093c0       ??_C@_1CK@FGOEJJCO@?$AAe?$AAn?$AAg?$AAl?$AAi?$AAs?$AAh?$AA?9?$AAs?$AAo?$AAu?$AAt?$AAh?$AA?5?$AAa@ 000000018004f3c0     libucrt:get_qualified_locale.obj
 0002:000093f0       ??_C@_1DE@PDBJPCJ@?$AAe?$AAn?$AAg?$AAl?$AAi?$AAs?$AAh?$AA?9?$AAt?$AAr?$AAi?$AAn?$AAi?$AAd?$AAa@ 000000018004f3f0     libucrt:get_qualified_locale.obj
 0002:00009428       ??_C@_1BG@JGCANDME@?$AAe?$AAn?$AAg?$AAl?$AAi?$AAs?$AAh?$AA?9?$AAu?$AAk@ 000000018004f428     libucrt:get_qualified_locale.obj
 0002:00009440       ??_C@_1BG@DINKMLE@?$AAe?$AAn?$AAg?$AAl?$AAi?$AAs?$AAh?$AA?9?$AAu?$AAs@ 000000018004f440     libucrt:get_qualified_locale.obj
 0002:00009458       ??_C@_1BI@NMFDBHJE@?$AAe?$AAn?$AAg?$AAl?$AAi?$AAs?$AAh?$AA?9?$AAu?$AAs?$AAa@ 000000018004f458     libucrt:get_qualified_locale.obj
 0002:00009470       ??_C@_1BO@OIHKJKII@?$AAf?$AAr?$AAe?$AAn?$AAc?$AAh?$AA?9?$AAb?$AAe?$AAl?$AAg?$AAi?$AAa?$AAn@ 000000018004f470     libucrt:get_qualified_locale.obj
 0002:00009490       ??_C@_1CA@NKAELJKI@?$AAf?$AAr?$AAe?$AAn?$AAc?$AAh?$AA?9?$AAc?$AAa?$AAn?$AAa?$AAd?$AAi?$AAa?$AAn@ 000000018004f490     libucrt:get_qualified_locale.obj
 0002:000094b0       ??_C@_1CE@MGKCNLGN@?$AAf?$AAr?$AAe?$AAn?$AAc?$AAh?$AA?9?$AAl?$AAu?$AAx?$AAe?$AAm?$AAb?$AAo?$AAu@ 000000018004f4b0     libucrt:get_qualified_locale.obj
 0002:000094d8       ??_C@_1BK@CEGEAILM@?$AAf?$AAr?$AAe?$AAn?$AAc?$AAh?$AA?9?$AAs?$AAw?$AAi?$AAs?$AAs@ 000000018004f4d8     libucrt:get_qualified_locale.obj
 0002:000094f8       ??_C@_1CA@PAFKEOCC@?$AAg?$AAe?$AAr?$AAm?$AAa?$AAn?$AA?9?$AAa?$AAu?$AAs?$AAt?$AAr?$AAi?$AAa?$AAn@ 000000018004f4f8     libucrt:get_qualified_locale.obj
 0002:00009518       ??_C@_1CI@HCFHGOFD@?$AAg?$AAe?$AAr?$AAm?$AAa?$AAn?$AA?9?$AAl?$AAi?$AAc?$AAh?$AAt?$AAe?$AAn?$AAs@ 000000018004f518     libucrt:get_qualified_locale.obj
 0002:00009540       ??_C@_1CE@FEDDNPDG@?$AAg?$AAe?$AAr?$AAm?$AAa?$AAn?$AA?9?$AAl?$AAu?$AAx?$AAe?$AAm?$AAb?$AAo?$AAu@ 000000018004f540     libucrt:get_qualified_locale.obj
 0002:00009568       ??_C@_1BK@LIMINNMN@?$AAg?$AAe?$AAr?$AAm?$AAa?$AAn?$AA?9?$AAs?$AAw?$AAi?$AAs?$AAs@ 000000018004f568     libucrt:get_qualified_locale.obj
 0002:00009588       ??_C@_1BM@LGMDBEPD@?$AAi?$AAr?$AAi?$AAs?$AAh?$AA?9?$AAe?$AAn?$AAg?$AAl?$AAi?$AAs?$AAh@ 000000018004f588     libucrt:get_qualified_locale.obj
 0002:000095a8       ??_C@_1BM@NNCFBAEE@?$AAi?$AAt?$AAa?$AAl?$AAi?$AAa?$AAn?$AA?9?$AAs?$AAw?$AAi?$AAs?$AAs@ 000000018004f5a8     libucrt:get_qualified_locale.obj
 0002:000095c8       ??_C@_1BE@FEDJNPIB@?$AAn?$AAo?$AAr?$AAw?$AAe?$AAg?$AAi?$AAa?$AAn@ 000000018004f5c8     libucrt:get_qualified_locale.obj
 0002:000095e0       ??_C@_1CC@CILKDEIE@?$AAn?$AAo?$AAr?$AAw?$AAe?$AAg?$AAi?$AAa?$AAn?$AA?9?$AAb?$AAo?$AAk?$AAm?$AAa@ 000000018004f5e0     libucrt:get_qualified_locale.obj
 0002:00009608       ??_C@_1CE@DHMMHEPL@?$AAn?$AAo?$AAr?$AAw?$AAe?$AAg?$AAi?$AAa?$AAn?$AA?9?$AAn?$AAy?$AAn?$AAo?$AAr@ 000000018004f608     libucrt:get_qualified_locale.obj
 0002:00009630       ??_C@_1CK@OPNMHECD@?$AAp?$AAo?$AAr?$AAt?$AAu?$AAg?$AAu?$AAe?$AAs?$AAe?$AA?9?$AAb?$AAr?$AAa?$AAz@ 000000018004f630     libucrt:get_qualified_locale.obj
 0002:00009660       ??_C@_1CE@KEEHCDB@?$AAs?$AAp?$AAa?$AAn?$AAi?$AAs?$AAh?$AA?9?$AAa?$AAr?$AAg?$AAe?$AAn?$AAt?$AAi@ 000000018004f660     libucrt:get_qualified_locale.obj
 0002:00009688       ??_C@_1CA@GIAOLHJD@?$AAs?$AAp?$AAa?$AAn?$AAi?$AAs?$AAh?$AA?9?$AAb?$AAo?$AAl?$AAi?$AAv?$AAi?$AAa@ 000000018004f688     libucrt:get_qualified_locale.obj
 0002:000096a8       ??_C@_1BM@OJNDFNPD@?$AAs?$AAp?$AAa?$AAn?$AAi?$AAs?$AAh?$AA?9?$AAc?$AAh?$AAi?$AAl?$AAe@ 000000018004f6a8     libucrt:get_qualified_locale.obj
 0002:000096c8       ??_C@_1CC@OCOLPALL@?$AAs?$AAp?$AAa?$AAn?$AAi?$AAs?$AAh?$AA?9?$AAc?$AAo?$AAl?$AAo?$AAm?$AAb?$AAi@ 000000018004f6c8     libucrt:get_qualified_locale.obj
 0002:000096f0       ??_C@_1CG@BPOFMKBB@?$AAs?$AAp?$AAa?$AAn?$AAi?$AAs?$AAh?$AA?9?$AAc?$AAo?$AAs?$AAt?$AAa?$AA?5?$AAr@ 000000018004f6f0     libucrt:get_qualified_locale.obj
 0002:00009718       ??_C@_1DG@IGOBAPBB@?$AAs?$AAp?$AAa?$AAn?$AAi?$AAs?$AAh?$AA?9?$AAd?$AAo?$AAm?$AAi?$AAn?$AAi?$AAc@ 000000018004f718     libucrt:get_qualified_locale.obj
 0002:00009750       ??_C@_1CA@JHAPGEGI@?$AAs?$AAp?$AAa?$AAn?$AAi?$AAs?$AAh?$AA?9?$AAe?$AAc?$AAu?$AAa?$AAd?$AAo?$AAr@ 000000018004f750     libucrt:get_qualified_locale.obj
 0002:00009770       ??_C@_1CI@LAPALJPP@?$AAs?$AAp?$AAa?$AAn?$AAi?$AAs?$AAh?$AA?9?$AAe?$AAl?$AA?5?$AAs?$AAa?$AAl?$AAv@ 000000018004f770     libucrt:get_qualified_locale.obj
 0002:00009798       ??_C@_1CE@PDGBOFOM@?$AAs?$AAp?$AAa?$AAn?$AAi?$AAs?$AAh?$AA?9?$AAg?$AAu?$AAa?$AAt?$AAe?$AAm?$AAa@ 000000018004f798     libucrt:get_qualified_locale.obj
 0002:000097c0       ??_C@_1CC@NBEBAODI@?$AAs?$AAp?$AAa?$AAn?$AAi?$AAs?$AAh?$AA?9?$AAh?$AAo?$AAn?$AAd?$AAu?$AAr?$AAa@ 000000018004f7c0     libucrt:get_qualified_locale.obj
 0002:000097e8       ??_C@_1CA@LLKGHBMF@?$AAs?$AAp?$AAa?$AAn?$AAi?$AAs?$AAh?$AA?9?$AAm?$AAe?$AAx?$AAi?$AAc?$AAa?$AAn@ 000000018004f7e8     libucrt:get_qualified_locale.obj
 0002:00009808       ??_C@_1BO@LKNDOIGD@?$AAs?$AAp?$AAa?$AAn?$AAi?$AAs?$AAh?$AA?9?$AAm?$AAo?$AAd?$AAe?$AAr?$AAn@ 000000018004f808     libucrt:get_qualified_locale.obj
 0002:00009828       ??_C@_1CE@NMDMOEEB@?$AAs?$AAp?$AAa?$AAn?$AAi?$AAs?$AAh?$AA?9?$AAn?$AAi?$AAc?$AAa?$AAr?$AAa?$AAg@ 000000018004f828     libucrt:get_qualified_locale.obj
 0002:00009850       ??_C@_1BO@LLCBEJGB@?$AAs?$AAp?$AAa?$AAn?$AAi?$AAs?$AAh?$AA?9?$AAp?$AAa?$AAn?$AAa?$AAm?$AAa@ 000000018004f850     libucrt:get_qualified_locale.obj
 0002:00009870       ??_C@_1CC@FKPGGIHO@?$AAs?$AAp?$AAa?$AAn?$AAi?$AAs?$AAh?$AA?9?$AAp?$AAa?$AAr?$AAa?$AAg?$AAu?$AAa@ 000000018004f870     libucrt:get_qualified_locale.obj
 0002:00009898       ??_C@_1BK@CDEIHOOP@?$AAs?$AAp?$AAa?$AAn?$AAi?$AAs?$AAh?$AA?9?$AAp?$AAe?$AAr?$AAu@ 000000018004f898     libucrt:get_qualified_locale.obj
 0002:000098b8       ??_C@_1CI@GAHAKKGP@?$AAs?$AAp?$AAa?$AAn?$AAi?$AAs?$AAh?$AA?9?$AAp?$AAu?$AAe?$AAr?$AAt?$AAo?$AA?5@ 000000018004f8b8     libucrt:get_qualified_locale.obj
 0002:000098e0       ??_C@_1CA@NKJBCAGP@?$AAs?$AAp?$AAa?$AAn?$AAi?$AAs?$AAh?$AA?9?$AAu?$AAr?$AAu?$AAg?$AAu?$AAa?$AAy@ 000000018004f8e0     libucrt:get_qualified_locale.obj
 0002:00009900       ??_C@_1CE@ODILCONM@?$AAs?$AAp?$AAa?$AAn?$AAi?$AAs?$AAh?$AA?9?$AAv?$AAe?$AAn?$AAe?$AAz?$AAu?$AAe@ 000000018004f900     libucrt:get_qualified_locale.obj
 0002:00009928       ??_C@_1CA@OBNMCGFO@?$AAs?$AAw?$AAe?$AAd?$AAi?$AAs?$AAh?$AA?9?$AAf?$AAi?$AAn?$AAl?$AAa?$AAn?$AAd@ 000000018004f928     libucrt:get_qualified_locale.obj
 0002:00009948       ??_C@_1M@PIPDDPPI@?$AAs?$AAw?$AAi?$AAs?$AAs@ 000000018004f948     libucrt:get_qualified_locale.obj
 0002:00009954       ??_C@_15GMFIMNFM@?$AAu?$AAs@ 000000018004f954     libucrt:get_qualified_locale.obj
 0002:00009960       ??_C@_17HAEBFAGL@?$AAu?$AAs?$AAa@ 000000018004f960     libucrt:get_qualified_locale.obj
 0002:00009968       ??_C@_1BA@DPFJEPHB@?$AAa?$AAm?$AAe?$AAr?$AAi?$AAc?$AAa@ 000000018004f968     libucrt:get_qualified_locale.obj
 0002:00009978       ??_C@_1BA@ELOGGFK@?$AAb?$AAr?$AAi?$AAt?$AAa?$AAi?$AAn@ 000000018004f978     libucrt:get_qualified_locale.obj
 0002:00009988       ??_C@_1M@GHBGIGDA@?$AAc?$AAh?$AAi?$AAn?$AAa@ 000000018004f988     libucrt:get_qualified_locale.obj
 0002:00009998       ??_C@_1M@NCHEJOPO@?$AAc?$AAz?$AAe?$AAc?$AAh@ 000000018004f998     libucrt:get_qualified_locale.obj
 0002:000099a8       ??_C@_1BA@BKPAPBLA@?$AAe?$AAn?$AAg?$AAl?$AAa?$AAn?$AAd@ 000000018004f9a8     libucrt:get_qualified_locale.obj
 0002:000099b8       ??_C@_1BM@HKBCKIPC@?$AAg?$AAr?$AAe?$AAa?$AAt?$AA?5?$AAb?$AAr?$AAi?$AAt?$AAa?$AAi?$AAn@ 000000018004f9b8     libucrt:get_qualified_locale.obj
 0002:000099d8       ??_C@_1BA@PPCHPGJB@?$AAh?$AAo?$AAl?$AAl?$AAa?$AAn?$AAd@ 000000018004f9d8     libucrt:get_qualified_locale.obj
 0002:000099e8       ??_C@_1BE@JBMPEGDG@?$AAh?$AAo?$AAn?$AAg?$AA?9?$AAk?$AAo?$AAn?$AAg@ 000000018004f9e8     libucrt:get_qualified_locale.obj
 0002:00009a00       ??_C@_1BI@KOELBBPJ@?$AAn?$AAe?$AAw?$AA?9?$AAz?$AAe?$AAa?$AAl?$AAa?$AAn?$AAd@ 000000018004fa00     libucrt:get_qualified_locale.obj
 0002:00009a18       ??_C@_15HIEBHAIO@?$AAn?$AAz@ 000000018004fa18     libucrt:get_qualified_locale.obj
 0002:00009a20       ??_C@_1BC@CHBCPFPI@?$AAp?$AAr?$AA?5?$AAc?$AAh?$AAi?$AAn?$AAa@ 000000018004fa20     libucrt:get_qualified_locale.obj
 0002:00009a38       ??_C@_1BC@JAOIIFKD@?$AAp?$AAr?$AA?9?$AAc?$AAh?$AAi?$AAn?$AAa@ 000000018004fa38     libucrt:get_qualified_locale.obj
 0002:00009a50       ??_C@_1BI@BEHPPHKC@?$AAp?$AAu?$AAe?$AAr?$AAt?$AAo?$AA?9?$AAr?$AAi?$AAc?$AAo@ 000000018004fa50     libucrt:get_qualified_locale.obj
 0002:00009a68       ??_C@_1O@PAEOFKDI@?$AAs?$AAl?$AAo?$AAv?$AAa?$AAk@ 000000018004fa68     libucrt:get_qualified_locale.obj
 0002:00009a78       ??_C@_1BK@FIHMCKAM@?$AAs?$AAo?$AAu?$AAt?$AAh?$AA?5?$AAa?$AAf?$AAr?$AAi?$AAc?$AAa@ 000000018004fa78     libucrt:get_qualified_locale.obj
 0002:00009a98       ??_C@_1BI@NAEOODKB@?$AAs?$AAo?$AAu?$AAt?$AAh?$AA?5?$AAk?$AAo?$AAr?$AAe?$AAa@ 000000018004fa98     libucrt:get_qualified_locale.obj
 0002:00009ab0       ??_C@_1BK@FBDGGIFF@?$AAs?$AAo?$AAu?$AAt?$AAh?$AA?9?$AAa?$AAf?$AAr?$AAi?$AAc?$AAa@ 000000018004fab0     libucrt:get_qualified_locale.obj
 0002:00009ad0       ??_C@_1BI@GHLEJDPK@?$AAs?$AAo?$AAu?$AAt?$AAh?$AA?9?$AAk?$AAo?$AAr?$AAe?$AAa@ 000000018004fad0     libucrt:get_qualified_locale.obj
 0002:00009ae8       ??_C@_1CE@PLHLOMJF@?$AAt?$AAr?$AAi?$AAn?$AAi?$AAd?$AAa?$AAd?$AA?5?$AA?$CG?$AA?5?$AAt?$AAo?$AAb?$AAa@ 000000018004fae8     libucrt:get_qualified_locale.obj
 0002:00009b10       ??_C@_1BO@MODIMHHI@?$AAu?$AAn?$AAi?$AAt?$AAe?$AAd?$AA?9?$AAk?$AAi?$AAn?$AAg?$AAd?$AAo?$AAm@ 000000018004fb10     libucrt:get_qualified_locale.obj
 0002:00009b30       ??_C@_1BM@FFHJONBJ@?$AAu?$AAn?$AAi?$AAt?$AAe?$AAd?$AA?9?$AAs?$AAt?$AAa?$AAt?$AAe?$AAs@ 000000018004fb30     libucrt:get_qualified_locale.obj
 0002:00009b50       ??_C@_19MPDNHKDG@?$AAu?$AAt?$AAf?$AA8@ 000000018004fb50     libucrt:get_qualified_locale.obj
 0002:00009b60       ??_C@_17DNCLJFIF@?$AAA?$AAC?$AAP@ 000000018004fb60     libucrt:get_qualified_locale.obj
 0002:00009b68       ??_C@_1M@FPEIIFAM@?$AAu?$AAt?$AAf?$AA?9?$AA8@ 000000018004fb68     libucrt:get_qualified_locale.obj
 0002:00009b78       ??_C@_17CIKBIHLH@?$AAO?$AAC?$AAP@ 000000018004fb78     libucrt:get_qualified_locale.obj
 0002:00009b80       __rglangidNotDefault       000000018004fb80     libucrt:getqloc_downlevel.obj
 0002:00009fb8       ??_C@_1BA@BALFACEM@?$AAC?$AAO?$AAN?$AAO?$AAU?$AAT?$AA$@ 000000018004ffb8     libucrt:initcon.obj
 0002:00009fc8       ??_C@_0BC@EOODALEL@Unknown?5exception@ 000000018004ffc8     format.obj
 0002:00009fe0       ??_C@_0BF@KINCDENJ@bad?5array?5new?5length@ 000000018004ffe0     format.obj
 0002:00009ff8       ??_C@_08EPJLHIJG@bad?5cast@ 000000018004fff8     format.obj
 0002:0000a008       ??_C@_0BA@JFNIOLAK@string?5too?5long@ 0000000180050008     format.obj
 0002:0000a018       ??_C@_00CNPNBAHC@@         0000000180050018     format.obj
 0002:0000a020       ??_C@_0MJ@HFBCCPGP@0001020304050607080910111213141@ 0000000180050020     format.obj
 0002:0000a0f0       ??_C@_0BA@ELKIONDK@bad?5locale?5name@ 00000001800500f0     format.obj
 0002:0000a100       ??_C@_05LAPONLG@false@     0000000180050100     format.obj
 0002:0000a108       ??_C@_04LOAJBDKD@true@     0000000180050108     format.obj
 0002:0000a110       ??_C@_0BD@DBEDGLNA@argument?5not?5found@ 0000000180050110     format.obj
 0002:0000a128       ??_C@_0BN@JNLAGDD@missing?5?8?$HN?8?5in?5format?5string@ 0000000180050128     format.obj
 0002:0000a148       ??_C@_0BH@IEEDMHI@string?5pointer?5is?5null@ 0000000180050148     format.obj
 0002:0000a160       ??_C@_0DJ@LMIJFHJI@cannot?5switch?5from?5automatic?5to@ 0000000180050160     format.obj
 0002:0000a1a0       ??_C@_0DJ@GHJONFIH@cannot?5switch?5from?5manual?5to?5au@ 00000001800501a0     format.obj
 0002:0000a1e0       ??_C@_0BH@CIKPCHEG@invalid?5type?5specifier@ 00000001800501e0     format.obj
 0002:0000a1f8       ??_C@_0BP@NMGMJOEM@unmatched?5?8?$HN?8?5in?5format?5string@ 00000001800501f8     format.obj
 0002:0000a218       ??_C@_0BG@PEJKJNLA@invalid?5format?5string@ 0000000180050218     format.obj
 0002:0000a230       ??_C@_0BJ@JNDNOEDN@unknown?5format?5specifier@ 0000000180050230     format.obj
 0002:0000a250       ??_C@_0BL@KNEDAEPA@invalid?5fill?5character?5?8?$HL?8@ 0000000180050250     format.obj
 0002:0000a270       ??_C@_0CL@CFEEEDMP@format?5specifier?5requires?5numer@ 0000000180050270     format.obj
 0002:0000a2a0       ??_C@_0BC@MDEIBHGE@number?5is?5too?5big@ 00000001800502a0     format.obj
 0002:0000a2b8       ??_C@_0CK@IBNNAPH@format?5specifier?5requires?5signe@ 00000001800502b8     format.obj
 0002:0000a2e8       ??_C@_0N@EFEDKJEI@invalid?5fill@ 00000001800502e8     format.obj
 0002:0000a2f8       ??_C@_0BM@IEKLBNBK@missing?5precision?5specifier@ 00000001800502f8     format.obj
 0002:0000a318       ??_C@_0CC@ELFJMMCC@invalid?5format?5specifier?5for?5ch@ 0000000180050318     format.obj
 0002:0000a340       ??_C@_0CN@KMEDLGAJ@precision?5not?5allowed?5for?5this?5@ 0000000180050340     format.obj
 0002:0000a370       ??_C@_03OEIAHPBN@INF@      0000000180050370     format.obj
 0002:0000a374       ??_C@_03OJHLLCGB@inf@      0000000180050374     format.obj
 0002:0000a378       ??_C@_03LKNCIKJB@NAN@      0000000180050378     format.obj
 0002:0000a37c       ??_C@_03LHCJEHON@nan@      000000018005037c     format.obj
 0002:0000a380       ??_C@_04MKBJPCKC@?$AA?9?$CL?5@ 0000000180050380     format.obj
 0002:0000a388       ??_C@_04MKAMHODJ@?$BP?$BP?$AA?$AB@ 0000000180050388     format.obj
 0002:0000a390       ??_C@_04CILMHOGK@?$AA?$BP?$AA?$AB@ 0000000180050390     format.obj
 0002:0000a398       ??_C@_0BB@JGGOGLEG@0123456789ABCDEF@ 0000000180050398     format.obj
 0002:0000a3b0       ??_C@_0BB@JCEFLFJE@0123456789abcdef@ 00000001800503b0     format.obj
 0002:0000a3c8       ??_C@_0P@DAPDPGEO@negative?5width@ 00000001800503c8     format.obj
 0002:0000a3d8       ??_C@_0BD@PKKFPMLC@negative?5precision@ 00000001800503d8     format.obj
 0002:0000a3f0       ??_C@_0BF@KEAPHPPE@width?5is?5not?5integer@ 00000001800503f0     format.obj
 0002:0000a408       ??_C@_0BJ@KKLAKOOL@precision?5is?5not?5integer@ 0000000180050408     format.obj
 0002:0000a430       ?pow10_significands@?1??get_cached_power@?$cache_accessor@N@dragonbox@detail@v8@fmt@@SA?AUuint128_wrapper@456@H@Z@4QBU7456@B 0000000180050430     format.obj
 0002:0000a5a0       ?pow10_significands@?1??get_cached_power@?$cache_accessor@M@dragonbox@detail@v8@fmt@@SA_KH@Z@4QB_KB 00000001800505a0     format.obj
 0002:0000a818       ??_7?$basic_memory_buffer@_W$0BPE@V?$allocator@_W@std@@@v8@fmt@@6B@ 0000000180050818     format.obj
 0002:0000a820       ?divtest_table@?1??divisible_by_power_of_5@dragonbox@detail@v8@fmt@@YA_NIH@Z@4QBU?$divtest_table_entry@I@2345@B 0000000180050820     format.obj
 0002:0000a880       ??_7?$basic_memory_buffer@H$0BPE@V?$allocator@H@std@@@v8@fmt@@6B@ 0000000180050880     format.obj
 0002:0000a890       ?power_of_10_64@?$basic_impl_data@X@detail@v8@fmt@@2QB_KB 0000000180050890     format.obj
 0002:0000a930       ?pow10_significands@?$basic_impl_data@X@detail@v8@fmt@@2QB_KB 0000000180050930     format.obj
 0002:0000abf0       ?pow10_exponents@?$basic_impl_data@X@detail@v8@fmt@@2QBFB 0000000180050bf0     format.obj
 0002:0000aca0       ?powers_of_5_64@?1??get_cached_power@?$cache_accessor@N@dragonbox@detail@v8@fmt@@SA?AUuint128_wrapper@456@H@Z@4QB_KB 0000000180050ca0     format.obj
 0002:0000ad80       ??_7format_error@v8@fmt@@6B@ 0000000180050d80     format.obj
 0002:0000ad90       ?bsr2log10@?1??do_count_digits@detail@v8@fmt@@YAH_K@Z@4QBEB 0000000180050d90     format.obj
 0002:0000add0       ?table@?1??do_count_digits@detail@v8@fmt@@YAHI@Z@4QB_KB 0000000180050dd0     format.obj
 0002:0000aed0       ?zero_or_powers_of_10@?1??do_count_digits@detail@v8@fmt@@YAH_K@Z@4QB_KB 0000000180050ed0     format.obj
 0002:0000af80       ?pow10_recovery_errors@?1??get_cached_power@?$cache_accessor@N@dragonbox@detail@v8@fmt@@SA?AUuint128_wrapper@456@H@Z@4QBIB 0000000180050f80     format.obj
 0002:0000b028       ??_7?$basic_memory_buffer@I$0CA@V?$allocator@I@std@@@v8@fmt@@6B@ 0000000180051028     format.obj
 0002:0000b030       ?divtest_table@?1??divisible_by_power_of_5@dragonbox@detail@v8@fmt@@YA_N_KH@Z@4QBU?$divtest_table_entry@_K@2345@B 0000000180051030     format.obj
 0002:0000b1b8       ??_7?$basic_memory_buffer@D$0BPE@V?$allocator@D@std@@@v8@fmt@@6B@ 00000001800511b8     format.obj
 0002:0000b1c0       ??_C@_1O@ECECHNAE@?$AA?$DM?$AAp?$AAi?$AAp?$AAe?$AA?$DO@ 00000001800511c0     handles.obj
 0002:0000b1d0       ??_C@_11LOCGONAA@@         00000001800511d0     handles.obj
 0002:0000b1d8       ??_C@_1BA@NMDNJJOO@?$AAP?$AAr?$AAo?$AAc?$AAe?$AAs?$AAs@ 00000001800511d8     handles.obj
 0002:0000b1e8       ??_C@_1O@CDOGJPJJ@?$AAT?$AAh?$AAr?$AAe?$AAa?$AAd@ 00000001800511e8     handles.obj
 0002:0000b1f8       ??_C@_17KACEIPNC@?$AAK?$AAe?$AAy@ 00000001800511f8     handles.obj
 0002:0000b200       ??_C@_19DDLLJDOO@?$AAF?$AAi?$AAl?$AAe@ 0000000180051200     handles.obj
 0002:0000b210       ??_C@_1BE@FGECLHKD@?$AA?$HL?$AA0?$AA?$HN?$AA?5?$AA?$CI?$AA?$HL?$AA1?$AA?$HN?$AA?$CJ@ 0000000180051210     handles.obj
 0002:0000b228       ??_C@_1BC@HBCEGEJN@?$AAT?$AAI?$AAD?$AA?3?$AA?5?$AA?$HL?$AA0?$AA?$HN@ 0000000180051228     handles.obj
 0002:0000b240       ??_C@_1BE@ELICABCK@?$AA?$DM?$AAu?$AAn?$AAk?$AAn?$AAo?$AAw?$AAn?$AA?$DO@ 0000000180051240     handles.obj
 0002:0000b258       ??_C@_1BG@OKCBELMP@?$AA?2?$AAR?$AAE?$AAG?$AAI?$AAS?$AAT?$AAR?$AAY?$AA?2@ 0000000180051258     handles.obj
 0002:0000b270       ??_C@_19KGHAHCFG@?$AAU?$AAS?$AAE?$AAR@ 0000000180051270     handles.obj
 0002:0000b280       ??_C@_1DC@OIDKFHBF@?$AAM?$AAA?$AAC?$AAH?$AAI?$AAN?$AAE?$AA?2?$AAS?$AAO?$AAF?$AAT?$AAW?$AAA?$AAR@ 0000000180051280     handles.obj
 0002:0000b2b8       ??_C@_1BA@INBMCOAP@?$AAM?$AAA?$AAC?$AAH?$AAI?$AAN?$AAE@ 00000001800512b8     handles.obj
 0002:0000b2c8       ??_C@_1BC@DCCOJFBE@?$AA_?$AAC?$AAL?$AAA?$AAS?$AAS?$AAE?$AAS@ 00000001800512c8     handles.obj
 0002:0000b2dc       ??_C@_13FPGAJAPJ@?$AA?2@   00000001800512dc     handles.obj
 0002:0000b2e0       ??_C@_19DIHHCHDI@?$AAH?$AAK?$AAU?$AA?2@ 00000001800512e0     handles.obj
 0002:0000b2f0       ??_C@_19JAPAIJDE@?$AAH?$AAK?$AAC?$AAU@ 00000001800512f0     handles.obj
 0002:0000b300       ??_C@_1BK@OEABCBLA@?$AAH?$AAK?$AAC?$AAU?$AA?2?$AAC?$AAl?$AAa?$AAs?$AAs?$AAe?$AAs@ 0000000180051300     handles.obj
 0002:0000b320       ??_C@_17PJOJPMPB@?$AAH?$AAK?$AAU@ 0000000180051320     handles.obj
 0002:0000b328       ??_C@_19NCHLBIN@?$AAH?$AAK?$AAC?$AAR@ 0000000180051328     handles.obj
 0002:0000b338       ??_C@_19PEALEEJB@?$AAH?$AAK?$AAL?$AAM@ 0000000180051338     handles.obj
 0002:0000b348       ??_C@_1DM@NGIMPLFP@?$AA?6?$AA?$HL?$AA0?$AA?$HN?$AA?3?$AA?6?$AA?$HL?$AA1?$AA?3?$AA6?$AA?$HN?$AA?5?$AA?$HL?$AA2?$AA?3@ 0000000180051348     handles.obj
 0002:0000b388       ??_C@_1DG@HOLPNCNP@?$AA?$HL?$AA0?$AA?3?$AA6?$AAX?$AA?$HN?$AA?5?$AA?$HL?$AA1?$AA?3?$AA0?$AA8?$AAX?$AA?$HN?$AA?5@ 0000000180051388     handles.obj
 0002:0000b3e8       ??_C@_1O@BJPKKLLM@?$AAC?$AAo?$AAn?$AAf?$AAi?$AAg@ 00000001800513e8     Pcfg.obj
 0002:0000b3f8       ??_C@_1BO@NGDOFANC@?$AAA?$AAd?$AAd?$AAT?$AAo?$AAD?$AAi?$AAs?$AAk?$AAs?$AAM?$AAe?$AAn?$AAu@ 00000001800513f8     Pcfg.obj
 0002:0000b418       ??_C@_1CC@PNNAOHJC@?$AAA?$AAd?$AAd?$AAT?$AAo?$AAP?$AAl?$AAu?$AAg?$AAi?$AAn?$AAs?$AAM?$AAe?$AAn@ 0000000180051418     Pcfg.obj
 0002:0000b440       ??_C@_1CE@JIPJNDMD@?$AAE?$AAx?$AAp?$AAo?$AAr?$AAt?$AAE?$AAn?$AAv?$AAi?$AAr?$AAo?$AAn?$AAm?$AAe@ 0000000180051440     Pcfg.obj
 0002:0000b468       ??_C@_1CC@OABICAMP@?$AAE?$AAx?$AAp?$AAo?$AAr?$AAt?$AAM?$AAo?$AAd?$AAu?$AAl?$AAe?$AAI?$AAn?$AAf@ 0000000180051468     Pcfg.obj
 0002:0000b490       ??_C@_1CI@OFLGHPDG@?$AAE?$AAx?$AAp?$AAo?$AAr?$AAt?$AAM?$AAo?$AAd?$AAu?$AAl?$AAe?$AAV?$AAe?$AAr@ 0000000180051490     Pcfg.obj
 0002:0000b4b8       ??_C@_1CE@GNMOKOAL@?$AAE?$AAx?$AAp?$AAo?$AAr?$AAt?$AAP?$AAe?$AAr?$AAf?$AAo?$AAr?$AAm?$AAa?$AAn@ 00000001800514b8     Pcfg.obj
 0002:0000b4e0       ??_C@_1BM@KMCHODLM@?$AAE?$AAx?$AAp?$AAo?$AAr?$AAt?$AAH?$AAa?$AAn?$AAd?$AAl?$AAe?$AAs@ 00000001800514e0     Pcfg.obj
 0002:0000b500       ??_C@_1CK@CLFOOHFA@?$AAE?$AAx?$AAp?$AAo?$AAr?$AAt?$AAH?$AAa?$AAn?$AAd?$AAl?$AAe?$AAs?$AAU?$AAn@ 0000000180051500     Pcfg.obj
 0002:0000b530       ??_C@_1BE@PKILIDFH@?$AAE?$AAn?$AAa?$AAb?$AAl?$AAe?$AAW?$AAM?$AAI@ 0000000180051530     Pcfg.obj
 0002:0000b550       ??_7PluginCheckBoxBinding@@6B@ 0000000180051550     Pcfg.obj
 0002:0000b7d8       ??_7PluginEditFieldBinding@@6B@ 00000001800517d8     Pclass.obj
 0002:0000b810       ??_C@_1BK@GMMKGKID@?$AA?$HL?$AA0?$AA?$HN?$AA?4?$AA?$HL?$AA1?$AA?3?$AA0?$AA?$HL?$AA2?$AA?$HN?$AA?$HN@ 0000000180051810     Pclass.obj
 0002:0000b830       ??_C@_1BA@BHJJFMCM@?$AAB?$AAK?$AAM?$AAG?$AAT?$AAP?$AAE@ 0000000180051830     Pclass.obj
 0002:0000b840       ??_C@_1BC@HGOMHBK@?$AA?$HL?$AA0?$AA?3?$AA?$DM?$AA2?$AA1?$AA?$HN?$AA?5@ 0000000180051840     Pclass.obj
 0002:0000b858       ??_C@_19LPDLLMEB@?$AA?$HL?$AA0?$AA?$HN?$AA?3@ 0000000180051858     Pclass.obj
 0002:0000b868       ??_C@_1BC@IALIJCAM@?$AAS?$AAo?$AAr?$AAt?$AAM?$AAo?$AAd?$AAe@ 0000000180051868     Pclass.obj
 0002:0000b880       ??_C@_1BO@OMKAPLPJ@?$AAS?$AAt?$AAa?$AAr?$AAt?$AAP?$AAa?$AAn?$AAe?$AAl?$AAM?$AAo?$AAd?$AAe@ 0000000180051880     Pclass.obj
 0002:0000b8a0       ??_C@_1BA@JOLGFBLP@?$AAM?$AAo?$AAd?$AAe?$AA?$HL?$AA0?$AA?$HN@ 00000001800518a0     Pclass.obj
 0002:0000b8b0       ??_C@_1CM@KGJLHHPG@?$AAN?$AA?0?$AAX?$AA1?$AA5?$AAF?$AA?0?$AAX?$AA1?$AA6?$AAF?$AA?0?$AAX?$AA1?$AA7@ 00000001800518b0     Pclass.obj
 0002:0000b8e0       ??_C@_1BG@MNPGDOEP@?$AA1?$AA2?$AA?0?$AA0?$AA?0?$AA0?$AA?0?$AA0?$AA?0?$AA4@ 00000001800518e0     Pclass.obj
 0002:0000b8f8       ??_C@_1CG@OHFJBKLN@?$AAN?$AA?0?$AAX?$AAI?$AA?0?$AAX?$AAB?$AA?0?$AAX?$AAP?$AA?0?$AAX?$AA0?$AAS?$AA?0@ 00000001800518f8     Pclass.obj
 0002:0000b920       ??_C@_1BI@EFANNANC@?$AA0?$AA?0?$AA6?$AA?0?$AA2?$AA?0?$AA2?$AA?0?$AA3?$AA?0?$AA9@ 0000000180051920     Pclass.obj
 0002:0000b938       ??_C@_17KNGPBKAK@?$AAN?$AA?0?$AAN@ 0000000180051938     Pclass.obj
 0002:0000b940       ??_C@_17JPFFEOAH@?$AA0?$AA?0?$AA0@ 0000000180051940     Pclass.obj
 0002:0000b948       ??_C@_1BO@JAFIOFIL@?$AAN?$AA?0?$AAX?$AAI?$AA?0?$AAX?$AAB?$AA?0?$AAX?$AAC?$AA?0?$AAD?$AA?0?$AAT@ 0000000180051948     Pclass.obj
 0002:0000b968       ??_C@_1BI@LFIMKDME@?$AA0?$AA?0?$AA6?$AA?0?$AA2?$AA?0?$AA6?$AA?0?$AA0?$AA?0?$AA0@ 0000000180051968     Pclass.obj
 0002:0000b980       ??_C@_1BK@IEHCCPMO@?$AAN?$AA?0?$AAX?$AAI?$AA?0?$AAX?$AA4?$AAF?$AA?0?$AAX?$AA6?$AAF@ 0000000180051980     Pclass.obj
 0002:0000b9a0       ??_C@_1BA@MMHHFCDG@?$AA0?$AA?0?$AA6?$AA?0?$AA9?$AA?0?$AA9@ 00000001800519a0     Pclass.obj
 0002:0000b9b0       ??_C@_1EA@CMHCGANC@?$AAN?$AA?0?$AAX?$AAI?$AA?0?$AAX?$AA4?$AAF?$AA?0?$AAX?$AA6?$AAF?$AA?0?$AAX?$AA1@ 00000001800519b0     Pclass.obj
 0002:0000b9f0       ??_C@_1CE@LPFIEDMN@?$AA0?$AA?0?$AA6?$AA?0?$AA9?$AA?0?$AA9?$AA?0?$AA9?$AA?0?$AA9?$AA?0?$AA8?$AA?0?$AA8@ 00000001800519f0     Pclass.obj
 0002:0000ba18       ??_C@_19ILLMDDHI@?$AAN?$AA?0?$AAZ?$AAD@ 0000000180051a18     Pclass.obj
 0002:0000ba28       ??_C@_19NMOJBHGD@?$AA1?$AA2?$AA?0?$AA0@ 0000000180051a28     Pclass.obj
 0002:0000ba40       ??_C@_1EC@OFLHMCFD@?$AAN?$AA?0?$AAX?$AAP?$AA?0?$AAX?$AA0?$AAS?$AA?0?$AAX?$AA1?$AAS?$AA?0?$AAX?$AA2@ 0000000180051a40     Pclass.obj
 0002:0000ba88       ??_C@_1CA@MGMNHCLL@?$AA0?$AA?0?$AA2?$AA?0?$AA3?$AA?0?$AA2?$AA?0?$AA2?$AA?0?$AA3?$AA?0?$AA4?$AA?0?$AA3@ 0000000180051a88     Pclass.obj
 0002:0000baa8       ??_C@_1O@JGFFCAGM@?$AAN?$AA?0?$AAX?$AAI?$AA?0?$AAO@ 0000000180051aa8     Pclass.obj
 0002:0000bab8       ??_C@_1O@FLEOANAI@?$AA0?$AA?0?$AA6?$AA?0?$AA1?$AA5@ 0000000180051ab8     Pclass.obj
 0002:0000bac8       ??_C@_1CC@FANCGEGE@?$AAN?$AA?0?$AAX?$AAI?$AA?0?$AAX?$AAT?$AA?0?$AAX?$AA3?$AA?0?$AAX?$AAG?$AA?0?$AAX@ 0000000180051ac8     Pclass.obj
 0002:0000baf0       ??_C@_1BI@PMPHDFGH@?$AA0?$AA?0?$AA6?$AA?0?$AA3?$AA?0?$AA4?$AA?0?$AA4?$AA?0?$AA4@ 0000000180051af0     Pclass.obj
 0002:0000bb08       ??_C@_1BG@COBJEPBB@?$AAN?$AA?0?$AAX?$AAI?$AA?0?$AAX?$AAT?$AA?0?$AAX?$AA3@ 0000000180051b08     Pclass.obj
 0002:0000bb20       ??_C@_1BA@KPNNJGCD@?$AA0?$AA?0?$AA6?$AA?0?$AA3?$AA?0?$AA4@ 0000000180051b20     Pclass.obj
 0002:0000bb30       ??_C@_1CA@HLBJOHGN@?$AAF?$AAu?$AAl?$AAl?$AAS?$AAc?$AAr?$AAe?$AAe?$AAn?$AAL?$AAo?$AAc?$AAa?$AAl@ 0000000180051b30     Pclass.obj
 0002:0000bb50       ??_C@_1CC@EBBNDNOD@?$AAF?$AAu?$AAl?$AAl?$AAS?$AAc?$AAr?$AAe?$AAe?$AAn?$AAR?$AAe?$AAm?$AAo?$AAt@ 0000000180051b50     Pclass.obj
 0002:0000bb78       ??_C@_1BK@HMOODHKK@?$AAC?$AAo?$AAl?$AAu?$AAm?$AAn?$AAs?$AAL?$AAo?$AAc?$AAa?$AAl@ 0000000180051b78     Pclass.obj
 0002:0000bb98       ??_C@_1BM@EDHFKJEJ@?$AAC?$AAo?$AAl?$AAu?$AAm?$AAn?$AAs?$AAR?$AAe?$AAm?$AAo?$AAt?$AAe@ 0000000180051b98     Pclass.obj
 0002:0000bbb8       ??_C@_1BI@FOOHDOCI@?$AAW?$AAi?$AAd?$AAt?$AAh?$AAs?$AAL?$AAo?$AAc?$AAa?$AAl@ 0000000180051bb8     Pclass.obj
 0002:0000bbd0       ??_C@_1BK@DDBMMJCN@?$AAW?$AAi?$AAd?$AAt?$AAh?$AAs?$AAR?$AAe?$AAm?$AAo?$AAt?$AAe@ 0000000180051bd0     Pclass.obj
 0002:0000bbec       ??_C@_13DEFPDAGF@?$AA?0@   0000000180051bec     Pclass.obj
 0002:0000bbf0       ??_C@_15LNKNCLHH@?$AAS?$AAs@ 0000000180051bf0     Pclass.obj
 0002:0000bbf8       ??_C@_1M@PBHOFL@?$AA?5?$AA?$HL?$AA0?$AA?$HN?$AA?5@ 0000000180051bf8     Pclass.obj
 0002:0000bc08       ??_C@_1BE@JJMDGICA@?$AA?$HL?$AA0?$AA?$HN?$AA?3?$AA?5?$AA?$HL?$AA1?$AA?$HN?$AA?5@ 0000000180051c08     Pclass.obj
 0002:0000bc1c       ??_C@_15JOGBDECP@?$AA?0?$AA?5@ 0000000180051c1c     Pclass.obj
 0002:0000bc24       ??_C@_15DNHPCDHG@?$AAT?$AAt@ 0000000180051c24     Pclass.obj
 0002:0000bc2c       ??_C@_15IJHBBPPC@?$AAF?$AAf@ 0000000180051c2c     Pclass.obj
 0002:0000bc38       ??_C@_1BC@OMEIHGFC@?$AAW?$AAS?$AA_?$AAP?$AAO?$AAP?$AAU?$AAP@ 0000000180051c38     Pclass.obj
 0002:0000bc50       ??_C@_1BC@ONEEOLLM@?$AAW?$AAS?$AA_?$AAC?$AAH?$AAI?$AAL?$AAD@ 0000000180051c50     Pclass.obj
 0002:0000bc68       ??_C@_1BI@GHDIGAD@?$AAW?$AAS?$AA_?$AAM?$AAI?$AAN?$AAI?$AAM?$AAI?$AAZ?$AAE@ 0000000180051c68     Pclass.obj
 0002:0000bc80       ??_C@_1BG@KLPFHNBP@?$AAW?$AAS?$AA_?$AAV?$AAI?$AAS?$AAI?$AAB?$AAL?$AAE@ 0000000180051c80     Pclass.obj
 0002:0000bc98       ??_C@_1BI@NKODCGOF@?$AAW?$AAS?$AA_?$AAD?$AAI?$AAS?$AAA?$AAB?$AAL?$AAE?$AAD@ 0000000180051c98     Pclass.obj
 0002:0000bcb0       ??_C@_1CA@PCFJBBHH@?$AAW?$AAS?$AA_?$AAC?$AAL?$AAI?$AAP?$AAS?$AAI?$AAB?$AAL?$AAI?$AAN?$AAG?$AAS@ 0000000180051cb0     Pclass.obj
 0002:0000bcd0       ??_C@_1CA@MPLGGIO@?$AAW?$AAS?$AA_?$AAC?$AAL?$AAI?$AAP?$AAC?$AAH?$AAI?$AAL?$AAD?$AAR?$AAE?$AAN@ 0000000180051cd0     Pclass.obj
 0002:0000bcf0       ??_C@_1BI@OLBAGOJG@?$AAW?$AAS?$AA_?$AAM?$AAA?$AAX?$AAI?$AAM?$AAI?$AAZ?$AAE@ 0000000180051cf0     Pclass.obj
 0002:0000bd08       ??_C@_1BE@DAMMEKNP@?$AAW?$AAS?$AA_?$AAB?$AAO?$AAR?$AAD?$AAE?$AAR@ 0000000180051d08     Pclass.obj
 0002:0000bd20       ??_C@_1BI@EDHINADK@?$AAW?$AAS?$AA_?$AAD?$AAL?$AAG?$AAF?$AAR?$AAA?$AAM?$AAE@ 0000000180051d20     Pclass.obj
 0002:0000bd38       ??_C@_1BG@CKCLFGFA@?$AAW?$AAS?$AA_?$AAV?$AAS?$AAC?$AAR?$AAO?$AAL?$AAL@ 0000000180051d38     Pclass.obj
 0002:0000bd50       ??_C@_1BG@OMIOJOGF@?$AAW?$AAS?$AA_?$AAH?$AAS?$AAC?$AAR?$AAO?$AAL?$AAL@ 0000000180051d50     Pclass.obj
 0002:0000bd68       ??_C@_1BG@KJOBMDJC@?$AAW?$AAS?$AA_?$AAS?$AAY?$AAS?$AAM?$AAE?$AAN?$AAU@ 0000000180051d68     Pclass.obj
 0002:0000bd80       ??_C@_1BM@GPNNOPCH@?$AAW?$AAS?$AA_?$AAT?$AAH?$AAI?$AAC?$AAK?$AAF?$AAR?$AAA?$AAM?$AAE@ 0000000180051d80     Pclass.obj
 0002:0000bda0       ??_C@_1BO@FODKBODI@?$AAW?$AAS?$AA_?$AAM?$AAI?$AAN?$AAI?$AAM?$AAI?$AAZ?$AAE?$AAB?$AAO?$AAX@ 0000000180051da0     Pclass.obj
 0002:0000bdc0       ??_C@_1BO@IDJMAOMI@?$AAW?$AAS?$AA_?$AAM?$AAA?$AAX?$AAI?$AAM?$AAI?$AAZ?$AAE?$AAB?$AAO?$AAX@ 0000000180051dc0     Pclass.obj
 0002:0000bde0       ??_C@_1CI@PKBCIOPN@?$AAW?$AAS?$AA_?$AAE?$AAX?$AA_?$AAD?$AAL?$AAG?$AAM?$AAO?$AAD?$AAA?$AAL?$AAF@ 0000000180051de0     Pclass.obj
 0002:0000be08       ??_C@_1CK@KJECLHMG@?$AAW?$AAS?$AA_?$AAE?$AAX?$AA_?$AAN?$AAO?$AAP?$AAA?$AAR?$AAE?$AAN?$AAT?$AAN@ 0000000180051e08     Pclass.obj
 0002:0000be38       ??_C@_1BM@OCBKBALE@?$AAW?$AAS?$AA_?$AAE?$AAX?$AA_?$AAT?$AAO?$AAP?$AAM?$AAO?$AAS?$AAT@ 0000000180051e38     Pclass.obj
 0002:0000be58       ??_C@_1CE@JIDMMICL@?$AAW?$AAS?$AA_?$AAE?$AAX?$AA_?$AAA?$AAC?$AAC?$AAE?$AAP?$AAT?$AAF?$AAI?$AAL@ 0000000180051e58     Pclass.obj
 0002:0000be80       ??_C@_1CE@PFFPBMCF@?$AAW?$AAS?$AA_?$AAE?$AAX?$AA_?$AAT?$AAR?$AAA?$AAN?$AAS?$AAP?$AAA?$AAR?$AAE@ 0000000180051e80     Pclass.obj
 0002:0000bea8       ??_C@_1BO@MEOEJPLO@?$AAW?$AAS?$AA_?$AAE?$AAX?$AA_?$AAM?$AAD?$AAI?$AAC?$AAH?$AAI?$AAL?$AAD@ 0000000180051ea8     Pclass.obj
 0002:0000bec8       ??_C@_1CC@IEIGGJGG@?$AAW?$AAS?$AA_?$AAE?$AAX?$AA_?$AAT?$AAO?$AAO?$AAL?$AAW?$AAI?$AAN?$AAD?$AAO@ 0000000180051ec8     Pclass.obj
 0002:0000bef0       ??_C@_1CC@PLPNIKGL@?$AAW?$AAS?$AA_?$AAE?$AAX?$AA_?$AAW?$AAI?$AAN?$AAD?$AAO?$AAW?$AAE?$AAD?$AAG@ 0000000180051ef0     Pclass.obj
 0002:0000bf18       ??_C@_1CC@IAPGCLEG@?$AAW?$AAS?$AA_?$AAE?$AAX?$AA_?$AAC?$AAL?$AAI?$AAE?$AAN?$AAT?$AAE?$AAD?$AAG@ 0000000180051f18     Pclass.obj
 0002:0000bf40       ??_C@_1CE@EANKNCIF@?$AAW?$AAS?$AA_?$AAE?$AAX?$AA_?$AAC?$AAO?$AAN?$AAT?$AAE?$AAX?$AAT?$AAH?$AAE@ 0000000180051f40     Pclass.obj
 0002:0000bf68       ??_C@_1BI@GFIADCMK@?$AAW?$AAS?$AA_?$AAE?$AAX?$AA_?$AAR?$AAI?$AAG?$AAH?$AAT@ 0000000180051f68     Pclass.obj
 0002:0000bf80       ??_C@_1CC@JOFCJJPB@?$AAW?$AAS?$AA_?$AAE?$AAX?$AA_?$AAR?$AAT?$AAL?$AAR?$AAE?$AAA?$AAD?$AAI?$AAN@ 0000000180051f80     Pclass.obj
 0002:0000bfa8       ??_C@_1CI@EFLDECAB@?$AAW?$AAS?$AA_?$AAE?$AAX?$AA_?$AAL?$AAE?$AAF?$AAT?$AAS?$AAC?$AAR?$AAO?$AAL@ 0000000180051fa8     Pclass.obj
 0002:0000bfd0       ??_C@_1CI@CIFGFFJB@?$AAW?$AAS?$AA_?$AAE?$AAX?$AA_?$AAC?$AAO?$AAN?$AAT?$AAR?$AAO?$AAL?$AAP?$AAA@ 0000000180051fd0     Pclass.obj
 0002:0000bff8       ??_C@_1CC@BGEPLDCA@?$AAW?$AAS?$AA_?$AAE?$AAX?$AA_?$AAS?$AAT?$AAA?$AAT?$AAI?$AAC?$AAE?$AAD?$AAG@ 0000000180051ff8     Pclass.obj
 0002:0000c020       ??_C@_1CA@DOAIHHLO@?$AAW?$AAS?$AA_?$AAE?$AAX?$AA_?$AAA?$AAP?$AAP?$AAW?$AAI?$AAN?$AAD?$AAO?$AAW@ 0000000180052020     Pclass.obj
 0002:0000c040       ??_C@_1BM@FAODAMGD@?$AAW?$AAS?$AA_?$AAE?$AAX?$AA_?$AAL?$AAA?$AAY?$AAE?$AAR?$AAE?$AAD@ 0000000180052040     Pclass.obj
 0002:0000c060       ??_C@_1CM@DJKNBOGD@?$AAW?$AAS?$AA_?$AAE?$AAX?$AA_?$AAN?$AAO?$AAI?$AAN?$AAH?$AAE?$AAR?$AAI?$AAT@ 0000000180052060     Pclass.obj
 0002:0000c090       ??_C@_1CA@KMHLBMFI@?$AAW?$AAS?$AA_?$AAE?$AAX?$AA_?$AAL?$AAA?$AAY?$AAO?$AAU?$AAT?$AAR?$AAT?$AAL@ 0000000180052090     Pclass.obj
 0002:0000c0b0       ??_C@_1CC@LOFMDOPL@?$AAW?$AAS?$AA_?$AAE?$AAX?$AA_?$AAN?$AAO?$AAA?$AAC?$AAT?$AAI?$AAV?$AAA?$AAT@ 00000001800520b0     Pclass.obj
 0002:0000c0d8       ??_C@_1BA@PCPLEJNM@?$AA?$HL?$AA0?$AA?3?$AA2?$AA0?$AA?$HN?$AA?6@ 00000001800520d8     Pclass.obj
 0002:0000c0e8       ??_C@_1CA@PGPHFLML@?$AA?$HL?$AA0?$AA?3?$AA?$DO?$AA2?$AA0?$AA?$HN?$AA?5?$AA?$HL?$AA1?$AA?3?$AA7?$AA?$HN?$AA?$CF?$AA?6@ 00000001800520e8     Pclass.obj
 0002:0000c108       ??_C@_1CE@BCAPNIMO@?$AA?$HL?$AA0?$AA?3?$AA2?$AA0?$AA?$HN?$AA?5?$AA?5?$AA?$HL?$AA1?$AA?3?$AA7?$AA?$HN?$AA?$HL?$AA2@ 0000000180052108     Pclass.obj
 0002:0000c130       ??_C@_1CA@CGMHBFCH@?$AA?$HL?$AA0?$AA?$HN?$AA?$HL?$AA1?$AA?$HN?$AA?0?$AA?5?$AA?$HL?$AA2?$AA?$HN?$AA?$HL?$AA3?$AA?$HN?$AA?6@ 0000000180052130     Pclass.obj
 0002:0000c150       ??_C@_1BA@BIAFDLFH@?$AA?$HL?$AA0?$AA?$HN?$AA?$HL?$AA1?$AA?$HN?$AA?6@ 0000000180052150     Pclass.obj
 0002:0000c160       ??_C@_1BI@DHFBAHCI@?$AA?$HL?$AA0?$AA?$HN?$AA?5?$AA?5?$AA?$CI?$AA?$HL?$AA1?$AA?$HN?$AA?$CJ?$AA?6@ 0000000180052160     Pclass.obj
 0002:0000c178       ??_C@_19EPBAEEOA@?$AA?$HL?$AA0?$AA?$HN?$AA?6@ 0000000180052178     Pclass.obj
 0002:0000c188       ??_C@_1BK@FKNCLDML@?$AA?6?$AA?$HL?$AA0?$AA?$HN?$AA?$HL?$AA1?$AA?$HN?$AA?5?$AA?$HL?$AA2?$AA?$HN?$AA?6@ 0000000180052188     Pclass.obj
 0002:0000c1a8       ??_C@_1BC@IBCAHKMA@?$AA?6?$AA?$HL?$AA0?$AA?$HN?$AA?$HL?$AA1?$AA?$HN?$AA?6@ 00000001800521a8     Pclass.obj
 0002:0000c1c0       ??_C@_1BG@JEKFNBAO@?$AA?6?$AA?$HL?$AA0?$AA?$HN?$AA?3?$AA?6?$AA?$HL?$AA1?$AA?$HN?$AA?6@ 00000001800521c0     Pclass.obj
 0002:0000c1d8       ??_C@_1CA@MEPGLLIO@?$AA?$HL?$AA0?$AA?$HN?$AA?$HL?$AA1?$AA?3?$AA0?$AA8?$AAX?$AA?$HN?$AA?5?$AA?$HL?$AA2?$AA?$HN?$AA?6@ 00000001800521d8     Pclass.obj
 0002:0000c1f8       ??_C@_1DG@MNBLGAON@?$AA?6?$AA?$HL?$AA0?$AA?$HN?$AA?3?$AA?6?$AA?$HL?$AA1?$AA?3?$AA?$DM?$AA?$HL?$AA2?$AA?$HN?$AA?$HN?$AA?5@ 00000001800521f8     Pclass.obj
 0002:0000c230       ??_C@_19GGNHIDOH@?$AA?4?$AAt?$AAx?$AAt@ 0000000180052230     Pclass.obj
 0002:0000c240       ??_C@_19OPNPIOHE@?$AAH?$AAW?$AAN?$AAD@ 0000000180052240     Pclass.obj
 0002:0000c24c       ??_C@_15GKIJICBO@?$AAZ?$AAC@ 000000018005224c     Pclass.obj
 0002:0000c258       ??_C@_17JJIMNMHK@?$AA?5?$AA?$CG?$AA?$FO@ 0000000180052258     Pclass.obj
 0002:0000c260       ??_C@_13HOIJIPNN@?$AA?5@   0000000180052260     Pclass.obj
 0002:0000c264       ??_C@_15LEKKCGMK@?$AA?2?$AA?2@ 0000000180052264     Pclass.obj
 0002:0000c270       ??_C@_1M@CHPAGEIC@?$AA?$CF?$AA?5?$AA?$HL?$AA0?$AA?$HN@ 0000000180052270     Pclass.obj
 0002:0000c280       ??_C@_1O@DLMEBHDD@?$AA?$HL?$AA0?$AA?$HN?$AA?$HL?$AA1?$AA?$HN@ 0000000180052280     Pclass.obj
 0002:0000c290       ??_C@_15DDHGOCBH@?$AA?4?$AA?4@ 0000000180052290     Pclass.obj
 0002:0000c298       ??_C@_17FJPEEFCB@?$AAp?$AAr?$AAc@ 0000000180052298     Pclass.obj
 0002:0000c2a0       ??_C@_1BC@ENICKDH@?$AAC?$AAo?$AAn?$AAt?$AAe?$AAn?$AAt?$AAs@ 00000001800522a0     Pclass.obj
 0002:0000c2b8       ??_C@_1CK@DGKCELDD@?$AAP?$AAr?$AAo?$AAc?$AAe?$AAs?$AAs?$AAL?$AAi?$AAs?$AAt?$AA?4?$AAC?$AAo?$AAm@ 00000001800522b8     Pclass.obj
 0002:0000c2e8       ??_C@_1CK@ECJCGOEK@?$AAP?$AAr?$AAo?$AAc?$AAe?$AAs?$AAs?$AAL?$AAi?$AAs?$AAt?$AA?4?$AAU?$AAs?$AAe@ 00000001800522e8     Pclass.obj
 0002:0000c320       ??_C@_1EA@IELLPLEF@?$AA?$HL?$AA0?$AA?$HN?$AA?5?$AA?$HL?$AA1?$AA?3?$AA0?$AA2?$AA?$HN?$AA?3?$AA?$HL?$AA2?$AA?3?$AA0@ 0000000180052320     Pclass.obj
 0002:0000c360       ??_C@_1DI@BCOMPFMM@?$AA?$HL?$AA0?$AA?3?$AA0?$AA2?$AA?$HN?$AA?3?$AA?$HL?$AA1?$AA?3?$AA0?$AA2?$AA?$HN?$AA?3?$AA?$HL@ 0000000180052360     Pclass.obj
 0002:0000c3a0       ??_C@_1EA@HECKBAAG@?$AA?2?$AAS?$AAt?$AAr?$AAi?$AAn?$AAg?$AAF?$AAi?$AAl?$AAe?$AAI?$AAn?$AAf?$AAo@ 00000001800523a0     Pclass.obj
 0002:0000c3e0       ??_C@_19JHEHLFPM@?$AA?2?$AA?$DP?$AA?$DP?$AA?2@ 00000001800523e0     Pclass.obj
 0002:0000c3f0       ??_C@_1DC@HCLBMGIA@?$AA?2?$AAV?$AAa?$AAr?$AAF?$AAi?$AAl?$AAe?$AAI?$AAn?$AAf?$AAo?$AA?2?$AAT?$AAr@ 00000001800523f0     Pclass.obj
 0002:0000c428       ??_C@_1BI@HCCAONKE@?$AAF?$AAi?$AAl?$AAe?$AAV?$AAe?$AAr?$AAs?$AAi?$AAo?$AAn@ 0000000180052428     Pclass.obj
 0002:0000c440       ??_C@_1CA@JGBAIPOO@?$AAF?$AAi?$AAl?$AAe?$AAD?$AAe?$AAs?$AAc?$AAr?$AAi?$AAp?$AAt?$AAi?$AAo?$AAn@ 0000000180052440     Pclass.obj
 0002:0000c460       ??_C@_19KBHGBEJO@?$AA?$HL?$AA0?$AA?$HN?$AA?2@ 0000000180052460     Pclass.obj
 0002:0000c470       ??_C@_1O@BMPPIAFP@?$AA?5?$AA?$CI?$AA?$HL?$AA0?$AA?$HN?$AA?$CJ@ 0000000180052470     Pclass.obj
 0002:0000c480       ??_C@_1BC@OMEIBLAI@?$AAw?$AAb?$AAe?$AAm?$AAc?$AAo?$AAm?$AAn@ 0000000180052480     Pclass.obj
 0002:0000c498       ??_C@_0BA@FOIKENOD@vector?5too?5long@ 0000000180052498     Pclass.obj
 0002:0000c4a8       ??_C@_0BI@CFPLBAOH@invalid?5string?5position@ 00000001800524a8     Pclass.obj
 0002:0000c4c0       ??_C@_15LGINNLBP@?$AA?$HL?$AA?$HN@ 00000001800524c0     Pclass.obj
 0002:0000c4c8       ??_C@_0BL@GOIGLPKN@unordered_map?1set?5too?5long@ 00000001800524c8     Pclass.obj
 0002:0000c4e8       ??_C@_0BK@OGNNAFAB@invalid?5hash?5bucket?5count@ 00000001800524e8     Pclass.obj
 0002:0000c510       ?Counters@@3QBUcounters@@B 0000000180052510     perfthread.obj
 0002:0000c670       ??_C@_1CC@DNHMJIKH@?$AA?$CF?$AA?5?$AAP?$AAr?$AAo?$AAc?$AAe?$AAs?$AAs?$AAo?$AAr?$AA?5?$AAT?$AAi?$AAm@ 0000000180052670     perfthread.obj
 0002:0000c698       ??_C@_1CE@FNEMIHOD@?$AA?$CF?$AA?5?$AAP?$AAr?$AAi?$AAv?$AAi?$AAl?$AAe?$AAg?$AAe?$AAd?$AA?5?$AAT?$AAi@ 0000000180052698     perfthread.obj
 0002:0000c6c0       ??_C@_1BI@IIOPEKIO@?$AA?$CF?$AA?5?$AAU?$AAs?$AAe?$AAr?$AA?5?$AAT?$AAi?$AAm?$AAe@ 00000001800526c0     perfthread.obj
 0002:0000c6d8       ??_C@_1BK@FAAJNJIB@?$AAH?$AAa?$AAn?$AAd?$AAl?$AAe?$AA?5?$AAC?$AAo?$AAu?$AAn?$AAt@ 00000001800526d8     perfthread.obj
 0002:0000c6f8       ??_C@_1CA@KJMNGIDJ@?$AAP?$AAa?$AAg?$AAe?$AA?5?$AAF?$AAi?$AAl?$AAe?$AA?5?$AAB?$AAy?$AAt?$AAe?$AAs@ 00000001800526f8     perfthread.obj
 0002:0000c718       ??_C@_1CK@FGGMBBIH@?$AAP?$AAa?$AAg?$AAe?$AA?5?$AAF?$AAi?$AAl?$AAe?$AA?5?$AAB?$AAy?$AAt?$AAe?$AAs@ 0000000180052718     perfthread.obj
 0002:0000c748       ??_C@_1BI@GCOMDKEO@?$AAW?$AAo?$AAr?$AAk?$AAi?$AAn?$AAg?$AA?5?$AAS?$AAe?$AAt@ 0000000180052748     perfthread.obj
 0002:0000c760       ??_C@_1CC@OFJLEPCP@?$AAW?$AAo?$AAr?$AAk?$AAi?$AAn?$AAg?$AA?5?$AAS?$AAe?$AAt?$AA?5?$AAP?$AAe?$AAa@ 0000000180052760     perfthread.obj
 0002:0000c788       ??_C@_1CI@LLKMGPEG@?$AAP?$AAo?$AAo?$AAl?$AA?5?$AAN?$AAo?$AAn?$AAp?$AAa?$AAg?$AAe?$AAd?$AA?5?$AAB@ 0000000180052788     perfthread.obj
 0002:0000c7b0       ??_C@_1CC@IMBAECJF@?$AAP?$AAo?$AAo?$AAl?$AA?5?$AAP?$AAa?$AAg?$AAe?$AAd?$AA?5?$AAB?$AAy?$AAt?$AAe@ 00000001800527b0     perfthread.obj
 0002:0000c7d8       ??_C@_1BM@DGDPAMAA@?$AAP?$AAr?$AAi?$AAv?$AAa?$AAt?$AAe?$AA?5?$AAB?$AAy?$AAt?$AAe?$AAs@ 00000001800527d8     perfthread.obj
 0002:0000c7f8       ??_C@_1CA@GADAGCME@?$AAP?$AAa?$AAg?$AAe?$AA?5?$AAF?$AAa?$AAu?$AAl?$AAt?$AAs?$AA?1?$AAs?$AAe?$AAc@ 00000001800527f8     perfthread.obj
 0002:0000c818       ??_C@_1BM@FMIOMJAE@?$AAV?$AAi?$AAr?$AAt?$AAu?$AAa?$AAl?$AA?5?$AAB?$AAy?$AAt?$AAe?$AAs@ 0000000180052818     perfthread.obj
 0002:0000c838       ??_C@_1CG@KJOKFONA@?$AAV?$AAi?$AAr?$AAt?$AAu?$AAa?$AAl?$AA?5?$AAB?$AAy?$AAt?$AAe?$AAs?$AA?5?$AAP@ 0000000180052838     perfthread.obj
 0002:0000c860       ??_C@_1CE@DFDFLLAO@?$AAI?$AAO?$AA?5?$AAD?$AAa?$AAt?$AAa?$AA?5?$AAB?$AAy?$AAt?$AAe?$AAs?$AA?1?$AAs@ 0000000180052860     perfthread.obj
 0002:0000c888       ??_C@_1CE@EFLEKJAB@?$AAI?$AAO?$AA?5?$AAR?$AAe?$AAa?$AAd?$AA?5?$AAB?$AAy?$AAt?$AAe?$AAs?$AA?1?$AAs@ 0000000180052888     perfthread.obj
 0002:0000c8b0       ??_C@_1CG@MEJHKKKF@?$AAI?$AAO?$AA?5?$AAW?$AAr?$AAi?$AAt?$AAe?$AA?5?$AAB?$AAy?$AAt?$AAe?$AAs?$AA?1@ 00000001800528b0     perfthread.obj
 0002:0000c8d8       ??_C@_1CG@LBBBPCJA@?$AAI?$AAO?$AA?5?$AAO?$AAt?$AAh?$AAe?$AAr?$AA?5?$AAB?$AAy?$AAt?$AAe?$AAs?$AA?1@ 00000001800528d8     perfthread.obj
 0002:0000c900       ??_C@_1CO@LIEOHDCC@?$AAI?$AAO?$AA?5?$AAD?$AAa?$AAt?$AAa?$AA?5?$AAO?$AAp?$AAe?$AAr?$AAa?$AAt?$AAi@ 0000000180052900     perfthread.obj
 0002:0000c930       ??_C@_1CO@LIIKBHDH@?$AAI?$AAO?$AA?5?$AAR?$AAe?$AAa?$AAd?$AA?5?$AAO?$AAp?$AAe?$AAr?$AAa?$AAt?$AAi@ 0000000180052930     perfthread.obj
 0002:0000c960       ??_C@_1DA@HICMAFKK@?$AAI?$AAO?$AA?5?$AAW?$AAr?$AAi?$AAt?$AAe?$AA?5?$AAO?$AAp?$AAe?$AAr?$AAa?$AAt@ 0000000180052960     perfthread.obj
 0002:0000c990       ??_C@_1DA@BEHINMGJ@?$AAI?$AAO?$AA?5?$AAO?$AAt?$AAh?$AAe?$AAr?$AA?5?$AAO?$AAp?$AAe?$AAr?$AAa?$AAt@ 0000000180052990     perfthread.obj
 0002:0000c9c0       ??_C@_1BA@MGJGGMO@?$AAC?$AAo?$AAu?$AAn?$AAt?$AAe?$AAr@ 00000001800529c0     perfthread.obj
 0002:0000c9d0       ??_C@_1BG@NKNJPBCD@?$AAI?$AAD?$AA?5?$AAP?$AAr?$AAo?$AAc?$AAe?$AAs?$AAs@ 00000001800529d0     perfthread.obj
 0002:0000c9e8       ??_C@_1BM@KCAKLHJN@?$AAP?$AAr?$AAi?$AAo?$AAr?$AAi?$AAt?$AAy?$AA?5?$AAB?$AAa?$AAs?$AAe@ 00000001800529e8     perfthread.obj
 0002:0000ca08       ??_C@_1BK@KCHPPKHP@?$AAT?$AAh?$AAr?$AAe?$AAa?$AAd?$AA?5?$AAC?$AAo?$AAu?$AAn?$AAt@ 0000000180052a08     perfthread.obj
 0002:0000ca28       ??_C@_1CI@FNIEMNAI@?$AAC?$AAr?$AAe?$AAa?$AAt?$AAi?$AAn?$AAg?$AA?5?$AAP?$AAr?$AAo?$AAc?$AAe?$AAs@ 0000000180052a28     perfthread.obj
 0002:0000ca50       ??_C@_1BK@IKAFHKBD@?$AAE?$AAl?$AAa?$AAp?$AAs?$AAe?$AAd?$AA?5?$AAT?$AAi?$AAm?$AAe@ 0000000180052a50     perfthread.obj
 0002:0000ca70       ??_C@_19DLCFHDFF@?$AAP?$AAE?$AAR?$AAF@ 0000000180052a70     perfthread.obj
 0002:0000ca80       ??_C@_19DOGDICKI@?$AA?4?$AAe?$AAx?$AAe@ 0000000180052a80     perfthread.obj
 0002:0000ca90       ??_C@_1O@NKAIMMPD@?$AA_?$AAT?$AAo?$AAt?$AAa?$AAl@ 0000000180052a90     Plist.obj
 0002:0000caa0       ??_C@_1CC@DMDJMJLM@?$AAS?$AAe?$AAD?$AAe?$AAb?$AAu?$AAg?$AAP?$AAr?$AAi?$AAv?$AAi?$AAl?$AAe?$AAg@ 0000000180052aa0     Plist.obj
 0002:0000cac8       ??_C@_1BE@KEEKBEOD@?$AA?$HL?$AA0?$AA?$HN?$AA?3?$AA?6?$AA?$HL?$AA1?$AA?$HN?$AA?6@ 0000000180052ac8     Plist.obj
 0002:0000cae0       ??_C@_1O@DMFBLLIP@?$AA?6?$AA?$HL?$AA0?$AA?$HN?$AA?3?$AA?6@ 0000000180052ae0     Plist.obj
 0002:0000caf0       ??_C@_1BG@JBKHLPML@?$AA?$HL?$AA0?$AA?$HN?$AA?5?$AA?$HL?$AA1?$AA?3?$AA8?$AAX?$AA?$HN@ 0000000180052af0     Plist.obj
 0002:0000cb08       ??_C@_19DPDNGGHD@?$AA?5?$AA?$HL?$AA0?$AA?$HN@ 0000000180052b08     Plist.obj
 0002:0000cb18       ??_C@_1BE@EMDGEBAH@?$AA?$HL?$AA0?$AA?3?$AA0?$AA?$HL?$AA1?$AA?$HN?$AAX?$AA?$HN@ 0000000180052b18     Plist.obj
 0002:0000cb38       ??_7?$_Func_impl_no_alloc@V<lambda_1>@?6??PrintModules@?$ipc_functions@$0A@@@SAXPEAX0AEAUoptions@@@Z@_NPEA_W_K@std@@6B@ 0000000180052b38     Plist.obj
 0002:0000cba0       ??_C@_1CA@CCAFOKCB@?$AAE?$AAr?$AAr?$AAo?$AAr?$AA?5?$AA0?$AAx?$AA?$HL?$AA0?$AA?3?$AA0?$AA8?$AAX?$AA?$HN@ 0000000180052ba0     Pmix.obj
 0002:0000cbc0       ??_C@_15JNBOKNOG@?$AA?$AN?$AA?6@ 0000000180052bc0     Pmix.obj
 0002:0000cbc8       ??_C@_1DC@LAIEFOLO@?$AAW?$AAi?$AAn?$AA3?$AA2?$AA_?$AAP?$AAr?$AAo?$AAc?$AAe?$AAs?$AAs?$AA?4?$AAH@ 0000000180052bc8     wmi.obj
 0002:0000cc00       ??_C@_1BO@CLCOBGDE@?$AAE?$AAx?$AAe?$AAc?$AAu?$AAt?$AAa?$AAb?$AAl?$AAe?$AAP?$AAa?$AAt?$AAh@ 0000000180052c00     wmi.obj
 0002:0000cc20       ??_C@_1BI@LPJNJKGA@?$AAC?$AAo?$AAm?$AAm?$AAa?$AAn?$AAd?$AAL?$AAi?$AAn?$AAe@ 0000000180052c20     wmi.obj
 0002:0000cc38       ??_C@_1BC@JHNNEHFE@?$AAP?$AAr?$AAi?$AAo?$AAr?$AAi?$AAt?$AAy@ 0000000180052c38     wmi.obj
 0002:0000cc50       ??_C@_1BC@HJJANEGO@?$AAG?$AAe?$AAt?$AAO?$AAw?$AAn?$AAe?$AAr@ 0000000180052c50     wmi.obj
 0002:0000cc68       ??_C@_19PIJILKAI@?$AAU?$AAs?$AAe?$AAr@ 0000000180052c68     wmi.obj
 0002:0000cc78       ??_C@_1O@OAMNPMOM@?$AAD?$AAo?$AAm?$AAa?$AAi?$AAn@ 0000000180052c78     wmi.obj
 0002:0000cc88       ??_C@_1BI@OIPNMPCL@?$AAG?$AAe?$AAt?$AAO?$AAw?$AAn?$AAe?$AAr?$AAS?$AAi?$AAd@ 0000000180052c88     wmi.obj
 0002:0000cca0       ??_C@_17NKMLOKHF@?$AAS?$AAi?$AAd@ 0000000180052ca0     wmi.obj
 0002:0000cca8       ??_C@_1BE@CFEJJKFE@?$AAS?$AAe?$AAs?$AAs?$AAi?$AAo?$AAn?$AAI?$AAd@ 0000000180052ca8     wmi.obj
 0002:0000ccc0       ??_C@_1BM@MLGLIGHJ@?$AAW?$AAi?$AAn?$AA3?$AA2?$AA_?$AAP?$AAr?$AAo?$AAc?$AAe?$AAs?$AAs@ 0000000180052cc0     wmi.obj
 0002:0000cce0       ??_C@_1BI@FLOHINJE@?$AAR?$AAe?$AAt?$AAu?$AAr?$AAn?$AAV?$AAa?$AAl?$AAu?$AAe@ 0000000180052ce0     wmi.obj
 0002:0000ccf8       ??_C@_1BI@NKNJJIDM@?$AAS?$AAe?$AAt?$AAP?$AAr?$AAi?$AAo?$AAr?$AAi?$AAt?$AAy@ 0000000180052cf8     wmi.obj
 0002:0000cd10       ??_C@_1O@GGHBFGJC@?$AAR?$AAe?$AAa?$AAs?$AAo?$AAn@ 0000000180052d10     wmi.obj
 0002:0000cd20       ??_C@_1BE@PBPGMODO@?$AAT?$AAe?$AAr?$AAm?$AAi?$AAn?$AAa?$AAt?$AAe@ 0000000180052d20     wmi.obj
 0002:0000cd38       ??_C@_1CC@OGNCBAIB@?$AA?2?$AA?2?$AA?$HL?$AA0?$AA?$HN?$AA?2?$AAr?$AAo?$AAo?$AAt?$AA?2?$AAc?$AAi?$AAm?$AAv@ 0000000180052d38     wmi.obj
 0002:0000cd5c       ??_C@_13JOFGPIOO@?$AA?4@   0000000180052d5c     wmi.obj
 0002:0000cdd0       ??_C@_1M@OAIMIKLP@?$AAn?$AAt?$AAd?$AAl?$AAl@ 0000000180052dd0     Proclist.obj
 0002:0000cde0       ??_C@_0BK@EGDDIFMK@NtQueryInformationProcess@ 0000000180052de0     Proclist.obj
 0002:0000ce00       ??_C@_0BJ@HKKELGGC@NtQueryInformationThread@ 0000000180052e00     Proclist.obj
 0002:0000ce20       ??_C@_0O@IFMDHOMC@NtQueryObject@ 0000000180052e20     Proclist.obj
 0002:0000ce30       ??_C@_0BJ@NDLOPGCH@NtQuerySystemInformation@ 0000000180052e30     Proclist.obj
 0002:0000ce50       ??_C@_0BH@DLPGICA@NtQueryInformationFile@ 0000000180052e50     Proclist.obj
 0002:0000ce68       ??_C@_0CB@GDPHBMJN@NtWow64QueryInformationProcess6@ 0000000180052e68     Proclist.obj
 0002:0000ce90       ??_C@_0BL@NJDHCDMK@NtWow64ReadVirtualMemory64@ 0000000180052e90     Proclist.obj
 0002:0000ceb0       ??_C@_1BC@GDMECMAK@?$AAk?$AAe?$AAr?$AAn?$AAe?$AAl?$AA3?$AA2@ 0000000180052eb0     Proclist.obj
 0002:0000cec8       ??_C@_0P@LKABJJMO@IsWow64Process@ 0000000180052ec8     Proclist.obj
 0002:0000ced8       ??_C@_1BC@DNHGCMLG@?$AAa?$AAd?$AAv?$AAa?$AAp?$AAi?$AA3?$AA2@ 0000000180052ed8     Proclist.obj
 0002:0000cef0       ??_C@_0L@KJHKJIPF@IsValidSid@ 0000000180052ef0     Proclist.obj
 0002:0000cf00       ??_C@_0BK@FIHGNING@GetSidIdentifierAuthority@ 0000000180052f00     Proclist.obj
 0002:0000cf20       ??_C@_0BI@LPFJALDI@GetSidSubAuthorityCount@ 0000000180052f20     Proclist.obj
 0002:0000cf38       ??_C@_0BD@LMGFHOAE@GetSidSubAuthority@ 0000000180052f38     Proclist.obj
 0002:0000cf50       ??_C@_1O@BCCLBEOE@?$AAu?$AAs?$AAe?$AAr?$AA3?$AA2@ 0000000180052f50     Proclist.obj
 0002:0000cf60       ??_C@_0BA@FKGDNIJG@GetGuiResources@ 0000000180052f60     Proclist.obj
 0002:0000cf70       ??_C@_1M@FFPAMFOB@?$AAo?$AAl?$AAe?$AA3?$AA2@ 0000000180052f70     Proclist.obj
 0002:0000cf80       ??_C@_0BC@IOEGILCE@CoSetProxyBlanket@ 0000000180052f80     Proclist.obj
 0002:0000cf98       ??_C@_1M@OMFDJDJC@?$AAp?$AAs?$AAa?$AAp?$AAi@ 0000000180052f98     Proclist.obj
 0002:0000cfa8       ??_C@_0BF@LEEEDPDK@EnumProcessModulesEx@ 0000000180052fa8     Proclist.obj
 0002:0000cfc0       ??_C@_1BC@PDEABLIN@?$AAP?$AAr?$AAo?$AAc?$AAL?$AAi?$AAs?$AAt@ 0000000180052fc0     Proclist.obj
 0002:0000cfd8       ??_C@_1DK@DCAMPEPJ@?$AAP?$AAr?$AAo?$AAc?$AAe?$AAs?$AAs?$AA?5?$AAL?$AAi?$AAs?$AAt?$AA?5?$AAf?$AAo@ 0000000180052fd8     Proclist.obj
 0002:0000d018       ??_C@_1DE@BGKMIKPD@?$AAE?$AAu?$AAg?$AAe?$AAn?$AAe?$AA?5?$AAR?$AAo?$AAs?$AAh?$AAa?$AAl?$AA?5?$AA?$CG@ 0000000180053018     Proclist.obj
 0002:0000d050       ??_C@_1M@MNPEKPKO@?$AAp?$AAl?$AAi?$AAs?$AAt@ 0000000180053050     Proclist.obj
 0002:0000d060       MenuGuid                   0000000180053060     Proclist.obj
 0002:0000d070       MainGuid                   0000000180053070     Proclist.obj
 0002:0000d080       ConfigDialogGuid           0000000180053080     Proclist.obj
 0002:0000e8e0       _load_config_used          00000001800548e0     LIBCMT:loadcfg.obj
 0002:0000ea80       ??_R4bad_function_call@std@@6B@ 0000000180054a80     libcpmt:xthrow.obj
 0002:0000eaa8       ??_R3bad_function_call@std@@8 0000000180054aa8     libcpmt:xthrow.obj
 0002:0000eac0       ??_R2bad_function_call@std@@8 0000000180054ac0     libcpmt:xthrow.obj
 0002:0000ead8       ??_R1A@?0A@EA@bad_function_call@std@@8 0000000180054ad8     libcpmt:xthrow.obj
 0002:0000eb00       ??_R4logic_error@std@@6B@  0000000180054b00     libcpmt:xthrow.obj
 0002:0000eb28       ??_R3logic_error@std@@8    0000000180054b28     libcpmt:xthrow.obj
 0002:0000eb40       ??_R2logic_error@std@@8    0000000180054b40     libcpmt:xthrow.obj
 0002:0000eb58       ??_R1A@?0A@EA@logic_error@std@@8 0000000180054b58     libcpmt:xthrow.obj
 0002:0000eb80       ??_R4length_error@std@@6B@ 0000000180054b80     libcpmt:xthrow.obj
 0002:0000eba8       ??_R3length_error@std@@8   0000000180054ba8     libcpmt:xthrow.obj
 0002:0000ebc0       ??_R2length_error@std@@8   0000000180054bc0     libcpmt:xthrow.obj
 0002:0000ebe0       ??_R1A@?0A@EA@length_error@std@@8 0000000180054be0     libcpmt:xthrow.obj
 0002:0000ec08       ??_R4out_of_range@std@@6B@ 0000000180054c08     libcpmt:xthrow.obj
 0002:0000ec30       ??_R3out_of_range@std@@8   0000000180054c30     libcpmt:xthrow.obj
 0002:0000ec48       ??_R2out_of_range@std@@8   0000000180054c48     libcpmt:xthrow.obj
 0002:0000ec68       ??_R1A@?0A@EA@out_of_range@std@@8 0000000180054c68     libcpmt:xthrow.obj
 0002:0000ec90       ??_R4_Locimp@locale@std@@6B@ 0000000180054c90     libcpmt:locale0.obj
 0002:0000ecb8       ??_R3_Locimp@locale@std@@8 0000000180054cb8     libcpmt:locale0.obj
 0002:0000ecd0       ??_R2_Locimp@locale@std@@8 0000000180054cd0     libcpmt:locale0.obj
 0002:0000ecf8       ??_R1A@?0A@EA@_Locimp@locale@std@@8 0000000180054cf8     libcpmt:locale0.obj
 0002:0000ed20       ??_R4type_info@@6B@        0000000180054d20     LIBCMT:std_type_info_static.obj
 0002:0000ed48       ??_R3type_info@@8          0000000180054d48     LIBCMT:std_type_info_static.obj
 0002:0000ed60       ??_R2type_info@@8          0000000180054d60     LIBCMT:std_type_info_static.obj
 0002:0000ed70       ??_R1A@?0A@EA@type_info@@8 0000000180054d70     LIBCMT:std_type_info_static.obj
 0002:0000ed98       ??_R4bad_exception@std@@6B@ 0000000180054d98     libvcruntime:frame.obj
 0002:0000edc0       ??_R3bad_exception@std@@8  0000000180054dc0     libvcruntime:frame.obj
 0002:0000edd8       ??_R2bad_exception@std@@8  0000000180054dd8     libvcruntime:frame.obj
 0002:0000edf0       ??_R1A@?0A@EA@bad_exception@std@@8 0000000180054df0     libvcruntime:frame.obj
 0002:0000ee18       ??_R1A@?0A@EA@?$basic_memory_buffer@D$0BPE@V?$allocator@D@std@@@v8@fmt@@8 0000000180054e18     format.obj
 0002:0000ee40       ??_R4exception@std@@6B@    0000000180054e40     format.obj
 0002:0000ee68       ??_R2bad_array_new_length@std@@8 0000000180054e68     format.obj
 0002:0000ee88       ??_R3?$buffer@H@detail@v8@fmt@@8 0000000180054e88     format.obj
 0002:0000eea0       ??_R1A@?0A@EA@?$buffer@H@detail@v8@fmt@@8 0000000180054ea0     format.obj
 0002:0000eec8       ??_R3?$basic_memory_buffer@H$0BPE@V?$allocator@H@std@@@v8@fmt@@8 0000000180054ec8     format.obj
 0002:0000eee0       ??_R4?$basic_memory_buffer@_W$0BPE@V?$allocator@_W@std@@@v8@fmt@@6B@ 0000000180054ee0     format.obj
 0002:0000ef08       ??_R4runtime_error@std@@6B@ 0000000180054f08     format.obj
 0002:0000ef30       ??_R3_Facet_base@std@@8    0000000180054f30     format.obj
 0002:0000ef48       ??_R1A@?0A@EA@bad_cast@std@@8 0000000180054f48     format.obj
 0002:0000ef70       ??_R1A@?0A@EA@?$buffer@I@detail@v8@fmt@@8 0000000180054f70     format.obj
 0002:0000ef98       ??_R2bad_alloc@std@@8      0000000180054f98     format.obj
 0002:0000efb0       ??_R3format_error@v8@fmt@@8 0000000180054fb0     format.obj
 0002:0000efc8       ??_R3_Crt_new_delete@std@@8 0000000180054fc8     format.obj
 0002:0000efe0       ??_R1A@?0A@EA@runtime_error@std@@8 0000000180054fe0     format.obj
 0002:0000f008       ??_R2?$buffer@_W@detail@v8@fmt@@8 0000000180055008     format.obj
 0002:0000f018       ??_R1A@?0A@EA@exception@std@@8 0000000180055018     format.obj
 0002:0000f040       ??_R2?$numpunct@_W@std@@8  0000000180055040     format.obj
 0002:0000f068       ??_R1A@?0A@EA@_Facet_base@std@@8 0000000180055068     format.obj
 0002:0000f090       ??_R1A@?0A@EA@bad_alloc@std@@8 0000000180055090     format.obj
 0002:0000f0b8       ??_R2format_error@v8@fmt@@8 00000001800550b8     format.obj
 0002:0000f0d8       ??_R3?$basic_memory_buffer@D$0BPE@V?$allocator@D@std@@@v8@fmt@@8 00000001800550d8     format.obj
 0002:0000f0f0       ??_R17?0A@EA@_Crt_new_delete@std@@8 00000001800550f0     format.obj
 0002:0000f118       ??_R2?$basic_memory_buffer@D$0BPE@V?$allocator@D@std@@@v8@fmt@@8 0000000180055118     format.obj
 0002:0000f130       ??_R3?$basic_memory_buffer@_W$0BPE@V?$allocator@_W@std@@@v8@fmt@@8 0000000180055130     format.obj
 0002:0000f148       ??_R2bad_cast@std@@8       0000000180055148     format.obj
 0002:0000f160       ??_R2exception@std@@8      0000000180055160     format.obj
 0002:0000f170       ??_R1A@?0A@EA@facet@locale@std@@8 0000000180055170     format.obj
 0002:0000f198       ??_R2?$buffer@I@detail@v8@fmt@@8 0000000180055198     format.obj
 0002:0000f1a8       ??_R3?$numpunct@_W@std@@8  00000001800551a8     format.obj
 0002:0000f1c0       ??_R3?$buffer@I@detail@v8@fmt@@8 00000001800551c0     format.obj
 0002:0000f1d8       ??_R4?$basic_memory_buffer@H$0BPE@V?$allocator@H@std@@@v8@fmt@@6B@ 00000001800551d8     format.obj
 0002:0000f200       ??_R1A@?0A@EA@?$numpunct@_W@std@@8 0000000180055200     format.obj
 0002:0000f228       ??_R2?$basic_memory_buffer@I$0CA@V?$allocator@I@std@@@v8@fmt@@8 0000000180055228     format.obj
 0002:0000f240       ??_R3exception@std@@8      0000000180055240     format.obj
 0002:0000f258       ??_R2?$buffer@D@detail@v8@fmt@@8 0000000180055258     format.obj
 0002:0000f268       ??_R3?$buffer@D@detail@v8@fmt@@8 0000000180055268     format.obj
 0002:0000f280       ??_R2?$buffer@H@detail@v8@fmt@@8 0000000180055280     format.obj
 0002:0000f290       ??_R3facet@locale@std@@8   0000000180055290     format.obj
 0002:0000f2a8       ??_R2?$basic_memory_buffer@_W$0BPE@V?$allocator@_W@std@@@v8@fmt@@8 00000001800552a8     format.obj
 0002:0000f2c0       ??_R3bad_cast@std@@8       00000001800552c0     format.obj
 0002:0000f2d8       ??_R4bad_alloc@std@@6B@    00000001800552d8     format.obj
 0002:0000f300       ??_R4bad_cast@std@@6B@     0000000180055300     format.obj
 0002:0000f328       ??_R1A@?0A@EA@_Crt_new_delete@std@@8 0000000180055328     format.obj
 0002:0000f350       ??_R2?$basic_memory_buffer@H$0BPE@V?$allocator@H@std@@@v8@fmt@@8 0000000180055350     format.obj
 0002:0000f368       ??_R4format_error@v8@fmt@@6B@ 0000000180055368     format.obj
 0002:0000f390       ??_R3bad_array_new_length@std@@8 0000000180055390     format.obj
 0002:0000f3a8       ??_R3bad_alloc@std@@8      00000001800553a8     format.obj
 0002:0000f3c0       ??_R4_Facet_base@std@@6B@  00000001800553c0     format.obj
 0002:0000f3e8       ??_R2runtime_error@std@@8  00000001800553e8     format.obj
 0002:0000f400       ??_R4?$numpunct@_W@std@@6B@ 0000000180055400     format.obj
 0002:0000f428       ??_R3?$buffer@_W@detail@v8@fmt@@8 0000000180055428     format.obj
 0002:0000f440       ??_R4bad_array_new_length@std@@6B@ 0000000180055440     format.obj
 0002:0000f468       ??_R1A@?0A@EA@?$buffer@_W@detail@v8@fmt@@8 0000000180055468     format.obj
 0002:0000f490       ??_R2_Crt_new_delete@std@@8 0000000180055490     format.obj
 0002:0000f4a0       ??_R1A@?0A@EA@?$buffer@D@detail@v8@fmt@@8 00000001800554a0     format.obj
 0002:0000f4c8       ??_R1A@?0A@EA@?$basic_memory_buffer@I$0CA@V?$allocator@I@std@@@v8@fmt@@8 00000001800554c8     format.obj
 0002:0000f4f0       ??_R1A@?0A@EA@bad_array_new_length@std@@8 00000001800554f0     format.obj
 0002:0000f518       ??_R3?$basic_memory_buffer@I$0CA@V?$allocator@I@std@@@v8@fmt@@8 0000000180055518     format.obj
 0002:0000f530       ??_R1A@?0A@EA@format_error@v8@fmt@@8 0000000180055530     format.obj
 0002:0000f558       ??_R2_Facet_base@std@@8    0000000180055558     format.obj
 0002:0000f568       ??_R2facet@locale@std@@8   0000000180055568     format.obj
 0002:0000f588       ??_R3runtime_error@std@@8  0000000180055588     format.obj
 0002:0000f5a0       ??_R4?$basic_memory_buffer@D$0BPE@V?$allocator@D@std@@@v8@fmt@@6B@ 00000001800555a0     format.obj
 0002:0000f5c8       ??_R1A@?0A@EA@?$basic_memory_buffer@H$0BPE@V?$allocator@H@std@@@v8@fmt@@8 00000001800555c8     format.obj
 0002:0000f5f0       ??_R1A@?0A@EA@?$basic_memory_buffer@_W$0BPE@V?$allocator@_W@std@@@v8@fmt@@8 00000001800555f0     format.obj
 0002:0000f618       ??_R4?$basic_memory_buffer@I$0CA@V?$allocator@I@std@@@v8@fmt@@6B@ 0000000180055618     format.obj
 0002:0000f640       ??_R3DialogAPIBinding@@8   0000000180055640     Pcfg.obj
 0002:0000f658       ??_R1A@?0A@EA@PluginCheckBoxBinding@@8 0000000180055658     Pcfg.obj
 0002:0000f680       ??_R3PluginCheckBoxBinding@@8 0000000180055680     Pcfg.obj
 0002:0000f698       ??_R2DialogAPIBinding@@8   0000000180055698     Pcfg.obj
 0002:0000f6a8       ??_R4PluginCheckBoxBinding@@6B@ 00000001800556a8     Pcfg.obj
 0002:0000f6d0       ??_R2PluginCheckBoxBinding@@8 00000001800556d0     Pcfg.obj
 0002:0000f6e8       ??_R1A@?0A@EA@DialogAPIBinding@@8 00000001800556e8     Pcfg.obj
 0002:0000f710       ??_R2PluginEditFieldBinding@@8 0000000180055710     Pclass.obj
 0002:0000f728       ??_R4PluginEditFieldBinding@@6B@ 0000000180055728     Pclass.obj
 0002:0000f750       ??_R3PluginEditFieldBinding@@8 0000000180055750     Pclass.obj
 0002:0000f768       ??_R1A@?0A@EA@PluginEditFieldBinding@@8 0000000180055768     Pclass.obj
 0002:0000f7c0       ??_R1A@?0A@EA@?$_Func_base@_NPEA_W_K@std@@8 00000001800557c0     Plist.obj
 0002:0000f7e8       ??_R3?$_Func_impl_no_alloc@V<lambda_1>@?6??PrintModules@?$ipc_functions@$0A@@@SAXPEAX0AEAUoptions@@@Z@_NPEA_W_K@std@@8 00000001800557e8     Plist.obj
 0002:0000f828       ??_R2?$_Func_base@_NPEA_W_K@std@@8 0000000180055828     Plist.obj
 0002:0000f838       ??_R3?$_Func_base@_NPEA_W_K@std@@8 0000000180055838     Plist.obj
 0002:0000f850       ??_R1A@?0A@EA@?$_Func_impl_no_alloc@V<lambda_1>@?6??PrintModules@?$ipc_functions@$0A@@@SAXPEAX0AEAUoptions@@@Z@_NPEA_W_K@std@@8 0000000180055850     Plist.obj
 0002:0000f878       ??_R2?$_Func_impl_no_alloc@V<lambda_1>@?6??PrintModules@?$ipc_functions@$0A@@@SAXPEAX0AEAUoptions@@@Z@_NPEA_W_K@std@@8 0000000180055878     Plist.obj
 0002:0000f8b8       ??_R4?$_Func_impl_no_alloc@V<lambda_1>@?6??PrintModules@?$ipc_functions@$0A@@@SAXPEAX0AEAUoptions@@@Z@_NPEA_W_K@std@@6B@ 00000001800558b8     Plist.obj
 0002:0000f938       ??_R1A@?0A@EA@?$_Func_base@XAEBUtagVARIANT@@@std@@8 0000000180055938     wmi.obj
 0002:0000f988       ??_R2?$_Func_base@XAEBUtagVARIANT@@@std@@8 0000000180055988     wmi.obj
 0002:0000f9c0       ??_R3?$_Func_base@XAEBUtagVARIANT@@@std@@8 00000001800559c0     wmi.obj
 0002:0000fdb8       __rtc_iaa                  0000000180055db8     LIBCMT:initsect.obj
 0002:0000fdc0       __rtc_izz                  0000000180055dc0     LIBCMT:initsect.obj
 0002:0000fdc8       __rtc_taa                  0000000180055dc8     LIBCMT:initsect.obj
 0002:0000fdd0       __rtc_tzz                  0000000180055dd0     LIBCMT:initsect.obj
 0002:00014978       _TI2?AVbad_alloc@std@@     000000018005a978     libcpmt:xthrow.obj
 0002:00014998       _CTA2?AVbad_alloc@std@@    000000018005a998     libcpmt:xthrow.obj
 0002:000149b0       _CT??_R0?AVlogic_error@std@@@8??0logic_error@std@@QEAA@AEBV01@@Z24 000000018005a9b0     libcpmt:xthrow.obj
 0002:000149d8       _TI3?AVlength_error@std@@  000000018005a9d8     libcpmt:xthrow.obj
 0002:000149f8       _CTA3?AVlength_error@std@@ 000000018005a9f8     libcpmt:xthrow.obj
 0002:00014a18       _CT??_R0?AVlength_error@std@@@8??0length_error@std@@QEAA@AEBV01@@Z24 000000018005aa18     libcpmt:xthrow.obj
 0002:00014a40       _TI3?AVout_of_range@std@@  000000018005aa40     libcpmt:xthrow.obj
 0002:00014a60       _CTA3?AVout_of_range@std@@ 000000018005aa60     libcpmt:xthrow.obj
 0002:00014a80       _CT??_R0?AVout_of_range@std@@@8??0out_of_range@std@@QEAA@AEBV01@@Z24 000000018005aa80     libcpmt:xthrow.obj
 0002:00014aa8       _TI2?AVbad_function_call@std@@ 000000018005aaa8     libcpmt:xthrow.obj
 0002:00014ac8       _CTA2?AVbad_function_call@std@@ 000000018005aac8     libcpmt:xthrow.obj
 0002:00014ae0       _CT??_R0?AVbad_function_call@std@@@8??0bad_function_call@std@@QEAA@AEBV01@@Z24 000000018005aae0     libcpmt:xthrow.obj
 0002:00014b08       _TI2?AVbad_exception@std@@ 000000018005ab08     libvcruntime:frame.obj
 0002:00014b28       _CTA2?AVbad_exception@std@@ 000000018005ab28     libvcruntime:frame.obj
 0002:00014b40       _CT??_R0?AVbad_exception@std@@@8??0bad_exception@std@@QEAA@AEBV01@@Z24 000000018005ab40     libvcruntime:frame.obj
 0002:00014b68       _CT??_R0?AVformat_error@v8@fmt@@@8??0format_error@v8@fmt@@QEAA@AEBV012@@Z24 000000018005ab68     format.obj
 0002:00014b90       _CTA3?AVformat_error@v8@fmt@@ 000000018005ab90     format.obj
 0002:00014bb0       _TI2?AVruntime_error@std@@ 000000018005abb0     format.obj
 0002:00014bd0       _CTA3?AVbad_array_new_length@std@@ 000000018005abd0     format.obj
 0002:00014bf0       _CTA2?AVbad_cast@std@@     000000018005abf0     format.obj
 0002:00014c08       _CTA2?AVruntime_error@std@@ 000000018005ac08     format.obj
 0002:00014c20       _TI2?AVbad_cast@std@@      000000018005ac20     format.obj
 0002:00014c40       _CT??_R0?AVbad_array_new_length@std@@@8??0bad_array_new_length@std@@QEAA@AEBV01@@Z24 000000018005ac40     format.obj
 0002:00014c68       _CT??_R0?AVruntime_error@std@@@8??0runtime_error@std@@QEAA@AEBV01@@Z24 000000018005ac68     format.obj
 0002:00014c90       _CT??_R0?AVbad_cast@std@@@8??0bad_cast@std@@QEAA@AEBV01@@Z24 000000018005ac90     format.obj
 0002:00014cb8       _CT??_R0?AVbad_alloc@std@@@8??0bad_alloc@std@@QEAA@AEBV01@@Z24 000000018005acb8     format.obj
 0002:00014ce0       _CT??_R0?AVexception@std@@@8??0exception@std@@QEAA@AEBV01@@Z24 000000018005ace0     format.obj
 0002:00014d08       _TI3?AVformat_error@v8@fmt@@ 000000018005ad08     format.obj
 0002:00014d28       _TI3?AVbad_array_new_length@std@@ 000000018005ad28     format.obj
 0002:00014ef0       __IMPORT_DESCRIPTOR_KERNEL32 000000018005aef0     kernel32:KERNEL32.dll
 0002:00014f04       __IMPORT_DESCRIPTOR_ADVAPI32 000000018005af04     advapi32:ADVAPI32.dll
 0002:00014f18       __IMPORT_DESCRIPTOR_USER32 000000018005af18     user32:USER32.dll
 0002:00014f2c       __IMPORT_DESCRIPTOR_MPR    000000018005af2c     mpr:MPR.dll
 0002:00014f40       __IMPORT_DESCRIPTOR_ole32  000000018005af40     ole32:ole32.dll
 0002:00014f54       __IMPORT_DESCRIPTOR_OLEAUT32 000000018005af54     oleaut32:OLEAUT32.dll
 0002:00014f68       __IMPORT_DESCRIPTOR_PSAPI  000000018005af68     psapi:PSAPI.DLL
 0002:00014f7c       __IMPORT_DESCRIPTOR_VERSION 000000018005af7c     version:VERSION.dll
 0002:00014f90       __NULL_IMPORT_DESCRIPTOR   000000018005af90     kernel32:KERNEL32.dll
 0003:00000010       __do_unsigned_char_lconv_initialization 000000018005c010     LIBCMT:lconv_unsigned_char.obj
 0003:00000014       __scrt_native_dllmain_reason 000000018005c014     LIBCMT:utility.obj
 0003:00000018       _fltused                   000000018005c018     LIBCMT:fltused.obj
 0003:00000020       __security_cookie          000000018005c020     LIBCMT:gs_cookie.obj
 0003:00000028       __security_cookie_complement 000000018005c028     LIBCMT:gs_cookie.obj
 0003:00000040       _iob                       000000018005c040     libucrt:_file.obj
 0003:00000150       __acrt_lconv_c             000000018005c150     libucrt:localeconv.obj
 0003:000001e8       __acrt_lconv               000000018005c1e8     libucrt:localeconv.obj
 0003:000001f0       __acrt_lconv_static_decimal 000000018005c1f0     libucrt:localeconv.obj
 0003:000001f4       __acrt_lconv_static_W_decimal 000000018005c1f4     libucrt:localeconv.obj
 0003:00000200       _pctype                    000000018005c200     libucrt:ctype.obj
 0003:00000208       _pwctype                   000000018005c208     libucrt:ctype.obj
 0003:00000210       __abort_behavior           000000018005c210     libucrt:abort.obj
 0003:00000220       __acrt_initial_locale_data 000000018005c220     libucrt:nlsdata.obj
 0003:00000378       __acrt_initial_locale_pointers 000000018005c378     libucrt:nlsdata.obj
 0003:00000388       __acrt_wide_c_locale_string 000000018005c388     libucrt:nlsdata.obj
 0003:0000038c       __mb_cur_max               000000018005c38c     libucrt:nlsdata.obj
 0003:00000390       __globallocalestatus       000000018005c390     libucrt:glstatus.obj
 0003:00000430       __acrt_initial_multibyte_data 000000018005c430     libucrt:mbctype.obj
 0003:00000970       _lookuptrailbytes          000000018005c970     libucrt:read.obj
 0003:00000b08       ?pGetGuiResources@@3P6AKPEAXK@ZEA 000000018005cb08     Proclist.obj
 0003:00000b10       ?pEnumProcessModulesEx@@3P6AHPEAXPEAPEAUHINSTANCE__@@KPEAKK@ZEA 000000018005cb10     Proclist.obj
 0003:00000b18       ?pCoSetProxyBlanket@@3P6AJPEAUIUnknown@@KKPEA_WKKPEAXK@ZEA 000000018005cb18     Proclist.obj
 0003:00000b20       ?pIsWow64Process@@3P6AHPEAXPEAH@ZEA 000000018005cb20     Proclist.obj
 0003:00000b28       ?pNtQuerySystemInformation@@3P6AJKPEAXKPEAK@ZEA 000000018005cb28     Proclist.obj
 0003:00000b30       ?pNtQueryInformationProcess@@3P6AJPEAXW4_PROCESSINFOCLASS@@0KPEAK@ZEA 000000018005cb30     Proclist.obj
 0003:00000b38       ?pNtQueryObject@@3P6AJPEAXK0K0@ZEA 000000018005cb38     Proclist.obj
 0003:00000b40       ?pNtQueryInformationThread@@3P6AJPEAXK0KPEAK@ZEA 000000018005cb40     Proclist.obj
 0003:00000b48       ?pNtQueryInformationFile@@3P6AJPEAX00KK@ZEA 000000018005cb48     Proclist.obj
 0003:00000b50       ?m_PanelModesDataRemote@Plist@@0V?$vector@Umode@@V?$allocator@Umode@@@std@@@std@@A 000000018005cb50     fileio.obj
 0003:00000b68       ?m_PanelModesDataLocal@Plist@@0V?$vector@Umode@@V?$allocator@Umode@@@std@@@std@@A 000000018005cb68     fileio.obj
 0003:00000b80       ??_R0?AVlogic_error@std@@@8 000000018005cb80     libcpmt:xthrow.obj
 0003:00000ba8       ??_R0?AVlength_error@std@@@8 000000018005cba8     libcpmt:xthrow.obj
 0003:00000bd0       ??_R0?AVout_of_range@std@@@8 000000018005cbd0     libcpmt:xthrow.obj
 0003:00000bf8       ??_R0?AVbad_function_call@std@@@8 000000018005cbf8     libcpmt:xthrow.obj
 0003:00000c28       ??_R0?AVbad_exception@std@@@8 000000018005cc28     libvcruntime:frame.obj
 0003:00000c50       ??_R0?AVruntime_error@std@@@8 000000018005cc50     format.obj
 0003:00000c78       ??_R0?AVbad_alloc@std@@@8  000000018005cc78     format.obj
 0003:00000ca0       ??_R0?AVbad_cast@std@@@8   000000018005cca0     format.obj
 0003:00000cc8       ??_R0?AVformat_error@v8@fmt@@@8 000000018005ccc8     format.obj
 0003:00000cf8       ??_R0?AVexception@std@@@8  000000018005ccf8     format.obj
 0003:00000d20       ??_R0?AVbad_array_new_length@std@@@8 000000018005cd20     format.obj
 0003:00000da0       ??_R0?AV<lambda_1>@?6??PrintModules@?$ipc_functions@$0A@@@SAXPEAX0AEAUoptions@@@Z@@8 000000018005cda0     Plist.obj
 0003:00000ef0       ??_R0?AV_Locimp@locale@std@@@8 000000018005cef0     libcpmt:locale0.obj
 0003:00000f20       ??_R0?AVtype_info@@@8      000000018005cf20     LIBCMT:std_type_info_static.obj
 0003:00000f40       ??_R0?AV?$basic_memory_buffer@H$0BPE@V?$allocator@H@std@@@v8@fmt@@@8 000000018005cf40     format.obj
 0003:00000f90       ??_R0?AV_Facet_base@std@@@8 000000018005cf90     format.obj
 0003:00000fb8       ??_R0?AU_Crt_new_delete@std@@@8 000000018005cfb8     format.obj
 0003:00000fe8       ??_R0?AV?$buffer@_W@detail@v8@fmt@@@8 000000018005cfe8     format.obj
 0003:00001018       ??_R0?AV?$numpunct@_W@std@@@8 000000018005d018     format.obj
 0003:00001040       ??_R0?AV?$buffer@D@detail@v8@fmt@@@8 000000018005d040     format.obj
 0003:00001070       ??_R0?AV?$buffer@H@detail@v8@fmt@@@8 000000018005d070     format.obj
 0003:000010a0       ??_R0?AV?$basic_memory_buffer@I$0CA@V?$allocator@I@std@@@v8@fmt@@@8 000000018005d0a0     format.obj
 0003:000010f0       ??_R0?AVfacet@locale@std@@@8 000000018005d0f0     format.obj
 0003:00001120       ??_R0?AV?$basic_memory_buffer@_W$0BPE@V?$allocator@_W@std@@@v8@fmt@@@8 000000018005d120     format.obj
 0003:00001178       ??_R0?AV?$buffer@I@detail@v8@fmt@@@8 000000018005d178     format.obj
 0003:000011b0       ??_R0?AV?$basic_memory_buffer@D$0BPE@V?$allocator@D@std@@@v8@fmt@@@8 000000018005d1b0     format.obj
 0003:00001200       ??_R0?AVDialogAPIBinding@@@8 000000018005d200     Pcfg.obj
 0003:00001228       ??_R0?AVPluginCheckBoxBinding@@@8 000000018005d228     Pcfg.obj
 0003:00001258       ??_R0?AVPluginEditFieldBinding@@@8 000000018005d258     Pclass.obj
 0003:00001288       ??_R0?AV?$_Func_base@_NPEA_W_K@std@@@8 000000018005d288     Plist.obj
 0003:00001340       ??_R0?AV?$_Func_impl_no_alloc@V<lambda_1>@?6??PrintModules@?$ipc_functions@$0A@@@SAXPEAX0AEAUoptions@@@Z@_NPEA_W_K@std@@@8 000000018005d340     Plist.obj
 0003:000013c8       ??_R0?AV?$_Func_base@XAEBUtagVARIANT@@@std@@@8 000000018005d3c8     wmi.obj
 0003:000016a8       ?_Id_cnt@id@locale@std@@0HA 000000018005d6a8     libcpmt:locale0.obj
 0003:000016b0       ?_Clocptr@_Locimp@locale@std@@0PEAV123@EA 000000018005d6b0     libcpmt:locale0.obj
 0003:000016b8       ?id@?$ctype@_W@std@@2V0locale@2@A 000000018005d6b8     libcpmt:locale0.obj
 0003:000016c0       ?id@?$ctype@D@std@@2V0locale@2@A 000000018005d6c0     libcpmt:locale0.obj
 0003:000016c8       ?id@?$codecvt@GDU_Mbstatet@@@std@@2V0locale@2@A 000000018005d6c8     libcpmt:locale0.obj
 0003:000016d0       ?id@?$ctype@G@std@@2V0locale@2@A 000000018005d6d0     libcpmt:locale0.obj
 0003:000016e8       ?id@?$codecvt@_WDU_Mbstatet@@@std@@2V0locale@2@A 000000018005d6e8     libcpmt:locale0.obj
 0003:00001710       ?id@?$num_get@DV?$istreambuf_iterator@DU?$char_traits@D@std@@@std@@@std@@2V0locale@2@A 000000018005d710     libcpmt:locale.obj
 0003:00001718       ?id@?$num_put@DV?$ostreambuf_iterator@DU?$char_traits@D@std@@@std@@@std@@2V0locale@2@A 000000018005d718     libcpmt:locale.obj
 0003:00001720       ?id@?$codecvt@DDU_Mbstatet@@@std@@2V0locale@2@A 000000018005d720     libcpmt:locale.obj
 0003:00001730       ?_Ptr_cin@std@@3PEAV?$basic_istream@DU?$char_traits@D@std@@@1@EA 000000018005d730     libcpmt:iosptrs.obj
 0003:00001738       ?_Ptr_cout@std@@3PEAV?$basic_ostream@DU?$char_traits@D@std@@@1@EA 000000018005d738     libcpmt:iosptrs.obj
 0003:00001740       ?_Ptr_cerr@std@@3PEAV?$basic_ostream@DU?$char_traits@D@std@@@1@EA 000000018005d740     libcpmt:iosptrs.obj
 0003:00001748       ?_Ptr_clog@std@@3PEAV?$basic_ostream@DU?$char_traits@D@std@@@1@EA 000000018005d748     libcpmt:iosptrs.obj
 0003:00001750       ?_Ptr_wcin@std@@3PEAV?$basic_istream@_WU?$char_traits@_W@std@@@1@EA 000000018005d750     libcpmt:iosptrs.obj
 0003:00001758       ?_Ptr_wcout@std@@3PEAV?$basic_ostream@_WU?$char_traits@_W@std@@@1@EA 000000018005d758     libcpmt:iosptrs.obj
 0003:00001760       ?_Ptr_wcerr@std@@3PEAV?$basic_ostream@_WU?$char_traits@_W@std@@@1@EA 000000018005d760     libcpmt:iosptrs.obj
 0003:00001768       ?_Ptr_wclog@std@@3PEAV?$basic_ostream@_WU?$char_traits@_W@std@@@1@EA 000000018005d768     libcpmt:iosptrs.obj
 0003:000017d0       ?id@?$time_put@_WV?$ostreambuf_iterator@_WU?$char_traits@_W@std@@@std@@@std@@2V0locale@2@A 000000018005d7d0     libcpmt:wlocale.obj
 0003:000017d8       ?id@?$num_get@_WV?$istreambuf_iterator@_WU?$char_traits@_W@std@@@std@@@std@@2V0locale@2@A 000000018005d7d8     libcpmt:wlocale.obj
 0003:000017e0       ?id@?$num_put@_WV?$ostreambuf_iterator@_WU?$char_traits@_W@std@@@std@@@std@@2V0locale@2@A 000000018005d7e0     libcpmt:wlocale.obj
 0003:000017e8       ?id@?$collate@_W@std@@2V0locale@2@A 000000018005d7e8     libcpmt:wlocale.obj
 0003:000017f0       ?id@?$messages@_W@std@@2V0locale@2@A 000000018005d7f0     libcpmt:wlocale.obj
 0003:000017f8       ?id@?$money_get@_WV?$istreambuf_iterator@_WU?$char_traits@_W@std@@@std@@@std@@2V0locale@2@A 000000018005d7f8     libcpmt:wlocale.obj
 0003:00001800       ?id@?$money_put@_WV?$ostreambuf_iterator@_WU?$char_traits@_W@std@@@std@@@std@@2V0locale@2@A 000000018005d800     libcpmt:wlocale.obj
 0003:00001808       ?id@?$moneypunct@_W$0A@@std@@2V0locale@2@A 000000018005d808     libcpmt:wlocale.obj
 0003:00001810       ?id@?$moneypunct@_W$00@std@@2V0locale@2@A 000000018005d810     libcpmt:wlocale.obj
 0003:00001818       ?id@?$time_get@_WV?$istreambuf_iterator@_WU?$char_traits@_W@std@@@std@@@std@@2V0locale@2@A 000000018005d818     libcpmt:wlocale.obj
 0003:00001820       ?id@?$num_get@GV?$istreambuf_iterator@GU?$char_traits@G@std@@@std@@@std@@2V0locale@2@A 000000018005d820     libcpmt:wlocale.obj
 0003:00001828       ?id@?$num_put@GV?$ostreambuf_iterator@GU?$char_traits@G@std@@@std@@@std@@2V0locale@2@A 000000018005d828     libcpmt:wlocale.obj
 0003:00001830       ?id@?$numpunct@G@std@@2V0locale@2@A 000000018005d830     libcpmt:wlocale.obj
 0003:00001838       ?id@?$collate@G@std@@2V0locale@2@A 000000018005d838     libcpmt:wlocale.obj
 0003:00001840       ?id@?$messages@G@std@@2V0locale@2@A 000000018005d840     libcpmt:wlocale.obj
 0003:00001848       ?id@?$money_get@GV?$istreambuf_iterator@GU?$char_traits@G@std@@@std@@@std@@2V0locale@2@A 000000018005d848     libcpmt:wlocale.obj
 0003:00001850       ?id@?$money_put@GV?$ostreambuf_iterator@GU?$char_traits@G@std@@@std@@@std@@2V0locale@2@A 000000018005d850     libcpmt:wlocale.obj
 0003:00001858       ?id@?$moneypunct@G$0A@@std@@2V0locale@2@A 000000018005d858     libcpmt:wlocale.obj
 0003:00001860       ?id@?$moneypunct@G$00@std@@2V0locale@2@A 000000018005d860     libcpmt:wlocale.obj
 0003:00001868       ?id@?$time_get@GV?$istreambuf_iterator@GU?$char_traits@G@std@@@std@@@std@@2V0locale@2@A 000000018005d868     libcpmt:wlocale.obj
 0003:00001870       ?id@?$time_put@GV?$ostreambuf_iterator@GU?$char_traits@G@std@@@std@@@std@@2V0locale@2@A 000000018005d870     libcpmt:wlocale.obj
 0003:00001878       ?id@?$collate@D@std@@2V0locale@2@A 000000018005d878     libcpmt:xlocale.obj
 0003:00001880       ?id@?$messages@D@std@@2V0locale@2@A 000000018005d880     libcpmt:xlocale.obj
 0003:00001888       ?id@?$money_get@DV?$istreambuf_iterator@DU?$char_traits@D@std@@@std@@@std@@2V0locale@2@A 000000018005d888     libcpmt:xlocale.obj
 0003:00001890       ?id@?$money_put@DV?$ostreambuf_iterator@DU?$char_traits@D@std@@@std@@@std@@2V0locale@2@A 000000018005d890     libcpmt:xlocale.obj
 0003:00001898       ?id@?$moneypunct@D$0A@@std@@2V0locale@2@A 000000018005d898     libcpmt:xlocale.obj
 0003:000018a0       ?id@?$moneypunct@D$00@std@@2V0locale@2@A 000000018005d8a0     libcpmt:xlocale.obj
 0003:000018a8       ?id@?$time_get@DV?$istreambuf_iterator@DU?$char_traits@D@std@@@std@@@std@@2V0locale@2@A 000000018005d8a8     libcpmt:xlocale.obj
 0003:000018b0       ?id@?$time_put@DV?$ostreambuf_iterator@DU?$char_traits@D@std@@@std@@@std@@2V0locale@2@A 000000018005d8b0     libcpmt:xlocale.obj
 0003:000018b8       __scrt_current_native_startup_state 000000018005d8b8     LIBCMT:utility.obj
 0003:000018c0       __scrt_native_startup_lock 000000018005d8c0     LIBCMT:utility.obj
 0003:00001900       __castguard_check_failure_os_handled_fptr 000000018005d900     LIBCMT:guard_support.obj
 0003:00001d40       ?__type_info_root_node@@3U__type_info_node@@A 000000018005dd40     LIBCMT:tncleanup.obj
 0003:00001d50       ?_OptionsStorage@?1??__local_stdio_scanf_options@@9@4_KA 000000018005dd50     LIBCMT:default_local_stdio_options.obj
 0003:00001d58       ?__WinRTOutOfMemoryExceptionCallback@@3P6APEAXXZEA 000000018005dd58     libvcruntime:ehhelpers.obj
 0003:00001de0       __pPurecall                000000018005dde0     libvcruntime:purevirt_data.obj
 0003:00001e40       ?pArgList@UnDecorator@@0PEAVReplicator@@EA 000000018005de40     libvcruntime:undname.obj
 0003:00001e48       ?pZNameList@UnDecorator@@0PEAVReplicator@@EA 000000018005de48     libvcruntime:undname.obj
 0003:00001e50       ?pTemplateArgList@UnDecorator@@0PEAVReplicator@@EA 000000018005de50     libvcruntime:undname.obj
 0003:00001e58       ?gName@UnDecorator@@0PEBDEB 000000018005de58     libvcruntime:undname.obj
 0003:00001e60       ?name@UnDecorator@@0PEBDEB 000000018005de60     libvcruntime:undname.obj
 0003:00001e68       ?disableFlags@UnDecorator@@0KA 000000018005de68     libvcruntime:undname.obj
 0003:00001e6c       ?fExplicitTemplateParams@UnDecorator@@0_NA 000000018005de6c     libvcruntime:undname.obj
 0003:00001e6d       ?fGetTemplateArgumentList@UnDecorator@@0_NA 000000018005de6d     libvcruntime:undname.obj
 0003:00001e70       ?m_pGetParameter@UnDecorator@@0P6APEADJ@ZEA 000000018005de70     libvcruntime:undname.obj
 0003:00001e78       ?m_CHPENameOffset@UnDecorator@@0KA 000000018005de78     libvcruntime:undname.obj
 0003:00001e7c       ?m_recursionLevel@UnDecorator@@0KA 000000018005de7c     libvcruntime:undname.obj
 0003:00001e80       _nstream                   000000018005de80     libucrt:_file.obj
 0003:00001e88       __piob                     000000018005de88     libucrt:_file.obj
 0003:00001e90       __acrt_lconv_static_null   000000018005de90     libucrt:localeconv.obj
 0003:00001e94       __acrt_lconv_static_W_null 000000018005de94     libucrt:localeconv.obj
 0003:000020e0       ?c_exit_complete@?1???R<lambda_6e4b09c48022b2350581041d5f6b0c4c>@@QEBA@XZ@4_NA 000000018005e0e0     libucrt:exit.obj
 0003:000021f8       _environ_table             000000018005e1f8     libucrt:environment_initialization.obj
 0003:00002200       _wenviron_table            000000018005e200     libucrt:environment_initialization.obj
 0003:00002208       __dcrt_initial_wide_environment 000000018005e208     libucrt:environment_initialization.obj
 0003:00002210       __dcrt_initial_narrow_environment 000000018005e210     libucrt:environment_initialization.obj
 0003:00002218       __acrt_atexit_table        000000018005e218     libucrt:onexit.obj
 0003:00002230       __acrt_at_quick_exit_table 000000018005e230     libucrt:onexit.obj
 0003:00002260       __pioinfo                  000000018005e260     libucrt:ioinit.obj
 0003:00002660       _nhandle                   000000018005e660     libucrt:ioinit.obj
 0003:00002838       __acrt_stdout_buffer       000000018005e838     libucrt:_sftbuf.obj
 0003:00002840       __acrt_stderr_buffer       000000018005e840     libucrt:_sftbuf.obj
 0003:00002848       __acrt_locale_changed_data 000000018005e848     libucrt:wsetlocale.obj
 0003:00002850       __acrt_current_locale_data 000000018005e850     libucrt:nlsdata.obj
 0003:00002880       ?_timezone@@3V?$dual_state_global@J@__crt_state_management@@A 000000018005e880     libucrt:timeset.obj
 0003:00002884       ?_daylight@@3V?$dual_state_global@H@__crt_state_management@@A 000000018005e884     libucrt:timeset.obj
 0003:00002888       ?_dstbias@@3V?$dual_state_global@J@__crt_state_management@@A 000000018005e888     libucrt:timeset.obj
 0003:00002950       _mbctype                   000000018005e950     libucrt:mbctype.obj
 0003:00002958       _mbcasemap                 000000018005e958     libucrt:mbctype.obj
 0003:00002960       __acrt_current_multibyte_data 000000018005e960     libucrt:mbctype.obj
 0003:00002970       _pgmptr                    000000018005e970     libucrt:argv_data.obj
 0003:00002978       __argc                     000000018005e978     libucrt:argv_data.obj
 0003:00002980       __argv                     000000018005e980     libucrt:argv_data.obj
 0003:00002988       __wargv                    000000018005e988     libucrt:argv_data.obj
 0003:00002990       _acmdln                    000000018005e990     libucrt:argv_data.obj
 0003:00002998       _wcmdln                    000000018005e998     libucrt:argv_data.obj
 0003:000029a0       __acrt_heap                000000018005e9a0     libucrt:heap_handle.obj
 0003:000029c8       ?_OptionsStorage@?1??__local_stdio_printf_options@@9@4_KA 000000018005e9c8     format.obj
 0003:000029d0       ?_Psave@?$_Facetptr@V?$numpunct@_W@std@@@std@@2PEBVfacet@locale@2@EB 000000018005e9d0     format.obj
 0003:00002af0       ?FSF@@3UFarStandardFunctions@@A 000000018005eaf0     Proclist.obj
 0003:00002c80       ?Opt@@3Uoptions@@A         000000018005ec80     Proclist.obj
 0003:00002cb0       ?PsInfo@@3UPluginStartupInfo@@A 000000018005ecb0     Proclist.obj
 0003:00002dc8       ?id@?$numpunct@_W@std@@2V0locale@2@A 000000018005edc8     format.obj
 0003:00002dd0       ?id@?$numpunct@D@std@@2V0locale@2@A 000000018005edd0     format.obj
 0003:00004110       __dyn_tls_init_callback    0000000180060110     <common>
 0003:00004118       __scrt_ucrt_dll_is_in_use  0000000180060118     <common>

 entry point at        0001:00029a98

 Static symbols

 0000:fff9a000       .debug$S                   0000000180000000     ProcList.exp
 0000:fff9a000       .debug$S                   0000000180000000     advapi32:ADVAPI32.dll
 0000:fff9a000       .debug$S                   0000000180000000     advapi32:ADVAPI32.dll
 0000:fff9a000       .debug$S                   0000000180000000     advapi32:ADVAPI32.dll
 0000:fff9a000       .debug$S                   0000000180000000     advapi32:ADVAPI32.dll
 0000:fff9a000       .debug$S                   0000000180000000     advapi32:ADVAPI32.dll
 0000:fff9a000       .debug$S                   0000000180000000     advapi32:ADVAPI32.dll
 0000:fff9a000       .debug$S                   0000000180000000     advapi32:ADVAPI32.dll
 0000:fff9a000       .debug$S                   0000000180000000     advapi32:ADVAPI32.dll
 0000:fff9a000       .debug$S                   0000000180000000     advapi32:ADVAPI32.dll
 0000:fff9a000       .debug$S                   0000000180000000     advapi32:ADVAPI32.dll
 0000:fff9a000       .debug$S                   0000000180000000     advapi32:ADVAPI32.dll
 0000:fff9a000       .debug$S                   0000000180000000     advapi32:ADVAPI32.dll
 0000:fff9a000       .debug$S                   0000000180000000     kernel32:KERNEL32.dll
 0000:fff9a000       .debug$S                   0000000180000000     kernel32:KERNEL32.dll
 0000:fff9a000       .debug$S                   0000000180000000     kernel32:KERNEL32.dll
 0000:fff9a000       .debug$S                   0000000180000000     kernel32:KERNEL32.dll
 0000:fff9a000       .debug$S                   0000000180000000     kernel32:KERNEL32.dll
 0000:fff9a000       .debug$S                   0000000180000000     kernel32:KERNEL32.dll
 0000:fff9a000       .debug$S                   0000000180000000     kernel32:KERNEL32.dll
 0000:fff9a000       .debug$S                   0000000180000000     kernel32:KERNEL32.dll
 0000:fff9a000       .debug$S                   0000000180000000     kernel32:KERNEL32.dll
 0000:fff9a000       .debug$S                   0000000180000000     kernel32:KERNEL32.dll
 0000:fff9a000       .debug$S                   0000000180000000     kernel32:KERNEL32.dll
 0000:fff9a000       .debug$S                   0000000180000000     kernel32:KERNEL32.dll
 0000:fff9a000       .debug$S                   0000000180000000     kernel32:KERNEL32.dll
 0000:fff9a000       .debug$S                   0000000180000000     kernel32:KERNEL32.dll
 0000:fff9a000       .debug$S                   0000000180000000     kernel32:KERNEL32.dll
 0000:fff9a000       .debug$S                   0000000180000000     kernel32:KERNEL32.dll
 0000:fff9a000       .debug$S                   0000000180000000     kernel32:KERNEL32.dll
 0000:fff9a000       .debug$S                   0000000180000000     kernel32:KERNEL32.dll
 0000:fff9a000       .debug$S                   0000000180000000     kernel32:KERNEL32.dll
 0000:fff9a000       .debug$S                   0000000180000000     kernel32:KERNEL32.dll
 0000:fff9a000       .debug$S                   0000000180000000     kernel32:KERNEL32.dll
 0000:fff9a000       .debug$S                   0000000180000000     kernel32:KERNEL32.dll
 0000:fff9a000       .debug$S                   0000000180000000     kernel32:KERNEL32.dll
 0000:fff9a000       .debug$S                   0000000180000000     kernel32:KERNEL32.dll
 0000:fff9a000       .debug$S                   0000000180000000     kernel32:KERNEL32.dll
 0000:fff9a000       .debug$S                   0000000180000000     kernel32:KERNEL32.dll
 0000:fff9a000       .debug$S                   0000000180000000     kernel32:KERNEL32.dll
 0000:fff9a000       .debug$S                   0000000180000000     kernel32:KERNEL32.dll
 0000:fff9a000       .debug$S                   0000000180000000     kernel32:KERNEL32.dll
 0000:fff9a000       .debug$S                   0000000180000000     kernel32:KERNEL32.dll
 0000:fff9a000       .debug$S                   0000000180000000     kernel32:KERNEL32.dll
 0000:fff9a000       .debug$S                   0000000180000000     kernel32:KERNEL32.dll
 0000:fff9a000       .debug$S                   0000000180000000     kernel32:KERNEL32.dll
 0000:fff9a000       .debug$S                   0000000180000000     kernel32:KERNEL32.dll
 0000:fff9a000       .debug$S                   0000000180000000     kernel32:KERNEL32.dll
 0000:fff9a000       .debug$S                   0000000180000000     kernel32:KERNEL32.dll
 0000:fff9a000       .debug$S                   0000000180000000     kernel32:KERNEL32.dll
 0000:fff9a000       .debug$S                   0000000180000000     kernel32:KERNEL32.dll
 0000:fff9a000       .debug$S                   0000000180000000     kernel32:KERNEL32.dll
 0000:fff9a000       .debug$S                   0000000180000000     kernel32:KERNEL32.dll
 0000:fff9a000       .debug$S                   0000000180000000     kernel32:KERNEL32.dll
 0000:fff9a000       .debug$S                   0000000180000000     kernel32:KERNEL32.dll
 0000:fff9a000       .debug$S                   0000000180000000     kernel32:KERNEL32.dll
 0000:fff9a000       .debug$S                   0000000180000000     kernel32:KERNEL32.dll
 0000:fff9a000       .debug$S                   0000000180000000     kernel32:KERNEL32.dll
 0000:fff9a000       .debug$S                   0000000180000000     kernel32:KERNEL32.dll
 0000:fff9a000       .debug$S                   0000000180000000     kernel32:KERNEL32.dll
 0000:fff9a000       .debug$S                   0000000180000000     kernel32:KERNEL32.dll
 0000:fff9a000       .debug$S                   0000000180000000     kernel32:KERNEL32.dll
 0000:fff9a000       .debug$S                   0000000180000000     kernel32:KERNEL32.dll
 0000:fff9a000       .debug$S                   0000000180000000     kernel32:KERNEL32.dll
 0000:fff9a000       .debug$S                   0000000180000000     kernel32:KERNEL32.dll
 0000:fff9a000       .debug$S                   0000000180000000     kernel32:KERNEL32.dll
 0000:fff9a000       .debug$S                   0000000180000000     kernel32:KERNEL32.dll
 0000:fff9a000       .debug$S                   0000000180000000     kernel32:KERNEL32.dll
 0000:fff9a000       .debug$S                   0000000180000000     kernel32:KERNEL32.dll
 0000:fff9a000       .debug$S                   0000000180000000     kernel32:KERNEL32.dll
 0000:fff9a000       .debug$S                   0000000180000000     kernel32:KERNEL32.dll
 0000:fff9a000       .debug$S                   0000000180000000     kernel32:KERNEL32.dll
 0000:fff9a000       .debug$S                   0000000180000000     kernel32:KERNEL32.dll
 0000:fff9a000       .debug$S                   0000000180000000     kernel32:KERNEL32.dll
 0000:fff9a000       .debug$S                   0000000180000000     kernel32:KERNEL32.dll
 0000:fff9a000       .debug$S                   0000000180000000     kernel32:KERNEL32.dll
 0000:fff9a000       .debug$S                   0000000180000000     kernel32:KERNEL32.dll
 0000:fff9a000       .debug$S                   0000000180000000     kernel32:KERNEL32.dll
 0000:fff9a000       .debug$S                   0000000180000000     kernel32:KERNEL32.dll
 0000:fff9a000       .debug$S                   0000000180000000     kernel32:KERNEL32.dll
 0000:fff9a000       .debug$S                   0000000180000000     kernel32:KERNEL32.dll
 0000:fff9a000       .debug$S                   0000000180000000     kernel32:KERNEL32.dll
 0000:fff9a000       .debug$S                   0000000180000000     kernel32:KERNEL32.dll
 0000:fff9a000       .debug$S                   0000000180000000     kernel32:KERNEL32.dll
 0000:fff9a000       .debug$S                   0000000180000000     kernel32:KERNEL32.dll
 0000:fff9a000       .debug$S                   0000000180000000     kernel32:KERNEL32.dll
 0000:fff9a000       .debug$S                   0000000180000000     kernel32:KERNEL32.dll
 0000:fff9a000       .debug$S                   0000000180000000     kernel32:KERNEL32.dll
 0000:fff9a000       .debug$S                   0000000180000000     kernel32:KERNEL32.dll
 0000:fff9a000       .debug$S                   0000000180000000     kernel32:KERNEL32.dll
 0000:fff9a000       .debug$S                   0000000180000000     kernel32:KERNEL32.dll
 0000:fff9a000       .debug$S                   0000000180000000     kernel32:KERNEL32.dll
 0000:fff9a000       .debug$S                   0000000180000000     kernel32:KERNEL32.dll
 0000:fff9a000       .debug$S                   0000000180000000     kernel32:KERNEL32.dll
 0000:fff9a000       .debug$S                   0000000180000000     kernel32:KERNEL32.dll
 0000:fff9a000       .debug$S                   0000000180000000     kernel32:KERNEL32.dll
 0000:fff9a000       .debug$S                   0000000180000000     kernel32:KERNEL32.dll
 0000:fff9a000       .debug$S                   0000000180000000     kernel32:KERNEL32.dll
 0000:fff9a000       .debug$S                   0000000180000000     kernel32:KERNEL32.dll
 0000:fff9a000       .debug$S                   0000000180000000     kernel32:KERNEL32.dll
 0000:fff9a000       .debug$S                   0000000180000000     kernel32:KERNEL32.dll
 0000:fff9a000       .debug$S                   0000000180000000     kernel32:KERNEL32.dll
 0000:fff9a000       .debug$S                   0000000180000000     kernel32:KERNEL32.dll
 0000:fff9a000       .debug$S                   0000000180000000     kernel32:KERNEL32.dll
 0000:fff9a000       .debug$S                   0000000180000000     kernel32:KERNEL32.dll
 0000:fff9a000       .debug$S                   0000000180000000     kernel32:KERNEL32.dll
 0000:fff9a000       .debug$S                   0000000180000000     kernel32:KERNEL32.dll
 0000:fff9a000       .debug$S                   0000000180000000     kernel32:KERNEL32.dll
 0000:fff9a000       .debug$S                   0000000180000000     kernel32:KERNEL32.dll
 0000:fff9a000       .debug$S                   0000000180000000     kernel32:KERNEL32.dll
 0000:fff9a000       .debug$S                   0000000180000000     kernel32:KERNEL32.dll
 0000:fff9a000       .debug$S                   0000000180000000     kernel32:KERNEL32.dll
 0000:fff9a000       .debug$S                   0000000180000000     kernel32:KERNEL32.dll
 0000:fff9a000       .debug$S                   0000000180000000     kernel32:KERNEL32.dll
 0000:fff9a000       .debug$S                   0000000180000000     kernel32:KERNEL32.dll
 0000:fff9a000       .debug$S                   0000000180000000     kernel32:KERNEL32.dll
 0000:fff9a000       .debug$S                   0000000180000000     kernel32:KERNEL32.dll
 0000:fff9a000       .debug$S                   0000000180000000     kernel32:KERNEL32.dll
 0000:fff9a000       .debug$S                   0000000180000000     kernel32:KERNEL32.dll
 0000:fff9a000       .debug$S                   0000000180000000     kernel32:KERNEL32.dll
 0000:fff9a000       .debug$S                   0000000180000000     kernel32:KERNEL32.dll
 0000:fff9a000       .debug$S                   0000000180000000     kernel32:KERNEL32.dll
 0000:fff9a000       .debug$S                   0000000180000000     kernel32:KERNEL32.dll
 0000:fff9a000       .debug$S                   0000000180000000     kernel32:KERNEL32.dll
 0000:fff9a000       .debug$S                   0000000180000000     kernel32:KERNEL32.dll
 0000:fff9a000       .debug$S                   0000000180000000     kernel32:KERNEL32.dll
 0000:fff9a000       .debug$S                   0000000180000000     kernel32:KERNEL32.dll
 0000:fff9a000       .debug$S                   0000000180000000     kernel32:KERNEL32.dll
 0000:fff9a000       .debug$S                   0000000180000000     kernel32:KERNEL32.dll
 0000:fff9a000       .debug$S                   0000000180000000     kernel32:KERNEL32.dll
 0000:fff9a000       .debug$S                   0000000180000000     kernel32:KERNEL32.dll
 0000:fff9a000       .debug$S                   0000000180000000     mpr:MPR.dll
 0000:fff9a000       .debug$S                   0000000180000000     mpr:MPR.dll
 0000:fff9a000       .debug$S                   0000000180000000     ole32:ole32.dll
 0000:fff9a000       .debug$S                   0000000180000000     ole32:ole32.dll
 0000:fff9a000       .debug$S                   0000000180000000     ole32:ole32.dll
 0000:fff9a000       .debug$S                   0000000180000000     oleaut32:OLEAUT32.dll
 0000:fff9a000       .debug$S                   0000000180000000     oleaut32:OLEAUT32.dll
 0000:fff9a000       .debug$S                   0000000180000000     oleaut32:OLEAUT32.dll
 0000:fff9a000       .debug$S                   0000000180000000     psapi:PSAPI.DLL
 0000:fff9a000       .debug$S                   0000000180000000     psapi:PSAPI.DLL
 0000:fff9a000       .debug$S                   0000000180000000     user32:USER32.dll
 0000:fff9a000       .debug$S                   0000000180000000     user32:USER32.dll
 0000:fff9a000       .debug$S                   0000000180000000     user32:USER32.dll
 0000:fff9a000       .debug$S                   0000000180000000     user32:USER32.dll
 0000:fff9a000       .debug$S                   0000000180000000     user32:USER32.dll
 0000:fff9a000       .debug$S                   0000000180000000     user32:USER32.dll
 0000:fff9a000       .debug$S                   0000000180000000     user32:USER32.dll
 0000:fff9a000       .debug$S                   0000000180000000     user32:USER32.dll
 0000:fff9a000       .debug$S                   0000000180000000     user32:USER32.dll
 0000:fff9a000       .debug$S                   0000000180000000     user32:USER32.dll
 0000:fff9a000       .debug$S                   0000000180000000     user32:USER32.dll
 0000:fff9a000       .debug$S                   0000000180000000     user32:USER32.dll
 0000:fff9a000       .debug$S                   0000000180000000     version:VERSION.dll
 0000:fff9a000       .debug$S                   0000000180000000     version:VERSION.dll
 0000:fff9a000       .debug$S                   0000000180000000     version:VERSION.dll
 0001:00000410       Table                      0000000180001410     libvcruntime:memset.obj
 0001:00000ae0       ??__F?m_PanelModesDataLocal@Plist@@0V?$vector@Umode@@V?$allocator@Umode@@@std@@@std@@A@@YAXXZ 0000000180001ae0 f   fileio.obj
 0001:00000af0       ??__F?m_PanelModesDataRemote@Plist@@0V?$vector@Umode@@V?$allocator@Umode@@@std@@@std@@A@@YAXXZ 0000000180001af0 f   fileio.obj
 0001:00000b00       ??__FhDebugToken@@YAXXZ    0000000180001b00 f   Plist.obj
 0001:00000b10       ??__Einitlocks@std@@YAXXZ  0000000180001b10 f   libcpmt:xlock.obj
 0001:00000b38       ??__Eclassic_locale@std@@YAXXZ 0000000180001b38 f   libcpmt:locale0.obj
 0001:00000b48       ??__F_Fac_tidy_reg@std@@YAXXZ 0000000180001b48 f   libcpmt:locale0.obj
 0001:00000b58       ??__Einitlocks@std@@YAXXZ  0000000180001b58 f   libcpmt:iosptrs.obj
 0001:00000b80       ??__Finit_atexit@@YAXXZ    0000000180001b80 f   libcpmt:iosptrs.obj
 0001:00001f30       $LN108                     0000000180002f30     format.obj
 0001:00001f31       $LN109                     0000000180002f31     format.obj
 0001:00001f32       $LN110                     0000000180002f32     format.obj
 0001:00001f33       $LN111                     0000000180002f33     format.obj
 0001:00001f34       $LN112                     0000000180002f34     format.obj
 0001:00001f35       $LN113                     0000000180002f35     format.obj
 0001:00001f36       $LN114                     0000000180002f36     format.obj
 0001:00001f37       $LN115                     0000000180002f37     format.obj
 0001:00001f38       $LN116                     0000000180002f38     format.obj
 0001:00001f39       $LN117                     0000000180002f39     format.obj
 0001:00001f3a       $LN118                     0000000180002f3a     format.obj
 0001:00001f3b       $LN119                     0000000180002f3b     format.obj
 0001:00002390       $LN35                      0000000180003390     format.obj
 0001:00002398       $LN36                      0000000180003398     format.obj
 0001:00004e78       $LN76                      0000000180005e78     format.obj
 0001:00005a18       $LN49                      0000000180006a18     format.obj
 0001:000066d0       ?GetFileName@@YA?AV?$basic_string@_WU?$char_traits@_W@std@@V?$allocator@_W@2@@std@@PEAX@Z 00000001800076d0 f   handles.obj
 0001:000068a8       $LN493                     00000001800078a8     handles.obj
 0001:000068b0       ?GetFileNameThread@test@?4??GetFileName@@YA?AV?$basic_string@_WU?$char_traits@_W@std@@V?$allocator@_W@2@@std@@PEAX@Z@SAK0@Z 00000001800078b0 f   handles.obj
 0001:000068f0       ??R<lambda_1>@?1??GetUserAccountID@@YA@XZ@QEBA?AV?$basic_string@_WU?$char_traits@_W@std@@V?$allocator@_W@2@@std@@XZ 00000001800078f0 f   handles.obj
 0001:00006ac0       ?GetNameByType@@YA?AV?$basic_string@_WU?$char_traits@_W@std@@V?$allocator@_W@2@@std@@PEAXGPEAVPerfThread@@@Z 0000000180007ac0 f   handles.obj
 0001:0000705c       $LN1239                    000000018000805c     handles.obj
 0001:00007060       $LN1240                    0000000180008060     handles.obj
 0001:00007064       $LN1241                    0000000180008064     handles.obj
 0001:00007068       $LN1242                    0000000180008068     handles.obj
 0001:0000706c       $LN1243                    000000018000806c     handles.obj
 0001:00007070       $LN1244                    0000000180008070     handles.obj
 0001:00007078       ?duplicate_handle@@YA?AV?$unique_ptr@XUhandle_closer@@@std@@PEAXK@Z 0000000180008078 f   handles.obj
 0001:00007828       $LN690                     0000000180008828     handles.obj
 0001:000084a0       $LN590                     00000001800094a0     handles.obj
 0001:000084a4       $LN591                     00000001800094a4     handles.obj
 0001:000084a8       $LN592                     00000001800094a8     handles.obj
 0001:000084ac       $LN593                     00000001800094ac     handles.obj
 0001:000084b0       $LN594                     00000001800094b0     handles.obj
 0001:000084b4       $LN595                     00000001800094b4     handles.obj
 0001:000084b8       $LN596                     00000001800094b8     handles.obj
 0001:000084bc       $LN597                     00000001800094bc     handles.obj
 0001:000084c0       $LN598                     00000001800094c0     handles.obj
 0001:000084c4       $LN599                     00000001800094c4     handles.obj
 0001:000084c8       $LN600                     00000001800094c8     handles.obj
 0001:000084cc       $LN601                     00000001800094cc     handles.obj
 0001:000084d0       $LN602                     00000001800094d0     handles.obj
 0001:000084d4       $LN603                     00000001800094d4     handles.obj
 0001:000084d8       $LN604                     00000001800094d8     handles.obj
 0001:00008bf0       $LN166                     0000000180009bf0     handles.obj
 0001:00008bf4       $LN167                     0000000180009bf4     handles.obj
 0001:00008bf8       $LN168                     0000000180009bf8     handles.obj
 0001:00008bfc       $LN169                     0000000180009bfc     handles.obj
 0001:00008c00       $LN170                     0000000180009c00     handles.obj
 0001:00008c04       $LN171                     0000000180009c04     handles.obj
 0001:00008c08       $LN172                     0000000180009c08     handles.obj
 0001:00008c0c       $LN173                     0000000180009c0c     handles.obj
 0001:00008c10       $LN174                     0000000180009c10     handles.obj
 0001:00008c14       $LN175                     0000000180009c14     handles.obj
 0001:00008c18       $LN176                     0000000180009c18     handles.obj
 0001:00008c1c       $LN177                     0000000180009c1c     handles.obj
 0001:00008c20       $LN178                     0000000180009c20     handles.obj
 0001:00008c24       $LN179                     0000000180009c24     handles.obj
 0001:00008c28       $LN180                     0000000180009c28     handles.obj
 0001:00009120       $LN25                      000000018000a120     handles.obj
 0001:00009121       $LN26                      000000018000a121     handles.obj
 0001:00009122       $LN27                      000000018000a122     handles.obj
 0001:00009123       $LN28                      000000018000a123     handles.obj
 0001:00009124       $LN29                      000000018000a124     handles.obj
 0001:00009125       $LN30                      000000018000a125     handles.obj
 0001:00009126       $LN31                      000000018000a126     handles.obj
 0001:00009127       $LN32                      000000018000a127     handles.obj
 0001:00009128       $LN33                      000000018000a128     handles.obj
 0001:00009129       $LN34                      000000018000a129     handles.obj
 0001:0000912a       $LN35                      000000018000a12a     handles.obj
 0001:0000912b       $LN36                      000000018000a12b     handles.obj
 0001:0000912c       $LN37                      000000018000a12c     handles.obj
 0001:0000912d       $LN38                      000000018000a12d     handles.obj
 0001:0000912e       $LN39                      000000018000a12e     handles.obj
 0001:0000912f       $LN40                      000000018000a12f     handles.obj
 0001:00009130       $LN41                      000000018000a130     handles.obj
 0001:00009131       $LN42                      000000018000a131     handles.obj
 0001:00009132       $LN43                      000000018000a132     handles.obj
 0001:00009133       $LN44                      000000018000a133     handles.obj
 0001:00009134       $LN45                      000000018000a134     handles.obj
 0001:00009135       $LN46                      000000018000a135     handles.obj
 0001:00009136       $LN47                      000000018000a136     handles.obj
 0001:00009137       $LN48                      000000018000a137     handles.obj
 0001:00009138       $LN49                      000000018000a138     handles.obj
 0001:00009139       $LN50                      000000018000a139     handles.obj
 0001:0000913a       $LN51                      000000018000a13a     handles.obj
 0001:0000913b       $LN52                      000000018000a13b     handles.obj
 0001:0000913c       $LN53                      000000018000a13c     handles.obj
 0001:0000913d       $LN54                      000000018000a13d     handles.obj
 0001:0000913e       $LN55                      000000018000a13e     handles.obj
 0001:0000913f       $LN56                      000000018000a13f     handles.obj
 0001:00009140       $LN57                      000000018000a140     handles.obj
 0001:00009141       $LN58                      000000018000a141     handles.obj
 0001:00009142       $LN59                      000000018000a142     handles.obj
 0001:00009143       $LN60                      000000018000a143     handles.obj
 0001:00009144       $LN61                      000000018000a144     handles.obj
 0001:00009145       $LN62                      000000018000a145     handles.obj
 0001:00009146       $LN63                      000000018000a146     handles.obj
 0001:00009147       $LN64                      000000018000a147     handles.obj
 0001:00009148       $LN65                      000000018000a148     handles.obj
 0001:00009149       $LN66                      000000018000a149     handles.obj
 0001:0000914a       $LN67                      000000018000a14a     handles.obj
 0001:0000914b       $LN68                      000000018000a14b     handles.obj
 0001:0000914c       $LN69                      000000018000a14c     handles.obj
 0001:0000914d       $LN70                      000000018000a14d     handles.obj
 0001:0000914e       $LN71                      000000018000a14e     handles.obj
 0001:0000914f       $LN72                      000000018000a14f     handles.obj
 0001:00009150       $LN73                      000000018000a150     handles.obj
 0001:00009151       $LN74                      000000018000a151     handles.obj
 0001:00009152       $LN75                      000000018000a152     handles.obj
 0001:00009153       $LN76                      000000018000a153     handles.obj
 0001:00009154       $LN77                      000000018000a154     handles.obj
 0001:00009155       $LN78                      000000018000a155     handles.obj
 0001:00009156       $LN79                      000000018000a156     handles.obj
 0001:00009157       $LN80                      000000018000a157     handles.obj
 0001:0000bf58       $LN132                     000000018000cf58     handles.obj
 0001:0000c2a8       $LN132                     000000018000d2a8     handles.obj
 0001:0000c45c       $LN45                      000000018000d45c     handles.obj
 0001:0000c45d       $LN46                      000000018000d45d     handles.obj
 0001:0000c45e       $LN47                      000000018000d45e     handles.obj
 0001:0000c45f       $LN48                      000000018000d45f     handles.obj
 0001:0000c460       $LN49                      000000018000d460     handles.obj
 0001:0000c461       $LN50                      000000018000d461     handles.obj
 0001:0000c462       $LN51                      000000018000d462     handles.obj
 0001:0000c463       $LN52                      000000018000d463     handles.obj
 0001:0000c464       $LN53                      000000018000d464     handles.obj
 0001:0000c465       $LN54                      000000018000d465     handles.obj
 0001:0000c466       $LN55                      000000018000d466     handles.obj
 0001:0000c467       $LN56                      000000018000d467     handles.obj
 0001:0000c468       $LN57                      000000018000d468     handles.obj
 0001:0000c469       $LN58                      000000018000d469     handles.obj
 0001:0000c46a       $LN59                      000000018000d46a     handles.obj
 0001:0000c46b       $LN60                      000000018000d46b     handles.obj
 0001:0000c6c8       $LN93                      000000018000d6c8     handles.obj
 0001:0000cd48       $LN184                     000000018000dd48     handles.obj
 0001:0000cd4c       $LN185                     000000018000dd4c     handles.obj
 0001:0000cd50       $LN186                     000000018000dd50     handles.obj
 0001:0000cd54       $LN187                     000000018000dd54     handles.obj
 0001:0000cd58       $LN188                     000000018000dd58     handles.obj
 0001:0000cd5c       $LN189                     000000018000dd5c     handles.obj
 0001:0000cd60       $LN190                     000000018000dd60     handles.obj
 0001:0000cd64       $LN191                     000000018000dd64     handles.obj
 0001:0000cd68       $LN192                     000000018000dd68     handles.obj
 0001:0000cd6c       $LN193                     000000018000dd6c     handles.obj
 0001:0000cd70       $LN194                     000000018000dd70     handles.obj
 0001:0000cd74       $LN195                     000000018000dd74     handles.obj
 0001:0000cd78       $LN196                     000000018000dd78     handles.obj
 0001:0000cd7c       $LN197                     000000018000dd7c     handles.obj
 0001:0000cd80       $LN198                     000000018000dd80     handles.obj
 0001:0000cd84       $LN199                     000000018000dd84     handles.obj
 0001:0000e84c       $LN172                     000000018000f84c     handles.obj
 0001:0000e850       $LN173                     000000018000f850     handles.obj
 0001:0000e854       $LN174                     000000018000f854     handles.obj
 0001:0000e858       $LN175                     000000018000f858     handles.obj
 0001:0000e85c       $LN176                     000000018000f85c     handles.obj
 0001:0000e860       $LN177                     000000018000f860     handles.obj
 0001:0000e864       $LN178                     000000018000f864     handles.obj
 0001:0000e868       $LN179                     000000018000f868     handles.obj
 0001:0000e86c       $LN180                     000000018000f86c     handles.obj
 0001:0000e870       $LN181                     000000018000f870     handles.obj
 0001:0000e874       $LN182                     000000018000f874     handles.obj
 0001:0000e878       $LN183                     000000018000f878     handles.obj
 0001:0000e87c       $LN184                     000000018000f87c     handles.obj
 0001:0000e880       $LN185                     000000018000f880     handles.obj
 0001:0000e884       $LN186                     000000018000f884     handles.obj
 0001:0000eb84       $LN172                     000000018000fb84     handles.obj
 0001:0000eb88       $LN173                     000000018000fb88     handles.obj
 0001:0000eb8c       $LN174                     000000018000fb8c     handles.obj
 0001:0000eb90       $LN175                     000000018000fb90     handles.obj
 0001:0000eb94       $LN176                     000000018000fb94     handles.obj
 0001:0000eb98       $LN177                     000000018000fb98     handles.obj
 0001:0000eb9c       $LN178                     000000018000fb9c     handles.obj
 0001:0000eba0       $LN179                     000000018000fba0     handles.obj
 0001:0000eba4       $LN180                     000000018000fba4     handles.obj
 0001:0000eba8       $LN181                     000000018000fba8     handles.obj
 0001:0000ebac       $LN182                     000000018000fbac     handles.obj
 0001:0000ebb0       $LN183                     000000018000fbb0     handles.obj
 0001:0000ebb4       $LN184                     000000018000fbb4     handles.obj
 0001:0000ebb8       $LN185                     000000018000fbb8     handles.obj
 0001:0000ebbc       $LN186                     000000018000fbbc     handles.obj
 0001:0000f068       $LN194                     0000000180010068     handles.obj
 0001:0000f06c       $LN195                     000000018001006c     handles.obj
 0001:0000f070       $LN196                     0000000180010070     handles.obj
 0001:0000f074       $LN197                     0000000180010074     handles.obj
 0001:0000f078       $LN198                     0000000180010078     handles.obj
 0001:0000f07c       $LN199                     000000018001007c     handles.obj
 0001:0000f080       $LN200                     0000000180010080     handles.obj
 0001:0000f084       $LN201                     0000000180010084     handles.obj
 0001:0000f088       $LN202                     0000000180010088     handles.obj
 0001:0000f08c       $LN203                     000000018001008c     handles.obj
 0001:0000f090       $LN204                     0000000180010090     handles.obj
 0001:0000f094       $LN205                     0000000180010094     handles.obj
 0001:0000f098       $LN206                     0000000180010098     handles.obj
 0001:0000f09c       $LN207                     000000018001009c     handles.obj
 0001:0000f0a0       $LN208                     00000001800100a0     handles.obj
 0001:0000f0a4       $LN209                     00000001800100a4     handles.obj
 0001:00014cd0       $LN42                      0000000180015cd0     Pcfg.obj
 0001:00014cd1       $LN43                      0000000180015cd1     Pcfg.obj
 0001:00014cd2       $LN44                      0000000180015cd2     Pcfg.obj
 0001:00014cd3       $LN45                      0000000180015cd3     Pcfg.obj
 0001:00014cd4       $LN46                      0000000180015cd4     Pcfg.obj
 0001:00014cd5       $LN47                      0000000180015cd5     Pcfg.obj
 0001:00014cd6       $LN48                      0000000180015cd6     Pcfg.obj
 0001:00014cd7       $LN49                      0000000180015cd7     Pcfg.obj
 0001:00014cd8       $LN50                      0000000180015cd8     Pcfg.obj
 0001:00014cd9       $LN51                      0000000180015cd9     Pcfg.obj
 0001:00014cda       $LN52                      0000000180015cda     Pcfg.obj
 0001:00014cdb       $LN53                      0000000180015cdb     Pcfg.obj
 0001:00014e9c       $LN50                      0000000180015e9c     Pcfg.obj
 0001:00014e9d       $LN51                      0000000180015e9d     Pcfg.obj
 0001:00014e9e       $LN52                      0000000180015e9e     Pcfg.obj
 0001:00014e9f       $LN53                      0000000180015e9f     Pcfg.obj
 0001:00014ea0       $LN54                      0000000180015ea0     Pcfg.obj
 0001:00014ea1       $LN55                      0000000180015ea1     Pcfg.obj
 0001:00014ea2       $LN56                      0000000180015ea2     Pcfg.obj
 0001:00014ea3       $LN57                      0000000180015ea3     Pcfg.obj
 0001:00014ea4       $LN58                      0000000180015ea4     Pcfg.obj
 0001:00014ea5       $LN59                      0000000180015ea5     Pcfg.obj
 0001:00014ea6       $LN60                      0000000180015ea6     Pcfg.obj
 0001:00014ea7       $LN61                      0000000180015ea7     Pcfg.obj
 0001:000151c8       $LN18                      00000001800161c8     Pcfg.obj
 0001:00015250       $LN21                      0000000180016250     Pcfg.obj
 0001:00015251       $LN22                      0000000180016251     Pcfg.obj
 0001:00015252       $LN23                      0000000180016252     Pcfg.obj
 0001:00015253       $LN24                      0000000180016253     Pcfg.obj
 0001:00015254       $LN25                      0000000180016254     Pcfg.obj
 0001:00015255       $LN26                      0000000180016255     Pcfg.obj
 0001:00015256       $LN27                      0000000180016256     Pcfg.obj
 0001:00015257       $LN28                      0000000180016257     Pcfg.obj
 0001:00015258       $LN29                      0000000180016258     Pcfg.obj
 0001:00015259       $LN30                      0000000180016259     Pcfg.obj
 0001:0001525a       $LN31                      000000018001625a     Pcfg.obj
 0001:0001525b       $LN32                      000000018001625b     Pcfg.obj
 0001:00015410       $LN48                      0000000180016410     Pcfg.obj
 0001:00015411       $LN49                      0000000180016411     Pcfg.obj
 0001:00015412       $LN50                      0000000180016412     Pcfg.obj
 0001:00015413       $LN51                      0000000180016413     Pcfg.obj
 0001:00015414       $LN52                      0000000180016414     Pcfg.obj
 0001:00015415       $LN53                      0000000180016415     Pcfg.obj
 0001:00015416       $LN54                      0000000180016416     Pcfg.obj
 0001:00015417       $LN55                      0000000180016417     Pcfg.obj
 0001:00015418       $LN56                      0000000180016418     Pcfg.obj
 0001:00015419       $LN57                      0000000180016419     Pcfg.obj
 0001:0001541a       $LN58                      000000018001641a     Pcfg.obj
 0001:0001541b       $LN59                      000000018001641b     Pcfg.obj
 0001:00015f28       ?ui64toa_width@@YA?AV?$basic_string@_WU?$char_traits@_W@std@@V?$allocator@_W@2@@std@@_KI_N@Z 0000000180016f28 f   Pclass.obj
 0001:000163c0       ?PrintTitle@@YA?AV?$basic_string@_WU?$char_traits@_W@std@@V?$allocator@_W@2@@std@@V?$basic_string_view@_WU?$char_traits@_W@std@@@2@@Z 00000001800173c0 f   Pclass.obj
 0001:000166b8       ?TranslateMode@@YA_NAEBV?$basic_string@_WU?$char_traits@_W@std@@V?$allocator@_W@2@@std@@AEAV12@@Z 00000001800176b8 f   Pclass.obj
 0001:0001690c       $LN450                     000000018001790c     Pclass.obj
 0001:0001690d       $LN451                     000000018001790d     Pclass.obj
 0001:0001690e       $LN452                     000000018001790e     Pclass.obj
 0001:0001690f       $LN453                     000000018001790f     Pclass.obj
 0001:00016910       $LN454                     0000000180017910     Pclass.obj
 0001:00016911       $LN455                     0000000180017911     Pclass.obj
 0001:00016912       $LN456                     0000000180017912     Pclass.obj
 0001:00016913       $LN457                     0000000180017913     Pclass.obj
 0001:00016914       $LN458                     0000000180017914     Pclass.obj
 0001:00016915       $LN459                     0000000180017915     Pclass.obj
 0001:00016916       $LN460                     0000000180017916     Pclass.obj
 0001:00016917       $LN461                     0000000180017917     Pclass.obj
 0001:00016918       $LN462                     0000000180017918     Pclass.obj
 0001:00016919       $LN463                     0000000180017919     Pclass.obj
 0001:0001691a       $LN464                     000000018001791a     Pclass.obj
 0001:0001691b       $LN465                     000000018001791b     Pclass.obj
 0001:0001691c       $LN466                     000000018001791c     Pclass.obj
 0001:0001691d       $LN467                     000000018001791d     Pclass.obj
 0001:0001691e       $LN468                     000000018001791e     Pclass.obj
 0001:0001691f       $LN469                     000000018001791f     Pclass.obj
 0001:00017588       ??$format@UFMT_COMPILE_STRING@?1???R<lambda_1>@?4??InitializePanelModes@Plist@@SAXXZ@QEBA@XZ@AEA_K@@YA?A_P$$QEAUFMT_COMPILE_STRING@?1???R<lambda_1>@?4??InitializePanelModes@Plist@@SAXXZ@QEBA@XZ@AEA_K@Z 0000000180018588 f   Pclass.obj
 0001:00017948       ?generate_titles@@YAXAEBV?$basic_string@_WU?$char_traits@_W@std@@V?$allocator@_W@2@@std@@AEAUPanelMode@@@Z 0000000180018948 f   Pclass.obj
 0001:00017b98       $LN92                      0000000180018b98     Pclass.obj
 0001:00017b99       $LN93                      0000000180018b99     Pclass.obj
 0001:00017b9a       $LN94                      0000000180018b9a     Pclass.obj
 0001:00017b9b       $LN95                      0000000180018b9b     Pclass.obj
 0001:00017b9c       $LN96                      0000000180018b9c     Pclass.obj
 0001:00017b9d       $LN97                      0000000180018b9d     Pclass.obj
 0001:00017b9e       $LN98                      0000000180018b9e     Pclass.obj
 0001:00017b9f       $LN99                      0000000180018b9f     Pclass.obj
 0001:00017ba0       $LN100                     0000000180018ba0     Pclass.obj
 0001:00017ba1       $LN101                     0000000180018ba1     Pclass.obj
 0001:00017ba2       $LN102                     0000000180018ba2     Pclass.obj
 0001:00017ba3       $LN103                     0000000180018ba3     Pclass.obj
 0001:00017ba4       $LN104                     0000000180018ba4     Pclass.obj
 0001:00017ba5       $LN105                     0000000180018ba5     Pclass.obj
 0001:00017ba6       $LN106                     0000000180018ba6     Pclass.obj
 0001:00017ba7       $LN107                     0000000180018ba7     Pclass.obj
 0001:00017ba8       $LN108                     0000000180018ba8     Pclass.obj
 0001:00017ba9       $LN109                     0000000180018ba9     Pclass.obj
 0001:00017baa       $LN110                     0000000180018baa     Pclass.obj
 0001:00017bab       $LN111                     0000000180018bab     Pclass.obj
 0001:00018060       ?EnumWndProc@@YAHPEAUHWND__@@_J@Z 0000000180019060 f   Pclass.obj
 0001:000181a0       $LN89                      00000001800191a0     Pclass.obj
 0001:00018da0       $LN1859                    0000000180019da0     Pclass.obj
 0001:00018da4       $LN1860                    0000000180019da4     Pclass.obj
 0001:00018da8       $LN1861                    0000000180019da8     Pclass.obj
 0001:00018dac       $LN1862                    0000000180019dac     Pclass.obj
 0001:00018db0       $LN1863                    0000000180019db0     Pclass.obj
 0001:00018db4       $LN1864                    0000000180019db4     Pclass.obj
 0001:00018db8       $LN1865                    0000000180019db8     Pclass.obj
 0001:00018dbc       $LN1866                    0000000180019dbc     Pclass.obj
 0001:00018dc0       $LN1867                    0000000180019dc0     Pclass.obj
 0001:00018dc4       $LN1868                    0000000180019dc4     Pclass.obj
 0001:00018dc8       $LN1869                    0000000180019dc8     Pclass.obj
 0001:00018dcc       $LN1870                    0000000180019dcc     Pclass.obj
 0001:00018dd0       $LN1871                    0000000180019dd0     Pclass.obj
 0001:00018dd4       $LN1872                    0000000180019dd4     Pclass.obj
 0001:00018dd8       $LN1873                    0000000180019dd8     Pclass.obj
 0001:00018ddc       $LN1874                    0000000180019ddc     Pclass.obj
 0001:00018de0       $LN1875                    0000000180019de0     Pclass.obj
 0001:00018de4       $LN1876                    0000000180019de4     Pclass.obj
 0001:00018de8       $LN1877                    0000000180019de8     Pclass.obj
 0001:00018dec       $LN1878                    0000000180019dec     Pclass.obj
 0001:00018e58       ?window_style@@YA@PEAUHWND__@@@Z 0000000180019e58 f   Pclass.obj
 0001:00019018       ?window_ex_style@@YA@PEAUHWND__@@@Z 000000018001a018 f   Pclass.obj
 0001:00019190       ?DumpNTCounters@@YAXPEAXAEAVPerfThread@@KK@Z 000000018001a190 f   Pclass.obj
 0001:0001b188       ??$format@UFMT_COMPILE_STRING@?1???R<lambda_18>@?EB@??GetFiles@Plist@@QEAAHPEAUPluginPanelItem@@_KHPEAPEB_W1AEAUoptions@@@Z@QEBA@XZ@PEB_WPEB_WHPEB_WPEB_W@@YA?A_P$$QEAUFMT_COMPILE_STRING@?1???R<lambda_18>@?EB@??GetFiles@Plist@@QEAAHPEAUPluginPanelItem@@_KHPEAPEB_W1AEAUoptions@@@Z@QEBA@XZ@$$QEAPEB_W5$$QEAH55@Z 000000018001c188 f   Pclass.obj
 0001:0001b88c       $LN872                     000000018001c88c     Pclass.obj
 0001:0001b890       $LN873                     000000018001c890     Pclass.obj
 0001:0001b894       $LN874                     000000018001c894     Pclass.obj
 0001:0001b898       $LN875                     000000018001c898     Pclass.obj
 0001:0001b89c       $LN876                     000000018001c89c     Pclass.obj
 0001:0001d7c0       $LN102                     000000018001e7c0     Pclass.obj
 0001:0001d7c8       $LN103                     000000018001e7c8     Pclass.obj
 0001:0001ed40       $LN61                      000000018001fd40     Pclass.obj
 0001:0001f718       $LN132                     0000000180020718     Pclass.obj
 0001:0001f9c0       $LN168                     00000001800209c0     Pclass.obj
 0001:0001fb48       $LN87                      0000000180020b48     Pclass.obj
 0001:00020078       $LN176                     0000000180021078     Pclass.obj
 0001:00020078       $LN148                     0000000180021078     perfthread.obj
 0001:00020d00       $LN944                     0000000180021d00     perfthread.obj
 0001:00021080       $LN114                     0000000180022080     perfthread.obj
 0001:00022d38       $LN1156                    0000000180023d38     perfthread.obj
 0001:000231b8       $LN62                      00000001800241b8     perfthread.obj
 0001:00023438       $LN229                     0000000180024438     perfthread.obj
 0001:00023640       $LN139                     0000000180024640     perfthread.obj
 0001:00023648       $LN140                     0000000180024648     perfthread.obj
 0001:00023650       ??$transform@V?$_List_const_iterator@V?$_List_val@U?$_List_simple_types@U?$pair@$$CBKUProcessPerfData@@@std@@@std@@@std@@@std@@V?$back_insert_iterator@V?$vector@UProcessPerfData@@V?$allocator@UProcessPerfData@@@std@@@std@@@2@V<lambda_1>@?2??RefreshWMIData@PerfThread@@AEAAXXZ@@std@@YA?AV?$back_insert_iterator@V?$vector@UProcessPerfData@@V?$allocator@UProcessPerfData@@@std@@@std@@@0@V?$_List_const_iterator@V?$_List_val@U?$_List_simple_types@U?$pair@$$CBKUProcessPerfData@@@std@@@std@@@std@@@0@0V10@V<lambda_1>@?2??RefreshWMIData@PerfThread@@AEAAXXZ@@Z 0000000180024650 f   perfthread.obj
 0001:00023fd0       $LN130                     0000000180024fd0     perfthread.obj
 0001:00024228       ?FreeUserData@@YAXQEAXQEBUFarPanelItemFreeInfo@@@Z 0000000180025228 f   Plist.obj
 0001:000246c8       $LN550                     00000001800256c8     Plist.obj
 0001:00024cf0       ?print_module_impl@@YAXQEAXAEBV?$basic_string@_WU?$char_traits@_W@std@@V?$allocator@_W@2@@std@@KAEBUoptions@@AEBV?$function@$$A6A_NPEA_W_K@Z@2@@Z 0000000180025cf0 f   Plist.obj
 0001:00025e20       ??$print_module@PEAX@@YAXQEAXPEAXKAEAUoptions@@AEBV?$function@$$A6A_NPEA_W_K@Z@std@@@Z 0000000180026e20 f   Plist.obj
 0001:00026150       $LN225                     0000000180027150     Plist.obj
 0001:00026158       $LN226                     0000000180027158     Plist.obj
 0001:00026160       ?_Delete_this@?$_Func_impl_no_alloc@V<lambda_3>@?N@??PrintModules@@YAXPEAXKAEAUoptions@@@Z@_NPEA_W_K@std@@EEAAX_N@Z 0000000180027160 f i Plist.obj
 0001:00026178       ?_Get@?$_Func_impl_no_alloc@V<lambda_3>@?N@??PrintModules@@YAXPEAXKAEAUoptions@@@Z@_NPEA_W_K@std@@EEBAPEBXXZ 0000000180027178 f i Plist.obj
 0001:00026178       ?_Get@?$_Func_impl_no_alloc@V<lambda_1>@?1??GetProcessInt@WMIConnection@@AEAAKKPEB_W@Z@XAEBUtagVARIANT@@@std@@EEBAPEBXXZ 0000000180027178 f i wmi.obj
 0001:00026178       ?_Get@?$_Func_impl_no_alloc@V<lambda_1>@?1??GetProcessString@WMIConnection@@AEAA?AV?$basic_string@_WU?$char_traits@_W@std@@V?$allocator@_W@2@@std@@KPEB_W@Z@XAEBUtagVARIANT@@@std@@EEBAPEBXXZ 0000000180027178 f i wmi.obj
 0001:000261f0       ?_Target_type@?$_Func_impl_no_alloc@V<lambda_3>@?N@??PrintModules@@YAXPEAXKAEAUoptions@@@Z@_NPEA_W_K@std@@EEBAAEBVtype_info@@XZ 00000001800271f0 f   Plist.obj
 0001:00026200       ?_Do_call@?$_Func_impl_no_alloc@V<lambda_3>@?N@??PrintModules@@YAXPEAXKAEAUoptions@@@Z@_NPEA_W_K@std@@EEAA_N$$QEAPEA_W$$QEA_K@Z 0000000180027200 f   Plist.obj
 0001:00026238       ?_Copy@?$_Func_impl_no_alloc@V<lambda_3>@?N@??PrintModules@@YAXPEAXKAEAUoptions@@@Z@_NPEA_W_K@std@@EEBAPEAV?$_Func_base@_NPEA_W_K@2@PEAX@Z 0000000180027238 f   Plist.obj
 0001:00026238       ?_Move@?$_Func_impl_no_alloc@V<lambda_3>@?N@??PrintModules@@YAXPEAXKAEAUoptions@@@Z@_NPEA_W_K@std@@EEAAPEAV?$_Func_base@_NPEA_W_K@2@PEAX@Z 0000000180027238 f   Plist.obj
 0001:00027638       ?_Delete_this@?$_Func_impl_no_alloc@V<lambda_1>@?1??GetProcessInt@WMIConnection@@AEAAKKPEB_W@Z@XAEBUtagVARIANT@@@std@@EEAAX_N@Z 0000000180028638 f   wmi.obj
 0001:00027638       ?_Delete_this@?$_Func_impl_no_alloc@V<lambda_1>@?1??GetProcessString@WMIConnection@@AEAA?AV?$basic_string@_WU?$char_traits@_W@std@@V?$allocator@_W@2@@std@@KPEB_W@Z@XAEBUtagVARIANT@@@std@@EEAAX_N@Z 0000000180028638 f   wmi.obj
 0001:00027650       ?_Target_type@?$_Func_impl_no_alloc@V<lambda_1>@?1??GetProcessString@WMIConnection@@AEAA?AV?$basic_string@_WU?$char_traits@_W@std@@V?$allocator@_W@2@@std@@KPEB_W@Z@XAEBUtagVARIANT@@@std@@EEBAAEBVtype_info@@XZ 0000000180028650 f   wmi.obj
 0001:00027660       ?_Do_call@?$_Func_impl_no_alloc@V<lambda_1>@?1??GetProcessString@WMIConnection@@AEAA?AV?$basic_string@_WU?$char_traits@_W@std@@V?$allocator@_W@2@@std@@KPEB_W@Z@XAEBUtagVARIANT@@@std@@EEAAXAEBUtagVARIANT@@@Z 0000000180028660 f   wmi.obj
 0001:00027698       ?_Copy@?$_Func_impl_no_alloc@V<lambda_1>@?1??GetProcessString@WMIConnection@@AEAA?AV?$basic_string@_WU?$char_traits@_W@std@@V?$allocator@_W@2@@std@@KPEB_W@Z@XAEBUtagVARIANT@@@std@@EEBAPEAV?$_Func_base@XAEBUtagVARIANT@@@2@PEAX@Z 0000000180028698 f   wmi.obj
 0001:00027698       ?_Move@?$_Func_impl_no_alloc@V<lambda_1>@?1??GetProcessString@WMIConnection@@AEAA?AV?$basic_string@_WU?$char_traits@_W@std@@V?$allocator@_W@2@@std@@KPEB_W@Z@XAEBUtagVARIANT@@@std@@EEAAPEAV?$_Func_base@XAEBUtagVARIANT@@@2@PEAX@Z 0000000180028698 f   wmi.obj
 0001:000276b8       ?_Target_type@?$_Func_impl_no_alloc@V<lambda_1>@?1??GetProcessInt@WMIConnection@@AEAAKKPEB_W@Z@XAEBUtagVARIANT@@@std@@EEBAAEBVtype_info@@XZ 00000001800286b8 f   wmi.obj
 0001:000276c8       ?_Do_call@?$_Func_impl_no_alloc@V<lambda_1>@?1??GetProcessInt@WMIConnection@@AEAAKKPEB_W@Z@XAEBUtagVARIANT@@@std@@EEAAXAEBUtagVARIANT@@@Z 00000001800286c8 f   wmi.obj
 0001:000276e8       ?_Copy@?$_Func_impl_no_alloc@V<lambda_1>@?1??GetProcessInt@WMIConnection@@AEAAKKPEB_W@Z@XAEBUtagVARIANT@@@std@@EEBAPEAV?$_Func_base@XAEBUtagVARIANT@@@2@PEAX@Z 00000001800286e8 f   wmi.obj
 0001:000276e8       ?_Move@?$_Func_impl_no_alloc@V<lambda_1>@?1??GetProcessInt@WMIConnection@@AEAAKKPEB_W@Z@XAEBUtagVARIANT@@@std@@EEAAPEAV?$_Func_base@XAEBUtagVARIANT@@@2@PEAX@Z 00000001800286e8 f   wmi.obj
 0001:00027708       ?fNtQueryInformationFile@@YAJPEAX00KK@Z 0000000180028708 f   Proclist.obj
 0001:00027708       ?fNtQueryInformationProcess@@YAJPEAXW4_PROCESSINFOCLASS@@0KPEAK@Z 0000000180028708 f   Proclist.obj
 0001:00027708       ?fNtQueryInformationThread@@YAJPEAXK0KPEAK@Z 0000000180028708 f   Proclist.obj
 0001:00027708       ?fNtQueryObject@@YAJPEAXK0K0@Z 0000000180028708 f   Proclist.obj
 0001:00027708       ?fNtQuerySystemInformation@@YAJKPEAXKPEAK@Z 0000000180028708 f   Proclist.obj
 0001:00027710       $LN4                       0000000180028710     Proclist.obj
 0001:00027710       $LN4                       0000000180028710     Proclist.obj
 0001:00027710       $LN4                       0000000180028710     Proclist.obj
 0001:00027710       $LN4                       0000000180028710     Proclist.obj
 0001:00027710       $LN4                       0000000180028710     Proclist.obj
 0001:00027718       ?fEnumProcessModulesEx@@YAHPEAXPEAPEAUHINSTANCE__@@KPEAKK@Z 0000000180028718 f   Proclist.obj
 0001:00027718       ?fGetGuiResources@@YAKPEAXK@Z 0000000180028718 f   Proclist.obj
 0001:00027718       ?fIsWow64Process@@YAHPEAXPEAH@Z 0000000180028718 f   Proclist.obj
 0001:00027718       no_op_initialize           0000000180028718 f   libucrt:wsetlocale.obj
 0001:00027720       ?fCoSetProxyBlanket@@YAJPEAUIUnknown@@KKPEA_WKKPEAXK@Z 0000000180028720 f   Proclist.obj
 0001:00027728       $LN4                       0000000180028728     Proclist.obj
 0001:00027730       ?dynamic_bind@@YAXXZ       0000000180028730 f   Proclist.obj
 0001:00028e28       tidy_global                0000000180029e28 f   libcpmt:locale0.obj
 0001:000296d0       ?dllmain_crt_dispatch@@YAHQEAUHINSTANCE__@@KQEAX@Z 000000018002a6d0 f   LIBCMT:dll_dllmain.obj
 0001:00029730       ?dllmain_crt_process_attach@@YAHQEAUHINSTANCE__@@QEAX@Z 000000018002a730 f   LIBCMT:dll_dllmain.obj
 0001:00029860       ?dllmain_crt_process_detach@@YAH_N@Z 000000018002a860 f   LIBCMT:dll_dllmain.obj
 0001:00029900       ?dllmain_dispatch@@YAHQEAUHINSTANCE__@@KQEAX@Z 000000018002a900 f   LIBCMT:dll_dllmain.obj
 0001:00029a38       ?dllmain_raw@@YAHQEAUHINSTANCE__@@KQEAX@Z 000000018002aa38 f   LIBCMT:dll_dllmain.obj
 0001:00029c18       initialize_environment     000000018002ac18 f   libucrt:initialization.obj
 0001:00029c18       initialize_global_state_isolation 000000018002ac18 f   libucrt:initialization.obj
 0001:00029c18       report_memory_leaks        000000018002ac18 f   libucrt:initialization.obj
 0001:00029c18       uninitialize_c             000000018002ac18 f   libucrt:initialization.obj
 0001:00029c18       uninitialize_global_state_isolation 000000018002ac18 f   libucrt:initialization.obj
 0001:00029d40       $LN9                       000000018002ad40     LIBCMT:gs_support.obj
 0001:00029d48       $LN10                      000000018002ad48     LIBCMT:gs_support.obj
 0001:0002a340       $LN6                       000000018002b340     libvcruntime:risctrnsctrl.obj
 0001:0002a5a8       $LN28                      000000018002b5a8     libvcruntime:ehhelpers.obj
 0001:0002a5ac       $LN29                      000000018002b5ac     libvcruntime:ehhelpers.obj
 0001:0002a6b0       $LN13                      000000018002b6b0     libvcruntime:ehhelpers.obj
 0001:0002a6b4       $LN14                      000000018002b6b4     libvcruntime:ehhelpers.obj
 0001:0002a6b8       $LN15                      000000018002b6b8     libvcruntime:ehhelpers.obj
 0001:0002aab0       $LN6                       000000018002bab0     libvcruntime:throw.obj
 0001:0002aab8       $LN7                       000000018002bab8     libvcruntime:throw.obj
 0001:0002aac0       $LN8                       000000018002bac0     libvcruntime:throw.obj
 0001:0002ae28       $LN54                      000000018002be28     libvcruntime:riscchandler.obj
 0001:0002b258       ??$BuildCatchObjectHelperInternal@V__FrameHandler3@@@@YAHPEAUEHExceptionRecord@@PEAXPEBU_s_HandlerType@@PEBU_s_CatchableType@@@Z 000000018002c258 f   libvcruntime:frame.obj
 0001:0002b440       ??$BuildCatchObjectInternal@V__FrameHandler3@@@@YAXPEAUEHExceptionRecord@@PEAXPEBU_s_HandlerType@@PEBU_s_CatchableType@@@Z 000000018002c440 f   libvcruntime:frame.obj
 0001:0002b520       ??$CatchIt@V__FrameHandler3@@@@YAXPEAUEHExceptionRecord@@PEA_KPEAU_CONTEXT@@PEAU_xDISPATCHER_CONTEXT@@PEBU_s_FuncInfo@@PEBU_s_HandlerType@@PEBU_s_CatchableType@@PEBU_s_TryBlockMapEntry@@H1EE@Z 000000018002c520 f   libvcruntime:frame.obj
 0001:0002b5f0       ??$FindHandler@V__FrameHandler3@@@@YAXPEAUEHExceptionRecord@@PEA_KPEAU_CONTEXT@@PEAU_xDISPATCHER_CONTEXT@@PEBU_s_FuncInfo@@EH1@Z 000000018002c5f0 f   libvcruntime:frame.obj
 0001:0002bb20       $LN128                     000000018002cb20     libvcruntime:frame.obj
 0001:0002bb24       $LN129                     000000018002cb24     libvcruntime:frame.obj
 0001:0002bb28       $LN130                     000000018002cb28     libvcruntime:frame.obj
 0001:0002bb30       ??$FindHandlerForForeignException@V__FrameHandler3@@@@YAXPEAUEHExceptionRecord@@PEA_KPEAU_CONTEXT@@PEAU_xDISPATCHER_CONTEXT@@PEBU_s_FuncInfo@@HH1@Z 000000018002cb30 f   libvcruntime:frame.obj
 0001:0002bd80       $LN54                      000000018002cd80     libvcruntime:frame.obj
 0001:0002bd84       $LN55                      000000018002cd84     libvcruntime:frame.obj
 0001:0002c110       $LN51                      000000018002d110     libvcruntime:frame.obj
 0001:0002c118       $LN47                      000000018002d118     libvcruntime:frame.obj
 0001:0002c11c       $LN48                      000000018002d11c     libvcruntime:frame.obj
 0001:0002c120       $LN49                      000000018002d120     libvcruntime:frame.obj
 0001:0002c124       $LN50                      000000018002d124     libvcruntime:frame.obj
 0001:0002c128       $LN52                      000000018002d128     libvcruntime:frame.obj
 0001:0002c3a8       $LN29                      000000018002d3a8     libvcruntime:frame.obj
 0001:0002c3ac       $LN30                      000000018002d3ac     libvcruntime:frame.obj
 0001:0002c3b0       ?ExFilterRethrow@@YAHPEAU_EXCEPTION_POINTERS@@PEAUEHExceptionRecord@@PEAH@Z 000000018002d3b0 f   libvcruntime:frame.obj
 0001:0002c468       $LN12                      000000018002d468     libvcruntime:frame.obj
 0001:0002c46c       $LN13                      000000018002d46c     libvcruntime:frame.obj
 0001:0002c6f8       ?IsInExceptionSpec@@YAEPEAUEHExceptionRecord@@PEBU_s_ESTypeList@@@Z 000000018002d6f8 f   libvcruntime:frame.obj
 0001:0002cee8       ??$common_vsprintf@Vformat_validation_base@__crt_stdio_output@@D@@YAH_KQEAD0QEBDQEAU__crt_locale_pointers@@1@Z 000000018002dee8 f   libucrt:output.obj
 0001:0002d80c       $LN116                     000000018002e80c     libucrt:output.obj
 0001:0002d80d       $LN117                     000000018002e80d     libucrt:output.obj
 0001:0002d80e       $LN118                     000000018002e80e     libucrt:output.obj
 0001:0002d80f       $LN119                     000000018002e80f     libucrt:output.obj
 0001:0002d810       $LN120                     000000018002e810     libucrt:output.obj
 0001:0002d811       $LN121                     000000018002e811     libucrt:output.obj
 0001:0002d812       $LN122                     000000018002e812     libucrt:output.obj
 0001:0002d813       $LN123                     000000018002e813     libucrt:output.obj
 0001:0002dd34       $LN92                      000000018002ed34     libucrt:output.obj
 0001:0002dd38       $LN93                      000000018002ed38     libucrt:output.obj
 0001:0002dd3c       $LN94                      000000018002ed3c     libucrt:output.obj
 0001:0002dd40       $LN95                      000000018002ed40     libucrt:output.obj
 0001:0002dd44       $LN96                      000000018002ed44     libucrt:output.obj
 0001:0002dd48       $LN97                      000000018002ed48     libucrt:output.obj
 0001:0002dd4c       $LN98                      000000018002ed4c     libucrt:output.obj
 0001:0002dd50       $LN99                      000000018002ed50     libucrt:output.obj
 0001:0002dd54       $LN100                     000000018002ed54     libucrt:output.obj
 0001:0002dd58       $LN101                     000000018002ed58     libucrt:output.obj
 0001:0002dd5c       $LN102                     000000018002ed5c     libucrt:output.obj
 0001:0002dd60       $LN103                     000000018002ed60     libucrt:output.obj
 0001:0002dd64       $LN104                     000000018002ed64     libucrt:output.obj
 0001:0002dd68       $LN105                     000000018002ed68     libucrt:output.obj
 0001:0002dd6c       $LN106                     000000018002ed6c     libucrt:output.obj
 0001:0002dd70       $LN107                     000000018002ed70     libucrt:output.obj
 0001:0002dd74       $LN108                     000000018002ed74     libucrt:output.obj
 0001:0002dd78       $LN109                     000000018002ed78     libucrt:output.obj
 0001:0002dd7c       $LN110                     000000018002ed7c     libucrt:output.obj
 0001:0002dd80       $LN111                     000000018002ed80     libucrt:output.obj
 0001:0002dd84       $LN112                     000000018002ed84     libucrt:output.obj
 0001:0002dd88       $LN113                     000000018002ed88     libucrt:output.obj
 0001:0002dd8c       $LN114                     000000018002ed8c     libucrt:output.obj
 0001:0002dd90       $LN115                     000000018002ed90     libucrt:output.obj
 0001:0002dd94       $LN116                     000000018002ed94     libucrt:output.obj
 0001:0002dd98       $LN117                     000000018002ed98     libucrt:output.obj
 0001:0002dd9c       $LN118                     000000018002ed9c     libucrt:output.obj
 0001:0002dda0       $LN119                     000000018002eda0     libucrt:output.obj
 0001:0002dda4       $LN120                     000000018002eda4     libucrt:output.obj
 0001:0002dda8       $LN121                     000000018002eda8     libucrt:output.obj
 0001:0002ddac       $LN122                     000000018002edac     libucrt:output.obj
 0001:0002ddb0       $LN123                     000000018002edb0     libucrt:output.obj
 0001:0002ddb4       $LN124                     000000018002edb4     libucrt:output.obj
 0001:0002ddb8       $LN125                     000000018002edb8     libucrt:output.obj
 0001:0002ddbc       $LN126                     000000018002edbc     libucrt:output.obj
 0001:0002ddc0       $LN127                     000000018002edc0     libucrt:output.obj
 0001:0002ddc4       $LN128                     000000018002edc4     libucrt:output.obj
 0001:0002ddc8       $LN129                     000000018002edc8     libucrt:output.obj
 0001:0002ddcc       $LN130                     000000018002edcc     libucrt:output.obj
 0001:0002ddd0       $LN131                     000000018002edd0     libucrt:output.obj
 0001:0002ddd4       $LN132                     000000018002edd4     libucrt:output.obj
 0001:0002ddd8       $LN133                     000000018002edd8     libucrt:output.obj
 0001:0002dddc       $LN134                     000000018002eddc     libucrt:output.obj
 0001:0002dde0       $LN135                     000000018002ede0     libucrt:output.obj
 0001:0002dde4       $LN136                     000000018002ede4     libucrt:output.obj
 0001:0002dde8       $LN137                     000000018002ede8     libucrt:output.obj
 0001:0002ddec       $LN138                     000000018002edec     libucrt:output.obj
 0001:0002ddf0       $LN139                     000000018002edf0     libucrt:output.obj
 0001:0002ddf4       $LN140                     000000018002edf4     libucrt:output.obj
 0001:0002ddf8       $LN141                     000000018002edf8     libucrt:output.obj
 0001:0002ddfc       $LN142                     000000018002edfc     libucrt:output.obj
 0001:0002de00       $LN143                     000000018002ee00     libucrt:output.obj
 0001:0002de04       $LN144                     000000018002ee04     libucrt:output.obj
 0001:0002de08       $LN145                     000000018002ee08     libucrt:output.obj
 0001:0002de0c       $LN146                     000000018002ee0c     libucrt:output.obj
 0001:0002de10       $LN147                     000000018002ee10     libucrt:output.obj
 0001:0002e3dc       $LN132                     000000018002f3dc     libucrt:output.obj
 0001:0002e3dd       $LN133                     000000018002f3dd     libucrt:output.obj
 0001:0002e3de       $LN134                     000000018002f3de     libucrt:output.obj
 0001:0002e3df       $LN135                     000000018002f3df     libucrt:output.obj
 0001:0002e3e0       $LN136                     000000018002f3e0     libucrt:output.obj
 0001:0002e3e1       $LN137                     000000018002f3e1     libucrt:output.obj
 0001:0002e3e2       $LN138                     000000018002f3e2     libucrt:output.obj
 0001:0002e3e3       $LN139                     000000018002f3e3     libucrt:output.obj
 0001:0002e3e4       $LN140                     000000018002f3e4     libucrt:output.obj
 0001:0002e3e5       $LN141                     000000018002f3e5     libucrt:output.obj
 0001:0002e3e6       $LN142                     000000018002f3e6     libucrt:output.obj
 0001:0002e3e7       $LN143                     000000018002f3e7     libucrt:output.obj
 0001:0002e494       $LN49                      000000018002f494     libucrt:output.obj
 0001:0002e495       $LN50                      000000018002f495     libucrt:output.obj
 0001:0002e496       $LN51                      000000018002f496     libucrt:output.obj
 0001:0002e497       $LN52                      000000018002f497     libucrt:output.obj
 0001:0002e498       $LN53                      000000018002f498     libucrt:output.obj
 0001:0002e499       $LN54                      000000018002f499     libucrt:output.obj
 0001:0002e49a       $LN55                      000000018002f49a     libucrt:output.obj
 0001:0002e49b       $LN56                      000000018002f49b     libucrt:output.obj
 0001:0002e49c       $LN57                      000000018002f49c     libucrt:output.obj
 0001:0002e49d       $LN58                      000000018002f49d     libucrt:output.obj
 0001:0002e49e       $LN59                      000000018002f49e     libucrt:output.obj
 0001:0002e49f       $LN60                      000000018002f49f     libucrt:output.obj
 0001:0002f230       ??$?RV<lambda_41e84717acc955b55e9d0d529e507b68>@@AEAV<lambda_b37934c380d97b75fd242ea49540127a>@@V<lambda_bb6db9f9ac473960206e0d4b942b5506>@@@?$__crt_seh_guarded_call@PEAD@@QEAAPEAD$$QEAV<lambda_41e84717acc955b55e9d0d529e507b68>@@AEAV<lambda_b37934c380d97b75fd242ea49540127a>@@$$QEAV<lambda_bb6db9f9ac473960206e0d4b942b5506>@@@Z 0000000180030230 f   libucrt:setlocale.obj
 0001:0002f278       ??R<lambda_b37934c380d97b75fd242ea49540127a>@@QEBAPEADXZ 0000000180030278 f   libucrt:setlocale.obj
 0001:00030c38       ??$?RV<lambda_d80eeec6fff315bfe5c115232f3240e3>@@AEAV<lambda_6e4b09c48022b2350581041d5f6b0c4c>@@V<lambda_2358e3775559c9db80273638284d5e45>@@@?$__crt_seh_guarded_call@X@@QEAAX$$QEAV<lambda_d80eeec6fff315bfe5c115232f3240e3>@@AEAV<lambda_6e4b09c48022b2350581041d5f6b0c4c>@@$$QEAV<lambda_2358e3775559c9db80273638284d5e45>@@@Z 0000000180031c38 f   libucrt:exit.obj
 0001:00030c78       ??R<lambda_6e4b09c48022b2350581041d5f6b0c4c>@@QEBA@XZ 0000000180031c78 f   libucrt:exit.obj
 0001:00030d88       ?atexit_exception_filter@@YAHK@Z 0000000180031d88 f   libucrt:exit.obj
 0001:00030da0       ?common_exit@@YAXHW4_crt_exit_cleanup_mode@@W4_crt_exit_return_mode@@@Z 0000000180031da0 f   libucrt:exit.obj
 0001:00030e78       ?exit_or_terminate_process@@YAXI@Z 0000000180031e78 f   libucrt:exit.obj
 0001:00030ee8       ?try_cor_exit_process@@YAXI@Z 0000000180031ee8 f   libucrt:exit.obj
 0001:00030fc0       ??$parse_command_line@D@@YAXPEADPEAPEAD0PEA_K2@Z 0000000180031fc0 f   libucrt:argv_parsing.obj
 0001:00031418       ??$common_initialize_environment_nolock@D@@YAHXZ 0000000180032418 f   libucrt:environment_initialization.obj
 0001:00031498       ??$create_environment@D@@YAQEAPEADQEAD@Z 0000000180032498 f   libucrt:environment_initialization.obj
 0001:000315c0       ??$uninitialize_environment_internal@D@@YAXAEAPEAPEAD@Z 00000001800325c0 f   libucrt:environment_initialization.obj
 0001:00031618       ??$uninitialize_environment_internal@_W@@YAXAEAPEAPEA_W@Z 0000000180032618 f   libucrt:environment_initialization.obj
 0001:00031708       ??$?RV<lambda_638799b9deba96c50f710eeac98168cd>@@AEAV<lambda_22ebabd17bc4fa466a2aca6d8deb888d>@@V<lambda_a6f7d7db0129f75315ebf26d50c089f1>@@@?$__crt_seh_guarded_call@H@@QEAAH$$QEAV<lambda_638799b9deba96c50f710eeac98168cd>@@AEAV<lambda_22ebabd17bc4fa466a2aca6d8deb888d>@@$$QEAV<lambda_a6f7d7db0129f75315ebf26d50c089f1>@@@Z 0000000180032708 f   libucrt:onexit.obj
 0001:00031750       ??$?RV<lambda_7777bce6b2f8c936911f934f8298dc43>@@AEAV<lambda_f03950bc5685219e0bcd2087efbe011e>@@V<lambda_3883c3dff614d5e0c5f61bb1ac94921c>@@@?$__crt_seh_guarded_call@H@@QEAAH$$QEAV<lambda_7777bce6b2f8c936911f934f8298dc43>@@AEAV<lambda_f03950bc5685219e0bcd2087efbe011e>@@$$QEAV<lambda_3883c3dff614d5e0c5f61bb1ac94921c>@@@Z 0000000180032750 f   libucrt:onexit.obj
 0001:00031798       ??R<lambda_22ebabd17bc4fa466a2aca6d8deb888d>@@QEBAHXZ 0000000180032798 f   libucrt:onexit.obj
 0001:00031958       ??R<lambda_f03950bc5685219e0bcd2087efbe011e>@@QEBAHXZ 0000000180032958 f   libucrt:onexit.obj
 0001:00031b68       initialize_global_variables 0000000180032b68 f   libucrt:initialization.obj
 0001:00031b80       initialize_c               0000000180032b80 f   libucrt:initialization.obj
 0001:00031bb0       uninitialize_environment   0000000180032bb0 f   libucrt:initialization.obj
 0001:00031bc8       initialize_pointers        0000000180032bc8 f   libucrt:initialization.obj
 0001:00031c18       uninitialize_vcruntime     0000000180032c18 f   libucrt:initialization.obj
 0001:00031c38       uninitialize_allocated_memory 0000000180032c38 f   libucrt:initialization.obj
 0001:00031c98       uninitialize_allocated_io_buffers 0000000180032c98 f   libucrt:initialization.obj
 0001:00032b50       ?initialize_inherited_file_handles_nolock@@YAXXZ 0000000180033b50 f   libucrt:ioinit.obj
 0001:00032c50       ?initialize_stdio_handles_nolock@@YAXXZ 0000000180033c50 f   libucrt:ioinit.obj
 0001:00032f48       ?<lambda_invoker_cdecl>@<lambda_795c6bd18aed400428efeb9a5f0e1479>@@CAHPEA_W@Z 0000000180033f48 f   libucrt:winapi_thunks.obj
 0001:00032fa0       ??$?RV<lambda_48fc4a32460bb0512d3b13f8499328be>@@AEAV<lambda_6c3dac0a4f3f9cefca9bb494422f9b77>@@V<lambda_0a2f2c9f9a56eb2b08bfa6ff61d331c5>@@@?$__crt_seh_guarded_call@H@@QEAAH$$QEAV<lambda_48fc4a32460bb0512d3b13f8499328be>@@AEAV<lambda_6c3dac0a4f3f9cefca9bb494422f9b77>@@$$QEAV<lambda_0a2f2c9f9a56eb2b08bfa6ff61d331c5>@@@Z 0000000180033fa0 f   libucrt:winapi_thunks.obj
 0001:00033038       ?try_get_function@@YAPEAXW4function_id@?A0x391cf84c@@QEBDQEBW4module_id@2@2@Z 0000000180034038 f   libucrt:winapi_thunks.obj
 0001:00033d00       ??$?RV<lambda_842d9ff0dc9ef11c61343bbaebe7f885>@@AEAV<lambda_c5860995281e5c4ce005b3de8f5874ee>@@V<lambda_d90129c13df834fdcbf8d2b88dafcf2d>@@@?$__crt_seh_guarded_call@X@@QEAAX$$QEAV<lambda_842d9ff0dc9ef11c61343bbaebe7f885>@@AEAV<lambda_c5860995281e5c4ce005b3de8f5874ee>@@$$QEAV<lambda_d90129c13df834fdcbf8d2b88dafcf2d>@@@Z 0000000180034d00 f   libucrt:fflush.obj
 0001:00033dc8       ??$?RV<lambda_886d6c58226a84441f68b9f2b8217b83>@@AEAV<lambda_ab61a845afdef5b7c387490eaf3616ee>@@V<lambda_f7f22ab5edc0698d5f6905b0d3f44752>@@@?$__crt_seh_guarded_call@X@@QEAAX$$QEAV<lambda_886d6c58226a84441f68b9f2b8217b83>@@AEAV<lambda_ab61a845afdef5b7c387490eaf3616ee>@@$$QEAV<lambda_f7f22ab5edc0698d5f6905b0d3f44752>@@@Z 0000000180034dc8 f   libucrt:fflush.obj
 0001:00033eb8       ?common_flush_all@@YAH_N@Z 0000000180034eb8 f   libucrt:fflush.obj
 0001:000346f0       ??$?RV<lambda_0ae27a3a962d80f24befdcbee591983d>@@AEAV<lambda_8d0ee55de4b1038c4002e0adecdf1839>@@V<lambda_dc504788e8f1664fe9b84e20bfb512f2>@@@?$__crt_seh_guarded_call@X@@QEAAX$$QEAV<lambda_0ae27a3a962d80f24befdcbee591983d>@@AEAV<lambda_8d0ee55de4b1038c4002e0adecdf1839>@@$$QEAV<lambda_dc504788e8f1664fe9b84e20bfb512f2>@@@Z 00000001800356f0 f   libucrt:per_thread_data.obj
 0001:00034748       ??$?RV<lambda_2d41944a1d46af3157314b8a01080d33>@@AEAV<lambda_8f455de75cd7d7f24b4096f044d8b9e6>@@V<lambda_aa500f224e6afead328df44964fe2772>@@@?$__crt_seh_guarded_call@X@@QEAAX$$QEAV<lambda_2d41944a1d46af3157314b8a01080d33>@@AEAV<lambda_8f455de75cd7d7f24b4096f044d8b9e6>@@$$QEAV<lambda_aa500f224e6afead328df44964fe2772>@@@Z 0000000180035748 f   libucrt:per_thread_data.obj
 0001:000347c8       ??$?RV<lambda_aa87e3671a710a21b5dc78c0bdf72e11>@@AEAV<lambda_92619d2358a28f41a33ba319515a20b9>@@V<lambda_6992ecaafeb10aed2b74cb1fae11a551>@@@?$__crt_seh_guarded_call@X@@QEAAX$$QEAV<lambda_aa87e3671a710a21b5dc78c0bdf72e11>@@AEAV<lambda_92619d2358a28f41a33ba319515a20b9>@@$$QEAV<lambda_6992ecaafeb10aed2b74cb1fae11a551>@@@Z 00000001800357c8 f   libucrt:per_thread_data.obj
 0001:00034818       ??$?RV<lambda_f2e299630e499de9f9a165e60fcd3db5>@@AEAV<lambda_2ae9d31cdba2644fcbeaf08da7c24588>@@V<lambda_40d01ff24d0e7b3814fdbdcee8eab3c7>@@@?$__crt_seh_guarded_call@X@@QEAAX$$QEAV<lambda_f2e299630e499de9f9a165e60fcd3db5>@@AEAV<lambda_2ae9d31cdba2644fcbeaf08da7c24588>@@$$QEAV<lambda_40d01ff24d0e7b3814fdbdcee8eab3c7>@@@Z 0000000180035818 f   libucrt:per_thread_data.obj
 0001:00034888       ?construct_ptd_array@@YAXQEAU__acrt_ptd@@@Z 0000000180035888 f   libucrt:per_thread_data.obj
 0001:00034950       ?destroy_fls@@YAXPEAX@Z    0000000180035950 f   libucrt:per_thread_data.obj
 0001:00034980       ?destroy_ptd_array@@YAXQEAU__acrt_ptd@@@Z 0000000180035980 f   libucrt:per_thread_data.obj
 0001:00034a70       ?replace_current_thread_locale_nolock@@YAXQEAU__acrt_ptd@@QEAU__crt_locale_data@@@Z 0000000180035a70 f   libucrt:per_thread_data.obj
 0001:00034ee8       ?fp_format_a@@YAHQEBNPEAD_KQEAD2H_NIQEAU__crt_locale_pointers@@@Z 0000000180035ee8 f   libucrt:cvt.obj
 0001:00035250       ?fp_format_e@@YAHQEBNQEAD_K12H_NIQEAU__crt_locale_pointers@@@Z 0000000180036250 f   libucrt:cvt.obj
 0001:00035320       ?fp_format_e_internal@@YAHQEAD_KH_NIQEAU_strflt@@2QEAU__crt_locale_pointers@@@Z 0000000180036320 f   libucrt:cvt.obj
 0001:00035558       ?fp_format_f_internal@@YAHQEAD_KHQEAU_strflt@@_NQEAU__crt_locale_pointers@@@Z 0000000180036558 f   libucrt:cvt.obj
 0001:000356e0       ?fp_format_g@@YAHQEBNQEAD_K12H_NIQEAU__crt_locale_pointers@@@Z 00000001800366e0 f   libucrt:cvt.obj
 0001:000357f8       ?fp_format_nan_or_infinity@@YAHW4__acrt_fp_class@@_NPEAD_K1@Z 00000001800367f8 f   libucrt:cvt.obj
 0001:00035ae8       ??$?RV<lambda_1d892b297fdedeee07ed8124eeb2f2fa>@@AEAV<lambda_ffc046909424fd52df0ac47e64813305>@@V<lambda_01a7098693036236037e7cdb9bca3d73>@@@?$__crt_seh_guarded_call@X@@QEAAX$$QEAV<lambda_1d892b297fdedeee07ed8124eeb2f2fa>@@AEAV<lambda_ffc046909424fd52df0ac47e64813305>@@$$QEAV<lambda_01a7098693036236037e7cdb9bca3d73>@@@Z 0000000180036ae8 f   libucrt:wsetlocale.obj
 0001:00035c50       ??$?RV<lambda_410d79af7f07d98d83a3f525b3859a53>@@AEAV<lambda_3e16ef9562a7dcce91392c22ab16ea36>@@V<lambda_38119f0e861e05405d8a144b9b982f0a>@@@?$__crt_seh_guarded_call@X@@QEAAX$$QEAV<lambda_410d79af7f07d98d83a3f525b3859a53>@@AEAV<lambda_3e16ef9562a7dcce91392c22ab16ea36>@@$$QEAV<lambda_38119f0e861e05405d8a144b9b982f0a>@@@Z 0000000180036c50 f   libucrt:wsetlocale.obj
 0001:00035cd0       ??$?RV<lambda_7f2adfce497ff2baa965cd4f576ecfd1>@@AEAV<lambda_2a444430fde8c29194d880d93eed5e8f>@@AEAV<lambda_8dff2cf36a5417162780cd64fa2883ef>@@@?$__crt_seh_guarded_call@X@@QEAAX$$QEAV<lambda_7f2adfce497ff2baa965cd4f576ecfd1>@@AEAV<lambda_2a444430fde8c29194d880d93eed5e8f>@@AEAV<lambda_8dff2cf36a5417162780cd64fa2883ef>@@@Z 0000000180036cd0 f   libucrt:wsetlocale.obj
 0001:00035d10       ??R<lambda_2a444430fde8c29194d880d93eed5e8f>@@QEBA@XZ 0000000180036d10 f   libucrt:wsetlocale.obj
 0001:00036050       _expandlocale              0000000180037050 f   libucrt:wsetlocale.obj
 0001:00036588       _wsetlocale_get_all        0000000180037588 f   libucrt:wsetlocale.obj
 0001:00036770       _wsetlocale_nolock         0000000180037770 f   libucrt:wsetlocale.obj
 0001:000369e0       _wsetlocale_set_cat        00000001800379e0 f   libucrt:wsetlocale.obj
 0001:00036d08       parse_bcp47                0000000180037d08 f   libucrt:wsetlocale.obj
 0001:00036f38       parse_bcp47_code_page      0000000180037f38 f   libucrt:wsetlocale.obj
 0001:00036f90       parse_bcp47_language       0000000180037f90 f   libucrt:wsetlocale.obj
 0001:00037028       parse_bcp47_region         0000000180038028 f   libucrt:wsetlocale.obj
 0001:00037128       parse_bcp47_script         0000000180038128 f   libucrt:wsetlocale.obj
 0001:000371c8       string_is_alpha            00000001800381c8 f   libucrt:wsetlocale.obj
 0001:00037238       ?write_double_translated_ansi_nolock@@YA?AUwrite_result@?A0x17268360@@HQEBDI@Z 0000000180038238 f   libucrt:write.obj
 0001:00037718       ?write_text_ansi_nolock@@YA?AUwrite_result@?A0x17268360@@HQEBDI@Z 0000000180038718 f   libucrt:write.obj
 0001:00037868       ?write_text_utf16le_nolock@@YA?AUwrite_result@?A0x17268360@@HQEBDI@Z 0000000180038868 f   libucrt:write.obj
 0001:000379c0       ?write_text_utf8_nolock@@YA?AUwrite_result@?A0x17268360@@HQEBDI@Z 00000001800389c0 f   libucrt:write.obj
 0001:00037f98       _exception_enabled         0000000180038f98 f   libucrt:libm_error.obj
 0001:000382a8       ?_mbstowcs_l_helper@@YA_KPEA_WPEBD_KPEAU__crt_locale_pointers@@@Z 00000001800392a8 f   libucrt:mbstowcs.obj
 0001:000385f8       ?_wcstombs_l_helper@@YA_KPEADPEB_W_KPEAU__crt_locale_pointers@@@Z 00000001800395f8 f   libucrt:wcstombs.obj
 0001:00038a18       ?InternalGetLocaleInfoA@@YAHQEAU__crt_locale_pointers@@QEB_WKQEADH@Z 0000000180039a18 f   libucrt:getlocaleinfoa.obj
 0001:00038f40       ?__acrt_LCMapStringA_stat@@YAHPEAU__crt_locale_pointers@@PEB_WKPEBDHPEADHHH@Z 0000000180039f40 f   libucrt:lcmapstringa.obj
 0001:0003a4b0       ??$?RV<lambda_450d765d439847d4c735a33c368b5fc0>@@AEAV<lambda_44731a7d0e6d81c3e6aa82d741081786>@@V<lambda_601a2a7da3b7a96e9554ac7215c4b07c>@@@?$__crt_seh_guarded_call@P6AXH@Z@@QEAAP6AXH@Z$$QEAV<lambda_450d765d439847d4c735a33c368b5fc0>@@AEAV<lambda_44731a7d0e6d81c3e6aa82d741081786>@@$$QEAV<lambda_601a2a7da3b7a96e9554ac7215c4b07c>@@@Z 000000018003b4b0 f   libucrt:signal.obj
 0001:0003a500       ?get_global_action_nolock@@YAPEAP6AXH@ZH@Z 000000018003b500 f   libucrt:signal.obj
 0001:0003ac00       ?<lambda_invoker_cdecl>@<lambda_a1ce4c8ae42411fd470c77163914f50e>@@CAHPEBX0@Z 000000018003bc00 f   libucrt:argv_wildcards.obj
 0001:0003adc0       ??$common_expand_argv_wildcards@D@@YAHQEAPEADQEAPEAPEAD@Z 000000018003bdc0 f   libucrt:argv_wildcards.obj
 0001:0003aff8       ??$copy_and_add_argument_to_buffer@D@@YAHQEBD0_KAEAV?$argument_list@D@?A0x5f5c8891@@@Z 000000018003bff8 f   libucrt:argv_wildcards.obj
 0001:0003b188       ??$expand_argument_wildcards@D@@YAHQEAD0AEAV?$argument_list@D@?A0x5f5c8891@@@Z 000000018003c188 f   libucrt:argv_wildcards.obj
 0001:0003b600       ??$?RV<lambda_efdfa57d1f175319df784efa44bb7b81>@@AEAV<lambda_5f0a4c1567f8adc6734073e5d1e1b35c>@@V<lambda_2e8a7d3640ea6ccb4c2413664c2db6fd>@@@?$__crt_seh_guarded_call@X@@QEAAX$$QEAV<lambda_efdfa57d1f175319df784efa44bb7b81>@@AEAV<lambda_5f0a4c1567f8adc6734073e5d1e1b35c>@@$$QEAV<lambda_2e8a7d3640ea6ccb4c2413664c2db6fd>@@@Z 000000018003c600 f   libucrt:mbctype.obj
 0001:0003b758       ?CPtoLocaleName@@YAPEB_WH@Z 000000018003c758 f   libucrt:mbctype.obj
 0001:0003b7a8       ?getSystemCP@@YAHH@Z       000000018003c7a8 f   libucrt:mbctype.obj
 0001:0003b850       ?setSBCS@@YAXPEAU__crt_multibyte_data@@@Z 000000018003c850 f   libucrt:mbctype.obj
 0001:0003b8d8       ?setSBUpLow@@YAXPEAU__crt_multibyte_data@@@Z 000000018003c8d8 f   libucrt:mbctype.obj
 0001:0003bae8       ?setmbcp_internal@@YAHH_NQEAU__acrt_ptd@@QEAPEAU__crt_multibyte_data@@@Z 000000018003cae8 f   libucrt:mbctype.obj
 0001:0003bc58       ?update_thread_multibyte_data_internal@@YAPEAU__crt_multibyte_data@@QEAU__acrt_ptd@@QEAPEAU1@@Z 000000018003cc58 f   libucrt:mbctype.obj
 0001:0003c040       ?x_ismbbtype_l@@YAHPEAU__crt_locale_pointers@@IHH@Z 000000018003d040 f   libucrt:ismbbyte.obj
 0001:0003c4f8       ??$common_lseek_nolock@_J@@YA_JH_JH@Z 000000018003d4f8 f   libucrt:lseek.obj
 0001:0003c978       ??$?RV<lambda_a37b2b86f63e897a80ea819b0eb08c01>@@AEAV<lambda_38ce7e780aa69e748d6df282ebc68efe>@@V<lambda_99fb1378e971ab6e7edea83e3a7a83a2>@@@?$__crt_seh_guarded_call@H@@QEAAH$$QEAV<lambda_a37b2b86f63e897a80ea819b0eb08c01>@@AEAV<lambda_38ce7e780aa69e748d6df282ebc68efe>@@$$QEAV<lambda_99fb1378e971ab6e7edea83e3a7a83a2>@@@Z 000000018003d978 f   libucrt:commit.obj
 0001:0003e788       memcpy_s                   000000018003f788 f   libucrt:cfout.obj
 0001:0003f1b8       ?free_crt_array_internal@@YAXQEAPEBX_K@Z 00000001800401b8 f   libucrt:inittime.obj
 0001:0003f208       ?initialize_lc_time@@YA_NQEAU__crt_lc_time_data@@QEAU__crt_locale_data@@@Z 0000000180040208 f   libucrt:inittime.obj
 0001:0003f778       GetLocaleNameFromLangCountry 0000000180040778 f   libucrt:get_qualified_locale.obj
 0001:0003f838       GetLocaleNameFromLanguage  0000000180040838 f   libucrt:get_qualified_locale.obj
 0001:0003f8c0       GetPrimaryLen              00000001800408c0 f   libucrt:get_qualified_locale.obj
 0001:0003f918       LangCountryEnumProcEx      0000000180040918 f   libucrt:get_qualified_locale.obj
 0001:0003fc50       LanguageEnumProcEx         0000000180040c50 f   libucrt:get_qualified_locale.obj
 0001:0003fd30       ProcessCodePage            0000000180040d30 f   libucrt:get_qualified_locale.obj
 0001:0003fdf8       TranslateName              0000000180040df8 f   libucrt:get_qualified_locale.obj
 0001:00040158       CountryEnumProc            0000000180041158 f   libucrt:getqloc_downlevel.obj
 0001:00040238       GetLcidFromLangCountry     0000000180041238 f   libucrt:getqloc_downlevel.obj
 0001:00040310       GetLcidFromLanguage        0000000180041310 f   libucrt:getqloc_downlevel.obj
 0001:000403a0       GetPrimaryLen              00000001800413a0 f   libucrt:getqloc_downlevel.obj
 0001:000403e8       LangCountryEnumProc        00000001800413e8 f   libucrt:getqloc_downlevel.obj
 0001:00040690       LanguageEnumProc           0000000180041690 f   libucrt:getqloc_downlevel.obj
 0001:00040788       LcidFromHexString          0000000180041788 f   libucrt:getqloc_downlevel.obj
 0001:000407f0       ProcessCodePage            00000001800417f0 f   libucrt:getqloc_downlevel.obj
 0001:000408c8       TestDefaultLanguage        00000001800418c8 f   libucrt:getqloc_downlevel.obj
 0001:00040978       TranslateName              0000000180041978 f   libucrt:getqloc_downlevel.obj
 0001:00040f50       _abstract_sw               0000000180041f50 f   libucrt:ieee.obj
 0001:00041610       ?initialize_multibyte@@YAHXZ 0000000180042610 f   libucrt:multibyte_initializer.obj
 0001:00041860       ??$?RV<lambda_751a882b2c74d4b022dec766aa51a29a>@@AEAV<lambda_628dfdc04ba53c8bfc02c9951375f3f5>@@V<lambda_f6c7be5f7998530c34de24c7437d6b54>@@@?$__crt_seh_guarded_call@H@@QEAAH$$QEAV<lambda_751a882b2c74d4b022dec766aa51a29a>@@AEAV<lambda_628dfdc04ba53c8bfc02c9951375f3f5>@@$$QEAV<lambda_f6c7be5f7998530c34de24c7437d6b54>@@@Z 0000000180042860 f   libucrt:close.obj
 0001:00041fd0       ??$common_xtox@K_W@@YAHKQEA_W_KI_N@Z 0000000180042fd0 f   libucrt:xtoa.obj
 0001:00042098       ??$common_xtox_s@K_W@@YAHKQEA_W_KI_N@Z 0000000180043098 f   libucrt:xtoa.obj
 0001:00042758       ?dtor$0@?0???$?RH$0A@@?$precision_checker@Uerror_handler@detail@v8@fmt@@@detail@v8@fmt@@QEAA_KH@Z@4HA 0000000180043758 f   format.obj
 0001:00042758       ?dtor$0@?0???$?RH$0A@@?$width_checker@Uerror_handler@detail@v8@fmt@@@detail@v8@fmt@@QEAA_KH@Z@4HA 0000000180043758 f   format.obj
 0001:00042758       ?dtor$0@?0???$?RM$0A@@?$precision_checker@Uerror_handler@detail@v8@fmt@@@detail@v8@fmt@@QEAA_KM@Z@4HA 0000000180043758 f   format.obj
 0001:00042758       ?dtor$0@?0???$?RM$0A@@?$width_checker@Uerror_handler@detail@v8@fmt@@@detail@v8@fmt@@QEAA_KM@Z@4HA 0000000180043758 f   format.obj
 0001:00042758       ?dtor$0@?0???$?RN$0A@@?$precision_checker@Uerror_handler@detail@v8@fmt@@@detail@v8@fmt@@QEAA_KN@Z@4HA 0000000180043758 f   format.obj
 0001:00042758       ?dtor$0@?0???$?RN$0A@@?$width_checker@Uerror_handler@detail@v8@fmt@@@detail@v8@fmt@@QEAA_KN@Z@4HA 0000000180043758 f   format.obj
 0001:00042758       ?dtor$0@?0???$?RO$0A@@?$precision_checker@Uerror_handler@detail@v8@fmt@@@detail@v8@fmt@@QEAA_KO@Z@4HA 0000000180043758 f   format.obj
 0001:00042758       ?dtor$0@?0???$?RO$0A@@?$width_checker@Uerror_handler@detail@v8@fmt@@@detail@v8@fmt@@QEAA_KO@Z@4HA 0000000180043758 f   format.obj
 0001:00042758       ?dtor$0@?0???$?RPEBX$0A@@?$precision_checker@Uerror_handler@detail@v8@fmt@@@detail@v8@fmt@@QEAA_KPEBX@Z@4HA 0000000180043758 f   format.obj
 0001:00042758       ?dtor$0@?0???$?RPEBX$0A@@?$width_checker@Uerror_handler@detail@v8@fmt@@@detail@v8@fmt@@QEAA_KPEBX@Z@4HA 0000000180043758 f   format.obj
 0001:00042758       ?dtor$0@?0???$?RUmonostate@v8@fmt@@$0A@@?$precision_checker@Uerror_handler@detail@v8@fmt@@@detail@v8@fmt@@QEAA_KUmonostate@23@@Z@4HA 0000000180043758 f   format.obj
 0001:00042758       ?dtor$0@?0???$?RUmonostate@v8@fmt@@$0A@@?$width_checker@Uerror_handler@detail@v8@fmt@@@detail@v8@fmt@@QEAA_KUmonostate@23@@Z@4HA 0000000180043758 f   format.obj
 0001:00042758       ?dtor$0@?0???$?R_J$0A@@?$precision_checker@Uerror_handler@detail@v8@fmt@@@detail@v8@fmt@@QEAA_K_J@Z@4HA 0000000180043758 f   format.obj
 0001:00042758       ?dtor$0@?0???$?R_J$0A@@?$width_checker@Uerror_handler@detail@v8@fmt@@@detail@v8@fmt@@QEAA_K_J@Z@4HA 0000000180043758 f   format.obj
 0001:00042758       ?dtor$0@?0???$?R_N$0A@@?$precision_checker@Uerror_handler@detail@v8@fmt@@@detail@v8@fmt@@QEAA_K_N@Z@4HA 0000000180043758 f   format.obj
 0001:00042758       ?dtor$0@?0???$?R_N$0A@@?$width_checker@Uerror_handler@detail@v8@fmt@@@detail@v8@fmt@@QEAA_K_N@Z@4HA 0000000180043758 f   format.obj
 0001:00042758       ?dtor$0@?0??on_error@error_handler@detail@v8@fmt@@QEAAXPEBD@Z@4HA 0000000180043758 f   format.obj
 0001:00042758       ?dtor$0@?0??throw_format_error@detail@v8@fmt@@YAXPEBD@Z@4HA 0000000180043758 f   format.obj
 0001:00042758       ?dtor$0@?0???$do_parse_arg_id@_WAEAUid_adapter@?1???$parse_replacement_field@_WAEAUformat_handler@?1???$vformat_to@_W@detail@v8@fmt@@YAXAEAV?$buffer@_W@234@V?$basic_string_view@_W@34@V?$basic_format_args@V?$basic_format_context@V?$back_insert_iterator@V?$buffer@_W@detail@v8@fmt@@@std@@_W@v8@fmt@@@34@Vlocale_ref@234@@Z@@detail@v8@fmt@@YAPEB_WPEB_W0AEAUformat_handler@?1???$vformat_to@_W@234@YAXAEAV?$buffer@_W@234@V?$basic_string_view@_W@34@V?$basic_format_args@V?$basic_format_context@V?$back_insert_iterator@V?$buffer@_W@detail@v8@fmt@@@std@@_W@v8@fmt@@@34@Vlocale_ref@234@@Z@@Z@@detail@v8@fmt@@YAPEB_WPEB_W0AEAUid_adapter@?1???$parse_replacement_field@_WAEAUformat_handler@?1???$vformat_to@_W@detail@v8@fmt@@YAXAEAV?$buffer@_W@234@V?$basic_string_view@_W@34@V?$basic_format_args@V?$basic_format_context@V?$back_insert_iterator@V?$buffer@_W@detail@v8@fmt@@@std@@_W@v8@fmt@@@34@Vlocale_ref@234@@Z@@012@YAPEB_W00AEAUformat_handler@?1???$vformat_to@_W@012@YAXAEAV?$buffer@_W@012@V?$basic_string_view@_W@12@V?$basic_format_args@V?$basic_format_context@V?$back_insert_iterator@V?$buffer@_W@detail@v8@fmt@@@std@@_W@v8@fmt@@@12@Vlocale_ref@012@@Z@@Z@@Z@4HA 0000000180043758 f   handles.obj
 0001:00042758       ?dtor$0@?0???$get_arg@V?$basic_format_context@V?$back_insert_iterator@V?$buffer@_W@detail@v8@fmt@@@std@@_W@v8@fmt@@H@detail@v8@fmt@@YA?AV?$basic_format_arg@V?$basic_format_context@V?$back_insert_iterator@V?$buffer@_W@detail@v8@fmt@@@std@@_W@v8@fmt@@@12@AEAV?$basic_format_context@V?$back_insert_iterator@V?$buffer@_W@detail@v8@fmt@@@std@@_W@12@H@Z@4HA 0000000180043758 f   handles.obj
 0001:00042758       ?dtor$0@?0???$write@_WV?$back_insert_iterator@V?$buffer@_W@detail@v8@fmt@@@std@@X$0A@@detail@v8@fmt@@YA?AV?$back_insert_iterator@V?$buffer@_W@detail@v8@fmt@@@std@@V34@PEBXAEBU?$basic_format_specs@_W@12@Vlocale_ref@012@@Z@4HA 0000000180043758 f   handles.obj
 0001:00042758       ?dtor$0@?0???$write_int@_WV?$back_insert_iterator@V?$buffer@_W@detail@v8@fmt@@@std@@I@detail@v8@fmt@@YA?AV?$back_insert_iterator@V?$buffer@_W@detail@v8@fmt@@@std@@V34@U?$write_int_arg@I@012@AEBU?$basic_format_specs@_W@12@Vlocale_ref@012@@Z@4HA 0000000180043758 f   handles.obj
 0001:00042758       ?dtor$0@?0???Rwriter@?1???$parse_format_string@$0A@_WUformat_handler@?1???$vformat_to@_W@detail@v8@fmt@@YAXAEAV?$buffer@_W@234@V?$basic_string_view@_W@34@V?$basic_format_args@V?$basic_format_context@V?$back_insert_iterator@V?$buffer@_W@detail@v8@fmt@@@std@@_W@v8@fmt@@@34@Vlocale_ref@234@@Z@@detail@v8@fmt@@YAXV?$basic_string_view@_W@23@$$QEAUformat_handler@?1???$vformat_to@_W@123@YAXAEAV?$buffer@_W@123@0V?$basic_format_args@V?$basic_format_context@V?$back_insert_iterator@V?$buffer@_W@detail@v8@fmt@@@std@@_W@v8@fmt@@@23@Vlocale_ref@123@@Z@@Z@QEAAXPEB_W5@Z@4HA 0000000180043758 f   handles.obj
 0001:00042758       ?dtor$0@?0??check_arg_id@?$basic_format_parse_context@_WUerror_handler@detail@v8@fmt@@@v8@fmt@@QEAAXH@Z@4HA 0000000180043758 f   handles.obj
 0001:00042758       ?dtor$0@?0??next_arg_id@?$basic_format_parse_context@_WUerror_handler@detail@v8@fmt@@@v8@fmt@@QEAAHXZ@4HA 0000000180043758 f   handles.obj
 0001:00042758       ?dtor$0@?0??on_error@?$specs_handler@_W@detail@v8@fmt@@QEAAXPEBD@Z@4HA 0000000180043758 f   handles.obj
 0001:00042758       ?dtor$0@?0??on_error@id_adapter@?1???$parse_replacement_field@_WAEAUformat_handler@?1???$vformat_to@_W@detail@v8@fmt@@YAXAEAV?$buffer@_W@234@V?$basic_string_view@_W@34@V?$basic_format_args@V?$basic_format_context@V?$back_insert_iterator@V?$buffer@_W@detail@v8@fmt@@@std@@_W@v8@fmt@@@34@Vlocale_ref@234@@Z@@detail@v8@fmt@@YAPEB_WPEB_W0AEAUformat_handler@?1???$vformat_to@_W@234@YAXAEAV?$buffer@_W@234@V?$basic_string_view@_W@34@V?$basic_format_args@V?$basic_format_context@V?$back_insert_iterator@V?$buffer@_W@detail@v8@fmt@@@std@@_W@v8@fmt@@@34@Vlocale_ref@234@@Z@@Z@QEAAXPEBD@Z@4HA 0000000180043758 f   handles.obj
 0001:00042758       ?dtor$0@?0??on_error@precision_adapter@?1???$parse_precision@_WAEAV?$specs_checker@V?$specs_handler@_W@detail@v8@fmt@@@detail@v8@fmt@@@detail@v8@fmt@@YAPEB_WPEB_W0AEAV?$specs_checker@V?$specs_handler@_W@detail@v8@fmt@@@234@@Z@QEAAXPEBD@Z@4HA 0000000180043758 f   handles.obj
 0001:00042758       ?dtor$0@?0??on_error@width_adapter@?1???$parse_width@_WAEAV?$specs_checker@V?$specs_handler@_W@detail@v8@fmt@@@detail@v8@fmt@@@detail@v8@fmt@@YAPEB_WPEB_W0AEAV?$specs_checker@V?$specs_handler@_W@detail@v8@fmt@@@234@@Z@QEAAXPEBD@Z@4HA 0000000180043758 f   handles.obj
 0001:00042758       ?dtor$0@?0??require_numeric_argument@?$specs_checker@V?$specs_handler@_W@detail@v8@fmt@@@detail@v8@fmt@@AEAAXXZ@4HA 0000000180043758 f   handles.obj
 0001:00042758       ?dtor$3@?0???$do_parse_arg_id@_WAEAUprecision_adapter@?1???$parse_precision@_WAEAV?$specs_checker@V?$specs_handler@_W@detail@v8@fmt@@@detail@v8@fmt@@@detail@v8@fmt@@YAPEB_WPEB_W0AEAV?$specs_checker@V?$specs_handler@_W@detail@v8@fmt@@@234@@Z@@detail@v8@fmt@@YAPEB_WPEB_W0AEAUprecision_adapter@?1???$parse_precision@_WAEAV?$specs_checker@V?$specs_handler@_W@detail@v8@fmt@@@detail@v8@fmt@@@012@YAPEB_W00AEAV?$specs_checker@V?$specs_handler@_W@detail@v8@fmt@@@012@@Z@@Z@4HA 0000000180043758 f   handles.obj
 0001:00042758       ?dtor$3@?0???$do_parse_arg_id@_WAEAUwidth_adapter@?1???$parse_width@_WAEAV?$specs_checker@V?$specs_handler@_W@detail@v8@fmt@@@detail@v8@fmt@@@detail@v8@fmt@@YAPEB_WPEB_W0AEAV?$specs_checker@V?$specs_handler@_W@detail@v8@fmt@@@234@@Z@@detail@v8@fmt@@YAPEB_WPEB_W0AEAUwidth_adapter@?1???$parse_width@_WAEAV?$specs_checker@V?$specs_handler@_W@detail@v8@fmt@@@detail@v8@fmt@@@012@YAPEB_W00AEAV?$specs_checker@V?$specs_handler@_W@detail@v8@fmt@@@012@@Z@@Z@4HA 0000000180043758 f   handles.obj
 0001:00042758       ?dtor$3@?0???$parse_align@_WAEAV?$specs_checker@V?$specs_handler@_W@detail@v8@fmt@@@detail@v8@fmt@@@detail@v8@fmt@@YAPEB_WPEB_W0AEAV?$specs_checker@V?$specs_handler@_W@detail@v8@fmt@@@012@@Z@4HA 0000000180043758 f   handles.obj
 0001:00042758       ?dtor$3@?0???$parse_precision@_WAEAV?$specs_checker@V?$specs_handler@_W@detail@v8@fmt@@@detail@v8@fmt@@@detail@v8@fmt@@YAPEB_WPEB_W0AEAV?$specs_checker@V?$specs_handler@_W@detail@v8@fmt@@@012@@Z@4HA 0000000180043758 f   handles.obj
 0001:00042758       ?dtor$3@?0???$parse_width@_WAEAV?$specs_checker@V?$specs_handler@_W@detail@v8@fmt@@@detail@v8@fmt@@@detail@v8@fmt@@YAPEB_WPEB_W0AEAV?$specs_checker@V?$specs_handler@_W@detail@v8@fmt@@@012@@Z@4HA 0000000180043758 f   handles.obj
 0001:00042758       ?dtor$6@?0???$visit_format_arg@V?$precision_checker@Uerror_handler@detail@v8@fmt@@@detail@v8@fmt@@V?$basic_format_context@V?$back_insert_iterator@V?$buffer@_W@detail@v8@fmt@@@std@@_W@34@@v8@fmt@@YA_K$$QEAV?$precision_checker@Uerror_handler@detail@v8@fmt@@@detail@01@AEBV?$basic_format_arg@V?$basic_format_context@V?$back_insert_iterator@V?$buffer@_W@detail@v8@fmt@@@std@@_W@v8@fmt@@@01@@Z@4HA 0000000180043758 f   handles.obj
 0001:00042758       ?dtor$6@?0???$visit_format_arg@V?$width_checker@Uerror_handler@detail@v8@fmt@@@detail@v8@fmt@@V?$basic_format_context@V?$back_insert_iterator@V?$buffer@_W@detail@v8@fmt@@@std@@_W@34@@v8@fmt@@YA_K$$QEAV?$width_checker@Uerror_handler@detail@v8@fmt@@@detail@01@AEBV?$basic_format_arg@V?$basic_format_context@V?$back_insert_iterator@V?$buffer@_W@detail@v8@fmt@@@std@@_W@v8@fmt@@@01@@Z@4HA 0000000180043758 f   handles.obj
 0001:0004276c       ?dtor$0@?0??square@bigint@detail@v8@fmt@@QEAAXXZ@4HA 000000018004376c f   format.obj
 0001:00042780       ?dtor$0@?0??format_dragon@detail@v8@fmt@@YAXUfp@123@_NHAEAV?$buffer@D@123@AEAH@Z@4HA 0000000180043780 f   format.obj
 0001:00042794       ?dtor$1@?0??format_dragon@detail@v8@fmt@@YAXUfp@123@_NHAEAV?$buffer@D@123@AEAH@Z@4HA 0000000180043794 f   format.obj
 0001:000427a8       ?dtor$2@?0??format_dragon@detail@v8@fmt@@YAXUfp@123@_NHAEAV?$buffer@D@123@AEAH@Z@4HA 00000001800437a8 f   format.obj
 0001:000427bc       ?dtor$3@?0??format_dragon@detail@v8@fmt@@YAXUfp@123@_NHAEAV?$buffer@D@123@AEAH@Z@4HA 00000001800437bc f   format.obj
 0001:000427d0       ?dtor$0@?0???$thousands_sep_impl@_W@detail@v8@fmt@@YA?AU?$thousands_sep_result@_W@012@Vlocale_ref@012@@Z@4HA 00000001800437d0 f   format.obj
 0001:000427e4       ?dtor$1@?0???$thousands_sep_impl@_W@detail@v8@fmt@@YA?AU?$thousands_sep_result@_W@012@Vlocale_ref@012@@Z@4HA 00000001800437e4 f   format.obj
 0001:000427f8       ?dtor$0@?0???$use_facet@V?$numpunct@_W@std@@@std@@YAAEBV?$numpunct@_W@0@AEBVlocale@0@@Z@4HA 00000001800437f8 f   format.obj
 0001:0004280c       ?dtor$1@?0???$use_facet@V?$numpunct@_W@std@@@std@@YAAEBV?$numpunct@_W@0@AEBVlocale@0@@Z@4HA 000000018004380c f   format.obj
 0001:00042820       ?dtor$0@?0??_Getcat@?$numpunct@_W@std@@SA_KPEAPEBVfacet@locale@2@PEBV42@@Z@4HA 0000000180043820 f   format.obj
 0001:00042838       ?dtor$1@?0??_Getcat@?$numpunct@_W@std@@SA_KPEAPEBVfacet@locale@2@PEBV42@@Z@4HA 0000000180043838 f   format.obj
 0001:00042868       ?dtor$2@?0??_Getcat@?$numpunct@_W@std@@SA_KPEAPEBVfacet@locale@2@PEBV42@@Z@4HA 0000000180043868 f   format.obj
 0001:0004287c       ?dtor$3@?0??_Getcat@?$numpunct@_W@std@@SA_KPEAPEBVfacet@locale@2@PEBV42@@Z@4HA 000000018004387c f   format.obj
 0001:00042894       ?dtor$4@?0??_Getcat@?$numpunct@_W@std@@SA_KPEAPEBVfacet@locale@2@PEBV42@@Z@4HA 0000000180043894 f   format.obj
 0001:000428ac       ?dtor$5@?0??_Getcat@?$numpunct@_W@std@@SA_KPEAPEBVfacet@locale@2@PEBV42@@Z@4HA 00000001800438ac f   format.obj
 0001:000428c4       ?dtor$6@?0??_Getcat@?$numpunct@_W@std@@SA_KPEAPEBVfacet@locale@2@PEBV42@@Z@4HA 00000001800438c4 f   format.obj
 0001:000428dc       ?dtor$7@?0??_Getcat@?$numpunct@_W@std@@SA_KPEAPEBVfacet@locale@2@PEBV42@@Z@4HA 00000001800438dc f   format.obj
 0001:000428f4       ?dtor$8@?0??_Getcat@?$numpunct@_W@std@@SA_KPEAPEBVfacet@locale@2@PEBV42@@Z@4HA 00000001800438f4 f   format.obj
 0001:0004290c       ?dtor$9@?0??_Getcat@?$numpunct@_W@std@@SA_KPEAPEBVfacet@locale@2@PEBV42@@Z@4HA 000000018004390c f   format.obj
 0001:00042920       ?dtor$0@?0??_Init@?$numpunct@_W@std@@IEAAXAEBV_Locinfo@2@_N@Z@4HA 0000000180043920 f   format.obj
 0001:00042934       ?dtor$0@?0???$decimal_point@_W@detail@v8@fmt@@YA_WVlocale_ref@012@@Z@4HA 0000000180043934 f   handles.obj
 0001:00042948       ?dtor$0@?0??GetFileName@@YA?AV?$basic_string@_WU?$char_traits@_W@std@@V?$allocator@_W@2@@std@@PEAX@Z@4HA 0000000180043948 f   handles.obj
 0001:0004295c       ?dtor$2@?0??GetFileName@@YA?AV?$basic_string@_WU?$char_traits@_W@std@@V?$allocator@_W@2@@std@@PEAX@Z@4HA 000000018004395c f   handles.obj
 0001:0004295c       ?dtor$7@?0??GetFileName@@YA?AV?$basic_string@_WU?$char_traits@_W@std@@V?$allocator@_W@2@@std@@PEAX@Z@4HA 000000018004395c f   handles.obj
 0001:00042970       ?dtor$1@?0???R<lambda_1>@?1??GetUserAccountID@@YA@XZ@QEBA?AV?$basic_string@_WU?$char_traits@_W@std@@V?$allocator@_W@2@@std@@XZ@4HA 0000000180043970 f   handles.obj
 0001:00042984       ?dtor$2@?0???R<lambda_1>@?1??GetUserAccountID@@YA@XZ@QEBA?AV?$basic_string@_WU?$char_traits@_W@std@@V?$allocator@_W@2@@std@@XZ@4HA 0000000180043984 f   handles.obj
 0001:00042998       ?dtor$0@?0??WinError@@YAHPEB_W@Z@4HA 0000000180043998 f   Pmix.obj
 0001:00042998       ?dtor$3@?0???R<lambda_1>@?1??GetUserAccountID@@YA@XZ@QEBA?AV?$basic_string@_WU?$char_traits@_W@std@@V?$allocator@_W@2@@std@@XZ@4HA 0000000180043998 f   handles.obj
 0001:000429ac       ?dtor$1@?0??GetNameByType@@YA?AV?$basic_string@_WU?$char_traits@_W@std@@V?$allocator@_W@2@@std@@PEAXGPEAVPerfThread@@@Z@4HA 00000001800439ac f   handles.obj
 0001:000429ac       ?dtor$6@?0??RefreshWMIData@PerfThread@@AEAAXXZ@4HA 00000001800439ac f   perfthread.obj
 0001:000429c0       ?dtor$20@?0??GetNameByType@@YA?AV?$basic_string@_WU?$char_traits@_W@std@@V?$allocator@_W@2@@std@@PEAXGPEAVPerfThread@@@Z@4HA 00000001800439c0 f   handles.obj
 0001:000429c0       ?dtor$2@?0??GetNameByType@@YA?AV?$basic_string@_WU?$char_traits@_W@std@@V?$allocator@_W@2@@std@@PEAXGPEAVPerfThread@@@Z@4HA 00000001800439c0 f   handles.obj
 0001:000429d4       ?dtor$0@?0??Connect@Plist@@QEAA_NPEB_W00@Z@4HA 00000001800439d4 f   Pclass.obj
 0001:000429d4       ?dtor$3@?0??GetNameByType@@YA?AV?$basic_string@_WU?$char_traits@_W@std@@V?$allocator@_W@2@@std@@PEAXGPEAVPerfThread@@@Z@4HA 00000001800439d4 f   handles.obj
 0001:000429e8       ?dtor$31@?0??GetNameByType@@YA?AV?$basic_string@_WU?$char_traits@_W@std@@V?$allocator@_W@2@@std@@PEAXGPEAVPerfThread@@@Z@4HA 00000001800439e8 f   handles.obj
 0001:00042a08       ?dtor$0@?0??PrintHandleInfo@@YA_NKPEAX_NPEAVPerfThread@@@Z@4HA 0000000180043a08 f   handles.obj
 0001:00042a1c       ?dtor$1@?0??PrintModules@@YAXPEAXKAEAUoptions@@@Z@4HA 0000000180043a1c f   Plist.obj
 0001:00042a1c       ?dtor$3@?0??PrintHandleInfo@@YA_NKPEAX_NPEAVPerfThread@@@Z@4HA 0000000180043a1c f   handles.obj
 0001:00042a30       ?dtor$5@?0??PrintHandleInfo@@YA_NKPEAX_NPEAVPerfThread@@@Z@4HA 0000000180043a30 f   handles.obj
 0001:00042a44       ?dtor$6@?0??PrintHandleInfo@@YA_NKPEAX_NPEAVPerfThread@@@Z@4HA 0000000180043a44 f   handles.obj
 0001:00042a58       ?dtor$11@?0??PrintHandleInfo@@YA_NKPEAX_NPEAVPerfThread@@@Z@4HA 0000000180043a58 f   handles.obj
 0001:00042a58       ?dtor$13@?0??PrintHandleInfo@@YA_NKPEAX_NPEAVPerfThread@@@Z@4HA 0000000180043a58 f   handles.obj
 0001:00042a6c       ?dtor$0@?0???$visit_format_arg@U?$default_arg_formatter@_W@detail@v8@fmt@@V?$basic_format_context@V?$back_insert_iterator@V?$buffer@_W@detail@v8@fmt@@@std@@_W@34@@v8@fmt@@YA?AV?$back_insert_iterator@V?$buffer@_W@detail@v8@fmt@@@std@@$$QEAU?$default_arg_formatter@_W@detail@01@AEBV?$basic_format_arg@V?$basic_format_context@V?$back_insert_iterator@V?$buffer@_W@detail@v8@fmt@@@std@@_W@v8@fmt@@@01@@Z@4HA 0000000180043a6c f   handles.obj
 0001:00042a80       ?dtor$0@?0???$parse_replacement_field@_WAEAUformat_handler@?1???$vformat_to@_W@detail@v8@fmt@@YAXAEAV?$buffer@_W@234@V?$basic_string_view@_W@34@V?$basic_format_args@V?$basic_format_context@V?$back_insert_iterator@V?$buffer@_W@detail@v8@fmt@@@std@@_W@v8@fmt@@@34@Vlocale_ref@234@@Z@@detail@v8@fmt@@YAPEB_WPEB_W0AEAUformat_handler@?1???$vformat_to@_W@012@YAXAEAV?$buffer@_W@012@V?$basic_string_view@_W@12@V?$basic_format_args@V?$basic_format_context@V?$back_insert_iterator@V?$buffer@_W@detail@v8@fmt@@@std@@_W@v8@fmt@@@12@Vlocale_ref@012@@Z@@Z@4HA 0000000180043a80 f   handles.obj
 0001:00042a80       ?dtor$0@?0???$visit_format_arg@AEAU?$arg_formatter@_W@detail@v8@fmt@@V?$basic_format_context@V?$back_insert_iterator@V?$buffer@_W@detail@v8@fmt@@@std@@_W@34@@v8@fmt@@YA?AV?$back_insert_iterator@V?$buffer@_W@detail@v8@fmt@@@std@@AEAU?$arg_formatter@_W@detail@01@AEBV?$basic_format_arg@V?$basic_format_context@V?$back_insert_iterator@V?$buffer@_W@detail@v8@fmt@@@std@@_W@v8@fmt@@@01@@Z@4HA 0000000180043a80 f   handles.obj
 0001:00042a94       ?dtor$0@?0???$parse_format_string@$0A@_WUformat_handler@?1???$vformat_to@_W@detail@v8@fmt@@YAXAEAV?$buffer@_W@234@V?$basic_string_view@_W@34@V?$basic_format_args@V?$basic_format_context@V?$back_insert_iterator@V?$buffer@_W@detail@v8@fmt@@@std@@_W@v8@fmt@@@34@Vlocale_ref@234@@Z@@detail@v8@fmt@@YAXV?$basic_string_view@_W@12@$$QEAUformat_handler@?1???$vformat_to@_W@012@YAXAEAV?$buffer@_W@012@0V?$basic_format_args@V?$basic_format_context@V?$back_insert_iterator@V?$buffer@_W@detail@v8@fmt@@@std@@_W@v8@fmt@@@12@Vlocale_ref@012@@Z@@Z@4HA 0000000180043a94 f   handles.obj
 0001:00042aa8       ?dtor$0@?0???$vformat@_W$0A@@v8@fmt@@YA?AV?$basic_string@_WU?$char_traits@_W@std@@V?$allocator@_W@2@@std@@V?$basic_string_view@_W@01@V?$basic_format_args@V?$basic_format_context@V?$back_insert_iterator@V?$buffer@_W@detail@v8@fmt@@@std@@_W@v8@fmt@@@01@@Z@4HA 0000000180043aa8 f   handles.obj
 0001:00042abc       ?dtor$2@?0???$vformat@_W$0A@@v8@fmt@@YA?AV?$basic_string@_WU?$char_traits@_W@std@@V?$allocator@_W@2@@std@@V?$basic_string_view@_W@01@V?$basic_format_args@V?$basic_format_context@V?$back_insert_iterator@V?$buffer@_W@detail@v8@fmt@@@std@@_W@v8@fmt@@@01@@Z@4HA 0000000180043abc f   handles.obj
 0001:00042ad0       ?dtor$0@?0???$do_parse_arg_id@_WAEAUprecision_adapter@?1???$parse_precision@_WAEAV?$specs_checker@V?$specs_handler@_W@detail@v8@fmt@@@detail@v8@fmt@@@detail@v8@fmt@@YAPEB_WPEB_W0AEAV?$specs_checker@V?$specs_handler@_W@detail@v8@fmt@@@234@@Z@@detail@v8@fmt@@YAPEB_WPEB_W0AEAUprecision_adapter@?1???$parse_precision@_WAEAV?$specs_checker@V?$specs_handler@_W@detail@v8@fmt@@@detail@v8@fmt@@@012@YAPEB_W00AEAV?$specs_checker@V?$specs_handler@_W@detail@v8@fmt@@@012@@Z@@Z@4HA 0000000180043ad0 f   handles.obj
 0001:00042ad0       ?dtor$0@?0???$do_parse_arg_id@_WAEAUwidth_adapter@?1???$parse_width@_WAEAV?$specs_checker@V?$specs_handler@_W@detail@v8@fmt@@@detail@v8@fmt@@@detail@v8@fmt@@YAPEB_WPEB_W0AEAV?$specs_checker@V?$specs_handler@_W@detail@v8@fmt@@@234@@Z@@detail@v8@fmt@@YAPEB_WPEB_W0AEAUwidth_adapter@?1???$parse_width@_WAEAV?$specs_checker@V?$specs_handler@_W@detail@v8@fmt@@@detail@v8@fmt@@@012@YAPEB_W00AEAV?$specs_checker@V?$specs_handler@_W@detail@v8@fmt@@@012@@Z@@Z@4HA 0000000180043ad0 f   handles.obj
 0001:00042ad0       ?dtor$0@?0???$parse_align@_WAEAV?$specs_checker@V?$specs_handler@_W@detail@v8@fmt@@@detail@v8@fmt@@@detail@v8@fmt@@YAPEB_WPEB_W0AEAV?$specs_checker@V?$specs_handler@_W@detail@v8@fmt@@@012@@Z@4HA 0000000180043ad0 f   handles.obj
 0001:00042ad0       ?dtor$0@?0???$parse_precision@_WAEAV?$specs_checker@V?$specs_handler@_W@detail@v8@fmt@@@detail@v8@fmt@@@detail@v8@fmt@@YAPEB_WPEB_W0AEAV?$specs_checker@V?$specs_handler@_W@detail@v8@fmt@@@012@@Z@4HA 0000000180043ad0 f   handles.obj
 0001:00042ad0       ?dtor$0@?0???$parse_width@_WAEAV?$specs_checker@V?$specs_handler@_W@detail@v8@fmt@@@detail@v8@fmt@@@detail@v8@fmt@@YAPEB_WPEB_W0AEAV?$specs_checker@V?$specs_handler@_W@detail@v8@fmt@@@012@@Z@4HA 0000000180043ad0 f   handles.obj
 0001:00042ad0       ?dtor$0@?0??get_arg@?$specs_handler@_W@detail@v8@fmt@@AEAA?AV?$basic_format_arg@V?$basic_format_context@V?$back_insert_iterator@V?$buffer@_W@detail@v8@fmt@@@std@@_W@v8@fmt@@@34@V?$basic_string_view@_W@34@@Z@4HA 0000000180043ad0 f   handles.obj
 0001:00042ad0       ?dtor$3@?0???$visit_format_arg@V?$precision_checker@Uerror_handler@detail@v8@fmt@@@detail@v8@fmt@@V?$basic_format_context@V?$back_insert_iterator@V?$buffer@_W@detail@v8@fmt@@@std@@_W@34@@v8@fmt@@YA_K$$QEAV?$precision_checker@Uerror_handler@detail@v8@fmt@@@detail@01@AEBV?$basic_format_arg@V?$basic_format_context@V?$back_insert_iterator@V?$buffer@_W@detail@v8@fmt@@@std@@_W@v8@fmt@@@01@@Z@4HA 0000000180043ad0 f   handles.obj
 0001:00042ad0       ?dtor$3@?0???$visit_format_arg@V?$width_checker@Uerror_handler@detail@v8@fmt@@@detail@v8@fmt@@V?$basic_format_context@V?$back_insert_iterator@V?$buffer@_W@detail@v8@fmt@@@std@@_W@34@@v8@fmt@@YA_K$$QEAV?$width_checker@Uerror_handler@detail@v8@fmt@@@detail@01@AEBV?$basic_format_arg@V?$basic_format_context@V?$back_insert_iterator@V?$buffer@_W@detail@v8@fmt@@@std@@_W@v8@fmt@@@01@@Z@4HA 0000000180043ad0 f   handles.obj
 0001:00042ae4       ?dtor$12@?0???$parse_precision@_WAEAV?$specs_checker@V?$specs_handler@_W@detail@v8@fmt@@@detail@v8@fmt@@@detail@v8@fmt@@YAPEB_WPEB_W0AEAV?$specs_checker@V?$specs_handler@_W@detail@v8@fmt@@@012@@Z@4HA 0000000180043ae4 f   handles.obj
 0001:00042ae4       ?dtor$6@?0???$parse_width@_WAEAV?$specs_checker@V?$specs_handler@_W@detail@v8@fmt@@@detail@v8@fmt@@@detail@v8@fmt@@YAPEB_WPEB_W0AEAV?$specs_checker@V?$specs_handler@_W@detail@v8@fmt@@@012@@Z@4HA 0000000180043ae4 f   handles.obj
 0001:00042ae4       ?dtor$9@?0???$visit_format_arg@V?$precision_checker@Uerror_handler@detail@v8@fmt@@@detail@v8@fmt@@V?$basic_format_context@V?$back_insert_iterator@V?$buffer@_W@detail@v8@fmt@@@std@@_W@34@@v8@fmt@@YA_K$$QEAV?$precision_checker@Uerror_handler@detail@v8@fmt@@@detail@01@AEBV?$basic_format_arg@V?$basic_format_context@V?$back_insert_iterator@V?$buffer@_W@detail@v8@fmt@@@std@@_W@v8@fmt@@@01@@Z@4HA 0000000180043ae4 f   handles.obj
 0001:00042ae4       ?dtor$9@?0???$visit_format_arg@V?$width_checker@Uerror_handler@detail@v8@fmt@@@detail@v8@fmt@@V?$basic_format_context@V?$back_insert_iterator@V?$buffer@_W@detail@v8@fmt@@@std@@_W@34@@v8@fmt@@YA_K$$QEAV?$width_checker@Uerror_handler@detail@v8@fmt@@@detail@01@AEBV?$basic_format_arg@V?$basic_format_context@V?$back_insert_iterator@V?$buffer@_W@detail@v8@fmt@@@std@@_W@v8@fmt@@@01@@Z@4HA 0000000180043ae4 f   handles.obj
 0001:00042af8       ?dtor$12@?0???$visit_format_arg@V?$precision_checker@Uerror_handler@detail@v8@fmt@@@detail@v8@fmt@@V?$basic_format_context@V?$back_insert_iterator@V?$buffer@_W@detail@v8@fmt@@@std@@_W@34@@v8@fmt@@YA_K$$QEAV?$precision_checker@Uerror_handler@detail@v8@fmt@@@detail@01@AEBV?$basic_format_arg@V?$basic_format_context@V?$back_insert_iterator@V?$buffer@_W@detail@v8@fmt@@@std@@_W@v8@fmt@@@01@@Z@4HA 0000000180043af8 f   handles.obj
 0001:00042af8       ?dtor$12@?0???$visit_format_arg@V?$width_checker@Uerror_handler@detail@v8@fmt@@@detail@v8@fmt@@V?$basic_format_context@V?$back_insert_iterator@V?$buffer@_W@detail@v8@fmt@@@std@@_W@34@@v8@fmt@@YA_K$$QEAV?$width_checker@Uerror_handler@detail@v8@fmt@@@detail@01@AEBV?$basic_format_arg@V?$basic_format_context@V?$back_insert_iterator@V?$buffer@_W@detail@v8@fmt@@@std@@_W@v8@fmt@@@01@@Z@4HA 0000000180043af8 f   handles.obj
 0001:00042af8       ?dtor$6@?0???$parse_precision@_WAEAV?$specs_checker@V?$specs_handler@_W@detail@v8@fmt@@@detail@v8@fmt@@@detail@v8@fmt@@YAPEB_WPEB_W0AEAV?$specs_checker@V?$specs_handler@_W@detail@v8@fmt@@@012@@Z@4HA 0000000180043af8 f   handles.obj
 0001:00042b0c       ?dtor$9@?0???$parse_precision@_WAEAV?$specs_checker@V?$specs_handler@_W@detail@v8@fmt@@@detail@v8@fmt@@@detail@v8@fmt@@YAPEB_WPEB_W0AEAV?$specs_checker@V?$specs_handler@_W@detail@v8@fmt@@@012@@Z@4HA 0000000180043b0c f   handles.obj
 0001:00042b20       ?dtor$3@?0???$parse_replacement_field@_WAEAUformat_handler@?1???$vformat_to@_W@detail@v8@fmt@@YAXAEAV?$buffer@_W@234@V?$basic_string_view@_W@34@V?$basic_format_args@V?$basic_format_context@V?$back_insert_iterator@V?$buffer@_W@detail@v8@fmt@@@std@@_W@v8@fmt@@@34@Vlocale_ref@234@@Z@@detail@v8@fmt@@YAPEB_WPEB_W0AEAUformat_handler@?1???$vformat_to@_W@012@YAXAEAV?$buffer@_W@012@V?$basic_string_view@_W@12@V?$basic_format_args@V?$basic_format_context@V?$back_insert_iterator@V?$buffer@_W@detail@v8@fmt@@@std@@_W@v8@fmt@@@12@Vlocale_ref@012@@Z@@Z@4HA 0000000180043b20 f   handles.obj
 0001:00042b34       ?dtor$0@?0???$parse_float_type_spec@Uerror_handler@detail@v8@fmt@@_W@detail@v8@fmt@@YA?AUfloat_specs@012@AEBU?$basic_format_specs@_W@12@$$QEAUerror_handler@012@@Z@4HA 0000000180043b34 f   handles.obj
 0001:00042b34       ?dtor$0@?0???$write@_WV?$back_insert_iterator@V?$buffer@_W@detail@v8@fmt@@@std@@@detail@v8@fmt@@YA?AV?$back_insert_iterator@V?$buffer@_W@detail@v8@fmt@@@std@@V34@V?$basic_string_view@_W@12@AEBU?$basic_format_specs@_W@12@Vlocale_ref@012@@Z@4HA 0000000180043b34 f   handles.obj
 0001:00042b34       ?dtor$0@?0???$write_int@_WV?$back_insert_iterator@V?$buffer@_W@detail@v8@fmt@@@std@@_K@detail@v8@fmt@@YA?AV?$back_insert_iterator@V?$buffer@_W@detail@v8@fmt@@@std@@V34@U?$write_int_arg@_K@012@AEBU?$basic_format_specs@_W@12@Vlocale_ref@012@@Z@4HA 0000000180043b34 f   handles.obj
 0001:00042b48       ?dtor$0@?0???$write@_WV?$back_insert_iterator@V?$buffer@_W@detail@v8@fmt@@@std@@@detail@v8@fmt@@YA?AV?$back_insert_iterator@V?$buffer@_W@detail@v8@fmt@@@std@@V34@_WAEBU?$basic_format_specs@_W@12@Vlocale_ref@012@@Z@4HA 0000000180043b48 f   handles.obj
 0001:00042b5c       ?dtor$3@?0???$write@_WV?$back_insert_iterator@V?$buffer@_W@detail@v8@fmt@@@std@@@detail@v8@fmt@@YA?AV?$back_insert_iterator@V?$buffer@_W@detail@v8@fmt@@@std@@V34@_WAEBU?$basic_format_specs@_W@12@Vlocale_ref@012@@Z@4HA 0000000180043b5c f   handles.obj
 0001:00042b70       ?dtor$0@?0???$write@_WV?$back_insert_iterator@V?$buffer@_W@detail@v8@fmt@@@std@@M$0A@@detail@v8@fmt@@YA?AV?$back_insert_iterator@V?$buffer@_W@detail@v8@fmt@@@std@@V34@MU?$basic_format_specs@_W@12@Vlocale_ref@012@@Z@4HA 0000000180043b70 f   handles.obj
 0001:00042b70       ?dtor$0@?0???$write@_WV?$back_insert_iterator@V?$buffer@_W@detail@v8@fmt@@@std@@N$0A@@detail@v8@fmt@@YA?AV?$back_insert_iterator@V?$buffer@_W@detail@v8@fmt@@@std@@V34@NU?$basic_format_specs@_W@12@Vlocale_ref@012@@Z@4HA 0000000180043b70 f   handles.obj
 0001:00042b70       ?dtor$0@?0???$write@_WV?$back_insert_iterator@V?$buffer@_W@detail@v8@fmt@@@std@@O$0A@@detail@v8@fmt@@YA?AV?$back_insert_iterator@V?$buffer@_W@detail@v8@fmt@@@std@@V34@OU?$basic_format_specs@_W@12@Vlocale_ref@012@@Z@4HA 0000000180043b70 f   handles.obj
 0001:00042b84       ?dtor$0@?0???$do_write_float@V?$back_insert_iterator@V?$buffer@_W@detail@v8@fmt@@@std@@U?$decimal_fp@M@dragonbox@detail@v8@fmt@@_WV?$digit_grouping@_W@567@@detail@v8@fmt@@YA?AV?$back_insert_iterator@V?$buffer@_W@detail@v8@fmt@@@std@@V34@AEBU?$decimal_fp@M@dragonbox@012@AEBU?$basic_format_specs@_W@12@Ufloat_specs@012@Vlocale_ref@012@@Z@4HA 0000000180043b84 f   handles.obj
 0001:00042b84       ?dtor$1@?0???$do_write_float@V?$back_insert_iterator@V?$buffer@_W@detail@v8@fmt@@@std@@U?$decimal_fp@M@dragonbox@detail@v8@fmt@@_WV?$digit_grouping@_W@567@@detail@v8@fmt@@YA?AV?$back_insert_iterator@V?$buffer@_W@detail@v8@fmt@@@std@@V34@AEBU?$decimal_fp@M@dragonbox@012@AEBU?$basic_format_specs@_W@12@Ufloat_specs@012@Vlocale_ref@012@@Z@4HA 0000000180043b84 f   handles.obj
 0001:00042b84       ?dtor$2@?0???$do_write_float@V?$back_insert_iterator@V?$buffer@_W@detail@v8@fmt@@@std@@U?$decimal_fp@M@dragonbox@detail@v8@fmt@@_WV?$digit_grouping@_W@567@@detail@v8@fmt@@YA?AV?$back_insert_iterator@V?$buffer@_W@detail@v8@fmt@@@std@@V34@AEBU?$decimal_fp@M@dragonbox@012@AEBU?$basic_format_specs@_W@12@Ufloat_specs@012@Vlocale_ref@012@@Z@4HA 0000000180043b84 f   handles.obj
 0001:00042b98       ?dtor$0@?0???R<lambda_3>@?BD@???$do_write_float@V?$back_insert_iterator@V?$buffer@_W@detail@v8@fmt@@@std@@U?$decimal_fp@M@dragonbox@detail@v8@fmt@@_WV?$digit_grouping@_W@567@@detail@v8@fmt@@YA?AV?$back_insert_iterator@V?$buffer@_W@detail@v8@fmt@@@std@@V45@AEBU?$decimal_fp@M@dragonbox@123@AEBU?$basic_format_specs@_W@23@Ufloat_specs@123@Vlocale_ref@123@@Z@QEBA@0@Z@4HA 0000000180043b98 f   handles.obj
 0001:00042b98       ?dtor$0@?0???R<lambda_3>@?BD@???$do_write_float@V?$back_insert_iterator@V?$buffer@_W@detail@v8@fmt@@@std@@U?$decimal_fp@N@dragonbox@detail@v8@fmt@@_WV?$digit_grouping@_W@567@@detail@v8@fmt@@YA?AV?$back_insert_iterator@V?$buffer@_W@detail@v8@fmt@@@std@@V45@AEBU?$decimal_fp@N@dragonbox@123@AEBU?$basic_format_specs@_W@23@Ufloat_specs@123@Vlocale_ref@123@@Z@QEBA@0@Z@4HA 0000000180043b98 f   handles.obj
 0001:00042bac       ?dtor$0@?0???$do_write_float@V?$back_insert_iterator@V?$buffer@_W@detail@v8@fmt@@@std@@U?$decimal_fp@N@dragonbox@detail@v8@fmt@@_WV?$digit_grouping@_W@567@@detail@v8@fmt@@YA?AV?$back_insert_iterator@V?$buffer@_W@detail@v8@fmt@@@std@@V34@AEBU?$decimal_fp@N@dragonbox@012@AEBU?$basic_format_specs@_W@12@Ufloat_specs@012@Vlocale_ref@012@@Z@4HA 0000000180043bac f   handles.obj
 0001:00042bac       ?dtor$0@?0???$do_write_float@V?$back_insert_iterator@V?$buffer@_W@detail@v8@fmt@@@std@@Ubig_decimal_fp@detail@v8@fmt@@_WV?$digit_grouping@_W@456@@detail@v8@fmt@@YA?AV?$back_insert_iterator@V?$buffer@_W@detail@v8@fmt@@@std@@V34@AEBUbig_decimal_fp@012@AEBU?$basic_format_specs@_W@12@Ufloat_specs@012@Vlocale_ref@012@@Z@4HA 0000000180043bac f   handles.obj
 0001:00042bac       ?dtor$1@?0???$do_write_float@V?$back_insert_iterator@V?$buffer@_W@detail@v8@fmt@@@std@@U?$decimal_fp@N@dragonbox@detail@v8@fmt@@_WV?$digit_grouping@_W@567@@detail@v8@fmt@@YA?AV?$back_insert_iterator@V?$buffer@_W@detail@v8@fmt@@@std@@V34@AEBU?$decimal_fp@N@dragonbox@012@AEBU?$basic_format_specs@_W@12@Ufloat_specs@012@Vlocale_ref@012@@Z@4HA 0000000180043bac f   handles.obj
 0001:00042bac       ?dtor$1@?0???$do_write_float@V?$back_insert_iterator@V?$buffer@_W@detail@v8@fmt@@@std@@Ubig_decimal_fp@detail@v8@fmt@@_WV?$digit_grouping@_W@456@@detail@v8@fmt@@YA?AV?$back_insert_iterator@V?$buffer@_W@detail@v8@fmt@@@std@@V34@AEBUbig_decimal_fp@012@AEBU?$basic_format_specs@_W@12@Ufloat_specs@012@Vlocale_ref@012@@Z@4HA 0000000180043bac f   handles.obj
 0001:00042bac       ?dtor$2@?0???$do_write_float@V?$back_insert_iterator@V?$buffer@_W@detail@v8@fmt@@@std@@U?$decimal_fp@N@dragonbox@detail@v8@fmt@@_WV?$digit_grouping@_W@567@@detail@v8@fmt@@YA?AV?$back_insert_iterator@V?$buffer@_W@detail@v8@fmt@@@std@@V34@AEBU?$decimal_fp@N@dragonbox@012@AEBU?$basic_format_specs@_W@12@Ufloat_specs@012@Vlocale_ref@012@@Z@4HA 0000000180043bac f   handles.obj
 0001:00042bac       ?dtor$2@?0???$do_write_float@V?$back_insert_iterator@V?$buffer@_W@detail@v8@fmt@@@std@@Ubig_decimal_fp@detail@v8@fmt@@_WV?$digit_grouping@_W@456@@detail@v8@fmt@@YA?AV?$back_insert_iterator@V?$buffer@_W@detail@v8@fmt@@@std@@V34@AEBUbig_decimal_fp@012@AEBU?$basic_format_specs@_W@12@Ufloat_specs@012@Vlocale_ref@012@@Z@4HA 0000000180043bac f   handles.obj
 0001:00042bc0       ?dtor$0@?0???$write_significand@V?$back_insert_iterator@V?$buffer@_W@detail@v8@fmt@@@std@@_WIV?$digit_grouping@_W@detail@v8@fmt@@@detail@v8@fmt@@YA?AV?$back_insert_iterator@V?$buffer@_W@detail@v8@fmt@@@std@@V34@IHH_WAEBV?$digit_grouping@_W@012@@Z@4HA 0000000180043bc0 f   handles.obj
 0001:00042bc0       ?dtor$0@?0???R<lambda_4>@?BO@???$do_write_float@V?$back_insert_iterator@V?$buffer@_W@detail@v8@fmt@@@std@@U?$decimal_fp@N@dragonbox@detail@v8@fmt@@_WV?$digit_grouping@_W@567@@detail@v8@fmt@@YA?AV?$back_insert_iterator@V?$buffer@_W@detail@v8@fmt@@@std@@V45@AEBU?$decimal_fp@N@dragonbox@123@AEBU?$basic_format_specs@_W@23@Ufloat_specs@123@Vlocale_ref@123@@Z@QEBA@0@Z@4HA 0000000180043bc0 f   handles.obj
 0001:00042bc0       ?dtor$0@?0???R<lambda_4>@?BO@???$do_write_float@V?$back_insert_iterator@V?$buffer@_W@detail@v8@fmt@@@std@@Ubig_decimal_fp@detail@v8@fmt@@_WV?$digit_grouping@_W@456@@detail@v8@fmt@@YA?AV?$back_insert_iterator@V?$buffer@_W@detail@v8@fmt@@@std@@V45@AEBUbig_decimal_fp@123@AEBU?$basic_format_specs@_W@23@Ufloat_specs@123@Vlocale_ref@123@@Z@QEBA@0@Z@4HA 0000000180043bc0 f   handles.obj
 0001:00042bd4       ?dtor$0@?0???0?$digit_grouping@_W@detail@v8@fmt@@QEAA@Vlocale_ref@123@_N@Z@4HA 0000000180043bd4 f   handles.obj
 0001:00042be8       ?dtor$0@?0???$write_int_localized@V?$back_insert_iterator@V?$buffer@_W@detail@v8@fmt@@@std@@_K_W@detail@v8@fmt@@YA_NAEAV?$back_insert_iterator@V?$buffer@_W@detail@v8@fmt@@@std@@_KIAEBU?$basic_format_specs@_W@12@Vlocale_ref@012@@Z@4HA 0000000180043be8 f   handles.obj
 0001:00042be8       ?dtor$1@?0???$write_int_localized@V?$back_insert_iterator@V?$buffer@_W@detail@v8@fmt@@@std@@_K_W@detail@v8@fmt@@YA_NAEAV?$back_insert_iterator@V?$buffer@_W@detail@v8@fmt@@@std@@_KIAEBU?$basic_format_specs@_W@12@Vlocale_ref@012@@Z@4HA 0000000180043be8 f   handles.obj
 0001:00042bfc       ?dtor$0@?0???$write_significand@_WV?$back_insert_iterator@V?$buffer@_W@detail@v8@fmt@@@std@@PEBDV?$digit_grouping@_W@detail@v8@fmt@@@detail@v8@fmt@@YA?AV?$back_insert_iterator@V?$buffer@_W@detail@v8@fmt@@@std@@V34@PEBDHHAEBV?$digit_grouping@_W@012@@Z@4HA 0000000180043bfc f   handles.obj
 0001:00042c10       ?dtor$0@?0???$apply@V?$back_insert_iterator@V?$buffer@_W@detail@v8@fmt@@@std@@D@?$digit_grouping@_W@detail@v8@fmt@@QEBA?AV?$back_insert_iterator@V?$buffer@_W@detail@v8@fmt@@@std@@V45@V?$basic_string_view@D@23@@Z@4HA 0000000180043c10 f   handles.obj
 0001:00042c10       ?dtor$0@?0???$apply@V?$back_insert_iterator@V?$buffer@_W@detail@v8@fmt@@@std@@_W@?$digit_grouping@_W@detail@v8@fmt@@QEBA?AV?$back_insert_iterator@V?$buffer@_W@detail@v8@fmt@@@std@@V45@V?$basic_string_view@_W@23@@Z@4HA 0000000180043c10 f   handles.obj
 0001:00042c24       ?dtor$0@?0??Config@@YAHXZ@4HA 0000000180043c24 f   Pcfg.obj
 0001:00042c38       ?dtor$0@?0??Write@options@@QEBAXXZ@4HA 0000000180043c38 f   Pcfg.obj
 0001:00042c4c       ?dtor$0@?0??Read@options@@QEAAXXZ@4HA 0000000180043c4c f   Pcfg.obj
 0001:00042c60       ?dtor$0@?0??ui64toa_width@@YA?AV?$basic_string@_WU?$char_traits@_W@std@@V?$allocator@_W@2@@std@@_KI_N@Z@4HA 0000000180043c60 f   Pclass.obj
 0001:00042c74       ?dtor$0@?0??PrintTitle@@YA?AV?$basic_string@_WU?$char_traits@_W@std@@V?$allocator@_W@2@@std@@V?$basic_string_view@_WU?$char_traits@_W@std@@@2@@Z@4HA 0000000180043c74 f   Pclass.obj
 0001:00042c88       ?dtor$0@?0???0Plist@@QEAA@XZ@4HA 0000000180043c88 f   Pclass.obj
 0001:00042ca0       ?dtor$1@?0???0Plist@@QEAA@XZ@4HA 0000000180043ca0 f   Pclass.obj
 0001:00042cb8       ?dtor$2@?0???0Plist@@QEAA@XZ@4HA 0000000180043cb8 f   Pclass.obj
 0001:00042cd0       ?dtor$3@?0???0Plist@@QEAA@XZ@4HA 0000000180043cd0 f   Pclass.obj
 0001:00042ce4       ?dtor$10@?0???0Plist@@QEAA@XZ@4HA 0000000180043ce4 f   Pclass.obj
 0001:00042cfc       ?dtor$0@?0??TranslateMode@@YA_NAEBV?$basic_string@_WU?$char_traits@_W@std@@V?$allocator@_W@2@@std@@AEAV12@@Z@4HA 0000000180043cfc f   Pclass.obj
 0001:00042cfc       ?dtor$0@?0??window_ex_style@@YA@PEAUHWND__@@@Z@4HA 0000000180043cfc f   Pclass.obj
 0001:00042cfc       ?dtor$0@?0??window_style@@YA@PEAUHWND__@@@Z@4HA 0000000180043cfc f   Pclass.obj
 0001:00042d10       ?dtor$0@?0??InitializePanelModes@Plist@@SAXXZ@4HA 0000000180043d10 f   Pclass.obj
 0001:00042d10       ?dtor$91@?0??InitializePanelModes@Plist@@SAXXZ@4HA 0000000180043d10 f   Pclass.obj
 0001:00042d24       ?dtor$8@?0??InitializePanelModes@Plist@@SAXXZ@4HA 0000000180043d24 f   Pclass.obj
 0001:00042d24       ?dtor$99@?0??InitializePanelModes@Plist@@SAXXZ@4HA 0000000180043d24 f   Pclass.obj
 0001:00042d38       ?dtor$100@?0??InitializePanelModes@Plist@@SAXXZ@4HA 0000000180043d38 f   Pclass.obj
 0001:00042d38       ?dtor$9@?0??InitializePanelModes@Plist@@SAXXZ@4HA 0000000180043d38 f   Pclass.obj
 0001:00042d4c       ?dtor$108@?0??InitializePanelModes@Plist@@SAXXZ@4HA 0000000180043d4c f   Pclass.obj
 0001:00042d4c       ?dtor$17@?0??InitializePanelModes@Plist@@SAXXZ@4HA 0000000180043d4c f   Pclass.obj
 0001:00042d60       ?dtor$109@?0??InitializePanelModes@Plist@@SAXXZ@4HA 0000000180043d60 f   Pclass.obj
 0001:00042d60       ?dtor$18@?0??InitializePanelModes@Plist@@SAXXZ@4HA 0000000180043d60 f   Pclass.obj
 0001:00042d74       ?dtor$117@?0??InitializePanelModes@Plist@@SAXXZ@4HA 0000000180043d74 f   Pclass.obj
 0001:00042d74       ?dtor$26@?0??InitializePanelModes@Plist@@SAXXZ@4HA 0000000180043d74 f   Pclass.obj
 0001:00042d88       ?dtor$118@?0??InitializePanelModes@Plist@@SAXXZ@4HA 0000000180043d88 f   Pclass.obj
 0001:00042d88       ?dtor$27@?0??InitializePanelModes@Plist@@SAXXZ@4HA 0000000180043d88 f   Pclass.obj
 0001:00042d9c       ?dtor$126@?0??InitializePanelModes@Plist@@SAXXZ@4HA 0000000180043d9c f   Pclass.obj
 0001:00042d9c       ?dtor$35@?0??InitializePanelModes@Plist@@SAXXZ@4HA 0000000180043d9c f   Pclass.obj
 0001:00042db0       ?dtor$127@?0??InitializePanelModes@Plist@@SAXXZ@4HA 0000000180043db0 f   Pclass.obj
 0001:00042db0       ?dtor$36@?0??InitializePanelModes@Plist@@SAXXZ@4HA 0000000180043db0 f   Pclass.obj
 0001:00042dc4       ?dtor$135@?0??InitializePanelModes@Plist@@SAXXZ@4HA 0000000180043dc4 f   Pclass.obj
 0001:00042dc4       ?dtor$44@?0??InitializePanelModes@Plist@@SAXXZ@4HA 0000000180043dc4 f   Pclass.obj
 0001:00042dd8       ?dtor$136@?0??InitializePanelModes@Plist@@SAXXZ@4HA 0000000180043dd8 f   Pclass.obj
 0001:00042dd8       ?dtor$45@?0??InitializePanelModes@Plist@@SAXXZ@4HA 0000000180043dd8 f   Pclass.obj
 0001:00042dec       ?dtor$144@?0??InitializePanelModes@Plist@@SAXXZ@4HA 0000000180043dec f   Pclass.obj
 0001:00042dec       ?dtor$53@?0??InitializePanelModes@Plist@@SAXXZ@4HA 0000000180043dec f   Pclass.obj
 0001:00042e00       ?dtor$145@?0??InitializePanelModes@Plist@@SAXXZ@4HA 0000000180043e00 f   Pclass.obj
 0001:00042e00       ?dtor$54@?0??InitializePanelModes@Plist@@SAXXZ@4HA 0000000180043e00 f   Pclass.obj
 0001:00042e14       ?dtor$153@?0??InitializePanelModes@Plist@@SAXXZ@4HA 0000000180043e14 f   Pclass.obj
 0001:00042e14       ?dtor$62@?0??InitializePanelModes@Plist@@SAXXZ@4HA 0000000180043e14 f   Pclass.obj
 0001:00042e28       ?dtor$154@?0??InitializePanelModes@Plist@@SAXXZ@4HA 0000000180043e28 f   Pclass.obj
 0001:00042e28       ?dtor$63@?0??InitializePanelModes@Plist@@SAXXZ@4HA 0000000180043e28 f   Pclass.obj
 0001:00042e3c       ?dtor$162@?0??InitializePanelModes@Plist@@SAXXZ@4HA 0000000180043e3c f   Pclass.obj
 0001:00042e3c       ?dtor$71@?0??InitializePanelModes@Plist@@SAXXZ@4HA 0000000180043e3c f   Pclass.obj
 0001:00042e50       ?dtor$163@?0??InitializePanelModes@Plist@@SAXXZ@4HA 0000000180043e50 f   Pclass.obj
 0001:00042e50       ?dtor$72@?0??InitializePanelModes@Plist@@SAXXZ@4HA 0000000180043e50 f   Pclass.obj
 0001:00042e64       ?dtor$171@?0??InitializePanelModes@Plist@@SAXXZ@4HA 0000000180043e64 f   Pclass.obj
 0001:00042e64       ?dtor$80@?0??InitializePanelModes@Plist@@SAXXZ@4HA 0000000180043e64 f   Pclass.obj
 0001:00042e78       ?dtor$172@?0??InitializePanelModes@Plist@@SAXXZ@4HA 0000000180043e78 f   Pclass.obj
 0001:00042e78       ?dtor$81@?0??InitializePanelModes@Plist@@SAXXZ@4HA 0000000180043e78 f   Pclass.obj
 0001:00042e8c       ?dtor$181@?0??InitializePanelModes@Plist@@SAXXZ@4HA 0000000180043e8c f   Pclass.obj
 0001:00042e8c       ?dtor$90@?0??InitializePanelModes@Plist@@SAXXZ@4HA 0000000180043e8c f   Pclass.obj
 0001:00042eb0       ?dtor$182@?0??InitializePanelModes@Plist@@SAXXZ@4HA 0000000180043eb0 f   Pclass.obj
 0001:00042ec4       ?dtor$183@?0??InitializePanelModes@Plist@@SAXXZ@4HA 0000000180043ec4 f   Pclass.obj
 0001:00042ed8       ?dtor$0@?0??SavePanelModes@Plist@@SAXXZ@4HA 0000000180043ed8 f   Pclass.obj
 0001:00042eec       ?dtor$1@?0??SavePanelModes@Plist@@SAXXZ@4HA 0000000180043eec f   Pclass.obj
 0001:00042f00       ?dtor$0@?0??generate_titles@@YAXAEBV?$basic_string@_WU?$char_traits@_W@std@@V?$allocator@_W@2@@std@@AEAUPanelMode@@@Z@4HA 0000000180043f00 f   Pclass.obj
 0001:00042f14       ?dtor$0@?0??GetOpenPanelInfo@Plist@@QEAAXPEAUOpenPanelInfo@@@Z@4HA 0000000180043f14 f   Pclass.obj
 0001:00042f28       ?dtor$0@?0??GetFindData@Plist@@QEAAHAEAPEAUPluginPanelItem@@AEA_K_K@Z@4HA 0000000180043f28 f   Pclass.obj
 0001:00042f3c       ?dtor$1@?0??GetFindData@Plist@@QEAAHAEAPEAUPluginPanelItem@@AEA_K_K@Z@4HA 0000000180043f3c f   Pclass.obj
 0001:00042f50       ?dtor$2@?0??GetFindData@Plist@@QEAAHAEAPEAUPluginPanelItem@@AEA_K_K@Z@4HA 0000000180043f50 f   Pclass.obj
 0001:00042f64       ?dtor$3@?0??GetFindData@Plist@@QEAAHAEAPEAUPluginPanelItem@@AEA_K_K@Z@4HA 0000000180043f64 f   Pclass.obj
 0001:00042f78       ?dtor$4@?0??GetFindData@Plist@@QEAAHAEAPEAUPluginPanelItem@@AEA_K_K@Z@4HA 0000000180043f78 f   Pclass.obj
 0001:00042f8c       ?dtor$5@?0??GetFindData@Plist@@QEAAHAEAPEAUPluginPanelItem@@AEA_K_K@Z@4HA 0000000180043f8c f   Pclass.obj
 0001:00042f8c       ?dtor$7@?0??GetFindData@Plist@@QEAAHAEAPEAUPluginPanelItem@@AEA_K_K@Z@4HA 0000000180043f8c f   Pclass.obj
 0001:00042fa0       ?dtor$6@?0??GetFindData@Plist@@QEAAHAEAPEAUPluginPanelItem@@AEA_K_K@Z@4HA 0000000180043fa0 f   Pclass.obj
 0001:00042fb4       ?dtor$8@?0??GetFindData@Plist@@QEAAHAEAPEAUPluginPanelItem@@AEA_K_K@Z@4HA 0000000180043fb4 f   Pclass.obj
 0001:00042fc8       ?dtor$13@?0??GetFindData@Plist@@QEAAHAEAPEAUPluginPanelItem@@AEA_K_K@Z@4HA 0000000180043fc8 f   Pclass.obj
 0001:00042fe0       ?dtor$14@?0??GetFindData@Plist@@QEAAHAEAPEAUPluginPanelItem@@AEA_K_K@Z@4HA 0000000180043fe0 f   Pclass.obj
 0001:00042ff8       ?dtor$0@?0??DumpNTCounters@@YAXPEAXAEAVPerfThread@@KK@Z@4HA 0000000180043ff8 f   Pclass.obj
 0001:0004300c       ?dtor$3@?0??DumpNTCounters@@YAXPEAXAEAVPerfThread@@KK@Z@4HA 000000018004400c f   Pclass.obj
 0001:00043020       ?dtor$6@?0??DumpNTCounters@@YAXPEAXAEAVPerfThread@@KK@Z@4HA 0000000180044020 f   Pclass.obj
 0001:00043034       ?dtor$0@?0??GetFiles@Plist@@QEAAHPEAUPluginPanelItem@@_KHPEAPEB_W1AEAUoptions@@@Z@4HA 0000000180044034 f   Pclass.obj
 0001:00043048       ?dtor$1@?0??GetFiles@Plist@@QEAAHPEAUPluginPanelItem@@_KHPEAPEB_W1AEAUoptions@@@Z@4HA 0000000180044048 f   Pclass.obj
 0001:0004305c       ?dtor$2@?0??GetFiles@Plist@@QEAAHPEAUPluginPanelItem@@_KHPEAPEB_W1AEAUoptions@@@Z@4HA 000000018004405c f   Pclass.obj
 0001:00043070       ?dtor$3@?0??GetFiles@Plist@@QEAAHPEAUPluginPanelItem@@_KHPEAPEB_W1AEAUoptions@@@Z@4HA 0000000180044070 f   Pclass.obj
 0001:00043084       ?dtor$14@?0??GetFiles@Plist@@QEAAHPEAUPluginPanelItem@@_KHPEAPEB_W1AEAUoptions@@@Z@4HA 0000000180044084 f   Pclass.obj
 0001:00043084       ?dtor$16@?0??GetFiles@Plist@@QEAAHPEAUPluginPanelItem@@_KHPEAPEB_W1AEAUoptions@@@Z@4HA 0000000180044084 f   Pclass.obj
 0001:00043084       ?dtor$18@?0??GetFiles@Plist@@QEAAHPEAUPluginPanelItem@@_KHPEAPEB_W1AEAUoptions@@@Z@4HA 0000000180044084 f   Pclass.obj
 0001:00043084       ?dtor$20@?0??GetFiles@Plist@@QEAAHPEAUPluginPanelItem@@_KHPEAPEB_W1AEAUoptions@@@Z@4HA 0000000180044084 f   Pclass.obj
 0001:00043084       ?dtor$22@?0??GetFiles@Plist@@QEAAHPEAUPluginPanelItem@@_KHPEAPEB_W1AEAUoptions@@@Z@4HA 0000000180044084 f   Pclass.obj
 0001:00043084       ?dtor$29@?0??GetFiles@Plist@@QEAAHPEAUPluginPanelItem@@_KHPEAPEB_W1AEAUoptions@@@Z@4HA 0000000180044084 f   Pclass.obj
 0001:00043084       ?dtor$31@?0??GetFiles@Plist@@QEAAHPEAUPluginPanelItem@@_KHPEAPEB_W1AEAUoptions@@@Z@4HA 0000000180044084 f   Pclass.obj
 0001:00043084       ?dtor$33@?0??GetFiles@Plist@@QEAAHPEAUPluginPanelItem@@_KHPEAPEB_W1AEAUoptions@@@Z@4HA 0000000180044084 f   Pclass.obj
 0001:00043084       ?dtor$35@?0??GetFiles@Plist@@QEAAHPEAUPluginPanelItem@@_KHPEAPEB_W1AEAUoptions@@@Z@4HA 0000000180044084 f   Pclass.obj
 0001:00043084       ?dtor$38@?0??GetFiles@Plist@@QEAAHPEAUPluginPanelItem@@_KHPEAPEB_W1AEAUoptions@@@Z@4HA 0000000180044084 f   Pclass.obj
 0001:00043084       ?dtor$41@?0??GetFiles@Plist@@QEAAHPEAUPluginPanelItem@@_KHPEAPEB_W1AEAUoptions@@@Z@4HA 0000000180044084 f   Pclass.obj
 0001:00043084       ?dtor$4@?0??GetFiles@Plist@@QEAAHPEAUPluginPanelItem@@_KHPEAPEB_W1AEAUoptions@@@Z@4HA 0000000180044084 f   Pclass.obj
 0001:00043084       ?dtor$6@?0??GetFiles@Plist@@QEAAHPEAUPluginPanelItem@@_KHPEAPEB_W1AEAUoptions@@@Z@4HA 0000000180044084 f   Pclass.obj
 0001:00043084       ?dtor$8@?0??GetFiles@Plist@@QEAAHPEAUPluginPanelItem@@_KHPEAPEB_W1AEAUoptions@@@Z@4HA 0000000180044084 f   Pclass.obj
 0001:00043098       ?dtor$11@?0??GetFiles@Plist@@QEAAHPEAUPluginPanelItem@@_KHPEAPEB_W1AEAUoptions@@@Z@4HA 0000000180044098 f   Pclass.obj
 0001:00043098       ?dtor$1@?0??RefreshWMIData@PerfThread@@AEAAXXZ@4HA 0000000180044098 f   perfthread.obj
 0001:000430ac       ?dtor$23@?0??GetFiles@Plist@@QEAAHPEAUPluginPanelItem@@_KHPEAPEB_W1AEAUoptions@@@Z@4HA 00000001800440ac f   Pclass.obj
 0001:000430ac       ?dtor$64@?0??GetFiles@Plist@@QEAAHPEAUPluginPanelItem@@_KHPEAPEB_W1AEAUoptions@@@Z@4HA 00000001800440ac f   Pclass.obj
 0001:000430c0       ?dtor$26@?0??GetFiles@Plist@@QEAAHPEAUPluginPanelItem@@_KHPEAPEB_W1AEAUoptions@@@Z@4HA 00000001800440c0 f   Pclass.obj
 0001:000430d4       ?dtor$27@?0??GetFiles@Plist@@QEAAHPEAUPluginPanelItem@@_KHPEAPEB_W1AEAUoptions@@@Z@4HA 00000001800440d4 f   Pclass.obj
 0001:000430e8       ?dtor$28@?0??GetFiles@Plist@@QEAAHPEAUPluginPanelItem@@_KHPEAPEB_W1AEAUoptions@@@Z@4HA 00000001800440e8 f   Pclass.obj
 0001:000430fc       ?dtor$37@?0??GetFiles@Plist@@QEAAHPEAUPluginPanelItem@@_KHPEAPEB_W1AEAUoptions@@@Z@4HA 00000001800440fc f   Pclass.obj
 0001:00043110       ?dtor$40@?0??GetFiles@Plist@@QEAAHPEAUPluginPanelItem@@_KHPEAPEB_W1AEAUoptions@@@Z@4HA 0000000180044110 f   Pclass.obj
 0001:00043124       ?dtor$76@?0??GetFiles@Plist@@QEAAHPEAUPluginPanelItem@@_KHPEAPEB_W1AEAUoptions@@@Z@4HA 0000000180044124 f   Pclass.obj
 0001:00043138       ?dtor$0@?0??DeleteFiles@Plist@@QEAAHPEAUPluginPanelItem@@_K1@Z@4HA 0000000180044138 f   Pclass.obj
 0001:0004314c       ?dtor$1@?0??DeleteFiles@Plist@@QEAAHPEAUPluginPanelItem@@_K1@Z@4HA 000000018004414c f   Pclass.obj
 0001:0004314c       ?dtor$4@?0??DeleteFiles@Plist@@QEAAHPEAUPluginPanelItem@@_K1@Z@4HA 000000018004414c f   Pclass.obj
 0001:00043160       ?dtor$1@?0??Connect@Plist@@QEAA_NPEB_W00@Z@4HA 0000000180044160 f   Pclass.obj
 0001:00043174       ?dtor$6@?0??Connect@Plist@@QEAA_NPEB_W00@Z@4HA 0000000180044174 f   Pclass.obj
 0001:0004318c       ?dtor$0@?0??ProcessKey@Plist@@QEAAHPEBU_INPUT_RECORD@@@Z@4HA 000000018004418c f   Pclass.obj
 0001:000431a8       ?dtor$11@?0??ProcessKey@Plist@@QEAAHPEBU_INPUT_RECORD@@@Z@4HA 00000001800441a8 f   Pclass.obj
 0001:000431a8       ?dtor$1@?0??ProcessKey@Plist@@QEAAHPEBU_INPUT_RECORD@@@Z@4HA 00000001800441a8 f   Pclass.obj
 0001:000431a8       ?dtor$2@?0??ProcessKey@Plist@@QEAAHPEBU_INPUT_RECORD@@@Z@4HA 00000001800441a8 f   Pclass.obj
 0001:000431a8       ?dtor$4@?0??ProcessKey@Plist@@QEAAHPEBU_INPUT_RECORD@@@Z@4HA 00000001800441a8 f   Pclass.obj
 0001:000431a8       ?dtor$9@?0??ProcessKey@Plist@@QEAAHPEBU_INPUT_RECORD@@@Z@4HA 00000001800441a8 f   Pclass.obj
 0001:000431c4       ?dtor$3@?0??ProcessKey@Plist@@QEAAHPEBU_INPUT_RECORD@@@Z@4HA 00000001800441c4 f   Pclass.obj
 0001:000431e0       ?dtor$5@?0??ProcessKey@Plist@@QEAAHPEBU_INPUT_RECORD@@@Z@4HA 00000001800441e0 f   Pclass.obj
 0001:000431fc       ?dtor$8@?0??ProcessKey@Plist@@QEAAHPEBU_INPUT_RECORD@@@Z@4HA 00000001800441fc f   Pclass.obj
 0001:00043218       ?dtor$10@?0??ProcessKey@Plist@@QEAAHPEBU_INPUT_RECORD@@@Z@4HA 0000000180044218 f   Pclass.obj
 0001:00043234       ?dtor$12@?0??ProcessKey@Plist@@QEAAHPEBU_INPUT_RECORD@@@Z@4HA 0000000180044234 f   Pclass.obj
 0001:00043250       ?dtor$13@?0??ProcessKey@Plist@@QEAAHPEBU_INPUT_RECORD@@@Z@4HA 0000000180044250 f   Pclass.obj
 0001:0004326c       ?dtor$14@?0??ProcessKey@Plist@@QEAAHPEBU_INPUT_RECORD@@@Z@4HA 000000018004426c f   Pclass.obj
 0001:00043288       ?dtor$15@?0??ProcessKey@Plist@@QEAAHPEBU_INPUT_RECORD@@@Z@4HA 0000000180044288 f   Pclass.obj
 0001:000432c0       ?dtor$16@?0??ProcessKey@Plist@@QEAAHPEBU_INPUT_RECORD@@@Z@4HA 00000001800442c0 f   Pclass.obj
 0001:000432f8       ?dtor$228@?0??ProcessKey@Plist@@QEAAHPEBU_INPUT_RECORD@@@Z@4HA 00000001800442f8 f   Pclass.obj
 0001:000432f8       ?dtor$230@?0??ProcessKey@Plist@@QEAAHPEBU_INPUT_RECORD@@@Z@4HA 00000001800442f8 f   Pclass.obj
 0001:00043318       ?dtor$233@?0??ProcessKey@Plist@@QEAAHPEBU_INPUT_RECORD@@@Z@4HA 0000000180044318 f   Pclass.obj
 0001:00043334       ?dtor$235@?0??ProcessKey@Plist@@QEAAHPEBU_INPUT_RECORD@@@Z@4HA 0000000180044334 f   Pclass.obj
 0001:00043350       ?dtor$1@?0??GetVersionInfo@Plist@@SA_NPEB_WAEAV?$unique_ptr@$$BY0A@DU?$default_delete@$$BY0A@D@std@@@std@@AEAPEB_W2@Z@4HA 0000000180044350 f   Pclass.obj
 0001:00043364       ?dtor$2@?0??GetVersionInfo@Plist@@SA_NPEB_WAEAV?$unique_ptr@$$BY0A@DU?$default_delete@$$BY0A@D@std@@@std@@AEAPEB_W2@Z@4HA 0000000180044364 f   Pclass.obj
 0001:00043364       ?dtor$4@?0??GetVersionInfo@Plist@@SA_NPEB_WAEAV?$unique_ptr@$$BY0A@DU?$default_delete@$$BY0A@D@std@@@std@@AEAPEB_W2@Z@4HA 0000000180044364 f   Pclass.obj
 0001:00043378       ?dtor$0@?0??PrintVersionInfo@Plist@@CAXPEAXPEB_W@Z@4HA 0000000180044378 f   Pclass.obj
 0001:0004338c       ?dtor$1@?0??PrintVersionInfo@Plist@@CAXPEAXPEB_W@Z@4HA 000000018004438c f   Pclass.obj
 0001:0004338c       ?dtor$3@?0??PrintVersionInfo@Plist@@CAXPEAXPEB_W@Z@4HA 000000018004438c f   Pclass.obj
 0001:0004338c       ?dtor$0@?0??PrintNTCurDirAndEnv@@YAXPEAX0H@Z@4HA 000000018004438c f   Plist.obj
 0001:000433a0       ?dtor$6@?0??PrintVersionInfo@Plist@@CAXPEAXPEB_W@Z@4HA 00000001800443a0 f   Pclass.obj
 0001:000433b4       ?dtor$18@?0??PrintVersionInfo@Plist@@CAXPEAXPEB_W@Z@4HA 00000001800443b4 f   Pclass.obj
 0001:000433b4       ?dtor$1@?0??PrintNTCurDirAndEnv@@YAXPEAX0H@Z@4HA 00000001800443b4 f   Plist.obj
 0001:000433b4       ?dtor$5@?0??GetProcessOwner@WMIConnection@@QEAA?AV?$basic_string@_WU?$char_traits@_W@std@@V?$allocator@_W@2@@std@@KPEAV23@@Z@4HA 00000001800443b4 f   wmi.obj
 0001:000433b4       ?dtor$5@?0??GetProcessUserSid@WMIConnection@@QEAA?AV?$basic_string@_WU?$char_traits@_W@std@@V?$allocator@_W@2@@std@@K@Z@4HA 00000001800443b4 f   wmi.obj
 0001:000433c8       ?dtor$0@?0??PrintOwnerInfo@Plist@@AEAAXPEAXK@Z@4HA 00000001800443c8 f   Pclass.obj
 0001:000433dc       ?dtor$1@?0??PrintOwnerInfo@Plist@@AEAAXPEAXK@Z@4HA 00000001800443dc f   Pclass.obj
 0001:000433f0       ?dtor$2@?0??PrintOwnerInfo@Plist@@AEAAXPEAXK@Z@4HA 00000001800443f0 f   Pclass.obj
 0001:00043404       ?dtor$6@?0??PrintOwnerInfo@Plist@@AEAAXPEAXK@Z@4HA 0000000180044404 f   Pclass.obj
 0001:00043418       ?dtor$13@?0??PrintOwnerInfo@Plist@@AEAAXPEAXK@Z@4HA 0000000180044418 f   Pclass.obj
 0001:0004342c       ?dtor$28@?0??PrintOwnerInfo@Plist@@AEAAXPEAXK@Z@4HA 000000018004442c f   Pclass.obj
 0001:00043440       ?dtor$0@?0??Compare@Plist@@QEBAHPEBUPluginPanelItem@@0I@Z@4HA 0000000180044440 f   Pclass.obj
 0001:00043454       ?dtor$1@?0??Compare@Plist@@QEBAHPEBUPluginPanelItem@@0I@Z@4HA 0000000180044454 f   Pclass.obj
 0001:00043468       ?dtor$0@?0???$_Try_emplace@AEBK$$V@?$_Hash@V?$_Umap_traits@KPEAUHWND__@@V?$_Uhash_compare@KU?$hash@K@std@@U?$equal_to@K@2@@std@@V?$allocator@U?$pair@$$CBKPEAUHWND__@@@std@@@3@$0A@@std@@@std@@IEAA?AU?$pair@PEAU?$_List_node@U?$pair@$$CBKPEAUHWND__@@@std@@PEAX@std@@_N@1@AEBK@Z@4HA 0000000180044468 f   Pclass.obj
 0001:00043468       ?dtor$1@?0???$_Try_emplace@AEBK$$V@?$_Hash@V?$_Umap_traits@KPEAUHWND__@@V?$_Uhash_compare@KU?$hash@K@std@@U?$equal_to@K@2@@std@@V?$allocator@U?$pair@$$CBKPEAUHWND__@@@std@@@3@$0A@@std@@@std@@IEAA?AU?$pair@PEAU?$_List_node@U?$pair@$$CBKPEAUHWND__@@@std@@PEAX@std@@_N@1@AEBK@Z@4HA 0000000180044468 f   Pclass.obj
 0001:0004347c       ?dtor$0@?0???$_Uninitialized_copy@PEBUmode@@V?$allocator@Umode@@@std@@@std@@YAPEAUmode@@QEBU1@0PEAU1@AEAV?$allocator@Umode@@@0@@Z@4HA 000000018004447c f   Pclass.obj
 0001:00043490       ?dtor$21@?0???$_Uninitialized_copy@PEBUmode@@V?$allocator@Umode@@@std@@@std@@YAPEAUmode@@QEBU1@0PEAU1@AEAV?$allocator@Umode@@@0@@Z@4HA 0000000180044490 f   Pclass.obj
 0001:000434a4       ?dtor$23@?0???$_Uninitialized_copy@PEBUmode@@V?$allocator@Umode@@@std@@@std@@YAPEAUmode@@QEBU1@0PEAU1@AEAV?$allocator@Umode@@@0@@Z@4HA 00000001800444a4 f   Pclass.obj
 0001:000434a4       ?dtor$32@?0???$_Uninitialized_copy@PEBUmode@@V?$allocator@Umode@@@std@@@std@@YAPEAUmode@@QEBU1@0PEAU1@AEAV?$allocator@Umode@@@0@@Z@4HA 00000001800444a4 f   Pclass.obj
 0001:000434b8       ?dtor$24@?0???$_Uninitialized_copy@PEBUmode@@V?$allocator@Umode@@@std@@@std@@YAPEAUmode@@QEBU1@0PEAU1@AEAV?$allocator@Umode@@@0@@Z@4HA 00000001800444b8 f   Pclass.obj
 0001:000434b8       ?dtor$33@?0???$_Uninitialized_copy@PEBUmode@@V?$allocator@Umode@@@std@@@std@@YAPEAUmode@@QEBU1@0PEAU1@AEAV?$allocator@Umode@@@0@@Z@4HA 00000001800444b8 f   Pclass.obj
 0001:000434d0       ?dtor$0@?0???0PerfThread@@QEAA@PEAVPlist@@PEB_W11@Z@4HA 00000001800444d0 f   perfthread.obj
 0001:000434e8       ?dtor$1@?0???0PerfThread@@QEAA@PEAVPlist@@PEB_W11@Z@4HA 00000001800444e8 f   perfthread.obj
 0001:00043500       ?dtor$2@?0???0PerfThread@@QEAA@PEAVPlist@@PEB_W11@Z@4HA 0000000180044500 f   perfthread.obj
 0001:00043518       ?dtor$3@?0???0PerfThread@@QEAA@PEAVPlist@@PEB_W11@Z@4HA 0000000180044518 f   perfthread.obj
 0001:00043530       ?dtor$4@?0???0PerfThread@@QEAA@PEAVPlist@@PEB_W11@Z@4HA 0000000180044530 f   perfthread.obj
 0001:00043548       ?dtor$5@?0???0PerfThread@@QEAA@PEAVPlist@@PEB_W11@Z@4HA 0000000180044548 f   perfthread.obj
 0001:00043560       ?dtor$6@?0???0PerfThread@@QEAA@PEAVPlist@@PEB_W11@Z@4HA 0000000180044560 f   perfthread.obj
 0001:00043578       ?dtor$7@?0???0PerfThread@@QEAA@PEAVPlist@@PEB_W11@Z@4HA 0000000180044578 f   perfthread.obj
 0001:00043590       ?dtor$8@?0???0PerfThread@@QEAA@PEAVPlist@@PEB_W11@Z@4HA 0000000180044590 f   perfthread.obj
 0001:000435a8       ?dtor$9@?0???0PerfThread@@QEAA@PEAVPlist@@PEB_W11@Z@4HA 00000001800445a8 f   perfthread.obj
 0001:000435c0       ?dtor$10@?0???0PerfThread@@QEAA@PEAVPlist@@PEB_W11@Z@4HA 00000001800445c0 f   perfthread.obj
 0001:000435d8       ?dtor$11@?0???0PerfThread@@QEAA@PEAVPlist@@PEB_W11@Z@4HA 00000001800445d8 f   perfthread.obj
 0001:000435f0       ?dtor$12@?0???0PerfThread@@QEAA@PEAVPlist@@PEB_W11@Z@4HA 00000001800445f0 f   perfthread.obj
 0001:00043604       ?dtor$13@?0???0PerfThread@@QEAA@PEAVPlist@@PEB_W11@Z@4HA 0000000180044604 f   perfthread.obj
 0001:00043618       ?dtor$0@?0??Refresh@PerfThread@@AEAAXXZ@4HA 0000000180044618 f   perfthread.obj
 0001:0004362c       ?dtor$1@?0??Refresh@PerfThread@@AEAAXXZ@4HA 000000018004462c f   perfthread.obj
 0001:00043640       ?dtor$2@?0??Refresh@PerfThread@@AEAAXXZ@4HA 0000000180044640 f   perfthread.obj
 0001:00043654       ?dtor$7@?0??Refresh@PerfThread@@AEAAXXZ@4HA 0000000180044654 f   perfthread.obj
 0001:00043668       ?dtor$11@?0??Refresh@PerfThread@@AEAAXXZ@4HA 0000000180044668 f   perfthread.obj
 0001:0004367c       ?dtor$17@?0??Refresh@PerfThread@@AEAAXXZ@4HA 000000018004467c f   perfthread.obj
 0001:00043694       ?dtor$18@?0??Refresh@PerfThread@@AEAAXXZ@4HA 0000000180044694 f   perfthread.obj
 0001:000436ac       ?dtor$0@?0??RefreshWMIData@PerfThread@@AEAAXXZ@4HA 00000001800446ac f   perfthread.obj
 0001:000436c0       ?dtor$4@?0??RefreshWMIData@PerfThread@@AEAAXXZ@4HA 00000001800446c0 f   perfthread.obj
 0001:000436d4       ?dtor$8@?0??RefreshWMIData@PerfThread@@AEAAXXZ@4HA 00000001800446d4 f   perfthread.obj
 0001:00043704       ?dtor$9@?0??RefreshWMIData@PerfThread@@AEAAXXZ@4HA 0000000180044704 f   perfthread.obj
 0001:00043718       ?dtor$21@?0??RefreshWMIData@PerfThread@@AEAAXXZ@4HA 0000000180044718 f   perfthread.obj
 0001:0004372c       ?dtor$28@?0??RefreshWMIData@PerfThread@@AEAAXXZ@4HA 000000018004472c f   perfthread.obj
 0001:0004375c       ?dtor$29@?0??RefreshWMIData@PerfThread@@AEAAXXZ@4HA 000000018004475c f   perfthread.obj
 0001:00043770       ?dtor$1@?0???0?$unordered_multimap@KUProcessPerfData@@U?$hash@K@std@@U?$equal_to@K@3@V?$allocator@U?$pair@$$CBKUProcessPerfData@@@std@@@3@@std@@QEAA@XZ@4HA 0000000180044770 f   perfthread.obj
 0001:00043788       ?dtor$2@?0???0?$unordered_multimap@KUProcessPerfData@@U?$hash@K@std@@U?$equal_to@K@3@V?$allocator@U?$pair@$$CBKUProcessPerfData@@@std@@@3@@std@@QEAA@XZ@4HA 0000000180044788 f   perfthread.obj
 0001:000437a0       ?dtor$0@?0???$insert@V?$_List_unchecked_const_iterator@V?$_List_val@U?$_List_simple_types@U?$pair@$$CBKUProcessPerfData@@@std@@@std@@@std@@U_Iterator_base0@2@@std@@@?$_Hash@V?$_Umap_traits@KUProcessPerfData@@V?$_Uhash_compare@KU?$hash@K@std@@U?$equal_to@K@2@@std@@V?$allocator@U?$pair@$$CBKUProcessPerfData@@@std@@@3@$00@std@@@std@@QEAAXV?$_List_unchecked_const_iterator@V?$_List_val@U?$_List_simple_types@U?$pair@$$CBKUProcessPerfData@@@std@@@std@@@std@@U_Iterator_base0@2@@1@0@Z@4HA 00000001800447a0 f   Plist.obj
 0001:000437a0       ?dtor$0@?0???$emplace@AEBKUProcessPerfData@@@?$_Hash@V?$_Umap_traits@KUProcessPerfData@@V?$_Uhash_compare@KU?$hash@K@std@@U?$equal_to@K@2@@std@@V?$allocator@U?$pair@$$CBKUProcessPerfData@@@std@@@3@$00@std@@@std@@QEAA?AV?$_List_iterator@V?$_List_val@U?$_List_simple_types@U?$pair@$$CBKUProcessPerfData@@@std@@@std@@@std@@@1@AEBK$$QEAUProcessPerfData@@@Z@4HA 00000001800447a0 f   perfthread.obj
 0001:000437b4       ?dtor$1@?0???$insert@V?$_List_unchecked_const_iterator@V?$_List_val@U?$_List_simple_types@U?$pair@$$CBKUProcessPerfData@@@std@@@std@@@std@@U_Iterator_base0@2@@std@@@?$_Hash@V?$_Umap_traits@KUProcessPerfData@@V?$_Uhash_compare@KU?$hash@K@std@@U?$equal_to@K@2@@std@@V?$allocator@U?$pair@$$CBKUProcessPerfData@@@std@@@3@$00@std@@@std@@QEAAXV?$_List_unchecked_const_iterator@V?$_List_val@U?$_List_simple_types@U?$pair@$$CBKUProcessPerfData@@@std@@@std@@@std@@U_Iterator_base0@2@@1@0@Z@4HA 00000001800447b4 f   Plist.obj
 0001:000437b4       ?dtor$1@?0???$emplace@AEBKUProcessPerfData@@@?$_Hash@V?$_Umap_traits@KUProcessPerfData@@V?$_Uhash_compare@KU?$hash@K@std@@U?$equal_to@K@2@@std@@V?$allocator@U?$pair@$$CBKUProcessPerfData@@@std@@@3@$00@std@@@std@@QEAA?AV?$_List_iterator@V?$_List_val@U?$_List_simple_types@U?$pair@$$CBKUProcessPerfData@@@std@@@std@@@std@@@1@AEBK$$QEAUProcessPerfData@@@Z@4HA 00000001800447b4 f   perfthread.obj
 0001:000437c8       ?dtor$0@?0???$transform@V?$_List_const_iterator@V?$_List_val@U?$_List_simple_types@U?$pair@$$CBKUProcessPerfData@@@std@@@std@@@std@@@std@@V?$back_insert_iterator@V?$vector@UProcessPerfData@@V?$allocator@UProcessPerfData@@@std@@@std@@@2@V<lambda_1>@?2??RefreshWMIData@PerfThread@@AEAAXXZ@@std@@YA?AV?$back_insert_iterator@V?$vector@UProcessPerfData@@V?$allocator@UProcessPerfData@@@std@@@std@@@0@V?$_List_const_iterator@V?$_List_val@U?$_List_simple_types@U?$pair@$$CBKUProcessPerfData@@@std@@@std@@@std@@@0@0V10@V<lambda_1>@?2??RefreshWMIData@PerfThread@@AEAAXXZ@@Z@4HA 00000001800447c8 f   perfthread.obj
 0001:000437dc       ?dtor$2@?0???$transform@V?$_List_const_iterator@V?$_List_val@U?$_List_simple_types@U?$pair@$$CBKUProcessPerfData@@@std@@@std@@@std@@@std@@V?$back_insert_iterator@V?$vector@UProcessPerfData@@V?$allocator@UProcessPerfData@@@std@@@std@@@2@V<lambda_1>@?2??RefreshWMIData@PerfThread@@AEAAXXZ@@std@@YA?AV?$back_insert_iterator@V?$vector@UProcessPerfData@@V?$allocator@UProcessPerfData@@@std@@@std@@@0@V?$_List_const_iterator@V?$_List_val@U?$_List_simple_types@U?$pair@$$CBKUProcessPerfData@@@std@@@std@@@std@@@0@0V10@V<lambda_1>@?2??RefreshWMIData@PerfThread@@AEAAXXZ@@Z@4HA 00000001800447dc f   perfthread.obj
 0001:000437f4       ?dtor$3@?0???$transform@V?$_List_const_iterator@V?$_List_val@U?$_List_simple_types@U?$pair@$$CBKUProcessPerfData@@@std@@@std@@@std@@@std@@V?$back_insert_iterator@V?$vector@UProcessPerfData@@V?$allocator@UProcessPerfData@@@std@@@std@@@2@V<lambda_1>@?2??RefreshWMIData@PerfThread@@AEAAXXZ@@std@@YA?AV?$back_insert_iterator@V?$vector@UProcessPerfData@@V?$allocator@UProcessPerfData@@@std@@@std@@@0@V?$_List_const_iterator@V?$_List_val@U?$_List_simple_types@U?$pair@$$CBKUProcessPerfData@@@std@@@std@@@std@@@0@0V10@V<lambda_1>@?2??RefreshWMIData@PerfThread@@AEAAXXZ@@Z@4HA 00000001800447f4 f   perfthread.obj
 0001:0004380c       ?dtor$4@?0???$transform@V?$_List_const_iterator@V?$_List_val@U?$_List_simple_types@U?$pair@$$CBKUProcessPerfData@@@std@@@std@@@std@@@std@@V?$back_insert_iterator@V?$vector@UProcessPerfData@@V?$allocator@UProcessPerfData@@@std@@@std@@@2@V<lambda_1>@?2??RefreshWMIData@PerfThread@@AEAAXXZ@@std@@YA?AV?$back_insert_iterator@V?$vector@UProcessPerfData@@V?$allocator@UProcessPerfData@@@std@@@std@@@0@V?$_List_const_iterator@V?$_List_val@U?$_List_simple_types@U?$pair@$$CBKUProcessPerfData@@@std@@@std@@@std@@@0@0V10@V<lambda_1>@?2??RefreshWMIData@PerfThread@@AEAAXXZ@@Z@4HA 000000018004480c f   perfthread.obj
 0001:00043824       ?dtor$0@?0???0ProcessPerfData@@QEAA@AEBU0@@Z@4HA 0000000180044824 f   perfthread.obj
 0001:0004383c       ?dtor$1@?0???0ProcessPerfData@@QEAA@AEBU0@@Z@4HA 000000018004483c f   perfthread.obj
 0001:00043854       ?dtor$2@?0???0ProcessPerfData@@QEAA@AEBU0@@Z@4HA 0000000180044854 f   perfthread.obj
 0001:0004386c       ?dtor$0@?0??GetList@@YA_NAEAPEAUPluginPanelItem@@AEA_KAEAVPerfThread@@@Z@4HA 000000018004486c f   Plist.obj
 0001:00043880       ?dtor$2@?0??GetList@@YA_NAEAPEAUPluginPanelItem@@AEA_KAEAVPerfThread@@@Z@4HA 0000000180044880 f   Plist.obj
 0001:00043898       ?dtor$3@?0??GetList@@YA_NAEAPEAUPluginPanelItem@@AEA_KAEAVPerfThread@@@Z@4HA 0000000180044898 f   Plist.obj
 0001:000438b0       ?dtor$0@?0??KillProcess@@YA_NKPEAUHWND__@@@Z@4HA 00000001800448b0 f   Plist.obj
 0001:000438c4       ?dtor$1@?0??KillProcess@@YA_NKPEAUHWND__@@@Z@4HA 00000001800448c4 f   Plist.obj
 0001:000438d8       ?dtor$2@?0??print_module_impl@@YAXQEAXAEBV?$basic_string@_WU?$char_traits@_W@std@@V?$allocator@_W@2@@std@@KAEBUoptions@@AEBV?$function@$$A6A_NPEA_W_K@Z@2@@Z@4HA 00000001800448d8 f   Plist.obj
 0001:000438ec       ?dtor$0@?0??PrintModules@@YAXPEAXKAEAUoptions@@@Z@4HA 00000001800448ec f   Plist.obj
 0001:00043900       ?dtor$2@?0??PrintModules@@YAXPEAXKAEAUoptions@@@Z@4HA 0000000180044900 f   Plist.obj
 0001:00043914       ?dtor$3@?0??PrintModules@@YAXPEAXKAEAUoptions@@@Z@4HA 0000000180044914 f   Plist.obj
 0001:00043928       ?dtor$0@?0??PrintModules@?$ipc_functions@$0A@@@SAXPEAX0AEAUoptions@@@Z@4HA 0000000180044928 f   Plist.obj
 0001:0004393c       ?dtor$1@?0??PrintModules@?$ipc_functions@$0A@@@SAXPEAX0AEAUoptions@@@Z@4HA 000000018004493c f   Plist.obj
 0001:00043950       ?dtor$0@?0???$print_module@PEAX@@YAXQEAXPEAXKAEAUoptions@@AEBV?$function@$$A6A_NPEA_W_K@Z@std@@@Z@4HA 0000000180044950 f   Plist.obj
 0001:00043950       ?dtor$1@?0??WinError@@YAHPEB_W@Z@4HA 0000000180044950 f   Pmix.obj
 0001:00043964       ?dtor$0@?0??ExecMethod@WMIConnection@@AEAAHKPEB_W0K@Z@4HA 0000000180044964 f   wmi.obj
 0001:00043964       ?dtor$0@?0??GetProcessOwner@WMIConnection@@QEAA?AV?$basic_string@_WU?$char_traits@_W@std@@V?$allocator@_W@2@@std@@KPEAV23@@Z@4HA 0000000180044964 f   wmi.obj
 0001:00043964       ?dtor$0@?0??GetProcessUserSid@WMIConnection@@QEAA?AV?$basic_string@_WU?$char_traits@_W@std@@V?$allocator@_W@2@@std@@K@Z@4HA 0000000180044964 f   wmi.obj
 0001:00043978       ?dtor$1@?0??GetProcessOwner@WMIConnection@@QEAA?AV?$basic_string@_WU?$char_traits@_W@std@@V?$allocator@_W@2@@std@@KPEAV23@@Z@4HA 0000000180044978 f   wmi.obj
 0001:0004398c       ?dtor$2@?0??GetProcessOwner@WMIConnection@@QEAA?AV?$basic_string@_WU?$char_traits@_W@std@@V?$allocator@_W@2@@std@@KPEAV23@@Z@4HA 000000018004498c f   wmi.obj
 0001:0004398c       ?dtor$2@?0??GetProcessUserSid@WMIConnection@@QEAA?AV?$basic_string@_WU?$char_traits@_W@std@@V?$allocator@_W@2@@std@@K@Z@4HA 000000018004498c f   wmi.obj
 0001:000439a0       ?dtor$10@?0??ExecMethod@WMIConnection@@AEAAHKPEB_W0K@Z@4HA 00000001800449a0 f   wmi.obj
 0001:000439a0       ?dtor$3@?0??GetProcessOwner@WMIConnection@@QEAA?AV?$basic_string@_WU?$char_traits@_W@std@@V?$allocator@_W@2@@std@@KPEAV23@@Z@4HA 00000001800449a0 f   wmi.obj
 0001:000439b4       ?dtor$1@?0??ExecMethod@WMIConnection@@AEAAHKPEB_W0K@Z@4HA 00000001800449b4 f   wmi.obj
 0001:000439b4       ?dtor$1@?0??GetProcessUserSid@WMIConnection@@QEAA?AV?$basic_string@_WU?$char_traits@_W@std@@V?$allocator@_W@2@@std@@K@Z@4HA 00000001800449b4 f   wmi.obj
 0001:000439b4       ?dtor$4@?0??ExecMethod@WMIConnection@@AEAAHKPEB_W0K@Z@4HA 00000001800449b4 f   wmi.obj
 0001:000439b4       ?dtor$6@?0??ExecMethod@WMIConnection@@AEAAHKPEB_W0K@Z@4HA 00000001800449b4 f   wmi.obj
 0001:000439c8       ?dtor$3@?0??GetProcessUserSid@WMIConnection@@QEAA?AV?$basic_string@_WU?$char_traits@_W@std@@V?$allocator@_W@2@@std@@K@Z@4HA 00000001800449c8 f   wmi.obj
 0001:000439dc       ?dtor$0@?0??GetProcessSessionId@WMIConnection@@QEAAKK@Z@4HA 00000001800449dc f   wmi.obj
 0001:000439f0       ?dtor$2@?0??ExecMethod@WMIConnection@@AEAAHKPEB_W0K@Z@4HA 00000001800449f0 f   wmi.obj
 0001:00043a04       ?dtor$3@?0??ExecMethod@WMIConnection@@AEAAHKPEB_W0K@Z@4HA 0000000180044a04 f   wmi.obj
 0001:00043a18       ?dtor$5@?0??ExecMethod@WMIConnection@@AEAAHKPEB_W0K@Z@4HA 0000000180044a18 f   wmi.obj
 0001:00043a2c       ?dtor$7@?0??ExecMethod@WMIConnection@@AEAAHKPEB_W0K@Z@4HA 0000000180044a2c f   wmi.obj
 0001:00043a40       ?dtor$8@?0??ExecMethod@WMIConnection@@AEAAHKPEB_W0K@Z@4HA 0000000180044a40 f   wmi.obj
 0001:00043a54       ?dtor$9@?0??ExecMethod@WMIConnection@@AEAAHKPEB_W0K@Z@4HA 0000000180044a54 f   wmi.obj
 0001:00043a68       ?dtor$0@?0??GetProcessProperty@WMIConnection@@AEAA_NKPEB_WAEBV?$function@$$A6AXAEBUtagVARIANT@@@Z@std@@@Z@4HA 0000000180044a68 f   wmi.obj
 0001:00043a7c       ?dtor$1@?0??GetProcessProperty@WMIConnection@@AEAA_NKPEB_WAEBV?$function@$$A6AXAEBUtagVARIANT@@@Z@std@@@Z@4HA 0000000180044a7c f   wmi.obj
 0001:00043a90       ?dtor$2@?0??GetProcessProperty@WMIConnection@@AEAA_NKPEB_WAEBV?$function@$$A6AXAEBUtagVARIANT@@@Z@std@@@Z@4HA 0000000180044a90 f   wmi.obj
 0001:00043aa4       ?dtor$0@?0??Connect@WMIConnection@@QEAA_NPEB_W00@Z@4HA 0000000180044aa4 f   wmi.obj
 0001:00043ac0       ?dtor$2@?0??Connect@WMIConnection@@QEAA_NPEB_W00@Z@4HA 0000000180044ac0 f   wmi.obj
 0001:00043adc       ?dtor$3@?0??Connect@WMIConnection@@QEAA_NPEB_W00@Z@4HA 0000000180044adc f   wmi.obj
 0001:00043af8       ?dtor$4@?0??Connect@WMIConnection@@QEAA_NPEB_W00@Z@4HA 0000000180044af8 f   wmi.obj
 0001:00043b14       ?dtor$5@?0??Connect@WMIConnection@@QEAA_NPEB_W00@Z@4HA 0000000180044b14 f   wmi.obj
 0001:00043b30       ?dtor$0@?0??_Init@locale@std@@CAPEAV_Locimp@12@_N@Z@4HA 0000000180044b30 f   libcpmt:locale0.obj
 0001:00043b44       __scrt_is_nonwritable_in_current_image$filt$0 0000000180044b44 f   LIBCMT:utility.obj
 0001:00043b6c       $LN31                      0000000180044b6c     LIBCMT:utility.obj
 0001:00043b70       ?fin$0@?0???_M@YAXPEAX_K1P6AX0@Z@Z@4HA 0000000180044b70 f   LIBCMT:ehvecdtr.obj
 0001:00043ba4       ?filt$0@?0??__ArrayUnwind@@YAXPEAX_K1P6AX0@Z@Z@4HA 0000000180044ba4 f   LIBCMT:ehvecdtr.obj
 0001:00043c3c       $LN26                      0000000180044c3c     LIBCMT:ehvecdtr.obj
 0001:00043c40       ?fin$0@?0??dllmain_crt_process_attach@@YAHQEAUHINSTANCE__@@QEAX@Z@4HA 0000000180044c40 f   LIBCMT:dll_dllmain.obj
 0001:00043c60       ?fin$0@?0??dllmain_crt_process_detach@@YAH_N@Z@4HA 0000000180044c60 f   LIBCMT:dll_dllmain.obj
 0001:00043c80       ?fin$1@?0??dllmain_crt_process_detach@@YAH_N@Z@4HA 0000000180044c80 f   LIBCMT:dll_dllmain.obj
 0001:00043c9c       ?filt$0@?0??dllmain_dispatch@@YAHQEAUHINSTANCE__@@KQEAX@Z@4HA 0000000180044c9c f   LIBCMT:dll_dllmain.obj
 0001:00043cd8       ?filt$0@?0???$_CallSETranslator@V__FrameHandler3@@@@YAHPEAUEHExceptionRecord@@PEA_KPEAU_CONTEXT@@PEAU_xDISPATCHER_CONTEXT@@PEBU_s_FuncInfo@@K1H@Z@4HA 0000000180044cd8 f   libvcruntime:risctrnsctrl.obj
 0001:00043d68       __DestructExceptionObject$filt$0 0000000180044d68 f   libvcruntime:ehhelpers.obj
 0001:00043e60       $LN30                      0000000180044e60     libvcruntime:ehhelpers.obj
 0001:00043e64       $LN31                      0000000180044e64     libvcruntime:ehhelpers.obj
 0001:00043e68       $LN32                      0000000180044e68     libvcruntime:ehhelpers.obj
 0001:00043e6c       $LN33                      0000000180044e6c     libvcruntime:ehhelpers.obj
 0001:00043e70       ?filt$0@?0??CxxCallCatchBlock@__FrameHandler3@@SAPEAXPEAU_EXCEPTION_RECORD@@@Z@4HA 0000000180044e70 f   libvcruntime:frame.obj
 0001:00043e98       ?fin$1@?0??CxxCallCatchBlock@__FrameHandler3@@SAPEAXPEAU_EXCEPTION_RECORD@@@Z@4HA 0000000180044e98 f   libvcruntime:frame.obj
 0001:00043f30       $LN31                      0000000180044f30     libvcruntime:frame.obj
 0001:00043f34       $LN32                      0000000180044f34     libvcruntime:frame.obj
 0001:00043f38       ?filt$0@?0??FrameUnwindToState@__FrameHandler3@@SAXPEA_KPEAU_xDISPATCHER_CONTEXT@@PEBU_s_FuncInfo@@H@Z@4HA 0000000180044f38 f   libvcruntime:frame.obj
 0001:00043f54       ?fin$1@?0??FrameUnwindToState@__FrameHandler3@@SAXPEA_KPEAU_xDISPATCHER_CONTEXT@@PEBU_s_FuncInfo@@H@Z@4HA 0000000180044f54 f   libvcruntime:frame.obj
 0001:00043f88       __acrt_initialize_lowio$fin$0 0000000180044f88 f   libucrt:ioinit.obj
 0001:00043f88       __acrt_lowio_ensure_fh_exists$fin$0 0000000180044f88 f   libucrt:osfinfo.obj
 0001:00043fa8       ?fin$0@?0???$?RV<lambda_0ae27a3a962d80f24befdcbee591983d>@@AEAV<lambda_8d0ee55de4b1038c4002e0adecdf1839>@@V<lambda_dc504788e8f1664fe9b84e20bfb512f2>@@@?$__crt_seh_guarded_call@X@@QEAAX$$QEAV<lambda_0ae27a3a962d80f24befdcbee591983d>@@AEAV<lambda_8d0ee55de4b1038c4002e0adecdf1839>@@$$QEAV<lambda_dc504788e8f1664fe9b84e20bfb512f2>@@@Z@4HA 0000000180044fa8 f   libucrt:per_thread_data.obj
 0001:00043fa8       ?fin$0@?0???$?RV<lambda_2d41944a1d46af3157314b8a01080d33>@@AEAV<lambda_8f455de75cd7d7f24b4096f044d8b9e6>@@V<lambda_aa500f224e6afead328df44964fe2772>@@@?$__crt_seh_guarded_call@X@@QEAAX$$QEAV<lambda_2d41944a1d46af3157314b8a01080d33>@@AEAV<lambda_8f455de75cd7d7f24b4096f044d8b9e6>@@$$QEAV<lambda_aa500f224e6afead328df44964fe2772>@@@Z@4HA 0000000180044fa8 f   libucrt:per_thread_data.obj
 0001:00043fa8       ?fin$0@?0???$?RV<lambda_aa87e3671a710a21b5dc78c0bdf72e11>@@AEAV<lambda_92619d2358a28f41a33ba319515a20b9>@@V<lambda_6992ecaafeb10aed2b74cb1fae11a551>@@@?$__crt_seh_guarded_call@X@@QEAAX$$QEAV<lambda_aa87e3671a710a21b5dc78c0bdf72e11>@@AEAV<lambda_92619d2358a28f41a33ba319515a20b9>@@$$QEAV<lambda_6992ecaafeb10aed2b74cb1fae11a551>@@@Z@4HA 0000000180044fa8 f   libucrt:per_thread_data.obj
 0001:00043fa8       ?fin$0@?0???$?RV<lambda_f2e299630e499de9f9a165e60fcd3db5>@@AEAV<lambda_2ae9d31cdba2644fcbeaf08da7c24588>@@V<lambda_40d01ff24d0e7b3814fdbdcee8eab3c7>@@@?$__crt_seh_guarded_call@X@@QEAAX$$QEAV<lambda_f2e299630e499de9f9a165e60fcd3db5>@@AEAV<lambda_2ae9d31cdba2644fcbeaf08da7c24588>@@$$QEAV<lambda_40d01ff24d0e7b3814fdbdcee8eab3c7>@@@Z@4HA 0000000180044fa8 f   libucrt:per_thread_data.obj
 0001:00043fa8       ?fin$0@?0???$?RV<lambda_48fc4a32460bb0512d3b13f8499328be>@@AEAV<lambda_6c3dac0a4f3f9cefca9bb494422f9b77>@@V<lambda_0a2f2c9f9a56eb2b08bfa6ff61d331c5>@@@?$__crt_seh_guarded_call@H@@QEAAH$$QEAV<lambda_48fc4a32460bb0512d3b13f8499328be>@@AEAV<lambda_6c3dac0a4f3f9cefca9bb494422f9b77>@@$$QEAV<lambda_0a2f2c9f9a56eb2b08bfa6ff61d331c5>@@@Z@4HA 0000000180044fa8 f   libucrt:winapi_thunks.obj
 0001:00043fa8       ?fin$0@?0???$?RV<lambda_41e84717acc955b55e9d0d529e507b68>@@AEAV<lambda_b37934c380d97b75fd242ea49540127a>@@V<lambda_bb6db9f9ac473960206e0d4b942b5506>@@@?$__crt_seh_guarded_call@PEAD@@QEAAPEAD$$QEAV<lambda_41e84717acc955b55e9d0d529e507b68>@@AEAV<lambda_b37934c380d97b75fd242ea49540127a>@@$$QEAV<lambda_bb6db9f9ac473960206e0d4b942b5506>@@@Z@4HA 0000000180044fa8 f   libucrt:setlocale.obj
 0001:00043fa8       ?fin$0@?0???$?RV<lambda_1d892b297fdedeee07ed8124eeb2f2fa>@@AEAV<lambda_ffc046909424fd52df0ac47e64813305>@@V<lambda_01a7098693036236037e7cdb9bca3d73>@@@?$__crt_seh_guarded_call@X@@QEAAX$$QEAV<lambda_1d892b297fdedeee07ed8124eeb2f2fa>@@AEAV<lambda_ffc046909424fd52df0ac47e64813305>@@$$QEAV<lambda_01a7098693036236037e7cdb9bca3d73>@@@Z@4HA 0000000180044fa8 f   libucrt:wsetlocale.obj
 0001:00043fa8       ?fin$0@?0???$?RV<lambda_efdfa57d1f175319df784efa44bb7b81>@@AEAV<lambda_5f0a4c1567f8adc6734073e5d1e1b35c>@@V<lambda_2e8a7d3640ea6ccb4c2413664c2db6fd>@@@?$__crt_seh_guarded_call@X@@QEAAX$$QEAV<lambda_efdfa57d1f175319df784efa44bb7b81>@@AEAV<lambda_5f0a4c1567f8adc6734073e5d1e1b35c>@@$$QEAV<lambda_2e8a7d3640ea6ccb4c2413664c2db6fd>@@@Z@4HA 0000000180044fa8 f   libucrt:mbctype.obj
 0001:00043fa8       ?fin$0@?0???$?RV<lambda_450d765d439847d4c735a33c368b5fc0>@@AEAV<lambda_44731a7d0e6d81c3e6aa82d741081786>@@V<lambda_601a2a7da3b7a96e9554ac7215c4b07c>@@@?$__crt_seh_guarded_call@P6AXH@Z@@QEAAP6AXH@Z$$QEAV<lambda_450d765d439847d4c735a33c368b5fc0>@@AEAV<lambda_44731a7d0e6d81c3e6aa82d741081786>@@$$QEAV<lambda_601a2a7da3b7a96e9554ac7215c4b07c>@@@Z@4HA 0000000180044fa8 f   libucrt:signal.obj
 0001:00043fa8       ?fin$0@?0???$?RV<lambda_d80eeec6fff315bfe5c115232f3240e3>@@AEAV<lambda_6e4b09c48022b2350581041d5f6b0c4c>@@V<lambda_2358e3775559c9db80273638284d5e45>@@@?$__crt_seh_guarded_call@X@@QEAAX$$QEAV<lambda_d80eeec6fff315bfe5c115232f3240e3>@@AEAV<lambda_6e4b09c48022b2350581041d5f6b0c4c>@@$$QEAV<lambda_2358e3775559c9db80273638284d5e45>@@@Z@4HA 0000000180044fa8 f   libucrt:exit.obj
 0001:00043fa8       ?fin$0@?0???$?RV<lambda_638799b9deba96c50f710eeac98168cd>@@AEAV<lambda_22ebabd17bc4fa466a2aca6d8deb888d>@@V<lambda_a6f7d7db0129f75315ebf26d50c089f1>@@@?$__crt_seh_guarded_call@H@@QEAAH$$QEAV<lambda_638799b9deba96c50f710eeac98168cd>@@AEAV<lambda_22ebabd17bc4fa466a2aca6d8deb888d>@@$$QEAV<lambda_a6f7d7db0129f75315ebf26d50c089f1>@@@Z@4HA 0000000180044fa8 f   libucrt:onexit.obj
 0001:00043fa8       ?fin$0@?0???$?RV<lambda_7777bce6b2f8c936911f934f8298dc43>@@AEAV<lambda_f03950bc5685219e0bcd2087efbe011e>@@V<lambda_3883c3dff614d5e0c5f61bb1ac94921c>@@@?$__crt_seh_guarded_call@H@@QEAAH$$QEAV<lambda_7777bce6b2f8c936911f934f8298dc43>@@AEAV<lambda_f03950bc5685219e0bcd2087efbe011e>@@$$QEAV<lambda_3883c3dff614d5e0c5f61bb1ac94921c>@@@Z@4HA 0000000180044fa8 f   libucrt:onexit.obj
 0001:00043fcc       ?filt$0@?0???R<lambda_6e4b09c48022b2350581041d5f6b0c4c>@@QEBA@XZ@4HA 0000000180044fcc f   libucrt:exit.obj
 0001:00043ff0       _query_new_handler$fin$0   0000000180044ff0 f   libucrt:new_handler.obj
 0001:00044010       _fcloseall$fin$0           0000000180045010 f   libucrt:closeall.obj
 0001:00044030       ?fin$0@?0???$?RV<lambda_842d9ff0dc9ef11c61343bbaebe7f885>@@AEAV<lambda_c5860995281e5c4ce005b3de8f5874ee>@@V<lambda_d90129c13df834fdcbf8d2b88dafcf2d>@@@?$__crt_seh_guarded_call@X@@QEAAX$$QEAV<lambda_842d9ff0dc9ef11c61343bbaebe7f885>@@AEAV<lambda_c5860995281e5c4ce005b3de8f5874ee>@@$$QEAV<lambda_d90129c13df834fdcbf8d2b88dafcf2d>@@@Z@4HA 0000000180045030 f   libucrt:fflush.obj
 0001:00044054       ?fin$0@?0???$?RV<lambda_886d6c58226a84441f68b9f2b8217b83>@@AEAV<lambda_ab61a845afdef5b7c387490eaf3616ee>@@V<lambda_f7f22ab5edc0698d5f6905b0d3f44752>@@@?$__crt_seh_guarded_call@X@@QEAAX$$QEAV<lambda_886d6c58226a84441f68b9f2b8217b83>@@AEAV<lambda_ab61a845afdef5b7c387490eaf3616ee>@@$$QEAV<lambda_f7f22ab5edc0698d5f6905b0d3f44752>@@@Z@4HA 0000000180045054 f   libucrt:fflush.obj
 0001:00044078       ?fin$0@?0???$?RV<lambda_410d79af7f07d98d83a3f525b3859a53>@@AEAV<lambda_3e16ef9562a7dcce91392c22ab16ea36>@@V<lambda_38119f0e861e05405d8a144b9b982f0a>@@@?$__crt_seh_guarded_call@X@@QEAAX$$QEAV<lambda_410d79af7f07d98d83a3f525b3859a53>@@AEAV<lambda_3e16ef9562a7dcce91392c22ab16ea36>@@$$QEAV<lambda_38119f0e861e05405d8a144b9b982f0a>@@@Z@4HA 0000000180045078 f   libucrt:wsetlocale.obj
 0001:0004409c       ?fin$0@?0???$?RV<lambda_7f2adfce497ff2baa965cd4f576ecfd1>@@AEAV<lambda_2a444430fde8c29194d880d93eed5e8f>@@AEAV<lambda_8dff2cf36a5417162780cd64fa2883ef>@@@?$__crt_seh_guarded_call@X@@QEAAX$$QEAV<lambda_7f2adfce497ff2baa965cd4f576ecfd1>@@AEAV<lambda_2a444430fde8c29194d880d93eed5e8f>@@AEAV<lambda_8dff2cf36a5417162780cd64fa2883ef>@@@Z@4HA 000000018004509c f   libucrt:wsetlocale.obj
 0001:000440c8       _write$fin$0               00000001800450c8 f   libucrt:write.obj
 0001:000440e8       ?dtor$0@?0??_wcstombs_l_helper@@YA_KPEADPEB_W_KPEAU__crt_locale_pointers@@@Z@4HA 00000001800450e8 f   libucrt:wcstombs.obj
 0001:000440fc       raise$fin$0                00000001800450fc f   libucrt:signal.obj
 0001:00044124       ?fin$0@?0??update_thread_multibyte_data_internal@@YAPEAU__crt_multibyte_data@@QEAU__acrt_ptd@@QEAPEAU1@@Z@4HA 0000000180045124 f   libucrt:mbctype.obj
 0001:00044144       fclose$fin$0               0000000180045144 f   libucrt:fclose.obj
 0001:00044164       ?fin$0@?0???$?RV<lambda_751a882b2c74d4b022dec766aa51a29a>@@AEAV<lambda_628dfdc04ba53c8bfc02c9951375f3f5>@@V<lambda_f6c7be5f7998530c34de24c7437d6b54>@@@?$__crt_seh_guarded_call@H@@QEAAH$$QEAV<lambda_751a882b2c74d4b022dec766aa51a29a>@@AEAV<lambda_628dfdc04ba53c8bfc02c9951375f3f5>@@$$QEAV<lambda_f6c7be5f7998530c34de24c7437d6b54>@@@Z@4HA 0000000180045164 f   libucrt:close.obj
 0001:00044164       ?fin$0@?0???$?RV<lambda_a37b2b86f63e897a80ea819b0eb08c01>@@AEAV<lambda_38ce7e780aa69e748d6df282ebc68efe>@@V<lambda_99fb1378e971ab6e7edea83e3a7a83a2>@@@?$__crt_seh_guarded_call@H@@QEAAH$$QEAV<lambda_a37b2b86f63e897a80ea819b0eb08c01>@@AEAV<lambda_38ce7e780aa69e748d6df282ebc68efe>@@$$QEAV<lambda_99fb1378e971ab6e7edea83e3a7a83a2>@@@Z@4HA 0000000180045164 f   libucrt:commit.obj
 0001:00044188       __acrt_update_thread_locale_data$fin$0 0000000180045188 f   libucrt:locale_refcounting.obj
 0001:000441a8       _IsNonwritableInCurrentImage$filt$0 00000001800451a8 f   LIBCMT:pesect.obj
 0001:000441d8       ??__F?m_PanelModesDataRemote@Plist@@0V?$vector@Umode@@V?$allocator@Umode@@@std@@@std@@A@@YAXXZ 00000001800451d8 f   fileio.obj
 0001:00044248       ??__F?m_PanelModesDataLocal@Plist@@0V?$vector@Umode@@V?$allocator@Umode@@@std@@@std@@A@@YAXXZ 0000000180045248 f   fileio.obj
 0001:000442b8       ??__FUserAccountID@?1??GetUserAccountID@@YA@XZ@YAXXZ 00000001800452b8 f   handles.obj
 0001:00044300       ??__FTitle@?1??GetOpenPanelInfo@Plist@@QEAAXPEAUOpenPanelInfo@@@Z@YAXXZ 0000000180045300 f   Pclass.obj
 0001:00044348       ??__FhDebugToken@@YAXXZ    0000000180045348 f   Plist.obj
 0001:00044368       ??__Finitlocks@std@@YAXXZ  0000000180045368 f   libcpmt:xlock.obj
 0001:00044378       ??__F_Fac_tidy_reg@std@@YAXXZ 0000000180045378 f   libcpmt:locale0.obj
 0001:00044388       ??__Fclassic_locale@std@@YAXXZ 0000000180045388 f   libcpmt:locale0.obj
 0001:00044400       ??__Finit_atexit@@YAXXZ    0000000180045400 f   libcpmt:iosptrs.obj
 0001:00044410       ??__Finitlocks@std@@YAXXZ  0000000180045410 f   libcpmt:iosptrs.obj
 0002:000004a8       ?initlocks$initializer$@std@@3P6AXXZEA 00000001800464a8     libcpmt:xlock.obj
 0002:000004b0       ?initlocks$initializer$@std@@3P6AXXZEA 00000001800464b0     libcpmt:iosptrs.obj
 0002:000004b8       ?init_atexit$initializer$@@3P6AXXZEA 00000001800464b8     libcpmt:iosptrs.obj
 0002:000004c0       ?_Fac_tidy_reg$initializer$@std@@3P6AXXZEA 00000001800464c0     libcpmt:locale0.obj
 0002:000004c8       ?classic_locale$initializer$@std@@3P6AXXZEA 00000001800464c8     libcpmt:locale0.obj
 0002:000004d0       ??m_PanelModesDataLocal$initializer$@Plist@@0P6AXXZEA@@3P6AXXZEA 00000001800464d0     fileio.obj
 0002:000004d8       ??m_PanelModesDataRemote$initializer$@Plist@@0P6AXXZEA@@3P6AXXZEA 00000001800464d8     fileio.obj
 0002:000004e0       ?hDebugToken$initializer$@@3P6AXXZEA 00000001800464e0     Plist.obj
 0002:000004f8       pinit                      00000001800464f8     LIBCMT:lconv_unsigned_char.obj
 0002:00000650       $cppxdata$?_Init@locale@std@@CAPEAV_Locimp@12@_N@Z 0000000180046650     libcpmt:locale0.obj
 0002:000006c0       ?_Win_errtab@?A0xf525aa19@@3QBU_Win_errtab_t@1@B 00000001800466c0     libcpmt:syserror.obj
 0002:00000940       ?_Sys_errtab@?A0xf525aa19@@3QBU_Sys_errtab_t@1@B 0000000180046940     libcpmt:syserror.obj
 0002:000014f0       $cppxdata$??1_Init_atexit@@QEAA@XZ 00000001800474f0     libcpmt:iosptrs.obj
 0002:00001520       ?_Whitespace_bitmap@?A0x8d5ed78e@@3U_Whitespace_bitmap_t@1@B 0000000180047520     libcpmt:syserror_import_lib.obj
 0002:00001688       digits                     0000000180047688     libcpmt:xstoul.obj
 0002:000016b0       ndigs                      00000001800476b0     libcpmt:xstoul.obj
 0002:000016d8       digits                     00000001800476d8     libcpmt:xstoull.obj
 0002:00001700       ndigs                      0000000180047700     libcpmt:xstoull.obj
 0002:00001740       GS_ExceptionPointers       0000000180047740     LIBCMT:gs_report.obj
 0002:00001750       ?ExceptionTemplate@?1??UnwindNestedFrames@__FrameHandler3@@SAXPEA_KPEAUEHExceptionRecord@@PEAU_CONTEXT@@0PEAXPEBU_s_FuncInfo@@HHPEBU_s_HandlerType@@PEAU_xDISPATCHER_CONTEXT@@E@Z@4U_EXCEPTION_RECORD@@B 0000000180047750     libvcruntime:risctrnsctrl.obj
 0002:00001820       ?tokenTable@@3QBUStringLiteral@@B 0000000180047820     libvcruntime:undname.obj
 0002:00001920       ?nameTable@@3QBUStringLiteral@@B 0000000180047920     libvcruntime:undname.obj
 0002:00001e50       ?rttiTable@@3QBUStringLiteral@@B 0000000180047e50     libvcruntime:undname.obj
 0002:00001ea0       ?IndirectionName@@3QBUStringLiteral@@B 0000000180047ea0     libvcruntime:undname.obj
 0002:00001f00       ?PrefixName@@3QBUStringLiteral@@B 0000000180047f00     libvcruntime:undname.obj
 0002:00002650       ?errtable@@3QBUerrentry@?A0x31fdb9ec@@B 0000000180048650     libucrt:errno.obj
 0002:000027c0       ?ln_lead_table@?1??log2@@9@9 00000001800487c0     libucrt:log2.obj
 0002:000029d0       ?ln_tail_table@?1??log2@@9@9 00000001800489d0     libucrt:log2.obj
 0002:00003d20       a1                         0000000180049d20     libucrt:pow.obj
 0002:00003db0       a2                         0000000180049db0     libucrt:pow.obj
 0002:00003df8       _ovfx                      0000000180049df8     libucrt:pow.obj
 0002:00003e00       _uflx                      0000000180049e00     libucrt:pow.obj
 0002:00003f10       __acrt_initializers        0000000180049f10     libucrt:initialization.obj
 0002:00004010       ?module_names@?A0x391cf84c@@3QBQEB_WB 000000018004a010     libucrt:winapi_thunks.obj
 0002:00004568       ?candidate_modules@?1??try_get_AreFileApisANSI@@YAP6AHXZXZ@4QBW4module_id@?A0x391cf84c@@B 000000018004a568     libucrt:winapi_thunks.obj
 0002:00004580       ?candidate_modules@?1??try_get_CompareStringEx@@YAP6AHPEB_WK0H0HPEAU_nlsversioninfo@@PEAX_J@ZXZ@4QBW4module_id@?A0x391cf84c@@B 000000018004a580     libucrt:winapi_thunks.obj
 0002:00004598       ?candidate_modules@?1??try_get_EnumSystemLocalesEx@@YAP6AHP6AHPEA_WK_J@ZK1PEAX@ZXZ@4QBW4module_id@?A0x391cf84c@@B 000000018004a598     libucrt:winapi_thunks.obj
 0002:000045b8       ?candidate_modules@?1??try_get_FlsAlloc@@YAP6AKP6AXPEAX@Z@ZXZ@4QBW4module_id@?A0x391cf84c@@B 000000018004a5b8     libucrt:winapi_thunks.obj
 0002:000045d0       ?candidate_modules@?1??try_get_FlsFree@@YAP6AHK@ZXZ@4QBW4module_id@?A0x391cf84c@@B 000000018004a5d0     libucrt:winapi_thunks.obj
 0002:000045e0       ?candidate_modules@?1??try_get_FlsGetValue@@YAP6APEAXK@ZXZ@4QBW4module_id@?A0x391cf84c@@B 000000018004a5e0     libucrt:winapi_thunks.obj
 0002:000045f8       ?candidate_modules@?1??try_get_FlsSetValue@@YAP6AHKPEAX@ZXZ@4QBW4module_id@?A0x391cf84c@@B 000000018004a5f8     libucrt:winapi_thunks.obj
 0002:00004610       ?candidate_modules@?1??try_get_GetDateFormatEx@@YAP6AHPEB_WKPEBU_SYSTEMTIME@@0PEA_WH0@ZXZ@4QBW4module_id@?A0x391cf84c@@B 000000018004a610     libucrt:winapi_thunks.obj
 0002:00004628       ?candidate_modules@?1??try_get_GetLocaleInfoEx@@YAP6AHPEB_WKPEA_WH@ZXZ@4QBW4module_id@?A0x391cf84c@@B 000000018004a628     libucrt:winapi_thunks.obj
 0002:00004640       ?candidate_modules@?1??try_get_GetTimeFormatEx@@YAP6AHPEB_WKPEBU_SYSTEMTIME@@0PEA_WH@ZXZ@4QBW4module_id@?A0x391cf84c@@B 000000018004a640     libucrt:winapi_thunks.obj
 0002:00004658       ?candidate_modules@?1??try_get_GetUserDefaultLocaleName@@YAP6AHPEA_WH@ZXZ@4QBW4module_id@?A0x391cf84c@@B 000000018004a658     libucrt:winapi_thunks.obj
 0002:00004680       ?candidate_modules@?1??try_get_InitializeCriticalSectionEx@@YAP6AHPEAU_RTL_CRITICAL_SECTION@@KK@ZXZ@4QBW4module_id@?A0x391cf84c@@B 000000018004a680     libucrt:winapi_thunks.obj
 0002:000046a8       ?candidate_modules@?1??try_get_IsValidLocaleName@@YAP6AHPEB_W@ZXZ@4QBW4module_id@?A0x391cf84c@@B 000000018004a6a8     libucrt:winapi_thunks.obj
 0002:000046c8       ?candidate_modules@?1??try_get_LCMapStringEx@@YAP6AHPEB_WK0HPEA_WHPEAU_nlsversioninfo@@PEAX_J@ZXZ@4QBW4module_id@?A0x391cf84c@@B 000000018004a6c8     libucrt:winapi_thunks.obj
 0002:000046e0       ?candidate_modules@?1??try_get_LCIDToLocaleName@@YAP6AHKPEA_WHK@ZXZ@4QBW4module_id@?A0x391cf84c@@B 000000018004a6e0     libucrt:winapi_thunks.obj
 0002:00004700       ?candidate_modules@?1??try_get_LocaleNameToLCID@@YAP6AKPEB_WK@ZXZ@4QBW4module_id@?A0x391cf84c@@B 000000018004a700     libucrt:winapi_thunks.obj
 0002:0000471c       ?candidate_modules@?1??try_get_AppPolicyGetProcessTerminationMethod@@YAP6AJPEAXPEAW4AppPolicyProcessTerminationMethod@@@ZXZ@4QBW4module_id@?A0x391cf84c@@B 000000018004a71c     libucrt:winapi_thunks.obj
 0002:00004748       ?mask@?P@??_d_int@@9@4QBGB 000000018004a748     libucrt:_test.obj
 0002:00004768       ?sub@?P@??_d_int@@9@4QB_KB 000000018004a768     libucrt:_test.obj
 0002:00004790       ?strings@?1??fp_format_nan_or_infinity@@YAHW4__acrt_fp_class@@_NPEAD_K1@Z@4QAY03QEBDA 000000018004a790     libucrt:cvt.obj
 0002:00004860       _first_127char             000000018004a860     libucrt:wsetlocale.obj
 0002:000050a0       $cppxdata$?_wcstombs_l_helper@@YA_KPEADPEB_W_KPEAU__crt_locale_pointers@@@Z 000000018004b0a0     libucrt:wcstombs.obj
 0002:000050d0       ?_names@?1??_get_fname@@9@9 000000018004b0d0     libucrt:fpexcept.obj
 0002:00005390       ?ln_lead_table@?1??log@@9@9 000000018004b390     libucrt:log.obj
 0002:000055a0       ?ln_tail_table@?1??log@@9@9 000000018004b5a0     libucrt:log.obj
 0002:000057f0       ?LcidToLocaleNameTable@?A0x881e4c05@@3QBULcidToLocaleName@1@B 000000018004b7f0     libucrt:lcidtoname_downlevel.obj
 0002:00007250       ?LocaleNameToIndexTable@?A0x881e4c05@@3QBULocaleNameIndex@1@B 000000018004d250     libucrt:lcidtoname_downlevel.obj
 0002:00008af0       ?large_power_indices@?1??multiply_by_power_of_ten@__crt_strtox@@YA_NAEAUbig_integer@2@I@Z@4QBUunpack_index@?1??12@YA_N0I@Z@B 000000018004eaf0     libucrt:cfout.obj
 0002:00009ba0       ?ln_lead_table@?1??log10@@9@9 000000018004fba0     libucrt:log10.obj
 0002:00009db0       ?ln_tail_table@?1??log10@@9@9 000000018004fdb0     libucrt:log10.obj
 0002:0000b3c0       ?constStrTypes@@3QBQEB_WB  00000001800513c0     handles.obj
 0002:0000b560       ?Styles@?1??window_style@@YA@PEAUHWND__@@@Z@4QBU?$pair@HPEB_W@std@@B 0000000180051560     Pclass.obj
 0002:0000b660       ?StatusCols@?1??InitializePanelModes@Plist@@SAXXZ@4QB_WB 0000000180051660     Pclass.obj
 0002:0000b670       ?Pr@?HF@??ProcessKey@Plist@@QEAAHPEBU_INPUT_RECORD@@@Z@4QBEB 0000000180051670     Pclass.obj
 0002:0000b680       ?ExtStyles@?1??window_ex_style@@YA@PEAUHWND__@@@Z@4QBU?$pair@HPEB_W@std@@B 0000000180051680     Pclass.obj
 0002:0000b7c0       ?StatusWidths@?1??InitializePanelModes@Plist@@SAXXZ@4QB_WB 00000001800517c0     Pclass.obj
 0002:0000b7e8       ?invalid_chars@?1??GetFiles@Plist@@QEAAHPEAUPluginPanelItem@@_KHPEAPEB_W1AEAUoptions@@@Z@4QB_WB 00000001800517e8     Pclass.obj
 0002:0000b800       ?PrClasses@?EH@??ProcessKey@Plist@@QEAAHPEBU_INPUT_RECORD@@@Z@4QBGB 0000000180051800     Pclass.obj
 0002:0000cb70       ??_7?$_Func_impl_no_alloc@V<lambda_3>@?N@??PrintModules@@YAXPEAXKAEAUoptions@@@Z@_NPEA_W_K@std@@6B@ 0000000180052b70     Plist.obj
 0002:0000cd68       ??_7?$_Func_impl_no_alloc@V<lambda_1>@?1??GetProcessInt@WMIConnection@@AEAAKKPEB_W@Z@XAEBUtagVARIANT@@@std@@6B@ 0000000180052d68     wmi.obj
 0002:0000cda0       ??_7?$_Func_impl_no_alloc@V<lambda_1>@?1??GetProcessString@WMIConnection@@AEAA?AV?$basic_string@_WU?$char_traits@_W@std@@V?$allocator@_W@2@@std@@KPEB_W@Z@XAEBUtagVARIANT@@@std@@6B@ 0000000180052da0     wmi.obj
 0002:0000d090       $cppxdata$??$?RM$0A@@?$precision_checker@Uerror_handler@detail@v8@fmt@@@detail@v8@fmt@@QEAA_KM@Z 0000000180053090     format.obj
 0002:0000d090       $cppxdata$??$?RN$0A@@?$precision_checker@Uerror_handler@detail@v8@fmt@@@detail@v8@fmt@@QEAA_KN@Z 0000000180053090     format.obj
 0002:0000d090       $cppxdata$??$?RO$0A@@?$precision_checker@Uerror_handler@detail@v8@fmt@@@detail@v8@fmt@@QEAA_KO@Z 0000000180053090     format.obj
 0002:0000d090       $cppxdata$??$?RPEBX$0A@@?$precision_checker@Uerror_handler@detail@v8@fmt@@@detail@v8@fmt@@QEAA_KPEBX@Z 0000000180053090     format.obj
 0002:0000d090       $cppxdata$??$?RUmonostate@v8@fmt@@$0A@@?$precision_checker@Uerror_handler@detail@v8@fmt@@@detail@v8@fmt@@QEAA_KUmonostate@23@@Z 0000000180053090     format.obj
 0002:0000d090       $cppxdata$??$?R_N$0A@@?$precision_checker@Uerror_handler@detail@v8@fmt@@@detail@v8@fmt@@QEAA_K_N@Z 0000000180053090     format.obj
 0002:0000d0c0       $cppxdata$??$?R_J$0A@@?$precision_checker@Uerror_handler@detail@v8@fmt@@@detail@v8@fmt@@QEAA_K_J@Z 00000001800530c0     format.obj
 0002:0000d0f0       $cppxdata$??$?RM$0A@@?$width_checker@Uerror_handler@detail@v8@fmt@@@detail@v8@fmt@@QEAA_KM@Z 00000001800530f0     format.obj
 0002:0000d0f0       $cppxdata$??$?RN$0A@@?$width_checker@Uerror_handler@detail@v8@fmt@@@detail@v8@fmt@@QEAA_KN@Z 00000001800530f0     format.obj
 0002:0000d0f0       $cppxdata$??$?RO$0A@@?$width_checker@Uerror_handler@detail@v8@fmt@@@detail@v8@fmt@@QEAA_KO@Z 00000001800530f0     format.obj
 0002:0000d0f0       $cppxdata$??$?RPEBX$0A@@?$width_checker@Uerror_handler@detail@v8@fmt@@@detail@v8@fmt@@QEAA_KPEBX@Z 00000001800530f0     format.obj
 0002:0000d0f0       $cppxdata$??$?RUmonostate@v8@fmt@@$0A@@?$width_checker@Uerror_handler@detail@v8@fmt@@@detail@v8@fmt@@QEAA_KUmonostate@23@@Z 00000001800530f0     format.obj
 0002:0000d0f0       $cppxdata$??$?R_N$0A@@?$width_checker@Uerror_handler@detail@v8@fmt@@@detail@v8@fmt@@QEAA_K_N@Z 00000001800530f0     format.obj
 0002:0000d120       $cppxdata$??$?R_J$0A@@?$width_checker@Uerror_handler@detail@v8@fmt@@@detail@v8@fmt@@QEAA_K_J@Z 0000000180053120     format.obj
 0002:0000d150       $cppxdata$??$?RH$0A@@?$precision_checker@Uerror_handler@detail@v8@fmt@@@detail@v8@fmt@@QEAA_KH@Z 0000000180053150     format.obj
 0002:0000d180       $cppxdata$??$?RH$0A@@?$width_checker@Uerror_handler@detail@v8@fmt@@@detail@v8@fmt@@QEAA_KH@Z 0000000180053180     format.obj
 0002:0000d1b0       $cppxdata$?_Init@?$numpunct@_W@std@@IEAAXAEBV_Locinfo@2@_N@Z 00000001800531b0     format.obj
 0002:0000d1e0       $cppxdata$?_Getcat@?$numpunct@_W@std@@SA_KPEAPEBVfacet@locale@2@PEBV42@@Z 00000001800531e0     format.obj
 0002:0000d210       $cppxdata$??$use_facet@V?$numpunct@_W@std@@@std@@YAAEBV?$numpunct@_W@0@AEBVlocale@0@@Z 0000000180053210     format.obj
 0002:0000d240       $cppxdata$??0?$basic_string@_WU?$char_traits@_W@std@@V?$allocator@_W@2@@std@@QEAA@QEB_W@Z 0000000180053240     format.obj
 0002:0000d270       $cppxdata$?do_grouping@?$numpunct@_W@std@@MEBA?AV?$basic_string@DU?$char_traits@D@std@@V?$allocator@D@2@@2@XZ 0000000180053270     format.obj
 0002:0000d2a0       $cppxdata$?do_falsename@?$numpunct@_W@std@@MEBA?AV?$basic_string@_WU?$char_traits@_W@std@@V?$allocator@_W@2@@2@XZ 00000001800532a0     format.obj
 0002:0000d2d0       $cppxdata$?do_truename@?$numpunct@_W@std@@MEBA?AV?$basic_string@_WU?$char_traits@_W@std@@V?$allocator@_W@2@@2@XZ 00000001800532d0     format.obj
 0002:0000d300       $cppxdata$??$thousands_sep_impl@_W@detail@v8@fmt@@YA?AU?$thousands_sep_result@_W@012@Vlocale_ref@012@@Z 0000000180053300     format.obj
 0002:0000d330       $cppxdata$?format_dragon@detail@v8@fmt@@YAXUfp@123@_NHAEAV?$buffer@D@123@AEAH@Z 0000000180053330     format.obj
 0002:0000d360       $cppxdata$?square@bigint@detail@v8@fmt@@QEAAXXZ 0000000180053360     format.obj
 0002:0000d390       $cppxdata$?throw_format_error@detail@v8@fmt@@YAXPEBD@Z 0000000180053390     format.obj
 0002:0000d3c0       $cppxdata$??1_Locinfo@std@@QEAA@XZ 00000001800533c0     format.obj
 0002:0000d3f0       $cppxdata$?on_error@error_handler@detail@v8@fmt@@QEAAXPEBD@Z 00000001800533f0     format.obj
 0002:0000d3f0       $cppxdata$?on_error@?$specs_handler@_W@detail@v8@fmt@@QEAAXPEBD@Z 00000001800533f0     handles.obj
 0002:0000d420       $cppxdata$??$apply@V?$back_insert_iterator@V?$buffer@_W@detail@v8@fmt@@@std@@_W@?$digit_grouping@_W@detail@v8@fmt@@QEBA?AV?$back_insert_iterator@V?$buffer@_W@detail@v8@fmt@@@std@@V45@V?$basic_string_view@_W@23@@Z 0000000180053420     handles.obj
 0002:0000d450       $cppxdata$??$apply@V?$back_insert_iterator@V?$buffer@_W@detail@v8@fmt@@@std@@D@?$digit_grouping@_W@detail@v8@fmt@@QEBA?AV?$back_insert_iterator@V?$buffer@_W@detail@v8@fmt@@@std@@V45@V?$basic_string_view@D@23@@Z 0000000180053450     handles.obj
 0002:0000d480       $cppxdata$??$write_significand@_WV?$back_insert_iterator@V?$buffer@_W@detail@v8@fmt@@@std@@PEBDV?$digit_grouping@_W@detail@v8@fmt@@@detail@v8@fmt@@YA?AV?$back_insert_iterator@V?$buffer@_W@detail@v8@fmt@@@std@@V34@PEBDHHAEBV?$digit_grouping@_W@012@@Z 0000000180053480     handles.obj
 0002:0000d4b0       $cppxdata$??$write_significand@V?$back_insert_iterator@V?$buffer@_W@detail@v8@fmt@@@std@@_WIV?$digit_grouping@_W@detail@v8@fmt@@@detail@v8@fmt@@YA?AV?$back_insert_iterator@V?$buffer@_W@detail@v8@fmt@@@std@@V34@IHH_WAEBV?$digit_grouping@_W@012@@Z 00000001800534b0     handles.obj
 0002:0000d4e0       $cppxdata$??$write_int_localized@V?$back_insert_iterator@V?$buffer@_W@detail@v8@fmt@@@std@@_K_W@detail@v8@fmt@@YA_NAEAV?$back_insert_iterator@V?$buffer@_W@detail@v8@fmt@@@std@@_KIAEBU?$basic_format_specs@_W@12@Vlocale_ref@012@@Z 00000001800534e0     handles.obj
 0002:0000d510       $cppxdata$??0?$digit_grouping@_W@detail@v8@fmt@@QEAA@Vlocale_ref@123@_N@Z 0000000180053510     handles.obj
 0002:0000d540       $cppxdata$??R<lambda_4>@?BO@???$do_write_float@V?$back_insert_iterator@V?$buffer@_W@detail@v8@fmt@@@std@@Ubig_decimal_fp@detail@v8@fmt@@_WV?$digit_grouping@_W@456@@detail@v8@fmt@@YA?AV?$back_insert_iterator@V?$buffer@_W@detail@v8@fmt@@@std@@V45@AEBUbig_decimal_fp@123@AEBU?$basic_format_specs@_W@23@Ufloat_specs@123@Vlocale_ref@123@@Z@QEBA@0@Z 0000000180053540     handles.obj
 0002:0000d570       $cppxdata$??$do_write_float@V?$back_insert_iterator@V?$buffer@_W@detail@v8@fmt@@@std@@Ubig_decimal_fp@detail@v8@fmt@@_WV?$digit_grouping@_W@456@@detail@v8@fmt@@YA?AV?$back_insert_iterator@V?$buffer@_W@detail@v8@fmt@@@std@@V34@AEBUbig_decimal_fp@012@AEBU?$basic_format_specs@_W@12@Ufloat_specs@012@Vlocale_ref@012@@Z 0000000180053570     handles.obj
 0002:0000d5a0       $cppxdata$??$write_int@_WV?$back_insert_iterator@V?$buffer@_W@detail@v8@fmt@@@std@@_K@detail@v8@fmt@@YA?AV?$back_insert_iterator@V?$buffer@_W@detail@v8@fmt@@@std@@V34@U?$write_int_arg@_K@012@AEBU?$basic_format_specs@_W@12@Vlocale_ref@012@@Z 00000001800535a0     handles.obj
 0002:0000d5d0       $cppxdata$??$visit_format_arg@V?$precision_checker@Uerror_handler@detail@v8@fmt@@@detail@v8@fmt@@V?$basic_format_context@V?$back_insert_iterator@V?$buffer@_W@detail@v8@fmt@@@std@@_W@34@@v8@fmt@@YA_K$$QEAV?$precision_checker@Uerror_handler@detail@v8@fmt@@@detail@01@AEBV?$basic_format_arg@V?$basic_format_context@V?$back_insert_iterator@V?$buffer@_W@detail@v8@fmt@@@std@@_W@v8@fmt@@@01@@Z 00000001800535d0     handles.obj
 0002:0000d600       $cppxdata$??$visit_format_arg@V?$width_checker@Uerror_handler@detail@v8@fmt@@@detail@v8@fmt@@V?$basic_format_context@V?$back_insert_iterator@V?$buffer@_W@detail@v8@fmt@@@std@@_W@34@@v8@fmt@@YA_K$$QEAV?$width_checker@Uerror_handler@detail@v8@fmt@@@detail@01@AEBV?$basic_format_arg@V?$basic_format_context@V?$back_insert_iterator@V?$buffer@_W@detail@v8@fmt@@@std@@_W@v8@fmt@@@01@@Z 0000000180053600     handles.obj
 0002:0000d630       $cppxdata$??R<lambda_4>@?BO@???$do_write_float@V?$back_insert_iterator@V?$buffer@_W@detail@v8@fmt@@@std@@U?$decimal_fp@N@dragonbox@detail@v8@fmt@@_WV?$digit_grouping@_W@567@@detail@v8@fmt@@YA?AV?$back_insert_iterator@V?$buffer@_W@detail@v8@fmt@@@std@@V45@AEBU?$decimal_fp@N@dragonbox@123@AEBU?$basic_format_specs@_W@23@Ufloat_specs@123@Vlocale_ref@123@@Z@QEBA@0@Z 0000000180053630     handles.obj
 0002:0000d660       $cppxdata$??R<lambda_3>@?BD@???$do_write_float@V?$back_insert_iterator@V?$buffer@_W@detail@v8@fmt@@@std@@U?$decimal_fp@N@dragonbox@detail@v8@fmt@@_WV?$digit_grouping@_W@567@@detail@v8@fmt@@YA?AV?$back_insert_iterator@V?$buffer@_W@detail@v8@fmt@@@std@@V45@AEBU?$decimal_fp@N@dragonbox@123@AEBU?$basic_format_specs@_W@23@Ufloat_specs@123@Vlocale_ref@123@@Z@QEBA@0@Z 0000000180053660     handles.obj
 0002:0000d690       $cppxdata$??$do_write_float@V?$back_insert_iterator@V?$buffer@_W@detail@v8@fmt@@@std@@U?$decimal_fp@N@dragonbox@detail@v8@fmt@@_WV?$digit_grouping@_W@567@@detail@v8@fmt@@YA?AV?$back_insert_iterator@V?$buffer@_W@detail@v8@fmt@@@std@@V34@AEBU?$decimal_fp@N@dragonbox@012@AEBU?$basic_format_specs@_W@12@Ufloat_specs@012@Vlocale_ref@012@@Z 0000000180053690     handles.obj
 0002:0000d6c0       $cppxdata$??R<lambda_3>@?BD@???$do_write_float@V?$back_insert_iterator@V?$buffer@_W@detail@v8@fmt@@@std@@U?$decimal_fp@M@dragonbox@detail@v8@fmt@@_WV?$digit_grouping@_W@567@@detail@v8@fmt@@YA?AV?$back_insert_iterator@V?$buffer@_W@detail@v8@fmt@@@std@@V45@AEBU?$decimal_fp@M@dragonbox@123@AEBU?$basic_format_specs@_W@23@Ufloat_specs@123@Vlocale_ref@123@@Z@QEBA@0@Z 00000001800536c0     handles.obj
 0002:0000d6f0       $cppxdata$??$do_write_float@V?$back_insert_iterator@V?$buffer@_W@detail@v8@fmt@@@std@@U?$decimal_fp@M@dragonbox@detail@v8@fmt@@_WV?$digit_grouping@_W@567@@detail@v8@fmt@@YA?AV?$back_insert_iterator@V?$buffer@_W@detail@v8@fmt@@@std@@V34@AEBU?$decimal_fp@M@dragonbox@012@AEBU?$basic_format_specs@_W@12@Ufloat_specs@012@Vlocale_ref@012@@Z 00000001800536f0     handles.obj
 0002:0000d720       $cppxdata$??$write_int@_WV?$back_insert_iterator@V?$buffer@_W@detail@v8@fmt@@@std@@I@detail@v8@fmt@@YA?AV?$back_insert_iterator@V?$buffer@_W@detail@v8@fmt@@@std@@V34@U?$write_int_arg@I@012@AEBU?$basic_format_specs@_W@12@Vlocale_ref@012@@Z 0000000180053720     handles.obj
 0002:0000d750       $cppxdata$??$do_parse_arg_id@_WAEAUid_adapter@?1???$parse_replacement_field@_WAEAUformat_handler@?1???$vformat_to@_W@detail@v8@fmt@@YAXAEAV?$buffer@_W@234@V?$basic_string_view@_W@34@V?$basic_format_args@V?$basic_format_context@V?$back_insert_iterator@V?$buffer@_W@detail@v8@fmt@@@std@@_W@v8@fmt@@@34@Vlocale_ref@234@@Z@@detail@v8@fmt@@YAPEB_WPEB_W0AEAUformat_handler@?1???$vformat_to@_W@234@YAXAEAV?$buffer@_W@234@V?$basic_string_view@_W@34@V?$basic_format_args@V?$basic_format_context@V?$back_insert_iterator@V?$buffer@_W@detail@v8@fmt@@@std@@_W@v8@fmt@@@34@Vlocale_ref@234@@Z@@Z@@detail@v8@fmt@@YAPEB_WPEB_W0AEAUid_adapter@?1???$parse_replacement_field@_WAEAUformat_handler@?1???$vformat_to@_W@detail@v8@fmt@@YAXAEAV?$buffer@_W@234@V?$basic_string_view@_W@34@V?$basic_format_args@V?$basic_format_context@V?$back_insert_iterator@V?$buffer@_W@detail@v8@fmt@@@std@@_W@v8@fmt@@@34@Vlocale_ref@234@@Z@@012@YAPEB_W00AEAUformat_handler@?1???$vformat_to@_W@012@YAXAEAV?$buffer@_W@012@V?$basic_string_view@_W@12@V?$basic_format_args@V?$basic_format_context@V?$back_insert_iterator@V?$buffer@_W@detail@v8@fmt@@@std@@_W@v8@fmt@@@12@Vlocale_ref@012@@Z@@Z@@Z 0000000180053750     handles.obj
 0002:0000d780       $cppxdata$??$parse_float_type_spec@Uerror_handler@detail@v8@fmt@@_W@detail@v8@fmt@@YA?AUfloat_specs@012@AEBU?$basic_format_specs@_W@12@$$QEAUerror_handler@012@@Z 0000000180053780     handles.obj
 0002:0000d7b0       $cppxdata$??$do_parse_arg_id@_WAEAUprecision_adapter@?1???$parse_precision@_WAEAV?$specs_checker@V?$specs_handler@_W@detail@v8@fmt@@@detail@v8@fmt@@@detail@v8@fmt@@YAPEB_WPEB_W0AEAV?$specs_checker@V?$specs_handler@_W@detail@v8@fmt@@@234@@Z@@detail@v8@fmt@@YAPEB_WPEB_W0AEAUprecision_adapter@?1???$parse_precision@_WAEAV?$specs_checker@V?$specs_handler@_W@detail@v8@fmt@@@detail@v8@fmt@@@012@YAPEB_W00AEAV?$specs_checker@V?$specs_handler@_W@detail@v8@fmt@@@012@@Z@@Z 00000001800537b0     handles.obj
 0002:0000d7e0       $cppxdata$??$do_parse_arg_id@_WAEAUwidth_adapter@?1???$parse_width@_WAEAV?$specs_checker@V?$specs_handler@_W@detail@v8@fmt@@@detail@v8@fmt@@@detail@v8@fmt@@YAPEB_WPEB_W0AEAV?$specs_checker@V?$specs_handler@_W@detail@v8@fmt@@@234@@Z@@detail@v8@fmt@@YAPEB_WPEB_W0AEAUwidth_adapter@?1???$parse_width@_WAEAV?$specs_checker@V?$specs_handler@_W@detail@v8@fmt@@@detail@v8@fmt@@@012@YAPEB_W00AEAV?$specs_checker@V?$specs_handler@_W@detail@v8@fmt@@@012@@Z@@Z 00000001800537e0     handles.obj
 0002:0000d810       $cppxdata$?get_arg@?$specs_handler@_W@detail@v8@fmt@@AEAA?AV?$basic_format_arg@V?$basic_format_context@V?$back_insert_iterator@V?$buffer@_W@detail@v8@fmt@@@std@@_W@v8@fmt@@@34@V?$basic_string_view@_W@34@@Z 0000000180053810     handles.obj
 0002:0000d840       $cppxdata$??$write@_WV?$back_insert_iterator@V?$buffer@_W@detail@v8@fmt@@@std@@O$0A@@detail@v8@fmt@@YA?AV?$back_insert_iterator@V?$buffer@_W@detail@v8@fmt@@@std@@V34@OU?$basic_format_specs@_W@12@Vlocale_ref@012@@Z 0000000180053840     handles.obj
 0002:0000d870       $cppxdata$??$write@_WV?$back_insert_iterator@V?$buffer@_W@detail@v8@fmt@@@std@@N$0A@@detail@v8@fmt@@YA?AV?$back_insert_iterator@V?$buffer@_W@detail@v8@fmt@@@std@@V34@NU?$basic_format_specs@_W@12@Vlocale_ref@012@@Z 0000000180053870     handles.obj
 0002:0000d8a0       $cppxdata$??$write@_WV?$back_insert_iterator@V?$buffer@_W@detail@v8@fmt@@@std@@M$0A@@detail@v8@fmt@@YA?AV?$back_insert_iterator@V?$buffer@_W@detail@v8@fmt@@@std@@V34@MU?$basic_format_specs@_W@12@Vlocale_ref@012@@Z 00000001800538a0     handles.obj
 0002:0000d8d0       $cppxdata$??$write@_WV?$back_insert_iterator@V?$buffer@_W@detail@v8@fmt@@@std@@@detail@v8@fmt@@YA?AV?$back_insert_iterator@V?$buffer@_W@detail@v8@fmt@@@std@@V34@_WAEBU?$basic_format_specs@_W@12@Vlocale_ref@012@@Z 00000001800538d0     handles.obj
 0002:0000d900       $cppxdata$??$write@_WV?$back_insert_iterator@V?$buffer@_W@detail@v8@fmt@@@std@@X$0A@@detail@v8@fmt@@YA?AV?$back_insert_iterator@V?$buffer@_W@detail@v8@fmt@@@std@@V34@PEBXAEBU?$basic_format_specs@_W@12@Vlocale_ref@012@@Z 0000000180053900     handles.obj
 0002:0000d930       $cppxdata$??$write@_WV?$back_insert_iterator@V?$buffer@_W@detail@v8@fmt@@@std@@@detail@v8@fmt@@YA?AV?$back_insert_iterator@V?$buffer@_W@detail@v8@fmt@@@std@@V34@V?$basic_string_view@_W@12@AEBU?$basic_format_specs@_W@12@Vlocale_ref@012@@Z 0000000180053930     handles.obj
 0002:0000d960       $cppxdata$?on_error@id_adapter@?1???$parse_replacement_field@_WAEAUformat_handler@?1???$vformat_to@_W@detail@v8@fmt@@YAXAEAV?$buffer@_W@234@V?$basic_string_view@_W@34@V?$basic_format_args@V?$basic_format_context@V?$back_insert_iterator@V?$buffer@_W@detail@v8@fmt@@@std@@_W@v8@fmt@@@34@Vlocale_ref@234@@Z@@detail@v8@fmt@@YAPEB_WPEB_W0AEAUformat_handler@?1???$vformat_to@_W@234@YAXAEAV?$buffer@_W@234@V?$basic_string_view@_W@34@V?$basic_format_args@V?$basic_format_context@V?$back_insert_iterator@V?$buffer@_W@detail@v8@fmt@@@std@@_W@v8@fmt@@@34@Vlocale_ref@234@@Z@@Z@QEAAXPEBD@Z 0000000180053960     handles.obj
 0002:0000d960       $cppxdata$?on_error@precision_adapter@?1???$parse_precision@_WAEAV?$specs_checker@V?$specs_handler@_W@detail@v8@fmt@@@detail@v8@fmt@@@detail@v8@fmt@@YAPEB_WPEB_W0AEAV?$specs_checker@V?$specs_handler@_W@detail@v8@fmt@@@234@@Z@QEAAXPEBD@Z 0000000180053960     handles.obj
 0002:0000d960       $cppxdata$?on_error@width_adapter@?1???$parse_width@_WAEAV?$specs_checker@V?$specs_handler@_W@detail@v8@fmt@@@detail@v8@fmt@@@detail@v8@fmt@@YAPEB_WPEB_W0AEAV?$specs_checker@V?$specs_handler@_W@detail@v8@fmt@@@234@@Z@QEAAXPEBD@Z 0000000180053960     handles.obj
 0002:0000d990       $cppxdata$??$parse_replacement_field@_WAEAUformat_handler@?1???$vformat_to@_W@detail@v8@fmt@@YAXAEAV?$buffer@_W@234@V?$basic_string_view@_W@34@V?$basic_format_args@V?$basic_format_context@V?$back_insert_iterator@V?$buffer@_W@detail@v8@fmt@@@std@@_W@v8@fmt@@@34@Vlocale_ref@234@@Z@@detail@v8@fmt@@YAPEB_WPEB_W0AEAUformat_handler@?1???$vformat_to@_W@012@YAXAEAV?$buffer@_W@012@V?$basic_string_view@_W@12@V?$basic_format_args@V?$basic_format_context@V?$back_insert_iterator@V?$buffer@_W@detail@v8@fmt@@@std@@_W@v8@fmt@@@12@Vlocale_ref@012@@Z@@Z 0000000180053990     handles.obj
 0002:0000d9c0       $cppxdata$??$parse_precision@_WAEAV?$specs_checker@V?$specs_handler@_W@detail@v8@fmt@@@detail@v8@fmt@@@detail@v8@fmt@@YAPEB_WPEB_W0AEAV?$specs_checker@V?$specs_handler@_W@detail@v8@fmt@@@012@@Z 00000001800539c0     handles.obj
 0002:0000d9f0       $cppxdata$??$parse_width@_WAEAV?$specs_checker@V?$specs_handler@_W@detail@v8@fmt@@@detail@v8@fmt@@@detail@v8@fmt@@YAPEB_WPEB_W0AEAV?$specs_checker@V?$specs_handler@_W@detail@v8@fmt@@@012@@Z 00000001800539f0     handles.obj
 0002:0000da20       $cppxdata$??$parse_align@_WAEAV?$specs_checker@V?$specs_handler@_W@detail@v8@fmt@@@detail@v8@fmt@@@detail@v8@fmt@@YAPEB_WPEB_W0AEAV?$specs_checker@V?$specs_handler@_W@detail@v8@fmt@@@012@@Z 0000000180053a20     handles.obj
 0002:0000da50       $cppxdata$?require_numeric_argument@?$specs_checker@V?$specs_handler@_W@detail@v8@fmt@@@detail@v8@fmt@@AEAAXXZ 0000000180053a50     handles.obj
 0002:0000da80       $cppxdata$??$vformat@_W$0A@@v8@fmt@@YA?AV?$basic_string@_WU?$char_traits@_W@std@@V?$allocator@_W@2@@std@@V?$basic_string_view@_W@01@V?$basic_format_args@V?$basic_format_context@V?$back_insert_iterator@V?$buffer@_W@detail@v8@fmt@@@std@@_W@v8@fmt@@@01@@Z 0000000180053a80     handles.obj
 0002:0000dab0       $cppxdata$??Rwriter@?1???$parse_format_string@$0A@_WUformat_handler@?1???$vformat_to@_W@detail@v8@fmt@@YAXAEAV?$buffer@_W@234@V?$basic_string_view@_W@34@V?$basic_format_args@V?$basic_format_context@V?$back_insert_iterator@V?$buffer@_W@detail@v8@fmt@@@std@@_W@v8@fmt@@@34@Vlocale_ref@234@@Z@@detail@v8@fmt@@YAXV?$basic_string_view@_W@23@$$QEAUformat_handler@?1???$vformat_to@_W@123@YAXAEAV?$buffer@_W@123@0V?$basic_format_args@V?$basic_format_context@V?$back_insert_iterator@V?$buffer@_W@detail@v8@fmt@@@std@@_W@v8@fmt@@@23@Vlocale_ref@123@@Z@@Z@QEAAXPEB_W5@Z 0000000180053ab0     handles.obj
 0002:0000dae0       $cppxdata$??$parse_format_string@$0A@_WUformat_handler@?1???$vformat_to@_W@detail@v8@fmt@@YAXAEAV?$buffer@_W@234@V?$basic_string_view@_W@34@V?$basic_format_args@V?$basic_format_context@V?$back_insert_iterator@V?$buffer@_W@detail@v8@fmt@@@std@@_W@v8@fmt@@@34@Vlocale_ref@234@@Z@@detail@v8@fmt@@YAXV?$basic_string_view@_W@12@$$QEAUformat_handler@?1???$vformat_to@_W@012@YAXAEAV?$buffer@_W@012@0V?$basic_format_args@V?$basic_format_context@V?$back_insert_iterator@V?$buffer@_W@detail@v8@fmt@@@std@@_W@v8@fmt@@@12@Vlocale_ref@012@@Z@@Z 0000000180053ae0     handles.obj
 0002:0000db10       $cppxdata$??$visit_format_arg@AEAU?$arg_formatter@_W@detail@v8@fmt@@V?$basic_format_context@V?$back_insert_iterator@V?$buffer@_W@detail@v8@fmt@@@std@@_W@34@@v8@fmt@@YA?AV?$back_insert_iterator@V?$buffer@_W@detail@v8@fmt@@@std@@AEAU?$arg_formatter@_W@detail@01@AEBV?$basic_format_arg@V?$basic_format_context@V?$back_insert_iterator@V?$buffer@_W@detail@v8@fmt@@@std@@_W@v8@fmt@@@01@@Z 0000000180053b10     handles.obj
 0002:0000db40       $cppxdata$??$get_arg@V?$basic_format_context@V?$back_insert_iterator@V?$buffer@_W@detail@v8@fmt@@@std@@_W@v8@fmt@@H@detail@v8@fmt@@YA?AV?$basic_format_arg@V?$basic_format_context@V?$back_insert_iterator@V?$buffer@_W@detail@v8@fmt@@@std@@_W@v8@fmt@@@12@AEAV?$basic_format_context@V?$back_insert_iterator@V?$buffer@_W@detail@v8@fmt@@@std@@_W@12@H@Z 0000000180053b40     handles.obj
 0002:0000db70       $cppxdata$??$visit_format_arg@U?$default_arg_formatter@_W@detail@v8@fmt@@V?$basic_format_context@V?$back_insert_iterator@V?$buffer@_W@detail@v8@fmt@@@std@@_W@34@@v8@fmt@@YA?AV?$back_insert_iterator@V?$buffer@_W@detail@v8@fmt@@@std@@$$QEAU?$default_arg_formatter@_W@detail@01@AEBV?$basic_format_arg@V?$basic_format_context@V?$back_insert_iterator@V?$buffer@_W@detail@v8@fmt@@@std@@_W@v8@fmt@@@01@@Z 0000000180053b70     handles.obj
 0002:0000dba0       $cppxdata$?next_arg_id@?$basic_format_parse_context@_WUerror_handler@detail@v8@fmt@@@v8@fmt@@QEAAHXZ 0000000180053ba0     handles.obj
 0002:0000dbd0       $cppxdata$?check_arg_id@?$basic_format_parse_context@_WUerror_handler@detail@v8@fmt@@@v8@fmt@@QEAAXH@Z 0000000180053bd0     handles.obj
 0002:0000dc00       $cppxdata$??0?$basic_string@_WU?$char_traits@_W@std@@V?$allocator@_W@2@@std@@QEAA@XZ 0000000180053c00     handles.obj
 0002:0000dc30       $cppxdata$?PrintHandleInfo@@YA_NKPEAX_NPEAVPerfThread@@@Z 0000000180053c30     handles.obj
 0002:0000dc60       $cppxdata$?GetNameByType@@YA?AV?$basic_string@_WU?$char_traits@_W@std@@V?$allocator@_W@2@@std@@PEAXGPEAVPerfThread@@@Z 0000000180053c60     handles.obj
 0002:0000dc90       $cppxdata$??R<lambda_1>@?1??GetUserAccountID@@YA@XZ@QEBA?AV?$basic_string@_WU?$char_traits@_W@std@@V?$allocator@_W@2@@std@@XZ 0000000180053c90     handles.obj
 0002:0000dcc0       $cppxdata$?GetFileName@@YA?AV?$basic_string@_WU?$char_traits@_W@std@@V?$allocator@_W@2@@std@@PEAX@Z 0000000180053cc0     handles.obj
 0002:0000dcf0       $cppxdata$??$decimal_point@_W@detail@v8@fmt@@YA_WVlocale_ref@012@@Z 0000000180053cf0     handles.obj
 0002:0000dd20       $cppxdata$?Read@options@@QEAAXXZ 0000000180053d20     Pcfg.obj
 0002:0000dd50       $cppxdata$?Write@options@@QEBAXXZ 0000000180053d50     Pcfg.obj
 0002:0000dd80       $cppxdata$?Config@@YAHXZ   0000000180053d80     Pcfg.obj
 0002:0000ddb0       $cppxdata$??1PluginDialogBuilder@@QEAA@XZ 0000000180053db0     Pcfg.obj
 0002:0000dde0       $cppxdata$??1PluginSettings@@QEAA@XZ 0000000180053de0     Pcfg.obj
 0002:0000de10       $cppxdata$??$_Uninitialized_copy@PEBUmode@@V?$allocator@Umode@@@std@@@std@@YAPEAUmode@@QEBU1@0PEAU1@AEAV?$allocator@Umode@@@0@@Z 0000000180053e10     Pclass.obj
 0002:0000de40       $cppxdata$?_Umove@?$vector@V?$basic_string@_WU?$char_traits@_W@std@@V?$allocator@_W@2@@std@@V?$allocator@V?$basic_string@_WU?$char_traits@_W@std@@V?$allocator@_W@2@@std@@@2@@std@@AEAAPEAV?$basic_string@_WU?$char_traits@_W@std@@V?$allocator@_W@2@@2@PEAV32@00@Z 0000000180053e40     Pclass.obj
 0002:0000de70       $cppxdata$??$_Try_emplace@AEBK$$V@?$_Hash@V?$_Umap_traits@KPEAUHWND__@@V?$_Uhash_compare@KU?$hash@K@std@@U?$equal_to@K@2@@std@@V?$allocator@U?$pair@$$CBKPEAUHWND__@@@std@@@3@$0A@@std@@@std@@IEAA?AU?$pair@PEAU?$_List_node@U?$pair@$$CBKPEAUHWND__@@@std@@PEAX@std@@_N@1@AEBK@Z 0000000180053e70     Pclass.obj
 0002:0000dea0       $cppxdata$??$_Emplace_reallocate@V?$basic_string@_WU?$char_traits@_W@std@@V?$allocator@_W@2@@std@@@?$vector@V?$basic_string@_WU?$char_traits@_W@std@@V?$allocator@_W@2@@std@@V?$allocator@V?$basic_string@_WU?$char_traits@_W@std@@V?$allocator@_W@2@@std@@@2@@std@@QEAAPEAV?$basic_string@_WU?$char_traits@_W@std@@V?$allocator@_W@2@@1@QEAV21@$$QEAV21@@Z 0000000180053ea0     Pclass.obj
 0002:0000ded0       $cppxdata$??R?$default_delete@VWMIConnection@@@std@@QEBAXPEAVWMIConnection@@@Z 0000000180053ed0     Pclass.obj
 0002:0000df00       $cppxdata$?_Reallocate_exactly@?$vector@V?$basic_string@_WU?$char_traits@_W@std@@V?$allocator@_W@2@@std@@V?$allocator@V?$basic_string@_WU?$char_traits@_W@std@@V?$allocator@_W@2@@std@@@2@@std@@AEAAX_K@Z 0000000180053f00     Pclass.obj
 0002:0000df30       $cppxdata$?Compare@Plist@@QEBAHPEBUPluginPanelItem@@0I@Z 0000000180053f30     Pclass.obj
 0002:0000df60       $cppxdata$?PrintOwnerInfo@Plist@@AEAAXPEAXK@Z 0000000180053f60     Pclass.obj
 0002:0000df90       $cppxdata$?PrintVersionInfo@Plist@@CAXPEAXPEB_W@Z 0000000180053f90     Pclass.obj
 0002:0000dfc0       $cppxdata$?GetVersionInfo@Plist@@SA_NPEB_WAEAV?$unique_ptr@$$BY0A@DU?$default_delete@$$BY0A@D@std@@@std@@AEAPEB_W2@Z 0000000180053fc0     Pclass.obj
 0002:0000dff0       $cppxdata$?ProcessKey@Plist@@QEAAHPEBU_INPUT_RECORD@@@Z 0000000180053ff0     Pclass.obj
 0002:0000e020       $cppxdata$?Connect@Plist@@QEAA_NPEB_W00@Z 0000000180054020     Pclass.obj
 0002:0000e050       $cppxdata$?DeleteFiles@Plist@@QEAAHPEAUPluginPanelItem@@_K1@Z 0000000180054050     Pclass.obj
 0002:0000e080       $cppxdata$?GetFiles@Plist@@QEAAHPEAUPluginPanelItem@@_KHPEAPEB_W1AEAUoptions@@@Z 0000000180054080     Pclass.obj
 0002:0000e0b0       $cppxdata$?DumpNTCounters@@YAXPEAXAEAVPerfThread@@KK@Z 00000001800540b0     Pclass.obj
 0002:0000e0e0       $cppxdata$?window_ex_style@@YA@PEAUHWND__@@@Z 00000001800540e0     Pclass.obj
 0002:0000e110       $cppxdata$?window_style@@YA@PEAUHWND__@@@Z 0000000180054110     Pclass.obj
 0002:0000e140       $cppxdata$?GetFindData@Plist@@QEAAHAEAPEAUPluginPanelItem@@AEA_K_K@Z 0000000180054140     Pclass.obj
 0002:0000e170       $cppxdata$?GetOpenPanelInfo@Plist@@QEAAXPEAUOpenPanelInfo@@@Z 0000000180054170     Pclass.obj
 0002:0000e1a0       $cppxdata$?generate_titles@@YAXAEBV?$basic_string@_WU?$char_traits@_W@std@@V?$allocator@_W@2@@std@@AEAUPanelMode@@@Z 00000001800541a0     Pclass.obj
 0002:0000e1d0       $cppxdata$?TranslateMode@@YA_NAEBV?$basic_string@_WU?$char_traits@_W@std@@V?$allocator@_W@2@@std@@AEAV12@@Z 00000001800541d0     Pclass.obj
 0002:0000e200       $cppxdata$??0Plist@@QEAA@XZ 0000000180054200     Pclass.obj
 0002:0000e230       $cppxdata$?PrintTitle@@YA?AV?$basic_string@_WU?$char_traits@_W@std@@V?$allocator@_W@2@@std@@V?$basic_string_view@_WU?$char_traits@_W@std@@@2@@Z 0000000180054230     Pclass.obj
 0002:0000e260       $cppxdata$?ui64toa_width@@YA?AV?$basic_string@_WU?$char_traits@_W@std@@V?$allocator@_W@2@@std@@_KI_N@Z 0000000180054260     Pclass.obj
 0002:0000e290       $cppxdata$?InitializePanelModes@Plist@@SAXXZ 0000000180054290     Pclass.obj
 0002:0000e2c0       $cppxdata$?SavePanelModes@Plist@@SAXXZ 00000001800542c0     Pclass.obj
 0002:0000e2f0       $cppxdata$??0ProcessPerfData@@QEAA@$$QEAU0@@Z 00000001800542f0     perfthread.obj
 0002:0000e320       $cppxdata$??0ProcessPerfData@@QEAA@AEBU0@@Z 0000000180054320     perfthread.obj
 0002:0000e350       $cppxdata$??$transform@V?$_List_const_iterator@V?$_List_val@U?$_List_simple_types@U?$pair@$$CBKUProcessPerfData@@@std@@@std@@@std@@@std@@V?$back_insert_iterator@V?$vector@UProcessPerfData@@V?$allocator@UProcessPerfData@@@std@@@std@@@2@V<lambda_1>@?2??RefreshWMIData@PerfThread@@AEAAXXZ@@std@@YA?AV?$back_insert_iterator@V?$vector@UProcessPerfData@@V?$allocator@UProcessPerfData@@@std@@@std@@@0@V?$_List_const_iterator@V?$_List_val@U?$_List_simple_types@U?$pair@$$CBKUProcessPerfData@@@std@@@std@@@std@@@0@0V10@V<lambda_1>@?2??RefreshWMIData@PerfThread@@AEAAXXZ@@Z 0000000180054350     perfthread.obj
 0002:0000e380       $cppxdata$??$emplace@AEBKUProcessPerfData@@@?$_Hash@V?$_Umap_traits@KUProcessPerfData@@V?$_Uhash_compare@KU?$hash@K@std@@U?$equal_to@K@2@@std@@V?$allocator@U?$pair@$$CBKUProcessPerfData@@@std@@@3@$00@std@@@std@@QEAA?AV?$_List_iterator@V?$_List_val@U?$_List_simple_types@U?$pair@$$CBKUProcessPerfData@@@std@@@std@@@std@@@1@AEBK$$QEAUProcessPerfData@@@Z 0000000180054380     perfthread.obj
 0002:0000e3b0       $cppxdata$??0?$unordered_multimap@KUProcessPerfData@@U?$hash@K@std@@U?$equal_to@K@3@V?$allocator@U?$pair@$$CBKUProcessPerfData@@@std@@@3@@std@@QEAA@XZ 00000001800543b0     perfthread.obj
 0002:0000e3e0       $cppxdata$?RefreshWMIData@PerfThread@@AEAAXXZ 00000001800543e0     perfthread.obj
 0002:0000e410       $cppxdata$?Refresh@PerfThread@@AEAAXXZ 0000000180054410     perfthread.obj
 0002:0000e440       $cppxdata$??1PerfThread@@QEAA@XZ 0000000180054440     perfthread.obj
 0002:0000e470       $cppxdata$??0PerfThread@@QEAA@PEAVPlist@@PEB_W11@Z 0000000180054470     perfthread.obj
 0002:0000e4a0       $cppxdata$??$insert@V?$_List_unchecked_const_iterator@V?$_List_val@U?$_List_simple_types@U?$pair@$$CBKUProcessPerfData@@@std@@@std@@@std@@U_Iterator_base0@2@@std@@@?$_Hash@V?$_Umap_traits@KUProcessPerfData@@V?$_Uhash_compare@KU?$hash@K@std@@U?$equal_to@K@2@@std@@V?$allocator@U?$pair@$$CBKUProcessPerfData@@@std@@@3@$00@std@@@std@@QEAAXV?$_List_unchecked_const_iterator@V?$_List_val@U?$_List_simple_types@U?$pair@$$CBKUProcessPerfData@@@std@@@std@@@std@@U_Iterator_base0@2@@1@0@Z 00000001800544a0     Plist.obj
 0002:0000e4d0       $cppxdata$??$print_module@PEAX@@YAXQEAXPEAXKAEAUoptions@@AEBV?$function@$$A6A_NPEA_W_K@Z@std@@@Z 00000001800544d0     Plist.obj
 0002:0000e500       $cppxdata$?read_string@?$ipc_functions@$0A@@@SA?AV?$basic_string@_WU?$char_traits@_W@std@@V?$allocator@_W@2@@std@@PEAXAEBUUNICODE_STRING_SAME@detail@@@Z 0000000180054500     Plist.obj
 0002:0000e530       $cppxdata$?GetOpenProcessData@?$ipc_functions@$0A@@@SAXPEAXPEAV?$basic_string@_WU?$char_traits@_W@std@@V?$allocator@_W@2@@std@@1111@Z 0000000180054530     Plist.obj
 0002:0000e560       $cppxdata$?PrintModules@?$ipc_functions@$0A@@@SAXPEAX0AEAUoptions@@@Z 0000000180054560     Plist.obj
 0002:0000e590       $cppxdata$?print_module_impl@@YAXQEAXAEBV?$basic_string@_WU?$char_traits@_W@std@@V?$allocator@_W@2@@std@@KAEBUoptions@@AEBV?$function@$$A6A_NPEA_W_K@Z@2@@Z 0000000180054590     Plist.obj
 0002:0000e5c0       $cppxdata$?GetList@@YA_NAEAPEAUPluginPanelItem@@AEA_KAEAVPerfThread@@@Z 00000001800545c0     Plist.obj
 0002:0000e5f0       $cppxdata$?KillProcess@@YA_NKPEAUHWND__@@@Z 00000001800545f0     Plist.obj
 0002:0000e620       $cppxdata$?PrintModules@@YAXPEAXKAEAUoptions@@@Z 0000000180054620     Plist.obj
 0002:0000e650       $cppxdata$?PrintNTCurDirAndEnv@@YAXPEAX0H@Z 0000000180054650     Plist.obj
 0002:0000e680       $cppxdata$?WinError@@YAHPEB_W@Z 0000000180054680     Pmix.obj
 0002:0000e6b0       $cppxdata$??1?$unique_ptr@UIWbemClassObject@@Ucom_closer@@@std@@QEAA@XZ 00000001800546b0     wmi.obj
 0002:0000e6b0       $cppxdata$??1?$unique_ptr@UIWbemLocator@@Ucom_closer@@@std@@QEAA@XZ 00000001800546b0     wmi.obj
 0002:0000e6e0       $cppxdata$??1?$ptr_setter@V?$unique_ptr@UIWbemClassObject@@Ucom_closer@@@std@@@@QEAA@XZ 00000001800546e0     wmi.obj
 0002:0000e710       $cppxdata$?GetProcessProperty@WMIConnection@@AEAA_NKPEB_WAEBV?$function@$$A6AXAEBUtagVARIANT@@@Z@std@@@Z 0000000180054710     wmi.obj
 0002:0000e740       $cppxdata$?ExecMethod@WMIConnection@@AEAAHKPEB_W0K@Z 0000000180054740     wmi.obj
 0002:0000e770       $cppxdata$?GetProcessSessionId@WMIConnection@@QEAAKK@Z 0000000180054770     wmi.obj
 0002:0000e7a0       $cppxdata$?GetProcessUserSid@WMIConnection@@QEAA?AV?$basic_string@_WU?$char_traits@_W@std@@V?$allocator@_W@2@@std@@K@Z 00000001800547a0     wmi.obj
 0002:0000e7d0       $cppxdata$?GetProcessOwner@WMIConnection@@QEAA?AV?$basic_string@_WU?$char_traits@_W@std@@V?$allocator@_W@2@@std@@KPEAV23@@Z 00000001800547d0     wmi.obj
 0002:0000e800       $cppxdata$?Connect@WMIConnection@@QEAA_NPEB_W00@Z 0000000180054800     wmi.obj
 0002:0000e830       $cppxdata$??1WMIConnection@@QEAA@XZ 0000000180054830     wmi.obj
 0002:0000e860       $cppxdata$ProcessPanelEventW 0000000180054860     Proclist.obj
 0002:0000f790       ??_R2?$_Func_impl_no_alloc@V<lambda_3>@?N@??PrintModules@@YAXPEAXKAEAUoptions@@@Z@_NPEA_W_K@std@@8 0000000180055790     Plist.obj
 0002:0000f7a8       ??_R3?$_Func_impl_no_alloc@V<lambda_3>@?N@??PrintModules@@YAXPEAXKAEAUoptions@@@Z@_NPEA_W_K@std@@8 00000001800557a8     Plist.obj
 0002:0000f800       ??_R1A@?0A@EA@?$_Func_impl_no_alloc@V<lambda_3>@?N@??PrintModules@@YAXPEAXKAEAUoptions@@@Z@_NPEA_W_K@std@@8 0000000180055800     Plist.obj
 0002:0000f890       ??_R4?$_Func_impl_no_alloc@V<lambda_3>@?N@??PrintModules@@YAXPEAXKAEAUoptions@@@Z@_NPEA_W_K@std@@6B@ 0000000180055890     Plist.obj
 0002:0000f8e0       ??_R3?$_Func_impl_no_alloc@V<lambda_1>@?1??GetProcessString@WMIConnection@@AEAA?AV?$basic_string@_WU?$char_traits@_W@std@@V?$allocator@_W@2@@std@@KPEB_W@Z@XAEBUtagVARIANT@@@std@@8 00000001800558e0     wmi.obj
 0002:0000f8f8       ??_R2?$_Func_impl_no_alloc@V<lambda_1>@?1??GetProcessInt@WMIConnection@@AEAAKKPEB_W@Z@XAEBUtagVARIANT@@@std@@8 00000001800558f8     wmi.obj
 0002:0000f910       ??_R4?$_Func_impl_no_alloc@V<lambda_1>@?1??GetProcessString@WMIConnection@@AEAA?AV?$basic_string@_WU?$char_traits@_W@std@@V?$allocator@_W@2@@std@@KPEB_W@Z@XAEBUtagVARIANT@@@std@@6B@ 0000000180055910     wmi.obj
 0002:0000f960       ??_R1A@?0A@EA@?$_Func_impl_no_alloc@V<lambda_1>@?1??GetProcessInt@WMIConnection@@AEAAKKPEB_W@Z@XAEBUtagVARIANT@@@std@@8 0000000180055960     wmi.obj
 0002:0000f998       ??_R4?$_Func_impl_no_alloc@V<lambda_1>@?1??GetProcessInt@WMIConnection@@AEAAKKPEB_W@Z@XAEBUtagVARIANT@@@std@@6B@ 0000000180055998     wmi.obj
 0002:0000f9d8       ??_R3?$_Func_impl_no_alloc@V<lambda_1>@?1??GetProcessInt@WMIConnection@@AEAAKKPEB_W@Z@XAEBUtagVARIANT@@@std@@8 00000001800559d8     wmi.obj
 0002:0000f9f0       ??_R2?$_Func_impl_no_alloc@V<lambda_1>@?1??GetProcessString@WMIConnection@@AEAA?AV?$basic_string@_WU?$char_traits@_W@std@@V?$allocator@_W@2@@std@@KPEB_W@Z@XAEBUtagVARIANT@@@std@@8 00000001800559f0     wmi.obj
 0002:0000fa08       ??_R1A@?0A@EA@?$_Func_impl_no_alloc@V<lambda_1>@?1??GetProcessString@WMIConnection@@AEAA?AV?$basic_string@_WU?$char_traits@_W@std@@V?$allocator@_W@2@@std@@KPEB_W@Z@XAEBUtagVARIANT@@@std@@8 0000000180055a08     wmi.obj
 0002:0000fde0       $unwind$?WriteToFile@@YA_KPEAXAEBV?$basic_string_view@_WU?$char_traits@_W@std@@@std@@@Z 0000000180055de0     fileio.obj
 0002:0000fdf0       $unwind$??1mode@@QEAA@XZ   0000000180055df0     fileio.obj
 0002:0000fdfc       $unwind$??1columns@@QEAA@XZ 0000000180055dfc     fileio.obj
 0002:0000fe08       $unwind$?_Throw_bad_array_new_length@std@@YAXXZ 0000000180055e08     format.obj
 0002:0000fe08       $unwind$?_Throw_bad_cast@std@@YAXXZ 0000000180055e08     format.obj
 0002:0000fe10       $unwind$?on_error@error_handler@detail@v8@fmt@@QEAAXPEBD@Z 0000000180055e10     format.obj
 0002:0000fe10       $unwind$?on_error@?$specs_handler@_W@detail@v8@fmt@@QEAAXPEBD@Z 0000000180055e10     handles.obj
 0002:0000fe24       $stateUnwindMap$??$?RH$0A@@?$precision_checker@Uerror_handler@detail@v8@fmt@@@detail@v8@fmt@@QEAA_KH@Z 0000000180055e24     format.obj
 0002:0000fe24       $stateUnwindMap$??$?RH$0A@@?$width_checker@Uerror_handler@detail@v8@fmt@@@detail@v8@fmt@@QEAA_KH@Z 0000000180055e24     format.obj
 0002:0000fe24       $stateUnwindMap$??$?RM$0A@@?$precision_checker@Uerror_handler@detail@v8@fmt@@@detail@v8@fmt@@QEAA_KM@Z 0000000180055e24     format.obj
 0002:0000fe24       $stateUnwindMap$??$?RM$0A@@?$width_checker@Uerror_handler@detail@v8@fmt@@@detail@v8@fmt@@QEAA_KM@Z 0000000180055e24     format.obj
 0002:0000fe24       $stateUnwindMap$??$?RN$0A@@?$precision_checker@Uerror_handler@detail@v8@fmt@@@detail@v8@fmt@@QEAA_KN@Z 0000000180055e24     format.obj
 0002:0000fe24       $stateUnwindMap$??$?RN$0A@@?$width_checker@Uerror_handler@detail@v8@fmt@@@detail@v8@fmt@@QEAA_KN@Z 0000000180055e24     format.obj
 0002:0000fe24       $stateUnwindMap$??$?RO$0A@@?$precision_checker@Uerror_handler@detail@v8@fmt@@@detail@v8@fmt@@QEAA_KO@Z 0000000180055e24     format.obj
 0002:0000fe24       $stateUnwindMap$??$?RO$0A@@?$width_checker@Uerror_handler@detail@v8@fmt@@@detail@v8@fmt@@QEAA_KO@Z 0000000180055e24     format.obj
 0002:0000fe24       $stateUnwindMap$??$?RPEBX$0A@@?$precision_checker@Uerror_handler@detail@v8@fmt@@@detail@v8@fmt@@QEAA_KPEBX@Z 0000000180055e24     format.obj
 0002:0000fe24       $stateUnwindMap$??$?RPEBX$0A@@?$width_checker@Uerror_handler@detail@v8@fmt@@@detail@v8@fmt@@QEAA_KPEBX@Z 0000000180055e24     format.obj
 0002:0000fe24       $stateUnwindMap$??$?RUmonostate@v8@fmt@@$0A@@?$precision_checker@Uerror_handler@detail@v8@fmt@@@detail@v8@fmt@@QEAA_KUmonostate@23@@Z 0000000180055e24     format.obj
 0002:0000fe24       $stateUnwindMap$??$?RUmonostate@v8@fmt@@$0A@@?$width_checker@Uerror_handler@detail@v8@fmt@@@detail@v8@fmt@@QEAA_KUmonostate@23@@Z 0000000180055e24     format.obj
 0002:0000fe24       $stateUnwindMap$??$?R_J$0A@@?$precision_checker@Uerror_handler@detail@v8@fmt@@@detail@v8@fmt@@QEAA_K_J@Z 0000000180055e24     format.obj
 0002:0000fe24       $stateUnwindMap$??$?R_J$0A@@?$width_checker@Uerror_handler@detail@v8@fmt@@@detail@v8@fmt@@QEAA_K_J@Z 0000000180055e24     format.obj
 0002:0000fe24       $stateUnwindMap$??$?R_N$0A@@?$precision_checker@Uerror_handler@detail@v8@fmt@@@detail@v8@fmt@@QEAA_K_N@Z 0000000180055e24     format.obj
 0002:0000fe24       $stateUnwindMap$??$?R_N$0A@@?$width_checker@Uerror_handler@detail@v8@fmt@@@detail@v8@fmt@@QEAA_K_N@Z 0000000180055e24     format.obj
 0002:0000fe24       $stateUnwindMap$?on_error@error_handler@detail@v8@fmt@@QEAAXPEBD@Z 0000000180055e24     format.obj
 0002:0000fe24       $stateUnwindMap$?throw_format_error@detail@v8@fmt@@YAXPEBD@Z 0000000180055e24     format.obj
 0002:0000fe24       $stateUnwindMap$??$do_parse_arg_id@_WAEAUid_adapter@?1???$parse_replacement_field@_WAEAUformat_handler@?1???$vformat_to@_W@detail@v8@fmt@@YAXAEAV?$buffer@_W@234@V?$basic_string_view@_W@34@V?$basic_format_args@V?$basic_format_context@V?$back_insert_iterator@V?$buffer@_W@detail@v8@fmt@@@std@@_W@v8@fmt@@@34@Vlocale_ref@234@@Z@@detail@v8@fmt@@YAPEB_WPEB_W0AEAUformat_handler@?1???$vformat_to@_W@234@YAXAEAV?$buffer@_W@234@V?$basic_string_view@_W@34@V?$basic_format_args@V?$basic_format_context@V?$back_insert_iterator@V?$buffer@_W@detail@v8@fmt@@@std@@_W@v8@fmt@@@34@Vlocale_ref@234@@Z@@Z@@detail@v8@fmt@@YAPEB_WPEB_W0AEAUid_adapter@?1???$parse_replacement_field@_WAEAUformat_handler@?1???$vformat_to@_W@detail@v8@fmt@@YAXAEAV?$buffer@_W@234@V?$basic_string_view@_W@34@V?$basic_format_args@V?$basic_format_context@V?$back_insert_iterator@V?$buffer@_W@detail@v8@fmt@@@std@@_W@v8@fmt@@@34@Vlocale_ref@234@@Z@@012@YAPEB_W00AEAUformat_handler@?1???$vformat_to@_W@012@YAXAEAV?$buffer@_W@012@V?$basic_string_view@_W@12@V?$basic_format_args@V?$basic_format_context@V?$back_insert_iterator@V?$buffer@_W@detail@v8@fmt@@@std@@_W@v8@fmt@@@12@Vlocale_ref@012@@Z@@Z@@Z 0000000180055e24     handles.obj
 0002:0000fe24       $stateUnwindMap$??$get_arg@V?$basic_format_context@V?$back_insert_iterator@V?$buffer@_W@detail@v8@fmt@@@std@@_W@v8@fmt@@H@detail@v8@fmt@@YA?AV?$basic_format_arg@V?$basic_format_context@V?$back_insert_iterator@V?$buffer@_W@detail@v8@fmt@@@std@@_W@v8@fmt@@@12@AEAV?$basic_format_context@V?$back_insert_iterator@V?$buffer@_W@detail@v8@fmt@@@std@@_W@12@H@Z 0000000180055e24     handles.obj
 0002:0000fe24       $stateUnwindMap$??$write@_WV?$back_insert_iterator@V?$buffer@_W@detail@v8@fmt@@@std@@X$0A@@detail@v8@fmt@@YA?AV?$back_insert_iterator@V?$buffer@_W@detail@v8@fmt@@@std@@V34@PEBXAEBU?$basic_format_specs@_W@12@Vlocale_ref@012@@Z 0000000180055e24     handles.obj
 0002:0000fe24       $stateUnwindMap$??$write_int@_WV?$back_insert_iterator@V?$buffer@_W@detail@v8@fmt@@@std@@I@detail@v8@fmt@@YA?AV?$back_insert_iterator@V?$buffer@_W@detail@v8@fmt@@@std@@V34@U?$write_int_arg@I@012@AEBU?$basic_format_specs@_W@12@Vlocale_ref@012@@Z 0000000180055e24     handles.obj
 0002:0000fe24       $stateUnwindMap$??Rwriter@?1???$parse_format_string@$0A@_WUformat_handler@?1???$vformat_to@_W@detail@v8@fmt@@YAXAEAV?$buffer@_W@234@V?$basic_string_view@_W@34@V?$basic_format_args@V?$basic_format_context@V?$back_insert_iterator@V?$buffer@_W@detail@v8@fmt@@@std@@_W@v8@fmt@@@34@Vlocale_ref@234@@Z@@detail@v8@fmt@@YAXV?$basic_string_view@_W@23@$$QEAUformat_handler@?1???$vformat_to@_W@123@YAXAEAV?$buffer@_W@123@0V?$basic_format_args@V?$basic_format_context@V?$back_insert_iterator@V?$buffer@_W@detail@v8@fmt@@@std@@_W@v8@fmt@@@23@Vlocale_ref@123@@Z@@Z@QEAAXPEB_W5@Z 0000000180055e24     handles.obj
 0002:0000fe24       $stateUnwindMap$?check_arg_id@?$basic_format_parse_context@_WUerror_handler@detail@v8@fmt@@@v8@fmt@@QEAAXH@Z 0000000180055e24     handles.obj
 0002:0000fe24       $stateUnwindMap$?next_arg_id@?$basic_format_parse_context@_WUerror_handler@detail@v8@fmt@@@v8@fmt@@QEAAHXZ 0000000180055e24     handles.obj
 0002:0000fe24       $stateUnwindMap$?on_error@?$specs_handler@_W@detail@v8@fmt@@QEAAXPEBD@Z 0000000180055e24     handles.obj
 0002:0000fe24       $stateUnwindMap$?on_error@id_adapter@?1???$parse_replacement_field@_WAEAUformat_handler@?1???$vformat_to@_W@detail@v8@fmt@@YAXAEAV?$buffer@_W@234@V?$basic_string_view@_W@34@V?$basic_format_args@V?$basic_format_context@V?$back_insert_iterator@V?$buffer@_W@detail@v8@fmt@@@std@@_W@v8@fmt@@@34@Vlocale_ref@234@@Z@@detail@v8@fmt@@YAPEB_WPEB_W0AEAUformat_handler@?1???$vformat_to@_W@234@YAXAEAV?$buffer@_W@234@V?$basic_string_view@_W@34@V?$basic_format_args@V?$basic_format_context@V?$back_insert_iterator@V?$buffer@_W@detail@v8@fmt@@@std@@_W@v8@fmt@@@34@Vlocale_ref@234@@Z@@Z@QEAAXPEBD@Z 0000000180055e24     handles.obj
 0002:0000fe24       $stateUnwindMap$?on_error@precision_adapter@?1???$parse_precision@_WAEAV?$specs_checker@V?$specs_handler@_W@detail@v8@fmt@@@detail@v8@fmt@@@detail@v8@fmt@@YAPEB_WPEB_W0AEAV?$specs_checker@V?$specs_handler@_W@detail@v8@fmt@@@234@@Z@QEAAXPEBD@Z 0000000180055e24     handles.obj
 0002:0000fe24       $stateUnwindMap$?on_error@width_adapter@?1???$parse_width@_WAEAV?$specs_checker@V?$specs_handler@_W@detail@v8@fmt@@@detail@v8@fmt@@@detail@v8@fmt@@YAPEB_WPEB_W0AEAV?$specs_checker@V?$specs_handler@_W@detail@v8@fmt@@@234@@Z@QEAAXPEBD@Z 0000000180055e24     handles.obj
 0002:0000fe24       $stateUnwindMap$?require_numeric_argument@?$specs_checker@V?$specs_handler@_W@detail@v8@fmt@@@detail@v8@fmt@@AEAAXXZ 0000000180055e24     handles.obj
 0002:0000fe30       $ip2state$?on_error@error_handler@detail@v8@fmt@@QEAAXPEBD@Z 0000000180055e30     format.obj
 0002:0000fe30       $ip2state$?on_error@?$specs_handler@_W@detail@v8@fmt@@QEAAXPEBD@Z 0000000180055e30     handles.obj
 0002:0000fe38       $unwind$?dtor$0@?0??Config@@YAHXZ@4HA 0000000180055e38     Pcfg.obj
 0002:0000fe38       $unwind$?dtor$0@?0??Read@options@@QEAAXXZ@4HA 0000000180055e38     Pcfg.obj
 0002:0000fe38       $unwind$?dtor$0@?0??Write@options@@QEBAXXZ@4HA 0000000180055e38     Pcfg.obj
 0002:0000fe38       $unwind$?dtor$0@?0???$_Try_emplace@AEBK$$V@?$_Hash@V?$_Umap_traits@KPEAUHWND__@@V?$_Uhash_compare@KU?$hash@K@std@@U?$equal_to@K@2@@std@@V?$allocator@U?$pair@$$CBKPEAUHWND__@@@std@@@3@$0A@@std@@@std@@IEAA?AU?$pair@PEAU?$_List_node@U?$pair@$$CBKPEAUHWND__@@@std@@PEAX@std@@_N@1@AEBK@Z@4HA 0000000180055e38     Pclass.obj
 0002:0000fe38       $unwind$?dtor$0@?0???$_Uninitialized_copy@PEBUmode@@V?$allocator@Umode@@@std@@@std@@YAPEAUmode@@QEBU1@0PEAU1@AEAV?$allocator@Umode@@@0@@Z@4HA 0000000180055e38     Pclass.obj
 0002:0000fe38       $unwind$?dtor$0@?0??Compare@Plist@@QEBAHPEBUPluginPanelItem@@0I@Z@4HA 0000000180055e38     Pclass.obj
 0002:0000fe38       $unwind$?dtor$0@?0??Connect@Plist@@QEAA_NPEB_W00@Z@4HA 0000000180055e38     Pclass.obj
 0002:0000fe38       $unwind$?dtor$0@?0??DeleteFiles@Plist@@QEAAHPEAUPluginPanelItem@@_K1@Z@4HA 0000000180055e38     Pclass.obj
 0002:0000fe38       $unwind$?dtor$0@?0??DumpNTCounters@@YAXPEAXAEAVPerfThread@@KK@Z@4HA 0000000180055e38     Pclass.obj
 0002:0000fe38       $unwind$?dtor$0@?0??GetFiles@Plist@@QEAAHPEAUPluginPanelItem@@_KHPEAPEB_W1AEAUoptions@@@Z@4HA 0000000180055e38     Pclass.obj
 0002:0000fe38       $unwind$?dtor$0@?0??GetFindData@Plist@@QEAAHAEAPEAUPluginPanelItem@@AEA_K_K@Z@4HA 0000000180055e38     Pclass.obj
 0002:0000fe38       $unwind$?dtor$0@?0??GetOpenPanelInfo@Plist@@QEAAXPEAUOpenPanelInfo@@@Z@4HA 0000000180055e38     Pclass.obj
 0002:0000fe38       $unwind$?dtor$0@?0??InitializePanelModes@Plist@@SAXXZ@4HA 0000000180055e38     Pclass.obj
 0002:0000fe38       $unwind$?dtor$0@?0??PrintOwnerInfo@Plist@@AEAAXPEAXK@Z@4HA 0000000180055e38     Pclass.obj
 0002:0000fe38       $unwind$?dtor$0@?0??PrintTitle@@YA?AV?$basic_string@_WU?$char_traits@_W@std@@V?$allocator@_W@2@@std@@V?$basic_string_view@_WU?$char_traits@_W@std@@@2@@Z@4HA 0000000180055e38     Pclass.obj
 0002:0000fe38       $unwind$?dtor$0@?0??PrintVersionInfo@Plist@@CAXPEAXPEB_W@Z@4HA 0000000180055e38     Pclass.obj
 0002:0000fe38       $unwind$?dtor$0@?0??SavePanelModes@Plist@@SAXXZ@4HA 0000000180055e38     Pclass.obj
 0002:0000fe38       $unwind$?dtor$0@?0??TranslateMode@@YA_NAEBV?$basic_string@_WU?$char_traits@_W@std@@V?$allocator@_W@2@@std@@AEAV12@@Z@4HA 0000000180055e38     Pclass.obj
 0002:0000fe38       $unwind$?dtor$0@?0??generate_titles@@YAXAEBV?$basic_string@_WU?$char_traits@_W@std@@V?$allocator@_W@2@@std@@AEAUPanelMode@@@Z@4HA 0000000180055e38     Pclass.obj
 0002:0000fe38       $unwind$?dtor$0@?0??ui64toa_width@@YA?AV?$basic_string@_WU?$char_traits@_W@std@@V?$allocator@_W@2@@std@@_KI_N@Z@4HA 0000000180055e38     Pclass.obj
 0002:0000fe38       $unwind$?dtor$0@?0??window_ex_style@@YA@PEAUHWND__@@@Z@4HA 0000000180055e38     Pclass.obj
 0002:0000fe38       $unwind$?dtor$0@?0??window_style@@YA@PEAUHWND__@@@Z@4HA 0000000180055e38     Pclass.obj
 0002:0000fe38       $unwind$?dtor$100@?0??InitializePanelModes@Plist@@SAXXZ@4HA 0000000180055e38     Pclass.obj
 0002:0000fe38       $unwind$?dtor$108@?0??InitializePanelModes@Plist@@SAXXZ@4HA 0000000180055e38     Pclass.obj
 0002:0000fe38       $unwind$?dtor$109@?0??InitializePanelModes@Plist@@SAXXZ@4HA 0000000180055e38     Pclass.obj
 0002:0000fe38       $unwind$?dtor$117@?0??InitializePanelModes@Plist@@SAXXZ@4HA 0000000180055e38     Pclass.obj
 0002:0000fe38       $unwind$?dtor$118@?0??InitializePanelModes@Plist@@SAXXZ@4HA 0000000180055e38     Pclass.obj
 0002:0000fe38       $unwind$?dtor$11@?0??GetFiles@Plist@@QEAAHPEAUPluginPanelItem@@_KHPEAPEB_W1AEAUoptions@@@Z@4HA 0000000180055e38     Pclass.obj
 0002:0000fe38       $unwind$?dtor$126@?0??InitializePanelModes@Plist@@SAXXZ@4HA 0000000180055e38     Pclass.obj
 0002:0000fe38       $unwind$?dtor$127@?0??InitializePanelModes@Plist@@SAXXZ@4HA 0000000180055e38     Pclass.obj
 0002:0000fe38       $unwind$?dtor$135@?0??InitializePanelModes@Plist@@SAXXZ@4HA 0000000180055e38     Pclass.obj
 0002:0000fe38       $unwind$?dtor$136@?0??InitializePanelModes@Plist@@SAXXZ@4HA 0000000180055e38     Pclass.obj
 0002:0000fe38       $unwind$?dtor$13@?0??PrintOwnerInfo@Plist@@AEAAXPEAXK@Z@4HA 0000000180055e38     Pclass.obj
 0002:0000fe38       $unwind$?dtor$144@?0??InitializePanelModes@Plist@@SAXXZ@4HA 0000000180055e38     Pclass.obj
 0002:0000fe38       $unwind$?dtor$145@?0??InitializePanelModes@Plist@@SAXXZ@4HA 0000000180055e38     Pclass.obj
 0002:0000fe38       $unwind$?dtor$14@?0??GetFiles@Plist@@QEAAHPEAUPluginPanelItem@@_KHPEAPEB_W1AEAUoptions@@@Z@4HA 0000000180055e38     Pclass.obj
 0002:0000fe38       $unwind$?dtor$153@?0??InitializePanelModes@Plist@@SAXXZ@4HA 0000000180055e38     Pclass.obj
 0002:0000fe38       $unwind$?dtor$154@?0??InitializePanelModes@Plist@@SAXXZ@4HA 0000000180055e38     Pclass.obj
 0002:0000fe38       $unwind$?dtor$162@?0??InitializePanelModes@Plist@@SAXXZ@4HA 0000000180055e38     Pclass.obj
 0002:0000fe38       $unwind$?dtor$163@?0??InitializePanelModes@Plist@@SAXXZ@4HA 0000000180055e38     Pclass.obj
 0002:0000fe38       $unwind$?dtor$16@?0??GetFiles@Plist@@QEAAHPEAUPluginPanelItem@@_KHPEAPEB_W1AEAUoptions@@@Z@4HA 0000000180055e38     Pclass.obj
 0002:0000fe38       $unwind$?dtor$171@?0??InitializePanelModes@Plist@@SAXXZ@4HA 0000000180055e38     Pclass.obj
 0002:0000fe38       $unwind$?dtor$172@?0??InitializePanelModes@Plist@@SAXXZ@4HA 0000000180055e38     Pclass.obj
 0002:0000fe38       $unwind$?dtor$17@?0??InitializePanelModes@Plist@@SAXXZ@4HA 0000000180055e38     Pclass.obj
 0002:0000fe38       $unwind$?dtor$182@?0??InitializePanelModes@Plist@@SAXXZ@4HA 0000000180055e38     Pclass.obj
 0002:0000fe38       $unwind$?dtor$183@?0??InitializePanelModes@Plist@@SAXXZ@4HA 0000000180055e38     Pclass.obj
 0002:0000fe38       $unwind$?dtor$18@?0??GetFiles@Plist@@QEAAHPEAUPluginPanelItem@@_KHPEAPEB_W1AEAUoptions@@@Z@4HA 0000000180055e38     Pclass.obj
 0002:0000fe38       $unwind$?dtor$18@?0??InitializePanelModes@Plist@@SAXXZ@4HA 0000000180055e38     Pclass.obj
 0002:0000fe38       $unwind$?dtor$18@?0??PrintVersionInfo@Plist@@CAXPEAXPEB_W@Z@4HA 0000000180055e38     Pclass.obj
 0002:0000fe38       $unwind$?dtor$1@?0???$_Try_emplace@AEBK$$V@?$_Hash@V?$_Umap_traits@KPEAUHWND__@@V?$_Uhash_compare@KU?$hash@K@std@@U?$equal_to@K@2@@std@@V?$allocator@U?$pair@$$CBKPEAUHWND__@@@std@@@3@$0A@@std@@@std@@IEAA?AU?$pair@PEAU?$_List_node@U?$pair@$$CBKPEAUHWND__@@@std@@PEAX@std@@_N@1@AEBK@Z@4HA 0000000180055e38     Pclass.obj
 0002:0000fe38       $unwind$?dtor$1@?0??Compare@Plist@@QEBAHPEBUPluginPanelItem@@0I@Z@4HA 0000000180055e38     Pclass.obj
 0002:0000fe38       $unwind$?dtor$1@?0??Connect@Plist@@QEAA_NPEB_W00@Z@4HA 0000000180055e38     Pclass.obj
 0002:0000fe38       $unwind$?dtor$1@?0??DeleteFiles@Plist@@QEAAHPEAUPluginPanelItem@@_K1@Z@4HA 0000000180055e38     Pclass.obj
 0002:0000fe38       $unwind$?dtor$1@?0??GetFiles@Plist@@QEAAHPEAUPluginPanelItem@@_KHPEAPEB_W1AEAUoptions@@@Z@4HA 0000000180055e38     Pclass.obj
 0002:0000fe38       $unwind$?dtor$1@?0??GetFindData@Plist@@QEAAHAEAPEAUPluginPanelItem@@AEA_K_K@Z@4HA 0000000180055e38     Pclass.obj
 0002:0000fe38       $unwind$?dtor$1@?0??GetVersionInfo@Plist@@SA_NPEB_WAEAV?$unique_ptr@$$BY0A@DU?$default_delete@$$BY0A@D@std@@@std@@AEAPEB_W2@Z@4HA 0000000180055e38     Pclass.obj
 0002:0000fe38       $unwind$?dtor$1@?0??PrintOwnerInfo@Plist@@AEAAXPEAXK@Z@4HA 0000000180055e38     Pclass.obj
 0002:0000fe38       $unwind$?dtor$1@?0??PrintVersionInfo@Plist@@CAXPEAXPEB_W@Z@4HA 0000000180055e38     Pclass.obj
 0002:0000fe38       $unwind$?dtor$1@?0??SavePanelModes@Plist@@SAXXZ@4HA 0000000180055e38     Pclass.obj
 0002:0000fe38       $unwind$?dtor$20@?0??GetFiles@Plist@@QEAAHPEAUPluginPanelItem@@_KHPEAPEB_W1AEAUoptions@@@Z@4HA 0000000180055e38     Pclass.obj
 0002:0000fe38       $unwind$?dtor$21@?0???$_Uninitialized_copy@PEBUmode@@V?$allocator@Umode@@@std@@@std@@YAPEAUmode@@QEBU1@0PEAU1@AEAV?$allocator@Umode@@@0@@Z@4HA 0000000180055e38     Pclass.obj
 0002:0000fe38       $unwind$?dtor$22@?0??GetFiles@Plist@@QEAAHPEAUPluginPanelItem@@_KHPEAPEB_W1AEAUoptions@@@Z@4HA 0000000180055e38     Pclass.obj
 0002:0000fe38       $unwind$?dtor$23@?0???$_Uninitialized_copy@PEBUmode@@V?$allocator@Umode@@@std@@@std@@YAPEAUmode@@QEBU1@0PEAU1@AEAV?$allocator@Umode@@@0@@Z@4HA 0000000180055e38     Pclass.obj
 0002:0000fe38       $unwind$?dtor$23@?0??GetFiles@Plist@@QEAAHPEAUPluginPanelItem@@_KHPEAPEB_W1AEAUoptions@@@Z@4HA 0000000180055e38     Pclass.obj
 0002:0000fe38       $unwind$?dtor$26@?0??GetFiles@Plist@@QEAAHPEAUPluginPanelItem@@_KHPEAPEB_W1AEAUoptions@@@Z@4HA 0000000180055e38     Pclass.obj
 0002:0000fe38       $unwind$?dtor$26@?0??InitializePanelModes@Plist@@SAXXZ@4HA 0000000180055e38     Pclass.obj
 0002:0000fe38       $unwind$?dtor$27@?0??GetFiles@Plist@@QEAAHPEAUPluginPanelItem@@_KHPEAPEB_W1AEAUoptions@@@Z@4HA 0000000180055e38     Pclass.obj
 0002:0000fe38       $unwind$?dtor$27@?0??InitializePanelModes@Plist@@SAXXZ@4HA 0000000180055e38     Pclass.obj
 0002:0000fe38       $unwind$?dtor$28@?0??GetFiles@Plist@@QEAAHPEAUPluginPanelItem@@_KHPEAPEB_W1AEAUoptions@@@Z@4HA 0000000180055e38     Pclass.obj
 0002:0000fe38       $unwind$?dtor$28@?0??PrintOwnerInfo@Plist@@AEAAXPEAXK@Z@4HA 0000000180055e38     Pclass.obj
 0002:0000fe38       $unwind$?dtor$29@?0??GetFiles@Plist@@QEAAHPEAUPluginPanelItem@@_KHPEAPEB_W1AEAUoptions@@@Z@4HA 0000000180055e38     Pclass.obj
 0002:0000fe38       $unwind$?dtor$2@?0??GetFiles@Plist@@QEAAHPEAUPluginPanelItem@@_KHPEAPEB_W1AEAUoptions@@@Z@4HA 0000000180055e38     Pclass.obj
 0002:0000fe38       $unwind$?dtor$2@?0??GetFindData@Plist@@QEAAHAEAPEAUPluginPanelItem@@AEA_K_K@Z@4HA 0000000180055e38     Pclass.obj
 0002:0000fe38       $unwind$?dtor$2@?0??GetVersionInfo@Plist@@SA_NPEB_WAEAV?$unique_ptr@$$BY0A@DU?$default_delete@$$BY0A@D@std@@@std@@AEAPEB_W2@Z@4HA 0000000180055e38     Pclass.obj
 0002:0000fe38       $unwind$?dtor$2@?0??PrintOwnerInfo@Plist@@AEAAXPEAXK@Z@4HA 0000000180055e38     Pclass.obj
 0002:0000fe38       $unwind$?dtor$31@?0??GetFiles@Plist@@QEAAHPEAUPluginPanelItem@@_KHPEAPEB_W1AEAUoptions@@@Z@4HA 0000000180055e38     Pclass.obj
 0002:0000fe38       $unwind$?dtor$32@?0???$_Uninitialized_copy@PEBUmode@@V?$allocator@Umode@@@std@@@std@@YAPEAUmode@@QEBU1@0PEAU1@AEAV?$allocator@Umode@@@0@@Z@4HA 0000000180055e38     Pclass.obj
 0002:0000fe38       $unwind$?dtor$33@?0??GetFiles@Plist@@QEAAHPEAUPluginPanelItem@@_KHPEAPEB_W1AEAUoptions@@@Z@4HA 0000000180055e38     Pclass.obj
 0002:0000fe38       $unwind$?dtor$35@?0??GetFiles@Plist@@QEAAHPEAUPluginPanelItem@@_KHPEAPEB_W1AEAUoptions@@@Z@4HA 0000000180055e38     Pclass.obj
 0002:0000fe38       $unwind$?dtor$35@?0??InitializePanelModes@Plist@@SAXXZ@4HA 0000000180055e38     Pclass.obj
 0002:0000fe38       $unwind$?dtor$36@?0??InitializePanelModes@Plist@@SAXXZ@4HA 0000000180055e38     Pclass.obj
 0002:0000fe38       $unwind$?dtor$37@?0??GetFiles@Plist@@QEAAHPEAUPluginPanelItem@@_KHPEAPEB_W1AEAUoptions@@@Z@4HA 0000000180055e38     Pclass.obj
 0002:0000fe38       $unwind$?dtor$38@?0??GetFiles@Plist@@QEAAHPEAUPluginPanelItem@@_KHPEAPEB_W1AEAUoptions@@@Z@4HA 0000000180055e38     Pclass.obj
 0002:0000fe38       $unwind$?dtor$3@?0???0Plist@@QEAA@XZ@4HA 0000000180055e38     Pclass.obj
 0002:0000fe38       $unwind$?dtor$3@?0??DumpNTCounters@@YAXPEAXAEAVPerfThread@@KK@Z@4HA 0000000180055e38     Pclass.obj
 0002:0000fe38       $unwind$?dtor$3@?0??GetFiles@Plist@@QEAAHPEAUPluginPanelItem@@_KHPEAPEB_W1AEAUoptions@@@Z@4HA 0000000180055e38     Pclass.obj
 0002:0000fe38       $unwind$?dtor$3@?0??GetFindData@Plist@@QEAAHAEAPEAUPluginPanelItem@@AEA_K_K@Z@4HA 0000000180055e38     Pclass.obj
 0002:0000fe38       $unwind$?dtor$3@?0??PrintVersionInfo@Plist@@CAXPEAXPEB_W@Z@4HA 0000000180055e38     Pclass.obj
 0002:0000fe38       $unwind$?dtor$40@?0??GetFiles@Plist@@QEAAHPEAUPluginPanelItem@@_KHPEAPEB_W1AEAUoptions@@@Z@4HA 0000000180055e38     Pclass.obj
 0002:0000fe38       $unwind$?dtor$41@?0??GetFiles@Plist@@QEAAHPEAUPluginPanelItem@@_KHPEAPEB_W1AEAUoptions@@@Z@4HA 0000000180055e38     Pclass.obj
 0002:0000fe38       $unwind$?dtor$44@?0??InitializePanelModes@Plist@@SAXXZ@4HA 0000000180055e38     Pclass.obj
 0002:0000fe38       $unwind$?dtor$45@?0??InitializePanelModes@Plist@@SAXXZ@4HA 0000000180055e38     Pclass.obj
 0002:0000fe38       $unwind$?dtor$4@?0??DeleteFiles@Plist@@QEAAHPEAUPluginPanelItem@@_K1@Z@4HA 0000000180055e38     Pclass.obj
 0002:0000fe38       $unwind$?dtor$4@?0??GetFiles@Plist@@QEAAHPEAUPluginPanelItem@@_KHPEAPEB_W1AEAUoptions@@@Z@4HA 0000000180055e38     Pclass.obj
 0002:0000fe38       $unwind$?dtor$4@?0??GetFindData@Plist@@QEAAHAEAPEAUPluginPanelItem@@AEA_K_K@Z@4HA 0000000180055e38     Pclass.obj
 0002:0000fe38       $unwind$?dtor$4@?0??GetVersionInfo@Plist@@SA_NPEB_WAEAV?$unique_ptr@$$BY0A@DU?$default_delete@$$BY0A@D@std@@@std@@AEAPEB_W2@Z@4HA 0000000180055e38     Pclass.obj
 0002:0000fe38       $unwind$?dtor$53@?0??InitializePanelModes@Plist@@SAXXZ@4HA 0000000180055e38     Pclass.obj
 0002:0000fe38       $unwind$?dtor$54@?0??InitializePanelModes@Plist@@SAXXZ@4HA 0000000180055e38     Pclass.obj
 0002:0000fe38       $unwind$?dtor$5@?0??GetFindData@Plist@@QEAAHAEAPEAUPluginPanelItem@@AEA_K_K@Z@4HA 0000000180055e38     Pclass.obj
 0002:0000fe38       $unwind$?dtor$62@?0??InitializePanelModes@Plist@@SAXXZ@4HA 0000000180055e38     Pclass.obj
 0002:0000fe38       $unwind$?dtor$63@?0??InitializePanelModes@Plist@@SAXXZ@4HA 0000000180055e38     Pclass.obj
 0002:0000fe38       $unwind$?dtor$64@?0??GetFiles@Plist@@QEAAHPEAUPluginPanelItem@@_KHPEAPEB_W1AEAUoptions@@@Z@4HA 0000000180055e38     Pclass.obj
 0002:0000fe38       $unwind$?dtor$6@?0??DumpNTCounters@@YAXPEAXAEAVPerfThread@@KK@Z@4HA 0000000180055e38     Pclass.obj
 0002:0000fe38       $unwind$?dtor$6@?0??GetFiles@Plist@@QEAAHPEAUPluginPanelItem@@_KHPEAPEB_W1AEAUoptions@@@Z@4HA 0000000180055e38     Pclass.obj
 0002:0000fe38       $unwind$?dtor$6@?0??GetFindData@Plist@@QEAAHAEAPEAUPluginPanelItem@@AEA_K_K@Z@4HA 0000000180055e38     Pclass.obj
 0002:0000fe38       $unwind$?dtor$6@?0??PrintOwnerInfo@Plist@@AEAAXPEAXK@Z@4HA 0000000180055e38     Pclass.obj
 0002:0000fe38       $unwind$?dtor$6@?0??PrintVersionInfo@Plist@@CAXPEAXPEB_W@Z@4HA 0000000180055e38     Pclass.obj
 0002:0000fe38       $unwind$?dtor$71@?0??InitializePanelModes@Plist@@SAXXZ@4HA 0000000180055e38     Pclass.obj
 0002:0000fe38       $unwind$?dtor$72@?0??InitializePanelModes@Plist@@SAXXZ@4HA 0000000180055e38     Pclass.obj
 0002:0000fe38       $unwind$?dtor$76@?0??GetFiles@Plist@@QEAAHPEAUPluginPanelItem@@_KHPEAPEB_W1AEAUoptions@@@Z@4HA 0000000180055e38     Pclass.obj
 0002:0000fe38       $unwind$?dtor$7@?0??GetFindData@Plist@@QEAAHAEAPEAUPluginPanelItem@@AEA_K_K@Z@4HA 0000000180055e38     Pclass.obj
 0002:0000fe38       $unwind$?dtor$80@?0??InitializePanelModes@Plist@@SAXXZ@4HA 0000000180055e38     Pclass.obj
 0002:0000fe38       $unwind$?dtor$81@?0??InitializePanelModes@Plist@@SAXXZ@4HA 0000000180055e38     Pclass.obj
 0002:0000fe38       $unwind$?dtor$8@?0??GetFiles@Plist@@QEAAHPEAUPluginPanelItem@@_KHPEAPEB_W1AEAUoptions@@@Z@4HA 0000000180055e38     Pclass.obj
 0002:0000fe38       $unwind$?dtor$8@?0??GetFindData@Plist@@QEAAHAEAPEAUPluginPanelItem@@AEA_K_K@Z@4HA 0000000180055e38     Pclass.obj
 0002:0000fe38       $unwind$?dtor$8@?0??InitializePanelModes@Plist@@SAXXZ@4HA 0000000180055e38     Pclass.obj
 0002:0000fe38       $unwind$?dtor$91@?0??InitializePanelModes@Plist@@SAXXZ@4HA 0000000180055e38     Pclass.obj
 0002:0000fe38       $unwind$?dtor$99@?0??InitializePanelModes@Plist@@SAXXZ@4HA 0000000180055e38     Pclass.obj
 0002:0000fe38       $unwind$?dtor$9@?0??InitializePanelModes@Plist@@SAXXZ@4HA 0000000180055e38     Pclass.obj
 0002:0000fe38       $unwind$?dtor$0@?0???$insert@V?$_List_unchecked_const_iterator@V?$_List_val@U?$_List_simple_types@U?$pair@$$CBKUProcessPerfData@@@std@@@std@@@std@@U_Iterator_base0@2@@std@@@?$_Hash@V?$_Umap_traits@KUProcessPerfData@@V?$_Uhash_compare@KU?$hash@K@std@@U?$equal_to@K@2@@std@@V?$allocator@U?$pair@$$CBKUProcessPerfData@@@std@@@3@$00@std@@@std@@QEAAXV?$_List_unchecked_const_iterator@V?$_List_val@U?$_List_simple_types@U?$pair@$$CBKUProcessPerfData@@@std@@@std@@@std@@U_Iterator_base0@2@@1@0@Z@4HA 0000000180055e38     Plist.obj
 0002:0000fe38       $unwind$?dtor$0@?0???$print_module@PEAX@@YAXQEAXPEAXKAEAUoptions@@AEBV?$function@$$A6A_NPEA_W_K@Z@std@@@Z@4HA 0000000180055e38     Plist.obj
 0002:0000fe38       $unwind$?dtor$0@?0??GetList@@YA_NAEAPEAUPluginPanelItem@@AEA_KAEAVPerfThread@@@Z@4HA 0000000180055e38     Plist.obj
 0002:0000fe38       $unwind$?dtor$0@?0??KillProcess@@YA_NKPEAUHWND__@@@Z@4HA 0000000180055e38     Plist.obj
 0002:0000fe38       $unwind$?dtor$0@?0??PrintModules@?$ipc_functions@$0A@@@SAXPEAX0AEAUoptions@@@Z@4HA 0000000180055e38     Plist.obj
 0002:0000fe38       $unwind$?dtor$0@?0??PrintModules@@YAXPEAXKAEAUoptions@@@Z@4HA 0000000180055e38     Plist.obj
 0002:0000fe38       $unwind$?dtor$0@?0??PrintNTCurDirAndEnv@@YAXPEAX0H@Z@4HA 0000000180055e38     Plist.obj
 0002:0000fe38       $unwind$?dtor$1@?0???$insert@V?$_List_unchecked_const_iterator@V?$_List_val@U?$_List_simple_types@U?$pair@$$CBKUProcessPerfData@@@std@@@std@@@std@@U_Iterator_base0@2@@std@@@?$_Hash@V?$_Umap_traits@KUProcessPerfData@@V?$_Uhash_compare@KU?$hash@K@std@@U?$equal_to@K@2@@std@@V?$allocator@U?$pair@$$CBKUProcessPerfData@@@std@@@3@$00@std@@@std@@QEAAXV?$_List_unchecked_const_iterator@V?$_List_val@U?$_List_simple_types@U?$pair@$$CBKUProcessPerfData@@@std@@@std@@@std@@U_Iterator_base0@2@@1@0@Z@4HA 0000000180055e38     Plist.obj
 0002:0000fe38       $unwind$?dtor$1@?0??KillProcess@@YA_NKPEAUHWND__@@@Z@4HA 0000000180055e38     Plist.obj
 0002:0000fe38       $unwind$?dtor$1@?0??PrintModules@?$ipc_functions@$0A@@@SAXPEAX0AEAUoptions@@@Z@4HA 0000000180055e38     Plist.obj
 0002:0000fe38       $unwind$?dtor$1@?0??PrintModules@@YAXPEAXKAEAUoptions@@@Z@4HA 0000000180055e38     Plist.obj
 0002:0000fe38       $unwind$?dtor$1@?0??PrintNTCurDirAndEnv@@YAXPEAX0H@Z@4HA 0000000180055e38     Plist.obj
 0002:0000fe38       $unwind$?dtor$2@?0??PrintModules@@YAXPEAXKAEAUoptions@@@Z@4HA 0000000180055e38     Plist.obj
 0002:0000fe38       $unwind$?dtor$2@?0??print_module_impl@@YAXQEAXAEBV?$basic_string@_WU?$char_traits@_W@std@@V?$allocator@_W@2@@std@@KAEBUoptions@@AEBV?$function@$$A6A_NPEA_W_K@Z@2@@Z@4HA 0000000180055e38     Plist.obj
 0002:0000fe38       $unwind$?dtor$3@?0??PrintModules@@YAXPEAXKAEAUoptions@@@Z@4HA 0000000180055e38     Plist.obj
 0002:0000fe38       $unwind$?dtor$0@?0??WinError@@YAHPEB_W@Z@4HA 0000000180055e38     Pmix.obj
 0002:0000fe38       $unwind$?dtor$1@?0??WinError@@YAHPEB_W@Z@4HA 0000000180055e38     Pmix.obj
 0002:0000fe38       $unwind$?dtor$0@?0???$?RH$0A@@?$precision_checker@Uerror_handler@detail@v8@fmt@@@detail@v8@fmt@@QEAA_KH@Z@4HA 0000000180055e38     format.obj
 0002:0000fe38       $unwind$?dtor$0@?0???$?RH$0A@@?$width_checker@Uerror_handler@detail@v8@fmt@@@detail@v8@fmt@@QEAA_KH@Z@4HA 0000000180055e38     format.obj
 0002:0000fe38       $unwind$?dtor$0@?0???$?RM$0A@@?$precision_checker@Uerror_handler@detail@v8@fmt@@@detail@v8@fmt@@QEAA_KM@Z@4HA 0000000180055e38     format.obj
 0002:0000fe38       $unwind$?dtor$0@?0???$?RM$0A@@?$width_checker@Uerror_handler@detail@v8@fmt@@@detail@v8@fmt@@QEAA_KM@Z@4HA 0000000180055e38     format.obj
 0002:0000fe38       $unwind$?dtor$0@?0???$?RN$0A@@?$precision_checker@Uerror_handler@detail@v8@fmt@@@detail@v8@fmt@@QEAA_KN@Z@4HA 0000000180055e38     format.obj
 0002:0000fe38       $unwind$?dtor$0@?0???$?RN$0A@@?$width_checker@Uerror_handler@detail@v8@fmt@@@detail@v8@fmt@@QEAA_KN@Z@4HA 0000000180055e38     format.obj
 0002:0000fe38       $unwind$?dtor$0@?0???$?RO$0A@@?$precision_checker@Uerror_handler@detail@v8@fmt@@@detail@v8@fmt@@QEAA_KO@Z@4HA 0000000180055e38     format.obj
 0002:0000fe38       $unwind$?dtor$0@?0???$?RO$0A@@?$width_checker@Uerror_handler@detail@v8@fmt@@@detail@v8@fmt@@QEAA_KO@Z@4HA 0000000180055e38     format.obj
 0002:0000fe38       $unwind$?dtor$0@?0???$?RPEBX$0A@@?$precision_checker@Uerror_handler@detail@v8@fmt@@@detail@v8@fmt@@QEAA_KPEBX@Z@4HA 0000000180055e38     format.obj
 0002:0000fe38       $unwind$?dtor$0@?0???$?RPEBX$0A@@?$width_checker@Uerror_handler@detail@v8@fmt@@@detail@v8@fmt@@QEAA_KPEBX@Z@4HA 0000000180055e38     format.obj
 0002:0000fe38       $unwind$?dtor$0@?0???$?RUmonostate@v8@fmt@@$0A@@?$precision_checker@Uerror_handler@detail@v8@fmt@@@detail@v8@fmt@@QEAA_KUmonostate@23@@Z@4HA 0000000180055e38     format.obj
 0002:0000fe38       $unwind$?dtor$0@?0???$?RUmonostate@v8@fmt@@$0A@@?$width_checker@Uerror_handler@detail@v8@fmt@@@detail@v8@fmt@@QEAA_KUmonostate@23@@Z@4HA 0000000180055e38     format.obj
 0002:0000fe38       $unwind$?dtor$0@?0???$?R_J$0A@@?$precision_checker@Uerror_handler@detail@v8@fmt@@@detail@v8@fmt@@QEAA_K_J@Z@4HA 0000000180055e38     format.obj
 0002:0000fe38       $unwind$?dtor$0@?0???$?R_J$0A@@?$width_checker@Uerror_handler@detail@v8@fmt@@@detail@v8@fmt@@QEAA_K_J@Z@4HA 0000000180055e38     format.obj
 0002:0000fe38       $unwind$?dtor$0@?0???$?R_N$0A@@?$precision_checker@Uerror_handler@detail@v8@fmt@@@detail@v8@fmt@@QEAA_K_N@Z@4HA 0000000180055e38     format.obj
 0002:0000fe38       $unwind$?dtor$0@?0???$?R_N$0A@@?$width_checker@Uerror_handler@detail@v8@fmt@@@detail@v8@fmt@@QEAA_K_N@Z@4HA 0000000180055e38     format.obj
 0002:0000fe38       $unwind$?dtor$0@?0???$thousands_sep_impl@_W@detail@v8@fmt@@YA?AU?$thousands_sep_result@_W@012@Vlocale_ref@012@@Z@4HA 0000000180055e38     format.obj
 0002:0000fe38       $unwind$?dtor$0@?0???$use_facet@V?$numpunct@_W@std@@@std@@YAAEBV?$numpunct@_W@0@AEBVlocale@0@@Z@4HA 0000000180055e38     format.obj
 0002:0000fe38       $unwind$?dtor$0@?0??_Init@?$numpunct@_W@std@@IEAAXAEBV_Locinfo@2@_N@Z@4HA 0000000180055e38     format.obj
 0002:0000fe38       $unwind$?dtor$0@?0??format_dragon@detail@v8@fmt@@YAXUfp@123@_NHAEAV?$buffer@D@123@AEAH@Z@4HA 0000000180055e38     format.obj
 0002:0000fe38       $unwind$?dtor$0@?0??on_error@error_handler@detail@v8@fmt@@QEAAXPEBD@Z@4HA 0000000180055e38     format.obj
 0002:0000fe38       $unwind$?dtor$0@?0??square@bigint@detail@v8@fmt@@QEAAXXZ@4HA 0000000180055e38     format.obj
 0002:0000fe38       $unwind$?dtor$0@?0??throw_format_error@detail@v8@fmt@@YAXPEBD@Z@4HA 0000000180055e38     format.obj
 0002:0000fe38       $unwind$?dtor$1@?0???$thousands_sep_impl@_W@detail@v8@fmt@@YA?AU?$thousands_sep_result@_W@012@Vlocale_ref@012@@Z@4HA 0000000180055e38     format.obj
 0002:0000fe38       $unwind$?dtor$1@?0???$use_facet@V?$numpunct@_W@std@@@std@@YAAEBV?$numpunct@_W@0@AEBVlocale@0@@Z@4HA 0000000180055e38     format.obj
 0002:0000fe38       $unwind$?dtor$1@?0??format_dragon@detail@v8@fmt@@YAXUfp@123@_NHAEAV?$buffer@D@123@AEAH@Z@4HA 0000000180055e38     format.obj
 0002:0000fe38       $unwind$?dtor$2@?0??_Getcat@?$numpunct@_W@std@@SA_KPEAPEBVfacet@locale@2@PEBV42@@Z@4HA 0000000180055e38     format.obj
 0002:0000fe38       $unwind$?dtor$2@?0??format_dragon@detail@v8@fmt@@YAXUfp@123@_NHAEAV?$buffer@D@123@AEAH@Z@4HA 0000000180055e38     format.obj
 0002:0000fe38       $unwind$?dtor$3@?0??format_dragon@detail@v8@fmt@@YAXUfp@123@_NHAEAV?$buffer@D@123@AEAH@Z@4HA 0000000180055e38     format.obj
 0002:0000fe38       $unwind$?dtor$9@?0??_Getcat@?$numpunct@_W@std@@SA_KPEAPEBVfacet@locale@2@PEBV42@@Z@4HA 0000000180055e38     format.obj
 0002:0000fe38       $unwind$?dtor$0@?0???$apply@V?$back_insert_iterator@V?$buffer@_W@detail@v8@fmt@@@std@@D@?$digit_grouping@_W@detail@v8@fmt@@QEBA?AV?$back_insert_iterator@V?$buffer@_W@detail@v8@fmt@@@std@@V45@V?$basic_string_view@D@23@@Z@4HA 0000000180055e38     handles.obj
 0002:0000fe38       $unwind$?dtor$0@?0???$apply@V?$back_insert_iterator@V?$buffer@_W@detail@v8@fmt@@@std@@_W@?$digit_grouping@_W@detail@v8@fmt@@QEBA?AV?$back_insert_iterator@V?$buffer@_W@detail@v8@fmt@@@std@@V45@V?$basic_string_view@_W@23@@Z@4HA 0000000180055e38     handles.obj
 0002:0000fe38       $unwind$?dtor$0@?0???$decimal_point@_W@detail@v8@fmt@@YA_WVlocale_ref@012@@Z@4HA 0000000180055e38     handles.obj
 0002:0000fe38       $unwind$?dtor$0@?0???$do_parse_arg_id@_WAEAUid_adapter@?1???$parse_replacement_field@_WAEAUformat_handler@?1???$vformat_to@_W@detail@v8@fmt@@YAXAEAV?$buffer@_W@234@V?$basic_string_view@_W@34@V?$basic_format_args@V?$basic_format_context@V?$back_insert_iterator@V?$buffer@_W@detail@v8@fmt@@@std@@_W@v8@fmt@@@34@Vlocale_ref@234@@Z@@detail@v8@fmt@@YAPEB_WPEB_W0AEAUformat_handler@?1???$vformat_to@_W@234@YAXAEAV?$buffer@_W@234@V?$basic_string_view@_W@34@V?$basic_format_args@V?$basic_format_context@V?$back_insert_iterator@V?$buffer@_W@detail@v8@fmt@@@std@@_W@v8@fmt@@@34@Vlocale_ref@234@@Z@@Z@@detail@v8@fmt@@YAPEB_WPEB_W0AEAUid_adapter@?1???$parse_replacement_field@_WAEAUformat_handler@?1???$vformat_to@_W@detail@v8@fmt@@YAXAEAV?$buffer@_W@234@V?$basic_string_view@_W@34@V?$basic_format_args@V?$basic_format_context@V?$back_insert_iterator@V?$buffer@_W@detail@v8@fmt@@@std@@_W@v8@fmt@@@34@Vlocale_ref@234@@Z@@012@YAPEB_W00AEAUformat_handler@?1???$vformat_to@_W@012@YAXAEAV?$buffer@_W@012@V?$basic_string_view@_W@12@V?$basic_format_args@V?$basic_format_context@V?$back_insert_iterator@V?$buffer@_W@detail@v8@fmt@@@std@@_W@v8@fmt@@@12@Vlocale_ref@012@@Z@@Z@@Z@4HA 0000000180055e38     handles.obj
 0002:0000fe38       $unwind$?dtor$0@?0???$do_parse_arg_id@_WAEAUprecision_adapter@?1???$parse_precision@_WAEAV?$specs_checker@V?$specs_handler@_W@detail@v8@fmt@@@detail@v8@fmt@@@detail@v8@fmt@@YAPEB_WPEB_W0AEAV?$specs_checker@V?$specs_handler@_W@detail@v8@fmt@@@234@@Z@@detail@v8@fmt@@YAPEB_WPEB_W0AEAUprecision_adapter@?1???$parse_precision@_WAEAV?$specs_checker@V?$specs_handler@_W@detail@v8@fmt@@@detail@v8@fmt@@@012@YAPEB_W00AEAV?$specs_checker@V?$specs_handler@_W@detail@v8@fmt@@@012@@Z@@Z@4HA 0000000180055e38     handles.obj
 0002:0000fe38       $unwind$?dtor$0@?0???$do_parse_arg_id@_WAEAUwidth_adapter@?1???$parse_width@_WAEAV?$specs_checker@V?$specs_handler@_W@detail@v8@fmt@@@detail@v8@fmt@@@detail@v8@fmt@@YAPEB_WPEB_W0AEAV?$specs_checker@V?$specs_handler@_W@detail@v8@fmt@@@234@@Z@@detail@v8@fmt@@YAPEB_WPEB_W0AEAUwidth_adapter@?1???$parse_width@_WAEAV?$specs_checker@V?$specs_handler@_W@detail@v8@fmt@@@detail@v8@fmt@@@012@YAPEB_W00AEAV?$specs_checker@V?$specs_handler@_W@detail@v8@fmt@@@012@@Z@@Z@4HA 0000000180055e38     handles.obj
 0002:0000fe38       $unwind$?dtor$0@?0???$do_write_float@V?$back_insert_iterator@V?$buffer@_W@detail@v8@fmt@@@std@@U?$decimal_fp@M@dragonbox@detail@v8@fmt@@_WV?$digit_grouping@_W@567@@detail@v8@fmt@@YA?AV?$back_insert_iterator@V?$buffer@_W@detail@v8@fmt@@@std@@V34@AEBU?$decimal_fp@M@dragonbox@012@AEBU?$basic_format_specs@_W@12@Ufloat_specs@012@Vlocale_ref@012@@Z@4HA 0000000180055e38     handles.obj
 0002:0000fe38       $unwind$?dtor$0@?0???$do_write_float@V?$back_insert_iterator@V?$buffer@_W@detail@v8@fmt@@@std@@U?$decimal_fp@N@dragonbox@detail@v8@fmt@@_WV?$digit_grouping@_W@567@@detail@v8@fmt@@YA?AV?$back_insert_iterator@V?$buffer@_W@detail@v8@fmt@@@std@@V34@AEBU?$decimal_fp@N@dragonbox@012@AEBU?$basic_format_specs@_W@12@Ufloat_specs@012@Vlocale_ref@012@@Z@4HA 0000000180055e38     handles.obj
 0002:0000fe38       $unwind$?dtor$0@?0???$do_write_float@V?$back_insert_iterator@V?$buffer@_W@detail@v8@fmt@@@std@@Ubig_decimal_fp@detail@v8@fmt@@_WV?$digit_grouping@_W@456@@detail@v8@fmt@@YA?AV?$back_insert_iterator@V?$buffer@_W@detail@v8@fmt@@@std@@V34@AEBUbig_decimal_fp@012@AEBU?$basic_format_specs@_W@12@Ufloat_specs@012@Vlocale_ref@012@@Z@4HA 0000000180055e38     handles.obj
 0002:0000fe38       $unwind$?dtor$0@?0???$get_arg@V?$basic_format_context@V?$back_insert_iterator@V?$buffer@_W@detail@v8@fmt@@@std@@_W@v8@fmt@@H@detail@v8@fmt@@YA?AV?$basic_format_arg@V?$basic_format_context@V?$back_insert_iterator@V?$buffer@_W@detail@v8@fmt@@@std@@_W@v8@fmt@@@12@AEAV?$basic_format_context@V?$back_insert_iterator@V?$buffer@_W@detail@v8@fmt@@@std@@_W@12@H@Z@4HA 0000000180055e38     handles.obj
 0002:0000fe38       $unwind$?dtor$0@?0???$parse_align@_WAEAV?$specs_checker@V?$specs_handler@_W@detail@v8@fmt@@@detail@v8@fmt@@@detail@v8@fmt@@YAPEB_WPEB_W0AEAV?$specs_checker@V?$specs_handler@_W@detail@v8@fmt@@@012@@Z@4HA 0000000180055e38     handles.obj
 0002:0000fe38       $unwind$?dtor$0@?0???$parse_float_type_spec@Uerror_handler@detail@v8@fmt@@_W@detail@v8@fmt@@YA?AUfloat_specs@012@AEBU?$basic_format_specs@_W@12@$$QEAUerror_handler@012@@Z@4HA 0000000180055e38     handles.obj
 0002:0000fe38       $unwind$?dtor$0@?0???$parse_format_string@$0A@_WUformat_handler@?1???$vformat_to@_W@detail@v8@fmt@@YAXAEAV?$buffer@_W@234@V?$basic_string_view@_W@34@V?$basic_format_args@V?$basic_format_context@V?$back_insert_iterator@V?$buffer@_W@detail@v8@fmt@@@std@@_W@v8@fmt@@@34@Vlocale_ref@234@@Z@@detail@v8@fmt@@YAXV?$basic_string_view@_W@12@$$QEAUformat_handler@?1???$vformat_to@_W@012@YAXAEAV?$buffer@_W@012@0V?$basic_format_args@V?$basic_format_context@V?$back_insert_iterator@V?$buffer@_W@detail@v8@fmt@@@std@@_W@v8@fmt@@@12@Vlocale_ref@012@@Z@@Z@4HA 0000000180055e38     handles.obj
 0002:0000fe38       $unwind$?dtor$0@?0???$parse_precision@_WAEAV?$specs_checker@V?$specs_handler@_W@detail@v8@fmt@@@detail@v8@fmt@@@detail@v8@fmt@@YAPEB_WPEB_W0AEAV?$specs_checker@V?$specs_handler@_W@detail@v8@fmt@@@012@@Z@4HA 0000000180055e38     handles.obj
 0002:0000fe38       $unwind$?dtor$0@?0???$parse_replacement_field@_WAEAUformat_handler@?1???$vformat_to@_W@detail@v8@fmt@@YAXAEAV?$buffer@_W@234@V?$basic_string_view@_W@34@V?$basic_format_args@V?$basic_format_context@V?$back_insert_iterator@V?$buffer@_W@detail@v8@fmt@@@std@@_W@v8@fmt@@@34@Vlocale_ref@234@@Z@@detail@v8@fmt@@YAPEB_WPEB_W0AEAUformat_handler@?1???$vformat_to@_W@012@YAXAEAV?$buffer@_W@012@V?$basic_string_view@_W@12@V?$basic_format_args@V?$basic_format_context@V?$back_insert_iterator@V?$buffer@_W@detail@v8@fmt@@@std@@_W@v8@fmt@@@12@Vlocale_ref@012@@Z@@Z@4HA 0000000180055e38     handles.obj
 0002:0000fe38       $unwind$?dtor$0@?0???$parse_width@_WAEAV?$specs_checker@V?$specs_handler@_W@detail@v8@fmt@@@detail@v8@fmt@@@detail@v8@fmt@@YAPEB_WPEB_W0AEAV?$specs_checker@V?$specs_handler@_W@detail@v8@fmt@@@012@@Z@4HA 0000000180055e38     handles.obj
 0002:0000fe38       $unwind$?dtor$0@?0???$vformat@_W$0A@@v8@fmt@@YA?AV?$basic_string@_WU?$char_traits@_W@std@@V?$allocator@_W@2@@std@@V?$basic_string_view@_W@01@V?$basic_format_args@V?$basic_format_context@V?$back_insert_iterator@V?$buffer@_W@detail@v8@fmt@@@std@@_W@v8@fmt@@@01@@Z@4HA 0000000180055e38     handles.obj
 0002:0000fe38       $unwind$?dtor$0@?0???$visit_format_arg@AEAU?$arg_formatter@_W@detail@v8@fmt@@V?$basic_format_context@V?$back_insert_iterator@V?$buffer@_W@detail@v8@fmt@@@std@@_W@34@@v8@fmt@@YA?AV?$back_insert_iterator@V?$buffer@_W@detail@v8@fmt@@@std@@AEAU?$arg_formatter@_W@detail@01@AEBV?$basic_format_arg@V?$basic_format_context@V?$back_insert_iterator@V?$buffer@_W@detail@v8@fmt@@@std@@_W@v8@fmt@@@01@@Z@4HA 0000000180055e38     handles.obj
 0002:0000fe38       $unwind$?dtor$0@?0???$visit_format_arg@U?$default_arg_formatter@_W@detail@v8@fmt@@V?$basic_format_context@V?$back_insert_iterator@V?$buffer@_W@detail@v8@fmt@@@std@@_W@34@@v8@fmt@@YA?AV?$back_insert_iterator@V?$buffer@_W@detail@v8@fmt@@@std@@$$QEAU?$default_arg_formatter@_W@detail@01@AEBV?$basic_format_arg@V?$basic_format_context@V?$back_insert_iterator@V?$buffer@_W@detail@v8@fmt@@@std@@_W@v8@fmt@@@01@@Z@4HA 0000000180055e38     handles.obj
 0002:0000fe38       $unwind$?dtor$0@?0???$write@_WV?$back_insert_iterator@V?$buffer@_W@detail@v8@fmt@@@std@@@detail@v8@fmt@@YA?AV?$back_insert_iterator@V?$buffer@_W@detail@v8@fmt@@@std@@V34@V?$basic_string_view@_W@12@AEBU?$basic_format_specs@_W@12@Vlocale_ref@012@@Z@4HA 0000000180055e38     handles.obj
 0002:0000fe38       $unwind$?dtor$0@?0???$write@_WV?$back_insert_iterator@V?$buffer@_W@detail@v8@fmt@@@std@@@detail@v8@fmt@@YA?AV?$back_insert_iterator@V?$buffer@_W@detail@v8@fmt@@@std@@V34@_WAEBU?$basic_format_specs@_W@12@Vlocale_ref@012@@Z@4HA 0000000180055e38     handles.obj
 0002:0000fe38       $unwind$?dtor$0@?0???$write@_WV?$back_insert_iterator@V?$buffer@_W@detail@v8@fmt@@@std@@M$0A@@detail@v8@fmt@@YA?AV?$back_insert_iterator@V?$buffer@_W@detail@v8@fmt@@@std@@V34@MU?$basic_format_specs@_W@12@Vlocale_ref@012@@Z@4HA 0000000180055e38     handles.obj
 0002:0000fe38       $unwind$?dtor$0@?0???$write@_WV?$back_insert_iterator@V?$buffer@_W@detail@v8@fmt@@@std@@N$0A@@detail@v8@fmt@@YA?AV?$back_insert_iterator@V?$buffer@_W@detail@v8@fmt@@@std@@V34@NU?$basic_format_specs@_W@12@Vlocale_ref@012@@Z@4HA 0000000180055e38     handles.obj
 0002:0000fe38       $unwind$?dtor$0@?0???$write@_WV?$back_insert_iterator@V?$buffer@_W@detail@v8@fmt@@@std@@O$0A@@detail@v8@fmt@@YA?AV?$back_insert_iterator@V?$buffer@_W@detail@v8@fmt@@@std@@V34@OU?$basic_format_specs@_W@12@Vlocale_ref@012@@Z@4HA 0000000180055e38     handles.obj
 0002:0000fe38       $unwind$?dtor$0@?0???$write@_WV?$back_insert_iterator@V?$buffer@_W@detail@v8@fmt@@@std@@X$0A@@detail@v8@fmt@@YA?AV?$back_insert_iterator@V?$buffer@_W@detail@v8@fmt@@@std@@V34@PEBXAEBU?$basic_format_specs@_W@12@Vlocale_ref@012@@Z@4HA 0000000180055e38     handles.obj
 0002:0000fe38       $unwind$?dtor$0@?0???$write_int@_WV?$back_insert_iterator@V?$buffer@_W@detail@v8@fmt@@@std@@I@detail@v8@fmt@@YA?AV?$back_insert_iterator@V?$buffer@_W@detail@v8@fmt@@@std@@V34@U?$write_int_arg@I@012@AEBU?$basic_format_specs@_W@12@Vlocale_ref@012@@Z@4HA 0000000180055e38     handles.obj
 0002:0000fe38       $unwind$?dtor$0@?0???$write_int@_WV?$back_insert_iterator@V?$buffer@_W@detail@v8@fmt@@@std@@_K@detail@v8@fmt@@YA?AV?$back_insert_iterator@V?$buffer@_W@detail@v8@fmt@@@std@@V34@U?$write_int_arg@_K@012@AEBU?$basic_format_specs@_W@12@Vlocale_ref@012@@Z@4HA 0000000180055e38     handles.obj
 0002:0000fe38       $unwind$?dtor$0@?0???$write_int_localized@V?$back_insert_iterator@V?$buffer@_W@detail@v8@fmt@@@std@@_K_W@detail@v8@fmt@@YA_NAEAV?$back_insert_iterator@V?$buffer@_W@detail@v8@fmt@@@std@@_KIAEBU?$basic_format_specs@_W@12@Vlocale_ref@012@@Z@4HA 0000000180055e38     handles.obj
 0002:0000fe38       $unwind$?dtor$0@?0???$write_significand@V?$back_insert_iterator@V?$buffer@_W@detail@v8@fmt@@@std@@_WIV?$digit_grouping@_W@detail@v8@fmt@@@detail@v8@fmt@@YA?AV?$back_insert_iterator@V?$buffer@_W@detail@v8@fmt@@@std@@V34@IHH_WAEBV?$digit_grouping@_W@012@@Z@4HA 0000000180055e38     handles.obj
 0002:0000fe38       $unwind$?dtor$0@?0???$write_significand@_WV?$back_insert_iterator@V?$buffer@_W@detail@v8@fmt@@@std@@PEBDV?$digit_grouping@_W@detail@v8@fmt@@@detail@v8@fmt@@YA?AV?$back_insert_iterator@V?$buffer@_W@detail@v8@fmt@@@std@@V34@PEBDHHAEBV?$digit_grouping@_W@012@@Z@4HA 0000000180055e38     handles.obj
 0002:0000fe38       $unwind$?dtor$0@?0???0?$digit_grouping@_W@detail@v8@fmt@@QEAA@Vlocale_ref@123@_N@Z@4HA 0000000180055e38     handles.obj
 0002:0000fe38       $unwind$?dtor$0@?0???R<lambda_3>@?BD@???$do_write_float@V?$back_insert_iterator@V?$buffer@_W@detail@v8@fmt@@@std@@U?$decimal_fp@M@dragonbox@detail@v8@fmt@@_WV?$digit_grouping@_W@567@@detail@v8@fmt@@YA?AV?$back_insert_iterator@V?$buffer@_W@detail@v8@fmt@@@std@@V45@AEBU?$decimal_fp@M@dragonbox@123@AEBU?$basic_format_specs@_W@23@Ufloat_specs@123@Vlocale_ref@123@@Z@QEBA@0@Z@4HA 0000000180055e38     handles.obj
 0002:0000fe38       $unwind$?dtor$0@?0???R<lambda_3>@?BD@???$do_write_float@V?$back_insert_iterator@V?$buffer@_W@detail@v8@fmt@@@std@@U?$decimal_fp@N@dragonbox@detail@v8@fmt@@_WV?$digit_grouping@_W@567@@detail@v8@fmt@@YA?AV?$back_insert_iterator@V?$buffer@_W@detail@v8@fmt@@@std@@V45@AEBU?$decimal_fp@N@dragonbox@123@AEBU?$basic_format_specs@_W@23@Ufloat_specs@123@Vlocale_ref@123@@Z@QEBA@0@Z@4HA 0000000180055e38     handles.obj
 0002:0000fe38       $unwind$?dtor$0@?0???R<lambda_4>@?BO@???$do_write_float@V?$back_insert_iterator@V?$buffer@_W@detail@v8@fmt@@@std@@U?$decimal_fp@N@dragonbox@detail@v8@fmt@@_WV?$digit_grouping@_W@567@@detail@v8@fmt@@YA?AV?$back_insert_iterator@V?$buffer@_W@detail@v8@fmt@@@std@@V45@AEBU?$decimal_fp@N@dragonbox@123@AEBU?$basic_format_specs@_W@23@Ufloat_specs@123@Vlocale_ref@123@@Z@QEBA@0@Z@4HA 0000000180055e38     handles.obj
 0002:0000fe38       $unwind$?dtor$0@?0???R<lambda_4>@?BO@???$do_write_float@V?$back_insert_iterator@V?$buffer@_W@detail@v8@fmt@@@std@@Ubig_decimal_fp@detail@v8@fmt@@_WV?$digit_grouping@_W@456@@detail@v8@fmt@@YA?AV?$back_insert_iterator@V?$buffer@_W@detail@v8@fmt@@@std@@V45@AEBUbig_decimal_fp@123@AEBU?$basic_format_specs@_W@23@Ufloat_specs@123@Vlocale_ref@123@@Z@QEBA@0@Z@4HA 0000000180055e38     handles.obj
 0002:0000fe38       $unwind$?dtor$0@?0???Rwriter@?1???$parse_format_string@$0A@_WUformat_handler@?1???$vformat_to@_W@detail@v8@fmt@@YAXAEAV?$buffer@_W@234@V?$basic_string_view@_W@34@V?$basic_format_args@V?$basic_format_context@V?$back_insert_iterator@V?$buffer@_W@detail@v8@fmt@@@std@@_W@v8@fmt@@@34@Vlocale_ref@234@@Z@@detail@v8@fmt@@YAXV?$basic_string_view@_W@23@$$QEAUformat_handler@?1???$vformat_to@_W@123@YAXAEAV?$buffer@_W@123@0V?$basic_format_args@V?$basic_format_context@V?$back_insert_iterator@V?$buffer@_W@detail@v8@fmt@@@std@@_W@v8@fmt@@@23@Vlocale_ref@123@@Z@@Z@QEAAXPEB_W5@Z@4HA 0000000180055e38     handles.obj
 0002:0000fe38       $unwind$?dtor$0@?0??GetFileName@@YA?AV?$basic_string@_WU?$char_traits@_W@std@@V?$allocator@_W@2@@std@@PEAX@Z@4HA 0000000180055e38     handles.obj
 0002:0000fe38       $unwind$?dtor$0@?0??PrintHandleInfo@@YA_NKPEAX_NPEAVPerfThread@@@Z@4HA 0000000180055e38     handles.obj
 0002:0000fe38       $unwind$?dtor$0@?0??check_arg_id@?$basic_format_parse_context@_WUerror_handler@detail@v8@fmt@@@v8@fmt@@QEAAXH@Z@4HA 0000000180055e38     handles.obj
 0002:0000fe38       $unwind$?dtor$0@?0??get_arg@?$specs_handler@_W@detail@v8@fmt@@AEAA?AV?$basic_format_arg@V?$basic_format_context@V?$back_insert_iterator@V?$buffer@_W@detail@v8@fmt@@@std@@_W@v8@fmt@@@34@V?$basic_string_view@_W@34@@Z@4HA 0000000180055e38     handles.obj
 0002:0000fe38       $unwind$?dtor$0@?0??next_arg_id@?$basic_format_parse_context@_WUerror_handler@detail@v8@fmt@@@v8@fmt@@QEAAHXZ@4HA 0000000180055e38     handles.obj
 0002:0000fe38       $unwind$?dtor$0@?0??on_error@?$specs_handler@_W@detail@v8@fmt@@QEAAXPEBD@Z@4HA 0000000180055e38     handles.obj
 0002:0000fe38       $unwind$?dtor$0@?0??on_error@id_adapter@?1???$parse_replacement_field@_WAEAUformat_handler@?1???$vformat_to@_W@detail@v8@fmt@@YAXAEAV?$buffer@_W@234@V?$basic_string_view@_W@34@V?$basic_format_args@V?$basic_format_context@V?$back_insert_iterator@V?$buffer@_W@detail@v8@fmt@@@std@@_W@v8@fmt@@@34@Vlocale_ref@234@@Z@@detail@v8@fmt@@YAPEB_WPEB_W0AEAUformat_handler@?1???$vformat_to@_W@234@YAXAEAV?$buffer@_W@234@V?$basic_string_view@_W@34@V?$basic_format_args@V?$basic_format_context@V?$back_insert_iterator@V?$buffer@_W@detail@v8@fmt@@@std@@_W@v8@fmt@@@34@Vlocale_ref@234@@Z@@Z@QEAAXPEBD@Z@4HA 0000000180055e38     handles.obj
 0002:0000fe38       $unwind$?dtor$0@?0??on_error@precision_adapter@?1???$parse_precision@_WAEAV?$specs_checker@V?$specs_handler@_W@detail@v8@fmt@@@detail@v8@fmt@@@detail@v8@fmt@@YAPEB_WPEB_W0AEAV?$specs_checker@V?$specs_handler@_W@detail@v8@fmt@@@234@@Z@QEAAXPEBD@Z@4HA 0000000180055e38     handles.obj
 0002:0000fe38       $unwind$?dtor$0@?0??on_error@width_adapter@?1???$parse_width@_WAEAV?$specs_checker@V?$specs_handler@_W@detail@v8@fmt@@@detail@v8@fmt@@@detail@v8@fmt@@YAPEB_WPEB_W0AEAV?$specs_checker@V?$specs_handler@_W@detail@v8@fmt@@@234@@Z@QEAAXPEBD@Z@4HA 0000000180055e38     handles.obj
 0002:0000fe38       $unwind$?dtor$0@?0??require_numeric_argument@?$specs_checker@V?$specs_handler@_W@detail@v8@fmt@@@detail@v8@fmt@@AEAAXXZ@4HA 0000000180055e38     handles.obj
 0002:0000fe38       $unwind$?dtor$11@?0??PrintHandleInfo@@YA_NKPEAX_NPEAVPerfThread@@@Z@4HA 0000000180055e38     handles.obj
 0002:0000fe38       $unwind$?dtor$12@?0???$parse_precision@_WAEAV?$specs_checker@V?$specs_handler@_W@detail@v8@fmt@@@detail@v8@fmt@@@detail@v8@fmt@@YAPEB_WPEB_W0AEAV?$specs_checker@V?$specs_handler@_W@detail@v8@fmt@@@012@@Z@4HA 0000000180055e38     handles.obj
 0002:0000fe38       $unwind$?dtor$12@?0???$visit_format_arg@V?$precision_checker@Uerror_handler@detail@v8@fmt@@@detail@v8@fmt@@V?$basic_format_context@V?$back_insert_iterator@V?$buffer@_W@detail@v8@fmt@@@std@@_W@34@@v8@fmt@@YA_K$$QEAV?$precision_checker@Uerror_handler@detail@v8@fmt@@@detail@01@AEBV?$basic_format_arg@V?$basic_format_context@V?$back_insert_iterator@V?$buffer@_W@detail@v8@fmt@@@std@@_W@v8@fmt@@@01@@Z@4HA 0000000180055e38     handles.obj
 0002:0000fe38       $unwind$?dtor$12@?0???$visit_format_arg@V?$width_checker@Uerror_handler@detail@v8@fmt@@@detail@v8@fmt@@V?$basic_format_context@V?$back_insert_iterator@V?$buffer@_W@detail@v8@fmt@@@std@@_W@34@@v8@fmt@@YA_K$$QEAV?$width_checker@Uerror_handler@detail@v8@fmt@@@detail@01@AEBV?$basic_format_arg@V?$basic_format_context@V?$back_insert_iterator@V?$buffer@_W@detail@v8@fmt@@@std@@_W@v8@fmt@@@01@@Z@4HA 0000000180055e38     handles.obj
 0002:0000fe38       $unwind$?dtor$13@?0??PrintHandleInfo@@YA_NKPEAX_NPEAVPerfThread@@@Z@4HA 0000000180055e38     handles.obj
 0002:0000fe38       $unwind$?dtor$1@?0???$do_write_float@V?$back_insert_iterator@V?$buffer@_W@detail@v8@fmt@@@std@@U?$decimal_fp@M@dragonbox@detail@v8@fmt@@_WV?$digit_grouping@_W@567@@detail@v8@fmt@@YA?AV?$back_insert_iterator@V?$buffer@_W@detail@v8@fmt@@@std@@V34@AEBU?$decimal_fp@M@dragonbox@012@AEBU?$basic_format_specs@_W@12@Ufloat_specs@012@Vlocale_ref@012@@Z@4HA 0000000180055e38     handles.obj
 0002:0000fe38       $unwind$?dtor$1@?0???$do_write_float@V?$back_insert_iterator@V?$buffer@_W@detail@v8@fmt@@@std@@U?$decimal_fp@N@dragonbox@detail@v8@fmt@@_WV?$digit_grouping@_W@567@@detail@v8@fmt@@YA?AV?$back_insert_iterator@V?$buffer@_W@detail@v8@fmt@@@std@@V34@AEBU?$decimal_fp@N@dragonbox@012@AEBU?$basic_format_specs@_W@12@Ufloat_specs@012@Vlocale_ref@012@@Z@4HA 0000000180055e38     handles.obj
 0002:0000fe38       $unwind$?dtor$1@?0???$do_write_float@V?$back_insert_iterator@V?$buffer@_W@detail@v8@fmt@@@std@@Ubig_decimal_fp@detail@v8@fmt@@_WV?$digit_grouping@_W@456@@detail@v8@fmt@@YA?AV?$back_insert_iterator@V?$buffer@_W@detail@v8@fmt@@@std@@V34@AEBUbig_decimal_fp@012@AEBU?$basic_format_specs@_W@12@Ufloat_specs@012@Vlocale_ref@012@@Z@4HA 0000000180055e38     handles.obj
 0002:0000fe38       $unwind$?dtor$1@?0???$write_int_localized@V?$back_insert_iterator@V?$buffer@_W@detail@v8@fmt@@@std@@_K_W@detail@v8@fmt@@YA_NAEAV?$back_insert_iterator@V?$buffer@_W@detail@v8@fmt@@@std@@_KIAEBU?$basic_format_specs@_W@12@Vlocale_ref@012@@Z@4HA 0000000180055e38     handles.obj
 0002:0000fe38       $unwind$?dtor$1@?0???R<lambda_1>@?1??GetUserAccountID@@YA@XZ@QEBA?AV?$basic_string@_WU?$char_traits@_W@std@@V?$allocator@_W@2@@std@@XZ@4HA 0000000180055e38     handles.obj
 0002:0000fe38       $unwind$?dtor$1@?0??GetNameByType@@YA?AV?$basic_string@_WU?$char_traits@_W@std@@V?$allocator@_W@2@@std@@PEAXGPEAVPerfThread@@@Z@4HA 0000000180055e38     handles.obj
 0002:0000fe38       $unwind$?dtor$20@?0??GetNameByType@@YA?AV?$basic_string@_WU?$char_traits@_W@std@@V?$allocator@_W@2@@std@@PEAXGPEAVPerfThread@@@Z@4HA 0000000180055e38     handles.obj
 0002:0000fe38       $unwind$?dtor$2@?0???$do_write_float@V?$back_insert_iterator@V?$buffer@_W@detail@v8@fmt@@@std@@U?$decimal_fp@M@dragonbox@detail@v8@fmt@@_WV?$digit_grouping@_W@567@@detail@v8@fmt@@YA?AV?$back_insert_iterator@V?$buffer@_W@detail@v8@fmt@@@std@@V34@AEBU?$decimal_fp@M@dragonbox@012@AEBU?$basic_format_specs@_W@12@Ufloat_specs@012@Vlocale_ref@012@@Z@4HA 0000000180055e38     handles.obj
 0002:0000fe38       $unwind$?dtor$2@?0???$do_write_float@V?$back_insert_iterator@V?$buffer@_W@detail@v8@fmt@@@std@@U?$decimal_fp@N@dragonbox@detail@v8@fmt@@_WV?$digit_grouping@_W@567@@detail@v8@fmt@@YA?AV?$back_insert_iterator@V?$buffer@_W@detail@v8@fmt@@@std@@V34@AEBU?$decimal_fp@N@dragonbox@012@AEBU?$basic_format_specs@_W@12@Ufloat_specs@012@Vlocale_ref@012@@Z@4HA 0000000180055e38     handles.obj
 0002:0000fe38       $unwind$?dtor$2@?0???$do_write_float@V?$back_insert_iterator@V?$buffer@_W@detail@v8@fmt@@@std@@Ubig_decimal_fp@detail@v8@fmt@@_WV?$digit_grouping@_W@456@@detail@v8@fmt@@YA?AV?$back_insert_iterator@V?$buffer@_W@detail@v8@fmt@@@std@@V34@AEBUbig_decimal_fp@012@AEBU?$basic_format_specs@_W@12@Ufloat_specs@012@Vlocale_ref@012@@Z@4HA 0000000180055e38     handles.obj
 0002:0000fe38       $unwind$?dtor$2@?0???$vformat@_W$0A@@v8@fmt@@YA?AV?$basic_string@_WU?$char_traits@_W@std@@V?$allocator@_W@2@@std@@V?$basic_string_view@_W@01@V?$basic_format_args@V?$basic_format_context@V?$back_insert_iterator@V?$buffer@_W@detail@v8@fmt@@@std@@_W@v8@fmt@@@01@@Z@4HA 0000000180055e38     handles.obj
 0002:0000fe38       $unwind$?dtor$2@?0???R<lambda_1>@?1??GetUserAccountID@@YA@XZ@QEBA?AV?$basic_string@_WU?$char_traits@_W@std@@V?$allocator@_W@2@@std@@XZ@4HA 0000000180055e38     handles.obj
 0002:0000fe38       $unwind$?dtor$2@?0??GetFileName@@YA?AV?$basic_string@_WU?$char_traits@_W@std@@V?$allocator@_W@2@@std@@PEAX@Z@4HA 0000000180055e38     handles.obj
 0002:0000fe38       $unwind$?dtor$2@?0??GetNameByType@@YA?AV?$basic_string@_WU?$char_traits@_W@std@@V?$allocator@_W@2@@std@@PEAXGPEAVPerfThread@@@Z@4HA 0000000180055e38     handles.obj
 0002:0000fe38       $unwind$?dtor$3@?0???$do_parse_arg_id@_WAEAUprecision_adapter@?1???$parse_precision@_WAEAV?$specs_checker@V?$specs_handler@_W@detail@v8@fmt@@@detail@v8@fmt@@@detail@v8@fmt@@YAPEB_WPEB_W0AEAV?$specs_checker@V?$specs_handler@_W@detail@v8@fmt@@@234@@Z@@detail@v8@fmt@@YAPEB_WPEB_W0AEAUprecision_adapter@?1???$parse_precision@_WAEAV?$specs_checker@V?$specs_handler@_W@detail@v8@fmt@@@detail@v8@fmt@@@012@YAPEB_W00AEAV?$specs_checker@V?$specs_handler@_W@detail@v8@fmt@@@012@@Z@@Z@4HA 0000000180055e38     handles.obj
 0002:0000fe38       $unwind$?dtor$3@?0???$do_parse_arg_id@_WAEAUwidth_adapter@?1???$parse_width@_WAEAV?$specs_checker@V?$specs_handler@_W@detail@v8@fmt@@@detail@v8@fmt@@@detail@v8@fmt@@YAPEB_WPEB_W0AEAV?$specs_checker@V?$specs_handler@_W@detail@v8@fmt@@@234@@Z@@detail@v8@fmt@@YAPEB_WPEB_W0AEAUwidth_adapter@?1???$parse_width@_WAEAV?$specs_checker@V?$specs_handler@_W@detail@v8@fmt@@@detail@v8@fmt@@@012@YAPEB_W00AEAV?$specs_checker@V?$specs_handler@_W@detail@v8@fmt@@@012@@Z@@Z@4HA 0000000180055e38     handles.obj
 0002:0000fe38       $unwind$?dtor$3@?0???$parse_align@_WAEAV?$specs_checker@V?$specs_handler@_W@detail@v8@fmt@@@detail@v8@fmt@@@detail@v8@fmt@@YAPEB_WPEB_W0AEAV?$specs_checker@V?$specs_handler@_W@detail@v8@fmt@@@012@@Z@4HA 0000000180055e38     handles.obj
 0002:0000fe38       $unwind$?dtor$3@?0???$parse_precision@_WAEAV?$specs_checker@V?$specs_handler@_W@detail@v8@fmt@@@detail@v8@fmt@@@detail@v8@fmt@@YAPEB_WPEB_W0AEAV?$specs_checker@V?$specs_handler@_W@detail@v8@fmt@@@012@@Z@4HA 0000000180055e38     handles.obj
 0002:0000fe38       $unwind$?dtor$3@?0???$parse_replacement_field@_WAEAUformat_handler@?1???$vformat_to@_W@detail@v8@fmt@@YAXAEAV?$buffer@_W@234@V?$basic_string_view@_W@34@V?$basic_format_args@V?$basic_format_context@V?$back_insert_iterator@V?$buffer@_W@detail@v8@fmt@@@std@@_W@v8@fmt@@@34@Vlocale_ref@234@@Z@@detail@v8@fmt@@YAPEB_WPEB_W0AEAUformat_handler@?1???$vformat_to@_W@012@YAXAEAV?$buffer@_W@012@V?$basic_string_view@_W@12@V?$basic_format_args@V?$basic_format_context@V?$back_insert_iterator@V?$buffer@_W@detail@v8@fmt@@@std@@_W@v8@fmt@@@12@Vlocale_ref@012@@Z@@Z@4HA 0000000180055e38     handles.obj
 0002:0000fe38       $unwind$?dtor$3@?0???$parse_width@_WAEAV?$specs_checker@V?$specs_handler@_W@detail@v8@fmt@@@detail@v8@fmt@@@detail@v8@fmt@@YAPEB_WPEB_W0AEAV?$specs_checker@V?$specs_handler@_W@detail@v8@fmt@@@012@@Z@4HA 0000000180055e38     handles.obj
 0002:0000fe38       $unwind$?dtor$3@?0???$visit_format_arg@V?$precision_checker@Uerror_handler@detail@v8@fmt@@@detail@v8@fmt@@V?$basic_format_context@V?$back_insert_iterator@V?$buffer@_W@detail@v8@fmt@@@std@@_W@34@@v8@fmt@@YA_K$$QEAV?$precision_checker@Uerror_handler@detail@v8@fmt@@@detail@01@AEBV?$basic_format_arg@V?$basic_format_context@V?$back_insert_iterator@V?$buffer@_W@detail@v8@fmt@@@std@@_W@v8@fmt@@@01@@Z@4HA 0000000180055e38     handles.obj
 0002:0000fe38       $unwind$?dtor$3@?0???$visit_format_arg@V?$width_checker@Uerror_handler@detail@v8@fmt@@@detail@v8@fmt@@V?$basic_format_context@V?$back_insert_iterator@V?$buffer@_W@detail@v8@fmt@@@std@@_W@34@@v8@fmt@@YA_K$$QEAV?$width_checker@Uerror_handler@detail@v8@fmt@@@detail@01@AEBV?$basic_format_arg@V?$basic_format_context@V?$back_insert_iterator@V?$buffer@_W@detail@v8@fmt@@@std@@_W@v8@fmt@@@01@@Z@4HA 0000000180055e38     handles.obj
 0002:0000fe38       $unwind$?dtor$3@?0???$write@_WV?$back_insert_iterator@V?$buffer@_W@detail@v8@fmt@@@std@@@detail@v8@fmt@@YA?AV?$back_insert_iterator@V?$buffer@_W@detail@v8@fmt@@@std@@V34@_WAEBU?$basic_format_specs@_W@12@Vlocale_ref@012@@Z@4HA 0000000180055e38     handles.obj
 0002:0000fe38       $unwind$?dtor$3@?0???R<lambda_1>@?1??GetUserAccountID@@YA@XZ@QEBA?AV?$basic_string@_WU?$char_traits@_W@std@@V?$allocator@_W@2@@std@@XZ@4HA 0000000180055e38     handles.obj
 0002:0000fe38       $unwind$?dtor$3@?0??GetNameByType@@YA?AV?$basic_string@_WU?$char_traits@_W@std@@V?$allocator@_W@2@@std@@PEAXGPEAVPerfThread@@@Z@4HA 0000000180055e38     handles.obj
 0002:0000fe38       $unwind$?dtor$3@?0??PrintHandleInfo@@YA_NKPEAX_NPEAVPerfThread@@@Z@4HA 0000000180055e38     handles.obj
 0002:0000fe38       $unwind$?dtor$5@?0??PrintHandleInfo@@YA_NKPEAX_NPEAVPerfThread@@@Z@4HA 0000000180055e38     handles.obj
 0002:0000fe38       $unwind$?dtor$6@?0???$parse_precision@_WAEAV?$specs_checker@V?$specs_handler@_W@detail@v8@fmt@@@detail@v8@fmt@@@detail@v8@fmt@@YAPEB_WPEB_W0AEAV?$specs_checker@V?$specs_handler@_W@detail@v8@fmt@@@012@@Z@4HA 0000000180055e38     handles.obj
 0002:0000fe38       $unwind$?dtor$6@?0???$parse_width@_WAEAV?$specs_checker@V?$specs_handler@_W@detail@v8@fmt@@@detail@v8@fmt@@@detail@v8@fmt@@YAPEB_WPEB_W0AEAV?$specs_checker@V?$specs_handler@_W@detail@v8@fmt@@@012@@Z@4HA 0000000180055e38     handles.obj
 0002:0000fe38       $unwind$?dtor$6@?0???$visit_format_arg@V?$precision_checker@Uerror_handler@detail@v8@fmt@@@detail@v8@fmt@@V?$basic_format_context@V?$back_insert_iterator@V?$buffer@_W@detail@v8@fmt@@@std@@_W@34@@v8@fmt@@YA_K$$QEAV?$precision_checker@Uerror_handler@detail@v8@fmt@@@detail@01@AEBV?$basic_format_arg@V?$basic_format_context@V?$back_insert_iterator@V?$buffer@_W@detail@v8@fmt@@@std@@_W@v8@fmt@@@01@@Z@4HA 0000000180055e38     handles.obj
 0002:0000fe38       $unwind$?dtor$6@?0???$visit_format_arg@V?$width_checker@Uerror_handler@detail@v8@fmt@@@detail@v8@fmt@@V?$basic_format_context@V?$back_insert_iterator@V?$buffer@_W@detail@v8@fmt@@@std@@_W@34@@v8@fmt@@YA_K$$QEAV?$width_checker@Uerror_handler@detail@v8@fmt@@@detail@01@AEBV?$basic_format_arg@V?$basic_format_context@V?$back_insert_iterator@V?$buffer@_W@detail@v8@fmt@@@std@@_W@v8@fmt@@@01@@Z@4HA 0000000180055e38     handles.obj
 0002:0000fe38       $unwind$?dtor$6@?0??PrintHandleInfo@@YA_NKPEAX_NPEAVPerfThread@@@Z@4HA 0000000180055e38     handles.obj
 0002:0000fe38       $unwind$?dtor$7@?0??GetFileName@@YA?AV?$basic_string@_WU?$char_traits@_W@std@@V?$allocator@_W@2@@std@@PEAX@Z@4HA 0000000180055e38     handles.obj
 0002:0000fe38       $unwind$?dtor$9@?0???$parse_precision@_WAEAV?$specs_checker@V?$specs_handler@_W@detail@v8@fmt@@@detail@v8@fmt@@@detail@v8@fmt@@YAPEB_WPEB_W0AEAV?$specs_checker@V?$specs_handler@_W@detail@v8@fmt@@@012@@Z@4HA 0000000180055e38     handles.obj
 0002:0000fe38       $unwind$?dtor$9@?0???$visit_format_arg@V?$precision_checker@Uerror_handler@detail@v8@fmt@@@detail@v8@fmt@@V?$basic_format_context@V?$back_insert_iterator@V?$buffer@_W@detail@v8@fmt@@@std@@_W@34@@v8@fmt@@YA_K$$QEAV?$precision_checker@Uerror_handler@detail@v8@fmt@@@detail@01@AEBV?$basic_format_arg@V?$basic_format_context@V?$back_insert_iterator@V?$buffer@_W@detail@v8@fmt@@@std@@_W@v8@fmt@@@01@@Z@4HA 0000000180055e38     handles.obj
 0002:0000fe38       $unwind$?dtor$9@?0???$visit_format_arg@V?$width_checker@Uerror_handler@detail@v8@fmt@@@detail@v8@fmt@@V?$basic_format_context@V?$back_insert_iterator@V?$buffer@_W@detail@v8@fmt@@@std@@_W@34@@v8@fmt@@YA_K$$QEAV?$width_checker@Uerror_handler@detail@v8@fmt@@@detail@01@AEBV?$basic_format_arg@V?$basic_format_context@V?$back_insert_iterator@V?$buffer@_W@detail@v8@fmt@@@std@@_W@v8@fmt@@@01@@Z@4HA 0000000180055e38     handles.obj
 0002:0000fe38       $unwind$?dtor$0@?0???$emplace@AEBKUProcessPerfData@@@?$_Hash@V?$_Umap_traits@KUProcessPerfData@@V?$_Uhash_compare@KU?$hash@K@std@@U?$equal_to@K@2@@std@@V?$allocator@U?$pair@$$CBKUProcessPerfData@@@std@@@3@$00@std@@@std@@QEAA?AV?$_List_iterator@V?$_List_val@U?$_List_simple_types@U?$pair@$$CBKUProcessPerfData@@@std@@@std@@@std@@@1@AEBK$$QEAUProcessPerfData@@@Z@4HA 0000000180055e38     perfthread.obj
 0002:0000fe38       $unwind$?dtor$0@?0???$transform@V?$_List_const_iterator@V?$_List_val@U?$_List_simple_types@U?$pair@$$CBKUProcessPerfData@@@std@@@std@@@std@@@std@@V?$back_insert_iterator@V?$vector@UProcessPerfData@@V?$allocator@UProcessPerfData@@@std@@@std@@@2@V<lambda_1>@?2??RefreshWMIData@PerfThread@@AEAAXXZ@@std@@YA?AV?$back_insert_iterator@V?$vector@UProcessPerfData@@V?$allocator@UProcessPerfData@@@std@@@std@@@0@V?$_List_const_iterator@V?$_List_val@U?$_List_simple_types@U?$pair@$$CBKUProcessPerfData@@@std@@@std@@@std@@@0@0V10@V<lambda_1>@?2??RefreshWMIData@PerfThread@@AEAAXXZ@@Z@4HA 0000000180055e38     perfthread.obj
 0002:0000fe38       $unwind$?dtor$0@?0??Refresh@PerfThread@@AEAAXXZ@4HA 0000000180055e38     perfthread.obj
 0002:0000fe38       $unwind$?dtor$0@?0??RefreshWMIData@PerfThread@@AEAAXXZ@4HA 0000000180055e38     perfthread.obj
 0002:0000fe38       $unwind$?dtor$11@?0??Refresh@PerfThread@@AEAAXXZ@4HA 0000000180055e38     perfthread.obj
 0002:0000fe38       $unwind$?dtor$12@?0???0PerfThread@@QEAA@PEAVPlist@@PEB_W11@Z@4HA 0000000180055e38     perfthread.obj
 0002:0000fe38       $unwind$?dtor$13@?0???0PerfThread@@QEAA@PEAVPlist@@PEB_W11@Z@4HA 0000000180055e38     perfthread.obj
 0002:0000fe38       $unwind$?dtor$1@?0???$emplace@AEBKUProcessPerfData@@@?$_Hash@V?$_Umap_traits@KUProcessPerfData@@V?$_Uhash_compare@KU?$hash@K@std@@U?$equal_to@K@2@@std@@V?$allocator@U?$pair@$$CBKUProcessPerfData@@@std@@@3@$00@std@@@std@@QEAA?AV?$_List_iterator@V?$_List_val@U?$_List_simple_types@U?$pair@$$CBKUProcessPerfData@@@std@@@std@@@std@@@1@AEBK$$QEAUProcessPerfData@@@Z@4HA 0000000180055e38     perfthread.obj
 0002:0000fe38       $unwind$?dtor$1@?0??Refresh@PerfThread@@AEAAXXZ@4HA 0000000180055e38     perfthread.obj
 0002:0000fe38       $unwind$?dtor$1@?0??RefreshWMIData@PerfThread@@AEAAXXZ@4HA 0000000180055e38     perfthread.obj
 0002:0000fe38       $unwind$?dtor$21@?0??RefreshWMIData@PerfThread@@AEAAXXZ@4HA 0000000180055e38     perfthread.obj
 0002:0000fe38       $unwind$?dtor$29@?0??RefreshWMIData@PerfThread@@AEAAXXZ@4HA 0000000180055e38     perfthread.obj
 0002:0000fe38       $unwind$?dtor$2@?0??Refresh@PerfThread@@AEAAXXZ@4HA 0000000180055e38     perfthread.obj
 0002:0000fe38       $unwind$?dtor$4@?0??RefreshWMIData@PerfThread@@AEAAXXZ@4HA 0000000180055e38     perfthread.obj
 0002:0000fe38       $unwind$?dtor$6@?0??RefreshWMIData@PerfThread@@AEAAXXZ@4HA 0000000180055e38     perfthread.obj
 0002:0000fe38       $unwind$?dtor$7@?0??Refresh@PerfThread@@AEAAXXZ@4HA 0000000180055e38     perfthread.obj
 0002:0000fe38       $unwind$?dtor$9@?0??RefreshWMIData@PerfThread@@AEAAXXZ@4HA 0000000180055e38     perfthread.obj
 0002:0000fe38       $unwind$?dtor$0@?0??ExecMethod@WMIConnection@@AEAAHKPEB_W0K@Z@4HA 0000000180055e38     wmi.obj
 0002:0000fe38       $unwind$?dtor$0@?0??GetProcessOwner@WMIConnection@@QEAA?AV?$basic_string@_WU?$char_traits@_W@std@@V?$allocator@_W@2@@std@@KPEAV23@@Z@4HA 0000000180055e38     wmi.obj
 0002:0000fe38       $unwind$?dtor$0@?0??GetProcessProperty@WMIConnection@@AEAA_NKPEB_WAEBV?$function@$$A6AXAEBUtagVARIANT@@@Z@std@@@Z@4HA 0000000180055e38     wmi.obj
 0002:0000fe38       $unwind$?dtor$0@?0??GetProcessSessionId@WMIConnection@@QEAAKK@Z@4HA 0000000180055e38     wmi.obj
 0002:0000fe38       $unwind$?dtor$0@?0??GetProcessUserSid@WMIConnection@@QEAA?AV?$basic_string@_WU?$char_traits@_W@std@@V?$allocator@_W@2@@std@@K@Z@4HA 0000000180055e38     wmi.obj
 0002:0000fe38       $unwind$?dtor$10@?0??ExecMethod@WMIConnection@@AEAAHKPEB_W0K@Z@4HA 0000000180055e38     wmi.obj
 0002:0000fe38       $unwind$?dtor$1@?0??ExecMethod@WMIConnection@@AEAAHKPEB_W0K@Z@4HA 0000000180055e38     wmi.obj
 0002:0000fe38       $unwind$?dtor$1@?0??GetProcessOwner@WMIConnection@@QEAA?AV?$basic_string@_WU?$char_traits@_W@std@@V?$allocator@_W@2@@std@@KPEAV23@@Z@4HA 0000000180055e38     wmi.obj
 0002:0000fe38       $unwind$?dtor$1@?0??GetProcessProperty@WMIConnection@@AEAA_NKPEB_WAEBV?$function@$$A6AXAEBUtagVARIANT@@@Z@std@@@Z@4HA 0000000180055e38     wmi.obj
 0002:0000fe38       $unwind$?dtor$1@?0??GetProcessUserSid@WMIConnection@@QEAA?AV?$basic_string@_WU?$char_traits@_W@std@@V?$allocator@_W@2@@std@@K@Z@4HA 0000000180055e38     wmi.obj
 0002:0000fe38       $unwind$?dtor$2@?0??ExecMethod@WMIConnection@@AEAAHKPEB_W0K@Z@4HA 0000000180055e38     wmi.obj
 0002:0000fe38       $unwind$?dtor$2@?0??GetProcessOwner@WMIConnection@@QEAA?AV?$basic_string@_WU?$char_traits@_W@std@@V?$allocator@_W@2@@std@@KPEAV23@@Z@4HA 0000000180055e38     wmi.obj
 0002:0000fe38       $unwind$?dtor$2@?0??GetProcessProperty@WMIConnection@@AEAA_NKPEB_WAEBV?$function@$$A6AXAEBUtagVARIANT@@@Z@std@@@Z@4HA 0000000180055e38     wmi.obj
 0002:0000fe38       $unwind$?dtor$2@?0??GetProcessUserSid@WMIConnection@@QEAA?AV?$basic_string@_WU?$char_traits@_W@std@@V?$allocator@_W@2@@std@@K@Z@4HA 0000000180055e38     wmi.obj
 0002:0000fe38       $unwind$?dtor$3@?0??ExecMethod@WMIConnection@@AEAAHKPEB_W0K@Z@4HA 0000000180055e38     wmi.obj
 0002:0000fe38       $unwind$?dtor$3@?0??GetProcessOwner@WMIConnection@@QEAA?AV?$basic_string@_WU?$char_traits@_W@std@@V?$allocator@_W@2@@std@@KPEAV23@@Z@4HA 0000000180055e38     wmi.obj
 0002:0000fe38       $unwind$?dtor$3@?0??GetProcessUserSid@WMIConnection@@QEAA?AV?$basic_string@_WU?$char_traits@_W@std@@V?$allocator@_W@2@@std@@K@Z@4HA 0000000180055e38     wmi.obj
 0002:0000fe38       $unwind$?dtor$4@?0??ExecMethod@WMIConnection@@AEAAHKPEB_W0K@Z@4HA 0000000180055e38     wmi.obj
 0002:0000fe38       $unwind$?dtor$5@?0??ExecMethod@WMIConnection@@AEAAHKPEB_W0K@Z@4HA 0000000180055e38     wmi.obj
 0002:0000fe38       $unwind$?dtor$5@?0??GetProcessOwner@WMIConnection@@QEAA?AV?$basic_string@_WU?$char_traits@_W@std@@V?$allocator@_W@2@@std@@KPEAV23@@Z@4HA 0000000180055e38     wmi.obj
 0002:0000fe38       $unwind$?dtor$5@?0??GetProcessUserSid@WMIConnection@@QEAA?AV?$basic_string@_WU?$char_traits@_W@std@@V?$allocator@_W@2@@std@@K@Z@4HA 0000000180055e38     wmi.obj
 0002:0000fe38       $unwind$?dtor$6@?0??ExecMethod@WMIConnection@@AEAAHKPEB_W0K@Z@4HA 0000000180055e38     wmi.obj
 0002:0000fe38       $unwind$?dtor$7@?0??ExecMethod@WMIConnection@@AEAAHKPEB_W0K@Z@4HA 0000000180055e38     wmi.obj
 0002:0000fe38       $unwind$?dtor$8@?0??ExecMethod@WMIConnection@@AEAAHKPEB_W0K@Z@4HA 0000000180055e38     wmi.obj
 0002:0000fe38       $unwind$?dtor$9@?0??ExecMethod@WMIConnection@@AEAAHKPEB_W0K@Z@4HA 0000000180055e38     wmi.obj
 0002:0000fe38       $unwind$?dtor$0@?0??_Init@locale@std@@CAPEAV_Locimp@12@_N@Z@4HA 0000000180055e38     libcpmt:locale0.obj
 0002:0000fe38       $unwind$?dtor$0@?0??_wcstombs_l_helper@@YA_KPEADPEB_W_KPEAU__crt_locale_pointers@@@Z@4HA 0000000180055e38     libucrt:wcstombs.obj
 0002:0000fe40       $unwind$??1_Locinfo@std@@QEAA@XZ 0000000180055e40     format.obj
 0002:0000fe58       $ip2state$??1_Locinfo@std@@QEAA@XZ 0000000180055e58     format.obj
 0002:0000fe60       $unwind$?throw_format_error@detail@v8@fmt@@YAXPEBD@Z 0000000180055e60     format.obj
 0002:0000fe78       $ip2state$?throw_format_error@detail@v8@fmt@@YAXPEBD@Z 0000000180055e78     format.obj
 0002:0000fe80       $unwind$?fmt_snprintf@detail@v8@fmt@@YAHPEAD_KPEBDZZ 0000000180055e80     format.obj
 0002:0000fe8c       $unwind$?add_compare@detail@v8@fmt@@YAHAEBVbigint@123@00@Z 0000000180055e8c     format.obj
 0002:0000fea0       $unwind$?assign_pow10@bigint@detail@v8@fmt@@QEAAXH@Z 0000000180055ea0     format.obj
 0002:0000feb4       $unwind$?square@bigint@detail@v8@fmt@@QEAAXXZ 0000000180055eb4     format.obj
 0002:0000fed0       $stateUnwindMap$?square@bigint@detail@v8@fmt@@QEAAXXZ 0000000180055ed0     format.obj
 0002:0000fee0       $ip2state$?square@bigint@detail@v8@fmt@@QEAAXXZ 0000000180055ee0     format.obj
 0002:0000fef8       $unwind$?get_cached_power@?$cache_accessor@N@dragonbox@detail@v8@fmt@@SA?AUuint128_wrapper@345@H@Z 0000000180055ef8     format.obj
 0002:0000ff08       $unwind$?format_dragon@detail@v8@fmt@@YAXUfp@123@_NHAEAV?$buffer@D@123@AEAH@Z 0000000180055f08     format.obj
 0002:0000ff28       $stateUnwindMap$?format_dragon@detail@v8@fmt@@YAXUfp@123@_NHAEAV?$buffer@D@123@AEAH@Z 0000000180055f28     format.obj
 0002:0000ff50       $ip2state$?format_dragon@detail@v8@fmt@@YAXUfp@123@_NHAEAV?$buffer@D@123@AEAH@Z 0000000180055f50     format.obj
 0002:0000ff60       $unwind$?assign@?$basic_string@_WU?$char_traits@_W@std@@V?$allocator@_W@2@@std@@QEAAAEAV12@QEB_W_K@Z 0000000180055f60     format.obj
 0002:0000ff70       $unwind$?assign@?$basic_string@DU?$char_traits@D@std@@V?$allocator@D@2@@std@@QEAAAEAV12@QEBD_K@Z 0000000180055f70     format.obj
 0002:0000ff80       $unwind$??$thousands_sep_impl@_W@detail@v8@fmt@@YA?AU?$thousands_sep_result@_W@012@Vlocale_ref@012@@Z 0000000180055f80     format.obj
 0002:0000ff98       $stateUnwindMap$??$thousands_sep_impl@_W@detail@v8@fmt@@YA?AU?$thousands_sep_result@_W@012@Vlocale_ref@012@@Z 0000000180055f98     format.obj
 0002:0000ffc0       $ip2state$??$thousands_sep_impl@_W@detail@v8@fmt@@YA?AU?$thousands_sep_result@_W@012@Vlocale_ref@012@@Z 0000000180055fc0     format.obj
 0002:0000ffe8       $unwind$?grow@?$basic_memory_buffer@H$0BPE@V?$allocator@H@std@@@v8@fmt@@MEAAX_K@Z 0000000180055fe8     format.obj
 0002:0000ffe8       $unwind$?grow@?$basic_memory_buffer@I$0CA@V?$allocator@I@std@@@v8@fmt@@MEAAX_K@Z 0000000180055fe8     format.obj
 0002:0000ffe8       $unwind$?grow@?$basic_memory_buffer@_W$0BPE@V?$allocator@_W@std@@@v8@fmt@@MEAAX_K@Z 0000000180055fe8     format.obj
 0002:0000fff8       $unwind$??$snprintf_float@N@detail@v8@fmt@@YAHNHUfloat_specs@012@AEAV?$buffer@D@012@@Z 0000000180055ff8     format.obj
 0002:00010010       $unwind$??$snprintf_float@O@detail@v8@fmt@@YAHOHUfloat_specs@012@AEAV?$buffer@D@012@@Z 0000000180056010     format.obj
 0002:00010028       $unwind$??$to_decimal@M@dragonbox@detail@v8@fmt@@YA?AU?$decimal_fp@M@0123@M@Z 0000000180056028     format.obj
 0002:00010044       $unwind$?do_truename@?$numpunct@_W@std@@MEBA?AV?$basic_string@_WU?$char_traits@_W@std@@V?$allocator@_W@2@@2@XZ 0000000180056044     format.obj
 0002:00010058       $stateUnwindMap$??R?$default_delete@VWMIConnection@@@std@@QEBAXPEAVWMIConnection@@@Z 0000000180056058     Pclass.obj
 0002:00010058       $stateUnwindMap$ProcessPanelEventW 0000000180056058     Proclist.obj
 0002:00010058       $stateUnwindMap$??0?$basic_string@_WU?$char_traits@_W@std@@V?$allocator@_W@2@@std@@QEAA@QEB_W@Z 0000000180056058     format.obj
 0002:00010058       $stateUnwindMap$?do_falsename@?$numpunct@_W@std@@MEBA?AV?$basic_string@_WU?$char_traits@_W@std@@V?$allocator@_W@2@@2@XZ 0000000180056058     format.obj
 0002:00010058       $stateUnwindMap$?do_grouping@?$numpunct@_W@std@@MEBA?AV?$basic_string@DU?$char_traits@D@std@@V?$allocator@D@2@@2@XZ 0000000180056058     format.obj
 0002:00010058       $stateUnwindMap$?do_truename@?$numpunct@_W@std@@MEBA?AV?$basic_string@_WU?$char_traits@_W@std@@V?$allocator@_W@2@@2@XZ 0000000180056058     format.obj
 0002:00010058       $stateUnwindMap$??0?$basic_string@_WU?$char_traits@_W@std@@V?$allocator@_W@2@@std@@QEAA@XZ 0000000180056058     handles.obj
 0002:00010058       $stateUnwindMap$??1PerfThread@@QEAA@XZ 0000000180056058     perfthread.obj
 0002:00010058       $stateUnwindMap$??1?$ptr_setter@V?$unique_ptr@UIWbemClassObject@@Ucom_closer@@@std@@@@QEAA@XZ 0000000180056058     wmi.obj
 0002:00010060       $ip2state$?do_truename@?$numpunct@_W@std@@MEBA?AV?$basic_string@_WU?$char_traits@_W@std@@V?$allocator@_W@2@@2@XZ 0000000180056060     format.obj
 0002:00010068       $unwind$?do_falsename@?$numpunct@_W@std@@MEBA?AV?$basic_string@_WU?$char_traits@_W@std@@V?$allocator@_W@2@@2@XZ 0000000180056068     format.obj
 0002:00010080       $ip2state$?do_falsename@?$numpunct@_W@std@@MEBA?AV?$basic_string@_WU?$char_traits@_W@std@@V?$allocator@_W@2@@2@XZ 0000000180056080     format.obj
 0002:00010088       $unwind$?do_grouping@?$numpunct@_W@std@@MEBA?AV?$basic_string@DU?$char_traits@D@std@@V?$allocator@D@2@@2@XZ 0000000180056088     format.obj
 0002:000100a0       $ip2state$?do_grouping@?$numpunct@_W@std@@MEBA?AV?$basic_string@DU?$char_traits@D@std@@V?$allocator@D@2@@2@XZ 00000001800560a0     format.obj
 0002:000100a8       $unwind$??0?$basic_string@_WU?$char_traits@_W@std@@V?$allocator@_W@2@@std@@QEAA@QEB_W@Z 00000001800560a8     format.obj
 0002:000100c0       $ip2state$??0?$basic_string@_WU?$char_traits@_W@std@@V?$allocator@_W@2@@std@@QEAA@QEB_W@Z 00000001800560c0     format.obj
 0002:000100c8       $unwind$??$use_facet@V?$numpunct@_W@std@@@std@@YAAEBV?$numpunct@_W@0@AEBVlocale@0@@Z 00000001800560c8     format.obj
 0002:000100e0       $stateUnwindMap$??$use_facet@V?$numpunct@_W@std@@@std@@YAAEBV?$numpunct@_W@0@AEBVlocale@0@@Z 00000001800560e0     format.obj
 0002:000100f0       $ip2state$??$use_facet@V?$numpunct@_W@std@@@std@@YAAEBV?$numpunct@_W@0@AEBVlocale@0@@Z 00000001800560f0     format.obj
 0002:00010110       $unwind$??$write@DVappender@v8@fmt@@I$0A@@detail@v8@fmt@@YA?AVappender@12@V312@I@Z 0000000180056110     format.obj
 0002:00010128       $unwind$??$write@DVappender@v8@fmt@@_K$0A@@detail@v8@fmt@@YA?AVappender@12@V312@_K@Z 0000000180056128     format.obj
 0002:00010140       $unwind$?_Getcat@?$numpunct@_W@std@@SA_KPEAPEBVfacet@locale@2@PEBV42@@Z 0000000180056140     format.obj
 0002:00010158       $stateUnwindMap$?_Getcat@?$numpunct@_W@std@@SA_KPEAPEBVfacet@locale@2@PEBV42@@Z 0000000180056158     format.obj
 0002:000101c0       $ip2state$?_Getcat@?$numpunct@_W@std@@SA_KPEAPEBVfacet@locale@2@PEBV42@@Z 00000001800561c0     format.obj
 0002:000101e8       $unwind$?dtor$0@?0???0Plist@@QEAA@XZ@4HA 00000001800561e8     Pclass.obj
 0002:000101e8       $unwind$?dtor$10@?0???0Plist@@QEAA@XZ@4HA 00000001800561e8     Pclass.obj
 0002:000101e8       $unwind$?dtor$13@?0??GetFindData@Plist@@QEAAHAEAPEAUPluginPanelItem@@AEA_K_K@Z@4HA 00000001800561e8     Pclass.obj
 0002:000101e8       $unwind$?dtor$14@?0??GetFindData@Plist@@QEAAHAEAPEAUPluginPanelItem@@AEA_K_K@Z@4HA 00000001800561e8     Pclass.obj
 0002:000101e8       $unwind$?dtor$1@?0???0Plist@@QEAA@XZ@4HA 00000001800561e8     Pclass.obj
 0002:000101e8       $unwind$?dtor$24@?0???$_Uninitialized_copy@PEBUmode@@V?$allocator@Umode@@@std@@@std@@YAPEAUmode@@QEBU1@0PEAU1@AEAV?$allocator@Umode@@@0@@Z@4HA 00000001800561e8     Pclass.obj
 0002:000101e8       $unwind$?dtor$2@?0???0Plist@@QEAA@XZ@4HA 00000001800561e8     Pclass.obj
 0002:000101e8       $unwind$?dtor$33@?0???$_Uninitialized_copy@PEBUmode@@V?$allocator@Umode@@@std@@@std@@YAPEAUmode@@QEBU1@0PEAU1@AEAV?$allocator@Umode@@@0@@Z@4HA 00000001800561e8     Pclass.obj
 0002:000101e8       $unwind$?dtor$6@?0??Connect@Plist@@QEAA_NPEB_W00@Z@4HA 00000001800561e8     Pclass.obj
 0002:000101e8       $unwind$?dtor$2@?0??GetList@@YA_NAEAPEAUPluginPanelItem@@AEA_KAEAVPerfThread@@@Z@4HA 00000001800561e8     Plist.obj
 0002:000101e8       $unwind$?dtor$3@?0??GetList@@YA_NAEAPEAUPluginPanelItem@@AEA_KAEAVPerfThread@@@Z@4HA 00000001800561e8     Plist.obj
 0002:000101e8       $unwind$?dtor$0@?0??_Getcat@?$numpunct@_W@std@@SA_KPEAPEBVfacet@locale@2@PEBV42@@Z@4HA 00000001800561e8     format.obj
 0002:000101e8       $unwind$?dtor$3@?0??_Getcat@?$numpunct@_W@std@@SA_KPEAPEBVfacet@locale@2@PEBV42@@Z@4HA 00000001800561e8     format.obj
 0002:000101e8       $unwind$?dtor$4@?0??_Getcat@?$numpunct@_W@std@@SA_KPEAPEBVfacet@locale@2@PEBV42@@Z@4HA 00000001800561e8     format.obj
 0002:000101e8       $unwind$?dtor$5@?0??_Getcat@?$numpunct@_W@std@@SA_KPEAPEBVfacet@locale@2@PEBV42@@Z@4HA 00000001800561e8     format.obj
 0002:000101e8       $unwind$?dtor$6@?0??_Getcat@?$numpunct@_W@std@@SA_KPEAPEBVfacet@locale@2@PEBV42@@Z@4HA 00000001800561e8     format.obj
 0002:000101e8       $unwind$?dtor$7@?0??_Getcat@?$numpunct@_W@std@@SA_KPEAPEBVfacet@locale@2@PEBV42@@Z@4HA 00000001800561e8     format.obj
 0002:000101e8       $unwind$?dtor$8@?0??_Getcat@?$numpunct@_W@std@@SA_KPEAPEBVfacet@locale@2@PEBV42@@Z@4HA 00000001800561e8     format.obj
 0002:000101e8       $unwind$?dtor$0@?0???0PerfThread@@QEAA@PEAVPlist@@PEB_W11@Z@4HA 00000001800561e8     perfthread.obj
 0002:000101e8       $unwind$?dtor$0@?0???0ProcessPerfData@@QEAA@AEBU0@@Z@4HA 00000001800561e8     perfthread.obj
 0002:000101e8       $unwind$?dtor$10@?0???0PerfThread@@QEAA@PEAVPlist@@PEB_W11@Z@4HA 00000001800561e8     perfthread.obj
 0002:000101e8       $unwind$?dtor$11@?0???0PerfThread@@QEAA@PEAVPlist@@PEB_W11@Z@4HA 00000001800561e8     perfthread.obj
 0002:000101e8       $unwind$?dtor$17@?0??Refresh@PerfThread@@AEAAXXZ@4HA 00000001800561e8     perfthread.obj
 0002:000101e8       $unwind$?dtor$18@?0??Refresh@PerfThread@@AEAAXXZ@4HA 00000001800561e8     perfthread.obj
 0002:000101e8       $unwind$?dtor$1@?0???0?$unordered_multimap@KUProcessPerfData@@U?$hash@K@std@@U?$equal_to@K@3@V?$allocator@U?$pair@$$CBKUProcessPerfData@@@std@@@3@@std@@QEAA@XZ@4HA 00000001800561e8     perfthread.obj
 0002:000101e8       $unwind$?dtor$1@?0???0PerfThread@@QEAA@PEAVPlist@@PEB_W11@Z@4HA 00000001800561e8     perfthread.obj
 0002:000101e8       $unwind$?dtor$1@?0???0ProcessPerfData@@QEAA@AEBU0@@Z@4HA 00000001800561e8     perfthread.obj
 0002:000101e8       $unwind$?dtor$2@?0???$transform@V?$_List_const_iterator@V?$_List_val@U?$_List_simple_types@U?$pair@$$CBKUProcessPerfData@@@std@@@std@@@std@@@std@@V?$back_insert_iterator@V?$vector@UProcessPerfData@@V?$allocator@UProcessPerfData@@@std@@@std@@@2@V<lambda_1>@?2??RefreshWMIData@PerfThread@@AEAAXXZ@@std@@YA?AV?$back_insert_iterator@V?$vector@UProcessPerfData@@V?$allocator@UProcessPerfData@@@std@@@std@@@0@V?$_List_const_iterator@V?$_List_val@U?$_List_simple_types@U?$pair@$$CBKUProcessPerfData@@@std@@@std@@@std@@@0@0V10@V<lambda_1>@?2??RefreshWMIData@PerfThread@@AEAAXXZ@@Z@4HA 00000001800561e8     perfthread.obj
 0002:000101e8       $unwind$?dtor$2@?0???0?$unordered_multimap@KUProcessPerfData@@U?$hash@K@std@@U?$equal_to@K@3@V?$allocator@U?$pair@$$CBKUProcessPerfData@@@std@@@3@@std@@QEAA@XZ@4HA 00000001800561e8     perfthread.obj
 0002:000101e8       $unwind$?dtor$2@?0???0PerfThread@@QEAA@PEAVPlist@@PEB_W11@Z@4HA 00000001800561e8     perfthread.obj
 0002:000101e8       $unwind$?dtor$2@?0???0ProcessPerfData@@QEAA@AEBU0@@Z@4HA 00000001800561e8     perfthread.obj
 0002:000101e8       $unwind$?dtor$3@?0???$transform@V?$_List_const_iterator@V?$_List_val@U?$_List_simple_types@U?$pair@$$CBKUProcessPerfData@@@std@@@std@@@std@@@std@@V?$back_insert_iterator@V?$vector@UProcessPerfData@@V?$allocator@UProcessPerfData@@@std@@@std@@@2@V<lambda_1>@?2??RefreshWMIData@PerfThread@@AEAAXXZ@@std@@YA?AV?$back_insert_iterator@V?$vector@UProcessPerfData@@V?$allocator@UProcessPerfData@@@std@@@std@@@0@V?$_List_const_iterator@V?$_List_val@U?$_List_simple_types@U?$pair@$$CBKUProcessPerfData@@@std@@@std@@@std@@@0@0V10@V<lambda_1>@?2??RefreshWMIData@PerfThread@@AEAAXXZ@@Z@4HA 00000001800561e8     perfthread.obj
 0002:000101e8       $unwind$?dtor$3@?0???0PerfThread@@QEAA@PEAVPlist@@PEB_W11@Z@4HA 00000001800561e8     perfthread.obj
 0002:000101e8       $unwind$?dtor$4@?0???$transform@V?$_List_const_iterator@V?$_List_val@U?$_List_simple_types@U?$pair@$$CBKUProcessPerfData@@@std@@@std@@@std@@@std@@V?$back_insert_iterator@V?$vector@UProcessPerfData@@V?$allocator@UProcessPerfData@@@std@@@std@@@2@V<lambda_1>@?2??RefreshWMIData@PerfThread@@AEAAXXZ@@std@@YA?AV?$back_insert_iterator@V?$vector@UProcessPerfData@@V?$allocator@UProcessPerfData@@@std@@@std@@@0@V?$_List_const_iterator@V?$_List_val@U?$_List_simple_types@U?$pair@$$CBKUProcessPerfData@@@std@@@std@@@std@@@0@0V10@V<lambda_1>@?2??RefreshWMIData@PerfThread@@AEAAXXZ@@Z@4HA 00000001800561e8     perfthread.obj
 0002:000101e8       $unwind$?dtor$4@?0???0PerfThread@@QEAA@PEAVPlist@@PEB_W11@Z@4HA 00000001800561e8     perfthread.obj
 0002:000101e8       $unwind$?dtor$5@?0???0PerfThread@@QEAA@PEAVPlist@@PEB_W11@Z@4HA 00000001800561e8     perfthread.obj
 0002:000101e8       $unwind$?dtor$6@?0???0PerfThread@@QEAA@PEAVPlist@@PEB_W11@Z@4HA 00000001800561e8     perfthread.obj
 0002:000101e8       $unwind$?dtor$7@?0???0PerfThread@@QEAA@PEAVPlist@@PEB_W11@Z@4HA 00000001800561e8     perfthread.obj
 0002:000101e8       $unwind$?dtor$8@?0???0PerfThread@@QEAA@PEAVPlist@@PEB_W11@Z@4HA 00000001800561e8     perfthread.obj
 0002:000101e8       $unwind$?dtor$9@?0???0PerfThread@@QEAA@PEAVPlist@@PEB_W11@Z@4HA 00000001800561e8     perfthread.obj
 0002:000101f0       $unwind$?dtor$1@?0??_Getcat@?$numpunct@_W@std@@SA_KPEAPEBVfacet@locale@2@PEBV42@@Z@4HA 00000001800561f0     format.obj
 0002:000101f0       $unwind$?dtor$28@?0??RefreshWMIData@PerfThread@@AEAAXXZ@4HA 00000001800561f0     perfthread.obj
 0002:000101f0       $unwind$?dtor$8@?0??RefreshWMIData@PerfThread@@AEAAXXZ@4HA 00000001800561f0     perfthread.obj
 0002:000101f8       $unwind$?_Init@?$numpunct@_W@std@@IEAAXAEBV_Locinfo@2@_N@Z 00000001800561f8     format.obj
 0002:0001021c       $stateUnwindMap$?_Init@?$numpunct@_W@std@@IEAAXAEBV_Locinfo@2@_N@Z 000000018005621c     format.obj
 0002:00010228       $ip2state$?_Init@?$numpunct@_W@std@@IEAAXAEBV_Locinfo@2@_N@Z 0000000180056228     format.obj
 0002:00010230       $unwind$??$format_decimal@DIVappender@v8@fmt@@$0A@@detail@v8@fmt@@YA?AU?$format_decimal_result@Vappender@v8@fmt@@@012@Vappender@12@IH@Z 0000000180056230     format.obj
 0002:00010244       $unwind$??$format_decimal@D_KVappender@v8@fmt@@$0A@@detail@v8@fmt@@YA?AU?$format_decimal_result@Vappender@v8@fmt@@@012@Vappender@12@_KH@Z 0000000180056244     format.obj
 0002:00010258       $unwind$??$?RH$0A@@?$width_checker@Uerror_handler@detail@v8@fmt@@@detail@v8@fmt@@QEAA_KH@Z 0000000180056258     format.obj
 0002:00010270       $ip2state$??$?RH$0A@@?$width_checker@Uerror_handler@detail@v8@fmt@@@detail@v8@fmt@@QEAA_KH@Z 0000000180056270     format.obj
 0002:00010278       $unwind$??$?RH$0A@@?$precision_checker@Uerror_handler@detail@v8@fmt@@@detail@v8@fmt@@QEAA_KH@Z 0000000180056278     format.obj
 0002:00010290       $ip2state$??$?RH$0A@@?$precision_checker@Uerror_handler@detail@v8@fmt@@@detail@v8@fmt@@QEAA_KH@Z 0000000180056290     format.obj
 0002:00010298       $unwind$??$?R_J$0A@@?$width_checker@Uerror_handler@detail@v8@fmt@@@detail@v8@fmt@@QEAA_K_J@Z 0000000180056298     format.obj
 0002:000102b0       $ip2state$??$?R_J$0A@@?$width_checker@Uerror_handler@detail@v8@fmt@@@detail@v8@fmt@@QEAA_K_J@Z 00000001800562b0     format.obj
 0002:000102b8       $unwind$??$?RM$0A@@?$width_checker@Uerror_handler@detail@v8@fmt@@@detail@v8@fmt@@QEAA_KM@Z 00000001800562b8     format.obj
 0002:000102b8       $unwind$??$?RN$0A@@?$width_checker@Uerror_handler@detail@v8@fmt@@@detail@v8@fmt@@QEAA_KN@Z 00000001800562b8     format.obj
 0002:000102b8       $unwind$??$?RO$0A@@?$width_checker@Uerror_handler@detail@v8@fmt@@@detail@v8@fmt@@QEAA_KO@Z 00000001800562b8     format.obj
 0002:000102b8       $unwind$??$?RPEBX$0A@@?$width_checker@Uerror_handler@detail@v8@fmt@@@detail@v8@fmt@@QEAA_KPEBX@Z 00000001800562b8     format.obj
 0002:000102b8       $unwind$??$?RUmonostate@v8@fmt@@$0A@@?$width_checker@Uerror_handler@detail@v8@fmt@@@detail@v8@fmt@@QEAA_KUmonostate@23@@Z 00000001800562b8     format.obj
 0002:000102b8       $unwind$??$?R_N$0A@@?$width_checker@Uerror_handler@detail@v8@fmt@@@detail@v8@fmt@@QEAA_K_N@Z 00000001800562b8     format.obj
 0002:000102d0       $ip2state$??$?RM$0A@@?$width_checker@Uerror_handler@detail@v8@fmt@@@detail@v8@fmt@@QEAA_KM@Z 00000001800562d0     format.obj
 0002:000102d0       $ip2state$??$?RN$0A@@?$width_checker@Uerror_handler@detail@v8@fmt@@@detail@v8@fmt@@QEAA_KN@Z 00000001800562d0     format.obj
 0002:000102d0       $ip2state$??$?RO$0A@@?$width_checker@Uerror_handler@detail@v8@fmt@@@detail@v8@fmt@@QEAA_KO@Z 00000001800562d0     format.obj
 0002:000102d0       $ip2state$??$?RPEBX$0A@@?$width_checker@Uerror_handler@detail@v8@fmt@@@detail@v8@fmt@@QEAA_KPEBX@Z 00000001800562d0     format.obj
 0002:000102d0       $ip2state$??$?RUmonostate@v8@fmt@@$0A@@?$width_checker@Uerror_handler@detail@v8@fmt@@@detail@v8@fmt@@QEAA_KUmonostate@23@@Z 00000001800562d0     format.obj
 0002:000102d0       $ip2state$??$?R_N$0A@@?$width_checker@Uerror_handler@detail@v8@fmt@@@detail@v8@fmt@@QEAA_K_N@Z 00000001800562d0     format.obj
 0002:000102d8       $unwind$??$?R_J$0A@@?$precision_checker@Uerror_handler@detail@v8@fmt@@@detail@v8@fmt@@QEAA_K_J@Z 00000001800562d8     format.obj
 0002:000102f0       $ip2state$??$?R_J$0A@@?$precision_checker@Uerror_handler@detail@v8@fmt@@@detail@v8@fmt@@QEAA_K_J@Z 00000001800562f0     format.obj
 0002:000102f8       $unwind$??$?RM$0A@@?$precision_checker@Uerror_handler@detail@v8@fmt@@@detail@v8@fmt@@QEAA_KM@Z 00000001800562f8     format.obj
 0002:000102f8       $unwind$??$?RN$0A@@?$precision_checker@Uerror_handler@detail@v8@fmt@@@detail@v8@fmt@@QEAA_KN@Z 00000001800562f8     format.obj
 0002:000102f8       $unwind$??$?RO$0A@@?$precision_checker@Uerror_handler@detail@v8@fmt@@@detail@v8@fmt@@QEAA_KO@Z 00000001800562f8     format.obj
 0002:000102f8       $unwind$??$?RPEBX$0A@@?$precision_checker@Uerror_handler@detail@v8@fmt@@@detail@v8@fmt@@QEAA_KPEBX@Z 00000001800562f8     format.obj
 0002:000102f8       $unwind$??$?RUmonostate@v8@fmt@@$0A@@?$precision_checker@Uerror_handler@detail@v8@fmt@@@detail@v8@fmt@@QEAA_KUmonostate@23@@Z 00000001800562f8     format.obj
 0002:000102f8       $unwind$??$?R_N$0A@@?$precision_checker@Uerror_handler@detail@v8@fmt@@@detail@v8@fmt@@QEAA_K_N@Z 00000001800562f8     format.obj
 0002:00010310       $ip2state$??$?RM$0A@@?$precision_checker@Uerror_handler@detail@v8@fmt@@@detail@v8@fmt@@QEAA_KM@Z 0000000180056310     format.obj
 0002:00010310       $ip2state$??$?RN$0A@@?$precision_checker@Uerror_handler@detail@v8@fmt@@@detail@v8@fmt@@QEAA_KN@Z 0000000180056310     format.obj
 0002:00010310       $ip2state$??$?RO$0A@@?$precision_checker@Uerror_handler@detail@v8@fmt@@@detail@v8@fmt@@QEAA_KO@Z 0000000180056310     format.obj
 0002:00010310       $ip2state$??$?RPEBX$0A@@?$precision_checker@Uerror_handler@detail@v8@fmt@@@detail@v8@fmt@@QEAA_KPEBX@Z 0000000180056310     format.obj
 0002:00010310       $ip2state$??$?RUmonostate@v8@fmt@@$0A@@?$precision_checker@Uerror_handler@detail@v8@fmt@@@detail@v8@fmt@@QEAA_KUmonostate@23@@Z 0000000180056310     format.obj
 0002:00010310       $ip2state$??$?R_N$0A@@?$precision_checker@Uerror_handler@detail@v8@fmt@@@detail@v8@fmt@@QEAA_K_N@Z 0000000180056310     format.obj
 0002:00010318       $unwind$??$decimal_point@_W@detail@v8@fmt@@YA_WVlocale_ref@012@@Z 0000000180056318     handles.obj
 0002:00010328       $stateUnwindMap$??$decimal_point@_W@detail@v8@fmt@@YA_WVlocale_ref@012@@Z 0000000180056328     handles.obj
 0002:00010340       $ip2state$??$decimal_point@_W@detail@v8@fmt@@YA_WVlocale_ref@012@@Z 0000000180056340     handles.obj
 0002:00010360       $unwind$?GetFileName@@YA?AV?$basic_string@_WU?$char_traits@_W@std@@V?$allocator@_W@2@@std@@PEAX@Z 0000000180056360     handles.obj
 0002:00010378       $stateUnwindMap$?GetFileName@@YA?AV?$basic_string@_WU?$char_traits@_W@std@@V?$allocator@_W@2@@std@@PEAX@Z 0000000180056378     handles.obj
 0002:000103a0       $ip2state$?GetFileName@@YA?AV?$basic_string@_WU?$char_traits@_W@std@@V?$allocator@_W@2@@std@@PEAX@Z 00000001800563a0     handles.obj
 0002:000103d8       $unwind$?GetFileNameThread@test@?4??GetFileName@@YA?AV?$basic_string@_WU?$char_traits@_W@std@@V?$allocator@_W@2@@std@@PEAX@Z@SAK0@Z 00000001800563d8     handles.obj
 0002:000103ec       $unwind$??R<lambda_1>@?1??GetUserAccountID@@YA@XZ@QEBA?AV?$basic_string@_WU?$char_traits@_W@std@@V?$allocator@_W@2@@std@@XZ 00000001800563ec     handles.obj
 0002:00010408       $stateUnwindMap$??R<lambda_1>@?1??GetUserAccountID@@YA@XZ@QEBA?AV?$basic_string@_WU?$char_traits@_W@std@@V?$allocator@_W@2@@std@@XZ 0000000180056408     handles.obj
 0002:00010440       $ip2state$??R<lambda_1>@?1??GetUserAccountID@@YA@XZ@QEBA?AV?$basic_string@_WU?$char_traits@_W@std@@V?$allocator@_W@2@@std@@XZ 0000000180056440     handles.obj
 0002:00010480       $unwind$?GetNameByType@@YA?AV?$basic_string@_WU?$char_traits@_W@std@@V?$allocator@_W@2@@std@@PEAXGPEAVPerfThread@@@Z 0000000180056480     handles.obj
 0002:000104a4       $stateUnwindMap$?GetNameByType@@YA?AV?$basic_string@_WU?$char_traits@_W@std@@V?$allocator@_W@2@@std@@PEAXGPEAVPerfThread@@@Z 00000001800564a4     handles.obj
 0002:000104e0       $ip2state$?GetNameByType@@YA?AV?$basic_string@_WU?$char_traits@_W@std@@V?$allocator@_W@2@@std@@PEAXGPEAVPerfThread@@@Z 00000001800564e0     handles.obj
 0002:00010540       $unwind$?dtor$31@?0??GetNameByType@@YA?AV?$basic_string@_WU?$char_traits@_W@std@@V?$allocator@_W@2@@std@@PEAXGPEAVPerfThread@@@Z@4HA 0000000180056540     handles.obj
 0002:00010548       $unwind$?PrintHandleInfo@@YA_NKPEAX_NPEAVPerfThread@@@Z 0000000180056548     handles.obj
 0002:0001056c       $stateUnwindMap$?PrintHandleInfo@@YA_NKPEAX_NPEAVPerfThread@@@Z 000000018005656c     handles.obj
 0002:000105b0       $ip2state$?PrintHandleInfo@@YA_NKPEAX_NPEAVPerfThread@@@Z 00000001800565b0     handles.obj
 0002:00010608       $unwind$??0?$basic_string@_WU?$char_traits@_W@std@@V?$allocator@_W@2@@std@@QEAA@XZ 0000000180056608     handles.obj
 0002:00010618       $unwind$??0?$basic_string@_WU?$char_traits@_W@std@@V?$allocator@_W@2@@std@@QEAA@AEBV01@@Z 0000000180056618     handles.obj
 0002:00010628       $unwind$?check_arg_id@?$basic_format_parse_context@_WUerror_handler@detail@v8@fmt@@@v8@fmt@@QEAAXH@Z 0000000180056628     handles.obj
 0002:00010640       $ip2state$?check_arg_id@?$basic_format_parse_context@_WUerror_handler@detail@v8@fmt@@@v8@fmt@@QEAAXH@Z 0000000180056640     handles.obj
 0002:00010648       $unwind$?next_arg_id@?$basic_format_parse_context@_WUerror_handler@detail@v8@fmt@@@v8@fmt@@QEAAHXZ 0000000180056648     handles.obj
 0002:00010660       $ip2state$?next_arg_id@?$basic_format_parse_context@_WUerror_handler@detail@v8@fmt@@@v8@fmt@@QEAAHXZ 0000000180056660     handles.obj
 0002:00010668       $unwind$?append@?$basic_string@_WU?$char_traits@_W@std@@V?$allocator@_W@2@@std@@QEAAAEAV12@QEB_W_K@Z 0000000180056668     handles.obj
 0002:0001067c       $unwind$??$visit_format_arg@U?$default_arg_formatter@_W@detail@v8@fmt@@V?$basic_format_context@V?$back_insert_iterator@V?$buffer@_W@detail@v8@fmt@@@std@@_W@34@@v8@fmt@@YA?AV?$back_insert_iterator@V?$buffer@_W@detail@v8@fmt@@@std@@$$QEAU?$default_arg_formatter@_W@detail@01@AEBV?$basic_format_arg@V?$basic_format_context@V?$back_insert_iterator@V?$buffer@_W@detail@v8@fmt@@@std@@_W@v8@fmt@@@01@@Z 000000018005667c     handles.obj
 0002:0001069c       $stateUnwindMap$??$visit_format_arg@U?$default_arg_formatter@_W@detail@v8@fmt@@V?$basic_format_context@V?$back_insert_iterator@V?$buffer@_W@detail@v8@fmt@@@std@@_W@34@@v8@fmt@@YA?AV?$back_insert_iterator@V?$buffer@_W@detail@v8@fmt@@@std@@$$QEAU?$default_arg_formatter@_W@detail@01@AEBV?$basic_format_arg@V?$basic_format_context@V?$back_insert_iterator@V?$buffer@_W@detail@v8@fmt@@@std@@_W@v8@fmt@@@01@@Z 000000018005669c     handles.obj
 0002:000106b0       $ip2state$??$visit_format_arg@U?$default_arg_formatter@_W@detail@v8@fmt@@V?$basic_format_context@V?$back_insert_iterator@V?$buffer@_W@detail@v8@fmt@@@std@@_W@34@@v8@fmt@@YA?AV?$back_insert_iterator@V?$buffer@_W@detail@v8@fmt@@@std@@$$QEAU?$default_arg_formatter@_W@detail@01@AEBV?$basic_format_arg@V?$basic_format_context@V?$back_insert_iterator@V?$buffer@_W@detail@v8@fmt@@@std@@_W@v8@fmt@@@01@@Z 00000001800566b0     handles.obj
 0002:000106d0       $unwind$??$get_arg@V?$basic_format_context@V?$back_insert_iterator@V?$buffer@_W@detail@v8@fmt@@@std@@_W@v8@fmt@@H@detail@v8@fmt@@YA?AV?$basic_format_arg@V?$basic_format_context@V?$back_insert_iterator@V?$buffer@_W@detail@v8@fmt@@@std@@_W@v8@fmt@@@12@AEAV?$basic_format_context@V?$back_insert_iterator@V?$buffer@_W@detail@v8@fmt@@@std@@_W@12@H@Z 00000001800566d0     handles.obj
 0002:000106f0       $ip2state$??$get_arg@V?$basic_format_context@V?$back_insert_iterator@V?$buffer@_W@detail@v8@fmt@@@std@@_W@v8@fmt@@H@detail@v8@fmt@@YA?AV?$basic_format_arg@V?$basic_format_context@V?$back_insert_iterator@V?$buffer@_W@detail@v8@fmt@@@std@@_W@v8@fmt@@@12@AEAV?$basic_format_context@V?$back_insert_iterator@V?$buffer@_W@detail@v8@fmt@@@std@@_W@12@H@Z 00000001800566f0     handles.obj
 0002:000106f8       $unwind$??$visit_format_arg@AEAU?$arg_formatter@_W@detail@v8@fmt@@V?$basic_format_context@V?$back_insert_iterator@V?$buffer@_W@detail@v8@fmt@@@std@@_W@34@@v8@fmt@@YA?AV?$back_insert_iterator@V?$buffer@_W@detail@v8@fmt@@@std@@AEAU?$arg_formatter@_W@detail@01@AEBV?$basic_format_arg@V?$basic_format_context@V?$back_insert_iterator@V?$buffer@_W@detail@v8@fmt@@@std@@_W@v8@fmt@@@01@@Z 00000001800566f8     handles.obj
 0002:00010718       $stateUnwindMap$??$visit_format_arg@AEAU?$arg_formatter@_W@detail@v8@fmt@@V?$basic_format_context@V?$back_insert_iterator@V?$buffer@_W@detail@v8@fmt@@@std@@_W@34@@v8@fmt@@YA?AV?$back_insert_iterator@V?$buffer@_W@detail@v8@fmt@@@std@@AEAU?$arg_formatter@_W@detail@01@AEBV?$basic_format_arg@V?$basic_format_context@V?$back_insert_iterator@V?$buffer@_W@detail@v8@fmt@@@std@@_W@v8@fmt@@@01@@Z 0000000180056718     handles.obj
 0002:00010720       $ip2state$??$visit_format_arg@AEAU?$arg_formatter@_W@detail@v8@fmt@@V?$basic_format_context@V?$back_insert_iterator@V?$buffer@_W@detail@v8@fmt@@@std@@_W@34@@v8@fmt@@YA?AV?$back_insert_iterator@V?$buffer@_W@detail@v8@fmt@@@std@@AEAU?$arg_formatter@_W@detail@01@AEBV?$basic_format_arg@V?$basic_format_context@V?$back_insert_iterator@V?$buffer@_W@detail@v8@fmt@@@std@@_W@v8@fmt@@@01@@Z 0000000180056720     handles.obj
 0002:00010760       $unwind$??$parse_format_string@$0A@_WUformat_handler@?1???$vformat_to@_W@detail@v8@fmt@@YAXAEAV?$buffer@_W@234@V?$basic_string_view@_W@34@V?$basic_format_args@V?$basic_format_context@V?$back_insert_iterator@V?$buffer@_W@detail@v8@fmt@@@std@@_W@v8@fmt@@@34@Vlocale_ref@234@@Z@@detail@v8@fmt@@YAXV?$basic_string_view@_W@12@$$QEAUformat_handler@?1???$vformat_to@_W@012@YAXAEAV?$buffer@_W@012@0V?$basic_format_args@V?$basic_format_context@V?$back_insert_iterator@V?$buffer@_W@detail@v8@fmt@@@std@@_W@v8@fmt@@@12@Vlocale_ref@012@@Z@@Z 0000000180056760     handles.obj
 0002:0001077c       $stateUnwindMap$??$parse_format_string@$0A@_WUformat_handler@?1???$vformat_to@_W@detail@v8@fmt@@YAXAEAV?$buffer@_W@234@V?$basic_string_view@_W@34@V?$basic_format_args@V?$basic_format_context@V?$back_insert_iterator@V?$buffer@_W@detail@v8@fmt@@@std@@_W@v8@fmt@@@34@Vlocale_ref@234@@Z@@detail@v8@fmt@@YAXV?$basic_string_view@_W@12@$$QEAUformat_handler@?1???$vformat_to@_W@012@YAXAEAV?$buffer@_W@012@0V?$basic_format_args@V?$basic_format_context@V?$back_insert_iterator@V?$buffer@_W@detail@v8@fmt@@@std@@_W@v8@fmt@@@12@Vlocale_ref@012@@Z@@Z 000000018005677c     handles.obj
 0002:00010790       $ip2state$??$parse_format_string@$0A@_WUformat_handler@?1???$vformat_to@_W@detail@v8@fmt@@YAXAEAV?$buffer@_W@234@V?$basic_string_view@_W@34@V?$basic_format_args@V?$basic_format_context@V?$back_insert_iterator@V?$buffer@_W@detail@v8@fmt@@@std@@_W@v8@fmt@@@34@Vlocale_ref@234@@Z@@detail@v8@fmt@@YAXV?$basic_string_view@_W@12@$$QEAUformat_handler@?1???$vformat_to@_W@012@YAXAEAV?$buffer@_W@012@0V?$basic_format_args@V?$basic_format_context@V?$back_insert_iterator@V?$buffer@_W@detail@v8@fmt@@@std@@_W@v8@fmt@@@12@Vlocale_ref@012@@Z@@Z 0000000180056790     handles.obj
 0002:000107b0       $unwind$??Rwriter@?1???$parse_format_string@$0A@_WUformat_handler@?1???$vformat_to@_W@detail@v8@fmt@@YAXAEAV?$buffer@_W@234@V?$basic_string_view@_W@34@V?$basic_format_args@V?$basic_format_context@V?$back_insert_iterator@V?$buffer@_W@detail@v8@fmt@@@std@@_W@v8@fmt@@@34@Vlocale_ref@234@@Z@@detail@v8@fmt@@YAXV?$basic_string_view@_W@23@$$QEAUformat_handler@?1???$vformat_to@_W@123@YAXAEAV?$buffer@_W@123@0V?$basic_format_args@V?$basic_format_context@V?$back_insert_iterator@V?$buffer@_W@detail@v8@fmt@@@std@@_W@v8@fmt@@@23@Vlocale_ref@123@@Z@@Z@QEAAXPEB_W5@Z 00000001800567b0     handles.obj
 0002:000107d0       $ip2state$??Rwriter@?1???$parse_format_string@$0A@_WUformat_handler@?1???$vformat_to@_W@detail@v8@fmt@@YAXAEAV?$buffer@_W@234@V?$basic_string_view@_W@34@V?$basic_format_args@V?$basic_format_context@V?$back_insert_iterator@V?$buffer@_W@detail@v8@fmt@@@std@@_W@v8@fmt@@@34@Vlocale_ref@234@@Z@@detail@v8@fmt@@YAXV?$basic_string_view@_W@23@$$QEAUformat_handler@?1???$vformat_to@_W@123@YAXAEAV?$buffer@_W@123@0V?$basic_format_args@V?$basic_format_context@V?$back_insert_iterator@V?$buffer@_W@detail@v8@fmt@@@std@@_W@v8@fmt@@@23@Vlocale_ref@123@@Z@@Z@QEAAXPEB_W5@Z 00000001800567d0     handles.obj
 0002:000107e0       $unwind$??$vformat@_W$0A@@v8@fmt@@YA?AV?$basic_string@_WU?$char_traits@_W@std@@V?$allocator@_W@2@@std@@V?$basic_string_view@_W@01@V?$basic_format_args@V?$basic_format_context@V?$back_insert_iterator@V?$buffer@_W@detail@v8@fmt@@@std@@_W@v8@fmt@@@01@@Z 00000001800567e0     handles.obj
 0002:00010800       $stateUnwindMap$??$vformat@_W$0A@@v8@fmt@@YA?AV?$basic_string@_WU?$char_traits@_W@std@@V?$allocator@_W@2@@std@@V?$basic_string_view@_W@01@V?$basic_format_args@V?$basic_format_context@V?$back_insert_iterator@V?$buffer@_W@detail@v8@fmt@@@std@@_W@v8@fmt@@@01@@Z 0000000180056800     handles.obj
 0002:00010820       $ip2state$??$vformat@_W$0A@@v8@fmt@@YA?AV?$basic_string@_WU?$char_traits@_W@std@@V?$allocator@_W@2@@std@@V?$basic_string_view@_W@01@V?$basic_format_args@V?$basic_format_context@V?$back_insert_iterator@V?$buffer@_W@detail@v8@fmt@@@std@@_W@v8@fmt@@@01@@Z 0000000180056820     handles.obj
 0002:00010840       $unwind$?require_numeric_argument@?$specs_checker@V?$specs_handler@_W@detail@v8@fmt@@@detail@v8@fmt@@AEAAXXZ 0000000180056840     handles.obj
 0002:00010858       $ip2state$?require_numeric_argument@?$specs_checker@V?$specs_handler@_W@detail@v8@fmt@@@detail@v8@fmt@@AEAAXXZ 0000000180056858     handles.obj
 0002:00010860       $unwind$??$?RM@?$default_arg_formatter@_W@detail@v8@fmt@@QEAA?AV?$back_insert_iterator@V?$buffer@_W@detail@v8@fmt@@@std@@M@Z 0000000180056860     handles.obj
 0002:00010860       $unwind$??$?RN@?$default_arg_formatter@_W@detail@v8@fmt@@QEAA?AV?$back_insert_iterator@V?$buffer@_W@detail@v8@fmt@@@std@@N@Z 0000000180056860     handles.obj
 0002:00010860       $unwind$??$?RO@?$default_arg_formatter@_W@detail@v8@fmt@@QEAA?AV?$back_insert_iterator@V?$buffer@_W@detail@v8@fmt@@@std@@O@Z 0000000180056860     handles.obj
 0002:00010878       $unwind$??$parse_align@_WAEAV?$specs_checker@V?$specs_handler@_W@detail@v8@fmt@@@detail@v8@fmt@@@detail@v8@fmt@@YAPEB_WPEB_W0AEAV?$specs_checker@V?$specs_handler@_W@detail@v8@fmt@@@012@@Z 0000000180056878     handles.obj
 0002:00010890       $stateUnwindMap$??$parse_align@_WAEAV?$specs_checker@V?$specs_handler@_W@detail@v8@fmt@@@detail@v8@fmt@@@detail@v8@fmt@@YAPEB_WPEB_W0AEAV?$specs_checker@V?$specs_handler@_W@detail@v8@fmt@@@012@@Z 0000000180056890     handles.obj
 0002:000108b0       $ip2state$??$parse_align@_WAEAV?$specs_checker@V?$specs_handler@_W@detail@v8@fmt@@@detail@v8@fmt@@@detail@v8@fmt@@YAPEB_WPEB_W0AEAV?$specs_checker@V?$specs_handler@_W@detail@v8@fmt@@@012@@Z 00000001800568b0     handles.obj
 0002:000108c0       $unwind$??$parse_width@_WAEAV?$specs_checker@V?$specs_handler@_W@detail@v8@fmt@@@detail@v8@fmt@@@detail@v8@fmt@@YAPEB_WPEB_W0AEAV?$specs_checker@V?$specs_handler@_W@detail@v8@fmt@@@012@@Z 00000001800568c0     handles.obj
 0002:000108d8       $stateUnwindMap$??$parse_width@_WAEAV?$specs_checker@V?$specs_handler@_W@detail@v8@fmt@@@detail@v8@fmt@@@detail@v8@fmt@@YAPEB_WPEB_W0AEAV?$specs_checker@V?$specs_handler@_W@detail@v8@fmt@@@012@@Z 00000001800568d8     handles.obj
 0002:000108f0       $ip2state$??$parse_width@_WAEAV?$specs_checker@V?$specs_handler@_W@detail@v8@fmt@@@detail@v8@fmt@@@detail@v8@fmt@@YAPEB_WPEB_W0AEAV?$specs_checker@V?$specs_handler@_W@detail@v8@fmt@@@012@@Z 00000001800568f0     handles.obj
 0002:00010910       $unwind$?on_error@id_adapter@?1???$parse_replacement_field@_WAEAUformat_handler@?1???$vformat_to@_W@detail@v8@fmt@@YAXAEAV?$buffer@_W@234@V?$basic_string_view@_W@34@V?$basic_format_args@V?$basic_format_context@V?$back_insert_iterator@V?$buffer@_W@detail@v8@fmt@@@std@@_W@v8@fmt@@@34@Vlocale_ref@234@@Z@@detail@v8@fmt@@YAPEB_WPEB_W0AEAUformat_handler@?1???$vformat_to@_W@234@YAXAEAV?$buffer@_W@234@V?$basic_string_view@_W@34@V?$basic_format_args@V?$basic_format_context@V?$back_insert_iterator@V?$buffer@_W@detail@v8@fmt@@@std@@_W@v8@fmt@@@34@Vlocale_ref@234@@Z@@Z@QEAAXPEBD@Z 0000000180056910     handles.obj
 0002:00010910       $unwind$?on_error@precision_adapter@?1???$parse_precision@_WAEAV?$specs_checker@V?$specs_handler@_W@detail@v8@fmt@@@detail@v8@fmt@@@detail@v8@fmt@@YAPEB_WPEB_W0AEAV?$specs_checker@V?$specs_handler@_W@detail@v8@fmt@@@234@@Z@QEAAXPEBD@Z 0000000180056910     handles.obj
 0002:00010910       $unwind$?on_error@width_adapter@?1???$parse_width@_WAEAV?$specs_checker@V?$specs_handler@_W@detail@v8@fmt@@@detail@v8@fmt@@@detail@v8@fmt@@YAPEB_WPEB_W0AEAV?$specs_checker@V?$specs_handler@_W@detail@v8@fmt@@@234@@Z@QEAAXPEBD@Z 0000000180056910     handles.obj
 0002:00010928       $ip2state$?on_error@id_adapter@?1???$parse_replacement_field@_WAEAUformat_handler@?1???$vformat_to@_W@detail@v8@fmt@@YAXAEAV?$buffer@_W@234@V?$basic_string_view@_W@34@V?$basic_format_args@V?$basic_format_context@V?$back_insert_iterator@V?$buffer@_W@detail@v8@fmt@@@std@@_W@v8@fmt@@@34@Vlocale_ref@234@@Z@@detail@v8@fmt@@YAPEB_WPEB_W0AEAUformat_handler@?1???$vformat_to@_W@234@YAXAEAV?$buffer@_W@234@V?$basic_string_view@_W@34@V?$basic_format_args@V?$basic_format_context@V?$back_insert_iterator@V?$buffer@_W@detail@v8@fmt@@@std@@_W@v8@fmt@@@34@Vlocale_ref@234@@Z@@Z@QEAAXPEBD@Z 0000000180056928     handles.obj
 0002:00010928       $ip2state$?on_error@precision_adapter@?1???$parse_precision@_WAEAV?$specs_checker@V?$specs_handler@_W@detail@v8@fmt@@@detail@v8@fmt@@@detail@v8@fmt@@YAPEB_WPEB_W0AEAV?$specs_checker@V?$specs_handler@_W@detail@v8@fmt@@@234@@Z@QEAAXPEBD@Z 0000000180056928     handles.obj
 0002:00010928       $ip2state$?on_error@width_adapter@?1???$parse_width@_WAEAV?$specs_checker@V?$specs_handler@_W@detail@v8@fmt@@@detail@v8@fmt@@@detail@v8@fmt@@YAPEB_WPEB_W0AEAV?$specs_checker@V?$specs_handler@_W@detail@v8@fmt@@@234@@Z@QEAAXPEBD@Z 0000000180056928     handles.obj
 0002:00010930       $unwind$??$parse_precision@_WAEAV?$specs_checker@V?$specs_handler@_W@detail@v8@fmt@@@detail@v8@fmt@@@detail@v8@fmt@@YAPEB_WPEB_W0AEAV?$specs_checker@V?$specs_handler@_W@detail@v8@fmt@@@012@@Z 0000000180056930     handles.obj
 0002:00010950       $stateUnwindMap$??$parse_precision@_WAEAV?$specs_checker@V?$specs_handler@_W@detail@v8@fmt@@@detail@v8@fmt@@@detail@v8@fmt@@YAPEB_WPEB_W0AEAV?$specs_checker@V?$specs_handler@_W@detail@v8@fmt@@@012@@Z 0000000180056950     handles.obj
 0002:00010980       $ip2state$??$parse_precision@_WAEAV?$specs_checker@V?$specs_handler@_W@detail@v8@fmt@@@detail@v8@fmt@@@detail@v8@fmt@@YAPEB_WPEB_W0AEAV?$specs_checker@V?$specs_handler@_W@detail@v8@fmt@@@012@@Z 0000000180056980     handles.obj
 0002:000109b8       $unwind$??$parse_replacement_field@_WAEAUformat_handler@?1???$vformat_to@_W@detail@v8@fmt@@YAXAEAV?$buffer@_W@234@V?$basic_string_view@_W@34@V?$basic_format_args@V?$basic_format_context@V?$back_insert_iterator@V?$buffer@_W@detail@v8@fmt@@@std@@_W@v8@fmt@@@34@Vlocale_ref@234@@Z@@detail@v8@fmt@@YAPEB_WPEB_W0AEAUformat_handler@?1???$vformat_to@_W@012@YAXAEAV?$buffer@_W@012@V?$basic_string_view@_W@12@V?$basic_format_args@V?$basic_format_context@V?$back_insert_iterator@V?$buffer@_W@detail@v8@fmt@@@std@@_W@v8@fmt@@@12@Vlocale_ref@012@@Z@@Z 00000001800569b8     handles.obj
 0002:000109d8       $stateUnwindMap$??$parse_replacement_field@_WAEAUformat_handler@?1???$vformat_to@_W@detail@v8@fmt@@YAXAEAV?$buffer@_W@234@V?$basic_string_view@_W@34@V?$basic_format_args@V?$basic_format_context@V?$back_insert_iterator@V?$buffer@_W@detail@v8@fmt@@@std@@_W@v8@fmt@@@34@Vlocale_ref@234@@Z@@detail@v8@fmt@@YAPEB_WPEB_W0AEAUformat_handler@?1???$vformat_to@_W@012@YAXAEAV?$buffer@_W@012@V?$basic_string_view@_W@12@V?$basic_format_args@V?$basic_format_context@V?$back_insert_iterator@V?$buffer@_W@detail@v8@fmt@@@std@@_W@v8@fmt@@@12@Vlocale_ref@012@@Z@@Z 00000001800569d8     handles.obj
 0002:000109f0       $ip2state$??$parse_replacement_field@_WAEAUformat_handler@?1???$vformat_to@_W@detail@v8@fmt@@YAXAEAV?$buffer@_W@234@V?$basic_string_view@_W@34@V?$basic_format_args@V?$basic_format_context@V?$back_insert_iterator@V?$buffer@_W@detail@v8@fmt@@@std@@_W@v8@fmt@@@34@Vlocale_ref@234@@Z@@detail@v8@fmt@@YAPEB_WPEB_W0AEAUformat_handler@?1???$vformat_to@_W@012@YAXAEAV?$buffer@_W@012@V?$basic_string_view@_W@12@V?$basic_format_args@V?$basic_format_context@V?$back_insert_iterator@V?$buffer@_W@detail@v8@fmt@@@std@@_W@v8@fmt@@@12@Vlocale_ref@012@@Z@@Z 00000001800569f0     handles.obj
 0002:00010a18       $unwind$??$write@_WV?$back_insert_iterator@V?$buffer@_W@detail@v8@fmt@@@std@@@detail@v8@fmt@@YA?AV?$back_insert_iterator@V?$buffer@_W@detail@v8@fmt@@@std@@V34@V?$basic_string_view@_W@12@AEBU?$basic_format_specs@_W@12@Vlocale_ref@012@@Z 0000000180056a18     handles.obj
 0002:00010a34       $stateUnwindMap$??$parse_float_type_spec@Uerror_handler@detail@v8@fmt@@_W@detail@v8@fmt@@YA?AUfloat_specs@012@AEBU?$basic_format_specs@_W@12@$$QEAUerror_handler@012@@Z 0000000180056a34     handles.obj
 0002:00010a34       $stateUnwindMap$??$write@_WV?$back_insert_iterator@V?$buffer@_W@detail@v8@fmt@@@std@@@detail@v8@fmt@@YA?AV?$back_insert_iterator@V?$buffer@_W@detail@v8@fmt@@@std@@V34@V?$basic_string_view@_W@12@AEBU?$basic_format_specs@_W@12@Vlocale_ref@012@@Z 0000000180056a34     handles.obj
 0002:00010a34       $stateUnwindMap$??$write_int@_WV?$back_insert_iterator@V?$buffer@_W@detail@v8@fmt@@@std@@_K@detail@v8@fmt@@YA?AV?$back_insert_iterator@V?$buffer@_W@detail@v8@fmt@@@std@@V34@U?$write_int_arg@_K@012@AEBU?$basic_format_specs@_W@12@Vlocale_ref@012@@Z 0000000180056a34     handles.obj
 0002:00010a40       $ip2state$??$write@_WV?$back_insert_iterator@V?$buffer@_W@detail@v8@fmt@@@std@@@detail@v8@fmt@@YA?AV?$back_insert_iterator@V?$buffer@_W@detail@v8@fmt@@@std@@V34@V?$basic_string_view@_W@12@AEBU?$basic_format_specs@_W@12@Vlocale_ref@012@@Z 0000000180056a40     handles.obj
 0002:00010a50       $unwind$??$write@_WV?$back_insert_iterator@V?$buffer@_W@detail@v8@fmt@@@std@@_N$0A@@detail@v8@fmt@@YA?AV?$back_insert_iterator@V?$buffer@_W@detail@v8@fmt@@@std@@V34@_NAEBU?$basic_format_specs@_W@12@Vlocale_ref@012@@Z 0000000180056a50     handles.obj
 0002:00010a64       $unwind$??$write@_WV?$back_insert_iterator@V?$buffer@_W@detail@v8@fmt@@@std@@X$0A@@detail@v8@fmt@@YA?AV?$back_insert_iterator@V?$buffer@_W@detail@v8@fmt@@@std@@V34@PEBXAEBU?$basic_format_specs@_W@12@Vlocale_ref@012@@Z 0000000180056a64     handles.obj
 0002:00010a80       $ip2state$??$write@_WV?$back_insert_iterator@V?$buffer@_W@detail@v8@fmt@@@std@@X$0A@@detail@v8@fmt@@YA?AV?$back_insert_iterator@V?$buffer@_W@detail@v8@fmt@@@std@@V34@PEBXAEBU?$basic_format_specs@_W@12@Vlocale_ref@012@@Z 0000000180056a80     handles.obj
 0002:00010a90       $unwind$??$write@_WV?$back_insert_iterator@V?$buffer@_W@detail@v8@fmt@@@std@@@detail@v8@fmt@@YA?AV?$back_insert_iterator@V?$buffer@_W@detail@v8@fmt@@@std@@V34@_WAEBU?$basic_format_specs@_W@12@Vlocale_ref@012@@Z 0000000180056a90     handles.obj
 0002:00010ab0       $stateUnwindMap$??$write@_WV?$back_insert_iterator@V?$buffer@_W@detail@v8@fmt@@@std@@@detail@v8@fmt@@YA?AV?$back_insert_iterator@V?$buffer@_W@detail@v8@fmt@@@std@@V34@_WAEBU?$basic_format_specs@_W@12@Vlocale_ref@012@@Z 0000000180056ab0     handles.obj
 0002:00010ac0       $ip2state$??$write@_WV?$back_insert_iterator@V?$buffer@_W@detail@v8@fmt@@@std@@@detail@v8@fmt@@YA?AV?$back_insert_iterator@V?$buffer@_W@detail@v8@fmt@@@std@@V34@_WAEBU?$basic_format_specs@_W@12@Vlocale_ref@012@@Z 0000000180056ac0     handles.obj
 0002:00010ad8       $unwind$??$write@_WV?$back_insert_iterator@V?$buffer@_W@detail@v8@fmt@@@std@@M$0A@@detail@v8@fmt@@YA?AV?$back_insert_iterator@V?$buffer@_W@detail@v8@fmt@@@std@@V34@MU?$basic_format_specs@_W@12@Vlocale_ref@012@@Z 0000000180056ad8     handles.obj
 0002:00010af8       $stateUnwindMap$??$write@_WV?$back_insert_iterator@V?$buffer@_W@detail@v8@fmt@@@std@@M$0A@@detail@v8@fmt@@YA?AV?$back_insert_iterator@V?$buffer@_W@detail@v8@fmt@@@std@@V34@MU?$basic_format_specs@_W@12@Vlocale_ref@012@@Z 0000000180056af8     handles.obj
 0002:00010af8       $stateUnwindMap$??$write@_WV?$back_insert_iterator@V?$buffer@_W@detail@v8@fmt@@@std@@N$0A@@detail@v8@fmt@@YA?AV?$back_insert_iterator@V?$buffer@_W@detail@v8@fmt@@@std@@V34@NU?$basic_format_specs@_W@12@Vlocale_ref@012@@Z 0000000180056af8     handles.obj
 0002:00010af8       $stateUnwindMap$??$write@_WV?$back_insert_iterator@V?$buffer@_W@detail@v8@fmt@@@std@@O$0A@@detail@v8@fmt@@YA?AV?$back_insert_iterator@V?$buffer@_W@detail@v8@fmt@@@std@@V34@OU?$basic_format_specs@_W@12@Vlocale_ref@012@@Z 0000000180056af8     handles.obj
 0002:00010b00       $ip2state$??$write@_WV?$back_insert_iterator@V?$buffer@_W@detail@v8@fmt@@@std@@M$0A@@detail@v8@fmt@@YA?AV?$back_insert_iterator@V?$buffer@_W@detail@v8@fmt@@@std@@V34@MU?$basic_format_specs@_W@12@Vlocale_ref@012@@Z 0000000180056b00     handles.obj
 0002:00010b18       $unwind$??$write@_WV?$back_insert_iterator@V?$buffer@_W@detail@v8@fmt@@@std@@N$0A@@detail@v8@fmt@@YA?AV?$back_insert_iterator@V?$buffer@_W@detail@v8@fmt@@@std@@V34@NU?$basic_format_specs@_W@12@Vlocale_ref@012@@Z 0000000180056b18     handles.obj
 0002:00010b40       $ip2state$??$write@_WV?$back_insert_iterator@V?$buffer@_W@detail@v8@fmt@@@std@@N$0A@@detail@v8@fmt@@YA?AV?$back_insert_iterator@V?$buffer@_W@detail@v8@fmt@@@std@@V34@NU?$basic_format_specs@_W@12@Vlocale_ref@012@@Z 0000000180056b40     handles.obj
 0002:00010b58       $unwind$??$write@_WV?$back_insert_iterator@V?$buffer@_W@detail@v8@fmt@@@std@@O$0A@@detail@v8@fmt@@YA?AV?$back_insert_iterator@V?$buffer@_W@detail@v8@fmt@@@std@@V34@OU?$basic_format_specs@_W@12@Vlocale_ref@012@@Z 0000000180056b58     handles.obj
 0002:00010b80       $ip2state$??$write@_WV?$back_insert_iterator@V?$buffer@_W@detail@v8@fmt@@@std@@O$0A@@detail@v8@fmt@@YA?AV?$back_insert_iterator@V?$buffer@_W@detail@v8@fmt@@@std@@V34@OU?$basic_format_specs@_W@12@Vlocale_ref@012@@Z 0000000180056b80     handles.obj
 0002:00010b98       $unwind$?get_arg@?$specs_handler@_W@detail@v8@fmt@@AEAA?AV?$basic_format_arg@V?$basic_format_context@V?$back_insert_iterator@V?$buffer@_W@detail@v8@fmt@@@std@@_W@v8@fmt@@@34@V?$basic_string_view@_W@34@@Z 0000000180056b98     handles.obj
 0002:00010bb0       $stateUnwindMap$?get_arg@?$specs_handler@_W@detail@v8@fmt@@AEAA?AV?$basic_format_arg@V?$basic_format_context@V?$back_insert_iterator@V?$buffer@_W@detail@v8@fmt@@@std@@_W@v8@fmt@@@34@V?$basic_string_view@_W@34@@Z 0000000180056bb0     handles.obj
 0002:00010bb8       $ip2state$?get_arg@?$specs_handler@_W@detail@v8@fmt@@AEAA?AV?$basic_format_arg@V?$basic_format_context@V?$back_insert_iterator@V?$buffer@_W@detail@v8@fmt@@@std@@_W@v8@fmt@@@34@V?$basic_string_view@_W@34@@Z 0000000180056bb8     handles.obj
 0002:00010bc0       $unwind$??$format_decimal@_WIV?$back_insert_iterator@V?$buffer@_W@detail@v8@fmt@@@std@@$0A@@detail@v8@fmt@@YA?AU?$format_decimal_result@V?$back_insert_iterator@V?$buffer@_W@detail@v8@fmt@@@std@@@012@V?$back_insert_iterator@V?$buffer@_W@detail@v8@fmt@@@std@@IH@Z 0000000180056bc0     handles.obj
 0002:00010bd4       $unwind$??$format_decimal@_W_KV?$back_insert_iterator@V?$buffer@_W@detail@v8@fmt@@@std@@$0A@@detail@v8@fmt@@YA?AU?$format_decimal_result@V?$back_insert_iterator@V?$buffer@_W@detail@v8@fmt@@@std@@@012@V?$back_insert_iterator@V?$buffer@_W@detail@v8@fmt@@@std@@_KH@Z 0000000180056bd4     handles.obj
 0002:00010be8       $unwind$??$write_ptr@_WV?$back_insert_iterator@V?$buffer@_W@detail@v8@fmt@@@std@@_K@detail@v8@fmt@@YA?AV?$back_insert_iterator@V?$buffer@_W@detail@v8@fmt@@@std@@V34@_KPEBU?$basic_format_specs@_W@12@@Z 0000000180056be8     handles.obj
 0002:00010c00       $unwind$??$do_parse_arg_id@_WAEAUwidth_adapter@?1???$parse_width@_WAEAV?$specs_checker@V?$specs_handler@_W@detail@v8@fmt@@@detail@v8@fmt@@@detail@v8@fmt@@YAPEB_WPEB_W0AEAV?$specs_checker@V?$specs_handler@_W@detail@v8@fmt@@@234@@Z@@detail@v8@fmt@@YAPEB_WPEB_W0AEAUwidth_adapter@?1???$parse_width@_WAEAV?$specs_checker@V?$specs_handler@_W@detail@v8@fmt@@@detail@v8@fmt@@@012@YAPEB_W00AEAV?$specs_checker@V?$specs_handler@_W@detail@v8@fmt@@@012@@Z@@Z 0000000180056c00     handles.obj
 0002:00010c24       $stateUnwindMap$??$do_parse_arg_id@_WAEAUprecision_adapter@?1???$parse_precision@_WAEAV?$specs_checker@V?$specs_handler@_W@detail@v8@fmt@@@detail@v8@fmt@@@detail@v8@fmt@@YAPEB_WPEB_W0AEAV?$specs_checker@V?$specs_handler@_W@detail@v8@fmt@@@234@@Z@@detail@v8@fmt@@YAPEB_WPEB_W0AEAUprecision_adapter@?1???$parse_precision@_WAEAV?$specs_checker@V?$specs_handler@_W@detail@v8@fmt@@@detail@v8@fmt@@@012@YAPEB_W00AEAV?$specs_checker@V?$specs_handler@_W@detail@v8@fmt@@@012@@Z@@Z 0000000180056c24     handles.obj
 0002:00010c24       $stateUnwindMap$??$do_parse_arg_id@_WAEAUwidth_adapter@?1???$parse_width@_WAEAV?$specs_checker@V?$specs_handler@_W@detail@v8@fmt@@@detail@v8@fmt@@@detail@v8@fmt@@YAPEB_WPEB_W0AEAV?$specs_checker@V?$specs_handler@_W@detail@v8@fmt@@@234@@Z@@detail@v8@fmt@@YAPEB_WPEB_W0AEAUwidth_adapter@?1???$parse_width@_WAEAV?$specs_checker@V?$specs_handler@_W@detail@v8@fmt@@@detail@v8@fmt@@@012@YAPEB_W00AEAV?$specs_checker@V?$specs_handler@_W@detail@v8@fmt@@@012@@Z@@Z 0000000180056c24     handles.obj
 0002:00010c40       $ip2state$??$do_parse_arg_id@_WAEAUwidth_adapter@?1???$parse_width@_WAEAV?$specs_checker@V?$specs_handler@_W@detail@v8@fmt@@@detail@v8@fmt@@@detail@v8@fmt@@YAPEB_WPEB_W0AEAV?$specs_checker@V?$specs_handler@_W@detail@v8@fmt@@@234@@Z@@detail@v8@fmt@@YAPEB_WPEB_W0AEAUwidth_adapter@?1???$parse_width@_WAEAV?$specs_checker@V?$specs_handler@_W@detail@v8@fmt@@@detail@v8@fmt@@@012@YAPEB_W00AEAV?$specs_checker@V?$specs_handler@_W@detail@v8@fmt@@@012@@Z@@Z 0000000180056c40     handles.obj
 0002:00010c78       $unwind$??$do_parse_arg_id@_WAEAUprecision_adapter@?1???$parse_precision@_WAEAV?$specs_checker@V?$specs_handler@_W@detail@v8@fmt@@@detail@v8@fmt@@@detail@v8@fmt@@YAPEB_WPEB_W0AEAV?$specs_checker@V?$specs_handler@_W@detail@v8@fmt@@@234@@Z@@detail@v8@fmt@@YAPEB_WPEB_W0AEAUprecision_adapter@?1???$parse_precision@_WAEAV?$specs_checker@V?$specs_handler@_W@detail@v8@fmt@@@detail@v8@fmt@@@012@YAPEB_W00AEAV?$specs_checker@V?$specs_handler@_W@detail@v8@fmt@@@012@@Z@@Z 0000000180056c78     handles.obj
 0002:00010ca0       $ip2state$??$do_parse_arg_id@_WAEAUprecision_adapter@?1???$parse_precision@_WAEAV?$specs_checker@V?$specs_handler@_W@detail@v8@fmt@@@detail@v8@fmt@@@detail@v8@fmt@@YAPEB_WPEB_W0AEAV?$specs_checker@V?$specs_handler@_W@detail@v8@fmt@@@234@@Z@@detail@v8@fmt@@YAPEB_WPEB_W0AEAUprecision_adapter@?1???$parse_precision@_WAEAV?$specs_checker@V?$specs_handler@_W@detail@v8@fmt@@@detail@v8@fmt@@@012@YAPEB_W00AEAV?$specs_checker@V?$specs_handler@_W@detail@v8@fmt@@@012@@Z@@Z 0000000180056ca0     handles.obj
 0002:00010cd8       $unwind$??$parse_float_type_spec@Uerror_handler@detail@v8@fmt@@_W@detail@v8@fmt@@YA?AUfloat_specs@012@AEBU?$basic_format_specs@_W@12@$$QEAUerror_handler@012@@Z 0000000180056cd8     handles.obj
 0002:00010d00       $ip2state$??$parse_float_type_spec@Uerror_handler@detail@v8@fmt@@_W@detail@v8@fmt@@YA?AUfloat_specs@012@AEBU?$basic_format_specs@_W@12@$$QEAUerror_handler@012@@Z 0000000180056d00     handles.obj
 0002:00010d08       $unwind$??$do_parse_arg_id@_WAEAUid_adapter@?1???$parse_replacement_field@_WAEAUformat_handler@?1???$vformat_to@_W@detail@v8@fmt@@YAXAEAV?$buffer@_W@234@V?$basic_string_view@_W@34@V?$basic_format_args@V?$basic_format_context@V?$back_insert_iterator@V?$buffer@_W@detail@v8@fmt@@@std@@_W@v8@fmt@@@34@Vlocale_ref@234@@Z@@detail@v8@fmt@@YAPEB_WPEB_W0AEAUformat_handler@?1???$vformat_to@_W@234@YAXAEAV?$buffer@_W@234@V?$basic_string_view@_W@34@V?$basic_format_args@V?$basic_format_context@V?$back_insert_iterator@V?$buffer@_W@detail@v8@fmt@@@std@@_W@v8@fmt@@@34@Vlocale_ref@234@@Z@@Z@@detail@v8@fmt@@YAPEB_WPEB_W0AEAUid_adapter@?1???$parse_replacement_field@_WAEAUformat_handler@?1???$vformat_to@_W@detail@v8@fmt@@YAXAEAV?$buffer@_W@234@V?$basic_string_view@_W@34@V?$basic_format_args@V?$basic_format_context@V?$back_insert_iterator@V?$buffer@_W@detail@v8@fmt@@@std@@_W@v8@fmt@@@34@Vlocale_ref@234@@Z@@012@YAPEB_W00AEAUformat_handler@?1???$vformat_to@_W@012@YAXAEAV?$buffer@_W@012@V?$basic_string_view@_W@12@V?$basic_format_args@V?$basic_format_context@V?$back_insert_iterator@V?$buffer@_W@detail@v8@fmt@@@std@@_W@v8@fmt@@@12@Vlocale_ref@012@@Z@@Z@@Z 0000000180056d08     handles.obj
 0002:00010d30       $ip2state$??$do_parse_arg_id@_WAEAUid_adapter@?1???$parse_replacement_field@_WAEAUformat_handler@?1???$vformat_to@_W@detail@v8@fmt@@YAXAEAV?$buffer@_W@234@V?$basic_string_view@_W@34@V?$basic_format_args@V?$basic_format_context@V?$back_insert_iterator@V?$buffer@_W@detail@v8@fmt@@@std@@_W@v8@fmt@@@34@Vlocale_ref@234@@Z@@detail@v8@fmt@@YAPEB_WPEB_W0AEAUformat_handler@?1???$vformat_to@_W@234@YAXAEAV?$buffer@_W@234@V?$basic_string_view@_W@34@V?$basic_format_args@V?$basic_format_context@V?$back_insert_iterator@V?$buffer@_W@detail@v8@fmt@@@std@@_W@v8@fmt@@@34@Vlocale_ref@234@@Z@@Z@@detail@v8@fmt@@YAPEB_WPEB_W0AEAUid_adapter@?1???$parse_replacement_field@_WAEAUformat_handler@?1???$vformat_to@_W@detail@v8@fmt@@YAXAEAV?$buffer@_W@234@V?$basic_string_view@_W@34@V?$basic_format_args@V?$basic_format_context@V?$back_insert_iterator@V?$buffer@_W@detail@v8@fmt@@@std@@_W@v8@fmt@@@34@Vlocale_ref@234@@Z@@012@YAPEB_W00AEAUformat_handler@?1???$vformat_to@_W@012@YAXAEAV?$buffer@_W@012@V?$basic_string_view@_W@12@V?$basic_format_args@V?$basic_format_context@V?$back_insert_iterator@V?$buffer@_W@detail@v8@fmt@@@std@@_W@v8@fmt@@@12@Vlocale_ref@012@@Z@@Z@@Z 0000000180056d30     handles.obj
 0002:00010d50       $unwind$??$write_int@_WV?$back_insert_iterator@V?$buffer@_W@detail@v8@fmt@@@std@@I@detail@v8@fmt@@YA?AV?$back_insert_iterator@V?$buffer@_W@detail@v8@fmt@@@std@@V34@U?$write_int_arg@I@012@AEBU?$basic_format_specs@_W@12@Vlocale_ref@012@@Z 0000000180056d50     handles.obj
 0002:00010d70       $ip2state$??$write_int@_WV?$back_insert_iterator@V?$buffer@_W@detail@v8@fmt@@@std@@I@detail@v8@fmt@@YA?AV?$back_insert_iterator@V?$buffer@_W@detail@v8@fmt@@@std@@V34@U?$write_int_arg@I@012@AEBU?$basic_format_specs@_W@12@Vlocale_ref@012@@Z 0000000180056d70     handles.obj
 0002:00010d90       $unwind$??R<lambda_2>@?8???$write_int@_WV?$back_insert_iterator@V?$buffer@_W@detail@v8@fmt@@@std@@I@detail@v8@fmt@@YA?AV?$back_insert_iterator@V?$buffer@_W@detail@v8@fmt@@@std@@V45@U?$write_int_arg@I@123@AEBU?$basic_format_specs@_W@23@Vlocale_ref@123@@Z@QEBA@0@Z 0000000180056d90     handles.obj
 0002:00010da8       $unwind$??$do_write_float@V?$back_insert_iterator@V?$buffer@_W@detail@v8@fmt@@@std@@U?$decimal_fp@M@dragonbox@detail@v8@fmt@@_WV?$digit_grouping@_W@567@@detail@v8@fmt@@YA?AV?$back_insert_iterator@V?$buffer@_W@detail@v8@fmt@@@std@@V34@AEBU?$decimal_fp@M@dragonbox@012@AEBU?$basic_format_specs@_W@12@Ufloat_specs@012@Vlocale_ref@012@@Z 0000000180056da8     handles.obj
 0002:00010dc4       $stateUnwindMap$??$do_write_float@V?$back_insert_iterator@V?$buffer@_W@detail@v8@fmt@@@std@@U?$decimal_fp@M@dragonbox@detail@v8@fmt@@_WV?$digit_grouping@_W@567@@detail@v8@fmt@@YA?AV?$back_insert_iterator@V?$buffer@_W@detail@v8@fmt@@@std@@V34@AEBU?$decimal_fp@M@dragonbox@012@AEBU?$basic_format_specs@_W@12@Ufloat_specs@012@Vlocale_ref@012@@Z 0000000180056dc4     handles.obj
 0002:00010e00       $ip2state$??$do_write_float@V?$back_insert_iterator@V?$buffer@_W@detail@v8@fmt@@@std@@U?$decimal_fp@M@dragonbox@detail@v8@fmt@@_WV?$digit_grouping@_W@567@@detail@v8@fmt@@YA?AV?$back_insert_iterator@V?$buffer@_W@detail@v8@fmt@@@std@@V34@AEBU?$decimal_fp@M@dragonbox@012@AEBU?$basic_format_specs@_W@12@Ufloat_specs@012@Vlocale_ref@012@@Z 0000000180056e00     handles.obj
 0002:00010e30       $unwind$??R<lambda_2>@?4???$do_write_float@V?$back_insert_iterator@V?$buffer@_W@detail@v8@fmt@@@std@@U?$decimal_fp@M@dragonbox@detail@v8@fmt@@_WV?$digit_grouping@_W@567@@detail@v8@fmt@@YA?AV?$back_insert_iterator@V?$buffer@_W@detail@v8@fmt@@@std@@V45@AEBU?$decimal_fp@M@dragonbox@123@AEBU?$basic_format_specs@_W@23@Ufloat_specs@123@Vlocale_ref@123@@Z@QEBA@0@Z 0000000180056e30     handles.obj
 0002:00010e48       $unwind$??R<lambda_3>@?BD@???$do_write_float@V?$back_insert_iterator@V?$buffer@_W@detail@v8@fmt@@@std@@U?$decimal_fp@M@dragonbox@detail@v8@fmt@@_WV?$digit_grouping@_W@567@@detail@v8@fmt@@YA?AV?$back_insert_iterator@V?$buffer@_W@detail@v8@fmt@@@std@@V45@AEBU?$decimal_fp@M@dragonbox@123@AEBU?$basic_format_specs@_W@23@Ufloat_specs@123@Vlocale_ref@123@@Z@QEBA@0@Z 0000000180056e48     handles.obj
 0002:00010e64       $stateUnwindMap$??R<lambda_3>@?BD@???$do_write_float@V?$back_insert_iterator@V?$buffer@_W@detail@v8@fmt@@@std@@U?$decimal_fp@M@dragonbox@detail@v8@fmt@@_WV?$digit_grouping@_W@567@@detail@v8@fmt@@YA?AV?$back_insert_iterator@V?$buffer@_W@detail@v8@fmt@@@std@@V45@AEBU?$decimal_fp@M@dragonbox@123@AEBU?$basic_format_specs@_W@23@Ufloat_specs@123@Vlocale_ref@123@@Z@QEBA@0@Z 0000000180056e64     handles.obj
 0002:00010e64       $stateUnwindMap$??R<lambda_3>@?BD@???$do_write_float@V?$back_insert_iterator@V?$buffer@_W@detail@v8@fmt@@@std@@U?$decimal_fp@N@dragonbox@detail@v8@fmt@@_WV?$digit_grouping@_W@567@@detail@v8@fmt@@YA?AV?$back_insert_iterator@V?$buffer@_W@detail@v8@fmt@@@std@@V45@AEBU?$decimal_fp@N@dragonbox@123@AEBU?$basic_format_specs@_W@23@Ufloat_specs@123@Vlocale_ref@123@@Z@QEBA@0@Z 0000000180056e64     handles.obj
 0002:00010e70       $ip2state$??R<lambda_3>@?BD@???$do_write_float@V?$back_insert_iterator@V?$buffer@_W@detail@v8@fmt@@@std@@U?$decimal_fp@M@dragonbox@detail@v8@fmt@@_WV?$digit_grouping@_W@567@@detail@v8@fmt@@YA?AV?$back_insert_iterator@V?$buffer@_W@detail@v8@fmt@@@std@@V45@AEBU?$decimal_fp@M@dragonbox@123@AEBU?$basic_format_specs@_W@23@Ufloat_specs@123@Vlocale_ref@123@@Z@QEBA@0@Z 0000000180056e70     handles.obj
 0002:00010e88       $unwind$??$do_write_float@V?$back_insert_iterator@V?$buffer@_W@detail@v8@fmt@@@std@@U?$decimal_fp@N@dragonbox@detail@v8@fmt@@_WV?$digit_grouping@_W@567@@detail@v8@fmt@@YA?AV?$back_insert_iterator@V?$buffer@_W@detail@v8@fmt@@@std@@V34@AEBU?$decimal_fp@N@dragonbox@012@AEBU?$basic_format_specs@_W@12@Ufloat_specs@012@Vlocale_ref@012@@Z 0000000180056e88     handles.obj
 0002:00010ea4       $stateUnwindMap$??$do_write_float@V?$back_insert_iterator@V?$buffer@_W@detail@v8@fmt@@@std@@U?$decimal_fp@N@dragonbox@detail@v8@fmt@@_WV?$digit_grouping@_W@567@@detail@v8@fmt@@YA?AV?$back_insert_iterator@V?$buffer@_W@detail@v8@fmt@@@std@@V34@AEBU?$decimal_fp@N@dragonbox@012@AEBU?$basic_format_specs@_W@12@Ufloat_specs@012@Vlocale_ref@012@@Z 0000000180056ea4     handles.obj
 0002:00010ea4       $stateUnwindMap$??$do_write_float@V?$back_insert_iterator@V?$buffer@_W@detail@v8@fmt@@@std@@Ubig_decimal_fp@detail@v8@fmt@@_WV?$digit_grouping@_W@456@@detail@v8@fmt@@YA?AV?$back_insert_iterator@V?$buffer@_W@detail@v8@fmt@@@std@@V34@AEBUbig_decimal_fp@012@AEBU?$basic_format_specs@_W@12@Ufloat_specs@012@Vlocale_ref@012@@Z 0000000180056ea4     handles.obj
 0002:00010ee0       $ip2state$??$do_write_float@V?$back_insert_iterator@V?$buffer@_W@detail@v8@fmt@@@std@@U?$decimal_fp@N@dragonbox@detail@v8@fmt@@_WV?$digit_grouping@_W@567@@detail@v8@fmt@@YA?AV?$back_insert_iterator@V?$buffer@_W@detail@v8@fmt@@@std@@V34@AEBU?$decimal_fp@N@dragonbox@012@AEBU?$basic_format_specs@_W@12@Ufloat_specs@012@Vlocale_ref@012@@Z 0000000180056ee0     handles.obj
 0002:00010f10       $unwind$??R<lambda_3>@?BD@???$do_write_float@V?$back_insert_iterator@V?$buffer@_W@detail@v8@fmt@@@std@@U?$decimal_fp@N@dragonbox@detail@v8@fmt@@_WV?$digit_grouping@_W@567@@detail@v8@fmt@@YA?AV?$back_insert_iterator@V?$buffer@_W@detail@v8@fmt@@@std@@V45@AEBU?$decimal_fp@N@dragonbox@123@AEBU?$basic_format_specs@_W@23@Ufloat_specs@123@Vlocale_ref@123@@Z@QEBA@0@Z 0000000180056f10     handles.obj
 0002:00010f30       $ip2state$??R<lambda_3>@?BD@???$do_write_float@V?$back_insert_iterator@V?$buffer@_W@detail@v8@fmt@@@std@@U?$decimal_fp@N@dragonbox@detail@v8@fmt@@_WV?$digit_grouping@_W@567@@detail@v8@fmt@@YA?AV?$back_insert_iterator@V?$buffer@_W@detail@v8@fmt@@@std@@V45@AEBU?$decimal_fp@N@dragonbox@123@AEBU?$basic_format_specs@_W@23@Ufloat_specs@123@Vlocale_ref@123@@Z@QEBA@0@Z 0000000180056f30     handles.obj
 0002:00010f48       $unwind$??R<lambda_4>@?BO@???$do_write_float@V?$back_insert_iterator@V?$buffer@_W@detail@v8@fmt@@@std@@U?$decimal_fp@N@dragonbox@detail@v8@fmt@@_WV?$digit_grouping@_W@567@@detail@v8@fmt@@YA?AV?$back_insert_iterator@V?$buffer@_W@detail@v8@fmt@@@std@@V45@AEBU?$decimal_fp@N@dragonbox@123@AEBU?$basic_format_specs@_W@23@Ufloat_specs@123@Vlocale_ref@123@@Z@QEBA@0@Z 0000000180056f48     handles.obj
 0002:00010f64       $stateUnwindMap$??$write_significand@V?$back_insert_iterator@V?$buffer@_W@detail@v8@fmt@@@std@@_WIV?$digit_grouping@_W@detail@v8@fmt@@@detail@v8@fmt@@YA?AV?$back_insert_iterator@V?$buffer@_W@detail@v8@fmt@@@std@@V34@IHH_WAEBV?$digit_grouping@_W@012@@Z 0000000180056f64     handles.obj
 0002:00010f64       $stateUnwindMap$??R<lambda_4>@?BO@???$do_write_float@V?$back_insert_iterator@V?$buffer@_W@detail@v8@fmt@@@std@@U?$decimal_fp@N@dragonbox@detail@v8@fmt@@_WV?$digit_grouping@_W@567@@detail@v8@fmt@@YA?AV?$back_insert_iterator@V?$buffer@_W@detail@v8@fmt@@@std@@V45@AEBU?$decimal_fp@N@dragonbox@123@AEBU?$basic_format_specs@_W@23@Ufloat_specs@123@Vlocale_ref@123@@Z@QEBA@0@Z 0000000180056f64     handles.obj
 0002:00010f64       $stateUnwindMap$??R<lambda_4>@?BO@???$do_write_float@V?$back_insert_iterator@V?$buffer@_W@detail@v8@fmt@@@std@@Ubig_decimal_fp@detail@v8@fmt@@_WV?$digit_grouping@_W@456@@detail@v8@fmt@@YA?AV?$back_insert_iterator@V?$buffer@_W@detail@v8@fmt@@@std@@V45@AEBUbig_decimal_fp@123@AEBU?$basic_format_specs@_W@23@Ufloat_specs@123@Vlocale_ref@123@@Z@QEBA@0@Z 0000000180056f64     handles.obj
 0002:00010f70       $ip2state$??R<lambda_4>@?BO@???$do_write_float@V?$back_insert_iterator@V?$buffer@_W@detail@v8@fmt@@@std@@U?$decimal_fp@N@dragonbox@detail@v8@fmt@@_WV?$digit_grouping@_W@567@@detail@v8@fmt@@YA?AV?$back_insert_iterator@V?$buffer@_W@detail@v8@fmt@@@std@@V45@AEBU?$decimal_fp@N@dragonbox@123@AEBU?$basic_format_specs@_W@23@Ufloat_specs@123@Vlocale_ref@123@@Z@QEBA@0@Z 0000000180056f70     handles.obj
 0002:00010f88       $unwind$??$format_uint@$03_WV?$back_insert_iterator@V?$buffer@_W@detail@v8@fmt@@@std@@_K@detail@v8@fmt@@YA?AV?$back_insert_iterator@V?$buffer@_W@detail@v8@fmt@@@std@@V34@_KH_N@Z 0000000180056f88     handles.obj
 0002:00010fa0       $unwind$??$visit_format_arg@V?$width_checker@Uerror_handler@detail@v8@fmt@@@detail@v8@fmt@@V?$basic_format_context@V?$back_insert_iterator@V?$buffer@_W@detail@v8@fmt@@@std@@_W@34@@v8@fmt@@YA_K$$QEAV?$width_checker@Uerror_handler@detail@v8@fmt@@@detail@01@AEBV?$basic_format_arg@V?$basic_format_context@V?$back_insert_iterator@V?$buffer@_W@detail@v8@fmt@@@std@@_W@v8@fmt@@@01@@Z 0000000180056fa0     handles.obj
 0002:00010fe8       $stateUnwindMap$??$visit_format_arg@V?$precision_checker@Uerror_handler@detail@v8@fmt@@@detail@v8@fmt@@V?$basic_format_context@V?$back_insert_iterator@V?$buffer@_W@detail@v8@fmt@@@std@@_W@34@@v8@fmt@@YA_K$$QEAV?$precision_checker@Uerror_handler@detail@v8@fmt@@@detail@01@AEBV?$basic_format_arg@V?$basic_format_context@V?$back_insert_iterator@V?$buffer@_W@detail@v8@fmt@@@std@@_W@v8@fmt@@@01@@Z 0000000180056fe8     handles.obj
 0002:00010fe8       $stateUnwindMap$??$visit_format_arg@V?$width_checker@Uerror_handler@detail@v8@fmt@@@detail@v8@fmt@@V?$basic_format_context@V?$back_insert_iterator@V?$buffer@_W@detail@v8@fmt@@@std@@_W@34@@v8@fmt@@YA_K$$QEAV?$width_checker@Uerror_handler@detail@v8@fmt@@@detail@01@AEBV?$basic_format_arg@V?$basic_format_context@V?$back_insert_iterator@V?$buffer@_W@detail@v8@fmt@@@std@@_W@v8@fmt@@@01@@Z 0000000180056fe8     handles.obj
 0002:00011010       $ip2state$??$visit_format_arg@V?$width_checker@Uerror_handler@detail@v8@fmt@@@detail@v8@fmt@@V?$basic_format_context@V?$back_insert_iterator@V?$buffer@_W@detail@v8@fmt@@@std@@_W@34@@v8@fmt@@YA_K$$QEAV?$width_checker@Uerror_handler@detail@v8@fmt@@@detail@01@AEBV?$basic_format_arg@V?$basic_format_context@V?$back_insert_iterator@V?$buffer@_W@detail@v8@fmt@@@std@@_W@v8@fmt@@@01@@Z 0000000180057010     handles.obj
 0002:00011060       $unwind$??$visit_format_arg@V?$precision_checker@Uerror_handler@detail@v8@fmt@@@detail@v8@fmt@@V?$basic_format_context@V?$back_insert_iterator@V?$buffer@_W@detail@v8@fmt@@@std@@_W@34@@v8@fmt@@YA_K$$QEAV?$precision_checker@Uerror_handler@detail@v8@fmt@@@detail@01@AEBV?$basic_format_arg@V?$basic_format_context@V?$back_insert_iterator@V?$buffer@_W@detail@v8@fmt@@@std@@_W@v8@fmt@@@01@@Z 0000000180057060     handles.obj
 0002:000110b0       $ip2state$??$visit_format_arg@V?$precision_checker@Uerror_handler@detail@v8@fmt@@@detail@v8@fmt@@V?$basic_format_context@V?$back_insert_iterator@V?$buffer@_W@detail@v8@fmt@@@std@@_W@34@@v8@fmt@@YA_K$$QEAV?$precision_checker@Uerror_handler@detail@v8@fmt@@@detail@01@AEBV?$basic_format_arg@V?$basic_format_context@V?$back_insert_iterator@V?$buffer@_W@detail@v8@fmt@@@std@@_W@v8@fmt@@@01@@Z 00000001800570b0     handles.obj
 0002:00011100       $unwind$??$write_int@_WV?$back_insert_iterator@V?$buffer@_W@detail@v8@fmt@@@std@@_K@detail@v8@fmt@@YA?AV?$back_insert_iterator@V?$buffer@_W@detail@v8@fmt@@@std@@V34@U?$write_int_arg@_K@012@AEBU?$basic_format_specs@_W@12@Vlocale_ref@012@@Z 0000000180057100     handles.obj
 0002:00011120       $ip2state$??$write_int@_WV?$back_insert_iterator@V?$buffer@_W@detail@v8@fmt@@@std@@_K@detail@v8@fmt@@YA?AV?$back_insert_iterator@V?$buffer@_W@detail@v8@fmt@@@std@@V34@U?$write_int_arg@_K@012@AEBU?$basic_format_specs@_W@12@Vlocale_ref@012@@Z 0000000180057120     handles.obj
 0002:00011130       $unwind$??$do_write_float@V?$back_insert_iterator@V?$buffer@_W@detail@v8@fmt@@@std@@Ubig_decimal_fp@detail@v8@fmt@@_WV?$digit_grouping@_W@456@@detail@v8@fmt@@YA?AV?$back_insert_iterator@V?$buffer@_W@detail@v8@fmt@@@std@@V34@AEBUbig_decimal_fp@012@AEBU?$basic_format_specs@_W@12@Ufloat_specs@012@Vlocale_ref@012@@Z 0000000180057130     handles.obj
 0002:00011150       $ip2state$??$do_write_float@V?$back_insert_iterator@V?$buffer@_W@detail@v8@fmt@@@std@@Ubig_decimal_fp@detail@v8@fmt@@_WV?$digit_grouping@_W@456@@detail@v8@fmt@@YA?AV?$back_insert_iterator@V?$buffer@_W@detail@v8@fmt@@@std@@V34@AEBUbig_decimal_fp@012@AEBU?$basic_format_specs@_W@12@Ufloat_specs@012@Vlocale_ref@012@@Z 0000000180057150     handles.obj
 0002:00011180       $unwind$??R<lambda_4>@?BO@???$do_write_float@V?$back_insert_iterator@V?$buffer@_W@detail@v8@fmt@@@std@@Ubig_decimal_fp@detail@v8@fmt@@_WV?$digit_grouping@_W@456@@detail@v8@fmt@@YA?AV?$back_insert_iterator@V?$buffer@_W@detail@v8@fmt@@@std@@V45@AEBUbig_decimal_fp@123@AEBU?$basic_format_specs@_W@23@Ufloat_specs@123@Vlocale_ref@123@@Z@QEBA@0@Z 0000000180057180     handles.obj
 0002:000111a0       $ip2state$??R<lambda_4>@?BO@???$do_write_float@V?$back_insert_iterator@V?$buffer@_W@detail@v8@fmt@@@std@@Ubig_decimal_fp@detail@v8@fmt@@_WV?$digit_grouping@_W@456@@detail@v8@fmt@@YA?AV?$back_insert_iterator@V?$buffer@_W@detail@v8@fmt@@@std@@V45@AEBUbig_decimal_fp@123@AEBU?$basic_format_specs@_W@23@Ufloat_specs@123@Vlocale_ref@123@@Z@QEBA@0@Z 00000001800571a0     handles.obj
 0002:000111b8       $unwind$??0?$digit_grouping@_W@detail@v8@fmt@@QEAA@Vlocale_ref@123@_N@Z 00000001800571b8     handles.obj
 0002:000111d0       $stateUnwindMap$??0?$digit_grouping@_W@detail@v8@fmt@@QEAA@Vlocale_ref@123@_N@Z 00000001800571d0     handles.obj
 0002:000111f0       $ip2state$??0?$digit_grouping@_W@detail@v8@fmt@@QEAA@Vlocale_ref@123@_N@Z 00000001800571f0     handles.obj
 0002:000111f8       $unwind$??$write_int_localized@V?$back_insert_iterator@V?$buffer@_W@detail@v8@fmt@@@std@@_K_W@detail@v8@fmt@@YA_NAEAV?$back_insert_iterator@V?$buffer@_W@detail@v8@fmt@@@std@@_KIAEBU?$basic_format_specs@_W@12@Vlocale_ref@012@@Z 00000001800571f8     handles.obj
 0002:00011214       $stateUnwindMap$??$write_int_localized@V?$back_insert_iterator@V?$buffer@_W@detail@v8@fmt@@@std@@_K_W@detail@v8@fmt@@YA_NAEAV?$back_insert_iterator@V?$buffer@_W@detail@v8@fmt@@@std@@_KIAEBU?$basic_format_specs@_W@12@Vlocale_ref@012@@Z 0000000180057214     handles.obj
 0002:00011240       $ip2state$??$write_int_localized@V?$back_insert_iterator@V?$buffer@_W@detail@v8@fmt@@@std@@_K_W@detail@v8@fmt@@YA_NAEAV?$back_insert_iterator@V?$buffer@_W@detail@v8@fmt@@@std@@_KIAEBU?$basic_format_specs@_W@12@Vlocale_ref@012@@Z 0000000180057240     handles.obj
 0002:00011250       $unwind$??$write_int@V?$back_insert_iterator@V?$buffer@_W@detail@v8@fmt@@@std@@_WV<lambda_3>@?M@???$write_int@_WV?$back_insert_iterator@V?$buffer@_W@detail@v8@fmt@@@std@@I@detail@v8@fmt@@YA?AV12@V12@U?$write_int_arg@I@456@AEBU?$basic_format_specs@_W@56@Vlocale_ref@456@@Z@@detail@v8@fmt@@YA?AV?$back_insert_iterator@V?$buffer@_W@detail@v8@fmt@@@std@@V34@HIAEBU?$basic_format_specs@_W@12@V<lambda_3>@?M@???$write_int@_WV?$back_insert_iterator@V?$buffer@_W@detail@v8@fmt@@@std@@I@012@YA?AV34@0U?$write_int_arg@I@012@1Vlocale_ref@012@@Z@@Z 0000000180057250     handles.obj
 0002:00011264       $unwind$??$write_int@V?$back_insert_iterator@V?$buffer@_W@detail@v8@fmt@@@std@@_WV<lambda_4>@?P@???$write_int@_WV?$back_insert_iterator@V?$buffer@_W@detail@v8@fmt@@@std@@I@detail@v8@fmt@@YA?AV12@V12@U?$write_int_arg@I@456@AEBU?$basic_format_specs@_W@56@Vlocale_ref@456@@Z@@detail@v8@fmt@@YA?AV?$back_insert_iterator@V?$buffer@_W@detail@v8@fmt@@@std@@V34@HIAEBU?$basic_format_specs@_W@12@V<lambda_4>@?P@???$write_int@_WV?$back_insert_iterator@V?$buffer@_W@detail@v8@fmt@@@std@@I@012@YA?AV34@0U?$write_int_arg@I@012@1Vlocale_ref@012@@Z@@Z 0000000180057264     handles.obj
 0002:00011278       $unwind$??$write_significand@V?$back_insert_iterator@V?$buffer@_W@detail@v8@fmt@@@std@@_WIV?$digit_grouping@_W@detail@v8@fmt@@@detail@v8@fmt@@YA?AV?$back_insert_iterator@V?$buffer@_W@detail@v8@fmt@@@std@@V34@IHH_WAEBV?$digit_grouping@_W@012@@Z 0000000180057278     handles.obj
 0002:000112a0       $ip2state$??$write_significand@V?$back_insert_iterator@V?$buffer@_W@detail@v8@fmt@@@std@@_WIV?$digit_grouping@_W@detail@v8@fmt@@@detail@v8@fmt@@YA?AV?$back_insert_iterator@V?$buffer@_W@detail@v8@fmt@@@std@@V34@IHH_WAEBV?$digit_grouping@_W@012@@Z 00000001800572a0     handles.obj
 0002:000112b8       $unwind$??$write_significand@V?$back_insert_iterator@V?$buffer@_W@detail@v8@fmt@@@std@@_K_W$0A@@detail@v8@fmt@@YA?AV?$back_insert_iterator@V?$buffer@_W@detail@v8@fmt@@@std@@V34@_KHH_W@Z 00000001800572b8     handles.obj
 0002:000112cc       $unwind$??$write_padded@$01V?$back_insert_iterator@V?$buffer@_W@detail@v8@fmt@@@std@@_WAEAV<lambda_1>@?1???$write_ptr@_WV?$back_insert_iterator@V?$buffer@_W@detail@v8@fmt@@@std@@_K@detail@v8@fmt@@YA?AV12@V12@_KPEBU?$basic_format_specs@_W@56@@Z@@detail@v8@fmt@@YA?AV?$back_insert_iterator@V?$buffer@_W@detail@v8@fmt@@@std@@V34@AEBU?$basic_format_specs@_W@12@_K2AEAV<lambda_1>@?1???$write_ptr@_WV?$back_insert_iterator@V?$buffer@_W@detail@v8@fmt@@@std@@_K@012@YA?AV34@02PEBU512@@Z@@Z 00000001800572cc     handles.obj
 0002:000112e8       $unwind$??$write_int@V?$back_insert_iterator@V?$buffer@_W@detail@v8@fmt@@@std@@_WV<lambda_3>@?M@???$write_int@_WV?$back_insert_iterator@V?$buffer@_W@detail@v8@fmt@@@std@@_K@detail@v8@fmt@@YA?AV12@V12@U?$write_int_arg@_K@456@AEBU?$basic_format_specs@_W@56@Vlocale_ref@456@@Z@@detail@v8@fmt@@YA?AV?$back_insert_iterator@V?$buffer@_W@detail@v8@fmt@@@std@@V34@HIAEBU?$basic_format_specs@_W@12@V<lambda_3>@?M@???$write_int@_WV?$back_insert_iterator@V?$buffer@_W@detail@v8@fmt@@@std@@_K@012@YA?AV34@0U?$write_int_arg@_K@012@1Vlocale_ref@012@@Z@@Z 00000001800572e8     handles.obj
 0002:000112fc       $unwind$??$write_int@V?$back_insert_iterator@V?$buffer@_W@detail@v8@fmt@@@std@@_WV<lambda_4>@?P@???$write_int@_WV?$back_insert_iterator@V?$buffer@_W@detail@v8@fmt@@@std@@_K@detail@v8@fmt@@YA?AV12@V12@U?$write_int_arg@_K@456@AEBU?$basic_format_specs@_W@56@Vlocale_ref@456@@Z@@detail@v8@fmt@@YA?AV?$back_insert_iterator@V?$buffer@_W@detail@v8@fmt@@@std@@V34@HIAEBU?$basic_format_specs@_W@12@V<lambda_4>@?P@???$write_int@_WV?$back_insert_iterator@V?$buffer@_W@detail@v8@fmt@@@std@@_K@012@YA?AV34@0U?$write_int_arg@_K@012@1Vlocale_ref@012@@Z@@Z 00000001800572fc     handles.obj
 0002:00011310       $unwind$??$write_significand@_WV?$back_insert_iterator@V?$buffer@_W@detail@v8@fmt@@@std@@PEBDV?$digit_grouping@_W@detail@v8@fmt@@@detail@v8@fmt@@YA?AV?$back_insert_iterator@V?$buffer@_W@detail@v8@fmt@@@std@@V34@PEBDHHAEBV?$digit_grouping@_W@012@@Z 0000000180057310     handles.obj
 0002:00011330       $stateUnwindMap$??$write_significand@_WV?$back_insert_iterator@V?$buffer@_W@detail@v8@fmt@@@std@@PEBDV?$digit_grouping@_W@detail@v8@fmt@@@detail@v8@fmt@@YA?AV?$back_insert_iterator@V?$buffer@_W@detail@v8@fmt@@@std@@V34@PEBDHHAEBV?$digit_grouping@_W@012@@Z 0000000180057330     handles.obj
 0002:00011340       $ip2state$??$write_significand@_WV?$back_insert_iterator@V?$buffer@_W@detail@v8@fmt@@@std@@PEBDV?$digit_grouping@_W@detail@v8@fmt@@@detail@v8@fmt@@YA?AV?$back_insert_iterator@V?$buffer@_W@detail@v8@fmt@@@std@@V34@PEBDHHAEBV?$digit_grouping@_W@012@@Z 0000000180057340     handles.obj
 0002:00011358       $unwind$??$write_significand@_WI$0A@@detail@v8@fmt@@YAPEA_WPEA_WIHH_W@Z 0000000180057358     handles.obj
 0002:0001136c       $unwind$??$apply@V?$back_insert_iterator@V?$buffer@_W@detail@v8@fmt@@@std@@D@?$digit_grouping@_W@detail@v8@fmt@@QEBA?AV?$back_insert_iterator@V?$buffer@_W@detail@v8@fmt@@@std@@V45@V?$basic_string_view@D@23@@Z 000000018005736c     handles.obj
 0002:00011390       $stateUnwindMap$??$apply@V?$back_insert_iterator@V?$buffer@_W@detail@v8@fmt@@@std@@D@?$digit_grouping@_W@detail@v8@fmt@@QEBA?AV?$back_insert_iterator@V?$buffer@_W@detail@v8@fmt@@@std@@V45@V?$basic_string_view@D@23@@Z 0000000180057390     handles.obj
 0002:00011390       $stateUnwindMap$??$apply@V?$back_insert_iterator@V?$buffer@_W@detail@v8@fmt@@@std@@_W@?$digit_grouping@_W@detail@v8@fmt@@QEBA?AV?$back_insert_iterator@V?$buffer@_W@detail@v8@fmt@@@std@@V45@V?$basic_string_view@_W@23@@Z 0000000180057390     handles.obj
 0002:000113a0       $ip2state$??$apply@V?$back_insert_iterator@V?$buffer@_W@detail@v8@fmt@@@std@@D@?$digit_grouping@_W@detail@v8@fmt@@QEBA?AV?$back_insert_iterator@V?$buffer@_W@detail@v8@fmt@@@std@@V45@V?$basic_string_view@D@23@@Z 00000001800573a0     handles.obj
 0002:000113b8       $unwind$??$apply@V?$back_insert_iterator@V?$buffer@_W@detail@v8@fmt@@@std@@_W@?$digit_grouping@_W@detail@v8@fmt@@QEBA?AV?$back_insert_iterator@V?$buffer@_W@detail@v8@fmt@@@std@@V45@V?$basic_string_view@_W@23@@Z 00000001800573b8     handles.obj
 0002:000113e0       $ip2state$??$apply@V?$back_insert_iterator@V?$buffer@_W@detail@v8@fmt@@@std@@_W@?$digit_grouping@_W@detail@v8@fmt@@QEBA?AV?$back_insert_iterator@V?$buffer@_W@detail@v8@fmt@@@std@@V45@V?$basic_string_view@_W@23@@Z 00000001800573e0     handles.obj
 0002:000113f8       $unwind$??$write_padded@$01V?$back_insert_iterator@V?$buffer@_W@detail@v8@fmt@@@std@@_WAEAV<lambda_1>@?1???$write_int@V?$back_insert_iterator@V?$buffer@_W@detail@v8@fmt@@@std@@_WV<lambda_3>@?M@???$write_int@_WV?$back_insert_iterator@V?$buffer@_W@detail@v8@fmt@@@std@@I@detail@v8@fmt@@YA?AV12@V12@U?$write_int_arg@I@456@AEBU?$basic_format_specs@_W@56@Vlocale_ref@456@@Z@@detail@v8@fmt@@YA?AV12@V12@HIAEBU?$basic_format_specs@_W@56@V<lambda_3>@?M@???$write_int@_WV?$back_insert_iterator@V?$buffer@_W@detail@v8@fmt@@@std@@I@456@YA?AV12@0U?$write_int_arg@I@456@1Vlocale_ref@456@@Z@@Z@@detail@v8@fmt@@YA?AV?$back_insert_iterator@V?$buffer@_W@detail@v8@fmt@@@std@@V34@AEBU?$basic_format_specs@_W@12@_K2AEAV<lambda_1>@?1???$write_int@V?$back_insert_iterator@V?$buffer@_W@detail@v8@fmt@@@std@@_WV<lambda_3>@?M@???$write_int@_WV?$back_insert_iterator@V?$buffer@_W@detail@v8@fmt@@@std@@I@detail@v8@fmt@@YA?AV12@V12@U?$write_int_arg@I@456@AEBU?$basic_format_specs@_W@56@Vlocale_ref@456@@Z@@012@YA?AV34@0HI1V<lambda_3>@?M@???$write_int@_WV?$back_insert_iterator@V?$buffer@_W@detail@v8@fmt@@@std@@I@012@YA?AV34@0U?$write_int_arg@I@012@1Vlocale_ref@012@@Z@@Z@@Z 00000001800573f8     handles.obj
 0002:00011414       $unwind$??$write_padded@$01V?$back_insert_iterator@V?$buffer@_W@detail@v8@fmt@@@std@@_WAEAV<lambda_1>@?1???$write_int@V?$back_insert_iterator@V?$buffer@_W@detail@v8@fmt@@@std@@_WV<lambda_4>@?P@???$write_int@_WV?$back_insert_iterator@V?$buffer@_W@detail@v8@fmt@@@std@@I@detail@v8@fmt@@YA?AV12@V12@U?$write_int_arg@I@456@AEBU?$basic_format_specs@_W@56@Vlocale_ref@456@@Z@@detail@v8@fmt@@YA?AV12@V12@HIAEBU?$basic_format_specs@_W@56@V<lambda_4>@?P@???$write_int@_WV?$back_insert_iterator@V?$buffer@_W@detail@v8@fmt@@@std@@I@456@YA?AV12@0U?$write_int_arg@I@456@1Vlocale_ref@456@@Z@@Z@@detail@v8@fmt@@YA?AV?$back_insert_iterator@V?$buffer@_W@detail@v8@fmt@@@std@@V34@AEBU?$basic_format_specs@_W@12@_K2AEAV<lambda_1>@?1???$write_int@V?$back_insert_iterator@V?$buffer@_W@detail@v8@fmt@@@std@@_WV<lambda_4>@?P@???$write_int@_WV?$back_insert_iterator@V?$buffer@_W@detail@v8@fmt@@@std@@I@detail@v8@fmt@@YA?AV12@V12@U?$write_int_arg@I@456@AEBU?$basic_format_specs@_W@56@Vlocale_ref@456@@Z@@012@YA?AV34@0HI1V<lambda_4>@?P@???$write_int@_WV?$back_insert_iterator@V?$buffer@_W@detail@v8@fmt@@@std@@I@012@YA?AV34@0U?$write_int_arg@I@012@1Vlocale_ref@012@@Z@@Z@@Z 0000000180057414     handles.obj
 0002:00011430       $unwind$??$write_padded@$01V?$back_insert_iterator@V?$buffer@_W@detail@v8@fmt@@@std@@_WAEAV<lambda_1>@?1???$write_int@V?$back_insert_iterator@V?$buffer@_W@detail@v8@fmt@@@std@@_WV<lambda_3>@?M@???$write_int@_WV?$back_insert_iterator@V?$buffer@_W@detail@v8@fmt@@@std@@_K@detail@v8@fmt@@YA?AV12@V12@U?$write_int_arg@_K@456@AEBU?$basic_format_specs@_W@56@Vlocale_ref@456@@Z@@detail@v8@fmt@@YA?AV12@V12@HIAEBU?$basic_format_specs@_W@56@V<lambda_3>@?M@???$write_int@_WV?$back_insert_iterator@V?$buffer@_W@detail@v8@fmt@@@std@@_K@456@YA?AV12@0U?$write_int_arg@_K@456@1Vlocale_ref@456@@Z@@Z@@detail@v8@fmt@@YA?AV?$back_insert_iterator@V?$buffer@_W@detail@v8@fmt@@@std@@V34@AEBU?$basic_format_specs@_W@12@_K2AEAV<lambda_1>@?1???$write_int@V?$back_insert_iterator@V?$buffer@_W@detail@v8@fmt@@@std@@_WV<lambda_3>@?M@???$write_int@_WV?$back_insert_iterator@V?$buffer@_W@detail@v8@fmt@@@std@@_K@detail@v8@fmt@@YA?AV12@V12@U?$write_int_arg@_K@456@AEBU?$basic_format_specs@_W@56@Vlocale_ref@456@@Z@@012@YA?AV34@0HI1V<lambda_3>@?M@???$write_int@_WV?$back_insert_iterator@V?$buffer@_W@detail@v8@fmt@@@std@@_K@012@YA?AV34@0U?$write_int_arg@_K@012@1Vlocale_ref@012@@Z@@Z@@Z 0000000180057430     handles.obj
 0002:0001144c       $unwind$??$write_padded@$01V?$back_insert_iterator@V?$buffer@_W@detail@v8@fmt@@@std@@_WAEAV<lambda_1>@?1???$write_int@V?$back_insert_iterator@V?$buffer@_W@detail@v8@fmt@@@std@@_WV<lambda_4>@?P@???$write_int@_WV?$back_insert_iterator@V?$buffer@_W@detail@v8@fmt@@@std@@_K@detail@v8@fmt@@YA?AV12@V12@U?$write_int_arg@_K@456@AEBU?$basic_format_specs@_W@56@Vlocale_ref@456@@Z@@detail@v8@fmt@@YA?AV12@V12@HIAEBU?$basic_format_specs@_W@56@V<lambda_4>@?P@???$write_int@_WV?$back_insert_iterator@V?$buffer@_W@detail@v8@fmt@@@std@@_K@456@YA?AV12@0U?$write_int_arg@_K@456@1Vlocale_ref@456@@Z@@Z@@detail@v8@fmt@@YA?AV?$back_insert_iterator@V?$buffer@_W@detail@v8@fmt@@@std@@V34@AEBU?$basic_format_specs@_W@12@_K2AEAV<lambda_1>@?1???$write_int@V?$back_insert_iterator@V?$buffer@_W@detail@v8@fmt@@@std@@_WV<lambda_4>@?P@???$write_int@_WV?$back_insert_iterator@V?$buffer@_W@detail@v8@fmt@@@std@@_K@detail@v8@fmt@@YA?AV12@V12@U?$write_int_arg@_K@456@AEBU?$basic_format_specs@_W@56@Vlocale_ref@456@@Z@@012@YA?AV34@0HI1V<lambda_4>@?P@???$write_int@_WV?$back_insert_iterator@V?$buffer@_W@detail@v8@fmt@@@std@@_K@012@YA?AV34@0U?$write_int_arg@_K@012@1Vlocale_ref@012@@Z@@Z@@Z 000000018005744c     handles.obj
 0002:00011468       $unwind$??0PluginSettings@@QEAA@AEBU_GUID@@P6A_JPEAXW4FAR_SETTINGS_CONTROL_COMMANDS@@_J1@Z@Z 0000000180057468     Pcfg.obj
 0002:0001147c       $unwind$??1PluginSettings@@QEAA@XZ 000000018005747c     Pcfg.obj
 0002:00011490       $ip2state$??1PluginSettings@@QEAA@XZ 0000000180057490     Pcfg.obj
 0002:00011498       $unwind$?SaveValue@PluginCheckBoxBinding@@UEAAXPEBUFarDialogItem@@H@Z 0000000180057498     Pcfg.obj
 0002:000114b0       $unwind$??1PluginDialogBuilder@@QEAA@XZ 00000001800574b0     Pcfg.obj
 0002:000114c0       $ip2state$??1PluginDialogBuilder@@QEAA@XZ 00000001800574c0     Pcfg.obj
 0002:000114c8       $unwind$?AddOKCancel@PluginDialogBuilder@@QEAAXHHH_N@Z 00000001800574c8     Pcfg.obj
 0002:000114e4       $unwind$?ItemWidth@PluginDialogBuilder@@CA_JAEBUFarDialogItem@@@Z 00000001800574e4     Pcfg.obj
 0002:000114fc       $unwind$?Config@@YAHXZ     00000001800574fc     Pcfg.obj
 0002:00011514       $stateUnwindMap$?Config@@YAHXZ 0000000180057514     Pcfg.obj
 0002:00011530       $ip2state$?Config@@YAHXZ   0000000180057530     Pcfg.obj
 0002:00011550       $unwind$?Write@options@@QEBAXXZ 0000000180057550     Pcfg.obj
 0002:0001156c       $stateUnwindMap$?Write@options@@QEBAXXZ 000000018005756c     Pcfg.obj
 0002:00011580       $ip2state$?Write@options@@QEBAXXZ 0000000180057580     Pcfg.obj
 0002:000115a0       $unwind$?Read@options@@QEAAXXZ 00000001800575a0     Pcfg.obj
 0002:000115bc       $stateUnwindMap$?Read@options@@QEAAXXZ 00000001800575bc     Pcfg.obj
 0002:000115d0       $ip2state$?Read@options@@QEAAXXZ 00000001800575d0     Pcfg.obj
 0002:000115f0       $unwind$?SmartReread@PerfThread@@QEAAXXZ 00000001800575f0     Pclass.obj
 0002:00011600       $unwind$?SaveValue@PluginEditFieldBinding@@UEAAXPEBUFarDialogItem@@H@Z 0000000180057600     Pclass.obj
 0002:00011610       $unwind$?ui64toa_width@@YA?AV?$basic_string@_WU?$char_traits@_W@std@@V?$allocator@_W@2@@std@@_KI_N@Z 0000000180057610     Pclass.obj
 0002:00011634       $stateUnwindMap$?ui64toa_width@@YA?AV?$basic_string@_WU?$char_traits@_W@std@@V?$allocator@_W@2@@std@@_KI_N@Z 0000000180057634     Pclass.obj
 0002:00011670       $ip2state$?ui64toa_width@@YA?AV?$basic_string@_WU?$char_traits@_W@std@@V?$allocator@_W@2@@std@@_KI_N@Z 0000000180057670     Pclass.obj
 0002:00011690       $unwind$?PrintTitle@@YA?AV?$basic_string@_WU?$char_traits@_W@std@@V?$allocator@_W@2@@std@@V?$basic_string_view@_WU?$char_traits@_W@std@@@2@@Z 0000000180057690     Pclass.obj
 0002:000116a8       $stateUnwindMap$?PrintTitle@@YA?AV?$basic_string@_WU?$char_traits@_W@std@@V?$allocator@_W@2@@std@@V?$basic_string_view@_WU?$char_traits@_W@std@@@2@@Z 00000001800576a8     Pclass.obj
 0002:000116b0       $ip2state$?PrintTitle@@YA?AV?$basic_string@_WU?$char_traits@_W@std@@V?$allocator@_W@2@@std@@V?$basic_string_view@_WU?$char_traits@_W@std@@@2@@Z 00000001800576b0     Pclass.obj
 0002:000116c0       $unwind$??0Plist@@QEAA@XZ  00000001800576c0     Pclass.obj
 0002:000116dc       $stateUnwindMap$??0Plist@@QEAA@XZ 00000001800576dc     Pclass.obj
 0002:00011720       $ip2state$??0Plist@@QEAA@XZ 0000000180057720     Pclass.obj
 0002:00011750       $unwind$?TranslateMode@@YA_NAEBV?$basic_string@_WU?$char_traits@_W@std@@V?$allocator@_W@2@@std@@AEAV12@@Z 0000000180057750     Pclass.obj
 0002:00011770       $stateUnwindMap$?TranslateMode@@YA_NAEBV?$basic_string@_WU?$char_traits@_W@std@@V?$allocator@_W@2@@std@@AEAV12@@Z 0000000180057770     Pclass.obj
 0002:00011790       $ip2state$?TranslateMode@@YA_NAEBV?$basic_string@_WU?$char_traits@_W@std@@V?$allocator@_W@2@@std@@AEAV12@@Z 0000000180057790     Pclass.obj
 0002:000117b0       $unwind$?InitializePanelModes@Plist@@SAXXZ 00000001800577b0     Pclass.obj
 0002:000117d0       $stateUnwindMap$?InitializePanelModes@Plist@@SAXXZ 00000001800577d0     Pclass.obj
 0002:000119c0       $ip2state$?InitializePanelModes@Plist@@SAXXZ 00000001800579c0     Pclass.obj
 0002:00011b40       $unwind$?dtor$181@?0??InitializePanelModes@Plist@@SAXXZ@4HA 0000000180057b40     Pclass.obj
 0002:00011b40       $unwind$?dtor$90@?0??InitializePanelModes@Plist@@SAXXZ@4HA 0000000180057b40     Pclass.obj
 0002:00011b48       $unwind$??$format@UFMT_COMPILE_STRING@?1???R<lambda_1>@?4??InitializePanelModes@Plist@@SAXXZ@QEBA@XZ@AEA_K@@YA?A_P$$QEAUFMT_COMPILE_STRING@?1???R<lambda_1>@?4??InitializePanelModes@Plist@@SAXXZ@QEBA@XZ@AEA_K@Z 0000000180057b48     Pclass.obj
 0002:00011b5c       $unwind$?SavePanelModes@Plist@@SAXXZ 0000000180057b5c     Pclass.obj
 0002:00011b7c       $stateUnwindMap$?SavePanelModes@Plist@@SAXXZ 0000000180057b7c     Pclass.obj
 0002:00011ba0       $ip2state$?SavePanelModes@Plist@@SAXXZ 0000000180057ba0     Pclass.obj
 0002:00011bd0       $unwind$?generate_titles@@YAXAEBV?$basic_string@_WU?$char_traits@_W@std@@V?$allocator@_W@2@@std@@AEAUPanelMode@@@Z 0000000180057bd0     Pclass.obj
 0002:00011bec       $stateUnwindMap$?generate_titles@@YAXAEBV?$basic_string@_WU?$char_traits@_W@std@@V?$allocator@_W@2@@std@@AEAUPanelMode@@@Z 0000000180057bec     Pclass.obj
 0002:00011c00       $ip2state$?generate_titles@@YAXAEBV?$basic_string@_WU?$char_traits@_W@std@@V?$allocator@_W@2@@std@@AEAUPanelMode@@@Z 0000000180057c00     Pclass.obj
 0002:00011c10       $unwind$?GetOpenPanelInfo@Plist@@QEAAXPEAUOpenPanelInfo@@@Z 0000000180057c10     Pclass.obj
 0002:00011c30       $stateUnwindMap$?GetOpenPanelInfo@Plist@@QEAAXPEAUOpenPanelInfo@@@Z 0000000180057c30     Pclass.obj
 0002:00011c50       $ip2state$?GetOpenPanelInfo@Plist@@QEAAXPEAUOpenPanelInfo@@@Z 0000000180057c50     Pclass.obj
 0002:00011c60       $unwind$?GetFindData@Plist@@QEAAHAEAPEAUPluginPanelItem@@AEA_K_K@Z 0000000180057c60     Pclass.obj
 0002:00011c84       $stateUnwindMap$?GetFindData@Plist@@QEAAHAEAPEAUPluginPanelItem@@AEA_K_K@Z 0000000180057c84     Pclass.obj
 0002:00011d20       $ip2state$?GetFindData@Plist@@QEAAHAEAPEAUPluginPanelItem@@AEA_K_K@Z 0000000180057d20     Pclass.obj
 0002:00011dc8       $unwind$?window_style@@YA@PEAUHWND__@@@Z 0000000180057dc8     Pclass.obj
 0002:00011de8       $stateUnwindMap$?window_ex_style@@YA@PEAUHWND__@@@Z 0000000180057de8     Pclass.obj
 0002:00011de8       $stateUnwindMap$?window_style@@YA@PEAUHWND__@@@Z 0000000180057de8     Pclass.obj
 0002:00011e00       $ip2state$?window_style@@YA@PEAUHWND__@@@Z 0000000180057e00     Pclass.obj
 0002:00011e20       $unwind$?window_ex_style@@YA@PEAUHWND__@@@Z 0000000180057e20     Pclass.obj
 0002:00011e40       $ip2state$?window_ex_style@@YA@PEAUHWND__@@@Z 0000000180057e40     Pclass.obj
 0002:00011e60       $unwind$?DumpNTCounters@@YAXPEAXAEAVPerfThread@@KK@Z 0000000180057e60     Pclass.obj
 0002:00011e80       $stateUnwindMap$?DumpNTCounters@@YAXPEAXAEAVPerfThread@@KK@Z 0000000180057e80     Pclass.obj
 0002:00011ea0       $ip2state$?DumpNTCounters@@YAXPEAXAEAVPerfThread@@KK@Z 0000000180057ea0     Pclass.obj
 0002:00011ed8       $unwind$?GetFiles@Plist@@QEAAHPEAUPluginPanelItem@@_KHPEAPEB_W1AEAUoptions@@@Z 0000000180057ed8     Pclass.obj
 0002:00011ef8       $stateUnwindMap$?GetFiles@Plist@@QEAAHPEAUPluginPanelItem@@_KHPEAPEB_W1AEAUoptions@@@Z 0000000180057ef8     Pclass.obj
 0002:00011fe0       $ip2state$?GetFiles@Plist@@QEAAHPEAUPluginPanelItem@@_KHPEAPEB_W1AEAUoptions@@@Z 0000000180057fe0     Pclass.obj
 0002:00012188       $unwind$??$format@UFMT_COMPILE_STRING@?1???R<lambda_18>@?EB@??GetFiles@Plist@@QEAAHPEAUPluginPanelItem@@_KHPEAPEB_W1AEAUoptions@@@Z@QEBA@XZ@PEB_WPEB_WHPEB_WPEB_W@@YA?A_P$$QEAUFMT_COMPILE_STRING@?1???R<lambda_18>@?EB@??GetFiles@Plist@@QEAAHPEAUPluginPanelItem@@_KHPEAPEB_W1AEAUoptions@@@Z@QEBA@XZ@$$QEAPEB_W5$$QEAH55@Z 0000000180058188     Pclass.obj
 0002:0001219c       $unwind$??1ProcessData@@QEAA@XZ 000000018005819c     Pclass.obj
 0002:000121a8       $unwind$?DeleteFiles@Plist@@QEAAHPEAUPluginPanelItem@@_K1@Z 00000001800581a8     Pclass.obj
 0002:000121cc       $stateUnwindMap$?DeleteFiles@Plist@@QEAAHPEAUPluginPanelItem@@_K1@Z 00000001800581cc     Pclass.obj
 0002:00012210       $ip2state$?DeleteFiles@Plist@@QEAAHPEAUPluginPanelItem@@_K1@Z 0000000180058210     Pclass.obj
 0002:00012240       $unwind$?Reread@Plist@@AEAAXXZ 0000000180058240     Pclass.obj
 0002:00012254       $unwind$?Connect@Plist@@QEAA_NPEB_W00@Z 0000000180058254     Pclass.obj
 0002:00012270       $stateUnwindMap$?Connect@Plist@@QEAA_NPEB_W00@Z 0000000180058270     Pclass.obj
 0002:000122a0       $ip2state$?Connect@Plist@@QEAA_NPEB_W00@Z 00000001800582a0     Pclass.obj
 0002:000122d0       $unwind$?ProcessKey@Plist@@QEAAHPEBU_INPUT_RECORD@@@Z 00000001800582d0     Pclass.obj
 0002:000122f4       $stateUnwindMap$?ProcessKey@Plist@@QEAAHPEBU_INPUT_RECORD@@@Z 00000001800582f4     Pclass.obj
 0002:000123b0       $ip2state$?ProcessKey@Plist@@QEAAHPEBU_INPUT_RECORD@@@Z 00000001800583b0     Pclass.obj
 0002:000124f0       $unwind$?dtor$0@?0??ProcessKey@Plist@@QEAAHPEBU_INPUT_RECORD@@@Z@4HA 00000001800584f0     Pclass.obj
 0002:000124f0       $unwind$?dtor$10@?0??ProcessKey@Plist@@QEAAHPEBU_INPUT_RECORD@@@Z@4HA 00000001800584f0     Pclass.obj
 0002:000124f0       $unwind$?dtor$11@?0??ProcessKey@Plist@@QEAAHPEBU_INPUT_RECORD@@@Z@4HA 00000001800584f0     Pclass.obj
 0002:000124f0       $unwind$?dtor$12@?0??ProcessKey@Plist@@QEAAHPEBU_INPUT_RECORD@@@Z@4HA 00000001800584f0     Pclass.obj
 0002:000124f0       $unwind$?dtor$13@?0??ProcessKey@Plist@@QEAAHPEBU_INPUT_RECORD@@@Z@4HA 00000001800584f0     Pclass.obj
 0002:000124f0       $unwind$?dtor$14@?0??ProcessKey@Plist@@QEAAHPEBU_INPUT_RECORD@@@Z@4HA 00000001800584f0     Pclass.obj
 0002:000124f0       $unwind$?dtor$1@?0??ProcessKey@Plist@@QEAAHPEBU_INPUT_RECORD@@@Z@4HA 00000001800584f0     Pclass.obj
 0002:000124f0       $unwind$?dtor$233@?0??ProcessKey@Plist@@QEAAHPEBU_INPUT_RECORD@@@Z@4HA 00000001800584f0     Pclass.obj
 0002:000124f0       $unwind$?dtor$235@?0??ProcessKey@Plist@@QEAAHPEBU_INPUT_RECORD@@@Z@4HA 00000001800584f0     Pclass.obj
 0002:000124f0       $unwind$?dtor$2@?0??ProcessKey@Plist@@QEAAHPEBU_INPUT_RECORD@@@Z@4HA 00000001800584f0     Pclass.obj
 0002:000124f0       $unwind$?dtor$3@?0??ProcessKey@Plist@@QEAAHPEBU_INPUT_RECORD@@@Z@4HA 00000001800584f0     Pclass.obj
 0002:000124f0       $unwind$?dtor$4@?0??ProcessKey@Plist@@QEAAHPEBU_INPUT_RECORD@@@Z@4HA 00000001800584f0     Pclass.obj
 0002:000124f0       $unwind$?dtor$5@?0??ProcessKey@Plist@@QEAAHPEBU_INPUT_RECORD@@@Z@4HA 00000001800584f0     Pclass.obj
 0002:000124f0       $unwind$?dtor$8@?0??ProcessKey@Plist@@QEAAHPEBU_INPUT_RECORD@@@Z@4HA 00000001800584f0     Pclass.obj
 0002:000124f0       $unwind$?dtor$9@?0??ProcessKey@Plist@@QEAAHPEBU_INPUT_RECORD@@@Z@4HA 00000001800584f0     Pclass.obj
 0002:000124f8       $unwind$?dtor$228@?0??ProcessKey@Plist@@QEAAHPEBU_INPUT_RECORD@@@Z@4HA 00000001800584f8     Pclass.obj
 0002:000124f8       $unwind$?dtor$230@?0??ProcessKey@Plist@@QEAAHPEBU_INPUT_RECORD@@@Z@4HA 00000001800584f8     Pclass.obj
 0002:00012500       $unwind$?dtor$15@?0??ProcessKey@Plist@@QEAAHPEBU_INPUT_RECORD@@@Z@4HA 0000000180058500     Pclass.obj
 0002:00012500       $unwind$?dtor$16@?0??ProcessKey@Plist@@QEAAHPEBU_INPUT_RECORD@@@Z@4HA 0000000180058500     Pclass.obj
 0002:00012508       $unwind$?DurationToText@@YA?AV?$basic_string@_WU?$char_traits@_W@std@@V?$allocator@_W@2@@std@@_K@Z 0000000180058508     Pclass.obj
 0002:00012520       $unwind$?GetVersionInfo@Plist@@SA_NPEB_WAEAV?$unique_ptr@$$BY0A@DU?$default_delete@$$BY0A@D@std@@@std@@AEAPEB_W2@Z 0000000180058520     Pclass.obj
 0002:0001253c       $stateUnwindMap$?GetVersionInfo@Plist@@SA_NPEB_WAEAV?$unique_ptr@$$BY0A@DU?$default_delete@$$BY0A@D@std@@@std@@AEAPEB_W2@Z 000000018005853c     Pclass.obj
 0002:00012580       $ip2state$?GetVersionInfo@Plist@@SA_NPEB_WAEAV?$unique_ptr@$$BY0A@DU?$default_delete@$$BY0A@D@std@@@std@@AEAPEB_W2@Z 0000000180058580     Pclass.obj
 0002:000125c0       $unwind$?PrintVersionInfo@Plist@@CAXPEAXPEB_W@Z 00000001800585c0     Pclass.obj
 0002:000125e0       $stateUnwindMap$?PrintVersionInfo@Plist@@CAXPEAXPEB_W@Z 00000001800585e0     Pclass.obj
 0002:00012610       $ip2state$?PrintVersionInfo@Plist@@CAXPEAXPEB_W@Z 0000000180058610     Pclass.obj
 0002:00012658       $unwind$?ConnectWMI@Plist@@AEAA_NXZ 0000000180058658     Pclass.obj
 0002:00012670       $unwind$?PrintOwnerInfo@Plist@@AEAAXPEAXK@Z 0000000180058670     Pclass.obj
 0002:00012690       $stateUnwindMap$?PrintOwnerInfo@Plist@@AEAAXPEAXK@Z 0000000180058690     Pclass.obj
 0002:000126d0       $ip2state$?PrintOwnerInfo@Plist@@AEAAXPEAXK@Z 00000001800586d0     Pclass.obj
 0002:00012720       $unwind$?Compare@Plist@@QEBAHPEBUPluginPanelItem@@0I@Z 0000000180058720     Pclass.obj
 0002:00012738       $stateUnwindMap$?Compare@Plist@@QEBAHPEBUPluginPanelItem@@0I@Z 0000000180058738     Pclass.obj
 0002:00012750       $ip2state$?Compare@Plist@@QEBAHPEBUPluginPanelItem@@0I@Z 0000000180058750     Pclass.obj
 0002:00012778       $unwind$??1?$vector@V?$basic_string@_WU?$char_traits@_W@std@@V?$allocator@_W@2@@std@@V?$allocator@V?$basic_string@_WU?$char_traits@_W@std@@V?$allocator@_W@2@@std@@@2@@std@@QEAA@XZ 0000000180058778     Pclass.obj
 0002:00012778       $unwind$?_Tidy@?$vector@V?$basic_string@_WU?$char_traits@_W@std@@V?$allocator@_W@2@@std@@V?$allocator@V?$basic_string@_WU?$char_traits@_W@std@@V?$allocator@_W@2@@std@@@2@@std@@AEAAXXZ 0000000180058778     Pclass.obj
 0002:00012784       $unwind$?push_back@?$basic_string@_WU?$char_traits@_W@std@@V?$allocator@_W@2@@std@@QEAAX_W@Z 0000000180058784     Pclass.obj
 0002:00012798       $unwind$?_Reallocate_exactly@?$vector@_KV?$allocator@_K@std@@@std@@AEAAX_K@Z 0000000180058798     Pclass.obj
 0002:000127a8       $unwind$?_Reallocate_exactly@?$vector@UFarMenuItem@@V?$allocator@UFarMenuItem@@@std@@@std@@AEAAX_K@Z 00000001800587a8     Pclass.obj
 0002:000127b8       $unwind$?_Reallocate_exactly@?$vector@V?$basic_string@_WU?$char_traits@_W@std@@V?$allocator@_W@2@@std@@V?$allocator@V?$basic_string@_WU?$char_traits@_W@std@@V?$allocator@_W@2@@std@@@2@@std@@AEAAX_K@Z 00000001800587b8     Pclass.obj
 0002:000127d0       $stateUnwindMap$?_Reallocate_exactly@?$vector@V?$basic_string@_WU?$char_traits@_W@std@@V?$allocator@_W@2@@std@@V?$allocator@V?$basic_string@_WU?$char_traits@_W@std@@V?$allocator@_W@2@@std@@@2@@std@@AEAAX_K@Z 00000001800587d0     Pclass.obj
 0002:00012800       $ip2state$?_Reallocate_exactly@?$vector@V?$basic_string@_WU?$char_traits@_W@std@@V?$allocator@_W@2@@std@@V?$allocator@V?$basic_string@_WU?$char_traits@_W@std@@V?$allocator@_W@2@@std@@@2@@std@@AEAAX_K@Z 0000000180058800     Pclass.obj
 0002:00012808       $unwind$??R?$default_delete@VWMIConnection@@@std@@QEBAXPEAVWMIConnection@@@Z 0000000180058808     Pclass.obj
 0002:00012820       $ip2state$??R?$default_delete@VWMIConnection@@@std@@QEBAXPEAVWMIConnection@@@Z 0000000180058820     Pclass.obj
 0002:00012830       $unwind$?insert@?$basic_string@_WU?$char_traits@_W@std@@V?$allocator@_W@2@@std@@QEAAAEAV12@_KQEB_W0@Z 0000000180058830     Pclass.obj
 0002:00012844       $unwind$?_Change_array@?$vector@V?$basic_string@_WU?$char_traits@_W@std@@V?$allocator@_W@2@@std@@V?$allocator@V?$basic_string@_WU?$char_traits@_W@std@@V?$allocator@_W@2@@std@@@2@@std@@AEAAXQEAV?$basic_string@_WU?$char_traits@_W@std@@V?$allocator@_W@2@@2@_K1@Z 0000000180058844     Pclass.obj
 0002:00012854       $unwind$?_Assign_grow@?$_Hash_vec@V?$allocator@V?$_List_unchecked_iterator@V?$_List_val@U?$_List_simple_types@U?$pair@$$CBKPEAUHWND__@@@std@@@std@@@std@@@std@@@std@@@std@@QEAAX_KV?$_List_unchecked_iterator@V?$_List_val@U?$_List_simple_types@U?$pair@$$CBKPEAUHWND__@@@std@@@std@@@std@@@2@@Z 0000000180058854     Pclass.obj
 0002:00012854       $unwind$?_Assign_grow@?$_Hash_vec@V?$allocator@V?$_List_unchecked_iterator@V?$_List_val@U?$_List_simple_types@U?$pair@$$CBKUProcessPerfData@@@std@@@std@@@std@@@std@@@std@@@std@@QEAAX_KV?$_List_unchecked_iterator@V?$_List_val@U?$_List_simple_types@U?$pair@$$CBKUProcessPerfData@@@std@@@std@@@std@@@2@@Z 0000000180058854     perfthread.obj
 0002:00012868       $unwind$??$_Emplace_reallocate@V?$basic_string@_WU?$char_traits@_W@std@@V?$allocator@_W@2@@std@@@?$vector@V?$basic_string@_WU?$char_traits@_W@std@@V?$allocator@_W@2@@std@@V?$allocator@V?$basic_string@_WU?$char_traits@_W@std@@V?$allocator@_W@2@@std@@@2@@std@@QEAAPEAV?$basic_string@_WU?$char_traits@_W@std@@V?$allocator@_W@2@@1@QEAV21@$$QEAV21@@Z 0000000180058868     Pclass.obj
 0002:00012884       $stateUnwindMap$??$_Emplace_reallocate@V?$basic_string@_WU?$char_traits@_W@std@@V?$allocator@_W@2@@std@@@?$vector@V?$basic_string@_WU?$char_traits@_W@std@@V?$allocator@_W@2@@std@@V?$allocator@V?$basic_string@_WU?$char_traits@_W@std@@V?$allocator@_W@2@@std@@@2@@std@@QEAAPEAV?$basic_string@_WU?$char_traits@_W@std@@V?$allocator@_W@2@@1@QEAV21@$$QEAV21@@Z 0000000180058884     Pclass.obj
 0002:000128f0       $ip2state$??$_Emplace_reallocate@V?$basic_string@_WU?$char_traits@_W@std@@V?$allocator@_W@2@@std@@@?$vector@V?$basic_string@_WU?$char_traits@_W@std@@V?$allocator@_W@2@@std@@V?$allocator@V?$basic_string@_WU?$char_traits@_W@std@@V?$allocator@_W@2@@std@@@2@@std@@QEAAPEAV?$basic_string@_WU?$char_traits@_W@std@@V?$allocator@_W@2@@1@QEAV21@$$QEAV21@@Z 00000001800588f0     Pclass.obj
 0002:00012908       $unwind$??$format@AEAV?$basic_string@_WU?$char_traits@_W@std@@V?$allocator@_W@2@@std@@AEAK@v8@fmt@@YA?AV?$basic_string@_WU?$char_traits@_W@std@@V?$allocator@_W@2@@std@@V?$basic_format_string@_WAEAV?$basic_string@_WU?$char_traits@_W@std@@V?$allocator@_W@2@@std@@AEAK@01@AEAV23@AEAK@Z 0000000180058908     Pclass.obj
 0002:0001291c       $unwind$??$_Emplace_reallocate@AEB_K@?$vector@_KV?$allocator@_K@std@@@std@@QEAAPEA_KQEA_KAEB_K@Z 000000018005891c     Pclass.obj
 0002:0001291c       $unwind$??$_Emplace_reallocate@_K@?$vector@_KV?$allocator@_K@std@@@std@@QEAAPEA_KQEA_K$$QEA_K@Z 000000018005891c     Pclass.obj
 0002:0001292c       $unwind$??$_Emplace_reallocate@UFarMenuItem@@@?$vector@UFarMenuItem@@V?$allocator@UFarMenuItem@@@std@@@std@@QEAAPEAUFarMenuItem@@QEAU2@$$QEAU2@@Z 000000018005892c     Pclass.obj
 0002:00012940       $unwind$??$_Try_emplace@AEBK$$V@?$_Hash@V?$_Umap_traits@KPEAUHWND__@@V?$_Uhash_compare@KU?$hash@K@std@@U?$equal_to@K@2@@std@@V?$allocator@U?$pair@$$CBKPEAUHWND__@@@std@@@3@$0A@@std@@@std@@IEAA?AU?$pair@PEAU?$_List_node@U?$pair@$$CBKPEAUHWND__@@@std@@PEAX@std@@_N@1@AEBK@Z 0000000180058940     Pclass.obj
 0002:0001295c       $stateUnwindMap$??$_Try_emplace@AEBK$$V@?$_Hash@V?$_Umap_traits@KPEAUHWND__@@V?$_Uhash_compare@KU?$hash@K@std@@U?$equal_to@K@2@@std@@V?$allocator@U?$pair@$$CBKPEAUHWND__@@@std@@@3@$0A@@std@@@std@@IEAA?AU?$pair@PEAU?$_List_node@U?$pair@$$CBKPEAUHWND__@@@std@@PEAX@std@@_N@1@AEBK@Z 000000018005895c     Pclass.obj
 0002:00012970       $ip2state$??$_Try_emplace@AEBK$$V@?$_Hash@V?$_Umap_traits@KPEAUHWND__@@V?$_Uhash_compare@KU?$hash@K@std@@U?$equal_to@K@2@@std@@V?$allocator@U?$pair@$$CBKPEAUHWND__@@@std@@@3@$0A@@std@@@std@@IEAA?AU?$pair@PEAU?$_List_node@U?$pair@$$CBKPEAUHWND__@@@std@@PEAX@std@@_N@1@AEBK@Z 0000000180058970     Pclass.obj
 0002:00012988       $unwind$??$_Assign_range@PEBUmode@@@?$vector@Umode@@V?$allocator@Umode@@@std@@@std@@AEAAXPEBUmode@@0Uforward_iterator_tag@1@@Z 0000000180058988     Pclass.obj
 0002:0001299c       $unwind$??$_Reallocate_grow_by@V<lambda_1>@?1??insert@?$basic_string@_WU?$char_traits@_W@std@@V?$allocator@_W@2@@std@@QEAAAEAV34@_K0_W@Z@_K_K_W@?$basic_string@_WU?$char_traits@_W@std@@V?$allocator@_W@2@@std@@AEAAAEAV01@_KV<lambda_1>@?1??insert@01@QEAAAEAV01@00_W@Z@_K3_W@Z 000000018005899c     Pclass.obj
 0002:000129b0       $unwind$??$_Reallocate_grow_by@V<lambda_1>@?1??append@?$basic_string@_WU?$char_traits@_W@std@@V?$allocator@_W@2@@std@@QEAAAEAV34@_K_W@Z@_K_W@?$basic_string@_WU?$char_traits@_W@std@@V?$allocator@_W@2@@std@@AEAAAEAV01@_KV<lambda_1>@?1??append@01@QEAAAEAV01@0_W@Z@_K_W@Z 00000001800589b0     Pclass.obj
 0002:000129c4       $unwind$?_Umove@?$vector@V?$basic_string@_WU?$char_traits@_W@std@@V?$allocator@_W@2@@std@@V?$allocator@V?$basic_string@_WU?$char_traits@_W@std@@V?$allocator@_W@2@@std@@@2@@std@@AEAAPEAV?$basic_string@_WU?$char_traits@_W@std@@V?$allocator@_W@2@@2@PEAV32@00@Z 00000001800589c4     Pclass.obj
 0002:000129d4       $stateUnwindMap$?_Umove@?$vector@V?$basic_string@_WU?$char_traits@_W@std@@V?$allocator@_W@2@@std@@V?$allocator@V?$basic_string@_WU?$char_traits@_W@std@@V?$allocator@_W@2@@std@@@2@@std@@AEAAPEAV?$basic_string@_WU?$char_traits@_W@std@@V?$allocator@_W@2@@2@PEAV32@00@Z 00000001800589d4     Pclass.obj
 0002:000129f4       $unwind$?_Forced_rehash@?$_Hash@V?$_Umap_traits@KPEAUHWND__@@V?$_Uhash_compare@KU?$hash@K@std@@U?$equal_to@K@2@@std@@V?$allocator@U?$pair@$$CBKPEAUHWND__@@@std@@@3@$0A@@std@@@std@@IEAAX_K@Z 00000001800589f4     Pclass.obj
 0002:000129f4       $unwind$?_Forced_rehash@?$_Hash@V?$_Umap_traits@KUProcessPerfData@@V?$_Uhash_compare@KU?$hash@K@std@@U?$equal_to@K@2@@std@@V?$allocator@U?$pair@$$CBKUProcessPerfData@@@std@@@3@$00@std@@@std@@IEAAX_K@Z 00000001800589f4     perfthread.obj
 0002:00012a00       $unwind$??$_Resize_reallocate@U_Value_init_tag@std@@@?$vector@PEB_WV?$allocator@PEB_W@std@@@std@@AEAAX_KAEBU_Value_init_tag@1@@Z 0000000180058a00     Pclass.obj
 0002:00012a00       $unwind$??$_Resize_reallocate@U_Value_init_tag@std@@@?$vector@PEAUHINSTANCE__@@V?$allocator@PEAUHINSTANCE__@@@std@@@std@@AEAAX_KAEBU_Value_init_tag@1@@Z 0000000180058a00     Plist.obj
 0002:00012a10       $unwind$??$_Uninitialized_copy@PEBUmode@@V?$allocator@Umode@@@std@@@std@@YAPEAUmode@@QEBU1@0PEAU1@AEAV?$allocator@Umode@@@0@@Z 0000000180058a10     Pclass.obj
 0002:00012a2c       $stateUnwindMap$??$_Uninitialized_copy@PEBUmode@@V?$allocator@Umode@@@std@@@std@@YAPEAUmode@@QEBU1@0PEAU1@AEAV?$allocator@Umode@@@0@@Z 0000000180058a2c     Pclass.obj
 0002:00012a90       $ip2state$??$_Uninitialized_copy@PEBUmode@@V?$allocator@Umode@@@std@@@std@@YAPEAUmode@@QEBU1@0PEAU1@AEAV?$allocator@Umode@@@0@@Z 0000000180058a90     Pclass.obj
 0002:00012ad8       $unwind$??0PerfThread@@QEAA@PEAVPlist@@PEB_W11@Z 0000000180058ad8     perfthread.obj
 0002:00012afc       $stateUnwindMap$??0PerfThread@@QEAA@PEAVPlist@@PEB_W11@Z 0000000180058afc     perfthread.obj
 0002:00012ba0       $ip2state$??0PerfThread@@QEAA@PEAVPlist@@PEB_W11@Z 0000000180058ba0     perfthread.obj
 0002:00012bf0       $unwind$??1PerfThread@@QEAA@XZ 0000000180058bf0     perfthread.obj
 0002:00012c10       $ip2state$??1PerfThread@@QEAA@XZ 0000000180058c10     perfthread.obj
 0002:00012c28       $unwind$?GetProcessData@PerfThread@@QEAAPEAUProcessPerfData@@KK@Z 0000000180058c28     perfthread.obj
 0002:00012c40       $unwind$?Refresh@PerfThread@@AEAAXXZ 0000000180058c40     perfthread.obj
 0002:00012c64       $stateUnwindMap$?Refresh@PerfThread@@AEAAXXZ 0000000180058c64     perfthread.obj
 0002:00012cb0       $ip2state$?Refresh@PerfThread@@AEAAXXZ 0000000180058cb0     perfthread.obj
 0002:00012d38       $unwind$??1ProcessPerfData@@QEAA@XZ 0000000180058d38     perfthread.obj
 0002:00012d44       $unwind$?RefreshWMIData@PerfThread@@AEAAXXZ 0000000180058d44     perfthread.obj
 0002:00012d68       $stateUnwindMap$?RefreshWMIData@PerfThread@@AEAAXXZ 0000000180058d68     perfthread.obj
 0002:00012de0       $ip2state$?RefreshWMIData@PerfThread@@AEAAXXZ 0000000180058de0     perfthread.obj
 0002:00012e60       $unwind$??0?$unordered_multimap@KUProcessPerfData@@U?$hash@K@std@@U?$equal_to@K@3@V?$allocator@U?$pair@$$CBKUProcessPerfData@@@std@@@3@@std@@QEAA@XZ 0000000180058e60     perfthread.obj
 0002:00012e74       $stateUnwindMap$??0?$unordered_multimap@KUProcessPerfData@@U?$hash@K@std@@U?$equal_to@K@3@V?$allocator@U?$pair@$$CBKUProcessPerfData@@@std@@@3@@std@@QEAA@XZ 0000000180058e74     perfthread.obj
 0002:00012e90       $ip2state$??0?$unordered_multimap@KUProcessPerfData@@U?$hash@K@std@@U?$equal_to@K@3@V?$allocator@U?$pair@$$CBKUProcessPerfData@@@std@@@3@@std@@QEAA@XZ 0000000180058e90     perfthread.obj
 0002:00012ea0       $unwind$?_Reallocate_exactly@?$vector@UProcessPerfData@@V?$allocator@UProcessPerfData@@@std@@@std@@AEAAX_K@Z 0000000180058ea0     perfthread.obj
 0002:00012eb0       $unwind$?_Unchecked_erase@?$_Hash@V?$_Umap_traits@KUProcessPerfData@@V?$_Uhash_compare@KU?$hash@K@std@@U?$equal_to@K@2@@std@@V?$allocator@U?$pair@$$CBKUProcessPerfData@@@std@@@3@$00@std@@@std@@AEAAPEAU?$_List_node@U?$pair@$$CBKUProcessPerfData@@@std@@PEAX@2@PEAU32@QEAU32@@Z 0000000180058eb0     perfthread.obj
 0002:00012ec4       $unwind$??$emplace@AEBKUProcessPerfData@@@?$_Hash@V?$_Umap_traits@KUProcessPerfData@@V?$_Uhash_compare@KU?$hash@K@std@@U?$equal_to@K@2@@std@@V?$allocator@U?$pair@$$CBKUProcessPerfData@@@std@@@3@$00@std@@@std@@QEAA?AV?$_List_iterator@V?$_List_val@U?$_List_simple_types@U?$pair@$$CBKUProcessPerfData@@@std@@@std@@@std@@@1@AEBK$$QEAUProcessPerfData@@@Z 0000000180058ec4     perfthread.obj
 0002:00012edc       $stateUnwindMap$??$insert@V?$_List_unchecked_const_iterator@V?$_List_val@U?$_List_simple_types@U?$pair@$$CBKUProcessPerfData@@@std@@@std@@@std@@U_Iterator_base0@2@@std@@@?$_Hash@V?$_Umap_traits@KUProcessPerfData@@V?$_Uhash_compare@KU?$hash@K@std@@U?$equal_to@K@2@@std@@V?$allocator@U?$pair@$$CBKUProcessPerfData@@@std@@@3@$00@std@@@std@@QEAAXV?$_List_unchecked_const_iterator@V?$_List_val@U?$_List_simple_types@U?$pair@$$CBKUProcessPerfData@@@std@@@std@@@std@@U_Iterator_base0@2@@1@0@Z 0000000180058edc     Plist.obj
 0002:00012edc       $stateUnwindMap$??$emplace@AEBKUProcessPerfData@@@?$_Hash@V?$_Umap_traits@KUProcessPerfData@@V?$_Uhash_compare@KU?$hash@K@std@@U?$equal_to@K@2@@std@@V?$allocator@U?$pair@$$CBKUProcessPerfData@@@std@@@3@$00@std@@@std@@QEAA?AV?$_List_iterator@V?$_List_val@U?$_List_simple_types@U?$pair@$$CBKUProcessPerfData@@@std@@@std@@@std@@@1@AEBK$$QEAUProcessPerfData@@@Z 0000000180058edc     perfthread.obj
 0002:00012ef0       $ip2state$??$emplace@AEBKUProcessPerfData@@@?$_Hash@V?$_Umap_traits@KUProcessPerfData@@V?$_Uhash_compare@KU?$hash@K@std@@U?$equal_to@K@2@@std@@V?$allocator@U?$pair@$$CBKUProcessPerfData@@@std@@@3@$00@std@@@std@@QEAA?AV?$_List_iterator@V?$_List_val@U?$_List_simple_types@U?$pair@$$CBKUProcessPerfData@@@std@@@std@@@std@@@1@AEBK$$QEAUProcessPerfData@@@Z 0000000180058ef0     perfthread.obj
 0002:00012f08       $unwind$??$transform@V?$_List_const_iterator@V?$_List_val@U?$_List_simple_types@U?$pair@$$CBKUProcessPerfData@@@std@@@std@@@std@@@std@@V?$back_insert_iterator@V?$vector@UProcessPerfData@@V?$allocator@UProcessPerfData@@@std@@@std@@@2@V<lambda_1>@?2??RefreshWMIData@PerfThread@@AEAAXXZ@@std@@YA?AV?$back_insert_iterator@V?$vector@UProcessPerfData@@V?$allocator@UProcessPerfData@@@std@@@std@@@0@V?$_List_const_iterator@V?$_List_val@U?$_List_simple_types@U?$pair@$$CBKUProcessPerfData@@@std@@@std@@@std@@@0@0V10@V<lambda_1>@?2??RefreshWMIData@PerfThread@@AEAAXXZ@@Z 0000000180058f08     perfthread.obj
 0002:00012f2c       $stateUnwindMap$??$transform@V?$_List_const_iterator@V?$_List_val@U?$_List_simple_types@U?$pair@$$CBKUProcessPerfData@@@std@@@std@@@std@@@std@@V?$back_insert_iterator@V?$vector@UProcessPerfData@@V?$allocator@UProcessPerfData@@@std@@@std@@@2@V<lambda_1>@?2??RefreshWMIData@PerfThread@@AEAAXXZ@@std@@YA?AV?$back_insert_iterator@V?$vector@UProcessPerfData@@V?$allocator@UProcessPerfData@@@std@@@std@@@0@V?$_List_const_iterator@V?$_List_val@U?$_List_simple_types@U?$pair@$$CBKUProcessPerfData@@@std@@@std@@@std@@@0@0V10@V<lambda_1>@?2??RefreshWMIData@PerfThread@@AEAAXXZ@@Z 0000000180058f2c     perfthread.obj
 0002:00012f50       $ip2state$??$transform@V?$_List_const_iterator@V?$_List_val@U?$_List_simple_types@U?$pair@$$CBKUProcessPerfData@@@std@@@std@@@std@@@std@@V?$back_insert_iterator@V?$vector@UProcessPerfData@@V?$allocator@UProcessPerfData@@@std@@@std@@@2@V<lambda_1>@?2??RefreshWMIData@PerfThread@@AEAAXXZ@@std@@YA?AV?$back_insert_iterator@V?$vector@UProcessPerfData@@V?$allocator@UProcessPerfData@@@std@@@std@@@0@V?$_List_const_iterator@V?$_List_val@U?$_List_simple_types@U?$pair@$$CBKUProcessPerfData@@@std@@@std@@@std@@@0@0V10@V<lambda_1>@?2??RefreshWMIData@PerfThread@@AEAAXXZ@@Z 0000000180058f50     perfthread.obj
 0002:00012f98       $unwind$??0ProcessPerfData@@QEAA@AEBU0@@Z 0000000180058f98     perfthread.obj
 0002:00012fa8       $stateUnwindMap$??0ProcessPerfData@@QEAA@AEBU0@@Z 0000000180058fa8     perfthread.obj
 0002:00012fc0       $ip2state$??0ProcessPerfData@@QEAA@AEBU0@@Z 0000000180058fc0     perfthread.obj
 0002:00012fe0       $unwind$??$_Free_non_head@V?$allocator@U?$_List_node@U?$pair@$$CBKUProcessPerfData@@@std@@PEAX@std@@@std@@@?$_List_node@U?$pair@$$CBKUProcessPerfData@@@std@@PEAX@std@@SAXAEAV?$allocator@U?$_List_node@U?$pair@$$CBKUProcessPerfData@@@std@@PEAX@std@@@1@PEAU01@@Z 0000000180058fe0     perfthread.obj
 0002:00012fec       $unwind$??$_Destroy_range@V?$allocator@UProcessPerfData@@@std@@@std@@YAXPEAUProcessPerfData@@QEAU1@AEAV?$allocator@UProcessPerfData@@@0@@Z 0000000180058fec     perfthread.obj
 0002:00012ff8       $unwind$??$_Resize_reallocate@U_Value_init_tag@std@@@?$vector@EV?$allocator@E@std@@@std@@AEAAX_KAEBU_Value_init_tag@1@@Z 0000000180058ff8     perfthread.obj
 0002:00013008       $unwind$??$_Emplace_reallocate@UProcessPerfData@@@?$vector@UProcessPerfData@@V?$allocator@UProcessPerfData@@@std@@@std@@QEAAPEAUProcessPerfData@@QEAU2@$$QEAU2@@Z 0000000180059008     perfthread.obj
 0002:0001301c       $unwind$??0ProcessPerfData@@QEAA@$$QEAU0@@Z 000000018005901c     perfthread.obj
 0002:0001302c       $stateUnwindMap$?GetOpenProcessData@?$ipc_functions@$0A@@@SAXPEAXPEAV?$basic_string@_WU?$char_traits@_W@std@@V?$allocator@_W@2@@std@@1111@Z 000000018005902c     Plist.obj
 0002:0001302c       $stateUnwindMap$??0ProcessPerfData@@QEAA@$$QEAU0@@Z 000000018005902c     perfthread.obj
 0002:00013054       $unwind$?GetPData@@YA_NAEAUProcessData@@AEBUProcessPerfData@@@Z 0000000180059054     Plist.obj
 0002:00013060       $unwind$?FreeUserData@@YAXQEAXQEBUFarPanelItemFreeInfo@@@Z 0000000180059060     Plist.obj
 0002:0001306c       $unwind$?GetList@@YA_NAEAPEAUPluginPanelItem@@AEA_KAEAVPerfThread@@@Z 000000018005906c     Plist.obj
 0002:00013088       $stateUnwindMap$?GetList@@YA_NAEAPEAUPluginPanelItem@@AEA_KAEAVPerfThread@@@Z 0000000180059088     Plist.obj
 0002:000130b0       $ip2state$?GetList@@YA_NAEAPEAUPluginPanelItem@@AEA_KAEAVPerfThread@@@Z 00000001800590b0     Plist.obj
 0002:000130f0       $unwind$?Enable@DebugToken@@QEAA_NXZ 00000001800590f0     Plist.obj
 0002:00013104       $unwind$?KillProcess@@YA_NKPEAUHWND__@@@Z 0000000180059104     Plist.obj
 0002:00013120       $stateUnwindMap$?KillProcess@@YA_NKPEAUHWND__@@@Z 0000000180059120     Plist.obj
 0002:00013130       $ip2state$?KillProcess@@YA_NKPEAUHWND__@@@Z 0000000180059130     Plist.obj
 0002:00013150       $unwind$?PrintNTCurDirAndEnv@@YAXPEAX0H@Z 0000000180059150     Plist.obj
 0002:00013170       $stateUnwindMap$?PrintNTCurDirAndEnv@@YAXPEAX0H@Z 0000000180059170     Plist.obj
 0002:00013190       $ip2state$?PrintNTCurDirAndEnv@@YAXPEAX0H@Z 0000000180059190     Plist.obj
 0002:000131a0       $unwind$?print_module_impl@@YAXQEAXAEBV?$basic_string@_WU?$char_traits@_W@std@@V?$allocator@_W@2@@std@@KAEBUoptions@@AEBV?$function@$$A6A_NPEA_W_K@Z@2@@Z 00000001800591a0     Plist.obj
 0002:000131c0       $stateUnwindMap$?print_module_impl@@YAXQEAXAEBV?$basic_string@_WU?$char_traits@_W@std@@V?$allocator@_W@2@@std@@KAEBUoptions@@AEBV?$function@$$A6A_NPEA_W_K@Z@2@@Z 00000001800591c0     Plist.obj
 0002:000131d0       $ip2state$?print_module_impl@@YAXQEAXAEBV?$basic_string@_WU?$char_traits@_W@std@@V?$allocator@_W@2@@std@@KAEBUoptions@@AEBV?$function@$$A6A_NPEA_W_K@Z@2@@Z 00000001800591d0     Plist.obj
 0002:000131e8       $unwind$?PrintModules@@YAXPEAXKAEAUoptions@@@Z 00000001800591e8     Plist.obj
 0002:00013208       $stateUnwindMap$?PrintModules@@YAXPEAXKAEAUoptions@@@Z 0000000180059208     Plist.obj
 0002:00013230       $ip2state$?PrintModules@@YAXPEAXKAEAUoptions@@@Z 0000000180059230     Plist.obj
 0002:00013280       $unwind$?PrintModules@?$ipc_functions@$0A@@@SAXPEAX0AEAUoptions@@@Z 0000000180059280     Plist.obj
 0002:000132a0       $stateUnwindMap$?PrintModules@?$ipc_functions@$0A@@@SAXPEAX0AEAUoptions@@@Z 00000001800592a0     Plist.obj
 0002:000132d0       $ip2state$?PrintModules@?$ipc_functions@$0A@@@SAXPEAX0AEAUoptions@@@Z 00000001800592d0     Plist.obj
 0002:000132f8       $unwind$?GetOpenProcessData@?$ipc_functions@$0A@@@SAXPEAXPEAV?$basic_string@_WU?$char_traits@_W@std@@V?$allocator@_W@2@@std@@1111@Z 00000001800592f8     Plist.obj
 0002:00013320       $ip2state$?GetOpenProcessData@?$ipc_functions@$0A@@@SAXPEAXPEAV?$basic_string@_WU?$char_traits@_W@std@@V?$allocator@_W@2@@std@@1111@Z 0000000180059320     Plist.obj
 0002:00013358       $unwind$?read_string@?$ipc_functions@$0A@@@SA?AV?$basic_string@_WU?$char_traits@_W@std@@V?$allocator@_W@2@@std@@PEAXAEBUUNICODE_STRING_SAME@detail@@@Z 0000000180059358     Plist.obj
 0002:00013374       $stateUnwindMap$?read_string@?$ipc_functions@$0A@@@SA?AV?$basic_string@_WU?$char_traits@_W@std@@V?$allocator@_W@2@@std@@PEAXAEBUUNICODE_STRING_SAME@detail@@@Z 0000000180059374     Plist.obj
 0002:00013390       $ip2state$?read_string@?$ipc_functions@$0A@@@SA?AV?$basic_string@_WU?$char_traits@_W@std@@V?$allocator@_W@2@@std@@PEAXAEBUUNICODE_STRING_SAME@detail@@@Z 0000000180059390     Plist.obj
 0002:000133a0       $unwind$?resize@?$basic_string@_WU?$char_traits@_W@std@@V?$allocator@_W@2@@std@@QEAAX_K_W@Z 00000001800593a0     Plist.obj
 0002:000133b4       $unwind$??$print_module@PEAX@@YAXQEAXPEAXKAEAUoptions@@AEBV?$function@$$A6A_NPEA_W_K@Z@std@@@Z 00000001800593b4     Plist.obj
 0002:000133d0       $stateUnwindMap$??$print_module@PEAX@@YAXQEAXPEAXKAEAUoptions@@AEBV?$function@$$A6A_NPEA_W_K@Z@std@@@Z 00000001800593d0     Plist.obj
 0002:000133f0       $ip2state$??$print_module@PEAX@@YAXQEAXPEAXKAEAUoptions@@AEBV?$function@$$A6A_NPEA_W_K@Z@std@@@Z 00000001800593f0     Plist.obj
 0002:00013400       $unwind$??$insert@V?$_List_unchecked_const_iterator@V?$_List_val@U?$_List_simple_types@U?$pair@$$CBKUProcessPerfData@@@std@@@std@@@std@@U_Iterator_base0@2@@std@@@?$_Hash@V?$_Umap_traits@KUProcessPerfData@@V?$_Uhash_compare@KU?$hash@K@std@@U?$equal_to@K@2@@std@@V?$allocator@U?$pair@$$CBKUProcessPerfData@@@std@@@3@$00@std@@@std@@QEAAXV?$_List_unchecked_const_iterator@V?$_List_val@U?$_List_simple_types@U?$pair@$$CBKUProcessPerfData@@@std@@@std@@@std@@U_Iterator_base0@2@@1@0@Z 0000000180059400     Plist.obj
 0002:00013420       $ip2state$??$insert@V?$_List_unchecked_const_iterator@V?$_List_val@U?$_List_simple_types@U?$pair@$$CBKUProcessPerfData@@@std@@@std@@@std@@U_Iterator_base0@2@@std@@@?$_Hash@V?$_Umap_traits@KUProcessPerfData@@V?$_Uhash_compare@KU?$hash@K@std@@U?$equal_to@K@2@@std@@V?$allocator@U?$pair@$$CBKUProcessPerfData@@@std@@@3@$00@std@@@std@@QEAAXV?$_List_unchecked_const_iterator@V?$_List_val@U?$_List_simple_types@U?$pair@$$CBKUProcessPerfData@@@std@@@std@@@std@@U_Iterator_base0@2@@1@0@Z 0000000180059420     Plist.obj
 0002:00013440       $unwind$?WinError@@YAHPEB_W@Z 0000000180059440     Pmix.obj
 0002:0001345c       $stateUnwindMap$?WinError@@YAHPEB_W@Z 000000018005945c     Pmix.obj
 0002:00013490       $ip2state$?WinError@@YAHPEB_W@Z 0000000180059490     Pmix.obj
 0002:000134c0       $unwind$?find_last_not_of@?$basic_string@_WU?$char_traits@_W@std@@V?$allocator@_W@2@@std@@QEBA_KQEB_W_K@Z 00000001800594c0     Pmix.obj
 0002:000134e0       $unwind$??1WMIConnection@@QEAA@XZ 00000001800594e0     wmi.obj
 0002:000134f8       $ip2state$??1WMIConnection@@QEAA@XZ 00000001800594f8     wmi.obj
 0002:00013500       $unwind$?GetProcessOwner@WMIConnection@@QEAA?AV?$basic_string@_WU?$char_traits@_W@std@@V?$allocator@_W@2@@std@@KPEAV23@@Z 0000000180059500     wmi.obj
 0002:00013520       $stateUnwindMap$?GetProcessOwner@WMIConnection@@QEAA?AV?$basic_string@_WU?$char_traits@_W@std@@V?$allocator@_W@2@@std@@KPEAV23@@Z 0000000180059520     wmi.obj
 0002:00013570       $ip2state$?GetProcessOwner@WMIConnection@@QEAA?AV?$basic_string@_WU?$char_traits@_W@std@@V?$allocator@_W@2@@std@@KPEAV23@@Z 0000000180059570     wmi.obj
 0002:000135c0       $unwind$?GetProcessUserSid@WMIConnection@@QEAA?AV?$basic_string@_WU?$char_traits@_W@std@@V?$allocator@_W@2@@std@@K@Z 00000001800595c0     wmi.obj
 0002:000135dc       $stateUnwindMap$?GetProcessUserSid@WMIConnection@@QEAA?AV?$basic_string@_WU?$char_traits@_W@std@@V?$allocator@_W@2@@std@@K@Z 00000001800595dc     wmi.obj
 0002:00013630       $ip2state$?GetProcessUserSid@WMIConnection@@QEAA?AV?$basic_string@_WU?$char_traits@_W@std@@V?$allocator@_W@2@@std@@K@Z 0000000180059630     wmi.obj
 0002:00013680       $unwind$?GetProcessSessionId@WMIConnection@@QEAAKK@Z 0000000180059680     wmi.obj
 0002:00013698       $stateUnwindMap$?GetProcessSessionId@WMIConnection@@QEAAKK@Z 0000000180059698     wmi.obj
 0002:000136a0       $ip2state$?GetProcessSessionId@WMIConnection@@QEAAKK@Z 00000001800596a0     wmi.obj
 0002:000136a8       $unwind$?ExecMethod@WMIConnection@@AEAAHKPEB_W0K@Z 00000001800596a8     wmi.obj
 0002:000136c8       $stateUnwindMap$?ExecMethod@WMIConnection@@AEAAHKPEB_W0K@Z 00000001800596c8     wmi.obj
 0002:00013750       $ip2state$?ExecMethod@WMIConnection@@AEAAHKPEB_W0K@Z 0000000180059750     wmi.obj
 0002:00013800       $unwind$?GetProcessProperty@WMIConnection@@AEAA_NKPEB_WAEBV?$function@$$A6AXAEBUtagVARIANT@@@Z@std@@@Z 0000000180059800     wmi.obj
 0002:00013820       $stateUnwindMap$?GetProcessProperty@WMIConnection@@AEAA_NKPEB_WAEBV?$function@$$A6AXAEBUtagVARIANT@@@Z@std@@@Z 0000000180059820     wmi.obj
 0002:00013860       $ip2state$?GetProcessProperty@WMIConnection@@AEAA_NKPEB_WAEBV?$function@$$A6AXAEBUtagVARIANT@@@Z@std@@@Z 0000000180059860     wmi.obj
 0002:000138a0       $unwind$?Connect@WMIConnection@@QEAA_NPEB_W00@Z 00000001800598a0     wmi.obj
 0002:000138bc       $stateUnwindMap$?Connect@WMIConnection@@QEAA_NPEB_W00@Z 00000001800598bc     wmi.obj
 0002:00013900       $ip2state$?Connect@WMIConnection@@QEAA_NPEB_W00@Z 0000000180059900     wmi.obj
 0002:00013960       $unwind$?dtor$0@?0??Connect@WMIConnection@@QEAA_NPEB_W00@Z@4HA 0000000180059960     wmi.obj
 0002:00013960       $unwind$?dtor$2@?0??Connect@WMIConnection@@QEAA_NPEB_W00@Z@4HA 0000000180059960     wmi.obj
 0002:00013960       $unwind$?dtor$3@?0??Connect@WMIConnection@@QEAA_NPEB_W00@Z@4HA 0000000180059960     wmi.obj
 0002:00013960       $unwind$?dtor$4@?0??Connect@WMIConnection@@QEAA_NPEB_W00@Z@4HA 0000000180059960     wmi.obj
 0002:00013960       $unwind$?dtor$5@?0??Connect@WMIConnection@@QEAA_NPEB_W00@Z@4HA 0000000180059960     wmi.obj
 0002:00013968       $unwind$??1?$unique_ptr@UIWbemClassObject@@Ucom_closer@@@std@@QEAA@XZ 0000000180059968     wmi.obj
 0002:00013968       $unwind$??1?$unique_ptr@UIWbemLocator@@Ucom_closer@@@std@@QEAA@XZ 0000000180059968     wmi.obj
 0002:00013978       $ip2state$??1?$unique_ptr@UIWbemClassObject@@Ucom_closer@@@std@@QEAA@XZ 0000000180059978     wmi.obj
 0002:00013978       $ip2state$??1?$unique_ptr@UIWbemLocator@@Ucom_closer@@@std@@QEAA@XZ 0000000180059978     wmi.obj
 0002:00013980       $unwind$??1?$ptr_setter@V?$unique_ptr@UIWbemClassObject@@Ucom_closer@@@std@@@@QEAA@XZ 0000000180059980     wmi.obj
 0002:00013990       $ip2state$??1?$ptr_setter@V?$unique_ptr@UIWbemClassObject@@Ucom_closer@@@std@@@@QEAA@XZ 0000000180059990     wmi.obj
 0002:00013998       $unwind$SetStartupInfoW    0000000180059998     Proclist.obj
 0002:000139ac       $unwind$OpenW              00000001800599ac     Proclist.obj
 0002:000139bc       $unwind$FreeFindDataW      00000001800599bc     Proclist.obj
 0002:000139cc       $unwind$ProcessPanelEventW 00000001800599cc     Proclist.obj
 0002:000139f0       $ip2state$ProcessPanelEventW 00000001800599f0     Proclist.obj
 0002:00013a08       $unwind$?__scrt_throw_std_bad_alloc@@YAXXZ 0000000180059a08     LIBCMT:throw_bad_alloc.obj
 0002:00013a08       $unwind$?__scrt_throw_std_bad_array_new_length@@YAXXZ 0000000180059a08     LIBCMT:throw_bad_alloc.obj
 0002:00013a08       $unwind$?_Xbad_alloc@std@@YAXXZ 0000000180059a08     libcpmt:xthrow.obj
 0002:00013a08       $unwind$?_Xbad_function_call@std@@YAXXZ 0000000180059a08     libcpmt:xthrow.obj
 0002:00013a10       $unwind$?_Xlength_error@std@@YAXPEBD@Z 0000000180059a10     libcpmt:xthrow.obj
 0002:00013a10       $unwind$?_Xout_of_range@std@@YAXPEBD@Z 0000000180059a10     libcpmt:xthrow.obj
 0002:00013a10       $unwind$?_Xruntime_error@std@@YAXPEBD@Z 0000000180059a10     libcpmt:xthrow.obj
 0002:00013a18       $unwind$?_Init@locale@std@@CAPEAV_Locimp@12@_N@Z 0000000180059a18     libcpmt:locale0.obj
 0002:00013a2c       $stateUnwindMap$?_Init@locale@std@@CAPEAV_Locimp@12@_N@Z 0000000180059a2c     libcpmt:locale0.obj
 0002:00013a40       $ip2state$?_Init@locale@std@@CAPEAV_Locimp@12@_N@Z 0000000180059a40     libcpmt:locale0.obj
 0002:00013a50       $unwind$?_Atexit@@YAXP6AXXZ@Z 0000000180059a50     libcpmt:iosptrs.obj
 0002:00013a60       $unwind$??1_Init_atexit@@QEAA@XZ 0000000180059a60     libcpmt:iosptrs.obj
 0002:00013a78       $ip2state$??1_Init_atexit@@QEAA@XZ 0000000180059a78     libcpmt:iosptrs.obj
 0002:00013a80       __security_check_cookie_xdata 0000000180059a80     LIBCMT:arm64secgs.obj
 0002:00013a88       __security_check_cookie_xdata_prolog 0000000180059a88     LIBCMT:arm64secgs.obj
 0002:00013a89       __security_check_cookie_xdata_epilog1 0000000180059a89     LIBCMT:arm64secgs.obj
 0002:00013a8c       __gsfailure_xdata          0000000180059a8c     LIBCMT:arm64secgs.obj
 0002:00013a8c       __security_check_cookie_xdata_end 0000000180059a8c     LIBCMT:arm64secgs.obj
 0002:00013a90       __gsfailure_xdata_prolog   0000000180059a90     LIBCMT:arm64secgs.obj
 0002:00013a94       __gsfailure_xdata_end      0000000180059a94     LIBCMT:arm64secgs.obj
 0002:00013a94       $unwind$__scrt_is_nonwritable_in_current_image 0000000180059a94     LIBCMT:utility.obj
 0002:00013ab4       $unwind$__scrt_is_nonwritable_in_current_image$filt$0 0000000180059ab4     LIBCMT:utility.obj
 0002:00013ac0       $unwind$__scrt_acquire_startup_lock 0000000180059ac0     LIBCMT:utility.obj
 0002:00013acc       $unwind$__scrt_initialize_onexit_tables 0000000180059acc     LIBCMT:utility.obj
 0002:00013ad8       $unwind$??2@YAPEAX_K@Z     0000000180059ad8     LIBCMT:new_scalar.obj
 0002:00013ae8       $unwind$??_M@YAXPEAX_K1P6AX0@Z@Z 0000000180059ae8     LIBCMT:ehvecdtr.obj
 0002:00013b0c       $unwind$?fin$0@?0???_M@YAXPEAX_K1P6AX0@Z@Z@4HA 0000000180059b0c     LIBCMT:ehvecdtr.obj
 0002:00013b0c       $unwind$?fin$1@?0??FrameUnwindToState@__FrameHandler3@@SAXPEA_KPEAU_xDISPATCHER_CONTEXT@@PEBU_s_FuncInfo@@H@Z@4HA 0000000180059b0c     libvcruntime:frame.obj
 0002:00013b18       $unwind$?__ArrayUnwind@@YAXPEAX_K1P6AX0@Z@Z 0000000180059b18     LIBCMT:ehvecdtr.obj
 0002:00013b3c       $unwind$?filt$0@?0??__ArrayUnwind@@YAXPEAX_K1P6AX0@Z@Z@4HA 0000000180059b3c     LIBCMT:ehvecdtr.obj
 0002:00013b48       $unwind$?dllmain_crt_process_attach@@YAHQEAUHINSTANCE__@@QEAX@Z 0000000180059b48     LIBCMT:dll_dllmain.obj
 0002:00013b80       $unwind$?fin$0@?0??dllmain_crt_process_attach@@YAHQEAUHINSTANCE__@@QEAX@Z@4HA 0000000180059b80     LIBCMT:dll_dllmain.obj
 0002:00013b80       $unwind$?fin$0@?0??dllmain_crt_process_detach@@YAH_N@Z@4HA 0000000180059b80     LIBCMT:dll_dllmain.obj
 0002:00013b80       $unwind$_query_new_handler$fin$0 0000000180059b80     libucrt:new_handler.obj
 0002:00013b80       $unwind$__acrt_update_thread_locale_data$fin$0 0000000180059b80     libucrt:locale_refcounting.obj
 0002:00013b80       $unwind$__acrt_initialize_lowio$fin$0 0000000180059b80     libucrt:ioinit.obj
 0002:00013b80       $unwind$__acrt_lowio_ensure_fh_exists$fin$0 0000000180059b80     libucrt:osfinfo.obj
 0002:00013b80       $unwind$_write$fin$0       0000000180059b80     libucrt:write.obj
 0002:00013b80       $unwind$?fin$0@?0??update_thread_multibyte_data_internal@@YAPEAU__crt_multibyte_data@@QEAU__acrt_ptd@@QEAPEAU1@@Z@4HA 0000000180059b80     libucrt:mbctype.obj
 0002:00013b80       $unwind$_fcloseall$fin$0   0000000180059b80     libucrt:closeall.obj
 0002:00013b80       $unwind$fclose$fin$0       0000000180059b80     libucrt:fclose.obj
 0002:00013b8c       $unwind$?dllmain_crt_process_detach@@YAH_N@Z 0000000180059b8c     LIBCMT:dll_dllmain.obj
 0002:00013be4       $unwind$?fin$1@?0??dllmain_crt_process_detach@@YAH_N@Z@4HA 0000000180059be4     LIBCMT:dll_dllmain.obj
 0002:00013be4       $unwind$?filt$0@?0??FrameUnwindToState@__FrameHandler3@@SAXPEA_KPEAU_xDISPATCHER_CONTEXT@@PEBU_s_FuncInfo@@H@Z@4HA 0000000180059be4     libvcruntime:frame.obj
 0002:00013bf0       $unwind$?dllmain_dispatch@@YAHQEAUHINSTANCE__@@KQEAX@Z 0000000180059bf0     LIBCMT:dll_dllmain.obj
 0002:00013c14       $unwind$?filt$0@?0??dllmain_dispatch@@YAHQEAUHINSTANCE__@@KQEAX@Z@4HA 0000000180059c14     LIBCMT:dll_dllmain.obj
 0002:00013c20       __security_push_cookie_xdata 0000000180059c20     LIBCMT:secpushpop.obj
 0002:00013c28       __security_push_cookie_xdata_prolog 0000000180059c28     LIBCMT:secpushpop.obj
 0002:00013c2a       __security_push_cookie_xdata_epilog1 0000000180059c2a     LIBCMT:secpushpop.obj
 0002:00013c2c       __security_pop_cookie_xdata 0000000180059c2c     LIBCMT:secpushpop.obj
 0002:00013c2c       __security_push_cookie_xdata_end 0000000180059c2c     LIBCMT:secpushpop.obj
 0002:00013c34       __security_pop_cookie_xdata_prolog 0000000180059c34     LIBCMT:secpushpop.obj
 0002:00013c35       __security_pop_cookie_xdata_epilog1 0000000180059c35     LIBCMT:secpushpop.obj
 0002:00013c3c       __ppgsfailure_xdata        0000000180059c3c     LIBCMT:secpushpop.obj
 0002:00013c3c       __security_pop_cookie_xdata_end 0000000180059c3c     LIBCMT:secpushpop.obj
 0002:00013c44       __ppgsfailure_xdata_prolog 0000000180059c44     LIBCMT:secpushpop.obj
 0002:00013c48       __ppgsfailure_xdata_epilog1 0000000180059c48     LIBCMT:secpushpop.obj
 0002:00013c4c       __chkstk_xdata             0000000180059c4c     LIBCMT:chkstk.obj
 0002:00013c4c       __ppgsfailure_xdata_end    0000000180059c4c     LIBCMT:secpushpop.obj
 0002:00013c50       __chkstk_xdata_prolog      0000000180059c50     LIBCMT:chkstk.obj
 0002:00013c54       __chkstk_xdata_end         0000000180059c54     LIBCMT:chkstk.obj
 0002:00013c54       $unwind$?UnwindNestedFrames@__FrameHandler3@@SAXPEA_KPEAUEHExceptionRecord@@PEAU_CONTEXT@@0PEAXPEBU_s_FuncInfo@@HHPEBU_s_HandlerType@@PEAU_xDISPATCHER_CONTEXT@@E@Z 0000000180059c54     libvcruntime:risctrnsctrl.obj
 0002:00013c68       $unwind$?GetRangeOfTrysToCheck@__FrameHandler3@@SA?AU?$pair@Viterator@TryBlockMap@__FrameHandler3@@V123@@std@@AEAVTryBlockMap@1@HPEAU_xDISPATCHER_CONTEXT@@PEBU_s_FuncInfo@@H@Z 0000000180059c68     libvcruntime:risctrnsctrl.obj
 0002:00013c78       $unwind$_FindAndUnlinkFrame 0000000180059c78     libvcruntime:risctrnsctrl.obj
 0002:00013c84       $unwind$??$_CallSETranslator@V__FrameHandler3@@@@YAHPEAUEHExceptionRecord@@PEA_KPEAU_CONTEXT@@PEAU_xDISPATCHER_CONTEXT@@PEBU_s_FuncInfo@@K1H@Z 0000000180059c84     libvcruntime:risctrnsctrl.obj
 0002:00013ca4       $unwind$?filt$0@?0???$_CallSETranslator@V__FrameHandler3@@@@YAHPEAUEHExceptionRecord@@PEA_KPEAU_CONTEXT@@PEAU_xDISPATCHER_CONTEXT@@PEBU_s_FuncInfo@@K1H@Z@4HA 0000000180059ca4     libvcruntime:risctrnsctrl.obj
 0002:00013cb0       $unwind$_IsExceptionObjectToBeDestroyed 0000000180059cb0     libvcruntime:ehhelpers.obj
 0002:00013cc0       $unwind$__FrameUnwindFilter 0000000180059cc0     libvcruntime:ehhelpers.obj
 0002:00013ccc       $unwind$__DestructExceptionObject 0000000180059ccc     libvcruntime:ehhelpers.obj
 0002:00013cf0       $unwind$__DestructExceptionObject$filt$0 0000000180059cf0     libvcruntime:ehhelpers.obj
 0002:00013cfc       $unwind$_purecall          0000000180059cfc     libvcruntime:purevirt.obj
 0002:00013d08       memcpy_xdata               0000000180059d08     libvcruntime:memcpy.obj
 0002:00013d0c       memcpy_xdata_prolog        0000000180059d0c     libvcruntime:memcpy.obj
 0002:00013d10       __memcpy_forward_large_neon_xdata 0000000180059d10     libvcruntime:memcpy.obj
 0002:00013d10       memcpy_xdata_end           0000000180059d10     libvcruntime:memcpy.obj
 0002:00013d14       __memcpy_forward_large_neon_xdata_prolog 0000000180059d14     libvcruntime:memcpy.obj
 0002:00013d18       __memcpy_forward_large_neon_xdata_end 0000000180059d18     libvcruntime:memcpy.obj
 0002:00013d18       __memcpy_reverse_xdata     0000000180059d18     libvcruntime:memcpy.obj
 0002:00013d1c       __memcpy_reverse_xdata_prolog 0000000180059d1c     libvcruntime:memcpy.obj
 0002:00013d20       __memcpy_reverse_large_neon_xdata 0000000180059d20     libvcruntime:memcpy.obj
 0002:00013d20       __memcpy_reverse_xdata_end 0000000180059d20     libvcruntime:memcpy.obj
 0002:00013d24       __memcpy_reverse_large_neon_xdata_prolog 0000000180059d24     libvcruntime:memcpy.obj
 0002:00013d28       __memcpy_reverse_large_neon_xdata_end 0000000180059d28     libvcruntime:memcpy.obj
 0002:00013d28       memset_xdata               0000000180059d28     libvcruntime:memset.obj
 0002:00013d2c       memset_xdata_prolog        0000000180059d2c     libvcruntime:memset.obj
 0002:00013d30       memcmp_xdata               0000000180059d30     libvcruntime:memcmp.obj
 0002:00013d30       memset_xdata_end           0000000180059d30     libvcruntime:memset.obj
 0002:00013d34       memcmp_xdata_prolog        0000000180059d34     libvcruntime:memcmp.obj
 0002:00013d38       memcmp_xdata_end           0000000180059d38     libvcruntime:memcmp.obj
 0002:00013d38       $unwind$__vcrt_getptd      0000000180059d38     libvcruntime:per_thread_data.obj
 0002:00013d44       $unwind$?FrameUnwindToState@__FrameHandler3@@SAXPEA_KPEAU_xDISPATCHER_CONTEXT@@PEBU_s_FuncInfo@@H@Z 0000000180059d44     libvcruntime:frame.obj
 0002:00013d90       $unwind$?CxxCallCatchBlock@__FrameHandler3@@SAPEAXPEAU_EXCEPTION_RECORD@@@Z 0000000180059d90     libvcruntime:frame.obj
 0002:00013dcc       $unwind$?filt$0@?0??CxxCallCatchBlock@__FrameHandler3@@SAPEAXPEAU_EXCEPTION_RECORD@@@Z@4HA 0000000180059dcc     libvcruntime:frame.obj
 0002:00013dcc       $unwind$raise$fin$0        0000000180059dcc     libucrt:signal.obj
 0002:00013dd8       $unwind$?fin$1@?0??CxxCallCatchBlock@__FrameHandler3@@SAPEAXPEAU_EXCEPTION_RECORD@@@Z@4HA 0000000180059dd8     libvcruntime:frame.obj
 0002:00013de4       $unwind$?IsInExceptionSpec@@YAEPEAUEHExceptionRecord@@PEBU_s_ESTypeList@@@Z 0000000180059de4     libvcruntime:frame.obj
 0002:00013df8       $unwind$??$__InternalCxxFrameHandler@V__FrameHandler3@@@@YA?AW4_EXCEPTION_DISPOSITION@@PEAUEHExceptionRecord@@PEA_KPEAU_CONTEXT@@PEAU_xDISPATCHER_CONTEXT@@PEBU_s_FuncInfo@@H1E@Z 0000000180059df8     libvcruntime:frame.obj
 0002:00013e0c       $unwind$??$BuildCatchObjectHelperInternal@V__FrameHandler3@@@@YAHPEAUEHExceptionRecord@@PEAXPEBU_s_HandlerType@@PEBU_s_CatchableType@@@Z 0000000180059e0c     libvcruntime:frame.obj
 0002:00013e44       $unwind$??$BuildCatchObjectInternal@V__FrameHandler3@@@@YAXPEAUEHExceptionRecord@@PEAXPEBU_s_HandlerType@@PEBU_s_CatchableType@@@Z 0000000180059e44     libvcruntime:frame.obj
 0002:00013e6c       $unwind$??$FindHandler@V__FrameHandler3@@@@YAXPEAUEHExceptionRecord@@PEA_KPEAU_CONTEXT@@PEAU_xDISPATCHER_CONTEXT@@PEBU_s_FuncInfo@@EH1@Z 0000000180059e6c     libvcruntime:frame.obj
 0002:00013e8c       $unwind$??$FindHandlerForForeignException@V__FrameHandler3@@@@YAXPEAUEHExceptionRecord@@PEA_KPEAU_CONTEXT@@PEAU_xDISPATCHER_CONTEXT@@PEBU_s_FuncInfo@@HH1@Z 0000000180059e8c     libvcruntime:frame.obj
 0002:00013ea0       _NLG_Notify_xdata          0000000180059ea0     libvcruntime:notify.obj
 0002:00013ea8       _NLG_Notify_xdata_prolog   0000000180059ea8     libvcruntime:notify.obj
 0002:00013eaa       _NLG_Notify_xdata_epilog1  0000000180059eaa     libvcruntime:notify.obj
 0002:00013eac       _NLG_Notify_xdata_end      0000000180059eac     libvcruntime:notify.obj
 0002:00013eac       __NLG_Return2_xdata        0000000180059eac     libvcruntime:notify.obj
 0002:00013eb0       __NLG_Return2_xdata_prolog 0000000180059eb0     libvcruntime:notify.obj
 0002:00013eb4       __C_ExecuteExceptionFilter_xdata 0000000180059eb4     libvcruntime:handler.obj
 0002:00013eb4       __NLG_Return2_xdata_end    0000000180059eb4     libvcruntime:notify.obj
 0002:00013ebc       __C_ExecuteExceptionFilter_xdata_prolog 0000000180059ebc     libvcruntime:handler.obj
 0002:00013ec9       __C_ExecuteExceptionFilter_xdata_epilog1 0000000180059ec9     libvcruntime:handler.obj
 0002:00013ed4       __C_ExecuteExceptionFilter_xdata_end 0000000180059ed4     libvcruntime:handler.obj
 0002:00013ed4       __C_ExecuteTerminationHandler_xdata 0000000180059ed4     libvcruntime:handler.obj
 0002:00013edc       __C_ExecuteTerminationHandler_xdata_prolog 0000000180059edc     libvcruntime:handler.obj
 0002:00013ee9       __C_ExecuteTerminationHandler_xdata_epilog1 0000000180059ee9     libvcruntime:handler.obj
 0002:00013ef4       __C_ExecuteTerminationHandler_xdata_end 0000000180059ef4     libvcruntime:handler.obj
 0002:00013ef4       _CallSettingFrame_xdata    0000000180059ef4     libvcruntime:handlers.obj
 0002:00013efc       _CallSettingFrame_xdata_prolog 0000000180059efc     libvcruntime:handlers.obj
 0002:00013f09       _CallSettingFrame_xdata_epilog1 0000000180059f09     libvcruntime:handlers.obj
 0002:00013f18       _CallSettingFrame_xdata_end 0000000180059f18     libvcruntime:handlers.obj
 0002:00013f18       $unwind$__acrt_lowio_ensure_fh_exists 0000000180059f18     libucrt:osfinfo.obj
 0002:00013f50       $unwind$??$common_vsprintf@Vformat_validation_base@__crt_stdio_output@@D@@YAH_KQEAD0QEBDQEAU__crt_locale_pointers@@1@Z 0000000180059f50     libucrt:output.obj
 0002:00013f6c       $unwind$?write_stored_string_tchar@?$output_processor@DV?$string_output_adapter@D@__crt_stdio_output@@V?$format_validation_base@DV?$string_output_adapter@D@__crt_stdio_output@@@2@@__crt_stdio_output@@AEAA_ND@Z 0000000180059f6c     libucrt:output.obj
 0002:00013f80       $unwind$terminate          0000000180059f80     libucrt:terminate.obj
 0002:00013fa4       $unwind$free               0000000180059fa4     libucrt:free.obj
 0002:00013fac       $unwind$strncpy_s          0000000180059fac     libucrt:strncpy_s.obj
 0002:00013fac       $unwind$wcsncpy_s          0000000180059fac     libucrt:wcsncpy_s.obj
 0002:00013fb8       $unwind$??R<lambda_b37934c380d97b75fd242ea49540127a>@@QEBAPEADXZ 0000000180059fb8     libucrt:setlocale.obj
 0002:00013fc8       $unwind$??$?RV<lambda_41e84717acc955b55e9d0d529e507b68>@@AEAV<lambda_b37934c380d97b75fd242ea49540127a>@@V<lambda_bb6db9f9ac473960206e0d4b942b5506>@@@?$__crt_seh_guarded_call@PEAD@@QEAAPEAD$$QEAV<lambda_41e84717acc955b55e9d0d529e507b68>@@AEAV<lambda_b37934c380d97b75fd242ea49540127a>@@$$QEAV<lambda_bb6db9f9ac473960206e0d4b942b5506>@@@Z 0000000180059fc8     libucrt:setlocale.obj
 0002:00013fe8       $unwind$?fin$0@?0???$?RV<lambda_0ae27a3a962d80f24befdcbee591983d>@@AEAV<lambda_8d0ee55de4b1038c4002e0adecdf1839>@@V<lambda_dc504788e8f1664fe9b84e20bfb512f2>@@@?$__crt_seh_guarded_call@X@@QEAAX$$QEAV<lambda_0ae27a3a962d80f24befdcbee591983d>@@AEAV<lambda_8d0ee55de4b1038c4002e0adecdf1839>@@$$QEAV<lambda_dc504788e8f1664fe9b84e20bfb512f2>@@@Z@4HA 0000000180059fe8     libucrt:per_thread_data.obj
 0002:00013fe8       $unwind$?fin$0@?0???$?RV<lambda_2d41944a1d46af3157314b8a01080d33>@@AEAV<lambda_8f455de75cd7d7f24b4096f044d8b9e6>@@V<lambda_aa500f224e6afead328df44964fe2772>@@@?$__crt_seh_guarded_call@X@@QEAAX$$QEAV<lambda_2d41944a1d46af3157314b8a01080d33>@@AEAV<lambda_8f455de75cd7d7f24b4096f044d8b9e6>@@$$QEAV<lambda_aa500f224e6afead328df44964fe2772>@@@Z@4HA 0000000180059fe8     libucrt:per_thread_data.obj
 0002:00013fe8       $unwind$?fin$0@?0???$?RV<lambda_aa87e3671a710a21b5dc78c0bdf72e11>@@AEAV<lambda_92619d2358a28f41a33ba319515a20b9>@@V<lambda_6992ecaafeb10aed2b74cb1fae11a551>@@@?$__crt_seh_guarded_call@X@@QEAAX$$QEAV<lambda_aa87e3671a710a21b5dc78c0bdf72e11>@@AEAV<lambda_92619d2358a28f41a33ba319515a20b9>@@$$QEAV<lambda_6992ecaafeb10aed2b74cb1fae11a551>@@@Z@4HA 0000000180059fe8     libucrt:per_thread_data.obj
 0002:00013fe8       $unwind$?fin$0@?0???$?RV<lambda_f2e299630e499de9f9a165e60fcd3db5>@@AEAV<lambda_2ae9d31cdba2644fcbeaf08da7c24588>@@V<lambda_40d01ff24d0e7b3814fdbdcee8eab3c7>@@@?$__crt_seh_guarded_call@X@@QEAAX$$QEAV<lambda_f2e299630e499de9f9a165e60fcd3db5>@@AEAV<lambda_2ae9d31cdba2644fcbeaf08da7c24588>@@$$QEAV<lambda_40d01ff24d0e7b3814fdbdcee8eab3c7>@@@Z@4HA 0000000180059fe8     libucrt:per_thread_data.obj
 0002:00013fe8       $unwind$?fin$0@?0???$?RV<lambda_48fc4a32460bb0512d3b13f8499328be>@@AEAV<lambda_6c3dac0a4f3f9cefca9bb494422f9b77>@@V<lambda_0a2f2c9f9a56eb2b08bfa6ff61d331c5>@@@?$__crt_seh_guarded_call@H@@QEAAH$$QEAV<lambda_48fc4a32460bb0512d3b13f8499328be>@@AEAV<lambda_6c3dac0a4f3f9cefca9bb494422f9b77>@@$$QEAV<lambda_0a2f2c9f9a56eb2b08bfa6ff61d331c5>@@@Z@4HA 0000000180059fe8     libucrt:winapi_thunks.obj
 0002:00013fe8       $unwind$?fin$0@?0???$?RV<lambda_41e84717acc955b55e9d0d529e507b68>@@AEAV<lambda_b37934c380d97b75fd242ea49540127a>@@V<lambda_bb6db9f9ac473960206e0d4b942b5506>@@@?$__crt_seh_guarded_call@PEAD@@QEAAPEAD$$QEAV<lambda_41e84717acc955b55e9d0d529e507b68>@@AEAV<lambda_b37934c380d97b75fd242ea49540127a>@@$$QEAV<lambda_bb6db9f9ac473960206e0d4b942b5506>@@@Z@4HA 0000000180059fe8     libucrt:setlocale.obj
 0002:00013fe8       $unwind$?fin$0@?0???$?RV<lambda_1d892b297fdedeee07ed8124eeb2f2fa>@@AEAV<lambda_ffc046909424fd52df0ac47e64813305>@@V<lambda_01a7098693036236037e7cdb9bca3d73>@@@?$__crt_seh_guarded_call@X@@QEAAX$$QEAV<lambda_1d892b297fdedeee07ed8124eeb2f2fa>@@AEAV<lambda_ffc046909424fd52df0ac47e64813305>@@$$QEAV<lambda_01a7098693036236037e7cdb9bca3d73>@@@Z@4HA 0000000180059fe8     libucrt:wsetlocale.obj
 0002:00013fe8       $unwind$?fin$0@?0???$?RV<lambda_410d79af7f07d98d83a3f525b3859a53>@@AEAV<lambda_3e16ef9562a7dcce91392c22ab16ea36>@@V<lambda_38119f0e861e05405d8a144b9b982f0a>@@@?$__crt_seh_guarded_call@X@@QEAAX$$QEAV<lambda_410d79af7f07d98d83a3f525b3859a53>@@AEAV<lambda_3e16ef9562a7dcce91392c22ab16ea36>@@$$QEAV<lambda_38119f0e861e05405d8a144b9b982f0a>@@@Z@4HA 0000000180059fe8     libucrt:wsetlocale.obj
 0002:00013fe8       $unwind$?fin$0@?0???$?RV<lambda_751a882b2c74d4b022dec766aa51a29a>@@AEAV<lambda_628dfdc04ba53c8bfc02c9951375f3f5>@@V<lambda_f6c7be5f7998530c34de24c7437d6b54>@@@?$__crt_seh_guarded_call@H@@QEAAH$$QEAV<lambda_751a882b2c74d4b022dec766aa51a29a>@@AEAV<lambda_628dfdc04ba53c8bfc02c9951375f3f5>@@$$QEAV<lambda_f6c7be5f7998530c34de24c7437d6b54>@@@Z@4HA 0000000180059fe8     libucrt:close.obj
 0002:00013fe8       $unwind$?fin$0@?0???$?RV<lambda_a37b2b86f63e897a80ea819b0eb08c01>@@AEAV<lambda_38ce7e780aa69e748d6df282ebc68efe>@@V<lambda_99fb1378e971ab6e7edea83e3a7a83a2>@@@?$__crt_seh_guarded_call@H@@QEAAH$$QEAV<lambda_a37b2b86f63e897a80ea819b0eb08c01>@@AEAV<lambda_38ce7e780aa69e748d6df282ebc68efe>@@$$QEAV<lambda_99fb1378e971ab6e7edea83e3a7a83a2>@@@Z@4HA 0000000180059fe8     libucrt:commit.obj
 0002:00013fe8       $unwind$?fin$0@?0???$?RV<lambda_efdfa57d1f175319df784efa44bb7b81>@@AEAV<lambda_5f0a4c1567f8adc6734073e5d1e1b35c>@@V<lambda_2e8a7d3640ea6ccb4c2413664c2db6fd>@@@?$__crt_seh_guarded_call@X@@QEAAX$$QEAV<lambda_efdfa57d1f175319df784efa44bb7b81>@@AEAV<lambda_5f0a4c1567f8adc6734073e5d1e1b35c>@@$$QEAV<lambda_2e8a7d3640ea6ccb4c2413664c2db6fd>@@@Z@4HA 0000000180059fe8     libucrt:mbctype.obj
 0002:00013fe8       $unwind$?fin$0@?0???$?RV<lambda_450d765d439847d4c735a33c368b5fc0>@@AEAV<lambda_44731a7d0e6d81c3e6aa82d741081786>@@V<lambda_601a2a7da3b7a96e9554ac7215c4b07c>@@@?$__crt_seh_guarded_call@P6AXH@Z@@QEAAP6AXH@Z$$QEAV<lambda_450d765d439847d4c735a33c368b5fc0>@@AEAV<lambda_44731a7d0e6d81c3e6aa82d741081786>@@$$QEAV<lambda_601a2a7da3b7a96e9554ac7215c4b07c>@@@Z@4HA 0000000180059fe8     libucrt:signal.obj
 0002:00013fe8       $unwind$?filt$0@?0???R<lambda_6e4b09c48022b2350581041d5f6b0c4c>@@QEBA@XZ@4HA 0000000180059fe8     libucrt:exit.obj
 0002:00013fe8       $unwind$?fin$0@?0???$?RV<lambda_d80eeec6fff315bfe5c115232f3240e3>@@AEAV<lambda_6e4b09c48022b2350581041d5f6b0c4c>@@V<lambda_2358e3775559c9db80273638284d5e45>@@@?$__crt_seh_guarded_call@X@@QEAAX$$QEAV<lambda_d80eeec6fff315bfe5c115232f3240e3>@@AEAV<lambda_6e4b09c48022b2350581041d5f6b0c4c>@@$$QEAV<lambda_2358e3775559c9db80273638284d5e45>@@@Z@4HA 0000000180059fe8     libucrt:exit.obj
 0002:00013fe8       $unwind$?fin$0@?0???$?RV<lambda_638799b9deba96c50f710eeac98168cd>@@AEAV<lambda_22ebabd17bc4fa466a2aca6d8deb888d>@@V<lambda_a6f7d7db0129f75315ebf26d50c089f1>@@@?$__crt_seh_guarded_call@H@@QEAAH$$QEAV<lambda_638799b9deba96c50f710eeac98168cd>@@AEAV<lambda_22ebabd17bc4fa466a2aca6d8deb888d>@@$$QEAV<lambda_a6f7d7db0129f75315ebf26d50c089f1>@@@Z@4HA 0000000180059fe8     libucrt:onexit.obj
 0002:00013fe8       $unwind$?fin$0@?0???$?RV<lambda_7777bce6b2f8c936911f934f8298dc43>@@AEAV<lambda_f03950bc5685219e0bcd2087efbe011e>@@V<lambda_3883c3dff614d5e0c5f61bb1ac94921c>@@@?$__crt_seh_guarded_call@H@@QEAAH$$QEAV<lambda_7777bce6b2f8c936911f934f8298dc43>@@AEAV<lambda_f03950bc5685219e0bcd2087efbe011e>@@$$QEAV<lambda_3883c3dff614d5e0c5f61bb1ac94921c>@@@Z@4HA 0000000180059fe8     libucrt:onexit.obj
 0002:00013fe8       $unwind$?fin$0@?0???$?RV<lambda_842d9ff0dc9ef11c61343bbaebe7f885>@@AEAV<lambda_c5860995281e5c4ce005b3de8f5874ee>@@V<lambda_d90129c13df834fdcbf8d2b88dafcf2d>@@@?$__crt_seh_guarded_call@X@@QEAAX$$QEAV<lambda_842d9ff0dc9ef11c61343bbaebe7f885>@@AEAV<lambda_c5860995281e5c4ce005b3de8f5874ee>@@$$QEAV<lambda_d90129c13df834fdcbf8d2b88dafcf2d>@@@Z@4HA 0000000180059fe8     libucrt:fflush.obj
 0002:00013fe8       $unwind$?fin$0@?0???$?RV<lambda_886d6c58226a84441f68b9f2b8217b83>@@AEAV<lambda_ab61a845afdef5b7c387490eaf3616ee>@@V<lambda_f7f22ab5edc0698d5f6905b0d3f44752>@@@?$__crt_seh_guarded_call@X@@QEAAX$$QEAV<lambda_886d6c58226a84441f68b9f2b8217b83>@@AEAV<lambda_ab61a845afdef5b7c387490eaf3616ee>@@$$QEAV<lambda_f7f22ab5edc0698d5f6905b0d3f44752>@@@Z@4HA 0000000180059fe8     libucrt:fflush.obj
 0002:00013ff4       $unwind$__acrt_locale_initialize_ctype 0000000180059ff4     libucrt:initctype.obj
 0002:00014010       $unwind$?divide@__crt_strtox@@YA_KAEAUbig_integer@1@AEBU21@@Z 000000018005a010     libucrt:strtod.obj
 0002:00014030       $unwind$abort              000000018005a030     libucrt:abort.obj
 0002:00014038       $unwind$_wcsdup            000000018005a038     libucrt:wcsdup.obj
 0002:00014048       $unwind$??$__acrt_wcs_to_mbs_cp@U__crt_win32_buffer_no_resizing@@@@YAHQEB_WAEAV?$__crt_win32_buffer@DU__crt_win32_buffer_no_resizing@@@@I@Z 000000018005a048     libucrt:strftime.obj
 0002:00014054       $unwind$?exit_or_terminate_process@@YAXI@Z 000000018005a054     libucrt:exit.obj
 0002:00014060       $unwind$?common_exit@@YAXHW4_crt_exit_cleanup_mode@@W4_crt_exit_return_mode@@@Z 000000018005a060     libucrt:exit.obj
 0002:00014070       $unwind$??R<lambda_6e4b09c48022b2350581041d5f6b0c4c>@@QEBA@XZ 000000018005a070     libucrt:exit.obj
 0002:00014098       $unwind$??$?RV<lambda_d80eeec6fff315bfe5c115232f3240e3>@@AEAV<lambda_6e4b09c48022b2350581041d5f6b0c4c>@@V<lambda_2358e3775559c9db80273638284d5e45>@@@?$__crt_seh_guarded_call@X@@QEAAX$$QEAV<lambda_d80eeec6fff315bfe5c115232f3240e3>@@AEAV<lambda_6e4b09c48022b2350581041d5f6b0c4c>@@$$QEAV<lambda_2358e3775559c9db80273638284d5e45>@@@Z 000000018005a098     libucrt:exit.obj
 0002:000140b8       $unwind$??$create_environment@D@@YAQEAPEADQEAD@Z 000000018005a0b8     libucrt:environment_initialization.obj
 0002:000140c8       $unwind$??$?RV<lambda_638799b9deba96c50f710eeac98168cd>@@AEAV<lambda_22ebabd17bc4fa466a2aca6d8deb888d>@@V<lambda_a6f7d7db0129f75315ebf26d50c089f1>@@@?$__crt_seh_guarded_call@H@@QEAAH$$QEAV<lambda_638799b9deba96c50f710eeac98168cd>@@AEAV<lambda_22ebabd17bc4fa466a2aca6d8deb888d>@@$$QEAV<lambda_a6f7d7db0129f75315ebf26d50c089f1>@@@Z 000000018005a0c8     libucrt:onexit.obj
 0002:000140e8       $unwind$??$?RV<lambda_7777bce6b2f8c936911f934f8298dc43>@@AEAV<lambda_f03950bc5685219e0bcd2087efbe011e>@@V<lambda_3883c3dff614d5e0c5f61bb1ac94921c>@@@?$__crt_seh_guarded_call@H@@QEAAH$$QEAV<lambda_7777bce6b2f8c936911f934f8298dc43>@@AEAV<lambda_f03950bc5685219e0bcd2087efbe011e>@@$$QEAV<lambda_3883c3dff614d5e0c5f61bb1ac94921c>@@@Z 000000018005a0e8     libucrt:onexit.obj
 0002:00014108       $unwind$_query_new_handler 000000018005a108     libucrt:new_handler.obj
 0002:0001412c       $unwind$_invalid_parameter 000000018005a12c     libucrt:invalid_parameter.obj
 0002:0001413c       $unwind$__acrt_initialize_lowio 000000018005a13c     libucrt:ioinit.obj
 0002:00014160       $unwind$??$?RV<lambda_48fc4a32460bb0512d3b13f8499328be>@@AEAV<lambda_6c3dac0a4f3f9cefca9bb494422f9b77>@@V<lambda_0a2f2c9f9a56eb2b08bfa6ff61d331c5>@@@?$__crt_seh_guarded_call@H@@QEAAH$$QEAV<lambda_48fc4a32460bb0512d3b13f8499328be>@@AEAV<lambda_6c3dac0a4f3f9cefca9bb494422f9b77>@@$$QEAV<lambda_0a2f2c9f9a56eb2b08bfa6ff61d331c5>@@@Z 000000018005a160     libucrt:winapi_thunks.obj
 0002:00014184       $unwind$_fcloseall         000000018005a184     libucrt:closeall.obj
 0002:000141a8       $unwind$??$?RV<lambda_842d9ff0dc9ef11c61343bbaebe7f885>@@AEAV<lambda_c5860995281e5c4ce005b3de8f5874ee>@@V<lambda_d90129c13df834fdcbf8d2b88dafcf2d>@@@?$__crt_seh_guarded_call@X@@QEAAX$$QEAV<lambda_842d9ff0dc9ef11c61343bbaebe7f885>@@AEAV<lambda_c5860995281e5c4ce005b3de8f5874ee>@@$$QEAV<lambda_d90129c13df834fdcbf8d2b88dafcf2d>@@@Z 000000018005a1a8     libucrt:fflush.obj
 0002:000141c8       $unwind$??$?RV<lambda_886d6c58226a84441f68b9f2b8217b83>@@AEAV<lambda_ab61a845afdef5b7c387490eaf3616ee>@@V<lambda_f7f22ab5edc0698d5f6905b0d3f44752>@@@?$__crt_seh_guarded_call@X@@QEAAX$$QEAV<lambda_886d6c58226a84441f68b9f2b8217b83>@@AEAV<lambda_ab61a845afdef5b7c387490eaf3616ee>@@$$QEAV<lambda_f7f22ab5edc0698d5f6905b0d3f44752>@@@Z 000000018005a1c8     libucrt:fflush.obj
 0002:000141ec       $unwind$_wctomb_s_l        000000018005a1ec     libucrt:wctomb.obj
 0002:000141fc       $unwind$__acrt_getptd      000000018005a1fc     libucrt:per_thread_data.obj
 0002:0001420c       $unwind$__acrt_getptd_head 000000018005a20c     libucrt:per_thread_data.obj
 0002:00014218       $unwind$??$?RV<lambda_0ae27a3a962d80f24befdcbee591983d>@@AEAV<lambda_8d0ee55de4b1038c4002e0adecdf1839>@@V<lambda_dc504788e8f1664fe9b84e20bfb512f2>@@@?$__crt_seh_guarded_call@X@@QEAAX$$QEAV<lambda_0ae27a3a962d80f24befdcbee591983d>@@AEAV<lambda_8d0ee55de4b1038c4002e0adecdf1839>@@$$QEAV<lambda_dc504788e8f1664fe9b84e20bfb512f2>@@@Z 000000018005a218     libucrt:per_thread_data.obj
 0002:00014238       $unwind$??$?RV<lambda_aa87e3671a710a21b5dc78c0bdf72e11>@@AEAV<lambda_92619d2358a28f41a33ba319515a20b9>@@V<lambda_6992ecaafeb10aed2b74cb1fae11a551>@@@?$__crt_seh_guarded_call@X@@QEAAX$$QEAV<lambda_aa87e3671a710a21b5dc78c0bdf72e11>@@AEAV<lambda_92619d2358a28f41a33ba319515a20b9>@@$$QEAV<lambda_6992ecaafeb10aed2b74cb1fae11a551>@@@Z 000000018005a238     libucrt:per_thread_data.obj
 0002:00014258       $unwind$??$?RV<lambda_f2e299630e499de9f9a165e60fcd3db5>@@AEAV<lambda_2ae9d31cdba2644fcbeaf08da7c24588>@@V<lambda_40d01ff24d0e7b3814fdbdcee8eab3c7>@@@?$__crt_seh_guarded_call@X@@QEAAX$$QEAV<lambda_f2e299630e499de9f9a165e60fcd3db5>@@AEAV<lambda_2ae9d31cdba2644fcbeaf08da7c24588>@@$$QEAV<lambda_40d01ff24d0e7b3814fdbdcee8eab3c7>@@@Z 000000018005a258     libucrt:per_thread_data.obj
 0002:00014278       $unwind$??$?RV<lambda_2d41944a1d46af3157314b8a01080d33>@@AEAV<lambda_8f455de75cd7d7f24b4096f044d8b9e6>@@V<lambda_aa500f224e6afead328df44964fe2772>@@@?$__crt_seh_guarded_call@X@@QEAAX$$QEAV<lambda_2d41944a1d46af3157314b8a01080d33>@@AEAV<lambda_8f455de75cd7d7f24b4096f044d8b9e6>@@$$QEAV<lambda_aa500f224e6afead328df44964fe2772>@@@Z 000000018005a278     libucrt:per_thread_data.obj
 0002:00014298       $unwind$?fp_format_nan_or_infinity@@YAHW4__acrt_fp_class@@_NPEAD_K1@Z 000000018005a298     libucrt:cvt.obj
 0002:000142a4       $unwind$?fp_format_e_internal@@YAHQEAD_KH_NIQEAU_strflt@@2QEAU__crt_locale_pointers@@@Z 000000018005a2a4     libucrt:cvt.obj
 0002:000142b8       $unwind$__acrt_copy_locale_name 000000018005a2b8     libucrt:wsetlocale.obj
 0002:000142c8       $unwind$_expandlocale      000000018005a2c8     libucrt:wsetlocale.obj
 0002:000142e8       $unwind$_wcscats           000000018005a2e8     libucrt:wsetlocale.obj
 0002:00014300       $unwind$__lc_lctowcs       000000018005a300     libucrt:wsetlocale.obj
 0002:00014310       $unwind$__lc_wcstolc       000000018005a310     libucrt:wsetlocale.obj
 0002:00014320       $unwind$_wsetlocale_set_cat 000000018005a320     libucrt:wsetlocale.obj
 0002:0001433c       $unwind$_wsetlocale_get_all 000000018005a33c     libucrt:wsetlocale.obj
 0002:00014350       $unwind$_wsetlocale_nolock 000000018005a350     libucrt:wsetlocale.obj
 0002:00014370       $unwind$string_is_alpha    000000018005a370     libucrt:wsetlocale.obj
 0002:00014380       $unwind$parse_bcp47_language 000000018005a380     libucrt:wsetlocale.obj
 0002:0001438c       $unwind$parse_bcp47_script 000000018005a38c     libucrt:wsetlocale.obj
 0002:00014398       $unwind$__acrt_DownlevelLCIDToLocaleName 000000018005a398     libucrt:lcidtoname_downlevel.obj
 0002:00014398       $unwind$parse_bcp47_region 000000018005a398     libucrt:wsetlocale.obj
 0002:000143a8       $unwind$parse_bcp47_code_page 000000018005a3a8     libucrt:wsetlocale.obj
 0002:000143b4       $unwind$parse_bcp47        000000018005a3b4     libucrt:wsetlocale.obj
 0002:000143cc       $unwind$??$?RV<lambda_410d79af7f07d98d83a3f525b3859a53>@@AEAV<lambda_3e16ef9562a7dcce91392c22ab16ea36>@@V<lambda_38119f0e861e05405d8a144b9b982f0a>@@@?$__crt_seh_guarded_call@X@@QEAAX$$QEAV<lambda_410d79af7f07d98d83a3f525b3859a53>@@AEAV<lambda_3e16ef9562a7dcce91392c22ab16ea36>@@$$QEAV<lambda_38119f0e861e05405d8a144b9b982f0a>@@@Z 000000018005a3cc     libucrt:wsetlocale.obj
 0002:000143f0       $unwind$??$?RV<lambda_1d892b297fdedeee07ed8124eeb2f2fa>@@AEAV<lambda_ffc046909424fd52df0ac47e64813305>@@V<lambda_01a7098693036236037e7cdb9bca3d73>@@@?$__crt_seh_guarded_call@X@@QEAAX$$QEAV<lambda_1d892b297fdedeee07ed8124eeb2f2fa>@@AEAV<lambda_ffc046909424fd52df0ac47e64813305>@@$$QEAV<lambda_01a7098693036236037e7cdb9bca3d73>@@@Z 000000018005a3f0     libucrt:wsetlocale.obj
 0002:00014414       $unwind$??$?RV<lambda_7f2adfce497ff2baa965cd4f576ecfd1>@@AEAV<lambda_2a444430fde8c29194d880d93eed5e8f>@@AEAV<lambda_8dff2cf36a5417162780cd64fa2883ef>@@@?$__crt_seh_guarded_call@X@@QEAAX$$QEAV<lambda_7f2adfce497ff2baa965cd4f576ecfd1>@@AEAV<lambda_2a444430fde8c29194d880d93eed5e8f>@@AEAV<lambda_8dff2cf36a5417162780cd64fa2883ef>@@@Z 000000018005a414     libucrt:wsetlocale.obj
 0002:00014438       $unwind$_IsNonwritableInCurrentImage$filt$0 000000018005a438     LIBCMT:pesect.obj
 0002:00014438       $unwind$?fin$0@?0???$?RV<lambda_7f2adfce497ff2baa965cd4f576ecfd1>@@AEAV<lambda_2a444430fde8c29194d880d93eed5e8f>@@AEAV<lambda_8dff2cf36a5417162780cd64fa2883ef>@@@?$__crt_seh_guarded_call@X@@QEAAX$$QEAV<lambda_7f2adfce497ff2baa965cd4f576ecfd1>@@AEAV<lambda_2a444430fde8c29194d880d93eed5e8f>@@AEAV<lambda_8dff2cf36a5417162780cd64fa2883ef>@@@Z@4HA 000000018005a438     libucrt:wsetlocale.obj
 0002:00014444       $unwind$_write             000000018005a444     libucrt:write.obj
 0002:0001446c       $unwind$_write_nolock      000000018005a46c     libucrt:write.obj
 0002:00014488       $unwind$?write_double_translated_ansi_nolock@@YA?AUwrite_result@?A0x17268360@@HQEBDI@Z 000000018005a488     libucrt:write.obj
 0002:000144a4       $unwind$?write_text_ansi_nolock@@YA?AUwrite_result@?A0x17268360@@HQEBDI@Z 000000018005a4a4     libucrt:write.obj
 0002:000144c0       $unwind$?write_text_utf16le_nolock@@YA?AUwrite_result@?A0x17268360@@HQEBDI@Z 000000018005a4c0     libucrt:write.obj
 0002:000144dc       $unwind$?write_text_utf8_nolock@@YA?AUwrite_result@?A0x17268360@@HQEBDI@Z 000000018005a4dc     libucrt:write.obj
 0002:000144f8       $unwind$_handle_error      000000018005a4f8     libucrt:libm_error.obj
 0002:00014518       $unwind$?_wcstombs_l_helper@@YA_KPEADPEB_W_KPEAU__crt_locale_pointers@@@Z 000000018005a518     libucrt:wcstombs.obj
 0002:00014534       $stateUnwindMap$?_wcstombs_l_helper@@YA_KPEADPEB_W_KPEAU__crt_locale_pointers@@@Z 000000018005a534     libucrt:wcstombs.obj
 0002:00014540       $ip2state$?_wcstombs_l_helper@@YA_KPEADPEB_W_KPEAU__crt_locale_pointers@@@Z 000000018005a540     libucrt:wcstombs.obj
 0002:00014550       $unwind$__acrt_GetLocaleInfoA 000000018005a550     libucrt:getlocaleinfoa.obj
 0002:0001456c       $unwind$?InternalGetLocaleInfoA@@YAHQEAU__crt_locale_pointers@@QEB_WKQEADH@Z 000000018005a56c     libucrt:getlocaleinfoa.obj
 0002:00014584       $unwind$__acrt_GetStringTypeA 000000018005a584     libucrt:getstringtypea.obj
 0002:000145a0       $unwind$?__acrt_LCMapStringA_stat@@YAHPEAU__crt_locale_pointers@@PEB_WKPEBDHPEADHHH@Z 000000018005a5a0     libucrt:lcmapstringa.obj
 0002:000145c0       $unwind$_except2           000000018005a5c0     libucrt:fpexcept.obj
 0002:000145dc       $unwind$_umatherr          000000018005a5dc     libucrt:fpexcept.obj
 0002:000145ec       $unwind$_d_inttype         000000018005a5ec     libucrt:powhlp.obj
 0002:000145f8       $unwind$_powhlp            000000018005a5f8     libucrt:powhlp.obj
 0002:00014604       $unwind$_frnd              000000018005a604     libucrt:frnd.obj
 0002:00014610       $unwind$raise              000000018005a610     libucrt:signal.obj
 0002:0001464c       $unwind$??$?RV<lambda_450d765d439847d4c735a33c368b5fc0>@@AEAV<lambda_44731a7d0e6d81c3e6aa82d741081786>@@V<lambda_601a2a7da3b7a96e9554ac7215c4b07c>@@@?$__crt_seh_guarded_call@P6AXH@Z@@QEAAP6AXH@Z$$QEAV<lambda_450d765d439847d4c735a33c368b5fc0>@@AEAV<lambda_44731a7d0e6d81c3e6aa82d741081786>@@$$QEAV<lambda_601a2a7da3b7a96e9554ac7215c4b07c>@@@Z 000000018005a64c     libucrt:signal.obj
 0002:0001466c       $unwind$??$__acrt_wcs_to_mbs_cp@U__crt_win32_buffer_internal_dynamic_resizing@@@@YAHQEB_WAEAV?$__crt_win32_buffer@DU__crt_win32_buffer_internal_dynamic_resizing@@@@I@Z 000000018005a66c     libucrt:argv_wildcards.obj
 0002:00014678       $unwind$??$common_expand_argv_wildcards@D@@YAHQEAPEADQEAPEAPEAD@Z 000000018005a678     libucrt:argv_wildcards.obj
 0002:0001468c       $unwind$??$copy_and_add_argument_to_buffer@D@@YAHQEBD0_KAEAV?$argument_list@D@?A0x5f5c8891@@@Z 000000018005a68c     libucrt:argv_wildcards.obj
 0002:000146a0       $unwind$??$expand_argument_wildcards@D@@YAHQEAD0AEAV?$argument_list@D@?A0x5f5c8891@@@Z 000000018005a6a0     libucrt:argv_wildcards.obj
 0002:000146bc       $unwind$__acrt_GetModuleFileNameA 000000018005a6bc     libucrt:getmodulefilenamea.obj
 0002:000146d0       $unwind$_setmbcp_nolock    000000018005a6d0     libucrt:mbctype.obj
 0002:000146e8       $unwind$?update_thread_multibyte_data_internal@@YAPEAU__crt_multibyte_data@@QEAU__acrt_ptd@@QEAPEAU1@@Z 000000018005a6e8     libucrt:mbctype.obj
 0002:00014710       $unwind$?setmbcp_internal@@YAHH_NQEAU__acrt_ptd@@QEAPEAU__crt_multibyte_data@@@Z 000000018005a710     libucrt:mbctype.obj
 0002:00014720       $unwind$?setSBUpLow@@YAXPEAU__crt_multibyte_data@@@Z 000000018005a720     libucrt:mbctype.obj
 0002:00014734       $unwind$??$?RV<lambda_efdfa57d1f175319df784efa44bb7b81>@@AEAV<lambda_5f0a4c1567f8adc6734073e5d1e1b35c>@@V<lambda_2e8a7d3640ea6ccb4c2413664c2db6fd>@@@?$__crt_seh_guarded_call@X@@QEAAX$$QEAV<lambda_efdfa57d1f175319df784efa44bb7b81>@@AEAV<lambda_5f0a4c1567f8adc6734073e5d1e1b35c>@@$$QEAV<lambda_2e8a7d3640ea6ccb4c2413664c2db6fd>@@@Z 000000018005a734     libucrt:mbctype.obj
 0002:00014758       $unwind$fclose             000000018005a758     libucrt:fclose.obj
 0002:0001477c       $unwind$??$?RV<lambda_a37b2b86f63e897a80ea819b0eb08c01>@@AEAV<lambda_38ce7e780aa69e748d6df282ebc68efe>@@V<lambda_99fb1378e971ab6e7edea83e3a7a83a2>@@@?$__crt_seh_guarded_call@H@@QEAAH$$QEAV<lambda_a37b2b86f63e897a80ea819b0eb08c01>@@AEAV<lambda_38ce7e780aa69e748d6df282ebc68efe>@@$$QEAV<lambda_99fb1378e971ab6e7edea83e3a7a83a2>@@@Z 000000018005a77c     libucrt:commit.obj
 0002:0001479c       $unwind$?__mbsrtowcs_utf8@__crt_mbstring@@YA_KPEA_WPEAPEBD_KPEAU_Mbstatet@@@Z 000000018005a79c     libucrt:mbrtowc.obj
 0002:000147b0       $unwind$__acrt_update_thread_locale_data 000000018005a7b0     libucrt:locale_refcounting.obj
 0002:000147d4       $unwind$memcpy_s           000000018005a7d4     libucrt:cfout.obj
 0002:000147e4       $unwind$__acrt_fltout      000000018005a7e4     libucrt:cfout.obj
 0002:00014804       $unwind$__acrt_locale_initialize_monetary 000000018005a804     libucrt:initmon.obj
 0002:00014818       $unwind$wcsncat_s          000000018005a818     libucrt:wcsncat_s.obj
 0002:00014824       $unwind$__acrt_get_qualified_locale 000000018005a824     libucrt:get_qualified_locale.obj
 0002:0001483c       $unwind$LangCountryEnumProcEx 000000018005a83c     libucrt:get_qualified_locale.obj
 0002:00014854       $unwind$LanguageEnumProcEx 000000018005a854     libucrt:get_qualified_locale.obj
 0002:0001486c       $unwind$ProcessCodePage    000000018005a86c     libucrt:get_qualified_locale.obj
 0002:00014878       $unwind$__acrt_get_qualified_locale_downlevel 000000018005a878     libucrt:getqloc_downlevel.obj
 0002:0001488c       $unwind$TranslateName      000000018005a88c     libucrt:getqloc_downlevel.obj
 0002:0001489c       $unwind$LangCountryEnumProc 000000018005a89c     libucrt:getqloc_downlevel.obj
 0002:000148b0       $unwind$LanguageEnumProc   000000018005a8b0     libucrt:getqloc_downlevel.obj
 0002:000148c4       $unwind$CountryEnumProc    000000018005a8c4     libucrt:getqloc_downlevel.obj
 0002:000148d8       $unwind$?__wcsrtombs_utf8@__crt_mbstring@@YA_KPEADPEAPEB_W_KPEAU_Mbstatet@@@Z 000000018005a8d8     libucrt:wcrtomb.obj
 0002:000148f4       $unwind$qsort              000000018005a8f4     libucrt:qsort.obj
 0002:00014914       $unwind$strpbrk            000000018005a914     libucrt:strpbrk.obj
 0002:00014928       $unwind$??$?RV<lambda_751a882b2c74d4b022dec766aa51a29a>@@AEAV<lambda_628dfdc04ba53c8bfc02c9951375f3f5>@@V<lambda_f6c7be5f7998530c34de24c7437d6b54>@@@?$__crt_seh_guarded_call@H@@QEAAH$$QEAV<lambda_751a882b2c74d4b022dec766aa51a29a>@@AEAV<lambda_628dfdc04ba53c8bfc02c9951375f3f5>@@$$QEAV<lambda_f6c7be5f7998530c34de24c7437d6b54>@@@Z 000000018005a928     libucrt:close.obj
 0002:00014948       $unwind$?__mbrtoc32_utf8@__crt_mbstring@@YA_KPEA_UPEBD_KPEAU_Mbstatet@@@Z 000000018005a948     libucrt:mbrtoc32.obj
 0002:00014958       $unwind$_IsNonwritableInCurrentImage 000000018005a958     LIBCMT:pesect.obj
 0002:00014d50       .edata                     000000018005ad50     ProcList.exp
 0002:00014d78       rgpv                       000000018005ad78     ProcList.exp
 0002:00014db4       rgszName                   000000018005adb4     ProcList.exp
 0002:00014df0       rgwOrd                     000000018005adf0     ProcList.exp
 0002:00014e0e       szName                     000000018005ae0e     ProcList.exp
 0002:00014e1b       $N00001                    000000018005ae1b     ProcList.exp
 0002:00014e27       $N00002                    000000018005ae27     ProcList.exp
 0002:00014e30       $N00003                    000000018005ae30     ProcList.exp
 0002:00014e3b       $N00004                    000000018005ae3b     ProcList.exp
 0002:00014e48       $N00005                    000000018005ae48     ProcList.exp
 0002:00014e56       $N00006                    000000018005ae56     ProcList.exp
 0002:00014e60       $N00007                    000000018005ae60     ProcList.exp
 0002:00014e6d       $N00008                    000000018005ae6d     ProcList.exp
 0002:00014e7c       $N00009                    000000018005ae7c     ProcList.exp
 0002:00014e8e       $N00010                    000000018005ae8e     ProcList.exp
 0002:00014e9d       $N00011                    000000018005ae9d     ProcList.exp
 0002:00014ea3       $N00012                    000000018005aea3     ProcList.exp
 0002:00014eb6       $N00013                    000000018005aeb6     ProcList.exp
 0002:00014ec9       $N00014                    000000018005aec9     ProcList.exp
 0002:00014ede       $N00015                    000000018005aede     ProcList.exp
 0002:00015750       .idata$6                   000000018005b750     kernel32:KERNEL32.dll
 0002:00015852       .idata$6                   000000018005b852     advapi32:ADVAPI32.dll
 0002:00015938       .idata$6                   000000018005b938     user32:USER32.dll
 0002:00015974       .idata$6                   000000018005b974     mpr:MPR.dll
 0002:000159b2       .idata$6                   000000018005b9b2     ole32:ole32.dll
 0002:000159bc       .idata$6                   000000018005b9bc     oleaut32:OLEAUT32.dll
 0002:000159fa       .idata$6                   000000018005b9fa     psapi:PSAPI.DLL
 0002:00015a46       .idata$6                   000000018005ba46     version:VERSION.dll
 0003:00000000       ?init@std@@3JA             000000018005c000     libcpmt:xlock.obj
 0003:00000008       ?atcount_cdecl@@3_KA       000000018005c008     libcpmt:iosptrs.obj
 0003:00000030       ?__vcrt_flsindex@@3KA      000000018005c030     libvcruntime:per_thread_data.obj
 0003:000001f8       ?errno_no_memory@@3HA      000000018005c1f8     libucrt:errno.obj
 0003:000001fc       ?doserrno_no_memory@@3KA   000000018005c1fc     libucrt:errno.obj
 0003:00000214       ?__acrt_flsindex@@3KA      000000018005c214     libucrt:per_thread_data.obj
 0003:00000218       _ctype_loc_style           000000018005c218     libucrt:wsetlocale.obj
 0003:000003a0       ?tzstd_program@@3PADA      000000018005c3a0     libucrt:timeset.obj
 0003:000003e0       ?tzdst_program@@3PADA      000000018005c3e0     libucrt:timeset.obj
 0003:00000420       ?tzname_states@@3PAY01PEADA 000000018005c420     libucrt:timeset.obj
 0003:00000660       _mbctypes                  000000018005c660     libucrt:mbctype.obj
 0003:00000770       _mbcasemaps                000000018005c770     libucrt:mbctype.obj
 0003:00000870       ?__rgctypeflag@@3PADA      000000018005c870     libucrt:mbctype.obj
 0003:00000880       ?__rgcode_page_info@@3PAUcode_page_info@@A 000000018005c880     libucrt:mbctype.obj
 0003:00000a70       ?__dcrt_lowio_console_output_handle@@3PEAXEA 000000018005ca70     libucrt:initcon.obj
 0003:00000a78       ?nr@?7??Connect@Plist@@QEAA_NPEB_W00@Z@4U_NETRESOURCEW@@A 000000018005ca78     Pclass.obj
 0003:00000aa8       ?kbt@?1??GetOpenPanelInfo@Plist@@QEAAXPEAUOpenPanelInfo@@@Z@4UKeyBarTitles@@A 000000018005caa8     Pclass.obj
 0003:00000ac0       ?FKeys@?1??GetOpenPanelInfo@Plist@@QEAAXPEAUOpenPanelInfo@@@Z@4PAGA 000000018005cac0     Pclass.obj
 0003:00000d50       ??_R0?AV<lambda_3>@?N@??PrintModules@@YAXPEAXKAEAUoptions@@@Z@@8 000000018005cd50     Plist.obj
 0003:00000e00       ??_R0?AV<lambda_1>@?1??GetProcessString@WMIConnection@@AEAA?AV?$basic_string@_WU?$char_traits@_W@std@@V?$allocator@_W@2@@std@@KPEB_W@Z@@8 000000018005ce00     wmi.obj
 0003:00000ea0       ??_R0?AV<lambda_1>@?1??GetProcessInt@WMIConnection@@AEAAKKPEB_W@Z@@8 000000018005cea0     wmi.obj
 0003:000012c0       ??_R0?AV?$_Func_impl_no_alloc@V<lambda_3>@?N@??PrintModules@@YAXPEAXKAEAUoptions@@@Z@_NPEA_W_K@std@@@8 000000018005d2c0     Plist.obj
 0003:00001410       ??_R0?AV?$_Func_impl_no_alloc@V<lambda_1>@?1??GetProcessString@WMIConnection@@AEAA?AV?$basic_string@_WU?$char_traits@_W@std@@V?$allocator@_W@2@@std@@KPEB_W@Z@XAEBUtagVARIANT@@@std@@@8 000000018005d410     wmi.obj
 0003:000014e0       ??_R0?AV?$_Func_impl_no_alloc@V<lambda_1>@?1??GetProcessInt@WMIConnection@@AEAAKKPEB_W@Z@XAEBUtagVARIANT@@@std@@@8 000000018005d4e0     wmi.obj
 0003:00001560       ?mtx@std@@3PAU_RTL_CRITICAL_SECTION@@A 000000018005d560     libcpmt:xlock.obj
 0003:000016a0       ?initlocks@std@@3V_Init_locks@1@A 000000018005d6a0     libcpmt:xlock.obj
 0003:000016d8       ?classic_locale@std@@3Vlocale@1@A 000000018005d6d8     libcpmt:locale0.obj
 0003:000016f0       ?_Fac_head@std@@3PEAU_Fac_node@1@EA 000000018005d6f0     libcpmt:locale0.obj
 0003:000016f8       ?_Fac_tidy_reg@std@@3U_Fac_tidy_reg_t@1@B 000000018005d6f8     libcpmt:locale0.obj
 0003:00001700       global_locale              000000018005d700     libcpmt:locale0.obj
 0003:00001708       ?registered@?1??_Setgloballocale@locale@std@@CAXPEAX@Z@4_NA 000000018005d708     libcpmt:locale0.obj
 0003:00001770       ?initlocks@std@@3V_Init_locks@1@A 000000018005d770     libcpmt:iosptrs.obj
 0003:00001771       ?init_atexit@@3U_Init_atexit@@A 000000018005d771     libcpmt:iosptrs.obj
 0003:00001780       ?atfuns_cdecl@@3PAP6AXXZA  000000018005d780     libcpmt:iosptrs.obj
 0003:000018bc       ?is_initialized_as_dll@@3_NA 000000018005d8bc     LIBCMT:utility.obj
 0003:000018c8       ?module_local_atexit_table@@3U_onexit_table_t@@A 000000018005d8c8     LIBCMT:utility.obj
 0003:000018e0       ?module_local_at_quick_exit_table@@3U_onexit_table_t@@A 000000018005d8e0     LIBCMT:utility.obj
 0003:000018f8       ?module_local_atexit_table_initialized@@3_NA 000000018005d8f8     LIBCMT:utility.obj
 0003:000018fc       ?__proc_attached@@3HA      000000018005d8fc     LIBCMT:dll_dllmain.obj
 0003:00001910       GS_ExceptionRecord         000000018005d910     LIBCMT:gs_report.obj
 0003:000019b0       GS_ContextRecord           000000018005d9b0     LIBCMT:gs_report.obj
 0003:00001d60       ?__vcrt_startup_thread_ptd@@3U__vcrt_ptd@@A 000000018005dd60     libvcruntime:per_thread_data.obj
 0003:00001de8       __vcrt_lock_table          000000018005dde8     libvcruntime:locks.obj
 0003:00001e10       __vcrt_locks_initialized   000000018005de10     libvcruntime:locks.obj
 0003:00001e18       ?heap@@3V_HeapManager@@A   000000018005de18     libvcruntime:undname.obj
 0003:00001ea0       ?__acrt_lock_table@@3PAU_RTL_CRITICAL_SECTION@@A 000000018005dea0     libucrt:locks.obj
 0003:000020d0       ?__acrt_locks_initialized@@3IA 000000018005e0d0     libucrt:locks.obj
 0003:000020d4       ?c_termination_complete@@3JA 000000018005e0d4     libucrt:exit.obj
 0003:000020d8       ?thread_local_exit_callback_func@@3P6AXPEAXK0@ZEA 000000018005e0d8     libucrt:exit.obj
 0003:000020f0       ?program_name@?1???$common_configure_argv@D@@YAHW4_crt_argv_mode@@@Z@4PADA 000000018005e0f0     libucrt:argv_parsing.obj
 0003:00002248       ?__acrt_new_handler@@3V?$dual_state_global@P6AH_K@Z@__crt_state_management@@A 000000018005e248     libucrt:new_handler.obj
 0003:00002250       ?__acrt_invalid_parameter_handler@@3V?$dual_state_global@P6AXPEB_W00I_K@Z@__crt_state_management@@A 000000018005e250     libucrt:invalid_parameter.obj
 0003:00002664       ?__acrt_app_type@@3W4_crt_app_type@@A 000000018005e664     libucrt:report_runtime_error.obj
 0003:00002670       ?module_handles@@3PAPEAUHINSTANCE__@@A 000000018005e670     libucrt:winapi_thunks.obj
 0003:00002710       ?encoded_function_pointers@@3PAPEAXA 000000018005e710     libucrt:winapi_thunks.obj
 0003:00002820       ?static_enum_proc@?1??enum_system_locales_ex_nolock@@YAHQ6AHPEA_WK_J@Z@Z@4P6AH0K1@ZEA 000000018005e820     libucrt:winapi_thunks.obj
 0003:00002828       ?internal_state@?1??_mbtowc_l@@9@4U_Mbstatet@@A 000000018005e828     libucrt:mbtowc.obj
 0003:00002830       ?enable_percent_n@@3_KA    000000018005e830     libucrt:printf_count_output.obj
 0003:00002858       ?ctrlc_action@@3V?$dual_state_global@P6AXH@Z@__crt_state_management@@A 000000018005e858     libucrt:signal.obj
 0003:00002860       ?ctrlbreak_action@@3V?$dual_state_global@P6AXH@Z@__crt_state_management@@A 000000018005e860     libucrt:signal.obj
 0003:00002868       ?abort_action@@3V?$dual_state_global@P6AXH@Z@__crt_state_management@@A 000000018005e868     libucrt:signal.obj
 0003:00002870       ?term_action@@3V?$dual_state_global@P6AXH@Z@__crt_state_management@@A 000000018005e870     libucrt:signal.obj
 0003:00002878       ?_tzname@@3V?$dual_state_global@PEAPEAD@__crt_state_management@@A 000000018005e878     libucrt:timeset.obj
 0003:00002890       ?tz_api_used@@3HA          000000018005e890     libucrt:tzset.obj
 0003:000028a0       ?tz_info@@3U_TIME_ZONE_INFORMATION@@A 000000018005e8a0     libucrt:tzset.obj
 0003:00002968       ?fSystemSet@@3HA           000000018005e968     libucrt:mbctype.obj
 0003:0000296c       ?initialized@?1??__acrt_initialize_multibyte@@9@4_NA 000000018005e96c     libucrt:mbctype.obj
 0003:000029a8       ?user_matherr@@3V?$dual_state_global@P6AHPEAU_exception@@@Z@__crt_state_management@@A 000000018005e9a8     libucrt:matherr.obj
 0003:000029b0       ?__acrt_global_new_mode@@3V?$dual_state_global@J@__crt_state_management@@A 000000018005e9b0     libucrt:new_mode.obj
 0003:000029b8       ?internal_pst@?1??__mbrtoc32_utf8@__crt_mbstring@@YA_KPEA_UPEBD_KPEAU_Mbstatet@@@Z@4U3@A 000000018005e9b8     libucrt:mbrtoc32.obj
 0003:000029c0       ?internal_pst@?1??__c16rtomb_utf8@__crt_mbstring@@YA_KPEAD_SPEAU_Mbstatet@@@Z@4U3@A 000000018005e9c0     libucrt:c16rtomb.obj
 0003:000029e0       ?kbl@?1??GetOpenPanelInfo@Plist@@QEAAXPEAUOpenPanelInfo@@@Z@4PAUKeyBarLabel@@A 000000018005e9e0     Pclass.obj
 0003:00002ae8       ?ArraysInited@?2??PanelModes@Plist@@QEAAPEAUPanelMode@@AEA_K@Z@4_NA 000000018005eae8     Pclass.obj
 0003:00002ae9       ?Inited@?1??dynamic_bind@@YAXXZ@4_NA 000000018005eae9     Proclist.obj
 0003:00002dd8       ?$S5@?1??GetUserAccountID@@YA@XZ@4IA 000000018005edd8     handles.obj
 0003:00002de0       ?UserAccountID@?1??GetUserAccountID@@YA@XZ@4V?$basic_string@_WU?$char_traits@_W@std@@V?$allocator@_W@2@@std@@B 000000018005ede0     handles.obj
 0003:00002e00       ?Title@?1??GetOpenPanelInfo@Plist@@QEAAXPEAUOpenPanelInfo@@@Z@4V?$basic_string@_WU?$char_traits@_W@std@@V?$allocator@_W@2@@std@@A 000000018005ee00     Pclass.obj
 0003:00002e20       ?$S5@?1??GetOpenPanelInfo@Plist@@QEAAXPEAUOpenPanelInfo@@@Z@4IA 000000018005ee20     Pclass.obj
 0003:00002e30       ?PanelModesRemote@?1??PanelModes@Plist@@QEAAPEAUPanelMode@@AEA_K@Z@4V?$array@UPanelMode@@$09@std@@A 000000018005ee30     Pclass.obj
 0003:00003010       ?PanelModesLocal@?1??PanelModes@Plist@@QEAAPEAUPanelMode@@AEA_K@Z@4V?$array@UPanelMode@@$09@std@@A 000000018005f010     Pclass.obj
 0003:000031f0       ?TitlesRemote@?1??PanelModes@Plist@@QEAAPEAUPanelMode@@AEA_K@Z@4V?$array@V?$array@PEA_W$0BI@@std@@$09@std@@A 000000018005f1f0     Pclass.obj
 0003:00003970       ?TitlesLocal@?1??PanelModes@Plist@@QEAAPEAUPanelMode@@AEA_K@Z@4V?$array@V?$array@PEA_W$0BI@@std@@$09@std@@A 000000018005f970     Pclass.obj
 0003:000040f0       ?hDebugToken@@3V?$unique_ptr@XUhandle_closer@@@std@@A 00000001800600f0     Plist.obj
 0003:000040f8       ?DiskMenuStrings@?7??GetPluginInfoW@@9@4PAPEB_WA 00000001800600f8     Proclist.obj
 0003:00004100       ?PluginCfgStrings@?1??GetPluginInfoW@@9@4PAPEB_WA 0000000180060100     Proclist.obj
 0003:00004108       ?PluginMenuStrings@?4??GetPluginInfoW@@9@4PAPEB_WA 0000000180060108     Proclist.obj
 0005:00000060       $R000000                   0000000180064060     ProcList.res
